 clark_support

 Timestamp is 5dee3682 (Mon Dec 09 18:56:50 2019)

 Preferred load address is 10000000

 Start         Length     Name                   Class
 0001:00000000 00002b1bH .text$di                CODE
 0001:00002b20 00016a08H .text$mn                CODE
 0001:00019530 000040e4H .text$x                 CODE
 0001:0001d620 00000a6bH .text$yd                CODE
 0002:00000000 00000918H .idata$5                DATA
 0002:00000918 00000004H .CRT$XCA                DATA
 0002:0000091c 0000023cH .CRT$XCU                DATA
 0002:00000b58 00000004H .CRT$XCZ                DATA
 0002:00000b5c 00000004H .CRT$XIA                DATA
 0002:00000b60 00000004H .CRT$XIAA               DATA
 0002:00000b64 00000004H .CRT$XIC                DATA
 0002:00000b68 00000004H .CRT$XIZ                DATA
 0002:00000b70 00003938H .rdata                  DATA
 0002:000044a8 00000074H .rdata$debug            DATA
 0002:0000451c 00001644H .rdata$r                DATA
 0002:00005b60 000002fcH .rdata$sxdata           DATA
 0002:00005e5c 00000004H .rtc$IAA                DATA
 0002:00005e60 00000004H .rtc$IZZ                DATA
 0002:00005e64 00000004H .rtc$TAA                DATA
 0002:00005e68 00000004H .rtc$TZZ                DATA
 0002:00005e70 0000487cH .xdata$x                DATA
 0002:0000a6f0 00000056H .edata                  DATA
 0002:0000a748 00000118H .idata$2                DATA
 0002:0000a860 00000014H .idata$3                DATA
 0002:0000a874 00000918H .idata$4                DATA
 0002:0000b18c 00007988H .idata$6                DATA
 0003:00000000 00000144H .data                   DATA
 0003:00000148 00000c10H .data$r                 DATA
 0003:00000d58 000006bcH .bss                    DATA
 0004:00000000 00000058H .rsrc$01                DATA
 0004:00000060 00000180H .rsrc$02                DATA

  Address         Publics by Value              Rva+Base       Lib:Object

 0000:00000000       ___guard_fids_count        00000000     <absolute>
 0000:00000000       __except_list              00000000     <absolute>
 0000:00000000       ___guard_fids_table        00000000     <absolute>
 0000:00000000       ___guard_flags             00000000     <absolute>
 0000:000000bf       ___safe_se_handler_count   000000bf     <absolute>
 0000:00009876       __ldused                   00009876     <absolute>
 0000:00009876       __fltused                  00009876     <absolute>
 0000:00000000       ___ImageBase               10000000     <linker-defined>
 0001:00002b20       ??$_Allocate@D@std@@YAPADIPAD@Z 10003b20 f i ClarkBuildWorker.obj
 0001:00002b50       ??$_Move@AAPAVDataType@U2@@@std@@YA$$QAPAVDataType@U2@@AAPAV12@@Z 10003b50 f i ClarkBuildWorker.obj
 0001:00002b60       ??$acquireMemoryFence@H@?$QGenericAtomicOps@U?$QAtomicOpsBySize@$03@@@@SAXABH@Z 10003b60 f i ClarkBuildWorker.obj
 0001:00002b70       ??$addressof@D@std@@YAPADAAD@Z 10003b70 f i ClarkBuildWorker.obj
 0001:00002b80       ??$atomic@H@?$QAtomicOpsBySize@$03@@CAPAJPAH@Z 10003b80 f i ClarkBuildWorker.obj
 0001:00002b90       ??$construct@PADAAPAD@?$_Wrap_alloc@V?$allocator@D@std@@@std@@QAEXPAPADAAPAD@Z 10003b90 f i ClarkBuildWorker.obj
 0001:00002bb0       ??$construct@PADAAPAD@?$allocator@D@std@@QAEXPAPADAAPAD@Z 10003bb0 f i ClarkBuildWorker.obj
 0001:00002bd0       ??$construct@PADAAPAD@?$allocator_traits@V?$allocator@D@std@@@std@@SAXAAV?$allocator@D@1@PAPADAAPAD@Z 10003bd0 f i ClarkBuildWorker.obj
 0001:00002bf0       ??$deref@H@?$QAtomicOpsBySize@$03@@SA_NAAH@Z 10003bf0 f i ClarkBuildWorker.obj
 0001:00002c10       ??$destroy@PAD@?$_Wrap_alloc@V?$allocator@D@std@@@std@@QAEXPAPAD@Z 10003c10 f i ClarkBuildWorker.obj
 0001:00002c20       ??$destroy@PAD@?$allocator@D@std@@QAEXPAPAD@Z 10003c20 f i ClarkBuildWorker.obj
 0001:00002c30       ??$destroy@PAD@?$allocator_traits@V?$allocator@D@std@@@std@@SAXAAV?$allocator@D@1@PAPAD@Z 10003c30 f i ClarkBuildWorker.obj
 0001:00002c40       ??$forward@AAPAD@std@@YAAAPADAAPAD@Z 10003c40 f i ClarkBuildWorker.obj
 0001:00002c50       ??$getAttributeValue@H@Attribute@U2@@QBEHPAVWorkflowContext@Workflow@1@@Z 10003c50 f i ClarkBuildWorker.obj
 0001:00003020       ??$getAttributeValue@V?$QList@VDataset@U2@@@@@Attribute@U2@@QBE?AV?$QList@VDataset@U2@@@@PAVWorkflowContext@Workflow@1@@Z 10004020 f i ClarkBuildWorker.obj
 0001:00003040       ??$getAttributeValue@VQString@@@Attribute@U2@@QBE?AVQString@@PAVWorkflowContext@Workflow@1@@Z 10004040 f i ClarkBuildWorker.obj
 0001:000033d0       ??$getAttributeValueWithoutScript@H@Attribute@U2@@QBEHXZ 100043d0 f i ClarkBuildWorker.obj
 0001:00003410       ??$getAttributeValueWithoutScript@V?$QList@VDataset@U2@@@@@Attribute@U2@@QBE?AV?$QList@VDataset@U2@@@@XZ 10004410 f i ClarkBuildWorker.obj
 0001:00003430       ??$getAttributeValueWithoutScript@VQString@@@Attribute@U2@@QBE?AVQString@@XZ 10004430 f i ClarkBuildWorker.obj
 0001:00003450       ??$getValue@H@BaseWorker@LocalWorkflow@U2@@IBEHABVQString@@@Z 10004450 f i ClarkBuildWorker.obj
 0001:00003480       ??$getValue@V?$QList@VDataset@U2@@@@@BaseWorker@LocalWorkflow@U2@@IBE?AV?$QList@VDataset@U2@@@@ABVQString@@@Z 10004480 f i ClarkBuildWorker.obj
 0001:000034d0       ??$getValue@VQString@@@BaseWorker@LocalWorkflow@U2@@IBE?AVQString@@ABV3@@Z 100044d0 f i ClarkBuildWorker.obj
 0001:000035e0       ??$load@H@?$QGenericAtomicOps@U?$QAtomicOpsBySize@$03@@@@SAHABH@Z 100045e0 f i ClarkBuildWorker.obj
 0001:000035f0       ??$loadAcquire@H@?$QGenericAtomicOps@U?$QAtomicOpsBySize@$03@@@@SAHABH@Z 100045f0 f i ClarkBuildWorker.obj
 0001:00003600       ??$orderedMemoryFence@H@?$QGenericAtomicOps@U?$QAtomicOpsBySize@$03@@@@SAXABH@Z 10004600 f i ClarkBuildWorker.obj
 0001:00003610       ??$qMapLessThanKey@VDescriptor@U2@@@@YA_NABVDescriptor@U2@@0@Z 10004610 f i ClarkBuildWorker.obj
 0001:00003630       ??$qMapLessThanKey@VQString@@@@YA_NABVQString@@0@Z 10004630 f i ClarkBuildWorker.obj
 0001:00003640       ??$qMetaTypeId@H@@YAHXZ    10004640 f i ClarkBuildWorker.obj
 0001:00003650       ??$qMetaTypeId@V?$QList@VDataset@U2@@@@@@YAHXZ 10004650 f i ClarkBuildWorker.obj
 0001:00003660       ??$qMetaTypeId@VQString@@@@YAHXZ 10004660 f i ClarkBuildWorker.obj
 0001:00003670       ??$qRegisterMetaType@V?$QList@VDataset@U2@@@@@@YAHPBDPAV?$QList@VDataset@U2@@@@W4DefinedType@?$MetaTypeDefinedHelper@V?$QList@VDataset@U2@@@@$00@QtPrivate@@@Z 10004670 f i ClarkBuildWorker.obj
 0001:00003730       ??$qRegisterNormalizedMetaType@V?$QList@VDataset@U2@@@@@@YAHABVQByteArray@@PAV?$QList@VDataset@U2@@@@W4DefinedType@?$MetaTypeDefinedHelper@V?$QList@VDataset@U2@@@@$00@QtPrivate@@@Z 10004730 f i ClarkBuildWorker.obj
 0001:00003790       ??$qSwap@PAVDataType@U2@@@@YAXAAPAVDataType@U2@@0@Z 10004790 f i ClarkBuildWorker.obj
 0001:000037b0       ??$qobject_cast@PAVClarkBuildTask@LocalWorkflow@U2@@@@YAPAVClarkBuildTask@LocalWorkflow@U2@@PAVQObject@@@Z 100047b0 f i ClarkBuildWorker.obj
 0001:000037d0       ??$qvariant_cast@H@@YAHABVQVariant@@@Z 100047d0 f i ClarkBuildWorker.obj
 0001:00003810       ??$qvariant_cast@V?$QList@VDataset@U2@@@@@@YA?AV?$QList@VDataset@U2@@@@ABVQVariant@@@Z 10004810 f i ClarkBuildWorker.obj
 0001:00003830       ??$qvariant_cast@VQString@@@@YA?AVQString@@ABVQVariant@@@Z 10004830 f i ClarkBuildWorker.obj
 0001:00003850       ??$ref@H@?$QAtomicOpsBySize@$03@@SA_NAAH@Z 10004850 f i ClarkBuildWorker.obj
 0001:00003870       ??$releaseMemoryFence@H@?$QGenericAtomicOps@U?$QAtomicOpsBySize@$03@@@@SAXABH@Z 10004870 f i ClarkBuildWorker.obj
 0001:00003880       ??$storeRelease@HH@?$QGenericAtomicOps@U?$QAtomicOpsBySize@$03@@@@SAXAAHH@Z 10004880 f i ClarkBuildWorker.obj
 0001:00003890       ??$swap@PAVDataType@U2@@@std@@YAXAAPAVDataType@U2@@0@Z 10004890 f i ClarkBuildWorker.obj
 0001:000038b0       ??$value@H@QVariant@@QBEHXZ 100048b0 f i ClarkBuildWorker.obj
 0001:000038f0       ??$value@V?$QList@VDataset@U2@@@@@QVariant@@QBE?AV?$QList@VDataset@U2@@@@XZ 100048f0 f i ClarkBuildWorker.obj
 0001:00003910       ??$value@VQString@@@QVariant@@QBE?AVQString@@XZ 10004910 f i ClarkBuildWorker.obj
 0001:00003930       ??0?$PrompterBase@VClarkBuildPrompter@LocalWorkflow@U2@@@U2@@QAE@PAVActor@Workflow@1@_N@Z 10004930 f i ClarkBuildWorker.obj
 0001:00003960       ??0?$QExplicitlySharedDataPointer@VDataType@U2@@@@QAE@ABV0@@Z 10004960 f i ClarkBuildWorker.obj
 0001:00003980       ??0?$QExplicitlySharedDataPointer@VDataType@U2@@@@QAE@PAVDataType@U2@@@Z 10004980 f i ClarkBuildWorker.obj
 0001:000039a0       ??0?$QExplicitlySharedDataPointer@VDataType@U2@@@@QAE@XZ 100049a0 f i ClarkBuildWorker.obj
 0001:000039b0       ??0?$QFlags@W4OpenModeFlag@QIODevice@@@@QAE@W4OpenModeFlag@QIODevice@@@Z 100049b0 f i ClarkBuildWorker.obj
 0001:000039c0       ??0?$QFlags@W4Option@URLDelegate@U2@@@@QAE@VQFlag@@@Z 100049c0 f i ClarkBuildWorker.obj
 0001:000039d0       ??0?$QFlags@W4Option@URLDelegate@U2@@@@QAE@W4Option@URLDelegate@U2@@@Z 100049d0 f i ClarkBuildWorker.obj
 0001:000039e0       ??0?$QFlags@W4TaskFlag@U2@@@@QAE@VQFlag@@@Z 100049e0 f i ClarkBuildWorker.obj
 0001:000039f0       ??0?$QFlags@W4TaskFlag@U2@@@@QAE@W4TaskFlag@U2@@@Z 100049f0 f i ClarkBuildWorker.obj
 0001:00003a00       ??0?$QFlags@W4TypeFlag@QMetaType@@@@QAE@VQFlag@@@Z 10004a00 f i ClarkBuildWorker.obj
 0001:00003a10       ??0?$QForeachContainer@$$CBVQStringList@@@@QAE@ABVQStringList@@@Z 10004a10 f i ClarkBuildWorker.obj
 0001:00003a50       ??0?$QForeachContainer@V?$QList@PAVPort@Workflow@U2@@@@@@QAE@ABV?$QList@PAVPort@Workflow@U2@@@@@Z 10004a50 f i ClarkBuildWorker.obj
 0001:00003a90       ??0?$QForeachContainer@V?$QList@VDescriptor@U2@@@@@@QAE@ABV?$QList@VDescriptor@U2@@@@@Z 10004a90 f i ClarkBuildWorker.obj
 0001:00003ad0       ??0?$QList@PAVAttribute@U2@@@@QAE@XZ 10004ad0 f i ClarkBuildWorker.obj
 0001:00003ae0       ??0?$QList@PAVPort@Workflow@U2@@@@QAE@ABV0@@Z 10004ae0 f i ClarkBuildWorker.obj
 0001:00003ba0       ??0?$QList@PAVPortDescriptor@Workflow@U2@@@@QAE@XZ 10004ba0 f i ClarkBuildWorker.obj
 0001:00003bb0       ??0?$QList@VDataset@U2@@@@QAE@$$QAV0@@Z 10004bb0 f i ClarkBuildWorker.obj
 0001:00003bd0       ??0?$QList@VDataset@U2@@@@QAE@ABV0@@Z 10004bd0 f i ClarkBuildWorker.obj
 0001:00003c90       ??0?$QList@VDataset@U2@@@@QAE@XZ 10004c90 f i ClarkBuildWorker.obj
 0001:00003ca0       ??0?$QList@VDescriptor@U2@@@@QAE@$$QAV0@@Z 10004ca0 f i ClarkBuildWorker.obj
 0001:00003cc0       ??0?$QList@VDescriptor@U2@@@@QAE@ABV0@@Z 10004cc0 f i ClarkBuildWorker.obj
 0001:00003d80       ??0?$QList@VDescriptor@U2@@@@QAE@XZ 10004d80 f i ClarkBuildWorker.obj
 0001:00003d90       ??0?$QList@VQString@@@@QAE@ABV0@@Z 10004d90 f i ClarkBuildWorker.obj
 0001:00003e50       ??0?$QList@VQString@@@@QAE@XZ 10004e50 f i ClarkBuildWorker.obj
 0001:00003e60       ??0?$QMap@VDescriptor@U2@@V?$QExplicitlySharedDataPointer@VDataType@U2@@@@@@QAE@XZ 10004e60 f i ClarkBuildWorker.obj
 0001:00003e70       ??0?$QMap@VQString@@PAVPropertyDelegate@U2@@@@QAE@XZ 10004e70 f i ClarkBuildWorker.obj
 0001:00003e80       ??0?$QMap@VQString@@VQScriptValue@@@@QAE@XZ 10004e80 f i ClarkBuildWorker.obj
 0001:00003e90       ??0?$QMap@VQString@@VQVariant@@@@QAE@XZ 10004e90 f i ClarkBuildWorker.obj
 0001:00003ea0       ??0?$QScopedPointer@VExternalToolRunTask@U2@@U?$QScopedPointerDeleter@VExternalToolRunTask@U2@@@@@@QAE@PAVExternalToolRunTask@U2@@@Z 10004ea0 f i ClarkBuildWorker.obj
 0001:00003eb0       ??0?$_String_alloc@$0A@U?$_String_base_types@DV?$allocator@D@std@@@std@@@std@@QAE@ABV?$allocator@D@1@@Z 10004eb0 f i ClarkBuildWorker.obj
 0001:00003ed0       ??0?$_String_val@U?$_Simple_types@D@std@@@std@@QAE@XZ 10004ed0 f i ClarkBuildWorker.obj
 0001:00003ef0       ??0?$_Wrap_alloc@V?$allocator@D@std@@@std@@QAE@XZ 10004ef0 f i ClarkBuildWorker.obj
 0001:00003f00       ??0?$allocator@D@std@@QAE@XZ 10004f00 f i ClarkBuildWorker.obj
 0001:00003f10       ??0?$basic_string@DU?$char_traits@D@std@@V?$allocator@D@2@@std@@QAE@PBD@Z 10004f10 f i ClarkBuildWorker.obj
 0001:00003f70       ??0ClarkBuildLogParser@LocalWorkflow@U2@@QAE@XZ 10004f70 f i ClarkBuildWorker.obj
 0001:00003f90       ??0ClarkBuildPrompter@LocalWorkflow@U2@@QAE@PAVActor@Workflow@2@@Z 10004f90 f i ClarkBuildWorker.obj
 0001:00003fc0       ??0ClarkBuildTask@LocalWorkflow@U2@@QAE@ABVQString@@ABVQStringList@@H0@Z 10004fc0 f   ClarkBuildWorker.obj
 0001:000041e0       ??0ClarkBuildValidator@LocalWorkflow@U2@@QAE@XZ 100051e0 f i ClarkBuildWorker.obj
 0001:000041f0       ??0ClarkBuildWorker@LocalWorkflow@U2@@QAE@PAVActor@Workflow@2@@Z 100051f0 f   ClarkBuildWorker.obj
 0001:00004230       ??0ClarkBuildWorkerFactory@LocalWorkflow@U2@@QAE@XZ 10005230 f i ClarkBuildWorker.obj
 0001:00004250       ??0QFlag@@QAE@H@Z          10005250 f i ClarkBuildWorker.obj
 0001:00004260       ??0QLatin1Char@@QAE@D@Z    10005260 f i ClarkBuildWorker.obj
 0001:00004270       ??0QStringList@@QAE@ABV0@@Z 10005270 f i ClarkBuildWorker.obj
 0001:00004290       ??0QStringList@@QAE@XZ     10005290 f i ClarkBuildWorker.obj
 0001:000042a0       ??0_Generic_error_category@std@@QAE@XZ 100052a0 f i ClarkBuildWorker.obj
 0001:000042b0       ??0_Ignore@std@@QAE@XZ     100052b0 f i ClarkBuildWorker.obj
 0001:000042c0       ??0_Iostream_error_category@std@@QAE@XZ 100052c0 f i ClarkBuildWorker.obj
 0001:000042d0       ??0_System_error_category@std@@QAE@XZ 100052d0 f i ClarkBuildWorker.obj
 0001:000042e0       ??0const_iterator@?$QList@PAVPort@Workflow@U2@@@@QAE@PAUNode@1@@Z 100052e0 f i ClarkBuildWorker.obj
 0001:000042f0       ??0const_iterator@?$QList@VDescriptor@U2@@@@QAE@PAUNode@1@@Z 100052f0 f i ClarkBuildWorker.obj
 0001:00004300       ??0const_iterator@?$QList@VQString@@@@QAE@PAUNode@1@@Z 10005300 f i ClarkBuildWorker.obj
 0001:00004310       ??0const_iterator@?$QMap@VDescriptor@U2@@VQVariant@@@@QAE@PBU?$QMapNode@VDescriptor@U2@@VQVariant@@@@@Z 10005310 f i ClarkBuildWorker.obj
 0001:00004320       ??0error_category@std@@QAE@XZ 10005320 f i ClarkBuildWorker.obj
 0001:00004330       ??0error_condition@std@@QAE@HABVerror_category@1@@Z 10005330 f i ClarkBuildWorker.obj
 0001:00004350       ??0iterator@?$QMap@VDescriptor@U2@@V?$QExplicitlySharedDataPointer@VDataType@U2@@@@@@QAE@PAU?$QMapNode@VDescriptor@U2@@V?$QExplicitlySharedDataPointer@VDataType@U2@@@@@@@Z 10005350 f i ClarkBuildWorker.obj
 0001:00004360       ??0iterator@?$QMap@VQString@@PAVPropertyDelegate@U2@@@@QAE@PAU?$QMapNode@VQString@@PAVPropertyDelegate@U2@@@@@Z 10005360 f i ClarkBuildWorker.obj
 0001:00004370       ??0iterator@?$QMap@VQString@@VQScriptValue@@@@QAE@PAU?$QMapNode@VQString@@VQScriptValue@@@@@Z 10005370 f i ClarkBuildWorker.obj
 0001:00004380       ??0iterator@?$QMap@VQString@@VQVariant@@@@QAE@PAU?$QMapNode@VQString@@VQVariant@@@@@Z 10005380 f i ClarkBuildWorker.obj
 0001:00004390       ??1?$PrompterBase@VClarkBuildPrompter@LocalWorkflow@U2@@@U2@@UAE@XZ 10005390 f i ClarkBuildWorker.obj
 0001:000043a0       ??1?$QExplicitlySharedDataPointer@VDataType@U2@@@@QAE@XZ 100053a0 f i ClarkBuildWorker.obj
 0001:000043c0       ??1?$QForeachContainer@$$CBVQStringList@@@@QAE@XZ 100053c0 f i ClarkBuildWorker.obj
 0001:000043d0       ??1?$QForeachContainer@V?$QList@PAVPort@Workflow@U2@@@@@@QAE@XZ 100053d0 f i ClarkBuildWorker.obj
 0001:00004400       ??1?$QForeachContainer@V?$QList@VDescriptor@U2@@@@@@QAE@XZ 10005400 f i ClarkBuildWorker.obj
 0001:00004430       ??1?$QList@PAVAttribute@U2@@@@QAE@XZ 10005430 f i ClarkBuildWorker.obj
 0001:00004460       ??1?$QList@PAVExternalToolListener@U2@@@@QAE@XZ 10005460 f i ClarkBuildWorker.obj
 0001:00004490       ??1?$QList@PAVPort@Workflow@U2@@@@QAE@XZ 10005490 f i ClarkBuildWorker.obj
 0001:000044c0       ??1?$QList@PAVPortDescriptor@Workflow@U2@@@@QAE@XZ 100054c0 f i ClarkBuildWorker.obj
 0001:000044f0       ??1?$QList@VDataset@U2@@@@QAE@XZ 100054f0 f i ClarkBuildWorker.obj
 0001:00004520       ??1?$QList@VDescriptor@U2@@@@QAE@XZ 10005520 f i ClarkBuildWorker.obj
 0001:00004550       ??1?$QList@VQString@@@@QAE@XZ 10005550 f i ClarkBuildWorker.obj
 0001:000045b0       ??1?$QMap@VDescriptor@U2@@V?$QExplicitlySharedDataPointer@VDataType@U2@@@@@@QAE@XZ 100055b0 f i ClarkBuildWorker.obj
 0001:00004600       ??1?$QMap@VQString@@PAVPropertyDelegate@U2@@@@QAE@XZ 10005600 f i ClarkBuildWorker.obj
 0001:00004670       ??1?$QMap@VQString@@VQScriptValue@@@@QAE@XZ 10005670 f i ClarkBuildWorker.obj
 0001:000046c0       ??1?$QMap@VQString@@VQVariant@@@@QAE@XZ 100056c0 f i ClarkBuildWorker.obj
 0001:00004710       ??1?$QScopedPointer@VExternalToolRunTask@U2@@U?$QScopedPointerDeleter@VExternalToolRunTask@U2@@@@@@QAE@XZ 10005710 f i ClarkBuildWorker.obj
 0001:00004720       ??1?$basic_string@DU?$char_traits@D@std@@V?$allocator@D@2@@std@@QAE@XZ 10005720 f i ClarkBuildWorker.obj
 0001:00004750       ??1ClarkBuildLogParser@LocalWorkflow@U2@@UAE@XZ 10005750 f i ClarkBuildWorker.obj
 0001:00004760       ??1ClarkBuildPrompter@LocalWorkflow@U2@@UAE@XZ 10005760 f i ClarkBuildWorker.obj
 0001:00004770       ??1ClarkBuildTask@LocalWorkflow@U2@@UAE@XZ 10005770 f i ClarkBuildWorker.obj
 0001:000047f0       ??1ClarkBuildValidator@LocalWorkflow@U2@@UAE@XZ 100057f0 f i ClarkBuildWorker.obj
 0001:00004800       ??1ClarkBuildWorker@LocalWorkflow@U2@@UAE@XZ 10005800 f i ClarkBuildWorker.obj
 0001:00004810       ??1ClarkBuildWorkerFactory@LocalWorkflow@U2@@UAE@XZ 10005810 f i ClarkBuildWorker.obj
 0001:00004820       ??1QStringList@@QAE@XZ     10005820 f i ClarkBuildWorker.obj
 0001:00004830       ??1_Generic_error_category@std@@UAE@XZ 10005830 f i ClarkBuildWorker.obj
 0001:00004840       ??1_Iostream_error_category@std@@UAE@XZ 10005840 f i ClarkBuildWorker.obj
 0001:00004850       ??1_System_error_category@std@@UAE@XZ 10005850 f i ClarkBuildWorker.obj
 0001:00004860       ??1error_category@std@@UAE@XZ 10005860 f i ClarkBuildWorker.obj
 0001:00004870       ??2@YAPAXIPAX@Z            10005870 f i ClarkBuildWorker.obj
 0001:00004880       ??3@YAXPAX0@Z              10005880 f i ClarkBuildWorker.obj
 0001:00004890       ??4?$QExplicitlySharedDataPointer@VDataType@U2@@@@QAEAAV0@$$QAV0@@Z 10005890 f i ClarkBuildWorker.obj
 0001:000048b0       ??4?$QExplicitlySharedDataPointer@VDataType@U2@@@@QAEAAV0@ABV0@@Z 100058b0 f i ClarkBuildWorker.obj
 0001:00004900       ??6?$QList@PAVAttribute@U2@@@@QAEAAV0@ABQAVAttribute@U2@@@Z 10005900 f i ClarkBuildWorker.obj
 0001:00004920       ??6?$QList@PAVPortDescriptor@Workflow@U2@@@@QAEAAV0@ABQAVPortDescriptor@Workflow@U2@@@Z 10005920 f i ClarkBuildWorker.obj
 0001:00004940       ??6?$QList@VWorkflowNotification@U2@@@@QAEAAV0@ABVWorkflowNotification@U2@@@Z 10005940 f i ClarkBuildWorker.obj
 0001:00004960       ??6QStringList@@QAEAAV0@ABVQString@@@Z 10005960 f i ClarkBuildWorker.obj
 0001:00004980       ??8const_iterator@?$QMap@VDescriptor@U2@@VQVariant@@@@QBE_NABV01@@Z 10005980 f i ClarkBuildWorker.obj
 0001:000049a0       ??8error_category@std@@QBE_NABV01@@Z 100059a0 f i ClarkBuildWorker.obj
 0001:000049b0       ??8error_condition@std@@QBE_NABV01@@Z 100059b0 f i ClarkBuildWorker.obj
 0001:000049d0       ??9const_iterator@?$QList@PAVPort@Workflow@U2@@@@QBE_NABV01@@Z 100059d0 f i ClarkBuildWorker.obj
 0001:000049f0       ??9const_iterator@?$QList@VDescriptor@U2@@@@QBE_NABV01@@Z 100059f0 f i ClarkBuildWorker.obj
 0001:00004a10       ??9const_iterator@?$QList@VQString@@@@QBE_NABV01@@Z 10005a10 f i ClarkBuildWorker.obj
 0001:00004a30       ??9const_iterator@?$QMap@VDescriptor@U2@@VQVariant@@@@QBE_NABV01@@Z 10005a30 f i ClarkBuildWorker.obj
 0001:00004a50       ??A?$QMap@VDescriptor@U2@@V?$QExplicitlySharedDataPointer@VDataType@U2@@@@@@QAEAAV?$QExplicitlySharedDataPointer@VDataType@U2@@@@ABVDescriptor@U2@@@Z 10005a50 f i ClarkBuildWorker.obj
 0001:00004b10       ??A?$QMap@VQString@@PAVPropertyDelegate@U2@@@@QAEAAPAVPropertyDelegate@U2@@ABVQString@@@Z 10005b10 f i ClarkBuildWorker.obj
 0001:00004b90       ??A?$QMap@VQString@@VQScriptValue@@@@QAEAAVQScriptValue@@ABVQString@@@Z 10005b90 f i ClarkBuildWorker.obj
 0001:00004c60       ??A?$QMap@VQString@@VQVariant@@@@QAEAAVQVariant@@ABVQString@@@Z 10005c60 f i ClarkBuildWorker.obj
 0001:00004d30       ??BQFlag@@QBEHXZ           10005d30 f i ClarkBuildWorker.obj
 0001:00004d40       ??Dconst_iterator@?$QList@PAVPort@Workflow@U2@@@@QBEABQAVPort@Workflow@U2@@XZ 10005d40 f i ClarkBuildWorker.obj
 0001:00004d50       ??Dconst_iterator@?$QList@VDescriptor@U2@@@@QBEABVDescriptor@U2@@XZ 10005d50 f i ClarkBuildWorker.obj
 0001:00004d60       ??Dconst_iterator@?$QList@VQString@@@@QBEABVQString@@XZ 10005d60 f i ClarkBuildWorker.obj
 0001:00004d70       ??Diterator@?$QMap@VDescriptor@U2@@V?$QExplicitlySharedDataPointer@VDataType@U2@@@@@@QBEAAV?$QExplicitlySharedDataPointer@VDataType@U2@@@@XZ 10005d70 f i ClarkBuildWorker.obj
 0001:00004d80       ??Diterator@?$QMap@VQString@@PAVPropertyDelegate@U2@@@@QBEAAPAVPropertyDelegate@U2@@XZ 10005d80 f i ClarkBuildWorker.obj
 0001:00004d90       ??Diterator@?$QMap@VQString@@VQScriptValue@@@@QBEAAVQScriptValue@@XZ 10005d90 f i ClarkBuildWorker.obj
 0001:00004da0       ??Diterator@?$QMap@VQString@@VQVariant@@@@QBEAAVQVariant@@XZ 10005da0 f i ClarkBuildWorker.obj
 0001:00004db0       ??Econst_iterator@?$QList@PAVPort@Workflow@U2@@@@QAEAAV01@XZ 10005db0 f i ClarkBuildWorker.obj
 0001:00004dc0       ??Econst_iterator@?$QList@VDescriptor@U2@@@@QAEAAV01@XZ 10005dc0 f i ClarkBuildWorker.obj
 0001:00004dd0       ??Econst_iterator@?$QList@VQString@@@@QAEAAV01@XZ 10005dd0 f i ClarkBuildWorker.obj
 0001:00004de0       ??Econst_iterator@?$QMap@VDescriptor@U2@@VQVariant@@@@QAEAAV01@XZ 10005de0 f i ClarkBuildWorker.obj
 0001:00004e00       ??H@YA?BVQString@@ABV0@PBD@Z 10005e00 f i ClarkBuildWorker.obj
 0001:00004ea0       ??U?$QFlags@W4Option@URLDelegate@U2@@@@QBE?AV0@W4Option@URLDelegate@U2@@@Z 10005ea0 f i ClarkBuildWorker.obj
 0001:00004ec0       ??U?$QFlags@W4TaskFlag@U2@@@@QBE?AV0@W4TaskFlag@U2@@@Z 10005ec0 f i ClarkBuildWorker.obj
 0001:00004ee0       ??U@YA?AV?$QFlags@W4Option@URLDelegate@U2@@@@W4Option@URLDelegate@U2@@0@Z 10005ee0 f i ClarkBuildWorker.obj
 0001:00004ef0       ??_5?$QFlags@W4TypeFlag@QMetaType@@@@QAEAAV0@W4TypeFlag@QMetaType@@@Z 10005ef0 f i ClarkBuildWorker.obj
 0001:00004efe       ??_E?$PrompterBase@VClarkBuildPrompter@LocalWorkflow@U2@@@U2@@WM@AEPAXI@Z 10005efe f i ClarkBuildWorker.obj
 0001:00004f06       ??_EClarkBuildPrompter@LocalWorkflow@U2@@WM@AEPAXI@Z 10005f06 f i ClarkBuildWorker.obj
 0001:00004f0e       ??_EClarkBuildWorker@LocalWorkflow@U2@@W7AEPAXI@Z 10005f0e f i ClarkBuildWorker.obj
 0001:00004f16       ??_EClarkBuildWorker@LocalWorkflow@U2@@WBA@AEPAXI@Z 10005f16 f i ClarkBuildWorker.obj
 0001:00004f1e       ??_EClarkBuildWorkerFactory@LocalWorkflow@U2@@W7AEPAXI@Z 10005f1e f i ClarkBuildWorker.obj
 0001:00004f26       ??_EIntegralBusActorPrototype@Workflow@U2@@W7AEPAXI@Z 10005f26 f i ClarkBuildWorker.obj
 0001:00004f30       ??_E?$PrompterBase@VClarkBuildPrompter@LocalWorkflow@U2@@@U2@@UAEPAXI@Z 10005f30 f i ClarkBuildWorker.obj
 0001:00004f30       ??_G?$PrompterBase@VClarkBuildPrompter@LocalWorkflow@U2@@@U2@@UAEPAXI@Z 10005f30 f i ClarkBuildWorker.obj
 0001:00004f60       ??_G?$QExplicitlySharedDataPointer@VDataType@U2@@@@QAEPAXI@Z 10005f60 f i ClarkBuildWorker.obj
 0001:00004fa0       ??_G?$QList@VDataset@U2@@@@QAEPAXI@Z 10005fa0 f i ClarkBuildWorker.obj
 0001:00004fe0       ??_EAttribute@U2@@UAEPAXI@Z 10005fe0 f i ClarkBuildWorker.obj
 0001:00004fe0       ??_GAttribute@U2@@UAEPAXI@Z 10005fe0 f i ClarkBuildWorker.obj
 0001:00005010       ??_EClarkBuildLogParser@LocalWorkflow@U2@@UAEPAXI@Z 10006010 f i ClarkBuildWorker.obj
 0001:00005010       ??_GClarkBuildLogParser@LocalWorkflow@U2@@UAEPAXI@Z 10006010 f i ClarkBuildWorker.obj
 0001:00005040       ??_EClarkBuildPrompter@LocalWorkflow@U2@@UAEPAXI@Z 10006040 f i ClarkBuildWorker.obj
 0001:00005040       ??_GClarkBuildPrompter@LocalWorkflow@U2@@UAEPAXI@Z 10006040 f i ClarkBuildWorker.obj
 0001:00005070       ??_EClarkBuildTask@LocalWorkflow@U2@@UAEPAXI@Z 10006070 f i ClarkBuildWorker.obj
 0001:00005070       ??_GClarkBuildTask@LocalWorkflow@U2@@UAEPAXI@Z 10006070 f i ClarkBuildWorker.obj
 0001:00005100       ??_EClarkBuildValidator@LocalWorkflow@U2@@UAEPAXI@Z 10006100 f i ClarkBuildWorker.obj
 0001:00005100       ??_GClarkBuildValidator@LocalWorkflow@U2@@UAEPAXI@Z 10006100 f i ClarkBuildWorker.obj
 0001:00005130       ??_EClarkBuildWorker@LocalWorkflow@U2@@UAEPAXI@Z 10006130 f i ClarkBuildWorker.obj
 0001:00005130       ??_GClarkBuildWorker@LocalWorkflow@U2@@UAEPAXI@Z 10006130 f i ClarkBuildWorker.obj
 0001:00005160       ??_GClarkBuildWorkerFactory@LocalWorkflow@U2@@UAEPAXI@Z 10006160 f i ClarkBuildWorker.obj
 0001:00005160       ??_EClarkBuildWorkerFactory@LocalWorkflow@U2@@UAEPAXI@Z 10006160 f i ClarkBuildWorker.obj
 0001:00005190       ??_EComboBoxDelegate@U2@@UAEPAXI@Z 10006190 f i ClarkBuildWorker.obj
 0001:00005190       ??_GComboBoxDelegate@U2@@UAEPAXI@Z 10006190 f i ClarkBuildWorker.obj
 0001:000051c0       ??_GDataset@U2@@QAEPAXI@Z  100061c0 f i ClarkBuildWorker.obj
 0001:000051f0       ??_GDelegateEditor@U2@@UAEPAXI@Z 100061f0 f i ClarkBuildWorker.obj
 0001:000051f0       ??_EDelegateEditor@U2@@UAEPAXI@Z 100061f0 f i ClarkBuildWorker.obj
 0001:00005220       ??_EDescriptor@U2@@UAEPAXI@Z 10006220 f i ClarkBuildWorker.obj
 0001:00005220       ??_GDescriptor@U2@@UAEPAXI@Z 10006220 f i ClarkBuildWorker.obj
 0001:00005250       ??_EExternalToolRunTask@U2@@UAEPAXI@Z 10006250 f i ClarkBuildWorker.obj
 0001:00005250       ??_GExternalToolRunTask@U2@@UAEPAXI@Z 10006250 f i ClarkBuildWorker.obj
 0001:00005280       ??_EFailTask@U2@@UAEPAXI@Z 10006280 f i ClarkBuildWorker.obj
 0001:00005280       ??_GFailTask@U2@@UAEPAXI@Z 10006280 f i ClarkBuildWorker.obj
 0001:000052b0       ??_EGenomicLibraryDelegate@LocalWorkflow@U2@@UAEPAXI@Z 100062b0 f i ClarkBuildWorker.obj
 0001:000052b0       ??_GGenomicLibraryDelegate@LocalWorkflow@U2@@UAEPAXI@Z 100062b0 f i ClarkBuildWorker.obj
 0001:000052e0       ??_GIntegralBusActorPrototype@Workflow@U2@@UAEPAXI@Z 100062e0 f i ClarkBuildWorker.obj
 0001:000052e0       ??_EIntegralBusActorPrototype@Workflow@U2@@UAEPAXI@Z 100062e0 f i ClarkBuildWorker.obj
 0001:00005310       ??_EMapDataType@U2@@UAEPAXI@Z 10006310 f i ClarkBuildWorker.obj
 0001:00005310       ??_GMapDataType@U2@@UAEPAXI@Z 10006310 f i ClarkBuildWorker.obj
 0001:00005340       ??_EPortDescriptor@Workflow@U2@@UAEPAXI@Z 10006340 f i ClarkBuildWorker.obj
 0001:00005340       ??_GPortDescriptor@Workflow@U2@@UAEPAXI@Z 10006340 f i ClarkBuildWorker.obj
 0001:00005370       ??_GQScriptValue@@QAEPAXI@Z 10006370 f i ClarkBuildWorker.obj
 0001:000053a0       ??_GQString@@QAEPAXI@Z     100063a0 f i ClarkBuildWorker.obj
 0001:000053d0       ??_GQVariant@@QAEPAXI@Z    100063d0 f i ClarkBuildWorker.obj
 0001:00005400       ??_ETaskSignalMapper@U2@@UAEPAXI@Z 10006400 f i ClarkBuildWorker.obj
 0001:00005400       ??_GTaskSignalMapper@U2@@UAEPAXI@Z 10006400 f i ClarkBuildWorker.obj
 0001:00005430       ??_EURLDelegate@U2@@UAEPAXI@Z 10006430 f i ClarkBuildWorker.obj
 0001:00005430       ??_GURLDelegate@U2@@UAEPAXI@Z 10006430 f i ClarkBuildWorker.obj
 0001:00005460       ??_GWorkflowNotification@U2@@QAEPAXI@Z 10006460 f i ClarkBuildWorker.obj
 0001:00005490       ??_G_Generic_error_category@std@@UAEPAXI@Z 10006490 f i ClarkBuildWorker.obj
 0001:00005490       ??_E_Generic_error_category@std@@UAEPAXI@Z 10006490 f i ClarkBuildWorker.obj
 0001:000054c0       ??_G_Iostream_error_category@std@@UAEPAXI@Z 100064c0 f i ClarkBuildWorker.obj
 0001:000054c0       ??_E_Iostream_error_category@std@@UAEPAXI@Z 100064c0 f i ClarkBuildWorker.obj
 0001:000054f0       ??_G_System_error_category@std@@UAEPAXI@Z 100064f0 f i ClarkBuildWorker.obj
 0001:000054f0       ??_E_System_error_category@std@@UAEPAXI@Z 100064f0 f i ClarkBuildWorker.obj
 0001:00005520       ??_Eerror_category@std@@UAEPAXI@Z 10006520 f i ClarkBuildWorker.obj
 0001:00005520       ??_Gerror_category@std@@UAEPAXI@Z 10006520 f i ClarkBuildWorker.obj
 0001:00005550       ?Construct@?$QMetaTypeFunctionHelper@V?$QList@VDataset@U2@@@@$00@QtMetaTypePrivate@@SAPAXPAXPBX@Z 10006550 f i ClarkBuildWorker.obj
 0001:000055e0       ?Create@?$QMetaTypeFunctionHelper@V?$QList@VDataset@U2@@@@$00@QtMetaTypePrivate@@SAPAXPBX@Z 100065e0 f i ClarkBuildWorker.obj
 0001:00005680       ?Delete@?$QMetaTypeFunctionHelper@V?$QList@VDataset@U2@@@@$00@QtMetaTypePrivate@@SAXPAX@Z 10006680 f i ClarkBuildWorker.obj
 0001:000056c0       ?Destruct@?$QMetaTypeFunctionHelper@V?$QList@VDataset@U2@@@@$00@QtMetaTypePrivate@@SAXPAX@Z 100066c0 f i ClarkBuildWorker.obj
 0001:000056f0       ?_Copy@?$basic_string@DU?$char_traits@D@std@@V?$allocator@D@2@@std@@QAEXII@Z 100066f0 f i ClarkBuildWorker.obj
 0001:00005840       ?_Eos@?$basic_string@DU?$char_traits@D@std@@V?$allocator@D@2@@std@@QAEXI@Z 10006840 f i ClarkBuildWorker.obj
 0001:00005870       ?_Getal@?$_String_alloc@$0A@U?$_String_base_types@DV?$allocator@D@std@@@std@@@std@@QBE?AU?$_Wrap_alloc@V?$allocator@D@std@@@2@XZ 10006870 f i ClarkBuildWorker.obj
 0001:00005880       ?_Grow@?$basic_string@DU?$char_traits@D@std@@V?$allocator@D@2@@std@@QAE_NI_N@Z 10006880 f i ClarkBuildWorker.obj
 0001:00005930       ?_Inside@?$basic_string@DU?$char_traits@D@std@@V?$allocator@D@2@@std@@QAE_NPBD@Z 10006930 f i ClarkBuildWorker.obj
 0001:00005970       ?_Myptr@?$_String_val@U?$_Simple_types@D@std@@@std@@QAEPADXZ 10006970 f i ClarkBuildWorker.obj
 0001:00005980       ?_Myptr@?$_String_val@U?$_Simple_types@D@std@@@std@@QBEPBDXZ 10006980 f i ClarkBuildWorker.obj
 0001:00005990       ?_Tidy@?$basic_string@DU?$char_traits@D@std@@V?$allocator@D@2@@std@@QAEX_NI@Z 10006990 f i ClarkBuildWorker.obj
 0001:000059e0       ?_Xlen@?$basic_string@DU?$char_traits@D@std@@V?$allocator@D@2@@std@@QBEXXZ 100069e0 f i ClarkBuildWorker.obj
 0001:000059f0       ?_Xran@?$basic_string@DU?$char_traits@D@std@@V?$allocator@D@2@@std@@QBEXXZ 100069f0 f i ClarkBuildWorker.obj
 0001:00005a00       ?allocate@?$_Wrap_alloc@V?$allocator@D@std@@@std@@QAEPADI@Z 10006a00 f i ClarkBuildWorker.obj
 0001:00005a30       ?allocate@?$allocator@D@std@@QAEPADI@Z 10006a30 f i ClarkBuildWorker.obj
 0001:00005a60       ?append@?$QList@PAVAttribute@U2@@@@QAEXABQAVAttribute@U2@@@Z 10006a60 f i ClarkBuildWorker.obj
 0001:00005af0       ?append@?$QList@PAVPortDescriptor@Workflow@U2@@@@QAEXABQAVPortDescriptor@Workflow@U2@@@Z 10006af0 f i ClarkBuildWorker.obj
 0001:00005b80       ?append@?$QList@VDescriptor@U2@@@@QAEXABVDescriptor@U2@@@Z 10006b80 f i ClarkBuildWorker.obj
 0001:00005c70       ?append@?$QList@VQString@@@@QAEXABVQString@@@Z 10006c70 f i ClarkBuildWorker.obj
 0001:00005d60       ?append@?$QList@VWorkflowNotification@U2@@@@QAEXABVWorkflowNotification@U2@@@Z 10006d60 f i ClarkBuildWorker.obj
 0001:00005e40       ?assign@?$basic_string@DU?$char_traits@D@std@@V?$allocator@D@2@@std@@QAEAAV12@ABV12@II@Z 10006e40 f i ClarkBuildWorker.obj
 0001:00005f60       ?assign@?$basic_string@DU?$char_traits@D@std@@V?$allocator@D@2@@std@@QAEAAV12@PBD@Z 10006f60 f i ClarkBuildWorker.obj
 0001:00005fa0       ?assign@?$basic_string@DU?$char_traits@D@std@@V?$allocator@D@2@@std@@QAEAAV12@PBDI@Z 10006fa0 f i ClarkBuildWorker.obj
 0001:000060a0       ?assign@?$char_traits@D@std@@SAXAADABD@Z 100070a0 f i ClarkBuildWorker.obj
 0001:000060b0       ?begin@?$QList@PAVPort@Workflow@U2@@@@QBE?AVconst_iterator@1@XZ 100070b0 f i ClarkBuildWorker.obj
 0001:000060d0       ?begin@?$QList@VDescriptor@U2@@@@QBE?AVconst_iterator@1@XZ 100070d0 f i ClarkBuildWorker.obj
 0001:000060f0       ?begin@?$QList@VQString@@@@QBE?AVconst_iterator@1@XZ 100070f0 f i ClarkBuildWorker.obj
 0001:00006110       ?begin@?$QMap@VDescriptor@U2@@VQVariant@@@@QBE?AVconst_iterator@1@XZ 10007110 f i ClarkBuildWorker.obj
 0001:00006130       ?begin@?$QMapData@VDescriptor@U2@@VQVariant@@@@QAEPAU?$QMapNode@VDescriptor@U2@@VQVariant@@@@XZ 10007130 f i ClarkBuildWorker.obj
 0001:00006140       ?category@error_code@std@@QBEABVerror_category@2@XZ 10007140 f i ClarkBuildWorker.obj
 0001:00006150       ?category@error_condition@std@@QBEABVerror_category@2@XZ 10007150 f i ClarkBuildWorker.obj
 0001:00006160       ?cleanup@?$QScopedPointerDeleter@VExternalToolRunTask@U2@@@@SAXPAVExternalToolRunTask@U2@@@Z 10007160 f i ClarkBuildWorker.obj
 0001:00006180       ?cleanup@ClarkBuildWorker@LocalWorkflow@U2@@MAEXXZ 10007180 f i ClarkBuildWorker.obj
 0001:00006190       ?cleanup@ClarkBuildWorkerFactory@LocalWorkflow@U2@@SAXXZ 10007190 f   ClarkBuildWorker.obj
 0001:000061e0       ?composeRichDoc@ClarkBuildPrompter@LocalWorkflow@U2@@MAE?AVQString@@XZ 100071e0 f   ClarkBuildWorker.obj
 0001:00006310       ?copy@?$QMapNode@VDescriptor@U2@@V?$QExplicitlySharedDataPointer@VDataType@U2@@@@@@QBEPAU1@PAU?$QMapData@VDescriptor@U2@@V?$QExplicitlySharedDataPointer@VDataType@U2@@@@@@@Z 10007310 f i ClarkBuildWorker.obj
 0001:000063a0       ?copy@?$QMapNode@VQString@@PAVPropertyDelegate@U2@@@@QBEPAU1@PAU?$QMapData@VQString@@PAVPropertyDelegate@U2@@@@@Z 100073a0 f i ClarkBuildWorker.obj
 0001:00006430       ?copy@?$QMapNode@VQString@@VQScriptValue@@@@QBEPAU1@PAU?$QMapData@VQString@@VQScriptValue@@@@@Z 10007430 f i ClarkBuildWorker.obj
 0001:000064c0       ?copy@?$QMapNode@VQString@@VQVariant@@@@QBEPAU1@PAU?$QMapData@VQString@@VQVariant@@@@@Z 100074c0 f i ClarkBuildWorker.obj
 0001:00006550       ?copy@?$char_traits@D@std@@SAPADPADPBDI@Z 10007550 f i ClarkBuildWorker.obj
 0001:00006570       ?create@?$QMapData@VDescriptor@U2@@V?$QExplicitlySharedDataPointer@VDataType@U2@@@@@@SAPAU1@XZ 10007570 f i ClarkBuildWorker.obj
 0001:00006580       ?create@?$QMapData@VQString@@PAVPropertyDelegate@U2@@@@SAPAU1@XZ 10007580 f i ClarkBuildWorker.obj
 0001:00006590       ?create@?$QMapData@VQString@@VQScriptValue@@@@SAPAU1@XZ 10007590 f i ClarkBuildWorker.obj
 0001:000065a0       ?create@?$QMapData@VQString@@VQVariant@@@@SAPAU1@XZ 100075a0 f i ClarkBuildWorker.obj
 0001:000065b0       ?createDescription@?$PrompterBase@VClarkBuildPrompter@LocalWorkflow@U2@@@U2@@UAEPAVActorDocument@Workflow@2@PAVActor@42@@Z 100075b0 f i ClarkBuildWorker.obj
 0001:00006850       ?createNode@?$QMapData@VDescriptor@U2@@V?$QExplicitlySharedDataPointer@VDataType@U2@@@@@@QAEPAU?$QMapNode@VDescriptor@U2@@V?$QExplicitlySharedDataPointer@VDataType@U2@@@@@@ABVDescriptor@U2@@ABV?$QExplicitlySharedDataPointer@VDataType@U2@@@@PAU2@_N@Z 10007850 f i ClarkBuildWorker.obj
 0001:00006910       ?createNode@?$QMapData@VQString@@PAVPropertyDelegate@U2@@@@QAEPAU?$QMapNode@VQString@@PAVPropertyDelegate@U2@@@@ABVQString@@ABQAVPropertyDelegate@U2@@PAU2@_N@Z 10007910 f i ClarkBuildWorker.obj
 0001:000069b0       ?createNode@?$QMapData@VQString@@VQScriptValue@@@@QAEPAU?$QMapNode@VQString@@VQScriptValue@@@@ABVQString@@ABVQScriptValue@@PAU2@_N@Z 100079b0 f i ClarkBuildWorker.obj
 0001:00006a70       ?createNode@?$QMapData@VQString@@VQVariant@@@@QAEPAU?$QMapNode@VQString@@VQVariant@@@@ABVQString@@ABVQVariant@@PAU2@_N@Z 10007a70 f i ClarkBuildWorker.obj
 0001:00006b30       ?createWorker@ClarkBuildWorkerFactory@LocalWorkflow@U2@@UAEPAVWorker@Workflow@3@PAVActor@53@@Z 10007b30 f i ClarkBuildWorker.obj
 0001:00006bc0       ?data@?$QScopedPointer@VExternalToolRunTask@U2@@U?$QScopedPointerDeleter@VExternalToolRunTask@U2@@@@@@QBEPAVExternalToolRunTask@U2@@XZ 10007bc0 f i ClarkBuildWorker.obj
 0001:00006bd0       ?dealloc@?$QList@PAVAttribute@U2@@@@AAEXPAUData@QListData@@@Z 10007bd0 f i ClarkBuildWorker.obj
 0001:00006bf0       ?dealloc@?$QList@PAVExternalToolListener@U2@@@@AAEXPAUData@QListData@@@Z 10007bf0 f i ClarkBuildWorker.obj
 0001:00006c10       ?dealloc@?$QList@PAVPort@Workflow@U2@@@@AAEXPAUData@QListData@@@Z 10007c10 f i ClarkBuildWorker.obj
 0001:00006c30       ?dealloc@?$QList@PAVPortDescriptor@Workflow@U2@@@@AAEXPAUData@QListData@@@Z 10007c30 f i ClarkBuildWorker.obj
 0001:00006c50       ?dealloc@?$QList@VDataset@U2@@@@AAEXPAUData@QListData@@@Z 10007c50 f i ClarkBuildWorker.obj
 0001:00006cb0       ?dealloc@?$QList@VDescriptor@U2@@@@AAEXPAUData@QListData@@@Z 10007cb0 f i ClarkBuildWorker.obj
 0001:00006d00       ?dealloc@?$QList@VQString@@@@AAEXPAUData@QListData@@@Z 10007d00 f i ClarkBuildWorker.obj
 0001:00006d40       ?dealloc@?$QList@VWorkflowNotification@U2@@@@AAEXPAUData@QListData@@@Z 10007d40 f i ClarkBuildWorker.obj
 0001:00006da0       ?deallocate@?$_Wrap_alloc@V?$allocator@D@std@@@std@@QAEXPADI@Z 10007da0 f i ClarkBuildWorker.obj
 0001:00006dc0       ?deallocate@?$allocator@D@std@@QAEXPADI@Z 10007dc0 f i ClarkBuildWorker.obj
 0001:00006de0       ?default_error_condition@_System_error_category@std@@UBE?AVerror_condition@2@H@Z 10007de0 f i ClarkBuildWorker.obj
 0001:00006e20       ?default_error_condition@error_category@std@@UBE?AVerror_condition@2@H@Z 10007e20 f i ClarkBuildWorker.obj
 0001:00006e40       ?deref@?$QBasicAtomicInteger@H@@QAE_NXZ 10007e40 f i ClarkBuildWorker.obj
 0001:00006e50       ?deref@RefCount@QtPrivate@@QAE_NXZ 10007e50 f i ClarkBuildWorker.obj
 0001:00006e70       ?destroy@?$QMapData@VDescriptor@U2@@V?$QExplicitlySharedDataPointer@VDataType@U2@@@@@@QAEXXZ 10007e70 f i ClarkBuildWorker.obj
 0001:00006ea0       ?destroy@?$QMapData@VQString@@PAVPropertyDelegate@U2@@@@QAEXXZ 10007ea0 f i ClarkBuildWorker.obj
 0001:00006ef0       ?destroy@?$QMapData@VQString@@VQScriptValue@@@@QAEXXZ 10007ef0 f i ClarkBuildWorker.obj
 0001:00006f20       ?destroy@?$QMapData@VQString@@VQVariant@@@@QAEXXZ 10007f20 f i ClarkBuildWorker.obj
 0001:00006f50       ?destroySubTree@?$QMapNode@VDescriptor@U2@@V?$QExplicitlySharedDataPointer@VDataType@U2@@@@@@QAEXXZ 10007f50 f i ClarkBuildWorker.obj
 0001:00006fa0       ?destroySubTree@?$QMapNode@VQString@@PAVPropertyDelegate@U2@@@@QAEXXZ 10007fa0 f i ClarkBuildWorker.obj
 0001:00006fd0       ?destroySubTree@?$QMapNode@VQString@@VQScriptValue@@@@QAEXXZ 10007fd0 f i ClarkBuildWorker.obj
 0001:00007010       ?destroySubTree@?$QMapNode@VQString@@VQVariant@@@@QAEXXZ 10008010 f i ClarkBuildWorker.obj
 0001:00007050       ?detach@?$QMap@VDescriptor@U2@@V?$QExplicitlySharedDataPointer@VDataType@U2@@@@@@QAEXXZ 10008050 f i ClarkBuildWorker.obj
 0001:00007070       ?detach@?$QMap@VQString@@PAVPropertyDelegate@U2@@@@QAEXXZ 10008070 f i ClarkBuildWorker.obj
 0001:00007090       ?detach@?$QMap@VQString@@VQScriptValue@@@@QAEXXZ 10008090 f i ClarkBuildWorker.obj
 0001:000070b0       ?detach@?$QMap@VQString@@VQVariant@@@@QAEXXZ 100080b0 f i ClarkBuildWorker.obj
 0001:000070d0       ?detach_helper@?$QList@VDescriptor@U2@@@@AAEXH@Z 100080d0 f i ClarkBuildWorker.obj
 0001:000071a0       ?detach_helper@?$QMap@VDescriptor@U2@@V?$QExplicitlySharedDataPointer@VDataType@U2@@@@@@AAEXXZ 100081a0 f i ClarkBuildWorker.obj
 0001:00007220       ?detach_helper@?$QMap@VQString@@PAVPropertyDelegate@U2@@@@AAEXXZ 10008220 f i ClarkBuildWorker.obj
 0001:000072d0       ?detach_helper@?$QMap@VQString@@VQScriptValue@@@@AAEXXZ 100082d0 f i ClarkBuildWorker.obj
 0001:00007350       ?detach_helper@?$QMap@VQString@@VQVariant@@@@AAEXXZ 10008350 f i ClarkBuildWorker.obj
 0001:000073d0       ?detach_helper_grow@?$QList@PAVAttribute@U2@@@@AAEPAUNode@1@HH@Z 100083d0 f i ClarkBuildWorker.obj
 0001:000074e0       ?detach_helper_grow@?$QList@PAVPortDescriptor@Workflow@U2@@@@AAEPAUNode@1@HH@Z 100084e0 f i ClarkBuildWorker.obj
 0001:000075f0       ?detach_helper_grow@?$QList@VDescriptor@U2@@@@AAEPAUNode@1@HH@Z 100085f0 f i ClarkBuildWorker.obj
 0001:00007740       ?detach_helper_grow@?$QList@VQString@@@@AAEPAUNode@1@HH@Z 10008740 f i ClarkBuildWorker.obj
 0001:000078c0       ?detach_helper_grow@?$QList@VWorkflowNotification@U2@@@@AAEPAUNode@1@HH@Z 100088c0 f i ClarkBuildWorker.obj
 0001:00007a10       ?end@?$QList@PAVPort@Workflow@U2@@@@QBE?AVconst_iterator@1@XZ 10008a10 f i ClarkBuildWorker.obj
 0001:00007a30       ?end@?$QList@VDescriptor@U2@@@@QBE?AVconst_iterator@1@XZ 10008a30 f i ClarkBuildWorker.obj
 0001:00007a50       ?end@?$QList@VQString@@@@QBE?AVconst_iterator@1@XZ 10008a50 f i ClarkBuildWorker.obj
 0001:00007a70       ?end@?$QMap@VDescriptor@U2@@VQVariant@@@@QBE?AVconst_iterator@1@XZ 10008a70 f i ClarkBuildWorker.obj
 0001:00007a90       ?end@?$QMapData@VDescriptor@U2@@V?$QExplicitlySharedDataPointer@VDataType@U2@@@@@@QAEPAU?$QMapNode@VDescriptor@U2@@V?$QExplicitlySharedDataPointer@VDataType@U2@@@@@@XZ 10008a90 f i ClarkBuildWorker.obj
 0001:00007aa0       ?end@?$QMapData@VDescriptor@U2@@VQVariant@@@@QAEPAU?$QMapNode@VDescriptor@U2@@VQVariant@@@@XZ 10008aa0 f i ClarkBuildWorker.obj
 0001:00007ab0       ?end@?$QMapData@VQString@@PAVPropertyDelegate@U2@@@@QAEPAU?$QMapNode@VQString@@PAVPropertyDelegate@U2@@@@XZ 10008ab0 f i ClarkBuildWorker.obj
 0001:00007ac0       ?end@?$QMapData@VQString@@VQScriptValue@@@@QAEPAU?$QMapNode@VQString@@VQScriptValue@@@@XZ 10008ac0 f i ClarkBuildWorker.obj
 0001:00007ad0       ?end@?$QMapData@VQString@@VQVariant@@@@QAEPAU?$QMapNode@VQString@@VQVariant@@@@XZ 10008ad0 f i ClarkBuildWorker.obj
 0001:00007ae0       ?equivalent@error_category@std@@UBE_NABVerror_code@2@H@Z 10008ae0 f i ClarkBuildWorker.obj
 0001:00007b00       ?equivalent@error_category@std@@UBE_NHABVerror_condition@2@@Z 10008b00 f i ClarkBuildWorker.obj
 0001:00007b40       ?erase@?$basic_string@DU?$char_traits@D@std@@V?$allocator@D@2@@std@@QAEAAV12@I@Z 10008b40 f i ClarkBuildWorker.obj
 0001:00007b80       ?erase@?$basic_string@DU?$char_traits@D@std@@V?$allocator@D@2@@std@@QAEAAV12@II@Z 10008b80 f i ClarkBuildWorker.obj
 0001:00007c20       ?findNode@?$QMapData@VDescriptor@U2@@V?$QExplicitlySharedDataPointer@VDataType@U2@@@@@@QBEPAU?$QMapNode@VDescriptor@U2@@V?$QExplicitlySharedDataPointer@VDataType@U2@@@@@@ABVDescriptor@U2@@@Z 10008c20 f i ClarkBuildWorker.obj
 0001:00007c60       ?findNode@?$QMapData@VDescriptor@U2@@VQVariant@@@@QBEPAU?$QMapNode@VDescriptor@U2@@VQVariant@@@@ABVDescriptor@U2@@@Z 10008c60 f i ClarkBuildWorker.obj
 0001:00007ca0       ?findNode@?$QMapData@VQString@@PAVIntegralBus@Workflow@U2@@@@QBEPAU?$QMapNode@VQString@@PAVIntegralBus@Workflow@U2@@@@ABVQString@@@Z 10008ca0 f i ClarkBuildWorker.obj
 0001:00007ce0       ?findNode@?$QMapData@VQString@@PAVPropertyDelegate@U2@@@@QBEPAU?$QMapNode@VQString@@PAVPropertyDelegate@U2@@@@ABVQString@@@Z 10008ce0 f i ClarkBuildWorker.obj
 0001:00007d20       ?findNode@?$QMapData@VQString@@VQScriptValue@@@@QBEPAU?$QMapNode@VQString@@VQScriptValue@@@@ABVQString@@@Z 10008d20 f i ClarkBuildWorker.obj
 0001:00007d60       ?findNode@?$QMapData@VQString@@VQVariant@@@@QBEPAU?$QMapNode@VQString@@VQVariant@@@@ABVQString@@@Z 10008d60 f i ClarkBuildWorker.obj
 0001:00007da0       ?generic_category@std@@YAABVerror_category@1@XZ 10008da0 f i ClarkBuildWorker.obj
 0001:00007db0       ?getArguments@ClarkBuildTask@LocalWorkflow@U2@@AAE?AVQStringList@@XZ 10008db0 f   ClarkBuildWorker.obj
 0001:00007e90       ?getDbUrl@ClarkBuildTask@LocalWorkflow@U2@@QBEABVQString@@XZ 10008e90 f i ClarkBuildWorker.obj
 0001:00007ea0       ?init@ClarkBuildWorker@LocalWorkflow@U2@@MAEXXZ 10008ea0 f   ClarkBuildWorker.obj
 0001:00008060       ?init@ClarkBuildWorkerFactory@LocalWorkflow@U2@@SAXXZ 10009060 f   ClarkBuildWorker.obj
 0001:00008c90       ?insert@?$QMap@VDescriptor@U2@@V?$QExplicitlySharedDataPointer@VDataType@U2@@@@@@QAE?AViterator@1@ABVDescriptor@U2@@ABV?$QExplicitlySharedDataPointer@VDataType@U2@@@@@Z 10009c90 f i ClarkBuildWorker.obj
 0001:00008d90       ?insert@?$QMap@VQString@@PAVPropertyDelegate@U2@@@@QAE?AViterator@1@ABVQString@@ABQAVPropertyDelegate@U2@@@Z 10009d90 f i ClarkBuildWorker.obj
 0001:00008e50       ?insert@?$QMap@VQString@@VQScriptValue@@@@QAE?AViterator@1@ABVQString@@ABVQScriptValue@@@Z 10009e50 f i ClarkBuildWorker.obj
 0001:00008f10       ?insert@?$QMap@VQString@@VQVariant@@@@QAE?AViterator@1@ABVQString@@ABVQVariant@@@Z 10009f10 f i ClarkBuildWorker.obj
 0001:00008fd0       ?invoke@?$MetaTypeInvoker@U?$QVariantValueHelper@H@QtPrivate@@ABVQVariant@@H@QtPrivate@@SAHABVQVariant@@@Z 10009fd0 f i ClarkBuildWorker.obj
 0001:00009010       ?invoke@?$MetaTypeInvoker@U?$QVariantValueHelper@V?$QList@VDataset@U2@@@@@QtPrivate@@ABVQVariant@@V?$QList@VDataset@U2@@@@@QtPrivate@@SA?AV?$QList@VDataset@U2@@@@ABVQVariant@@@Z 1000a010 f i ClarkBuildWorker.obj
 0001:00009030       ?invoke@?$MetaTypeInvoker@U?$QVariantValueHelper@VQString@@@QtPrivate@@ABVQVariant@@VQString@@@QtPrivate@@SA?AVQString@@ABVQVariant@@@Z 1000a030 f i ClarkBuildWorker.obj
 0001:00009050       ?isEmpty@?$QList@VQString@@@@QBE_NXZ 1000a050 f i ClarkBuildWorker.obj
 0001:00009060       ?isError@ClarkBuildLogParser@LocalWorkflow@U2@@EBE_NABVQString@@@Z 1000a060 f i ClarkBuildWorker.obj
 0001:000091d0       ?isShared@RefCount@QtPrivate@@QBE_NXZ 1000a1d0 f i ClarkBuildWorker.obj
 0001:000091f0       ?join@QStringList@@QBE?AVQString@@ABV2@@Z 1000a1f0 f i ClarkBuildWorker.obj
 0001:00009230       ?key@const_iterator@?$QMap@VDescriptor@U2@@VQVariant@@@@QBEABVDescriptor@U2@@XZ 1000a230 f i ClarkBuildWorker.obj
 0001:00009240       ?leftNode@?$QMapNode@VDescriptor@U2@@V?$QExplicitlySharedDataPointer@VDataType@U2@@@@@@QBEPAU1@XZ 1000a240 f i ClarkBuildWorker.obj
 0001:00009250       ?leftNode@?$QMapNode@VDescriptor@U2@@VQVariant@@@@QBEPAU1@XZ 1000a250 f i ClarkBuildWorker.obj
 0001:00009260       ?leftNode@?$QMapNode@VQString@@PAVIntegralBus@Workflow@U2@@@@QBEPAU1@XZ 1000a260 f i ClarkBuildWorker.obj
 0001:00009270       ?leftNode@?$QMapNode@VQString@@PAVPropertyDelegate@U2@@@@QBEPAU1@XZ 1000a270 f i ClarkBuildWorker.obj
 0001:00009280       ?leftNode@?$QMapNode@VQString@@VQScriptValue@@@@QBEPAU1@XZ 1000a280 f i ClarkBuildWorker.obj
 0001:00009290       ?leftNode@?$QMapNode@VQString@@VQVariant@@@@QBEPAU1@XZ 1000a290 f i ClarkBuildWorker.obj
 0001:000092a0       ?length@?$char_traits@D@std@@SAIPBD@Z 1000a2a0 f i ClarkBuildWorker.obj
 0001:000092c0       ?load@?$QBasicAtomicInteger@H@@QBEHXZ 1000a2c0 f i ClarkBuildWorker.obj
 0001:000092d0       ?loadAcquire@?$QBasicAtomicInteger@H@@QBEHXZ 1000a2d0 f i ClarkBuildWorker.obj
 0001:000092e0       ?lowerBound@?$QMapNode@VDescriptor@U2@@V?$QExplicitlySharedDataPointer@VDataType@U2@@@@@@QAEPAU1@ABVDescriptor@U2@@@Z 1000a2e0 f i ClarkBuildWorker.obj
 0001:00009320       ?lowerBound@?$QMapNode@VDescriptor@U2@@VQVariant@@@@QAEPAU1@ABVDescriptor@U2@@@Z 1000a320 f i ClarkBuildWorker.obj
 0001:00009360       ?lowerBound@?$QMapNode@VQString@@PAVIntegralBus@Workflow@U2@@@@QAEPAU1@ABVQString@@@Z 1000a360 f i ClarkBuildWorker.obj
 0001:000093a0       ?lowerBound@?$QMapNode@VQString@@PAVPropertyDelegate@U2@@@@QAEPAU1@ABVQString@@@Z 1000a3a0 f i ClarkBuildWorker.obj
 0001:000093e0       ?lowerBound@?$QMapNode@VQString@@VQScriptValue@@@@QAEPAU1@ABVQString@@@Z 1000a3e0 f i ClarkBuildWorker.obj
 0001:00009420       ?lowerBound@?$QMapNode@VQString@@VQVariant@@@@QAEPAU1@ABVQString@@@Z 1000a420 f i ClarkBuildWorker.obj
 0001:00009460       ?max_size@?$_Wrap_alloc@V?$allocator@D@std@@@std@@QBEIXZ 1000a460 f i ClarkBuildWorker.obj
 0001:00009470       ?max_size@?$allocator@D@std@@QBEIXZ 1000a470 f i ClarkBuildWorker.obj
 0001:00009480       ?max_size@?$allocator_traits@V?$allocator@D@std@@@std@@SAIABV?$allocator@D@2@@Z 1000a480 f i ClarkBuildWorker.obj
 0001:00009490       ?max_size@?$basic_string@DU?$char_traits@D@std@@V?$allocator@D@2@@std@@QBEIXZ 1000a490 f i ClarkBuildWorker.obj
 0001:000094a0       ?message@_Generic_error_category@std@@UBE?AV?$basic_string@DU?$char_traits@D@std@@V?$allocator@D@2@@2@H@Z 1000a4a0 f i ClarkBuildWorker.obj
 0001:00009520       ?message@_Iostream_error_category@std@@UBE?AV?$basic_string@DU?$char_traits@D@std@@V?$allocator@D@2@@2@H@Z 1000a520 f i ClarkBuildWorker.obj
 0001:00009570       ?message@_System_error_category@std@@UBE?AV?$basic_string@DU?$char_traits@D@std@@V?$allocator@D@2@@2@H@Z 1000a570 f i ClarkBuildWorker.obj
 0001:000095f0       ?metaType@?$QVariantValueHelper@H@QtPrivate@@SAHABVQVariant@@@Z 1000a5f0 f i ClarkBuildWorker.obj
 0001:00009630       ?metaType@?$QVariantValueHelper@V?$QList@VDataset@U2@@@@@QtPrivate@@SA?AV?$QList@VDataset@U2@@@@ABVQVariant@@@Z 1000a630 f i ClarkBuildWorker.obj
 0001:00009720       ?metaType@?$QVariantValueHelper@VQString@@@QtPrivate@@SA?AVQString@@ABVQVariant@@@Z 1000a720 f i ClarkBuildWorker.obj
 0001:000097e0       ?move@?$char_traits@D@std@@SAPADPADPBDI@Z 1000a7e0 f i ClarkBuildWorker.obj
 0001:00009800       ?name@_Generic_error_category@std@@UBEPBDXZ 1000a800 f i ClarkBuildWorker.obj
 0001:00009810       ?name@_Iostream_error_category@std@@UBEPBDXZ 1000a810 f i ClarkBuildWorker.obj
 0001:00009820       ?name@_System_error_category@std@@UBEPBDXZ 1000a820 f i ClarkBuildWorker.obj
 0001:00009830       ?nextNode@?$QMapNode@VDescriptor@U2@@VQVariant@@@@QBEPBU1@XZ 1000a830 f i ClarkBuildWorker.obj
 0001:00009840       ?node_construct@?$QList@PAVAttribute@U2@@@@AAEXPAUNode@1@ABQAVAttribute@U2@@@Z 1000a840 f i ClarkBuildWorker.obj
 0001:00009860       ?node_construct@?$QList@PAVPortDescriptor@Workflow@U2@@@@AAEXPAUNode@1@ABQAVPortDescriptor@Workflow@U2@@@Z 1000a860 f i ClarkBuildWorker.obj
 0001:00009880       ?node_construct@?$QList@VDescriptor@U2@@@@AAEXPAUNode@1@ABVDescriptor@U2@@@Z 1000a880 f i ClarkBuildWorker.obj
 0001:00009910       ?node_construct@?$QList@VQString@@@@AAEXPAUNode@1@ABVQString@@@Z 1000a910 f i ClarkBuildWorker.obj
 0001:00009960       ?node_construct@?$QList@VWorkflowNotification@U2@@@@AAEXPAUNode@1@ABVWorkflowNotification@U2@@@Z 1000a960 f i ClarkBuildWorker.obj
 0001:000099e0       ?node_copy@?$QList@PAVAttribute@U2@@@@AAEXPAUNode@1@00@Z 1000a9e0 f i ClarkBuildWorker.obj
 0001:00009a10       ?node_copy@?$QList@PAVPort@Workflow@U2@@@@AAEXPAUNode@1@00@Z 1000aa10 f i ClarkBuildWorker.obj
 0001:00009a40       ?node_copy@?$QList@PAVPortDescriptor@Workflow@U2@@@@AAEXPAUNode@1@00@Z 1000aa40 f i ClarkBuildWorker.obj
 0001:00009a70       ?node_copy@?$QList@VDataset@U2@@@@AAEXPAUNode@1@00@Z 1000aa70 f i ClarkBuildWorker.obj
 0001:00009b40       ?node_copy@?$QList@VDescriptor@U2@@@@AAEXPAUNode@1@00@Z 1000ab40 f i ClarkBuildWorker.obj
 0001:00009c10       ?node_copy@?$QList@VQString@@@@AAEXPAUNode@1@00@Z 1000ac10 f i ClarkBuildWorker.obj
 0001:00009cb0       ?node_copy@?$QList@VWorkflowNotification@U2@@@@AAEXPAUNode@1@00@Z 1000acb0 f i ClarkBuildWorker.obj
 0001:00009d80       ?node_destruct@?$QList@PAVAttribute@U2@@@@AAEXPAUNode@1@0@Z 1000ad80 f i ClarkBuildWorker.obj
 0001:00009d90       ?node_destruct@?$QList@PAVAttribute@U2@@@@AAEXPAUNode@1@@Z 1000ad90 f i ClarkBuildWorker.obj
 0001:00009da0       ?node_destruct@?$QList@PAVExternalToolListener@U2@@@@AAEXPAUNode@1@0@Z 1000ada0 f i ClarkBuildWorker.obj
 0001:00009db0       ?node_destruct@?$QList@PAVPort@Workflow@U2@@@@AAEXPAUNode@1@0@Z 1000adb0 f i ClarkBuildWorker.obj
 0001:00009dc0       ?node_destruct@?$QList@PAVPortDescriptor@Workflow@U2@@@@AAEXPAUNode@1@0@Z 1000adc0 f i ClarkBuildWorker.obj
 0001:00009dd0       ?node_destruct@?$QList@PAVPortDescriptor@Workflow@U2@@@@AAEXPAUNode@1@@Z 1000add0 f i ClarkBuildWorker.obj
 0001:00009de0       ?node_destruct@?$QList@VDataset@U2@@@@AAEXPAUNode@1@0@Z 1000ade0 f i ClarkBuildWorker.obj
 0001:00009e20       ?node_destruct@?$QList@VDescriptor@U2@@@@AAEXPAUNode@1@0@Z 1000ae20 f i ClarkBuildWorker.obj
 0001:00009e50       ?node_destruct@?$QList@VDescriptor@U2@@@@AAEXPAUNode@1@@Z 1000ae50 f i ClarkBuildWorker.obj
 0001:00009e70       ?node_destruct@?$QList@VQString@@@@AAEXPAUNode@1@0@Z 1000ae70 f i ClarkBuildWorker.obj
 0001:00009ea0       ?node_destruct@?$QList@VQString@@@@AAEXPAUNode@1@@Z 1000aea0 f i ClarkBuildWorker.obj
 0001:00009eb0       ?node_destruct@?$QList@VWorkflowNotification@U2@@@@AAEXPAUNode@1@0@Z 1000aeb0 f i ClarkBuildWorker.obj
 0001:00009ef0       ?node_destruct@?$QList@VWorkflowNotification@U2@@@@AAEXPAUNode@1@@Z 1000aef0 f i ClarkBuildWorker.obj
 0001:00009f20       ?prepare@ClarkBuildTask@LocalWorkflow@U2@@EAEXXZ 1000af20 f   ClarkBuildWorker.obj
 0001:0000a300       ?qt_metatype_id@?$QMetaTypeId2@H@@SAHXZ 1000b300 f i ClarkBuildWorker.obj
 0001:0000a310       ?qt_metatype_id@?$QMetaTypeId2@V?$QList@VDataset@U2@@@@@@SAHXZ 1000b310 f i ClarkBuildWorker.obj
 0001:0000a320       ?qt_metatype_id@?$QMetaTypeId2@VQString@@@@SAHXZ 1000b320 f i ClarkBuildWorker.obj
 0001:0000a330       ?qt_metatype_id@?$QMetaTypeId@V?$QList@VDataset@U2@@@@@@SAHXZ 1000b330 f i ClarkBuildWorker.obj
 0001:0000a3d0       ?qt_metatype_id@?$QMetaTypeIdHelper@V?$QList@VDataset@U2@@@@$00@QtPrivate@@SAHXZ 1000b3d0 f i ClarkBuildWorker.obj
 0001:0000a3e0       ?qt_noop@@YAXXZ            1000b3e0 f i ClarkBuildWorker.obj
 0001:0000a3f0       ?ref@?$QBasicAtomicInteger@H@@QAE_NXZ 1000b3f0 f i ClarkBuildWorker.obj
 0001:0000a410       ?ref@RefCount@QtPrivate@@QAE_NXZ 1000b410 f i ClarkBuildWorker.obj
 0001:0000a430       ?registerConverter@?$AssociativeContainerConverterHelper@V?$QList@VDataset@U2@@@@$0A@@QtPrivate@@SA_NH@Z 1000b430 f i ClarkBuildWorker.obj
 0001:0000a440       ?registerConverter@?$IsPair@V?$QList@VDataset@U2@@@@@QtPrivate@@SA_NH@Z 1000b440 f i ClarkBuildWorker.obj
 0001:0000a450       ?registerConverter@?$MetaTypeSmartPointerHelper@V?$QList@VDataset@U2@@@@X@QtPrivate@@SA_NH@Z 1000b450 f i ClarkBuildWorker.obj
 0001:0000a460       ?registerConverter@?$ValueTypeIsMetaType@V?$QList@VDataset@U2@@@@$0A@@QtPrivate@@SA_NH@Z 1000b460 f i ClarkBuildWorker.obj
 0001:0000a470       ?reserve@?$QList@VDescriptor@U2@@@@QAEXH@Z 1000b470 f i ClarkBuildWorker.obj
 0001:0000a4a0       ?rightNode@?$QMapNode@VDescriptor@U2@@V?$QExplicitlySharedDataPointer@VDataType@U2@@@@@@QBEPAU1@XZ 1000b4a0 f i ClarkBuildWorker.obj
 0001:0000a4b0       ?rightNode@?$QMapNode@VDescriptor@U2@@VQVariant@@@@QBEPAU1@XZ 1000b4b0 f i ClarkBuildWorker.obj
 0001:0000a4c0       ?rightNode@?$QMapNode@VQString@@PAVIntegralBus@Workflow@U2@@@@QBEPAU1@XZ 1000b4c0 f i ClarkBuildWorker.obj
 0001:0000a4d0       ?rightNode@?$QMapNode@VQString@@PAVPropertyDelegate@U2@@@@QBEPAU1@XZ 1000b4d0 f i ClarkBuildWorker.obj
 0001:0000a4e0       ?rightNode@?$QMapNode@VQString@@VQScriptValue@@@@QBEPAU1@XZ 1000b4e0 f i ClarkBuildWorker.obj
 0001:0000a4f0       ?rightNode@?$QMapNode@VQString@@VQVariant@@@@QBEPAU1@XZ 1000b4f0 f i ClarkBuildWorker.obj
 0001:0000a500       ?root@?$QMapData@VDescriptor@U2@@V?$QExplicitlySharedDataPointer@VDataType@U2@@@@@@QBEPAU?$QMapNode@VDescriptor@U2@@V?$QExplicitlySharedDataPointer@VDataType@U2@@@@@@XZ 1000b500 f i ClarkBuildWorker.obj
 0001:0000a510       ?root@?$QMapData@VDescriptor@U2@@VQVariant@@@@QBEPAU?$QMapNode@VDescriptor@U2@@VQVariant@@@@XZ 1000b510 f i ClarkBuildWorker.obj
 0001:0000a520       ?root@?$QMapData@VQString@@PAVIntegralBus@Workflow@U2@@@@QBEPAU?$QMapNode@VQString@@PAVIntegralBus@Workflow@U2@@@@XZ 1000b520 f i ClarkBuildWorker.obj
 0001:0000a530       ?root@?$QMapData@VQString@@PAVPropertyDelegate@U2@@@@QBEPAU?$QMapNode@VQString@@PAVPropertyDelegate@U2@@@@XZ 1000b530 f i ClarkBuildWorker.obj
 0001:0000a540       ?root@?$QMapData@VQString@@VQScriptValue@@@@QBEPAU?$QMapNode@VQString@@VQScriptValue@@@@XZ 1000b540 f i ClarkBuildWorker.obj
 0001:0000a550       ?root@?$QMapData@VQString@@VQVariant@@@@QBEPAU?$QMapNode@VQString@@VQVariant@@@@XZ 1000b550 f i ClarkBuildWorker.obj
 0001:0000a560       ?size@?$QMap@VDescriptor@U2@@VQVariant@@@@QBEHXZ 1000b560 f i ClarkBuildWorker.obj
 0001:0000a570       ?size@?$basic_string@DU?$char_traits@D@std@@V?$allocator@D@2@@std@@QBEIXZ 1000b570 f i ClarkBuildWorker.obj
 0001:0000a580       ?sl_taskFinished@ClarkBuildWorker@LocalWorkflow@U2@@AAEXPAVTask@3@@Z 1000b580 f   ClarkBuildWorker.obj
 0001:0000a8d0       ?storeRelease@?$QBasicAtomicInteger@H@@QAEXH@Z 1000b8d0 f i ClarkBuildWorker.obj
 0001:0000a8e0       ?system_category@std@@YAABVerror_category@1@XZ 1000b8e0 f i ClarkBuildWorker.obj
 0001:0000a8f0       ?t@Node@?$QList@PAVPort@Workflow@U2@@@@QAEAAPAVPort@Workflow@U2@@XZ 1000b8f0 f i ClarkBuildWorker.obj
 0001:0000a900       ?t@Node@?$QList@VDescriptor@U2@@@@QAEAAVDescriptor@U2@@XZ 1000b900 f i ClarkBuildWorker.obj
 0001:0000a910       ?t@Node@?$QList@VQString@@@@QAEAAVQString@@XZ 1000b910 f i ClarkBuildWorker.obj
 0001:0000a920       ?take@?$QScopedPointer@VExternalToolRunTask@U2@@U?$QScopedPointerDeleter@VExternalToolRunTask@U2@@@@@@QAEPAVExternalToolRunTask@U2@@XZ 1000b920 f i ClarkBuildWorker.obj
 0001:0000a930       ?tick@ClarkBuildWorker@LocalWorkflow@U2@@MAEPAVTask@3@XZ 1000b930 f   ClarkBuildWorker.obj
 0001:0000ac30       ?tr@ClarkBuildPrompter@LocalWorkflow@U2@@SA?AVQString@@PBD0H@Z 1000bc30 f i ClarkBuildWorker.obj
 0001:0000ac60       ?tr@ClarkBuildTask@LocalWorkflow@U2@@SA?AVQString@@PBD0H@Z 1000bc60 f i ClarkBuildWorker.obj
 0001:0000ac90       ?tr@ClarkBuildValidator@LocalWorkflow@U2@@SA?AVQString@@PBD0H@Z 1000bc90 f i ClarkBuildWorker.obj
 0001:0000acc0       ?tr@ClarkBuildWorker@LocalWorkflow@U2@@SA?AVQString@@PBD0H@Z 1000bcc0 f i ClarkBuildWorker.obj
 0001:0000acf0       ?uniqueKeys@?$QMap@VDescriptor@U2@@VQVariant@@@@QBE?AV?$QList@VDescriptor@U2@@@@XZ 1000bcf0 f i ClarkBuildWorker.obj
 0001:0000adf0       ?validate@ClarkBuildValidator@LocalWorkflow@U2@@UBE_NPBVActor@Workflow@3@AAV?$QList@VWorkflowNotification@U2@@@@ABV?$QMap@VQString@@V1@@@@Z 1000bdf0 f   ClarkBuildWorker.obj
 0001:0000ae10       ?validateTaxonomy@ClarkBuildValidator@LocalWorkflow@U2@@ABE_NPBVActor@Workflow@3@AAV?$QList@VWorkflowNotification@U2@@@@@Z 1000be10 f   ClarkBuildWorker.obj
 0001:0000b2f0       ?value@?$MetaObjectForType@V?$QList@VDataset@U2@@@@$0A@@QtPrivate@@SAPBUQMetaObject@@XZ 1000c2f0 f i ClarkBuildWorker.obj
 0001:0000b300       ?value@?$QMap@VDescriptor@U2@@VQVariant@@@@QBE?BVQVariant@@ABVDescriptor@U2@@ABV2@@Z 1000c300 f i ClarkBuildWorker.obj
 0001:0000b360       ?value@?$QMap@VQString@@PAVIntegralBus@Workflow@U2@@@@QBEQAVIntegralBus@Workflow@U2@@ABVQString@@ABQAV234@@Z 1000c360 f i ClarkBuildWorker.obj
 0001:0000b3b0       ?value@error_code@std@@QBEHXZ 1000c3b0 f i ClarkBuildWorker.obj
 0001:0000b3c0       ?value@error_condition@std@@QBEHXZ 1000c3c0 f i ClarkBuildWorker.obj
 0001:0000b3d0       _hypot                     1000c3d0 f i ClarkBuildWorker.obj
 0001:0000b400       ??$?0V?$QMap@VQString@@I@@@QAssociativeIterableImpl@QtMetaTypePrivate@@QAE@PBV?$QMap@VQString@@I@@@Z 1000c400 f i ClarkClassifyWorker.obj
 0001:0000b470       ??$_Advance@Vconst_iterator@?$QMap@VQString@@I@@H@std@@YAXAAVconst_iterator@?$QMap@VQString@@I@@HUbidirectional_iterator_tag@0@@Z 1000c470 f i ClarkClassifyWorker.obj
 0001:0000b4b0       ??$_Distance2@Vconst_iterator@?$QMap@VQString@@I@@H@std@@YAXVconst_iterator@?$QMap@VQString@@I@@0AAHUbidirectional_iterator_tag@0@@Z 1000c4b0 f i ClarkClassifyWorker.obj
 0001:0000b4e0       ??$_Iter_cat@Vconst_iterator@?$QMap@VQString@@I@@@std@@YA?AUbidirectional_iterator_tag@0@ABVconst_iterator@?$QMap@VQString@@I@@@Z 1000c4e0 f i ClarkClassifyWorker.obj
 0001:0000b4f0       ??$advance@Vconst_iterator@?$QMap@VQString@@I@@H@std@@YAXAAVconst_iterator@?$QMap@VQString@@I@@H@Z 1000c4f0 f i ClarkClassifyWorker.obj
 0001:0000b530       ??$advanceImpl@V?$QMap@VQString@@I@@@QAssociativeIterableImpl@QtMetaTypePrivate@@SAXPAPAXH@Z 1000c530 f i ClarkClassifyWorker.obj
 0001:0000b570       ??$beginImpl@V?$QMap@VQString@@I@@@QAssociativeIterableImpl@QtMetaTypePrivate@@SAXPBXPAPAX@Z 1000c570 f i ClarkClassifyWorker.obj
 0001:0000b5b0       ??$distance@Vconst_iterator@?$QMap@VQString@@I@@@std@@YAHVconst_iterator@?$QMap@VQString@@I@@0@Z 1000c5b0 f i ClarkClassifyWorker.obj
 0001:0000b5e0       ??$endImpl@V?$QMap@VQString@@I@@@QAssociativeIterableImpl@QtMetaTypePrivate@@SAXPBXPAPAX@Z 1000c5e0 f i ClarkClassifyWorker.obj
 0001:0000b610       ??$findImpl@V?$QMap@VQString@@I@@@QAssociativeIterableImpl@QtMetaTypePrivate@@SAXPBX0PAPAX@Z 1000c610 f i ClarkClassifyWorker.obj
 0001:0000b670       ??$fromValue@V?$QMap@VQString@@I@@@QVariant@@SA?AV0@ABV?$QMap@VQString@@I@@@Z 1000c670 f i ClarkClassifyWorker.obj
 0001:0000b690       ??$getAttributeValue@_N@Attribute@U2@@QBE_NPAVWorkflowContext@Workflow@1@@Z 1000c690 f i ClarkClassifyWorker.obj
 0001:0000b6d0       ??$getAttributeValueWithoutScript@_N@Attribute@U2@@QBE_NXZ 1000c6d0 f i ClarkClassifyWorker.obj
 0001:0000b710       ??$getKeyImpl@V?$QMap@VQString@@I@@@QAssociativeIterableImpl@QtMetaTypePrivate@@SA?AUVariantData@1@PBQAXHI@Z 1000c710 f i ClarkClassifyWorker.obj
 0001:0000b730       ??$getValue@_N@BaseWorker@LocalWorkflow@U2@@IBE_NABVQString@@@Z 1000c730 f i ClarkClassifyWorker.obj
 0001:0000b790       ??$getValueImpl@V?$QMap@VQString@@I@@@QAssociativeIterableImpl@QtMetaTypePrivate@@SA?AUVariantData@1@PBQAXHI@Z 1000c790 f i ClarkClassifyWorker.obj
 0001:0000b7b0       ??$qMetaTypeId@I@@YAHXZ    1000c7b0 f i ClarkClassifyWorker.obj
 0001:0000b7c0       ??$qMetaTypeId@V?$QMap@VQString@@I@@@@YAHXZ 1000c7c0 f i ClarkClassifyWorker.obj
 0001:0000b7d0       ??$qMetaTypeId@VQAssociativeIterableImpl@QtMetaTypePrivate@@@@YAHXZ 1000c7d0 f i ClarkClassifyWorker.obj
 0001:0000b7e0       ??$qMetaTypeId@_N@@YAHXZ   1000c7e0 f i ClarkClassifyWorker.obj
 0001:0000b7f0       ??$qRegisterMetaType@V?$QMap@VQString@@I@@@@YAHPBDPAV?$QMap@VQString@@I@@W4DefinedType@?$MetaTypeDefinedHelper@V?$QMap@VQString@@I@@$00@QtPrivate@@@Z 1000c7f0 f i ClarkClassifyWorker.obj
 0001:0000b860       ??$qRegisterMetaType@VQAssociativeIterableImpl@QtMetaTypePrivate@@@@YAHPBDPAVQAssociativeIterableImpl@QtMetaTypePrivate@@W4DefinedType@?$MetaTypeDefinedHelper@VQAssociativeIterableImpl@QtMetaTypePrivate@@$00@QtPrivate@@@Z 1000c860 f i ClarkClassifyWorker.obj
 0001:0000b920       ??$qRegisterNormalizedMetaType@V?$QMap@VQString@@I@@@@YAHABVQByteArray@@PAV?$QMap@VQString@@I@@W4DefinedType@?$MetaTypeDefinedHelper@V?$QMap@VQString@@I@@$00@QtPrivate@@@Z 1000c920 f i ClarkClassifyWorker.obj
 0001:0000b990       ??$qRegisterNormalizedMetaType@VQAssociativeIterableImpl@QtMetaTypePrivate@@@@YAHABVQByteArray@@PAVQAssociativeIterableImpl@QtMetaTypePrivate@@W4DefinedType@?$MetaTypeDefinedHelper@VQAssociativeIterableImpl@QtMetaTypePrivate@@$00@QtPrivate@@@Z 1000c990 f i ClarkClassifyWorker.obj
 0001:0000b9f0       ??$qVariantFromValue@V?$QMap@VQString@@I@@@@YA?AVQVariant@@ABV?$QMap@VQString@@I@@@Z 1000c9f0 f i ClarkClassifyWorker.obj
 0001:0000ba20       ??$qobject_cast@PAVClarkClassifyTask@LocalWorkflow@U2@@@@YAPAVClarkClassifyTask@LocalWorkflow@U2@@PAVQObject@@@Z 1000ca20 f i ClarkClassifyWorker.obj
 0001:0000ba40       ??$qvariant_cast@_N@@YA_NABVQVariant@@@Z 1000ca40 f i ClarkClassifyWorker.obj
 0001:0000ba80       ??$sizeImpl@V?$QMap@VQString@@I@@@QAssociativeIterableImpl@QtMetaTypePrivate@@SAHPBX@Z 1000ca80 f i ClarkClassifyWorker.obj
 0001:0000bac0       ??$value@_N@QVariant@@QBE_NXZ 1000cac0 f i ClarkClassifyWorker.obj
 0001:0000bb00       ??0?$ConverterFunctor@V?$QMap@VQString@@I@@VQAssociativeIterableImpl@QtMetaTypePrivate@@U?$QAssociativeIterableConvertFunctor@V?$QMap@VQString@@I@@@3@@QtPrivate@@QAE@U?$QAssociativeIterableConvertFunctor@V?$QMap@VQString@@I@@@QtMetaTypePrivate@@@Z 1000cb00 f i ClarkClassifyWorker.obj
 0001:0000bb10       ??0?$PrompterBase@VClarkClassifyPrompter@LocalWorkflow@U2@@@U2@@QAE@PAVActor@Workflow@1@_N@Z 1000cb10 f i ClarkClassifyWorker.obj
 0001:0000bb40       ??0?$QFlags@W4Filter@QDir@@@@QAE@W4Filter@QDir@@@Z 1000cb40 f i ClarkClassifyWorker.obj
 0001:0000bb50       ??0?$QFlags@W4Flag@Attribute@U2@@@@QAE@VQFlag@@@Z 1000cb50 f i ClarkClassifyWorker.obj
 0001:0000bb60       ??0?$QFlags@W4Flag@Attribute@U2@@@@QAE@W4Flag@Attribute@U2@@@Z 1000cb60 f i ClarkClassifyWorker.obj
 0001:0000bb70       ??0?$QFlags@W4SortFlag@QDir@@@@QAE@W4SortFlag@QDir@@@Z 1000cb70 f i ClarkClassifyWorker.obj
 0001:0000bb80       ??0?$QForeachContainer@V?$QList@VQString@@@@@@QAE@ABV?$QList@VQString@@@@@Z 1000cb80 f i ClarkClassifyWorker.obj
 0001:0000bbc0       ??0?$QForeachContainer@VQStringList@@@@QAE@ABVQStringList@@@Z 1000cbc0 f i ClarkClassifyWorker.obj
 0001:0000bc00       ??0?$QHash@VQString@@UQHashDummyValue@@@@QAE@XZ 1000cc00 f i ClarkClassifyWorker.obj
 0001:0000bc10       ??0?$QList@U?$QPair@VQString@@V1@@@@@QAE@XZ 1000cc10 f i ClarkClassifyWorker.obj
 0001:0000bc20       ??0?$QList@VQString@@@@QAE@$$QAV0@@Z 1000cc20 f i ClarkClassifyWorker.obj
 0001:0000bc40       ??0?$QList@VQVariant@@@@QAE@XZ 1000cc40 f i ClarkClassifyWorker.obj
 0001:0000bc50       ??0?$QMap@VQString@@I@@QAE@ABV0@@Z 1000cc50 f i ClarkClassifyWorker.obj
 0001:0000bcc0       ??0?$QMap@VQString@@I@@QAE@XZ 1000ccc0 f i ClarkClassifyWorker.obj
 0001:0000bcd0       ??0?$QMap@VQString@@V1@@@QAE@$$QAV0@@Z 1000ccd0 f i ClarkClassifyWorker.obj
 0001:0000bcf0       ??0?$QMap@VQString@@V1@@@QAE@XZ 1000ccf0 f i ClarkClassifyWorker.obj
 0001:0000bd00       ??0?$QPair@VQString@@V1@@@QAE@ABU0@@Z 1000cd00 f i ClarkClassifyWorker.obj
 0001:0000bd60       ??0?$QPair@VQString@@V1@@@QAE@ABVQString@@0@Z 1000cd60 f i ClarkClassifyWorker.obj
 0001:0000bdc0       ??0?$QSet@VQString@@@@QAE@XZ 1000cdc0 f i ClarkClassifyWorker.obj
 0001:0000bdd0       ??0AbstractConverterFunction@QtPrivate@@QAE@P6A_NPBU01@PBXPAX@Z@Z 1000cdd0 f i ClarkClassifyWorker.obj
 0001:0000bde0       ??0ClarkClassifyPrompter@LocalWorkflow@U2@@QAE@PAVActor@Workflow@2@@Z 1000cde0 f i ClarkClassifyWorker.obj
 0001:0000be10       ??0ClarkClassifySettings@LocalWorkflow@U2@@QAE@ABV012@@Z 1000ce10 f i ClarkClassifyWorker.obj
 0001:0000bea0       ??0ClarkClassifySettings@LocalWorkflow@U2@@QAE@XZ 1000cea0 f   ClarkClassifyWorker.obj
 0001:0000bf30       ??0ClarkClassifyTask@LocalWorkflow@U2@@QAE@ABVClarkClassifySettings@12@ABVQString@@11@Z 1000cf30 f   ClarkClassifyWorker.obj
 0001:0000c180       ??0ClarkClassifyValidator@LocalWorkflow@U2@@QAE@XZ 1000d180 f i ClarkClassifyWorker.obj
 0001:0000c190       ??0ClarkClassifyWorker@LocalWorkflow@U2@@QAE@PAVActor@Workflow@2@@Z 1000d190 f   ClarkClassifyWorker.obj
 0001:0000c260       ??0ClarkClassifyWorkerFactory@LocalWorkflow@U2@@QAE@XZ 1000d260 f i ClarkClassifyWorker.obj
 0001:0000c280       ??0ClarkLogParser@LocalWorkflow@U2@@QAE@XZ 1000d280 f   ClarkClassifyWorker.obj
 0001:0000c2a0       ??0QAssociativeIterableImpl@QtMetaTypePrivate@@QAE@XZ 1000d2a0 f i ClarkClassifyWorker.obj
 0001:0000c310       ??0QStringList@@QAE@ABVQString@@@Z 1000d310 f i ClarkClassifyWorker.obj
 0001:0000c370       ??0VariantData@QtMetaTypePrivate@@QAE@HPBXI@Z 1000d370 f i ClarkClassifyWorker.obj
 0001:0000c390       ??0const_iterator@?$QMap@VQString@@I@@QAE@PBU?$QMapNode@VQString@@I@@@Z 1000d390 f i ClarkClassifyWorker.obj
 0001:0000c3a0       ??0const_iterator@?$QMap@VQString@@I@@QAE@XZ 1000d3a0 f i ClarkClassifyWorker.obj
 0001:0000c3b0       ??0const_iterator@?$QMap@VQString@@V1@@@QAE@PBU?$QMapNode@VQString@@V1@@@@Z 1000d3b0 f i ClarkClassifyWorker.obj
 0001:0000c3c0       ??0iterator@?$QMap@VQString@@I@@QAE@PAU?$QMapNode@VQString@@I@@@Z 1000d3c0 f i ClarkClassifyWorker.obj
 0001:0000c3d0       ??0iterator@?$QMap@VQString@@V1@@@QAE@PAU?$QMapNode@VQString@@V1@@@@Z 1000d3d0 f i ClarkClassifyWorker.obj
 0001:0000c3e0       ??1?$ConverterFunctor@V?$QMap@VQString@@I@@VQAssociativeIterableImpl@QtMetaTypePrivate@@U?$QAssociativeIterableConvertFunctor@V?$QMap@VQString@@I@@@3@@QtPrivate@@QAE@XZ 1000d3e0 f i ClarkClassifyWorker.obj
 0001:0000c400       ??1?$PrompterBase@VClarkClassifyPrompter@LocalWorkflow@U2@@@U2@@UAE@XZ 1000d400 f i ClarkClassifyWorker.obj
 0001:0000c410       ??1?$QForeachContainer@V?$QList@VQString@@@@@@QAE@XZ 1000d410 f i ClarkClassifyWorker.obj
 0001:0000c420       ??1?$QForeachContainer@VQStringList@@@@QAE@XZ 1000d420 f i ClarkClassifyWorker.obj
 0001:0000c430       ??1?$QHash@VQString@@UQHashDummyValue@@@@QAE@XZ 1000d430 f i ClarkClassifyWorker.obj
 0001:0000c460       ??1?$QHashNode@VQString@@UQHashDummyValue@@@@QAE@XZ 1000d460 f i ClarkClassifyWorker.obj
 0001:0000c470       ??1?$QList@U?$QPair@VQString@@V1@@@@@QAE@XZ 1000d470 f i ClarkClassifyWorker.obj
 0001:0000c4c0       ??1?$QList@VQByteArray@@@@QAE@XZ 1000d4c0 f i ClarkClassifyWorker.obj
 0001:0000c520       ??1?$QList@VQFileInfo@@@@QAE@XZ 1000d520 f i ClarkClassifyWorker.obj
 0001:0000c590       ??1?$QList@VQVariant@@@@QAE@XZ 1000d590 f i ClarkClassifyWorker.obj
 0001:0000c5c0       ??1?$QMap@VQString@@I@@QAE@XZ 1000d5c0 f i ClarkClassifyWorker.obj
 0001:0000c630       ??1?$QMap@VQString@@V1@@@QAE@XZ 1000d630 f i ClarkClassifyWorker.obj
 0001:0000c680       ??1?$QPair@VQString@@V1@@@QAE@XZ 1000d680 f i ClarkClassifyWorker.obj
 0001:0000c6e0       ??1?$QSet@VQString@@@@QAE@XZ 1000d6e0 f i ClarkClassifyWorker.obj
 0001:0000c710       ??1ClarkClassifyPrompter@LocalWorkflow@U2@@UAE@XZ 1000d710 f i ClarkClassifyWorker.obj
 0001:0000c720       ??1ClarkClassifySettings@LocalWorkflow@U2@@QAE@XZ 1000d720 f i ClarkClassifyWorker.obj
 0001:0000c780       ??1ClarkClassifyTask@LocalWorkflow@U2@@UAE@XZ 1000d780 f i ClarkClassifyWorker.obj
 0001:0000c830       ??1ClarkClassifyValidator@LocalWorkflow@U2@@UAE@XZ 1000d830 f i ClarkClassifyWorker.obj
 0001:0000c840       ??1ClarkClassifyWorker@LocalWorkflow@U2@@UAE@XZ 1000d840 f i ClarkClassifyWorker.obj
 0001:0000c8c0       ??1ClarkClassifyWorkerFactory@LocalWorkflow@U2@@UAE@XZ 1000d8c0 f i ClarkClassifyWorker.obj
 0001:0000c8d0       ??1ClarkLogParser@LocalWorkflow@U2@@UAE@XZ 1000d8d0 f i ClarkClassifyWorker.obj
 0001:0000c8e0       ??6?$QList@U?$QPair@VQString@@V1@@@@@QAEAAV0@ABU?$QPair@VQString@@V1@@@@Z 1000d8e0 f i ClarkClassifyWorker.obj
 0001:0000c900       ??6?$QList@VQVariant@@@@QAEAAV0@ABVQVariant@@@Z 1000d900 f i ClarkClassifyWorker.obj
 0001:0000c920       ??8const_iterator@?$QMap@VQString@@I@@QBE_NABV01@@Z 1000d920 f i ClarkClassifyWorker.obj
 0001:0000c940       ??9@YA_NABVQByteArray@@PBD@Z 1000d940 f i ClarkClassifyWorker.obj
 0001:0000c970       ??9const_iterator@?$QMap@VQString@@I@@QBE_NABV01@@Z 1000d970 f i ClarkClassifyWorker.obj
 0001:0000c990       ??9const_iterator@?$QMap@VQString@@V1@@@QBE_NABV01@@Z 1000d990 f i ClarkClassifyWorker.obj
 0001:0000c9b0       ??Econst_iterator@?$QMap@VQString@@I@@QAEAAV01@XZ 1000d9b0 f i ClarkClassifyWorker.obj
 0001:0000c9d0       ??Econst_iterator@?$QMap@VQString@@V1@@@QAEAAV01@XZ 1000d9d0 f i ClarkClassifyWorker.obj
 0001:0000c9f0       ??Fconst_iterator@?$QMap@VQString@@I@@QAEAAV01@XZ 1000d9f0 f i ClarkClassifyWorker.obj
 0001:0000ca10       ??H@YA?BVQString@@ABV0@0@Z 1000da10 f i ClarkClassifyWorker.obj
 0001:0000ca80       ??R?$QAssociativeIterableConvertFunctor@V?$QMap@VQString@@I@@@QtMetaTypePrivate@@QBE?AVQAssociativeIterableImpl@1@ABV?$QMap@VQString@@I@@@Z 1000da80 f i ClarkClassifyWorker.obj
 0001:0000caa0       ??U?$QFlags@W4Flag@Attribute@U2@@@@QBE?AV0@W4Flag@Attribute@U2@@@Z 1000daa0 f i ClarkClassifyWorker.obj
 0001:0000cac0       ??U@YA?AV?$QFlags@W4Flag@Attribute@U2@@@@W4Flag@Attribute@U2@@0@Z 1000dac0 f i ClarkClassifyWorker.obj
 0001:0000cad0       ??_E?$PrompterBase@VClarkClassifyPrompter@LocalWorkflow@U2@@@U2@@WM@AEPAXI@Z 1000dad0 f i ClarkClassifyWorker.obj
 0001:0000cad8       ??_EClarkClassifyPrompter@LocalWorkflow@U2@@WM@AEPAXI@Z 1000dad8 f i ClarkClassifyWorker.obj
 0001:0000cae0       ??_EClarkClassifyWorker@LocalWorkflow@U2@@W7AEPAXI@Z 1000dae0 f i ClarkClassifyWorker.obj
 0001:0000cae8       ??_EClarkClassifyWorker@LocalWorkflow@U2@@WBA@AEPAXI@Z 1000dae8 f i ClarkClassifyWorker.obj
 0001:0000caf0       ??_EClarkClassifyWorkerFactory@LocalWorkflow@U2@@W7AEPAXI@Z 1000daf0 f i ClarkClassifyWorker.obj
 0001:0000cb00       ??_G?$PrompterBase@VClarkClassifyPrompter@LocalWorkflow@U2@@@U2@@UAEPAXI@Z 1000db00 f i ClarkClassifyWorker.obj
 0001:0000cb00       ??_E?$PrompterBase@VClarkClassifyPrompter@LocalWorkflow@U2@@@U2@@UAEPAXI@Z 1000db00 f i ClarkClassifyWorker.obj
 0001:0000cb30       ??_G?$QHashNode@VQString@@UQHashDummyValue@@@@QAEPAXI@Z 1000db30 f i ClarkClassifyWorker.obj
 0001:0000cb60       ??_G?$QMap@VQString@@I@@QAEPAXI@Z 1000db60 f i ClarkClassifyWorker.obj
 0001:0000cb90       ??_G?$QPair@VQString@@V1@@@QAEPAXI@Z 1000db90 f i ClarkClassifyWorker.obj
 0001:0000cc00       ??_EClarkClassifyPrompter@LocalWorkflow@U2@@UAEPAXI@Z 1000dc00 f i ClarkClassifyWorker.obj
 0001:0000cc00       ??_GClarkClassifyPrompter@LocalWorkflow@U2@@UAEPAXI@Z 1000dc00 f i ClarkClassifyWorker.obj
 0001:0000cc30       ??_GClarkClassifyTask@LocalWorkflow@U2@@UAEPAXI@Z 1000dc30 f i ClarkClassifyWorker.obj
 0001:0000cc30       ??_EClarkClassifyTask@LocalWorkflow@U2@@UAEPAXI@Z 1000dc30 f i ClarkClassifyWorker.obj
 0001:0000cc60       ??_GClarkClassifyValidator@LocalWorkflow@U2@@UAEPAXI@Z 1000dc60 f i ClarkClassifyWorker.obj
 0001:0000cc60       ??_EClarkClassifyValidator@LocalWorkflow@U2@@UAEPAXI@Z 1000dc60 f i ClarkClassifyWorker.obj
 0001:0000cc90       ??_EClarkClassifyWorker@LocalWorkflow@U2@@UAEPAXI@Z 1000dc90 f i ClarkClassifyWorker.obj
 0001:0000cc90       ??_GClarkClassifyWorker@LocalWorkflow@U2@@UAEPAXI@Z 1000dc90 f i ClarkClassifyWorker.obj
 0001:0000cd20       ??_GClarkClassifyWorkerFactory@LocalWorkflow@U2@@UAEPAXI@Z 1000dd20 f i ClarkClassifyWorker.obj
 0001:0000cd20       ??_EClarkClassifyWorkerFactory@LocalWorkflow@U2@@UAEPAXI@Z 1000dd20 f i ClarkClassifyWorker.obj
 0001:0000cd50       ??_EClarkLogParser@LocalWorkflow@U2@@UAEPAXI@Z 1000dd50 f i ClarkClassifyWorker.obj
 0001:0000cd50       ??_GClarkLogParser@LocalWorkflow@U2@@UAEPAXI@Z 1000dd50 f i ClarkClassifyWorker.obj
 0001:0000cd80       ??_GDatabaseDelegate@LocalWorkflow@U2@@UAEPAXI@Z 1000dd80 f i ClarkClassifyWorker.obj
 0001:0000cd80       ??_EDatabaseDelegate@LocalWorkflow@U2@@UAEPAXI@Z 1000dd80 f i ClarkClassifyWorker.obj
 0001:0000cdb0       ??_EPairedReadsPortValidator@Workflow@U2@@UAEPAXI@Z 1000ddb0 f i ClarkClassifyWorker.obj
 0001:0000cdb0       ??_GPairedReadsPortValidator@Workflow@U2@@UAEPAXI@Z 1000ddb0 f i ClarkClassifyWorker.obj
 0001:0000cde0       ??_GQByteArray@@QAEPAXI@Z  1000dde0 f i ClarkClassifyWorker.obj
 0001:0000ce10       ??_GQFileInfo@@QAEPAXI@Z   1000de10 f i ClarkClassifyWorker.obj
 0001:0000ce40       ??_ESlotRelationDescriptor@U2@@UAEPAXI@Z 1000de40 f i ClarkClassifyWorker.obj
 0001:0000ce40       ??_GSlotRelationDescriptor@U2@@UAEPAXI@Z 1000de40 f i ClarkClassifyWorker.obj
 0001:0000ce70       ??_GSpinBoxDelegate@U2@@UAEPAXI@Z 1000de70 f i ClarkClassifyWorker.obj
 0001:0000ce70       ??_ESpinBoxDelegate@U2@@UAEPAXI@Z 1000de70 f i ClarkClassifyWorker.obj
 0001:0000cea0       ??_EVisibilityRelation@U2@@UAEPAXI@Z 1000dea0 f i ClarkClassifyWorker.obj
 0001:0000cea0       ??_GVisibilityRelation@U2@@UAEPAXI@Z 1000dea0 f i ClarkClassifyWorker.obj
 0001:0000ced0       ?Construct@?$QMetaTypeFunctionHelper@V?$QMap@VQString@@I@@$00@QtMetaTypePrivate@@SAPAXPAXPBX@Z 1000ded0 f i ClarkClassifyWorker.obj
 0001:0000cf60       ?Construct@?$QMetaTypeFunctionHelper@VQAssociativeIterableImpl@QtMetaTypePrivate@@$00@QtMetaTypePrivate@@SAPAXPAXPBX@Z 1000df60 f i ClarkClassifyWorker.obj
 0001:0000cfb0       ?Create@?$QMetaTypeFunctionHelper@V?$QMap@VQString@@I@@$00@QtMetaTypePrivate@@SAPAXPBX@Z 1000dfb0 f i ClarkClassifyWorker.obj
 0001:0000d050       ?Create@?$QMetaTypeFunctionHelper@VQAssociativeIterableImpl@QtMetaTypePrivate@@$00@QtMetaTypePrivate@@SAPAXPBX@Z 1000e050 f i ClarkClassifyWorker.obj
 0001:0000d0b0       ?Delete@?$QMetaTypeFunctionHelper@V?$QMap@VQString@@I@@$00@QtMetaTypePrivate@@SAXPAX@Z 1000e0b0 f i ClarkClassifyWorker.obj
 0001:0000d0d0       ?Delete@?$QMetaTypeFunctionHelper@VQAssociativeIterableImpl@QtMetaTypePrivate@@$00@QtMetaTypePrivate@@SAXPAX@Z 1000e0d0 f i ClarkClassifyWorker.obj
 0001:0000d0e0       ?Destruct@?$QMetaTypeFunctionHelper@V?$QMap@VQString@@I@@$00@QtMetaTypePrivate@@SAXPAX@Z 1000e0e0 f i ClarkClassifyWorker.obj
 0001:0000d0f0       ?Destruct@?$QMetaTypeFunctionHelper@VQAssociativeIterableImpl@QtMetaTypePrivate@@$00@QtMetaTypePrivate@@SAXPAX@Z 1000e0f0 f i ClarkClassifyWorker.obj
 0001:0000d100       ?append@?$QList@U?$QPair@VQString@@V1@@@@@QAEXABU?$QPair@VQString@@V1@@@@Z 1000e100 f i ClarkClassifyWorker.obj
 0001:0000d190       ?append@?$QList@VQVariant@@@@QAEXABVQVariant@@@Z 1000e190 f i ClarkClassifyWorker.obj
 0001:0000d270       ?assign@?$IteratorOwnerCommon@Vconst_iterator@?$QMap@VQString@@I@@@QtMetaTypePrivate@@SAXPAPAXPBQAX@Z 1000e270 f i ClarkClassifyWorker.obj
 0001:0000d2a0       ?assign@?$IteratorOwnerCommon@Vconst_iterator@?$QMap@VQString@@I@@@QtMetaTypePrivate@@SAXPAPAXVconst_iterator@?$QMap@VQString@@I@@@Z 1000e2a0 f i ClarkClassifyWorker.obj
 0001:0000d2d0       ?at@?$QList@VQByteArray@@@@QBEABVQByteArray@@H@Z 1000e2d0 f i ClarkClassifyWorker.obj
 0001:0000d2f0       ?begin@?$QMap@VQString@@I@@QBE?AVconst_iterator@1@XZ 1000e2f0 f i ClarkClassifyWorker.obj
 0001:0000d310       ?begin@?$QMap@VQString@@V1@@@QBE?AVconst_iterator@1@XZ 1000e310 f i ClarkClassifyWorker.obj
 0001:0000d330       ?begin@?$QMapData@VQString@@I@@QAEPAU?$QMapNode@VQString@@I@@XZ 1000e330 f i ClarkClassifyWorker.obj
 0001:0000d340       ?begin@?$QMapData@VQString@@V1@@@QAEPAU?$QMapNode@VQString@@V1@@@XZ 1000e340 f i ClarkClassifyWorker.obj
 0001:0000d350       ?checkRefseqAvailability@ClarkClassifyValidator@LocalWorkflow@U2@@ABE_NPBVActor@Workflow@3@AAV?$QList@VWorkflowNotification@U2@@@@ABVQString@@@Z 1000e350 f   ClarkClassifyWorker.obj
 0001:0000d440       ?cleanup@ClarkClassifyWorker@LocalWorkflow@U2@@MAEXXZ 1000e440 f   ClarkClassifyWorker.obj
 0001:0000d450       ?cleanup@ClarkClassifyWorkerFactory@LocalWorkflow@U2@@SAXXZ 1000e450 f   ClarkClassifyWorker.obj
 0001:0000d4a0       ?composeRichDoc@ClarkClassifyPrompter@LocalWorkflow@U2@@MAE?AVQString@@XZ 1000e4a0 f   ClarkClassifyWorker.obj
 0001:0000d720       ?concrete@?$QHash@VQString@@UQHashDummyValue@@@@CAPAU?$QHashNode@VQString@@UQHashDummyValue@@@@PAUNode@QHashData@@@Z 1000e720 f i ClarkClassifyWorker.obj
 0001:0000d730       ?constFind@?$QMap@VQString@@I@@QBE?AVconst_iterator@1@ABVQString@@@Z 1000e730 f i ClarkClassifyWorker.obj
 0001:0000d780       ?contains@?$QMap@VQString@@I@@QBE_NABVQString@@@Z 1000e780 f i ClarkClassifyWorker.obj
 0001:0000d7c0       ?convert@?$ConverterFunctor@V?$QMap@VQString@@I@@VQAssociativeIterableImpl@QtMetaTypePrivate@@U?$QAssociativeIterableConvertFunctor@V?$QMap@VQString@@I@@@3@@QtPrivate@@SA_NPBUAbstractConverterFunction@2@PBXPAX@Z 1000e7c0 f i ClarkClassifyWorker.obj
 0001:0000d810       ?copy@?$QMapNode@VQString@@I@@QBEPAU1@PAU?$QMapData@VQString@@I@@@Z 1000e810 f i ClarkClassifyWorker.obj
 0001:0000d8a0       ?copy@?$QMapNode@VQString@@V1@@@QBEPAU1@PAU?$QMapData@VQString@@V1@@@@Z 1000e8a0 f i ClarkClassifyWorker.obj
 0001:0000d930       ?create@?$QMapData@VQString@@I@@SAPAU1@XZ 1000e930 f i ClarkClassifyWorker.obj
 0001:0000d940       ?create@?$QMapData@VQString@@V1@@@SAPAU1@XZ 1000e940 f i ClarkClassifyWorker.obj
 0001:0000d950       ?createDescription@?$PrompterBase@VClarkClassifyPrompter@LocalWorkflow@U2@@@U2@@UAEPAVActorDocument@Workflow@2@PAVActor@42@@Z 1000e950 f i ClarkClassifyWorker.obj
 0001:0000dbf0       ?createNode@?$QMapData@VQString@@I@@QAEPAU?$QMapNode@VQString@@I@@ABVQString@@ABIPAU2@_N@Z 1000ebf0 f i ClarkClassifyWorker.obj
 0001:0000dc90       ?createNode@?$QMapData@VQString@@V1@@@QAEPAU?$QMapNode@VQString@@V1@@@ABVQString@@0PAU2@_N@Z 1000ec90 f i ClarkClassifyWorker.obj
 0001:0000dd50       ?createWorker@ClarkClassifyWorkerFactory@LocalWorkflow@U2@@UAEPAVWorker@Workflow@3@PAVActor@53@@Z 1000ed50 f i ClarkClassifyWorker.obj
 0001:0000ddc0       ?dealloc@?$QList@U?$QPair@VQString@@V1@@@@@AAEXPAUData@QListData@@@Z 1000edc0 f i ClarkClassifyWorker.obj
 0001:0000ddf0       ?dealloc@?$QList@VQByteArray@@@@AAEXPAUData@QListData@@@Z 1000edf0 f i ClarkClassifyWorker.obj
 0001:0000de30       ?dealloc@?$QList@VQFileInfo@@@@AAEXPAUData@QListData@@@Z 1000ee30 f i ClarkClassifyWorker.obj
 0001:0000de80       ?dealloc@?$QList@VQVariant@@@@AAEXPAUData@QListData@@@Z 1000ee80 f i ClarkClassifyWorker.obj
 0001:0000dee0       ?deleteNode2@?$QHash@VQString@@UQHashDummyValue@@@@CAXPAUNode@QHashData@@@Z 1000eee0 f i ClarkClassifyWorker.obj
 0001:0000def0       ?destroy@?$IteratorOwnerCommon@Vconst_iterator@?$QMap@VQString@@I@@@QtMetaTypePrivate@@SAXPAPAX@Z 1000eef0 f i ClarkClassifyWorker.obj
 0001:0000df10       ?destroy@?$QMapData@VQString@@I@@QAEXXZ 1000ef10 f i ClarkClassifyWorker.obj
 0001:0000df60       ?destroy@?$QMapData@VQString@@V1@@@QAEXXZ 1000ef60 f i ClarkClassifyWorker.obj
 0001:0000df90       ?destroySubTree@?$QMapNode@VQString@@I@@QAEXXZ 1000ef90 f i ClarkClassifyWorker.obj
 0001:0000dfc0       ?destroySubTree@?$QMapNode@VQString@@V1@@@QAEXXZ 1000efc0 f i ClarkClassifyWorker.obj
 0001:0000dff0       ?detach@?$QMap@VQString@@I@@QAEXXZ 1000eff0 f i ClarkClassifyWorker.obj
 0001:0000e010       ?detach@?$QMap@VQString@@V1@@@QAEXXZ 1000f010 f i ClarkClassifyWorker.obj
 0001:0000e030       ?detach_helper@?$QList@VQString@@@@AAEXH@Z 1000f030 f i ClarkClassifyWorker.obj
 0001:0000e120       ?detach_helper@?$QMap@VQString@@I@@AAEXXZ 1000f120 f i ClarkClassifyWorker.obj
 0001:0000e1d0       ?detach_helper@?$QMap@VQString@@V1@@@AAEXXZ 1000f1d0 f i ClarkClassifyWorker.obj
 0001:0000e250       ?detach_helper_grow@?$QList@U?$QPair@VQString@@V1@@@@@AAEPAUNode@1@HH@Z 1000f250 f i ClarkClassifyWorker.obj
 0001:0000e3c0       ?detach_helper_grow@?$QList@VQVariant@@@@AAEPAUNode@1@HH@Z 1000f3c0 f i ClarkClassifyWorker.obj
 0001:0000e510       ?end@?$QMap@VQString@@I@@QBE?AVconst_iterator@1@XZ 1000f510 f i ClarkClassifyWorker.obj
 0001:0000e530       ?end@?$QMap@VQString@@V1@@@QBE?AVconst_iterator@1@XZ 1000f530 f i ClarkClassifyWorker.obj
 0001:0000e550       ?end@?$QMapData@VQString@@I@@QAEPAU?$QMapNode@VQString@@I@@XZ 1000f550 f i ClarkClassifyWorker.obj
 0001:0000e560       ?end@?$QMapData@VQString@@V1@@@QAEPAU?$QMapNode@VQString@@V1@@@XZ 1000f560 f i ClarkClassifyWorker.obj
 0001:0000e570       ?equal@?$IteratorOwnerCommon@Vconst_iterator@?$QMap@VQString@@I@@@QtMetaTypePrivate@@SA_NPBQAX0@Z 1000f570 f i ClarkClassifyWorker.obj
 0001:0000e590       ?find@?$QMap@VQString@@I@@QBE?AVconst_iterator@1@ABVQString@@@Z 1000f590 f i ClarkClassifyWorker.obj
 0001:0000e5e0       ?findNode@?$QMapData@VQString@@I@@QBEPAU?$QMapNode@VQString@@I@@ABVQString@@@Z 1000f5e0 f i ClarkClassifyWorker.obj
 0001:0000e620       ?findNode@?$QMapData@VQString@@V1@@@QBEPAU?$QMapNode@VQString@@V1@@@ABVQString@@@Z 1000f620 f i ClarkClassifyWorker.obj
 0001:0000e660       ?freeData@?$QHash@VQString@@UQHashDummyValue@@@@AAEXPAUQHashData@@@Z 1000f660 f i ClarkClassifyWorker.obj
 0001:0000e680       ?getArguments@ClarkClassifyTask@LocalWorkflow@U2@@AAE?AVQStringList@@XZ 1000f680 f   ClarkClassifyWorker.obj
 0001:0000ec20       ?getKey@?$AssociativeContainerAccessor@V?$QMap@VQString@@I@@$00@QtMetaTypePrivate@@SAABVQString@@ABVconst_iterator@?$QMap@VQString@@I@@@Z 1000fc20 f i ClarkClassifyWorker.obj
 0001:0000ec30       ?getParsedReport@ClarkClassifyTask@LocalWorkflow@U2@@QBEABV?$QMap@VQString@@I@@XZ 1000fc30 f   ClarkClassifyWorker.obj
 0001:0000ec40       ?getReportUrl@ClarkClassifyTask@LocalWorkflow@U2@@QBEABVQString@@XZ 1000fc40 f i ClarkClassifyWorker.obj
 0001:0000ec50       ?getValue@?$AssociativeContainerAccessor@V?$QMap@VQString@@I@@$00@QtMetaTypePrivate@@SAABIABVconst_iterator@?$QMap@VQString@@I@@@Z 1000fc50 f i ClarkClassifyWorker.obj
 0001:0000ec60       ?init@ClarkClassifyWorker@LocalWorkflow@U2@@MAEXXZ 1000fc60 f   ClarkClassifyWorker.obj
 0001:0000f1c0       ?init@ClarkClassifyWorkerFactory@LocalWorkflow@U2@@SAXXZ 100101c0 f   ClarkClassifyWorker.obj
 0001:000117d0       ?initWellKnownErrors@ClarkLogParser@LocalWorkflow@U2@@CA?AV?$QMap@VQString@@V1@@@XZ 100127d0 f   ClarkClassifyWorker.obj
 0001:000118e0       ?insert@?$QMap@VQString@@I@@QAE?AViterator@1@ABVQString@@ABI@Z 100128e0 f i ClarkClassifyWorker.obj
 0001:000119a0       ?insert@?$QMap@VQString@@V1@@@QAE?AViterator@1@ABVQString@@0@Z 100129a0 f i ClarkClassifyWorker.obj
 0001:00011a60       ?invoke@?$MetaTypeInvoker@U?$QVariantValueHelper@_N@QtPrivate@@ABVQVariant@@_N@QtPrivate@@SA_NABVQVariant@@@Z 10012a60 f i ClarkClassifyWorker.obj
 0001:00011aa0       ?isDatabaseAlreadyBuilt@ClarkClassifyValidator@LocalWorkflow@U2@@ABE_NPBVActor@Workflow@3@@Z 10012aa0 f   ClarkClassifyWorker.obj
 0001:00011df0       ?isError@ClarkLogParser@LocalWorkflow@U2@@EBE_NABVQString@@@Z 10012df0 f   ClarkClassifyWorker.obj
 0001:00011f80       ?key@const_iterator@?$QMap@VQString@@I@@QBEABVQString@@XZ 10012f80 f i ClarkClassifyWorker.obj
 0001:00011f90       ?key@const_iterator@?$QMap@VQString@@V1@@@QBEABVQString@@XZ 10012f90 f i ClarkClassifyWorker.obj
 0001:00011fa0       ?keys@?$QMap@VQString@@V1@@@QBE?AV?$QList@VQString@@@@XZ 10012fa0 f i ClarkClassifyWorker.obj
 0001:00012060       ?leftNode@?$QMapNode@VQString@@I@@QBEPAU1@XZ 10013060 f i ClarkClassifyWorker.obj
 0001:00012070       ?leftNode@?$QMapNode@VQString@@V1@@@QBEPAU1@XZ 10013070 f i ClarkClassifyWorker.obj
 0001:00012080       ?lowerBound@?$QMapNode@VQString@@I@@QAEPAU1@ABVQString@@@Z 10013080 f i ClarkClassifyWorker.obj
 0001:000120c0       ?lowerBound@?$QMapNode@VQString@@V1@@@QAEPAU1@ABVQString@@@Z 100130c0 f i ClarkClassifyWorker.obj
 0001:00012100       ?metaType@?$QVariantValueHelper@_N@QtPrivate@@SA_NABVQVariant@@@Z 10013100 f i ClarkClassifyWorker.obj
 0001:00012140       ?nextNode@?$QMapNode@VQString@@I@@QBEPBU1@XZ 10013140 f i ClarkClassifyWorker.obj
 0001:00012150       ?nextNode@?$QMapNode@VQString@@V1@@@QBEPBU1@XZ 10013150 f i ClarkClassifyWorker.obj
 0001:00012160       ?node_construct@?$QList@U?$QPair@VQString@@V1@@@@@AAEXPAUNode@1@ABU?$QPair@VQString@@V1@@@@Z 10013160 f i ClarkClassifyWorker.obj
 0001:000121f0       ?node_construct@?$QList@VQVariant@@@@AAEXPAUNode@1@ABVQVariant@@@Z 100131f0 f i ClarkClassifyWorker.obj
 0001:00012270       ?node_copy@?$QList@U?$QPair@VQString@@V1@@@@@AAEXPAUNode@1@00@Z 10013270 f i ClarkClassifyWorker.obj
 0001:00012370       ?node_copy@?$QList@VQVariant@@@@AAEXPAUNode@1@00@Z 10013370 f i ClarkClassifyWorker.obj
 0001:00012440       ?node_destruct@?$QList@U?$QPair@VQString@@V1@@@@@AAEXPAUNode@1@0@Z 10013440 f i ClarkClassifyWorker.obj
 0001:000124c0       ?node_destruct@?$QList@U?$QPair@VQString@@V1@@@@@AAEXPAUNode@1@@Z 100134c0 f i ClarkClassifyWorker.obj
 0001:00012530       ?node_destruct@?$QList@VQByteArray@@@@AAEXPAUNode@1@0@Z 10013530 f i ClarkClassifyWorker.obj
 0001:00012560       ?node_destruct@?$QList@VQFileInfo@@@@AAEXPAUNode@1@0@Z 10013560 f i ClarkClassifyWorker.obj
 0001:00012590       ?node_destruct@?$QList@VQVariant@@@@AAEXPAUNode@1@0@Z 10013590 f i ClarkClassifyWorker.obj
 0001:000125d0       ?node_destruct@?$QList@VQVariant@@@@AAEXPAUNode@1@@Z 100135d0 f i ClarkClassifyWorker.obj
 0001:00012600       ?prepare@ClarkClassifyTask@LocalWorkflow@U2@@EAEXXZ 10013600 f   ClarkClassifyWorker.obj
 0001:00012820       ?previousNode@?$QMapNode@VQString@@I@@QBEPBU1@XZ 10013820 f i ClarkClassifyWorker.obj
 0001:00012830       ?qt_metatype_id@?$QMetaTypeId2@I@@SAHXZ 10013830 f i ClarkClassifyWorker.obj
 0001:00012840       ?qt_metatype_id@?$QMetaTypeId2@V?$QMap@VQString@@I@@@@SAHXZ 10013840 f i ClarkClassifyWorker.obj
 0001:00012850       ?qt_metatype_id@?$QMetaTypeId2@VQAssociativeIterableImpl@QtMetaTypePrivate@@@@SAHXZ 10013850 f i ClarkClassifyWorker.obj
 0001:00012860       ?qt_metatype_id@?$QMetaTypeId2@_N@@SAHXZ 10013860 f i ClarkClassifyWorker.obj
 0001:00012870       ?qt_metatype_id@?$QMetaTypeId@V?$QMap@VQString@@I@@@@SAHXZ 10013870 f i ClarkClassifyWorker.obj
 0001:00012920       ?qt_metatype_id@?$QMetaTypeId@VQAssociativeIterableImpl@QtMetaTypePrivate@@@@SAHXZ 10013920 f i ClarkClassifyWorker.obj
 0001:000129c0       ?qt_metatype_id@?$QMetaTypeIdHelper@V?$QMap@VQString@@I@@$00@QtPrivate@@SAHXZ 100139c0 f i ClarkClassifyWorker.obj
 0001:000129d0       ?qt_metatype_id@?$QMetaTypeIdHelper@VQAssociativeIterableImpl@QtMetaTypePrivate@@$00@QtPrivate@@SAHXZ 100139d0 f i ClarkClassifyWorker.obj
 0001:000129e0       ?registerConverter@?$AssociativeContainerConverterHelper@VQAssociativeIterableImpl@QtMetaTypePrivate@@$0A@@QtPrivate@@SA_NH@Z 100139e0 f i ClarkClassifyWorker.obj
 0001:000129f0       ?registerConverter@?$AssociativeValueTypeIsMetaType@V?$QMap@VQString@@I@@$00@QtPrivate@@SA_NH@Z 100139f0 f i ClarkClassifyWorker.obj
 0001:00012a60       ?registerConverter@?$IsPair@V?$QMap@VQString@@I@@@QtPrivate@@SA_NH@Z 10013a60 f i ClarkClassifyWorker.obj
 0001:00012a70       ?registerConverter@?$IsPair@VQAssociativeIterableImpl@QtMetaTypePrivate@@@QtPrivate@@SA_NH@Z 10013a70 f i ClarkClassifyWorker.obj
 0001:00012a80       ?registerConverter@?$MetaTypeSmartPointerHelper@V?$QMap@VQString@@I@@X@QtPrivate@@SA_NH@Z 10013a80 f i ClarkClassifyWorker.obj
 0001:00012a90       ?registerConverter@?$MetaTypeSmartPointerHelper@VQAssociativeIterableImpl@QtMetaTypePrivate@@X@QtPrivate@@SA_NH@Z 10013a90 f i ClarkClassifyWorker.obj
 0001:00012aa0       ?registerConverter@?$SequentialContainerConverterHelper@V?$QMap@VQString@@I@@$0A@@QtPrivate@@SA_NH@Z 10013aa0 f i ClarkClassifyWorker.obj
 0001:00012ab0       ?registerConverter@?$SequentialContainerConverterHelper@VQAssociativeIterableImpl@QtMetaTypePrivate@@$0A@@QtPrivate@@SA_NH@Z 10013ab0 f i ClarkClassifyWorker.obj
 0001:00012ac0       ?reserve@?$QList@VQString@@@@QAEXH@Z 10013ac0 f i ClarkClassifyWorker.obj
 0001:00012af0       ?rightNode@?$QMapNode@VQString@@I@@QBEPAU1@XZ 10013af0 f i ClarkClassifyWorker.obj
 0001:00012b00       ?rightNode@?$QMapNode@VQString@@V1@@@QBEPAU1@XZ 10013b00 f i ClarkClassifyWorker.obj
 0001:00012b10       ?root@?$QMapData@VQString@@I@@QBEPAU?$QMapNode@VQString@@I@@XZ 10013b10 f i ClarkClassifyWorker.obj
 0001:00012b20       ?root@?$QMapData@VQString@@V1@@@QBEPAU?$QMapNode@VQString@@V1@@@XZ 10013b20 f i ClarkClassifyWorker.obj
 0001:00012b30       ?run@ClarkClassifyTask@LocalWorkflow@U2@@EAEXXZ 10013b30 f   ClarkClassifyWorker.obj
 0001:00013100       ?setLastError@ClarkLogParser@LocalWorkflow@U2@@EAEXABVQString@@@Z 10014100 f   ClarkClassifyWorker.obj
 0001:00013280       ?size@?$QList@VQByteArray@@@@QBEHXZ 10014280 f i ClarkClassifyWorker.obj
 0001:00013290       ?size@?$QList@VQFileInfo@@@@QBEHXZ 10014290 f i ClarkClassifyWorker.obj
 0001:000132a0       ?size@?$QMap@VQString@@I@@QBEHXZ 100142a0 f i ClarkClassifyWorker.obj
 0001:000132b0       ?size@?$QMap@VQString@@V1@@@QBEHXZ 100142b0 f i ClarkClassifyWorker.obj
 0001:000132c0       ?sl_taskFinished@ClarkClassifyWorker@LocalWorkflow@U2@@AAEXPAVTask@3@@Z 100142c0 f   ClarkClassifyWorker.obj
 0001:000136d0       ?t@Node@?$QList@VQByteArray@@@@QAEAAVQByteArray@@XZ 100146d0 f i ClarkClassifyWorker.obj
 0001:000136e0       ?tick@ClarkClassifyWorker@LocalWorkflow@U2@@MAEPAVTask@3@XZ 100146e0 f   ClarkClassifyWorker.obj
 0001:00013f60       ?tr@ClarkClassifyPrompter@LocalWorkflow@U2@@SA?AVQString@@PBD0H@Z 10014f60 f i ClarkClassifyWorker.obj
 0001:00013f90       ?tr@ClarkClassifyTask@LocalWorkflow@U2@@SA?AVQString@@PBD0H@Z 10014f90 f i ClarkClassifyWorker.obj
 0001:00013fc0       ?tr@ClarkClassifyValidator@LocalWorkflow@U2@@SA?AVQString@@PBD0H@Z 10014fc0 f i ClarkClassifyWorker.obj
 0001:00013ff0       ?tr@ClarkClassifyWorker@LocalWorkflow@U2@@SA?AVQString@@PBD0H@Z 10014ff0 f i ClarkClassifyWorker.obj
 0001:00014020       ?validate@ClarkClassifyValidator@LocalWorkflow@U2@@UBE_NPBVActor@Workflow@3@AAV?$QList@VWorkflowNotification@U2@@@@ABV?$QMap@VQString@@V1@@@@Z 10015020 f   ClarkClassifyWorker.obj
 0001:00014060       ?validateDatabase@ClarkClassifyValidator@LocalWorkflow@U2@@ABE_NPBVActor@Workflow@3@AAV?$QList@VWorkflowNotification@U2@@@@@Z 10015060 f   ClarkClassifyWorker.obj
 0001:00014620       ?validateRefseqAvailability@ClarkClassifyValidator@LocalWorkflow@U2@@ABE_NPBVActor@Workflow@3@AAV?$QList@VWorkflowNotification@U2@@@@@Z 10015620 f   ClarkClassifyWorker.obj
 0001:000147c0       ?value@?$MetaObjectForType@V?$QMap@VQString@@I@@$0A@@QtPrivate@@SAPBUQMetaObject@@XZ 100157c0 f i ClarkClassifyWorker.obj
 0001:000147d0       ?value@?$MetaObjectForType@VQAssociativeIterableImpl@QtMetaTypePrivate@@$0A@@QtPrivate@@SAPBUQMetaObject@@XZ 100157d0 f i ClarkClassifyWorker.obj
 0001:000147e0       ?value@?$QMap@VQString@@V1@@@QBE?BVQString@@ABV2@0@Z 100157e0 f i ClarkClassifyWorker.obj
 0001:00014850       ?value@const_iterator@?$QMap@VQString@@I@@QBEABIXZ 10015850 f i ClarkClassifyWorker.obj
 0001:00014860       ??0?$AbstractId@H@U2@@IAE@ABH@Z 10015860 f i ClarkSupport.obj
 0001:00014880       ??0AbstractInt32Id@U2@@IAE@H@Z 10015880 f i ClarkSupport.obj
 0001:000148a0       ??0ClarkSupport@U2@@QAE@ABVQString@@00@Z 100158a0 f   ClarkSupport.obj
 0001:00014c00       ??0ServiceType@U2@@QAE@H@Z 10015c00 f i ClarkSupport.obj
 0001:00014c20       ??1?$AbstractId@H@U2@@MAE@XZ 10015c20 f i ClarkSupport.obj
 0001:00014c30       ??1AbstractInt32Id@U2@@UAE@XZ 10015c30 f i ClarkSupport.obj
 0001:00014c40       ??1ClarkSupport@U2@@UAE@XZ 10015c40 f i ClarkSupport.obj
 0001:00014c50       ??1ServiceType@U2@@UAE@XZ  10015c50 f i ClarkSupport.obj
 0001:00014c60       ??H@YA?BVQString@@PBDABV0@@Z 10015c60 f i ClarkSupport.obj
 0001:00014cd0       ??_G?$AbstractId@H@U2@@MAEPAXI@Z 10015cd0 f i ClarkSupport.obj
 0001:00014cd0       ??_E?$AbstractId@H@U2@@MAEPAXI@Z 10015cd0 f i ClarkSupport.obj
 0001:00014d00       ??_EAbstractInt32Id@U2@@UAEPAXI@Z 10015d00 f i ClarkSupport.obj
 0001:00014d00       ??_GAbstractInt32Id@U2@@UAEPAXI@Z 10015d00 f i ClarkSupport.obj
 0001:00014d30       ??_GClarkSupport@U2@@UAEPAXI@Z 10015d30 f i ClarkSupport.obj
 0001:00014d30       ??_EClarkSupport@U2@@UAEPAXI@Z 10015d30 f i ClarkSupport.obj
 0001:00014d60       ??_EServiceType@U2@@UAEPAXI@Z 10015d60 f i ClarkSupport.obj
 0001:00014d60       ??_GServiceType@U2@@UAEPAXI@Z 10015d60 f i ClarkSupport.obj
 0001:00014d90       ?isValid@AbstractInt32Id@U2@@UBE_NXZ 10015d90 f i ClarkSupport.obj
 0001:00014da0       ?registerTools@ClarkSupport@U2@@SAXPAVExternalToolRegistry@2@@Z 10015da0 f   ClarkSupport.obj
 0001:000150e0       ?tr@ClarkSupport@U2@@SA?AVQString@@PBD0H@Z 100160e0 f i ClarkSupport.obj
 0001:00015110       ?unregisterTools@ClarkSupport@U2@@SAXPAVExternalToolRegistry@2@@Z 10016110 f   ClarkSupport.obj
 0001:00015160       ??$_Move@AAPAUData@QListData@@@std@@YA$$QAPAUData@QListData@@AAPAU12@@Z 10016160 f i ClarkSupportPlugin.obj
 0001:00015170       ??$qDeleteAll@V?$QList@PAVXMLTestFactory@U2@@@@@@YAXABV?$QList@PAVXMLTestFactory@U2@@@@@Z 10016170 f i ClarkSupportPlugin.obj
 0001:000151b0       ??$qDeleteAll@Vconst_iterator@?$QList@PAVXMLTestFactory@U2@@@@@@YAXVconst_iterator@?$QList@PAVXMLTestFactory@U2@@@@0@Z 100161b0 f i ClarkSupportPlugin.obj
 0001:000151e0       ??$qSwap@PAUData@QListData@@@@YAXAAPAUData@QListData@@0@Z 100161e0 f i ClarkSupportPlugin.obj
 0001:00015200       ??$qobject_cast@PAVXMLTestFormat@U2@@@@YAPAVXMLTestFormat@U2@@PAVQObject@@@Z 10016200 f i ClarkSupportPlugin.obj
 0001:00015220       ??$swap@PAUData@QListData@@@std@@YAXAAPAUData@QListData@@0@Z 10016220 f i ClarkSupportPlugin.obj
 0001:00015240       ??0?$GAutoDeleteList@VXMLTestFactory@U2@@@U2@@QAE@PAVQObject@@@Z 10016240 f i ClarkSupportPlugin.obj
 0001:00015270       ??0?$QForeachContainer@V?$QList@PAVXMLTestFactory@U2@@@@@@QAE@ABV?$QList@PAVXMLTestFactory@U2@@@@@Z 10016270 f i ClarkSupportPlugin.obj
 0001:000152b0       ??0?$QList@PAVXMLTestFactory@U2@@@@QAE@ABV0@@Z 100162b0 f i ClarkSupportPlugin.obj
 0001:00015370       ??0?$QList@PAVXMLTestFactory@U2@@@@QAE@XZ 10016370 f i ClarkSupportPlugin.obj
 0001:00015380       ??0ClarkSupportPlugin@U2@@QAE@XZ 10016380 f   ClarkSupportPlugin.obj
 0001:00015680       ??0const_iterator@?$QList@PAVXMLTestFactory@U2@@@@QAE@PAUNode@1@@Z 10016680 f i ClarkSupportPlugin.obj
 0001:00015690       ??1?$GAutoDeleteList@VXMLTestFactory@U2@@@U2@@UAE@XZ 10016690 f i ClarkSupportPlugin.obj
 0001:00015750       ??1?$QForeachContainer@V?$QList@PAVXMLTestFactory@U2@@@@@@QAE@XZ 10016750 f i ClarkSupportPlugin.obj
 0001:00015780       ??1?$QList@PAVXMLTestFactory@U2@@@@QAE@XZ 10016780 f i ClarkSupportPlugin.obj
 0001:000157b0       ??1ClarkSupportPlugin@U2@@UAE@XZ 100167b0 f   ClarkSupportPlugin.obj
 0001:00015a00       ??4?$QList@PAVXMLTestFactory@U2@@@@QAEAAV0@$$QAV0@@Z 10016a00 f i ClarkSupportPlugin.obj
 0001:00015a20       ??9const_iterator@?$QList@PAVXMLTestFactory@U2@@@@QBE_NABV01@@Z 10016a20 f i ClarkSupportPlugin.obj
 0001:00015a40       ??Dconst_iterator@?$QList@PAVXMLTestFactory@U2@@@@QBEABQAVXMLTestFactory@U2@@XZ 10016a40 f i ClarkSupportPlugin.obj
 0001:00015a50       ??Econst_iterator@?$QList@PAVXMLTestFactory@U2@@@@QAEAAV01@XZ 10016a50 f i ClarkSupportPlugin.obj
 0001:00015a60       ??_E?$GAutoDeleteList@VXMLTestFactory@U2@@@U2@@UAEPAXI@Z 10016a60 f i ClarkSupportPlugin.obj
 0001:00015a60       ??_G?$GAutoDeleteList@VXMLTestFactory@U2@@@U2@@UAEPAXI@Z 10016a60 f i ClarkSupportPlugin.obj
 0001:00015a90       ??_EClarkSupportPlugin@U2@@UAEPAXI@Z 10016a90 f i ClarkSupportPlugin.obj
 0001:00015a90       ??_GClarkSupportPlugin@U2@@UAEPAXI@Z 10016a90 f i ClarkSupportPlugin.obj
 0001:00015ac0       ?begin@?$QList@PAVXMLTestFactory@U2@@@@QBE?AVconst_iterator@1@XZ 10016ac0 f i ClarkSupportPlugin.obj
 0001:00015ae0       ?dealloc@?$QList@PAVXMLTestFactory@U2@@@@AAEXPAUData@QListData@@@Z 10016ae0 f i ClarkSupportPlugin.obj
 0001:00015b00       ?end@?$QList@PAVXMLTestFactory@U2@@@@QBE?AVconst_iterator@1@XZ 10016b00 f i ClarkSupportPlugin.obj
 0001:00015b20       ?node_copy@?$QList@PAVXMLTestFactory@U2@@@@AAEXPAUNode@1@00@Z 10016b20 f i ClarkSupportPlugin.obj
 0001:00015b50       ?node_destruct@?$QList@PAVXMLTestFactory@U2@@@@AAEXPAUNode@1@0@Z 10016b50 f i ClarkSupportPlugin.obj
 0001:00015b60       ?t@Node@?$QList@PAVXMLTestFactory@U2@@@@QAEAAPAVXMLTestFactory@U2@@XZ 10016b60 f i ClarkSupportPlugin.obj
 0001:00015b70       _ugene_plugin_init         10016b70 f   ClarkSupportPlugin.obj
 0001:00015b90       ??$_Copy_impl@PBQAVXMLTestFactory@U2@@V?$back_insert_iterator@V?$QList@PAVXMLTestFactory@U2@@@@@std@@@std@@YA?AV?$back_insert_iterator@V?$QList@PAVXMLTestFactory@U2@@@@@0@PBQAVXMLTestFactory@U2@@0V10@@Z 10016b90 f i ClarkTests.obj
 0001:00015bc0       ??$_Copy_impl@PBQAVXMLTestFactory@U2@@V?$back_insert_iterator@V?$QList@PAVXMLTestFactory@U2@@@@@std@@@std@@YA?AV?$back_insert_iterator@V?$QList@PAVXMLTestFactory@U2@@@@@0@PBQAVXMLTestFactory@U2@@0V10@U_Nonscalar_ptr_iterator_tag@0@@Z 10016bc0 f i ClarkTests.obj
 0001:00015bf0       ??$_Copy_impl@PBVQString@@V?$back_insert_iterator@V?$QList@VQString@@@@@std@@@std@@YA?AV?$back_insert_iterator@V?$QList@VQString@@@@@0@PBVQString@@0V10@@Z 10016bf0 f i ClarkTests.obj
 0001:00015c20       ??$_Copy_impl@PBVQString@@V?$back_insert_iterator@V?$QList@VQString@@@@@std@@@std@@YA?AV?$back_insert_iterator@V?$QList@VQString@@@@@0@PBVQString@@0V10@U_Nonscalar_ptr_iterator_tag@0@@Z 10016c20 f i ClarkTests.obj
 0001:00015c50       ??$_Ptr_cat@PBQAVXMLTestFactory@U2@@V?$back_insert_iterator@V?$QList@PAVXMLTestFactory@U2@@@@@std@@@std@@YA?AU_Nonscalar_ptr_iterator_tag@0@AAPBQAVXMLTestFactory@U2@@AAV?$back_insert_iterator@V?$QList@PAVXMLTestFactory@U2@@@@@0@@Z 10016c50 f i ClarkTests.obj
 0001:00015c60       ??$_Ptr_cat@PBVQString@@V?$back_insert_iterator@V?$QList@VQString@@@@@std@@@std@@YA?AU_Nonscalar_ptr_iterator_tag@0@AAPBVQString@@AAV?$back_insert_iterator@V?$QList@VQString@@@@@0@@Z 10016c60 f i ClarkTests.obj
 0001:00015c70       ??$_Rechecked@V?$back_insert_iterator@V?$QList@PAVXMLTestFactory@U2@@@@@std@@V12@@std@@YAAAV?$back_insert_iterator@V?$QList@PAVXMLTestFactory@U2@@@@@0@AAV10@V10@@Z 10016c70 f i ClarkTests.obj
 0001:00015c80       ??$_Rechecked@V?$back_insert_iterator@V?$QList@VQString@@@@@std@@V12@@std@@YAAAV?$back_insert_iterator@V?$QList@VQString@@@@@0@AAV10@V10@@Z 10016c80 f i ClarkTests.obj
 0001:00015c90       ??$_Unchecked@PBQAVXMLTestFactory@U2@@@std@@YAPBQAVXMLTestFactory@U2@@PBQAV12@@Z 10016c90 f i ClarkTests.obj
 0001:00015ca0       ??$_Unchecked@PBVQString@@@std@@YAPBVQString@@PBV1@@Z 10016ca0 f i ClarkTests.obj
 0001:00015cb0       ??$_Unchecked@V?$back_insert_iterator@V?$QList@PAVXMLTestFactory@U2@@@@@std@@@std@@YA?AV?$back_insert_iterator@V?$QList@PAVXMLTestFactory@U2@@@@@0@V10@@Z 10016cb0 f i ClarkTests.obj
 0001:00015cc0       ??$_Unchecked@V?$back_insert_iterator@V?$QList@VQString@@@@@std@@@std@@YA?AV?$back_insert_iterator@V?$QList@VQString@@@@@0@V10@@Z 10016cc0 f i ClarkTests.obj
 0001:00015cd0       ??$addressof@V?$QList@PAVXMLTestFactory@U2@@@@@std@@YAPAV?$QList@PAVXMLTestFactory@U2@@@@AAV1@@Z 10016cd0 f i ClarkTests.obj
 0001:00015ce0       ??$addressof@V?$QList@VQString@@@@@std@@YAPAV?$QList@VQString@@@@AAV1@@Z 10016ce0 f i ClarkTests.obj
 0001:00015cf0       ??$back_inserter@V?$QList@PAVXMLTestFactory@U2@@@@@std@@YA?AV?$back_insert_iterator@V?$QList@PAVXMLTestFactory@U2@@@@@0@AAV?$QList@PAVXMLTestFactory@U2@@@@@Z 10016cf0 f i ClarkTests.obj
 0001:00015d00       ??$back_inserter@V?$QList@VQString@@@@@std@@YA?AV?$back_insert_iterator@V?$QList@VQString@@@@@0@AAV?$QList@VQString@@@@@Z 10016d00 f i ClarkTests.obj
 0001:00015d10       ??$copy@PBQAVXMLTestFactory@U2@@V?$back_insert_iterator@V?$QList@PAVXMLTestFactory@U2@@@@@std@@@std@@YA?AV?$back_insert_iterator@V?$QList@PAVXMLTestFactory@U2@@@@@0@PBQAVXMLTestFactory@U2@@0V10@@Z 10016d10 f i ClarkTests.obj
 0001:00015d40       ??$copy@PBVQString@@V?$back_insert_iterator@V?$QList@VQString@@@@@std@@@std@@YA?AV?$back_insert_iterator@V?$QList@VQString@@@@@0@PBVQString@@0V10@@Z 10016d40 f i ClarkTests.obj
 0001:00015d70       ??0?$QList@PAVXMLTestFactory@U2@@@@QAE@V?$initializer_list@PAVXMLTestFactory@U2@@@std@@@Z 10016d70 f i ClarkTests.obj
 0001:00015de0       ??0?$QList@VQString@@@@QAE@V?$initializer_list@VQString@@@std@@@Z 10016de0 f i ClarkTests.obj
 0001:00015e50       ??0?$back_insert_iterator@V?$QList@PAVXMLTestFactory@U2@@@@@std@@QAE@AAV?$QList@PAVXMLTestFactory@U2@@@@@Z 10016e50 f i ClarkTests.obj
 0001:00015e60       ??0?$back_insert_iterator@V?$QList@VQString@@@@@std@@QAE@AAV?$QList@VQString@@@@@Z 10016e60 f i ClarkTests.obj
 0001:00015e70       ??0?$initializer_list@PAVXMLTestFactory@U2@@@std@@QAE@PBQAVXMLTestFactory@U2@@0@Z 10016e70 f i ClarkTests.obj
 0001:00015e90       ??0?$initializer_list@VQString@@@std@@QAE@PBVQString@@0@Z 10016e90 f i ClarkTests.obj
 0001:00015eb0       ??0GTest_CompareClarkDatabaseMetafiles@U2@@QAE@PAVXMLTestFormat@1@ABVQString@@PAVGTest@1@PBVGTestEnvironment@1@ABV?$QList@PAVGTest@U2@@@@ABVQDomElement@@@Z 10016eb0 f i ClarkTests.obj
 0001:00015f60       ??0GTest_CompareClarkDatabaseMetafilesFactory@GTest_CompareClarkDatabaseMetafiles@U2@@QAE@XZ 10016f60 f i ClarkTests.obj
 0001:00015fe0       ??0QStringList@@QAE@V?$initializer_list@VQString@@@std@@@Z 10016fe0 f i ClarkTests.obj
 0001:00016000       ??1GTest_CompareClarkDatabaseMetafiles@U2@@UAE@XZ 10017000 f i ClarkTests.obj
 0001:00016090       ??1GTest_CompareClarkDatabaseMetafilesFactory@GTest_CompareClarkDatabaseMetafiles@U2@@UAE@XZ 10017090 f i ClarkTests.obj
 0001:000160a0       ??4?$back_insert_iterator@V?$QList@PAVXMLTestFactory@U2@@@@@std@@QAEAAV01@ABQAVXMLTestFactory@U2@@@Z 100170a0 f i ClarkTests.obj
 0001:000160c0       ??4?$back_insert_iterator@V?$QList@VQString@@@@@std@@QAEAAV01@ABVQString@@@Z 100170c0 f i ClarkTests.obj
 0001:000160e0       ??D?$back_insert_iterator@V?$QList@PAVXMLTestFactory@U2@@@@@std@@QAEAAV01@XZ 100170e0 f i ClarkTests.obj
 0001:000160f0       ??D?$back_insert_iterator@V?$QList@VQString@@@@@std@@QAEAAV01@XZ 100170f0 f i ClarkTests.obj
 0001:00016100       ??E?$back_insert_iterator@V?$QList@PAVXMLTestFactory@U2@@@@@std@@QAEAAV01@XZ 10017100 f i ClarkTests.obj
 0001:00016110       ??E?$back_insert_iterator@V?$QList@VQString@@@@@std@@QAEAAV01@XZ 10017110 f i ClarkTests.obj
 0001:00016120       ??_EGTest_CompareClarkDatabaseMetafiles@U2@@UAEPAXI@Z 10017120 f i ClarkTests.obj
 0001:00016120       ??_GGTest_CompareClarkDatabaseMetafiles@U2@@UAEPAXI@Z 10017120 f i ClarkTests.obj
 0001:000161c0       ??_GGTest_CompareClarkDatabaseMetafilesFactory@GTest_CompareClarkDatabaseMetafiles@U2@@UAEPAXI@Z 100171c0 f i ClarkTests.obj
 0001:000161c0       ??_EGTest_CompareClarkDatabaseMetafilesFactory@GTest_CompareClarkDatabaseMetafiles@U2@@UAEPAXI@Z 100171c0 f i ClarkTests.obj
 0001:000161f0       ?append@?$QList@PAVXMLTestFactory@U2@@@@QAEXABQAVXMLTestFactory@U2@@@Z 100171f0 f i ClarkTests.obj
 0001:00016280       ?begin@?$initializer_list@PAVXMLTestFactory@U2@@@std@@QBEPBQAVXMLTestFactory@U2@@XZ 10017280 f i ClarkTests.obj
 0001:00016290       ?begin@?$initializer_list@VQString@@@std@@QBEPBVQString@@XZ 10017290 f i ClarkTests.obj
 0001:000162a0       ?createFactory@GTest_CompareClarkDatabaseMetafiles@U2@@SAPAVXMLTestFactory@2@XZ 100172a0 f i ClarkTests.obj
 0001:00016340       ?createTest@GTest_CompareClarkDatabaseMetafilesFactory@GTest_CompareClarkDatabaseMetafiles@U2@@UAEPAVGTest@3@PAVXMLTestFormat@3@ABVQString@@PAV43@PBVGTestEnvironment@3@ABV?$QList@PAVGTest@U2@@@@ABVQDomElement@@@Z 10017340 f i ClarkTests.obj
 0001:000163c0       ?createTestFactories@ClarkTests@U2@@SA?AV?$QList@PAVXMLTestFactory@U2@@@@XZ 100173c0 f   ClarkTests.obj
 0001:000163f0       ?detach_helper@?$QList@PAVXMLTestFactory@U2@@@@AAEXH@Z 100173f0 f i ClarkTests.obj
 0001:000164c0       ?detach_helper_grow@?$QList@PAVXMLTestFactory@U2@@@@AAEPAUNode@1@HH@Z 100174c0 f i ClarkTests.obj
 0001:000165d0       ?end@?$initializer_list@PAVXMLTestFactory@U2@@@std@@QBEPBQAVXMLTestFactory@U2@@XZ 100175d0 f i ClarkTests.obj
 0001:000165e0       ?end@?$initializer_list@VQString@@@std@@QBEPBVQString@@XZ 100175e0 f i ClarkTests.obj
 0001:000165f0       ?init@GTest_CompareClarkDatabaseMetafiles@U2@@QAEXPAVXMLTestFormat@2@ABVQDomElement@@@Z 100175f0 f   ClarkTests.obj
 0001:000169f0       ?node_construct@?$QList@PAVXMLTestFactory@U2@@@@AAEXPAUNode@1@ABQAVXMLTestFactory@U2@@@Z 100179f0 f i ClarkTests.obj
 0001:00016a10       ?node_destruct@?$QList@PAVXMLTestFactory@U2@@@@AAEXPAUNode@1@@Z 10017a10 f i ClarkTests.obj
 0001:00016a20       ?push_back@?$QList@PAVXMLTestFactory@U2@@@@QAEXABQAVXMLTestFactory@U2@@@Z 10017a20 f i ClarkTests.obj
 0001:00016a30       ?push_back@?$QList@VQString@@@@QAEXABVQString@@@Z 10017a30 f i ClarkTests.obj
 0001:00016a40       ?report@GTest_CompareClarkDatabaseMetafiles@U2@@EAE?AW4ReportResult@Task@2@XZ 10017a40 f   ClarkTests.obj
 0001:000173d0       ?reserve@?$QList@PAVXMLTestFactory@U2@@@@QAEXH@Z 100183d0 f i ClarkTests.obj
 0001:00017400       ?size@?$initializer_list@PAVXMLTestFactory@U2@@@std@@QBEIXZ 10018400 f i ClarkTests.obj
 0001:00017410       ?size@?$initializer_list@VQString@@@std@@QBEIXZ 10018410 f i ClarkTests.obj
 0001:00017420       ??$qMetaTypeId@PAVTask@U2@@@@YAHXZ 10018420 f i moc_ClarkBuildWorker.obj
 0001:00017430       ??$qRegisterMetaType@PAVTask@U2@@@@YAHXZ 10018430 f i moc_ClarkBuildWorker.obj
 0001:00017440       ??$qRegisterNormalizedMetaType@PAVTask@U2@@@@YAHABVQByteArray@@PAPAVTask@U2@@W4DefinedType@?$MetaTypeDefinedHelper@PAVTask@U2@@$00@QtPrivate@@@Z 10018440 f i moc_ClarkBuildWorker.obj
 0001:000174a0       ??C?$QScopedPointer@VQObjectData@@U?$QScopedPointerDeleter@VQObjectData@@@@@@QBEPAVQObjectData@@XZ 100184a0 f i moc_ClarkBuildWorker.obj
 0001:000174b0       ?Construct@?$QMetaTypeFunctionHelper@PAVTask@U2@@$00@QtMetaTypePrivate@@SAPAXPAXPBX@Z 100184b0 f i moc_ClarkBuildWorker.obj
 0001:000174e0       ?Create@?$QMetaTypeFunctionHelper@PAVTask@U2@@$00@QtMetaTypePrivate@@SAPAXPBX@Z 100184e0 f i moc_ClarkBuildWorker.obj
 0001:00017520       ?Delete@?$QMetaTypeFunctionHelper@PAVTask@U2@@$00@QtMetaTypePrivate@@SAXPAX@Z 10018520 f i moc_ClarkBuildWorker.obj
 0001:00017530       ?Destruct@?$QMetaTypeFunctionHelper@PAVTask@U2@@$00@QtMetaTypePrivate@@SAXPAX@Z 10018530 f i moc_ClarkBuildWorker.obj
 0001:00017540       ?metaObject@ClarkBuildPrompter@LocalWorkflow@U2@@UBEPBUQMetaObject@@XZ 10018540 f   moc_ClarkBuildWorker.obj
 0001:00017560       ?metaObject@ClarkBuildTask@LocalWorkflow@U2@@UBEPBUQMetaObject@@XZ 10018560 f   moc_ClarkBuildWorker.obj
 0001:00017580       ?metaObject@ClarkBuildWorker@LocalWorkflow@U2@@UBEPBUQMetaObject@@XZ 10018580 f   moc_ClarkBuildWorker.obj
 0001:000175a0       ?qt_metacall@ClarkBuildPrompter@LocalWorkflow@U2@@UAEHW4Call@QMetaObject@@HPAPAX@Z 100185a0 f   moc_ClarkBuildWorker.obj
 0001:000175b0       ?qt_metacall@ClarkBuildTask@LocalWorkflow@U2@@UAEHW4Call@QMetaObject@@HPAPAX@Z 100185b0 f   moc_ClarkBuildWorker.obj
 0001:000175c0       ?qt_metacall@ClarkBuildWorker@LocalWorkflow@U2@@UAEHW4Call@QMetaObject@@HPAPAX@Z 100185c0 f   moc_ClarkBuildWorker.obj
 0001:00017620       ?qt_metacast@ClarkBuildPrompter@LocalWorkflow@U2@@UAEPAXPBD@Z 10018620 f   moc_ClarkBuildWorker.obj
 0001:00017680       ?qt_metacast@ClarkBuildTask@LocalWorkflow@U2@@UAEPAXPBD@Z 10018680 f   moc_ClarkBuildWorker.obj
 0001:000176e0       ?qt_metacast@ClarkBuildWorker@LocalWorkflow@U2@@UAEPAXPBD@Z 100186e0 f   moc_ClarkBuildWorker.obj
 0001:00017740       ?qt_metatype_id@?$QMetaTypeId2@PAVTask@U2@@@@SAHXZ 10018740 f i moc_ClarkBuildWorker.obj
 0001:00017750       ?qt_metatype_id@?$QMetaTypeIdHelper@PAVTask@U2@@$00@QtPrivate@@SAHXZ 10018750 f i moc_ClarkBuildWorker.obj
 0001:00017760       ?qt_metatype_id@?$QMetaTypeIdQObject@PAVTask@U2@@$00@@SAHXZ 10018760 f i moc_ClarkBuildWorker.obj
 0001:00017840       ?qt_static_metacall@ClarkBuildPrompter@LocalWorkflow@U2@@CAXPAVQObject@@W4Call@QMetaObject@@HPAPAX@Z 10018840 f   moc_ClarkBuildWorker.obj
 0001:00017850       ?qt_static_metacall@ClarkBuildTask@LocalWorkflow@U2@@CAXPAVQObject@@W4Call@QMetaObject@@HPAPAX@Z 10018850 f   moc_ClarkBuildWorker.obj
 0001:00017860       ?qt_static_metacall@ClarkBuildWorker@LocalWorkflow@U2@@CAXPAVQObject@@W4Call@QMetaObject@@HPAPAX@Z 10018860 f   moc_ClarkBuildWorker.obj
 0001:000178c0       ?registerConverter@?$AssociativeContainerConverterHelper@PAVTask@U2@@$0A@@QtPrivate@@SA_NH@Z 100188c0 f i moc_ClarkBuildWorker.obj
 0001:000178d0       ?registerConverter@?$IsPair@PAVTask@U2@@@QtPrivate@@SA_NH@Z 100188d0 f i moc_ClarkBuildWorker.obj
 0001:000178e0       ?registerConverter@?$MetaTypeSmartPointerHelper@PAVTask@U2@@X@QtPrivate@@SA_NH@Z 100188e0 f i moc_ClarkBuildWorker.obj
 0001:000178f0       ?registerConverter@?$SequentialContainerConverterHelper@PAVTask@U2@@$0A@@QtPrivate@@SA_NH@Z 100188f0 f i moc_ClarkBuildWorker.obj
 0001:00017900       ?value@?$MetaObjectForType@PAVTask@U2@@$00@QtPrivate@@SAPBUQMetaObject@@XZ 10018900 f i moc_ClarkBuildWorker.obj
 0001:00017910       ?metaObject@ClarkClassifyPrompter@LocalWorkflow@U2@@UBEPBUQMetaObject@@XZ 10018910 f   moc_ClarkClassifyWorker.obj
 0001:00017930       ?metaObject@ClarkClassifyTask@LocalWorkflow@U2@@UBEPBUQMetaObject@@XZ 10018930 f   moc_ClarkClassifyWorker.obj
 0001:00017950       ?metaObject@ClarkClassifyWorker@LocalWorkflow@U2@@UBEPBUQMetaObject@@XZ 10018950 f   moc_ClarkClassifyWorker.obj
 0001:00017970       ?qt_metacall@ClarkClassifyPrompter@LocalWorkflow@U2@@UAEHW4Call@QMetaObject@@HPAPAX@Z 10018970 f   moc_ClarkClassifyWorker.obj
 0001:00017980       ?qt_metacall@ClarkClassifyTask@LocalWorkflow@U2@@UAEHW4Call@QMetaObject@@HPAPAX@Z 10018980 f   moc_ClarkClassifyWorker.obj
 0001:00017990       ?qt_metacall@ClarkClassifyWorker@LocalWorkflow@U2@@UAEHW4Call@QMetaObject@@HPAPAX@Z 10018990 f   moc_ClarkClassifyWorker.obj
 0001:000179f0       ?qt_metacast@ClarkClassifyPrompter@LocalWorkflow@U2@@UAEPAXPBD@Z 100189f0 f   moc_ClarkClassifyWorker.obj
 0001:00017a50       ?qt_metacast@ClarkClassifyTask@LocalWorkflow@U2@@UAEPAXPBD@Z 10018a50 f   moc_ClarkClassifyWorker.obj
 0001:00017ab0       ?qt_metacast@ClarkClassifyWorker@LocalWorkflow@U2@@UAEPAXPBD@Z 10018ab0 f   moc_ClarkClassifyWorker.obj
 0001:00017b10       ?qt_static_metacall@ClarkClassifyPrompter@LocalWorkflow@U2@@CAXPAVQObject@@W4Call@QMetaObject@@HPAPAX@Z 10018b10 f   moc_ClarkClassifyWorker.obj
 0001:00017b20       ?qt_static_metacall@ClarkClassifyTask@LocalWorkflow@U2@@CAXPAVQObject@@W4Call@QMetaObject@@HPAPAX@Z 10018b20 f   moc_ClarkClassifyWorker.obj
 0001:00017b30       ?qt_static_metacall@ClarkClassifyWorker@LocalWorkflow@U2@@CAXPAVQObject@@W4Call@QMetaObject@@HPAPAX@Z 10018b30 f   moc_ClarkClassifyWorker.obj
 0001:00017b90       ?metaObject@ClarkSupport@U2@@UBEPBUQMetaObject@@XZ 10018b90 f   moc_ClarkSupport.obj
 0001:00017bb0       ?qt_metacall@ClarkSupport@U2@@UAEHW4Call@QMetaObject@@HPAPAX@Z 10018bb0 f   moc_ClarkSupport.obj
 0001:00017bc0       ?qt_metacast@ClarkSupport@U2@@UAEPAXPBD@Z 10018bc0 f   moc_ClarkSupport.obj
 0001:00017c20       ?qt_static_metacall@ClarkSupport@U2@@CAXPAVQObject@@W4Call@QMetaObject@@HPAPAX@Z 10018c20 f   moc_ClarkSupport.obj
 0001:00017c30       ?metaObject@ClarkSupportPlugin@U2@@UBEPBUQMetaObject@@XZ 10018c30 f   moc_ClarkSupportPlugin.obj
 0001:00017c50       ?qt_metacall@ClarkSupportPlugin@U2@@UAEHW4Call@QMetaObject@@HPAPAX@Z 10018c50 f   moc_ClarkSupportPlugin.obj
 0001:00017c60       ?qt_metacast@ClarkSupportPlugin@U2@@UAEPAXPBD@Z 10018c60 f   moc_ClarkSupportPlugin.obj
 0001:00017cc0       ?qt_static_metacall@ClarkSupportPlugin@U2@@CAXPAVQObject@@W4Call@QMetaObject@@HPAPAX@Z 10018cc0 f   moc_ClarkSupportPlugin.obj
 0001:00017cc2       ?getDataPathRegistry@AppContext@U2@@SAPAVU2DataPathRegistry@2@XZ 10018cc2 f   U2Core:U2Core.dll
 0001:00017cc8       ??1GCounter@U2@@UAE@XZ     10018cc8 f   U2Core:U2Core.dll
 0001:00017cce       ??0GReportableCounter@U2@@QAE@ABVQString@@0N@Z 10018cce f   U2Core:U2Core.dll
 0001:00017cd4       ??1SimpleEventCounter@U2@@UAE@XZ 10018cd4 f   U2Core:U2Core.dll
 0001:00017cda       ?getPath@U2DataPath@U2@@QBEABVQString@@XZ 10018cda f   U2Core:U2Core.dll
 0001:00017ce0       ?isValid@U2DataPath@U2@@QBE_NXZ 10018ce0 f   U2Core:U2Core.dll
 0001:00017ce6       ?getPathByName@U2DataPath@U2@@QBE?AVQString@@ABV3@@Z 10018ce6 f   U2Core:U2Core.dll
 0001:00017cec       ?getDataPathByName@U2DataPathRegistry@U2@@QAEPAVU2DataPath@2@ABVQString@@@Z 10018cec f   U2Core:U2Core.dll
 0001:00017cf2       ??0Logger@U2@@QAE@ABVQString@@@Z 10018cf2 f   U2Core:U2Core.dll
 0001:00017cf8       ??1Logger@U2@@UAE@XZ       10018cf8 f   U2Core:U2Core.dll
 0001:00017cfe       ?trace@Logger@U2@@QAEXABVQString@@@Z 10018cfe f   U2Core:U2Core.dll
 0001:00017d04       ?error@Logger@U2@@QAEXABVQString@@@Z 10018d04 f   U2Core:U2Core.dll
 0001:00017d0a       ??0TaskStateInfo@U2@@QAE@XZ 10018d0a f   U2Core:U2Core.dll
 0001:00017d10       ?getError@TaskStateInfo@U2@@UBE?AVQString@@XZ 10018d10 f   U2Core:U2Core.dll
 0001:00017d16       ?setError@TaskStateInfo@U2@@UAEXABVQString@@@Z 10018d16 f   U2Core:U2Core.dll
 0001:00017d1c       ??1TaskStateInfo@U2@@UAE@XZ 10018d1c f   U2Core:U2Core.dll
 0001:00017d22       ?addSubTask@Task@U2@@QAEXPAV12@@Z 10018d22 f   U2Core:U2Core.dll
 0001:00017d28       ?hasError@Task@U2@@QBE_NXZ 10018d28 f   U2Core:U2Core.dll
 0001:00017d2e       ?setError@Task@U2@@QAEXABVQString@@@Z 10018d2e f   U2Core:U2Core.dll
 0001:00017d34       ??0FailTask@U2@@QAE@ABVQString@@@Z 10018d34 f   U2Core:U2Core.dll
 0001:00017d3a       ??1FailTask@U2@@UAE@XZ     10018d3a f   U2Core:U2Core.dll
 0001:00017d40       ?required@L10N@U2@@SA?AVQString@@XZ 10018d40 f   U2Core:U2Core.dll
 0001:00017d46       ??0TaskSignalMapper@U2@@QAE@PAVTask@1@@Z 10018d46 f   U2Core:U2Core.dll
 0001:00017d4c       ?runScript@ScriptTask@U2@@SA?AVQScriptValue@@PAVQScriptEngine@@ABV?$QMap@VQString@@VQScriptValue@@@@ABVQString@@AAVTaskStateInfo@2@@Z 10018d4c f   U2Core:U2Core.dll
 0001:00017d52       ??0ExternalToolRunTask@U2@@QAE@ABVQString@@ABVQStringList@@PAVExternalToolLogParser@1@010_N@Z 10018d52 f   U2Core:U2Core.dll
 0001:00017d58       ??1ExternalToolRunTask@U2@@UAE@XZ 10018d58 f   U2Core:U2Core.dll
 0001:00017d5e       ??0ExternalToolSupportTask@U2@@QAE@ABVQString@@V?$QFlags@W4TaskFlag@U2@@@@@Z 10018d5e f   U2Core:U2Core.dll
 0001:00017d64       ??1ExternalToolSupportTask@U2@@UAE@XZ 10018d64 f   U2Core:U2Core.dll
 0001:00017d6a       ?addListeners@ExternalToolSupportTask@U2@@QAEXABV?$QList@PAVExternalToolListener@U2@@@@@Z 10018d6a f   U2Core:U2Core.dll
 0001:00017d70       ??0ExternalToolLogParser@U2@@QAE@_N@Z 10018d70 f   U2Core:U2Core.dll
 0001:00017d76       ??1ExternalToolLogParser@U2@@UAE@XZ 10018d76 f   U2Core:U2Core.dll
 0001:00017d7c       ?cleanup@Task@U2@@UAEXXZ   10018d7c f   U2Core:U2Core.dll
 0001:00017d82       ?generateReport@Task@U2@@UBE?AVQString@@XZ 10018d82 f   U2Core:U2Core.dll
 0001:00017d88       ?getNumParallelSubtasks@Task@U2@@UBEHXZ 10018d88 f   U2Core:U2Core.dll
 0001:00017d8e       ?getParentTask@Task@U2@@UBEPAV12@XZ 10018d8e f   U2Core:U2Core.dll
 0001:00017d94       ?getProgress@ExternalToolLogParser@U2@@UAEHXZ 10018d94 f   U2Core:U2Core.dll
 0001:00017d9a       ?getSubtaskWithErrors@Task@U2@@UBEPAV12@XZ 10018d9a f   U2Core:U2Core.dll
 0001:00017da0       ?getTaskId@Task@U2@@UBE_JXZ 10018da0 f   U2Core:U2Core.dll
 0001:00017da6       ?getTopLevelParentTask@Task@U2@@UAEPAV12@XZ 10018da6 f   U2Core:U2Core.dll
 0001:00017dac       ?getWarnings@Task@U2@@UBE?AVQStringList@@XZ 10018dac f   U2Core:U2Core.dll
 0001:00017db2       ?hasSubtasksWithErrors@Task@U2@@UBE_NXZ 10018db2 f   U2Core:U2Core.dll
 0001:00017db8       ?hasWarning@Task@U2@@UBE_NXZ 10018db8 f   U2Core:U2Core.dll
 0001:00017dbe       ?isNotificationReport@Task@U2@@UBE_NXZ 10018dbe f   U2Core:U2Core.dll
 0001:00017dc4       ?isReportingEnabled@Task@U2@@UBE_NXZ 10018dc4 f   U2Core:U2Core.dll
 0001:00017dca       ?isReportingSupported@Task@U2@@UBE_NXZ 10018dca f   U2Core:U2Core.dll
 0001:00017dd0       ?isTopLevelTask@Task@U2@@UBE_NXZ 10018dd0 f   U2Core:U2Core.dll
 0001:00017dd6       ?metaObject@ExternalToolLogParser@U2@@UBEPBUQMetaObject@@XZ 10018dd6 f   U2Core:U2Core.dll
 0001:00017ddc       ?metaObject@ExternalToolRunTask@U2@@UBEPBUQMetaObject@@XZ 10018ddc f   U2Core:U2Core.dll
 0001:00017de2       ?metaObject@FailTask@U2@@UBEPBUQMetaObject@@XZ 10018de2 f   U2Core:U2Core.dll
 0001:00017de8       ?metaObject@TaskSignalMapper@U2@@UBEPBUQMetaObject@@XZ 10018de8 f   U2Core:U2Core.dll
 0001:00017dee       ?onSubTaskFinished@Task@U2@@MAE?AV?$QList@PAVTask@U2@@@@PAV12@@Z 10018dee f   U2Core:U2Core.dll
 0001:00017df4       ?parseErrOutput@ExternalToolLogParser@U2@@UAEXABVQString@@@Z 10018df4 f   U2Core:U2Core.dll
 0001:00017dfa       ?parseOutput@ExternalToolLogParser@U2@@UAEXABVQString@@@Z 10018dfa f   U2Core:U2Core.dll
 0001:00017e00       ?prepare@Task@U2@@UAEXXZ   10018e00 f   U2Core:U2Core.dll
 0001:00017e06       ?processErrLine@ExternalToolLogParser@U2@@MAEXABVQString@@@Z 10018e06 f   U2Core:U2Core.dll
 0001:00017e0c       ?processLine@ExternalToolLogParser@U2@@MAEXABVQString@@@Z 10018e0c f   U2Core:U2Core.dll
 0001:00017e12       ?propagateSubtaskError@Task@U2@@UAE_NXZ 10018e12 f   U2Core:U2Core.dll
 0001:00017e18       ?qt_metacall@ExternalToolLogParser@U2@@UAEHW4Call@QMetaObject@@HPAPAX@Z 10018e18 f   U2Core:U2Core.dll
 0001:00017e1e       ?qt_metacall@ExternalToolRunTask@U2@@UAEHW4Call@QMetaObject@@HPAPAX@Z 10018e1e f   U2Core:U2Core.dll
 0001:00017e24       ?qt_metacall@FailTask@U2@@UAEHW4Call@QMetaObject@@HPAPAX@Z 10018e24 f   U2Core:U2Core.dll
 0001:00017e2a       ?qt_metacall@TaskSignalMapper@U2@@UAEHW4Call@QMetaObject@@HPAPAX@Z 10018e2a f   U2Core:U2Core.dll
 0001:00017e30       ?qt_metacast@ExternalToolLogParser@U2@@UAEPAXPBD@Z 10018e30 f   U2Core:U2Core.dll
 0001:00017e36       ?qt_metacast@ExternalToolRunTask@U2@@UAEPAXPBD@Z 10018e36 f   U2Core:U2Core.dll
 0001:00017e3c       ?qt_metacast@FailTask@U2@@UAEPAXPBD@Z 10018e3c f   U2Core:U2Core.dll
 0001:00017e42       ?qt_metacast@TaskSignalMapper@U2@@UAEPAXPBD@Z 10018e42 f   U2Core:U2Core.dll
 0001:00017e48       ?report@Task@U2@@UAE?AW4ReportResult@12@XZ 10018e48 f   U2Core:U2Core.dll
 0001:00017e4e       ?run@ExternalToolRunTask@U2@@UAEXXZ 10018e4e f   U2Core:U2Core.dll
 0001:00017e54       ?run@Task@U2@@UAEXXZ       10018e54 f   U2Core:U2Core.dll
 0001:00017e5a       ?setCollectChildrensWarningsFlag@Task@U2@@UAEX_N@Z 10018e5a f   U2Core:U2Core.dll
 0001:00017e60       ?setLastError@ExternalToolLogParser@U2@@MAEXABVQString@@@Z 10018e60 f   U2Core:U2Core.dll
 0001:00017e66       ?setListenerForHelper@ExternalToolSupportTask@U2@@MAEXPAVExternalToolRunTaskHelper@2@H@Z 10018e66 f   U2Core:U2Core.dll
 0001:00017e6c       ?setListenerForTask@ExternalToolSupportTask@U2@@MAEXPAVExternalToolRunTask@2@H@Z 10018e6c f   U2Core:U2Core.dll
 0001:00017e72       ?setNoAutoDelete@Task@U2@@UAEX_N@Z 10018e72 f   U2Core:U2Core.dll
 0001:00017e78       ?setNotificationReport@Task@U2@@UAEX_N@Z 10018e78 f   U2Core:U2Core.dll
 0001:00017e7e       ?setReportingEnabled@Task@U2@@UAEX_N@Z 10018e7e f   U2Core:U2Core.dll
 0001:00017e84       ?setReportingSupported@Task@U2@@UAEX_N@Z 10018e84 f   U2Core:U2Core.dll
 0001:00017e8a       ?getAppSettings@AppContext@U2@@SAPAVAppSettings@2@XZ 10018e8a f   U2Core:U2Core.dll
 0001:00017e90       ?details@Logger@U2@@QAEXABVQString@@@Z 10018e90 f   U2Core:U2Core.dll
 0001:00017e96       ?info@Logger@U2@@QAEXABVQString@@@Z 10018e96 f   U2Core:U2Core.dll
 0001:00017e9c       ?isCoR@U2OpStatus@U2@@UBE_NXZ 10018e9c f   U2Core:U2Core.dll
 0001:00017ea2       ?instance@AppResourcePool@U2@@SAPAV12@XZ 10018ea2 f   U2Core:U2Core.dll
 0001:00017ea8       ??0GUrl@U2@@QAE@ABVQString@@@Z 10018ea8 f   U2Core:U2Core.dll
 0001:00017eae       ??1GUrl@U2@@QAE@XZ         10018eae f   U2Core:U2Core.dll
 0001:00017eb4       ?createWorkingDir@FileAndDirectoryUtils@U2@@SA?AVQString@@ABV3@H00@Z 10018eb4 f   U2Core:U2Core.dll
 0001:00017eba       ?ensureFileExt@GUrlUtils@U2@@SA?AVGUrl@2@ABV32@ABVQStringList@@@Z 10018eba f   U2Core:U2Core.dll
 0001:00017ec0       ?rollFileName@GUrlUtils@U2@@SA?AVQString@@ABV3@0ABV?$QSet@VQString@@@@@Z 10018ec0 f   U2Core:U2Core.dll
 0001:00017ec6       ?createDirectory@GUrlUtils@U2@@SA?AVQString@@ABV3@0AAVU2OpStatus@2@@Z 10018ec6 f   U2Core:U2Core.dll
 0001:00017ecc       ??0U2OpStatusImpl@U2@@QAE@XZ 10018ecc f   U2Core:U2Core.dll
 0001:00017ed2       ?getError@U2OpStatusImpl@U2@@UBE?AVQString@@XZ 10018ed2 f   U2Core:U2Core.dll
 0001:00017ed8       ??1U2OpStatusImpl@U2@@UAE@XZ 10018ed8 f   U2Core:U2Core.dll
 0001:00017ede       ?tr@ExternalToolLogParser@U2@@SA?AVQString@@PBD0H@Z 10018ede f   U2Core:U2Core.dll
 0001:00017ee4       ??0ExternalTool@U2@@QAE@VQString@@00@Z 10018ee4 f   U2Core:U2Core.dll
 0001:00017eea       ??1ExternalTool@U2@@UAE@XZ 10018eea f   U2Core:U2Core.dll
 0001:00017ef0       ?registerEntry@ExternalToolRegistry@U2@@QAE_NPAVExternalTool@2@@Z 10018ef0 f   U2Core:U2Core.dll
 0001:00017ef6       ?unregisterEntry@ExternalToolRegistry@U2@@QAEXABVQString@@@Z 10018ef6 f   U2Core:U2Core.dll
 0001:00017efc       ?setToolkitDescription@ExternalToolRegistry@U2@@QAEXABVQString@@0@Z 10018efc f   U2Core:U2Core.dll
 0001:00017f02       ?getMainWindow@AppContext@U2@@SAPAVMainWindow@2@XZ 10018f02 f   U2Core:U2Core.dll
 0001:00017f08       ?extractAdditionalParameters@ExternalTool@U2@@UAEXABVQString@@@Z 10018f08 f   U2Core:U2Core.dll
 0001:00017f0e       ?getAdditionalPaths@ExternalTool@U2@@UBE?AVQStringList@@XZ 10018f0e f   U2Core:U2Core.dll
 0001:00017f14       ?getRunParameters@ExternalTool@U2@@UBE?AVQStringList@@XZ 10018f14 f   U2Core:U2Core.dll
 0001:00017f1a       ?getToolRunnerAdditionalOptions@ExternalTool@U2@@UBE?AVQStringList@@XZ 10018f1a f   U2Core:U2Core.dll
 0001:00017f20       ?performAdditionalChecks@ExternalTool@U2@@UAEXABVQString@@@Z 10018f20 f   U2Core:U2Core.dll
 0001:00017f26       ?getTestFramework@AppContext@U2@@SAPAVTestFramework@2@XZ 10018f26 f   U2Core:U2Core.dll
 0001:00017f2c       ?getExternalToolRegistry@AppContext@U2@@SAPAVExternalToolRegistry@2@XZ 10018f2c f   U2Core:U2Core.dll
 0001:00017f32       ??0Plugin@U2@@QAE@ABVQString@@0_NW4PluginState@1@@Z 10018f32 f   U2Core:U2Core.dll
 0001:00017f38       ??1Plugin@U2@@UAE@XZ       10018f38 f   U2Core:U2Core.dll
 0001:00017f3e       ?qt_metacast@Task@U2@@UAEPAXPBD@Z 10018f3e f   U2Core:U2Core.dll
 0001:00017f44       ?qt_metacall@Task@U2@@UAEHW4Call@QMetaObject@@HPAPAX@Z 10018f44 f   U2Core:U2Core.dll
 0001:00017f4a       ?qt_metacast@ExternalTool@U2@@UAEPAXPBD@Z 10018f4a f   U2Core:U2Core.dll
 0001:00017f50       ?qt_metacall@ExternalTool@U2@@UAEHW4Call@QMetaObject@@HPAPAX@Z 10018f50 f   U2Core:U2Core.dll
 0001:00017f56       ?qt_metacast@Plugin@U2@@UAEPAXPBD@Z 10018f56 f   U2Core:U2Core.dll
 0001:00017f5c       ?qt_metacall@Plugin@U2@@UAEHW4Call@QMetaObject@@HPAPAX@Z 10018f5c f   U2Core:U2Core.dll
 0001:00017f62       ?prepareFileFilter@DialogUtils@U2@@SA?AVQString@@ABV3@ABVQStringList@@_N1@Z 10018f62 f   U2Gui:U2Gui.dll
 0001:00017f68       ?findFormat@GTestFormatRegistry@U2@@QAEPAVGTestFormat@2@ABVQString@@@Z 10018f68 f   U2Test:U2Test.dll
 0001:00017f6e       ??0XMLTestFactory@U2@@QAE@ABVQString@@@Z 10018f6e f   U2Test:U2Test.dll
 0001:00017f74       ??1XMLTestFactory@U2@@UAE@XZ 10018f74 f   U2Test:U2Test.dll
 0001:00017f7a       ??0XmlTest@U2@@QAE@ABVQString@@PAVGTest@1@PBVGTestEnvironment@1@V?$QFlags@W4TaskFlag@U2@@@@ABV?$QList@PAVGTest@U2@@@@@Z 10018f7a f   U2Test:U2Test.dll
 0001:00017f80       ?checkNecessaryAttributeExistence@XmlTest@U2@@QAEXABVQDomElement@@ABVQString@@@Z 10018f80 f   U2Test:U2Test.dll
 0001:00017f86       ??1XmlTest@U2@@UAE@XZ      10018f86 f   U2Test:U2Test.dll
 0001:00017f8c       ?replacePrefix@XMLTestUtils@U2@@SAXPBVGTestEnvironment@2@AAVQString@@@Z 10018f8c f   U2Test:U2Test.dll
 0001:00017f92       ?metaObject@GTest@U2@@UBEPBUQMetaObject@@XZ 10018f92 f   U2Test:U2Test.dll
 0001:00017f98       ?qt_metacall@GTest@U2@@UAEHW4Call@QMetaObject@@HPAPAX@Z 10018f98 f   U2Test:U2Test.dll
 0001:00017f9e       ?qt_metacast@GTest@U2@@UAEPAXPBD@Z 10018f9e f   U2Test:U2Test.dll
 0001:00017fa4       ??0Descriptor@U2@@QAE@ABVQString@@00@Z 10018fa4 f   U2Lang:U2Lang.dll
 0001:00017faa       ??0Descriptor@U2@@QAE@ABVQString@@@Z 10018faa f   U2Lang:U2Lang.dll
 0001:00017fb0       ??0Descriptor@U2@@QAE@PBD@Z 10018fb0 f   U2Lang:U2Lang.dll
 0001:00017fb6       ??1Descriptor@U2@@UAE@XZ   10018fb6 f   U2Lang:U2Lang.dll
 0001:00017fbc       ?getId@Descriptor@U2@@QBE?AVQString@@XZ 10018fbc f   U2Lang:U2Lang.dll
 0001:00017fc2       ??0Descriptor@U2@@QAE@ABV01@@Z 10018fc2 f   U2Lang:U2Lang.dll
 0001:00017fc8       ??0MapDataType@U2@@QAE@ABVDescriptor@1@ABV?$QMap@VDescriptor@U2@@V?$QExplicitlySharedDataPointer@VDataType@U2@@@@@@@Z 10018fc8 f   U2Lang:U2Lang.dll
 0001:00017fce       ??1MapDataType@U2@@UAE@XZ  10018fce f   U2Lang:U2Lang.dll
 0001:00017fd4       ?initEngine@WorkflowScriptLibrary@U2@@SAXPAVWorkflowScriptEngine@2@@Z 10018fd4 f   U2Lang:U2Lang.dll
 0001:00017fda       ??0WorkflowNotification@U2@@QAE@ABVQString@@00@Z 10018fda f   U2Lang:U2Lang.dll
 0001:00017fe0       ??1WorkflowNotification@U2@@QAE@XZ 10018fe0 f   U2Lang:U2Lang.dll
 0001:00017fe6       ??0WorkflowNotification@U2@@QAE@ABV01@@Z 10018fe6 f   U2Lang:U2Lang.dll
 0001:00017fec       ??0MessageMetadata@U2@@QAE@ABVQString@@@Z 10018fec f   U2Lang:U2Lang.dll
 0001:00017ff2       ?getId@MessageMetadata@U2@@QBEHXZ 10018ff2 f   U2Lang:U2Lang.dll
 0001:00017ff8       ??1MessageMetadata@U2@@QAE@XZ 10018ff8 f   U2Lang:U2Lang.dll
 0001:00017ffe       ?put@MessageMetadataStorage@U2@@QAEXABVMessageMetadata@2@@Z 10018ffe f   U2Lang:U2Lang.dll
 0001:00018004       ?getMonitor@WorkflowContext@Workflow@U2@@QAEPAVWorkflowMonitor@23@XZ 10019004 f   U2Lang:U2Lang.dll
 0001:0001800a       ?absolutePath@WorkflowContext@Workflow@U2@@QBE?AVQString@@ABV4@@Z 1001900a f   U2Lang:U2Lang.dll
 0001:00018010       ?getMetadataStorage@WorkflowContext@Workflow@U2@@QAEAAVMessageMetadataStorage@3@XZ 10019010 f   U2Lang:U2Lang.dll
 0001:00018016       ??0WorkflowScriptEngine@U2@@QAE@PAVWorkflowContext@Workflow@1@@Z 10019016 f   U2Lang:U2Lang.dll
 0001:0001801c       ??1WorkflowScriptEngine@U2@@UAE@XZ 1001901c f   U2Lang:U2Lang.dll
 0001:00018022       ?isEmpty@AttributeScript@U2@@QBE_NXZ 10019022 f   U2Lang:U2Lang.dll
 0001:00018028       ?getScriptText@AttributeScript@U2@@QBEABVQString@@XZ 10019028 f   U2Lang:U2Lang.dll
 0001:0001802e       ?getScriptVars@AttributeScript@U2@@QBEABV?$QMap@VDescriptor@U2@@VQVariant@@@@XZ 1001902e f   U2Lang:U2Lang.dll
 0001:00018034       ??0Attribute@U2@@QAE@ABVDescriptor@1@V?$QExplicitlySharedDataPointer@VDataType@U2@@@@_NABVQVariant@@@Z 10019034 f   U2Lang:U2Lang.dll
 0001:0001803a       ??1Attribute@U2@@UAE@XZ    1001903a f   U2Lang:U2Lang.dll
 0001:00018040       ?isOutUrlAttribute@RFSUtils@U2@@SA_NPAVAttribute@2@PAVActor@Workflow@2@AA_N@Z 10019040 f   U2Lang:U2Lang.dll
 0001:00018046       ??1PropertyDelegate@U2@@UAE@XZ 10019046 f   U2Lang:U2Lang.dll
 0001:0001804c       ??0DelegateTags@U2@@QAE@PAVQObject@@@Z 1001904c f   U2Lang:U2Lang.dll
 0001:00018052       ?set@DelegateTags@U2@@QAEXABVQString@@ABVQVariant@@@Z 10019052 f   U2Lang:U2Lang.dll
 0001:00018058       ??1DelegateTags@U2@@UAE@XZ 10019058 f   U2Lang:U2Lang.dll
 0001:0001805e       ?getId@Actor@Workflow@U2@@QBE?AVQString@@XZ 1001905e f   U2Lang:U2Lang.dll
 0001:00018064       ?getInputPorts@Actor@Workflow@U2@@QBE?AV?$QList@PAVPort@Workflow@U2@@@@XZ 10019064 f   U2Lang:U2Lang.dll
 0001:0001806a       ?getOutputPorts@Actor@Workflow@U2@@QBE?AV?$QList@PAVPort@Workflow@U2@@@@XZ 1001906a f   U2Lang:U2Lang.dll
 0001:00018070       ??0PortDescriptor@Workflow@U2@@QAE@ABVDescriptor@2@V?$QExplicitlySharedDataPointer@VDataType@U2@@@@_N2I@Z 10019070 f   U2Lang:U2Lang.dll
 0001:00018076       ??1PortDescriptor@Workflow@U2@@UAE@XZ 10019076 f   U2Lang:U2Lang.dll
 0001:0001807c       ??0ActorPrototype@Workflow@U2@@QAE@ABVDescriptor@2@ABV?$QList@PAVPortDescriptor@Workflow@U2@@@@ABV?$QList@PAVAttribute@U2@@@@@Z 1001907c f   U2Lang:U2Lang.dll
 0001:00018082       ??1ActorPrototype@Workflow@U2@@UAE@XZ 10019082 f   U2Lang:U2Lang.dll
 0001:00018088       ?setEditor@ActorPrototype@Workflow@U2@@QAEXPAVConfigurationEditor@3@@Z 10019088 f   U2Lang:U2Lang.dll
 0001:0001808e       ?setValidator@ActorPrototype@Workflow@U2@@QAEXPAVConfigurationValidator@3@@Z 1001908e f   U2Lang:U2Lang.dll
 0001:00018094       ?setPrompter@ActorPrototype@Workflow@U2@@QAEXPAVPrompter@23@@Z 10019094 f   U2Lang:U2Lang.dll
 0001:0001809a       ?addExternalTool@ActorPrototype@Workflow@U2@@QAEXABVQString@@0@Z 1001909a f   U2Lang:U2Lang.dll
 0001:000180a0       ?registerProto@ActorPrototypeRegistry@Workflow@U2@@QAE_NABVDescriptor@3@PAVActorPrototype@23@@Z 100190a0 f   U2Lang:U2Lang.dll
 0001:000180a6       ?unregisterProto@ActorPrototypeRegistry@Workflow@U2@@QAEPAVActorPrototype@23@ABVQString@@@Z 100190a6 f   U2Lang:U2Lang.dll
 0001:000180ac       ?URL_SLOT@BaseSlots@Workflow@U2@@SA?BVDescriptor@3@XZ 100190ac f   U2Lang:U2Lang.dll
 0001:000180b2       ?STRING_TYPE@BaseTypes@U2@@SA?AV?$QExplicitlySharedDataPointer@VDataType@U2@@@@XZ 100190b2 f   U2Lang:U2Lang.dll
 0001:000180b8       ?NUM_TYPE@BaseTypes@U2@@SA?AV?$QExplicitlySharedDataPointer@VDataType@U2@@@@XZ 100190b8 f   U2Lang:U2Lang.dll
 0001:000180be       ?URL_DATASETS_TYPE@BaseTypes@U2@@SA?AV?$QExplicitlySharedDataPointer@VDataType@U2@@@@XZ 100190be f   U2Lang:U2Lang.dll
 0001:000180c4       ??0Dataset@U2@@QAE@ABV01@@Z 100190c4 f   U2Lang:U2Lang.dll
 0001:000180ca       ??1Dataset@U2@@QAE@XZ      100190ca f   U2Lang:U2Lang.dll
 0001:000180d0       ??0DatasetFilesIterator@U2@@QAE@ABV?$QList@VDataset@U2@@@@@Z 100190d0 f   U2Lang:U2Lang.dll
 0001:000180d6       ??1DatasetFilesIterator@U2@@UAE@XZ 100190d6 f   U2Lang:U2Lang.dll
 0001:000180dc       ?getNextFile@DatasetFilesIterator@U2@@UAE?AVQString@@XZ 100190dc f   U2Lang:U2Lang.dll
 0001:000180e2       ?hasNext@DatasetFilesIterator@U2@@UAE_NXZ 100190e2 f   U2Lang:U2Lang.dll
 0001:000180e8       ?getInstance@WorkflowEnv@Workflow@U2@@KAPAV123@XZ 100190e8 f   U2Lang:U2Lang.dll
 0001:000180ee       ??0Message@Workflow@U2@@QAE@V?$QExplicitlySharedDataPointer@VDataType@U2@@@@ABVQVariant@@H@Z 100190ee f   U2Lang:U2Lang.dll
 0001:000180f4       ??1Message@Workflow@U2@@QAE@XZ 100190f4 f   U2Lang:U2Lang.dll
 0001:000180fa       ??0DomainFactory@Workflow@U2@@QAE@ABVQString@@@Z 100190fa f   U2Lang:U2Lang.dll
 0001:00018100       ??1DomainFactory@Workflow@U2@@UAE@XZ 10019100 f   U2Lang:U2Lang.dll
 0001:00018106       ?addOutputFile@WorkflowMonitor@Workflow@U2@@QAEXABVQString@@0_N@Z 10019106 f   U2Lang:U2Lang.dll
 0001:0001810c       ?getBusType@IntegralBus@Workflow@U2@@QBE?AV?$QExplicitlySharedDataPointer@VDataType@U2@@@@XZ 1001910c f   U2Lang:U2Lang.dll
 0001:00018112       ??0BaseWorker@LocalWorkflow@U2@@QAE@PAVActor@Workflow@2@_N@Z 10019112 f   U2Lang:U2Lang.dll
 0001:00018118       ??1BaseWorker@LocalWorkflow@U2@@UAE@XZ 10019118 f   U2Lang:U2Lang.dll
 0001:0001811e       ?createLogListeners@BaseWorker@LocalWorkflow@U2@@QBE?AV?$QList@PAVExternalToolListener@U2@@@@H@Z 1001911e f   U2Lang:U2Lang.dll
 0001:00018124       ??0PrompterBaseImpl@U2@@QAE@PAVActor@Workflow@1@@Z 10019124 f   U2Lang:U2Lang.dll
 0001:0001812a       ?getURL@PrompterBaseImpl@U2@@QAE?AVQString@@ABV3@PA_N00@Z 1001912a f   U2Lang:U2Lang.dll
 0001:00018130       ?getHyperlink@PrompterBaseImpl@U2@@SA?AVQString@@ABV3@0@Z 10019130 f   U2Lang:U2Lang.dll
 0001:00018136       ??1PrompterBaseImpl@U2@@UAE@XZ 10019136 f   U2Lang:U2Lang.dll
 0001:0001813c       ?addCommunication@BaseWorker@LocalWorkflow@U2@@UAE_NABVQString@@PAVCommunicationChannel@Workflow@3@@Z 1001913c f   U2Lang:U2Lang.dll
 0001:00018142       ?canTaskBeCanceled@BaseWorker@LocalWorkflow@U2@@MBE_NPAVTask@3@@Z 10019142 f   U2Lang:U2Lang.dll
 0001:00018148       ?clone@Attribute@U2@@UAEPAV12@XZ 10019148 f   U2Lang:U2Lang.dll
 0001:0001814e       ?createConnection@DomainFactory@Workflow@U2@@UAEPAVCommunicationChannel@23@PAVLink@23@@Z 1001914e f   U2Lang:U2Lang.dll
 0001:00018154       ?createInstance@ActorPrototype@Workflow@U2@@UAEPAVActor@23@ABVQString@@PAVAttributeScript@3@ABV?$QMap@VQString@@VQVariant@@@@@Z 10019154 f   U2Lang:U2Lang.dll
 0001:0001815a       ?createPort@IntegralBusActorPrototype@Workflow@U2@@UAEPAVPort@23@ABVPortDescriptor@23@PAVActor@23@@Z 1001915a f   U2Lang:U2Lang.dll
 0001:00018160       ?createScheduler@DomainFactory@Workflow@U2@@UAEPAVScheduler@23@PAVSchema@23@@Z 10019160 f   U2Lang:U2Lang.dll
 0001:00018166       ?destroy@DomainFactory@Workflow@U2@@UAEXPAVScheduler@23@PAVSchema@23@@Z 10019166 f   U2Lang:U2Lang.dll
 0001:0001816c       ?getActorId@BaseWorker@LocalWorkflow@U2@@UBE?AVQString@@XZ 1001916c f   U2Lang:U2Lang.dll
 0001:00018172       ?getAllDescriptors@MapDataType@U2@@UBE?AV?$QList@VDescriptor@U2@@@@XZ 10019172 f   U2Lang:U2Lang.dll
 0001:00018178       ?getAllEntries@?$IdRegistry@VDomainFactory@Workflow@U2@@@U2@@UBE?AV?$QList@PAVDomainFactory@Workflow@U2@@@@XZ 10019178 f   U2Lang:U2Lang.dll
 0001:0001817e       ?getAllIds@?$IdRegistry@VDomainFactory@Workflow@U2@@@U2@@UBE?AV?$QList@VQString@@@@XZ 1001917e f   U2Lang:U2Lang.dll
 0001:00018184       ?getAttributePureValue@Attribute@U2@@UBEABVQVariant@@XZ 10019184 f   U2Lang:U2Lang.dll
 0001:0001818a       ?getById@?$IdRegistry@VDomainFactory@Workflow@U2@@@U2@@UAEPAVDomainFactory@Workflow@2@ABVQString@@@Z 1001918a f   U2Lang:U2Lang.dll
 0001:00018190       ?getCommunication@BaseWorker@LocalWorkflow@U2@@UAEPAVCommunicationChannel@Workflow@3@ABVQString@@@Z 10019190 f   U2Lang:U2Lang.dll
 0001:00018196       ?getDatatypeByDescriptor@MapDataType@U2@@UBE?AV?$QExplicitlySharedDataPointer@VDataType@U2@@@@ABVDescriptor@2@@Z 10019196 f   U2Lang:U2Lang.dll
 0001:0001819c       ?getDatatypesMap@MapDataType@U2@@UBE?AV?$QMap@VDescriptor@U2@@V?$QExplicitlySharedDataPointer@VDataType@U2@@@@@@XZ 1001919c f   U2Lang:U2Lang.dll
 0001:000181a2       ?getDefaultPureValue@Attribute@U2@@UBEABVQVariant@@XZ 100191a2 f   U2Lang:U2Lang.dll
 0001:000181a8       ?getGroup@Attribute@U2@@UAE?AW4AttributeGroup@2@XZ 100191a8 f   U2Lang:U2Lang.dll
 0001:000181ae       ?getItems@PropertyDelegate@U2@@UBEXAAV?$QMap@VQString@@VQVariant@@@@@Z 100191ae f   U2Lang:U2Lang.dll
 0001:000181b4       ?getMessageAndSetupScriptValues@BaseWorker@LocalWorkflow@U2@@UAE?AVMessage@Workflow@3@PAVCommunicationChannel@53@@Z 100191b4 f   U2Lang:U2Lang.dll
 0001:000181ba       ?getOutputFiles@BaseWorker@LocalWorkflow@U2@@UAE?AVQStringList@@XZ 100191ba f   U2Lang:U2Lang.dll
 0001:000181c0       ?getType@PortDescriptor@Workflow@U2@@UBE?AV?$QExplicitlySharedDataPointer@VDataType@U2@@@@XZ 100191c0 f   U2Lang:U2Lang.dll
 0001:000181c6       ?getWidget@ConfigurationEditor@U2@@UAEPAVQWidget@@XZ 100191c6 f   U2Lang:U2Lang.dll
 0001:000181cc       ?isAcceptableDrop@ActorPrototype@Workflow@U2@@UBE_NPBVQMimeData@@PAV?$QMap@VQString@@VQVariant@@@@@Z 100191cc f   U2Lang:U2Lang.dll
 0001:000181d2       ?isDefaultValue@Attribute@U2@@UBE_NXZ 100191d2 f   U2Lang:U2Lang.dll
 0001:000181d8       ?isDone@BaseWorker@LocalWorkflow@U2@@UBE_NXZ 100191d8 f   U2Lang:U2Lang.dll
 0001:000181de       ?isEmpty@Attribute@U2@@UBE_NXZ 100191de f   U2Lang:U2Lang.dll
 0001:000181e4       ?isEmpty@ConfigurationEditor@U2@@UBE_NXZ 100191e4 f   U2Lang:U2Lang.dll
 0001:000181ea       ?isReady@BaseWorker@LocalWorkflow@U2@@UBE_NXZ 100191ea f   U2Lang:U2Lang.dll
 0001:000181f0       ?kind@MapDataType@U2@@UBE?AW4Kind@DataType@2@XZ 100191f0 f   U2Lang:U2Lang.dll
 0001:000181f6       ?metaObject@ActorPrototype@Workflow@U2@@UBEPBUQMetaObject@@XZ 100191f6 f   U2Lang:U2Lang.dll
 0001:000181fc       ?metaObject@PrompterBaseImpl@U2@@UBEPBUQMetaObject@@XZ 100191fc f   U2Lang:U2Lang.dll
 0001:00018202       ?qt_metacall@ActorPrototype@Workflow@U2@@UAEHW4Call@QMetaObject@@HPAPAX@Z 10019202 f   U2Lang:U2Lang.dll
 0001:00018208       ?qt_metacall@PrompterBaseImpl@U2@@UAEHW4Call@QMetaObject@@HPAPAX@Z 10019208 f   U2Lang:U2Lang.dll
 0001:0001820e       ?qt_metacast@ActorPrototype@Workflow@U2@@UAEPAXPBD@Z 1001920e f   U2Lang:U2Lang.dll
 0001:00018214       ?qt_metacast@PrompterBaseImpl@U2@@UAEPAXPBD@Z 10019214 f   U2Lang:U2Lang.dll
 0001:0001821a       ?registerEntry@?$IdRegistry@VDomainFactory@Workflow@U2@@@U2@@UAE_NPAVDomainFactory@Workflow@2@@Z 1001921a f   U2Lang:U2Lang.dll
 0001:00018220       ?setAttributeValue@Attribute@U2@@UAEXABVQVariant@@@Z 10019220 f   U2Lang:U2Lang.dll
 0001:00018226       ?setDisplayName@ActorPrototype@Workflow@U2@@UAEXABVQString@@@Z 10019226 f   U2Lang:U2Lang.dll
 0001:0001822c       ?setDisplayName@Descriptor@U2@@UAEXABVQString@@@Z 1001922c f   U2Lang:U2Lang.dll
 0001:00018232       ?setDocumentation@ActorPrototype@Workflow@U2@@UAEXABVQString@@@Z 10019232 f   U2Lang:U2Lang.dll
 0001:00018238       ?setDocumentation@Descriptor@U2@@UAEXABVQString@@@Z 10019238 f   U2Lang:U2Lang.dll
 0001:0001823e       ?setDone@BaseWorker@LocalWorkflow@U2@@UAEXXZ 1001923e f   U2Lang:U2Lang.dll
 0001:00018244       ?setVisibleSlot@PortDescriptor@Workflow@U2@@UAEXABVQString@@_N@Z 10019244 f   U2Lang:U2Lang.dll
 0001:0001824a       ?sl_actorModified@PrompterBaseImpl@U2@@MAEXXZ 1001924a f   U2Lang:U2Lang.dll
 0001:00018250       ?type@PropertyDelegate@U2@@UBE?AW4Type@12@XZ 10019250 f   U2Lang:U2Lang.dll
 0001:00018256       ?unregisterEntry@?$IdRegistry@VDomainFactory@Workflow@U2@@@U2@@UAEPAVDomainFactory@Workflow@2@ABVQString@@@Z 10019256 f   U2Lang:U2Lang.dll
 0001:0001825c       ?update@PrompterBaseImpl@U2@@UAEXABV?$QMap@VQString@@VQVariant@@@@@Z 1001925c f   U2Lang:U2Lang.dll
 0001:00018262       ?update@PropertyDelegate@U2@@UAEXXZ 10019262 f   U2Lang:U2Lang.dll
 0001:00018268       ?updateActorIds@Attribute@U2@@UAEXABV?$QMap@VQString@@V1@@@@Z 10019268 f   U2Lang:U2Lang.dll
 0001:0001826e       ?validate@ActorValidator@Workflow@U2@@UBE_NPBVConfiguration@3@AAV?$QList@VWorkflowNotification@U2@@@@@Z 1001926e f   U2Lang:U2Lang.dll
 0001:00018274       ?validate@Attribute@U2@@UAE_NAAV?$QList@VWorkflowNotification@U2@@@@@Z 10019274 f   U2Lang:U2Lang.dll
 0001:0001827a       ??0VisibilityRelation@U2@@QAE@ABVQString@@ABVQVariant@@_N@Z 1001927a f   U2Lang:U2Lang.dll
 0001:00018280       ??1VisibilityRelation@U2@@UAE@XZ 10019280 f   U2Lang:U2Lang.dll
 0001:00018286       ?getFileUrl@MessageMetadata@U2@@QBEABVQString@@XZ 10019286 f   U2Lang:U2Lang.dll
 0001:0001828c       ?get@MessageMetadataStorage@U2@@QBE?AVMessageMetadata@2@H@Z 1001928c f   U2Lang:U2Lang.dll
 0001:00018292       ?workingDir@WorkflowContext@Workflow@U2@@QBE?AVQString@@XZ 10019292 f   U2Lang:U2Lang.dll
 0001:00018298       ??0SlotRelationDescriptor@U2@@QAE@ABVQString@@0ABV?$QList@VQVariant@@@@@Z 10019298 f   U2Lang:U2Lang.dll
 0001:0001829e       ??1SlotRelationDescriptor@U2@@UAE@XZ 1001929e f   U2Lang:U2Lang.dll
 0001:000182a4       ??0Attribute@U2@@QAE@ABVDescriptor@1@V?$QExplicitlySharedDataPointer@VDataType@U2@@@@V?$QFlags@W4Flag@Attribute@U2@@@@ABVQVariant@@@Z 100192a4 f   U2Lang:U2Lang.dll
 0001:000182aa       ?addRelation@Attribute@U2@@QAEXPBVAttributeRelation@2@@Z 100192aa f   U2Lang:U2Lang.dll
 0001:000182b0       ?addSlotRelation@Attribute@U2@@QAEXPAVSlotRelationDescriptor@2@@Z 100192b0 f   U2Lang:U2Lang.dll
 0001:000182b6       ?setPortValidator@ActorPrototype@Workflow@U2@@QAEXABVQString@@PAVConfigurationValidator@3@@Z 100192b6 f   U2Lang:U2Lang.dll
 0001:000182bc       ?BOOL_TYPE@BaseTypes@U2@@SA?AV?$QExplicitlySharedDataPointer@VDataType@U2@@@@XZ 100192bc f   U2Lang:U2Lang.dll
 0001:000182c2       ??0PairedReadsPortValidator@Workflow@U2@@QAE@ABVQString@@0@Z 100192c2 f   U2Lang:U2Lang.dll
 0001:000182c8       ??1PairedReadsPortValidator@Workflow@U2@@UAE@XZ 100192c8 f   U2Lang:U2Lang.dll
 0001:000182ce       ?getData@Message@Workflow@U2@@QBE?AVQVariant@@XZ 100192ce f   U2Lang:U2Lang.dll
 0001:000182d4       ?getMetadataId@Message@Workflow@U2@@QBEHXZ 100192d4 f   U2Lang:U2Lang.dll
 0001:000182da       ?addInfo@WorkflowMonitor@Workflow@U2@@QAEXABVQString@@00@Z 100192da f   U2Lang:U2Lang.dll
 0001:000182e0       ?reportError@BaseWorker@LocalWorkflow@U2@@IAEXABVQString@@@Z 100192e0 f   U2Lang:U2Lang.dll
 0001:000182e6       ?getParameter@PrompterBaseImpl@U2@@QAE?AVQVariant@@ABVQString@@@Z 100192e6 f   U2Lang:U2Lang.dll
 0001:000182ec       ?getProducersOrUnset@PrompterBaseImpl@U2@@QAE?AVQString@@ABV3@0@Z 100192ec f   U2Lang:U2Lang.dll
 0001:000182f2       ?clone@SlotRelationDescriptor@U2@@UBEPAV12@XZ 100192f2 f   U2Lang:U2Lang.dll
 0001:000182f8       ?clone@VisibilityRelation@U2@@UBEPAV12@XZ 100192f8 f   U2Lang:U2Lang.dll
 0001:000182fe       ?getAffectResult@VisibilityRelation@U2@@UBE?AVQVariant@@ABV3@0PAVDelegateTags@2@1@Z 100192fe f   U2Lang:U2Lang.dll
 0001:00018304       ?getType@VisibilityRelation@U2@@UBE?AW4RelationType@2@XZ 10019304 f   U2Lang:U2Lang.dll
 0001:0001830a       ?isSlotEnabled@SlotRelationDescriptor@U2@@UBE_NABVQVariant@@@Z 1001930a f   U2Lang:U2Lang.dll
 0001:00018310       ?updateDelegateTags@AttributeRelation@U2@@UBEXABVQVariant@@PAVDelegateTags@2@@Z 10019310 f   U2Lang:U2Lang.dll
 0001:00018316       ?validate@PairedReadsPortValidator@Workflow@U2@@UBE_NPBVIntegralBusPort@23@AAV?$QList@VWorkflowNotification@U2@@@@@Z 10019316 f   U2Lang:U2Lang.dll
 0001:0001831c       ?validate@PortValidator@Workflow@U2@@UBE_NPBVConfiguration@3@AAV?$QList@VWorkflowNotification@U2@@@@@Z 1001931c f   U2Lang:U2Lang.dll
 0001:00018322       ?valueChangingRelation@VisibilityRelation@U2@@UBE_NXZ 10019322 f   U2Lang:U2Lang.dll
 0001:00018328       ?qt_metacast@BaseWorker@LocalWorkflow@U2@@UAEPAXPBD@Z 10019328 f   U2Lang:U2Lang.dll
 0001:0001832e       ?qt_metacall@BaseWorker@LocalWorkflow@U2@@UAEHW4Call@QMetaObject@@HPAPAX@Z 1001932e f   U2Lang:U2Lang.dll
 0001:00018334       ??0DelegateEditor@U2@@QAE@ABV?$QMap@VQString@@PAVPropertyDelegate@U2@@@@@Z 10019334 f   U2Designer:U2Designer.dll
 0001:0001833a       ??1DelegateEditor@U2@@UAE@XZ 1001933a f   U2Designer:U2Designer.dll
 0001:00018340       ??0URLDelegate@U2@@QAE@ABVDelegateTags@1@ABVQString@@ABV?$QFlags@W4Option@URLDelegate@U2@@@@PAVQObject@@@Z 10019340 f   U2Designer:U2Designer.dll
 0001:00018346       ??1URLDelegate@U2@@UAE@XZ  10019346 f   U2Designer:U2Designer.dll
 0001:0001834c       ??0ComboBoxDelegate@U2@@QAE@ABV?$QMap@VQString@@VQVariant@@@@PAVQObject@@@Z 1001934c f   U2Designer:U2Designer.dll
 0001:00018352       ??1ComboBoxDelegate@U2@@UAE@XZ 10019352 f   U2Designer:U2Designer.dll
 0001:00018358       ?addDelegate@DelegateEditor@U2@@UAEXPAVPropertyDelegate@2@ABVQString@@@Z 10019358 f   U2Designer:U2Designer.dll
 0001:0001835e       ?clone@ComboBoxDelegate@U2@@UAEPAVPropertyDelegate@2@XZ 1001935e f   U2Designer:U2Designer.dll
 0001:00018364       ?clone@DelegateEditor@U2@@UAEPAVConfigurationEditor@2@XZ 10019364 f   U2Designer:U2Designer.dll
 0001:0001836a       ?clone@URLDelegate@U2@@UAEPAVPropertyDelegate@2@XZ 1001936a f   U2Designer:U2Designer.dll
 0001:00018370       ?commit@DelegateEditor@U2@@UAEXXZ 10019370 f   U2Designer:U2Designer.dll
 0001:00018376       ?createEditor@ComboBoxDelegate@U2@@UBEPAVQWidget@@PAV3@ABVQStyleOptionViewItem@@ABVQModelIndex@@@Z 10019376 f   U2Designer:U2Designer.dll
 0001:0001837c       ?createEditor@URLDelegate@U2@@UBEPAVQWidget@@PAV3@ABVQStyleOptionViewItem@@ABVQModelIndex@@@Z 1001937c f   U2Designer:U2Designer.dll
 0001:00018382       ?createWizardWidget@ComboBoxDelegate@U2@@UBEPAVPropertyWidget@2@AAVU2OpStatus@2@PAVQWidget@@@Z 10019382 f   U2Designer:U2Designer.dll
 0001:00018388       ?createWizardWidget@URLDelegate@U2@@UBEPAVPropertyWidget@2@AAVU2OpStatus@2@PAVQWidget@@@Z 10019388 f   U2Designer:U2Designer.dll
 0001:0001838e       ?getDelegate@DelegateEditor@U2@@UAEPAVPropertyDelegate@2@ABVQString@@@Z 1001938e f   U2Designer:U2Designer.dll
 0001:00018394       ?getDisplayValue@ComboBoxDelegate@U2@@UBE?AVQVariant@@ABV3@@Z 10019394 f   U2Designer:U2Designer.dll
 0001:0001839a       ?getDisplayValue@URLDelegate@U2@@UBE?AVQVariant@@ABV3@@Z 1001939a f   U2Designer:U2Designer.dll
 0001:000183a0       ?getItems@ComboBoxDelegate@U2@@UBEXAAV?$QMap@VQString@@VQVariant@@@@@Z 100193a0 f   U2Designer:U2Designer.dll
 0001:000183a6       ?metaObject@ComboBoxDelegate@U2@@UBEPBUQMetaObject@@XZ 100193a6 f   U2Designer:U2Designer.dll
 0001:000183ac       ?metaObject@DelegateEditor@U2@@UBEPBUQMetaObject@@XZ 100193ac f   U2Designer:U2Designer.dll
 0001:000183b2       ?metaObject@URLDelegate@U2@@UBEPBUQMetaObject@@XZ 100193b2 f   U2Designer:U2Designer.dll
 0001:000183b8       ?qt_metacall@ComboBoxDelegate@U2@@UAEHW4Call@QMetaObject@@HPAPAX@Z 100193b8 f   U2Designer:U2Designer.dll
 0001:000183be       ?qt_metacall@DelegateEditor@U2@@UAEHW4Call@QMetaObject@@HPAPAX@Z 100193be f   U2Designer:U2Designer.dll
 0001:000183c4       ?qt_metacall@URLDelegate@U2@@UAEHW4Call@QMetaObject@@HPAPAX@Z 100193c4 f   U2Designer:U2Designer.dll
 0001:000183ca       ?qt_metacast@ComboBoxDelegate@U2@@UAEPAXPBD@Z 100193ca f   U2Designer:U2Designer.dll
 0001:000183d0       ?qt_metacast@DelegateEditor@U2@@UAEPAXPBD@Z 100193d0 f   U2Designer:U2Designer.dll
 0001:000183d6       ?qt_metacast@URLDelegate@U2@@UAEPAXPBD@Z 100193d6 f   U2Designer:U2Designer.dll
 0001:000183dc       ?removeDelegate@DelegateEditor@U2@@UAEPAVPropertyDelegate@2@ABVQString@@@Z 100193dc f   U2Designer:U2Designer.dll
 0001:000183e2       ?setEditorData@ComboBoxDelegate@U2@@UBEXPAVQWidget@@ABVQModelIndex@@@Z 100193e2 f   U2Designer:U2Designer.dll
 0001:000183e8       ?setEditorData@URLDelegate@U2@@UBEXPAVQWidget@@ABVQModelIndex@@@Z 100193e8 f   U2Designer:U2Designer.dll
 0001:000183ee       ?setModelData@ComboBoxDelegate@U2@@UBEXPAVQWidget@@PAVQAbstractItemModel@@ABVQModelIndex@@@Z 100193ee f   U2Designer:U2Designer.dll
 0001:000183f4       ?setModelData@URLDelegate@U2@@UBEXPAVQWidget@@PAVQAbstractItemModel@@ABVQModelIndex@@@Z 100193f4 f   U2Designer:U2Designer.dll
 0001:000183fa       ?type@URLDelegate@U2@@UBE?AW4Type@PropertyDelegate@2@XZ 100193fa f   U2Designer:U2Designer.dll
 0001:00018400       ?updateDelegate@DelegateEditor@U2@@UAEXABVQString@@@Z 10019400 f   U2Designer:U2Designer.dll
 0001:00018406       ?updateDelegates@DelegateEditor@U2@@UAEXXZ 10019406 f   U2Designer:U2Designer.dll
 0001:0001840c       ??0URLDelegate@U2@@QAE@ABVDelegateTags@1@ABVQString@@_N22PAVQObject@@22@Z 1001940c f   U2Designer:U2Designer.dll
 0001:00018412       ??0SpinBoxDelegate@U2@@QAE@ABV?$QMap@VQString@@VQVariant@@@@PAVQObject@@@Z 10019412 f   U2Designer:U2Designer.dll
 0001:00018418       ??1SpinBoxDelegate@U2@@UAE@XZ 10019418 f   U2Designer:U2Designer.dll
 0001:0001841e       ?clone@SpinBoxDelegate@U2@@UAEPAVPropertyDelegate@2@XZ 1001941e f   U2Designer:U2Designer.dll
 0001:00018424       ?createEditor@SpinBoxDelegate@U2@@UBEPAVQWidget@@PAV3@ABVQStyleOptionViewItem@@ABVQModelIndex@@@Z 10019424 f   U2Designer:U2Designer.dll
 0001:0001842a       ?createWizardWidget@SpinBoxDelegate@U2@@UBEPAVPropertyWidget@2@AAVU2OpStatus@2@PAVQWidget@@@Z 1001942a f   U2Designer:U2Designer.dll
 0001:00018430       ?getDisplayValue@SpinBoxDelegate@U2@@UBE?AVQVariant@@ABV3@@Z 10019430 f   U2Designer:U2Designer.dll
 0001:00018436       ?getItems@SpinBoxDelegate@U2@@UBEXAAV?$QMap@VQString@@VQVariant@@@@@Z 10019436 f   U2Designer:U2Designer.dll
 0001:0001843c       ?metaObject@SpinBoxDelegate@U2@@UBEPBUQMetaObject@@XZ 1001943c f   U2Designer:U2Designer.dll
 0001:00018442       ?qt_metacall@SpinBoxDelegate@U2@@UAEHW4Call@QMetaObject@@HPAPAX@Z 10019442 f   U2Designer:U2Designer.dll
 0001:00018448       ?qt_metacast@SpinBoxDelegate@U2@@UAEPAXPBD@Z 10019448 f   U2Designer:U2Designer.dll
 0001:0001844e       ?setEditorData@SpinBoxDelegate@U2@@UBEXPAVQWidget@@ABVQModelIndex@@@Z 1001944e f   U2Designer:U2Designer.dll
 0001:00018454       ?setModelData@SpinBoxDelegate@U2@@UBEXPAVQWidget@@PAVQAbstractItemModel@@ABVQModelIndex@@@Z 10019454 f   U2Designer:U2Designer.dll
 0001:0001845a       ??0GenomicLibraryDelegate@LocalWorkflow@U2@@QAE@PAVQObject@@@Z 1001945a f   ngs_reads_classification:ngs_reads_classification.dll
 0001:00018460       ?clone@GenomicLibraryDelegate@LocalWorkflow@U2@@UAEPAVPropertyDelegate@3@XZ 10019460 f   ngs_reads_classification:ngs_reads_classification.dll
 0001:00018466       ?createEditor@GenomicLibraryDelegate@LocalWorkflow@U2@@UBEPAVQWidget@@PAV4@ABVQStyleOptionViewItem@@ABVQModelIndex@@@Z 10019466 f   ngs_reads_classification:ngs_reads_classification.dll
 0001:0001846c       ?createWizardWidget@GenomicLibraryDelegate@LocalWorkflow@U2@@UBEPAVPropertyWidget@3@AAVU2OpStatus@3@PAVQWidget@@@Z 1001946c f   ngs_reads_classification:ngs_reads_classification.dll
 0001:00018472       ?getDisplayValue@GenomicLibraryDelegate@LocalWorkflow@U2@@UBE?AVQVariant@@ABV4@@Z 10019472 f   ngs_reads_classification:ngs_reads_classification.dll
 0001:00018478       ?metaObject@GenomicLibraryDelegate@LocalWorkflow@U2@@UBEPBUQMetaObject@@XZ 10019478 f   ngs_reads_classification:ngs_reads_classification.dll
 0001:0001847e       ?qt_metacall@GenomicLibraryDelegate@LocalWorkflow@U2@@UAEHW4Call@QMetaObject@@HPAPAX@Z 1001947e f   ngs_reads_classification:ngs_reads_classification.dll
 0001:00018484       ?qt_metacast@GenomicLibraryDelegate@LocalWorkflow@U2@@UAEPAXPBD@Z 10019484 f   ngs_reads_classification:ngs_reads_classification.dll
 0001:0001848a       ?setEditorData@GenomicLibraryDelegate@LocalWorkflow@U2@@UBEXPAVQWidget@@ABVQModelIndex@@@Z 1001948a f   ngs_reads_classification:ngs_reads_classification.dll
 0001:00018490       ?setModelData@GenomicLibraryDelegate@LocalWorkflow@U2@@UBEXPAVQWidget@@PAVQAbstractItemModel@@ABVQModelIndex@@@Z 10019490 f   ngs_reads_classification:ngs_reads_classification.dll
 0001:00018496       ?TAXONOMY_CLASSIFICATION_SLOT@TaxonomySupport@LocalWorkflow@U2@@SA?BVDescriptor@3@XZ 10019496 f   ngs_reads_classification:ngs_reads_classification.dll
 0001:0001849c       ?TAXONOMY_CLASSIFICATION_TYPE@TaxonomySupport@LocalWorkflow@U2@@SA?AV?$QExplicitlySharedDataPointer@VDataType@U2@@@@XZ 1001949c f   ngs_reads_classification:ngs_reads_classification.dll
 0001:000184a2       ??0DatabaseDelegate@LocalWorkflow@U2@@QAE@ABVQString@@0ABV?$QList@U?$QPair@VQString@@V1@@@@@0_N@Z 100194a2 f   ngs_reads_classification:ngs_reads_classification.dll
 0001:000184a8       ??1DatabaseDelegate@LocalWorkflow@U2@@UAE@XZ 100194a8 f   ngs_reads_classification:ngs_reads_classification.dll
 0001:000184ae       ?getBaseFileNameWithSuffixes@NgsReadsClassificationUtils@U2@@SA?AVQString@@ABV3@ABVQStringList@@0_N@Z 100194ae f   ngs_reads_classification:ngs_reads_classification.dll
 0001:000184b4       ?countClassified@NgsReadsClassificationUtils@U2@@SAHABV?$QMap@VQString@@I@@@Z 100194b4 f   ngs_reads_classification:ngs_reads_classification.dll
 0001:000184ba       ?update@DatabaseDelegate@LocalWorkflow@U2@@UAEXXZ 100194ba f   ngs_reads_classification:ngs_reads_classification.dll
 0001:000184c0       ?destroyEditor@QAbstractItemDelegate@@UBEXPAVQWidget@@ABVQModelIndex@@@Z 100194c0 f   Qt5Widgets:Qt5Widgets.dll
 0001:000184c6       ?drawCheck@QItemDelegate@@MBEXPAVQPainter@@ABVQStyleOptionViewItem@@ABVQRect@@W4CheckState@Qt@@@Z 100194c6 f   Qt5Widgets:Qt5Widgets.dll
 0001:000184cc       ?drawDecoration@QItemDelegate@@MBEXPAVQPainter@@ABVQStyleOptionViewItem@@ABVQRect@@ABVQPixmap@@@Z 100194cc f   Qt5Widgets:Qt5Widgets.dll
 0001:000184d2       ?drawDisplay@QItemDelegate@@MBEXPAVQPainter@@ABVQStyleOptionViewItem@@ABVQRect@@ABVQString@@@Z 100194d2 f   Qt5Widgets:Qt5Widgets.dll
 0001:000184d8       ?drawFocus@QItemDelegate@@MBEXPAVQPainter@@ABVQStyleOptionViewItem@@ABVQRect@@@Z 100194d8 f   Qt5Widgets:Qt5Widgets.dll
 0001:000184de       ?editorEvent@QItemDelegate@@MAE_NPAVQEvent@@PAVQAbstractItemModel@@ABVQStyleOptionViewItem@@ABVQModelIndex@@@Z 100194de f   Qt5Widgets:Qt5Widgets.dll
 0001:000184e4       ?eventFilter@QItemDelegate@@MAE_NPAVQObject@@PAVQEvent@@@Z 100194e4 f   Qt5Widgets:Qt5Widgets.dll
 0001:000184ea       ?helpEvent@QAbstractItemDelegate@@UAE_NPAVQHelpEvent@@PAVQAbstractItemView@@ABVQStyleOptionViewItem@@ABVQModelIndex@@@Z 100194ea f   Qt5Widgets:Qt5Widgets.dll
 0001:000184f0       ?paint@QItemDelegate@@UBEXPAVQPainter@@ABVQStyleOptionViewItem@@ABVQModelIndex@@@Z 100194f0 f   Qt5Widgets:Qt5Widgets.dll
 0001:000184f6       ?paintingRoles@QAbstractItemDelegate@@UBE?AV?$QVector@H@@XZ 100194f6 f   Qt5Widgets:Qt5Widgets.dll
 0001:000184fc       ?sizeHint@QItemDelegate@@UBE?AVQSize@@ABVQStyleOptionViewItem@@ABVQModelIndex@@@Z 100194fc f   Qt5Widgets:Qt5Widgets.dll
 0001:00018502       ?updateEditorGeometry@QItemDelegate@@UBEXPAVQWidget@@ABVQStyleOptionViewItem@@ABVQModelIndex@@@Z 10019502 f   Qt5Widgets:Qt5Widgets.dll
 0001:00018508       ?clear@QTextDocument@@UAEXXZ 10019508 f   Qt5Gui:Qt5Gui.dll
 0001:0001850e       ?createObject@QTextDocument@@MAEPAVQTextObject@@ABVQTextFormat@@@Z 1001950e f   Qt5Gui:Qt5Gui.dll
 0001:00018514       ?loadResource@QTextDocument@@MAE?AVQVariant@@HABVQUrl@@@Z 10019514 f   Qt5Gui:Qt5Gui.dll
 0001:0001851a       ??0QIcon@@QAE@ABVQString@@@Z 1001951a f   Qt5Gui:Qt5Gui.dll
 0001:00018520       ??1QIcon@@QAE@XZ           10019520 f   Qt5Gui:Qt5Gui.dll
 0001:00018526       ??4QIcon@@QAEAAV0@$$QAV0@@Z 10019526 f   Qt5Gui:Qt5Gui.dll
 0001:0001852c       ??0QScriptValue@@QAE@XZ    1001952c f   Qt5Script:Qt5Script.dll
 0001:00018532       ??1QScriptValue@@QAE@XZ    10019532 f   Qt5Script:Qt5Script.dll
 0001:00018538       ??0QScriptValue@@QAE@ABV0@@Z 10019538 f   Qt5Script:Qt5Script.dll
 0001:0001853e       ??4QScriptValue@@QAEAAV0@ABV0@@Z 1001953e f   Qt5Script:Qt5Script.dll
 0001:00018544       ?isNumber@QScriptValue@@QBE_NXZ 10019544 f   Qt5Script:Qt5Script.dll
 0001:0001854a       ?isString@QScriptValue@@QBE_NXZ 1001954a f   Qt5Script:Qt5Script.dll
 0001:00018550       ?toString@QScriptValue@@QBE?AVQString@@XZ 10019550 f   Qt5Script:Qt5Script.dll
 0001:00018556       ?toInt32@QScriptValue@@QBEHXZ 10019556 f   Qt5Script:Qt5Script.dll
 0001:0001855c       ??1QScriptEngine@@UAE@XZ   1001955c f   Qt5Script:Qt5Script.dll
 0001:00018562       ?newVariant@QScriptEngine@@QAE?AVQScriptValue@@ABVQVariant@@@Z 10019562 f   Qt5Script:Qt5Script.dll
 0001:00018568       ?attribute@QDomElement@@QBE?AVQString@@ABV2@0@Z 10019568 f   Qt5Xml:Qt5Xml.dll
 0001:0001856e       ?cast@QMetaObject@@QBEPAVQObject@@PAV2@@Z 1001956e f   Qt5Core:Qt5Core.dll
 0001:00018574       ?tr@QMetaObject@@QBE?AVQString@@PBD0H@Z 10019574 f   Qt5Core:Qt5Core.dll
 0001:0001857a       ?normalizedType@QMetaObject@@SA?AVQByteArray@@PBD@Z 1001957a f   Qt5Core:Qt5Core.dll
 0001:00018580       ??1Connection@QMetaObject@@QAE@XZ 10019580 f   Qt5Core:Qt5Core.dll
 0001:00018586       ??0QChar@@QAE@UQLatin1Char@@@Z 10019586 f   Qt5Core:Qt5Core.dll
 0001:0001858c       ??1QByteArray@@QAE@XZ      1001958c f   Qt5Core:Qt5Core.dll
 0001:00018592       ??0QString@@QAE@XZ         10019592 f   Qt5Core:Qt5Core.dll
 0001:00018598       ??0QString@@QAE@ABV0@@Z    10019598 f   Qt5Core:Qt5Core.dll
 0001:0001859e       ??1QString@@QAE@XZ         1001959e f   Qt5Core:Qt5Core.dll
 0001:000185a4       ??0QString@@QAE@$$QAV0@@Z  100195a4 f   Qt5Core:Qt5Core.dll
 0001:000185aa       ?constData@QString@@QBEPBVQChar@@XZ 100195aa f   Qt5Core:Qt5Core.dll
 0001:000185b0       ?arg@QString@@QBE?AV1@HHHVQChar@@@Z 100195b0 f   Qt5Core:Qt5Core.dll
 0001:000185b6       ?arg@QString@@QBE?AV1@ABV1@HVQChar@@@Z 100195b6 f   Qt5Core:Qt5Core.dll
 0001:000185bc       ?indexOf@QString@@QBEHABV1@HW4CaseSensitivity@Qt@@@Z 100195bc f   Qt5Core:Qt5Core.dll
 0001:000185c2       ?append@QString@@QAEAAV1@ABV1@@Z 100195c2 f   Qt5Core:Qt5Core.dll
 0001:000185c8       ?toLocal8Bit@QString@@QBE?AVQByteArray@@XZ 100195c8 f   Qt5Core:Qt5Core.dll
 0001:000185ce       ?fromUtf8@QString@@SA?AV1@PBDH@Z 100195ce f   Qt5Core:Qt5Core.dll
 0001:000185d4       ?number@QString@@SA?AV1@HH@Z 100195d4 f   Qt5Core:Qt5Core.dll
 0001:000185da       ??M@YA_NABVQString@@0@Z    100195da f   Qt5Core:Qt5Core.dll
 0001:000185e0       ?fromAscii_helper@QString@@CAPAU?$QTypedArrayData@G@@PBDH@Z 100195e0 f   Qt5Core:Qt5Core.dll
 0001:000185e6       ?detach@QListData@@QAEPAUData@1@H@Z 100195e6 f   Qt5Core:Qt5Core.dll
 0001:000185ec       ?detach_grow@QListData@@QAEPAUData@1@PAHH@Z 100195ec f   Qt5Core:Qt5Core.dll
 0001:000185f2       ?realloc@QListData@@QAEXH@Z 100195f2 f   Qt5Core:Qt5Core.dll
 0001:000185f8       ?dispose@QListData@@SAXPAUData@1@@Z 100195f8 f   Qt5Core:Qt5Core.dll
 0001:000185fe       ?append@QListData@@QAEPAPAXXZ 100195fe f   Qt5Core:Qt5Core.dll
 0001:00018604       ?registerNormalizedType@QMetaType@@SAHABVQByteArray@@P6AXPAX@ZP6APAXPBX@Z2P6APAX13@ZHV?$QFlags@W4TypeFlag@QMetaType@@@@PBUQMetaObject@@@Z 10019604 f   Qt5Core:Qt5Core.dll
 0001:0001860a       ?registerNormalizedTypedef@QMetaType@@SAHABVQByteArray@@H@Z 1001960a f   Qt5Core:Qt5Core.dll
 0001:00018610       ??1QObject@@UAE@XZ         10019610 f   Qt5Core:Qt5Core.dll
 0001:00018616       ?connect@QObject@@QBE?AVConnection@QMetaObject@@PBV1@PBD1W4ConnectionType@Qt@@@Z 10019616 f   Qt5Core:Qt5Core.dll
 0001:0001861c       ?nextNode@QMapNodeBase@@QBEPBU1@XZ 1001961c f   Qt5Core:Qt5Core.dll
 0001:00018622       ?freeNodeAndRebalance@QMapDataBase@@QAEXPAUQMapNodeBase@@@Z 10019622 f   Qt5Core:Qt5Core.dll
 0001:00018628       ?recalcMostLeftNode@QMapDataBase@@QAEXXZ 10019628 f   Qt5Core:Qt5Core.dll
 0001:0001862e       ?createNode@QMapDataBase@@QAEPAUQMapNodeBase@@HHPAU2@_N@Z 1001962e f   Qt5Core:Qt5Core.dll
 0001:00018634       ?freeTree@QMapDataBase@@QAEXPAUQMapNodeBase@@H@Z 10019634 f   Qt5Core:Qt5Core.dll
 0001:0001863a       ?createData@QMapDataBase@@SAPAU1@XZ 1001963a f   Qt5Core:Qt5Core.dll
 0001:00018640       ?freeData@QMapDataBase@@SAXPAU1@@Z 10019640 f   Qt5Core:Qt5Core.dll
 0001:00018646       ?write@QIODevice@@QAE_JABVQByteArray@@@Z 10019646 f   Qt5Core:Qt5Core.dll
 0001:0001864c       ?errorString@QIODevice@@QBE?AVQString@@XZ 1001964c f   Qt5Core:Qt5Core.dll
 0001:00018652       ?QStringList_join@QtPrivate@@YA?AVQString@@PBVQStringList@@PBVQChar@@H@Z 10019652 f   Qt5Core:Qt5Core.dll
 0001:00018658       ??0QVariant@@QAE@XZ        10019658 f   Qt5Core:Qt5Core.dll
 0001:0001865e       ??1QVariant@@QAE@XZ        1001965e f   Qt5Core:Qt5Core.dll
 0001:00018664       ??0QVariant@@QAE@ABV0@@Z   10019664 f   Qt5Core:Qt5Core.dll
 0001:0001866a       ??0QVariant@@QAE@H@Z       1001966a f   Qt5Core:Qt5Core.dll
 0001:00018670       ??0QVariant@@QAE@ABVQString@@@Z 10019670 f   Qt5Core:Qt5Core.dll
 0001:00018676       ??0QVariant@@QAE@ABV?$QMap@VQString@@VQVariant@@@@@Z 10019676 f   Qt5Core:Qt5Core.dll
 0001:0001867c       ??4QVariant@@QAEAAV0@ABV0@@Z 1001967c f   Qt5Core:Qt5Core.dll
 0001:00018682       ??4QVariant@@QAEAAV0@$$QAV0@@Z 10019682 f   Qt5Core:Qt5Core.dll
 0001:00018688       ?userType@QVariant@@QBEHXZ 10019688 f   Qt5Core:Qt5Core.dll
 0001:0001868e       ?constData@QVariant@@QBEPBXXZ 1001968e f   Qt5Core:Qt5Core.dll
 0001:00018694       ?convert@QVariant@@QBE_NHPAX@Z 10019694 f   Qt5Core:Qt5Core.dll
 0001:0001869a       ?close@QFileDevice@@UAEXXZ 1001969a f   Qt5Core:Qt5Core.dll
 0001:000186a0       ??0QFile@@QAE@ABVQString@@@Z 100196a0 f   Qt5Core:Qt5Core.dll
 0001:000186a6       ??1QFile@@UAE@XZ           100196a6 f   Qt5Core:Qt5Core.dll
 0001:000186ac       ?open@QFile@@UAE_NV?$QFlags@W4OpenModeFlag@QIODevice@@@@@Z 100196ac f   Qt5Core:Qt5Core.dll
 0001:000186b2       ??0QDir@@QAE@ABVQString@@@Z 100196b2 f   Qt5Core:Qt5Core.dll
 0001:000186b8       ??1QDir@@QAE@XZ            100196b8 f   Qt5Core:Qt5Core.dll
 0001:000186be       ?mkpath@QDir@@QBE_NABVQString@@@Z 100196be f   Qt5Core:Qt5Core.dll
 0001:000186c4       ?translate@QCoreApplication@@SA?AVQString@@PBD00H@Z 100196c4 f   Qt5Core:Qt5Core.dll
 0001:000186ca       ?childEvent@QObject@@MAEXPAVQChildEvent@@@Z 100196ca f   Qt5Core:Qt5Core.dll
 0001:000186d0       ?connectNotify@QObject@@MAEXABVQMetaMethod@@@Z 100196d0 f   Qt5Core:Qt5Core.dll
 0001:000186d6       ?customEvent@QObject@@MAEXPAVQEvent@@@Z 100196d6 f   Qt5Core:Qt5Core.dll
 0001:000186dc       ?disconnectNotify@QObject@@MAEXABVQMetaMethod@@@Z 100196dc f   Qt5Core:Qt5Core.dll
 0001:000186e2       ?event@QObject@@UAE_NPAVQEvent@@@Z 100196e2 f   Qt5Core:Qt5Core.dll
 0001:000186e8       ?eventFilter@QObject@@UAE_NPAV1@PAVQEvent@@@Z 100196e8 f   Qt5Core:Qt5Core.dll
 0001:000186ee       ?timerEvent@QObject@@MAEXPAVQTimerEvent@@@Z 100196ee f   Qt5Core:Qt5Core.dll
 0001:000186f4       ?qstrcmp@@YAHABVQByteArray@@PBD@Z 100196f4 f   Qt5Core:Qt5Core.dll
 0001:000186fa       ??0QByteArray@@QAE@PBDH@Z  100196fa f   Qt5Core:Qt5Core.dll
 0001:00018700       ??4QByteArray@@QAEAAV0@$$QAV0@@Z 10019700 f   Qt5Core:Qt5Core.dll
 0001:00018706       ?startsWith@QByteArray@@QBE_NABV1@@Z 10019706 f   Qt5Core:Qt5Core.dll
 0001:0001870c       ?endsWith@QByteArray@@QBE_NABV1@@Z 1001970c f   Qt5Core:Qt5Core.dll
 0001:00018712       ?trimmed@QByteArray@@QBE?AV1@XZ 10019712 f   Qt5Core:Qt5Core.dll
 0001:00018718       ?split@QByteArray@@QBE?AV?$QList@VQByteArray@@@@D@Z 10019718 f   Qt5Core:Qt5Core.dll
 0001:0001871e       ?toUInt@QByteArray@@QBEIPA_NH@Z 1001971e f   Qt5Core:Qt5Core.dll
 0001:00018724       ??4QString@@QAEAAV0@ABV0@@Z 10019724 f   Qt5Core:Qt5Core.dll
 0001:0001872a       ??4QString@@QAEAAV0@$$QAV0@@Z 1001972a f   Qt5Core:Qt5Core.dll
 0001:00018730       ?endsWith@QString@@QBE_NABV1@W4CaseSensitivity@Qt@@@Z 10019730 f   Qt5Core:Qt5Core.dll
 0001:00018736       ?toLower@QString@@QBE?AV1@XZ 10019736 f   Qt5Core:Qt5Core.dll
 0001:0001873c       ?compare@QString@@QBEHABV1@W4CaseSensitivity@Qt@@@Z 1001973c f   Qt5Core:Qt5Core.dll
 0001:00018742       ??8@YA_NABVQString@@0@Z    10019742 f   Qt5Core:Qt5Core.dll
 0001:00018748       ??0QString@@QAE@ABVQByteArray@@@Z 10019748 f   Qt5Core:Qt5Core.dll
 0001:0001874e       ??YQString@@QAEAAV0@PBD@Z  1001974e f   Qt5Core:Qt5Core.dll
 0001:00018754       ?hasRegisteredConverterFunction@QMetaType@@SA_NHH@Z 10019754 f   Qt5Core:Qt5Core.dll
 0001:0001875a       ?registerConverterFunction@QMetaType@@SA_NPBUAbstractConverterFunction@QtPrivate@@HH@Z 1001975a f   Qt5Core:Qt5Core.dll
 0001:00018760       ?unregisterConverterFunction@QMetaType@@SAXHH@Z 10019760 f   Qt5Core:Qt5Core.dll
 0001:00018766       ?readLine@QIODevice@@QAE?AVQByteArray@@_J@Z 10019766 f   Qt5Core:Qt5Core.dll
 0001:0001876c       ?free_helper@QHashData@@QAEXP6AXPAUNode@1@@Z@Z 1001976c f   Qt5Core:Qt5Core.dll
 0001:00018772       ??0QFileInfo@@QAE@ABVQString@@@Z 10019772 f   Qt5Core:Qt5Core.dll
 0001:00018778       ??1QFileInfo@@QAE@XZ       10019778 f   Qt5Core:Qt5Core.dll
 0001:0001877e       ?exists@QFileInfo@@QBE_NXZ 1001977e f   Qt5Core:Qt5Core.dll
 0001:00018784       ?completeBaseName@QFileInfo@@QBE?AVQString@@XZ 10019784 f   Qt5Core:Qt5Core.dll
 0001:0001878a       ?dir@QFileInfo@@QBE?AVQDir@@XZ 1001978a f   Qt5Core:Qt5Core.dll
 0001:00018790       ?previousNode@QMapNodeBase@@QBEPBU1@XZ 10019790 f   Qt5Core:Qt5Core.dll
 0001:00018796       ??0QVariant@@QAE@HPBXI@Z   10019796 f   Qt5Core:Qt5Core.dll
 0001:0001879c       ??0QVariant@@QAE@_N@Z      1001979c f   Qt5Core:Qt5Core.dll
 0001:000187a2       ??0QVariant@@QAE@PBD@Z     100197a2 f   Qt5Core:Qt5Core.dll
 0001:000187a8       ?toString@QVariant@@QBE?AVQString@@XZ 100197a8 f   Qt5Core:Qt5Core.dll
 0001:000187ae       ?toMap@QVariant@@QBE?AV?$QMap@VQString@@VQVariant@@@@XZ 100197ae f   Qt5Core:Qt5Core.dll
 0001:000187b4       ?path@QDir@@QBE?AVQString@@XZ 100197b4 f   Qt5Core:Qt5Core.dll
 0001:000187ba       ?entryInfoList@QDir@@QBE?AV?$QList@VQFileInfo@@@@ABVQStringList@@V?$QFlags@W4Filter@QDir@@@@V?$QFlags@W4SortFlag@QDir@@@@@Z 100197ba f   Qt5Core:Qt5Core.dll
 0001:000187c0       ??4QString@@QAEAAV0@PBD@Z  100197c0 f   Qt5Core:Qt5Core.dll
 0001:000187c6       ??0QRegExp@@QAE@ABVQString@@W4CaseSensitivity@Qt@@W4PatternSyntax@0@@Z 100197c6 f   Qt5Core:Qt5Core.dll
 0001:000187cc       ??1QRegExp@@QAE@XZ         100197cc f   Qt5Core:Qt5Core.dll
 0001:000187d2       ??4QRegExp@@QAEAAV0@$$QAV0@@Z 100197d2 f   Qt5Core:Qt5Core.dll
 0001:000187d8       ?tr@QObject@@SA?AVQString@@PBD0H@Z 100197d8 f   Qt5Core:Qt5Core.dll
 0001:000187de       ??0QObject@@QAE@PAV0@@Z    100197de f   Qt5Core:Qt5Core.dll
 0001:000187e4       ?metaObject@QObject@@UBEPBUQMetaObject@@XZ 100197e4 f   Qt5Core:Qt5Core.dll
 0001:000187ea       ?qt_metacall@QObject@@UAEHW4Call@QMetaObject@@HPAPAX@Z 100197ea f   Qt5Core:Qt5Core.dll
 0001:000187f0       ?qt_metacast@QObject@@UAEPAXPBD@Z 100197f0 f   Qt5Core:Qt5Core.dll
 0001:000187f6       ?replace@QString@@QAEAAV1@ABV1@0W4CaseSensitivity@Qt@@@Z 100197f6 f   Qt5Core:Qt5Core.dll
 0001:000187fc       ?split@QString@@QBE?AVQStringList@@ABV1@W4SplitBehavior@1@W4CaseSensitivity@Qt@@@Z 100197fc f   Qt5Core:Qt5Core.dll
 0001:00018802       ?fileName@QFile@@UBE?AVQString@@XZ 10019802 f   Qt5Core:Qt5Core.dll
 0001:00018808       ?exists@QFileInfo@@SA_NABVQString@@@Z 10019808 f   Qt5Core:Qt5Core.dll
 0001:0001880e       ?isDir@QFileInfo@@QBE_NXZ  1001980e f   Qt5Core:Qt5Core.dll
 0001:00018814       ??0QTextStream@@QAE@PAVQIODevice@@@Z 10019814 f   Qt5Core:Qt5Core.dll
 0001:0001881a       ??1QTextStream@@UAE@XZ     1001981a f   Qt5Core:Qt5Core.dll
 0001:00018820       ?atEnd@QTextStream@@QBE_NXZ 10019820 f   Qt5Core:Qt5Core.dll
 0001:00018826       ?readLine@QTextStream@@QAE?AVQString@@_J@Z 10019826 f   Qt5Core:Qt5Core.dll
 0001:0001882c       ??0QByteArray@@QAE@XZ      1001982c f   Qt5Core:Qt5Core.dll
 0001:00018832       ?reserve@QByteArray@@QAEXH@Z 10019832 f   Qt5Core:Qt5Core.dll
 0001:00018838       ?append@QByteArray@@QAEAAV1@D@Z 10019838 f   Qt5Core:Qt5Core.dll
 0001:0001883e       ?append@QByteArray@@QAEAAV1@PBD@Z 1001983e f   Qt5Core:Qt5Core.dll
 0001:00018844       ?className@QMetaObject@@QBEPBDXZ 10019844 f   Qt5Core:Qt5Core.dll
 0001:0001884a       ?dynamicMetaObject@QObjectData@@QBEPAUQMetaObject@@XZ 1001984a f   Qt5Core:Qt5Core.dll
 0001:00018850       ?_Xbad_alloc@std@@YAXXZ    10019850 f   msvcprt:MSVCP120.dll
 0001:00018856       ?_Xlength_error@std@@YAXPBD@Z 10019856 f   msvcprt:MSVCP120.dll
 0001:0001885c       ?_Xout_of_range@std@@YAXPBD@Z 1001985c f   msvcprt:MSVCP120.dll
 0001:00018862       ?_Syserror_map@std@@YAPBDH@Z 10019862 f   msvcprt:MSVCP120.dll
 0001:00018868       ?_Winerror_map@std@@YAPBDH@Z 10019868 f   msvcprt:MSVCP120.dll
 0001:0001886e       __purecall                 1001986e f   MSVCRT:MSVCR120.dll
 0001:00018874       ??2@YAPAXI@Z               10019874 f   MSVCRT:MSVCR120.dll
 0001:0001887a       ??3@YAXPAX@Z               1001987a f   MSVCRT:MSVCR120.dll
 0001:00018880       ___atonexitinit            10019880 f   MSVCRT:atonexit.obj
 0001:000188bc       __onexit                   100198bc f   MSVCRT:atonexit.obj
 0001:00018965       _atexit                    10019965 f   MSVCRT:atonexit.obj
 0001:0001897a       _memmove                   1001997a f   MSVCRT:MSVCR120.dll
 0001:00018980       __hypot                    10019980 f   MSVCRT:MSVCR120.dll
 0001:00018986       @__security_check_cookie@4 10019986 f   MSVCRT:secchk.obj
 0001:00018996       __CxxThrowException@8      10019996 f   MSVCRT:MSVCR120.dll
 0001:0001899c       ___CxxFrameHandler3        1001999c f   MSVCRT:MSVCR120.dll
 0001:000189a2       _memcpy                    100199a2 f   MSVCRT:MSVCR120.dll
 0001:000189a8       ??0type_info@@AAE@ABV0@@Z  100199a8 f   MSVCRT:ti_inst.obj
 0001:000189b3       ??4type_info@@AAEAAV0@ABV0@@Z 100199b3 f   MSVCRT:ti_inst.obj
 0001:000189b8       ??_Etype_info@@UAEPAXI@Z   100199b8 f i MSVCRT:ti_inst.obj
 0001:00018a10       ??_M@YGXPAXIHP6EX0@Z@Z     10019a10 f   MSVCRT:ehvecdtr.obj
 0001:00018a98       ?__ArrayUnwind@@YGXPAXIHP6EX0@Z@Z 10019a98 f   MSVCRT:ehvecdtr.obj
 0001:00018b42       _NtCurrentTeb              10019b42 f i MSVCRT:crtdll.obj
 0001:00018b49       __CRT_INIT@12              10019b49 f   MSVCRT:crtdll.obj
 0001:00018d40       __DllMainCRTStartup@12     10019d40 f   MSVCRT:crtdll.obj
 0001:00018e96       __lock                     10019e96 f   MSVCRT:MSVCR120.dll
 0001:00018e9c       __unlock                   10019e9c f   MSVCRT:MSVCR120.dll
 0001:00018ea2       __calloc_crt               10019ea2 f   MSVCRT:MSVCR120.dll
 0001:00018ea8       ___dllonexit               10019ea8 f   MSVCRT:MSVCR120.dll
 0001:00018eb0       __SEH_prolog4              10019eb0 f   MSVCRT:sehprolg4.obj
 0001:00018ef5       __SEH_epilog4              10019ef5 f   MSVCRT:sehprolg4.obj
 0001:00018f09       __except_handler4          10019f09 f   MSVCRT:chandler4gs.obj
 0001:00018f2c       ___raise_securityfailure   10019f2c f   MSVCRT:gs_report.obj
 0001:00018f6a       ___report_gsfailure        10019f6a f   MSVCRT:gs_report.obj
 0001:00019065       ___report_rangecheckfailure 1001a065 f   MSVCRT:gs_report.obj
 0001:00019071       ___report_securityfailure  1001a071 f   MSVCRT:gs_report.obj
 0001:00019141       ___report_securityfailureEx 1001a141 f   MSVCRT:gs_report.obj
 0001:00019258       ??1type_info@@UAE@XZ       1001a258 f   MSVCRT:MSVCR120.dll
 0001:0001925e       ?terminate@@YAXXZ          1001a25e f   MSVCRT:MSVCR120.dll
 0001:00019264       ___CppXcptFilter           1001a264 f   MSVCRT:MSVCR120.dll
 0001:0001926a       __amsg_exit                1001a26a f   MSVCRT:MSVCR120.dll
 0001:00019270       __FindPESection            1001a270 f   MSVCRT:pesect.obj
 0001:000192c0       __IsNonwritableInCurrentImage 1001a2c0 f   MSVCRT:pesect.obj
 0001:00019380       __ValidateImageBase        1001a380 f   MSVCRT:pesect.obj
 0001:000193b2       _free                      1001a3b2 f   MSVCRT:MSVCR120.dll
 0001:000193b8       ___security_init_cookie    1001a3b8 f   MSVCRT:gs_support.obj
 0001:00019454       _DllMain@12                1001a454 f   MSVCRT:dllmain.obj
 0001:00019476       __malloc_crt               1001a476 f   MSVCRT:MSVCR120.dll
 0001:0001947c       __RTC_Initialize           1001a47c f   MSVCRT:initsect.obj
 0001:0001949c       __RTC_Terminate            1001a49c f   MSVCRT:initsect.obj
 0001:000194bc       __initterm                 1001a4bc f   MSVCRT:MSVCR120.dll
 0001:000194c2       __initterm_e               1001a4c2 f   MSVCRT:MSVCR120.dll
 0001:000194c8       ___clean_type_info_names   1001a4c8 f   MSVCRT:tncleanup.obj
 0001:000194d4       __except_handler4_common   1001a4d4 f   MSVCRT:MSVCR120.dll
 0001:000194da       __crt_debugger_hook        1001a4da f   MSVCRT:MSVCR120.dll
 0001:000194e0       ___crtUnhandledException   1001a4e0 f   MSVCRT:MSVCR120.dll
 0001:000194e6       ___crtTerminateProcess     1001a4e6 f   MSVCRT:MSVCR120.dll
 0001:000194ec       ___clean_type_info_names_internal 1001a4ec f   MSVCRT:MSVCR120.dll
 0001:000194f2       _EncodePointer@4           1001a4f2 f   kernel32:KERNEL32.dll
 0001:000194f8       _DecodePointer@4           1001a4f8 f   kernel32:KERNEL32.dll
 0001:000194fe       _IsDebuggerPresent@0       1001a4fe f   kernel32:KERNEL32.dll
 0001:00019504       _IsProcessorFeaturePresent@4 1001a504 f   kernel32:KERNEL32.dll
 0001:0001950a       _QueryPerformanceCounter@4 1001a50a f   kernel32:KERNEL32.dll
 0001:00019510       _GetCurrentProcessId@0     1001a510 f   kernel32:KERNEL32.dll
 0001:00019516       _GetCurrentThreadId@0      1001a516 f   kernel32:KERNEL32.dll
 0001:0001951c       _GetSystemTimeAsFileTime@4 1001a51c f   kernel32:KERNEL32.dll
 0001:00019522       _DisableThreadLibraryCalls@4 1001a522 f   kernel32:KERNEL32.dll
 0001:0001d9c0       ??__Ff@?4??registerConverter@?$AssociativeValueTypeIsMetaType@V?$QMap@VQString@@I@@$00@QtPrivate@@SA_NH@Z@YAXXZ 1001e9c0 f i ClarkClassifyWorker.obj
 0002:00000000       __imp__GetSystemTimeAsFileTime@4 10020000     kernel32:KERNEL32.dll
 0002:00000004       __imp__GetCurrentThreadId@0 10020004     kernel32:KERNEL32.dll
 0002:00000008       __imp__GetCurrentProcessId@0 10020008     kernel32:KERNEL32.dll
 0002:0000000c       __imp__QueryPerformanceCounter@4 1002000c     kernel32:KERNEL32.dll
 0002:00000010       __imp__IsProcessorFeaturePresent@4 10020010     kernel32:KERNEL32.dll
 0002:00000014       __imp__EncodePointer@4     10020014     kernel32:KERNEL32.dll
 0002:00000018       __imp__DecodePointer@4     10020018     kernel32:KERNEL32.dll
 0002:0000001c       __imp__IsDebuggerPresent@0 1002001c     kernel32:KERNEL32.dll
 0002:00000020       __imp__DisableThreadLibraryCalls@4 10020020     kernel32:KERNEL32.dll
 0002:00000024       \177KERNEL32_NULL_THUNK_DATA 10020024     kernel32:KERNEL32.dll
 0002:00000028       __imp_?_Syserror_map@std@@YAPBDH@Z 10020028     msvcprt:MSVCP120.dll
 0002:0000002c       __imp_?_Xout_of_range@std@@YAXPBD@Z 1002002c     msvcprt:MSVCP120.dll
 0002:00000030       __imp_?_Xlength_error@std@@YAXPBD@Z 10020030     msvcprt:MSVCP120.dll
 0002:00000034       __imp_?_Winerror_map@std@@YAPBDH@Z 10020034     msvcprt:MSVCP120.dll
 0002:00000038       __imp_?_Xbad_alloc@std@@YAXXZ 10020038     msvcprt:MSVCP120.dll
 0002:0000003c       \177MSVCP120_NULL_THUNK_DATA 1002003c     msvcprt:MSVCP120.dll
 0002:00000040       __imp___purecall           10020040     MSVCRT:MSVCR120.dll
 0002:00000044       __imp_??3@YAXPAX@Z         10020044     MSVCRT:MSVCR120.dll
 0002:00000048       __imp__memmove             10020048     MSVCRT:MSVCR120.dll
 0002:0000004c       __imp___hypot              1002004c     MSVCRT:MSVCR120.dll
 0002:00000050       __imp___CxxThrowException@8 10020050     MSVCRT:MSVCR120.dll
 0002:00000054       __imp____CxxFrameHandler3  10020054     MSVCRT:MSVCR120.dll
 0002:00000058       __imp__memcpy              10020058     MSVCRT:MSVCR120.dll
 0002:0000005c       __imp___lock               1002005c     MSVCRT:MSVCR120.dll
 0002:00000060       __imp___unlock             10020060     MSVCRT:MSVCR120.dll
 0002:00000064       __imp___calloc_crt         10020064     MSVCRT:MSVCR120.dll
 0002:00000068       __imp____dllonexit         10020068     MSVCRT:MSVCR120.dll
 0002:0000006c       __imp___onexit             1002006c     MSVCRT:MSVCR120.dll
 0002:00000070       __imp_??1type_info@@UAE@XZ 10020070     MSVCRT:MSVCR120.dll
 0002:00000074       __imp_?terminate@@YAXXZ    10020074     MSVCRT:MSVCR120.dll
 0002:00000078       __imp____CppXcptFilter     10020078     MSVCRT:MSVCR120.dll
 0002:0000007c       __imp___amsg_exit          1002007c     MSVCRT:MSVCR120.dll
 0002:00000080       __imp__free                10020080     MSVCRT:MSVCR120.dll
 0002:00000084       __imp___malloc_crt         10020084     MSVCRT:MSVCR120.dll
 0002:00000088       __imp___initterm           10020088     MSVCRT:MSVCR120.dll
 0002:0000008c       __imp___initterm_e         1002008c     MSVCRT:MSVCR120.dll
 0002:00000090       __imp___except_handler4_common 10020090     MSVCRT:MSVCR120.dll
 0002:00000094       __imp___crt_debugger_hook  10020094     MSVCRT:MSVCR120.dll
 0002:00000098       __imp____crtUnhandledException 10020098     MSVCRT:MSVCR120.dll
 0002:0000009c       __imp____crtTerminateProcess 1002009c     MSVCRT:MSVCR120.dll
 0002:000000a0       __imp____clean_type_info_names_internal 100200a0     MSVCRT:MSVCR120.dll
 0002:000000a4       __imp_??2@YAPAXI@Z         100200a4     MSVCRT:MSVCR120.dll
 0002:000000a8       \177MSVCR120_NULL_THUNK_DATA 100200a8     MSVCRT:MSVCR120.dll
 0002:000000ac       __imp_??0QVariant@@QAE@H@Z 100200ac     Qt5Core:Qt5Core.dll
 0002:000000b0       __imp_??0QVariant@@QAE@ABVQString@@@Z 100200b0     Qt5Core:Qt5Core.dll
 0002:000000b4       __imp_??0QVariant@@QAE@ABV?$QMap@VQString@@VQVariant@@@@@Z 100200b4     Qt5Core:Qt5Core.dll
 0002:000000b8       __imp_??4QVariant@@QAEAAV0@ABV0@@Z 100200b8     Qt5Core:Qt5Core.dll
 0002:000000bc       __imp_??4QVariant@@QAEAAV0@$$QAV0@@Z 100200bc     Qt5Core:Qt5Core.dll
 0002:000000c0       __imp_?userType@QVariant@@QBEHXZ 100200c0     Qt5Core:Qt5Core.dll
 0002:000000c4       __imp_?constData@QVariant@@QBEPBXXZ 100200c4     Qt5Core:Qt5Core.dll
 0002:000000c8       __imp_?convert@QVariant@@QBE_NHPAX@Z 100200c8     Qt5Core:Qt5Core.dll
 0002:000000cc       __imp_?close@QFileDevice@@UAEXXZ 100200cc     Qt5Core:Qt5Core.dll
 0002:000000d0       __imp_??0QFile@@QAE@ABVQString@@@Z 100200d0     Qt5Core:Qt5Core.dll
 0002:000000d4       __imp_??1QFile@@UAE@XZ     100200d4     Qt5Core:Qt5Core.dll
 0002:000000d8       __imp_?open@QFile@@UAE_NV?$QFlags@W4OpenModeFlag@QIODevice@@@@@Z 100200d8     Qt5Core:Qt5Core.dll
 0002:000000dc       __imp_??0QDir@@QAE@ABVQString@@@Z 100200dc     Qt5Core:Qt5Core.dll
 0002:000000e0       __imp_??1QDir@@QAE@XZ      100200e0     Qt5Core:Qt5Core.dll
 0002:000000e4       __imp_?mkpath@QDir@@QBE_NABVQString@@@Z 100200e4     Qt5Core:Qt5Core.dll
 0002:000000e8       __imp_?translate@QCoreApplication@@SA?AVQString@@PBD00H@Z 100200e8     Qt5Core:Qt5Core.dll
 0002:000000ec       __imp_?childEvent@QObject@@MAEXPAVQChildEvent@@@Z 100200ec     Qt5Core:Qt5Core.dll
 0002:000000f0       __imp_?connectNotify@QObject@@MAEXABVQMetaMethod@@@Z 100200f0     Qt5Core:Qt5Core.dll
 0002:000000f4       __imp_?customEvent@QObject@@MAEXPAVQEvent@@@Z 100200f4     Qt5Core:Qt5Core.dll
 0002:000000f8       __imp_?disconnectNotify@QObject@@MAEXABVQMetaMethod@@@Z 100200f8     Qt5Core:Qt5Core.dll
 0002:000000fc       __imp_?event@QObject@@UAE_NPAVQEvent@@@Z 100200fc     Qt5Core:Qt5Core.dll
 0002:00000100       __imp_?eventFilter@QObject@@UAE_NPAV1@PAVQEvent@@@Z 10020100     Qt5Core:Qt5Core.dll
 0002:00000104       __imp_?timerEvent@QObject@@MAEXPAVQTimerEvent@@@Z 10020104     Qt5Core:Qt5Core.dll
 0002:00000108       __imp_?shared_null@QListData@@2UData@1@B 10020108     Qt5Core:Qt5Core.dll
 0002:0000010c       __imp_?shared_null@QMapDataBase@@2U1@B 1002010c     Qt5Core:Qt5Core.dll
 0002:00000110       __imp_?qstrcmp@@YAHABVQByteArray@@PBD@Z 10020110     Qt5Core:Qt5Core.dll
 0002:00000114       __imp_??0QByteArray@@QAE@PBDH@Z 10020114     Qt5Core:Qt5Core.dll
 0002:00000118       __imp_??4QByteArray@@QAEAAV0@$$QAV0@@Z 10020118     Qt5Core:Qt5Core.dll
 0002:0000011c       __imp_?startsWith@QByteArray@@QBE_NABV1@@Z 1002011c     Qt5Core:Qt5Core.dll
 0002:00000120       __imp_?endsWith@QByteArray@@QBE_NABV1@@Z 10020120     Qt5Core:Qt5Core.dll
 0002:00000124       __imp_?trimmed@QByteArray@@QBE?AV1@XZ 10020124     Qt5Core:Qt5Core.dll
 0002:00000128       __imp_?split@QByteArray@@QBE?AV?$QList@VQByteArray@@@@D@Z 10020128     Qt5Core:Qt5Core.dll
 0002:0000012c       __imp_?toUInt@QByteArray@@QBEIPA_NH@Z 1002012c     Qt5Core:Qt5Core.dll
 0002:00000130       __imp_??4QString@@QAEAAV0@ABV0@@Z 10020130     Qt5Core:Qt5Core.dll
 0002:00000134       __imp_??4QString@@QAEAAV0@$$QAV0@@Z 10020134     Qt5Core:Qt5Core.dll
 0002:00000138       __imp_?endsWith@QString@@QBE_NABV1@W4CaseSensitivity@Qt@@@Z 10020138     Qt5Core:Qt5Core.dll
 0002:0000013c       __imp_?append@QString@@QAEAAV1@ABV1@@Z 1002013c     Qt5Core:Qt5Core.dll
 0002:00000140       __imp_?compare@QString@@QBEHABV1@W4CaseSensitivity@Qt@@@Z 10020140     Qt5Core:Qt5Core.dll
 0002:00000144       __imp_??8@YA_NABVQString@@0@Z 10020144     Qt5Core:Qt5Core.dll
 0002:00000148       __imp_??0QString@@QAE@ABVQByteArray@@@Z 10020148     Qt5Core:Qt5Core.dll
 0002:0000014c       __imp_??YQString@@QAEAAV0@PBD@Z 1002014c     Qt5Core:Qt5Core.dll
 0002:00000150       __imp_??0QVariant@@QAE@ABV0@@Z 10020150     Qt5Core:Qt5Core.dll
 0002:00000154       __imp_?registerConverterFunction@QMetaType@@SA_NPBUAbstractConverterFunction@QtPrivate@@HH@Z 10020154     Qt5Core:Qt5Core.dll
 0002:00000158       __imp_?unregisterConverterFunction@QMetaType@@SAXHH@Z 10020158     Qt5Core:Qt5Core.dll
 0002:0000015c       __imp_?readLine@QIODevice@@QAE?AVQByteArray@@_J@Z 1002015c     Qt5Core:Qt5Core.dll
 0002:00000160       __imp_?free_helper@QHashData@@QAEXP6AXPAUNode@1@@Z@Z 10020160     Qt5Core:Qt5Core.dll
 0002:00000164       __imp_??0QFileInfo@@QAE@ABVQString@@@Z 10020164     Qt5Core:Qt5Core.dll
 0002:00000168       __imp_??1QFileInfo@@QAE@XZ 10020168     Qt5Core:Qt5Core.dll
 0002:0000016c       __imp_?exists@QFileInfo@@QBE_NXZ 1002016c     Qt5Core:Qt5Core.dll
 0002:00000170       __imp_?completeBaseName@QFileInfo@@QBE?AVQString@@XZ 10020170     Qt5Core:Qt5Core.dll
 0002:00000174       __imp_?dir@QFileInfo@@QBE?AVQDir@@XZ 10020174     Qt5Core:Qt5Core.dll
 0002:00000178       __imp_?previousNode@QMapNodeBase@@QBEPBU1@XZ 10020178     Qt5Core:Qt5Core.dll
 0002:0000017c       __imp_??0QVariant@@QAE@HPBXI@Z 1002017c     Qt5Core:Qt5Core.dll
 0002:00000180       __imp_??0QVariant@@QAE@_N@Z 10020180     Qt5Core:Qt5Core.dll
 0002:00000184       __imp_??0QVariant@@QAE@PBD@Z 10020184     Qt5Core:Qt5Core.dll
 0002:00000188       __imp_?toString@QVariant@@QBE?AVQString@@XZ 10020188     Qt5Core:Qt5Core.dll
 0002:0000018c       __imp_?toMap@QVariant@@QBE?AV?$QMap@VQString@@VQVariant@@@@XZ 1002018c     Qt5Core:Qt5Core.dll
 0002:00000190       __imp_?path@QDir@@QBE?AVQString@@XZ 10020190     Qt5Core:Qt5Core.dll
 0002:00000194       __imp_?entryInfoList@QDir@@QBE?AV?$QList@VQFileInfo@@@@ABVQStringList@@V?$QFlags@W4Filter@QDir@@@@V?$QFlags@W4SortFlag@QDir@@@@@Z 10020194     Qt5Core:Qt5Core.dll
 0002:00000198       __imp_?shared_null@QHashData@@2U1@B 10020198     Qt5Core:Qt5Core.dll
 0002:0000019c       __imp_??4QString@@QAEAAV0@PBD@Z 1002019c     Qt5Core:Qt5Core.dll
 0002:000001a0       __imp_??0QRegExp@@QAE@ABVQString@@W4CaseSensitivity@Qt@@W4PatternSyntax@0@@Z 100201a0     Qt5Core:Qt5Core.dll
 0002:000001a4       __imp_??1QRegExp@@QAE@XZ   100201a4     Qt5Core:Qt5Core.dll
 0002:000001a8       __imp_??4QRegExp@@QAEAAV0@$$QAV0@@Z 100201a8     Qt5Core:Qt5Core.dll
 0002:000001ac       __imp_?tr@QObject@@SA?AVQString@@PBD0H@Z 100201ac     Qt5Core:Qt5Core.dll
 0002:000001b0       __imp_??0QObject@@QAE@PAV0@@Z 100201b0     Qt5Core:Qt5Core.dll
 0002:000001b4       __imp_?metaObject@QObject@@UBEPBUQMetaObject@@XZ 100201b4     Qt5Core:Qt5Core.dll
 0002:000001b8       __imp_?qt_metacall@QObject@@UAEHW4Call@QMetaObject@@HPAPAX@Z 100201b8     Qt5Core:Qt5Core.dll
 0002:000001bc       __imp_?qt_metacast@QObject@@UAEPAXPBD@Z 100201bc     Qt5Core:Qt5Core.dll
 0002:000001c0       __imp_?replace@QString@@QAEAAV1@ABV1@0W4CaseSensitivity@Qt@@@Z 100201c0     Qt5Core:Qt5Core.dll
 0002:000001c4       __imp_?split@QString@@QBE?AVQStringList@@ABV1@W4SplitBehavior@1@W4CaseSensitivity@Qt@@@Z 100201c4     Qt5Core:Qt5Core.dll
 0002:000001c8       __imp_?fileName@QFile@@UBE?AVQString@@XZ 100201c8     Qt5Core:Qt5Core.dll
 0002:000001cc       __imp_?exists@QFileInfo@@SA_NABVQString@@@Z 100201cc     Qt5Core:Qt5Core.dll
 0002:000001d0       __imp_?isDir@QFileInfo@@QBE_NXZ 100201d0     Qt5Core:Qt5Core.dll
 0002:000001d4       __imp_?indexOf@QString@@QBEHABV1@HW4CaseSensitivity@Qt@@@Z 100201d4     Qt5Core:Qt5Core.dll
 0002:000001d8       __imp_?arg@QString@@QBE?AV1@ABV1@HVQChar@@@Z 100201d8     Qt5Core:Qt5Core.dll
 0002:000001dc       __imp_?arg@QString@@QBE?AV1@HHHVQChar@@@Z 100201dc     Qt5Core:Qt5Core.dll
 0002:000001e0       __imp_?constData@QString@@QBEPBVQChar@@XZ 100201e0     Qt5Core:Qt5Core.dll
 0002:000001e4       __imp_??0QString@@QAE@$$QAV0@@Z 100201e4     Qt5Core:Qt5Core.dll
 0002:000001e8       __imp_??1QString@@QAE@XZ   100201e8     Qt5Core:Qt5Core.dll
 0002:000001ec       __imp_??0QString@@QAE@ABV0@@Z 100201ec     Qt5Core:Qt5Core.dll
 0002:000001f0       __imp_??0QString@@QAE@XZ   100201f0     Qt5Core:Qt5Core.dll
 0002:000001f4       __imp_??1QByteArray@@QAE@XZ 100201f4     Qt5Core:Qt5Core.dll
 0002:000001f8       __imp_??1QVariant@@QAE@XZ  100201f8     Qt5Core:Qt5Core.dll
 0002:000001fc       __imp_??0QVariant@@QAE@XZ  100201fc     Qt5Core:Qt5Core.dll
 0002:00000200       __imp_?QStringList_join@QtPrivate@@YA?AVQString@@PBVQStringList@@PBVQChar@@H@Z 10020200     Qt5Core:Qt5Core.dll
 0002:00000204       __imp_?errorString@QIODevice@@QBE?AVQString@@XZ 10020204     Qt5Core:Qt5Core.dll
 0002:00000208       __imp_?write@QIODevice@@QAE_JABVQByteArray@@@Z 10020208     Qt5Core:Qt5Core.dll
 0002:0000020c       __imp_?freeData@QMapDataBase@@SAXPAU1@@Z 1002020c     Qt5Core:Qt5Core.dll
 0002:00000210       __imp_?createData@QMapDataBase@@SAPAU1@XZ 10020210     Qt5Core:Qt5Core.dll
 0002:00000214       __imp_?freeTree@QMapDataBase@@QAEXPAUQMapNodeBase@@H@Z 10020214     Qt5Core:Qt5Core.dll
 0002:00000218       __imp_?createNode@QMapDataBase@@QAEPAUQMapNodeBase@@HHPAU2@_N@Z 10020218     Qt5Core:Qt5Core.dll
 0002:0000021c       __imp_?recalcMostLeftNode@QMapDataBase@@QAEXXZ 1002021c     Qt5Core:Qt5Core.dll
 0002:00000220       __imp_?freeNodeAndRebalance@QMapDataBase@@QAEXPAUQMapNodeBase@@@Z 10020220     Qt5Core:Qt5Core.dll
 0002:00000224       __imp_?nextNode@QMapNodeBase@@QBEPBU1@XZ 10020224     Qt5Core:Qt5Core.dll
 0002:00000228       __imp_?connect@QObject@@QBE?AVConnection@QMetaObject@@PBV1@PBD1W4ConnectionType@Qt@@@Z 10020228     Qt5Core:Qt5Core.dll
 0002:0000022c       __imp_??1QObject@@UAE@XZ   1002022c     Qt5Core:Qt5Core.dll
 0002:00000230       __imp_?registerNormalizedTypedef@QMetaType@@SAHABVQByteArray@@H@Z 10020230     Qt5Core:Qt5Core.dll
 0002:00000234       __imp_?registerNormalizedType@QMetaType@@SAHABVQByteArray@@P6AXPAX@ZP6APAXPBX@Z2P6APAX13@ZHV?$QFlags@W4TypeFlag@QMetaType@@@@PBUQMetaObject@@@Z 10020234     Qt5Core:Qt5Core.dll
 0002:00000238       __imp_?append@QListData@@QAEPAPAXXZ 10020238     Qt5Core:Qt5Core.dll
 0002:0000023c       __imp_?dispose@QListData@@SAXPAUData@1@@Z 1002023c     Qt5Core:Qt5Core.dll
 0002:00000240       __imp_?realloc@QListData@@QAEXH@Z 10020240     Qt5Core:Qt5Core.dll
 0002:00000244       __imp_?detach_grow@QListData@@QAEPAUData@1@PAHH@Z 10020244     Qt5Core:Qt5Core.dll
 0002:00000248       __imp_?detach@QListData@@QAEPAUData@1@H@Z 10020248     Qt5Core:Qt5Core.dll
 0002:0000024c       __imp_?fromAscii_helper@QString@@CAPAU?$QTypedArrayData@G@@PBDH@Z 1002024c     Qt5Core:Qt5Core.dll
 0002:00000250       __imp_??M@YA_NABVQString@@0@Z 10020250     Qt5Core:Qt5Core.dll
 0002:00000254       __imp_?number@QString@@SA?AV1@HH@Z 10020254     Qt5Core:Qt5Core.dll
 0002:00000258       __imp_?fromUtf8@QString@@SA?AV1@PBDH@Z 10020258     Qt5Core:Qt5Core.dll
 0002:0000025c       __imp_?hasRegisteredConverterFunction@QMetaType@@SA_NHH@Z 1002025c     Qt5Core:Qt5Core.dll
 0002:00000260       __imp_?toLocal8Bit@QString@@QBE?AVQByteArray@@XZ 10020260     Qt5Core:Qt5Core.dll
 0002:00000264       __imp_??0QChar@@QAE@UQLatin1Char@@@Z 10020264     Qt5Core:Qt5Core.dll
 0002:00000268       __imp_??1Connection@QMetaObject@@QAE@XZ 10020268     Qt5Core:Qt5Core.dll
 0002:0000026c       __imp_?normalizedType@QMetaObject@@SA?AVQByteArray@@PBD@Z 1002026c     Qt5Core:Qt5Core.dll
 0002:00000270       __imp_?tr@QMetaObject@@QBE?AVQString@@PBD0H@Z 10020270     Qt5Core:Qt5Core.dll
 0002:00000274       __imp_?cast@QMetaObject@@QBEPAVQObject@@PAV2@@Z 10020274     Qt5Core:Qt5Core.dll
 0002:00000278       __imp_?toLower@QString@@QBE?AV1@XZ 10020278     Qt5Core:Qt5Core.dll
 0002:0000027c       __imp_?dynamicMetaObject@QObjectData@@QBEPAUQMetaObject@@XZ 1002027c     Qt5Core:Qt5Core.dll
 0002:00000280       __imp_?className@QMetaObject@@QBEPBDXZ 10020280     Qt5Core:Qt5Core.dll
 0002:00000284       __imp_?append@QByteArray@@QAEAAV1@PBD@Z 10020284     Qt5Core:Qt5Core.dll
 0002:00000288       __imp_?append@QByteArray@@QAEAAV1@D@Z 10020288     Qt5Core:Qt5Core.dll
 0002:0000028c       __imp_?reserve@QByteArray@@QAEXH@Z 1002028c     Qt5Core:Qt5Core.dll
 0002:00000290       __imp_??0QByteArray@@QAE@XZ 10020290     Qt5Core:Qt5Core.dll
 0002:00000294       __imp_?readLine@QTextStream@@QAE?AVQString@@_J@Z 10020294     Qt5Core:Qt5Core.dll
 0002:00000298       __imp_?atEnd@QTextStream@@QBE_NXZ 10020298     Qt5Core:Qt5Core.dll
 0002:0000029c       __imp_??1QTextStream@@UAE@XZ 1002029c     Qt5Core:Qt5Core.dll
 0002:000002a0       __imp_??0QTextStream@@QAE@PAVQIODevice@@@Z 100202a0     Qt5Core:Qt5Core.dll
 0002:000002a4       \177Qt5Core_NULL_THUNK_DATA 100202a4     Qt5Core:Qt5Core.dll
 0002:000002a8       __imp_??0QIcon@@QAE@ABVQString@@@Z 100202a8     Qt5Gui:Qt5Gui.dll
 0002:000002ac       __imp_??1QIcon@@QAE@XZ     100202ac     Qt5Gui:Qt5Gui.dll
 0002:000002b0       __imp_?loadResource@QTextDocument@@MAE?AVQVariant@@HABVQUrl@@@Z 100202b0     Qt5Gui:Qt5Gui.dll
 0002:000002b4       __imp_?createObject@QTextDocument@@MAEPAVQTextObject@@ABVQTextFormat@@@Z 100202b4     Qt5Gui:Qt5Gui.dll
 0002:000002b8       __imp_?clear@QTextDocument@@UAEXXZ 100202b8     Qt5Gui:Qt5Gui.dll
 0002:000002bc       __imp_??4QIcon@@QAEAAV0@$$QAV0@@Z 100202bc     Qt5Gui:Qt5Gui.dll
 0002:000002c0       \177Qt5Gui_NULL_THUNK_DATA 100202c0     Qt5Gui:Qt5Gui.dll
 0002:000002c4       __imp_??4QScriptValue@@QAEAAV0@ABV0@@Z 100202c4     Qt5Script:Qt5Script.dll
 0002:000002c8       __imp_??0QScriptValue@@QAE@ABV0@@Z 100202c8     Qt5Script:Qt5Script.dll
 0002:000002cc       __imp_?isNumber@QScriptValue@@QBE_NXZ 100202cc     Qt5Script:Qt5Script.dll
 0002:000002d0       __imp_??0QScriptValue@@QAE@XZ 100202d0     Qt5Script:Qt5Script.dll
 0002:000002d4       __imp_?isString@QScriptValue@@QBE_NXZ 100202d4     Qt5Script:Qt5Script.dll
 0002:000002d8       __imp_?toString@QScriptValue@@QBE?AVQString@@XZ 100202d8     Qt5Script:Qt5Script.dll
 0002:000002dc       __imp_?toInt32@QScriptValue@@QBEHXZ 100202dc     Qt5Script:Qt5Script.dll
 0002:000002e0       __imp_??1QScriptEngine@@UAE@XZ 100202e0     Qt5Script:Qt5Script.dll
 0002:000002e4       __imp_?newVariant@QScriptEngine@@QAE?AVQScriptValue@@ABVQVariant@@@Z 100202e4     Qt5Script:Qt5Script.dll
 0002:000002e8       __imp_??1QScriptValue@@QAE@XZ 100202e8     Qt5Script:Qt5Script.dll
 0002:000002ec       \177Qt5Script_NULL_THUNK_DATA 100202ec     Qt5Script:Qt5Script.dll
 0002:000002f0       __imp_?updateEditorGeometry@QItemDelegate@@UBEXPAVQWidget@@ABVQStyleOptionViewItem@@ABVQModelIndex@@@Z 100202f0     Qt5Widgets:Qt5Widgets.dll
 0002:000002f4       __imp_?sizeHint@QItemDelegate@@UBE?AVQSize@@ABVQStyleOptionViewItem@@ABVQModelIndex@@@Z 100202f4     Qt5Widgets:Qt5Widgets.dll
 0002:000002f8       __imp_?paintingRoles@QAbstractItemDelegate@@UBE?AV?$QVector@H@@XZ 100202f8     Qt5Widgets:Qt5Widgets.dll
 0002:000002fc       __imp_?paint@QItemDelegate@@UBEXPAVQPainter@@ABVQStyleOptionViewItem@@ABVQModelIndex@@@Z 100202fc     Qt5Widgets:Qt5Widgets.dll
 0002:00000300       __imp_?helpEvent@QAbstractItemDelegate@@UAE_NPAVQHelpEvent@@PAVQAbstractItemView@@ABVQStyleOptionViewItem@@ABVQModelIndex@@@Z 10020300     Qt5Widgets:Qt5Widgets.dll
 0002:00000304       __imp_?eventFilter@QItemDelegate@@MAE_NPAVQObject@@PAVQEvent@@@Z 10020304     Qt5Widgets:Qt5Widgets.dll
 0002:00000308       __imp_?editorEvent@QItemDelegate@@MAE_NPAVQEvent@@PAVQAbstractItemModel@@ABVQStyleOptionViewItem@@ABVQModelIndex@@@Z 10020308     Qt5Widgets:Qt5Widgets.dll
 0002:0000030c       __imp_?drawFocus@QItemDelegate@@MBEXPAVQPainter@@ABVQStyleOptionViewItem@@ABVQRect@@@Z 1002030c     Qt5Widgets:Qt5Widgets.dll
 0002:00000310       __imp_?drawDisplay@QItemDelegate@@MBEXPAVQPainter@@ABVQStyleOptionViewItem@@ABVQRect@@ABVQString@@@Z 10020310     Qt5Widgets:Qt5Widgets.dll
 0002:00000314       __imp_?drawDecoration@QItemDelegate@@MBEXPAVQPainter@@ABVQStyleOptionViewItem@@ABVQRect@@ABVQPixmap@@@Z 10020314     Qt5Widgets:Qt5Widgets.dll
 0002:00000318       __imp_?destroyEditor@QAbstractItemDelegate@@UBEXPAVQWidget@@ABVQModelIndex@@@Z 10020318     Qt5Widgets:Qt5Widgets.dll
 0002:0000031c       __imp_?drawCheck@QItemDelegate@@MBEXPAVQPainter@@ABVQStyleOptionViewItem@@ABVQRect@@W4CheckState@Qt@@@Z 1002031c     Qt5Widgets:Qt5Widgets.dll
 0002:00000320       \177Qt5Widgets_NULL_THUNK_DATA 10020320     Qt5Widgets:Qt5Widgets.dll
 0002:00000324       __imp_?attribute@QDomElement@@QBE?AVQString@@ABV2@0@Z 10020324     Qt5Xml:Qt5Xml.dll
 0002:00000328       \177Qt5Xml_NULL_THUNK_DATA 10020328     Qt5Xml:Qt5Xml.dll
 0002:0000032c       __imp_??1GUrl@U2@@QAE@XZ   1002032c     U2Core:U2Core.dll
 0002:00000330       __imp_??0GUrl@U2@@QAE@ABVQString@@@Z 10020330     U2Core:U2Core.dll
 0002:00000334       __imp_?instance@AppResourcePool@U2@@SAPAV12@XZ 10020334     U2Core:U2Core.dll
 0002:00000338       __imp_?isCoR@U2OpStatus@U2@@UBE_NXZ 10020338     U2Core:U2Core.dll
 0002:0000033c       __imp_?info@Logger@U2@@QAEXABVQString@@@Z 1002033c     U2Core:U2Core.dll
 0002:00000340       __imp_?details@Logger@U2@@QAEXABVQString@@@Z 10020340     U2Core:U2Core.dll
 0002:00000344       __imp_?getAppSettings@AppContext@U2@@SAPAVAppSettings@2@XZ 10020344     U2Core:U2Core.dll
 0002:00000348       __imp_??_7SimpleEventCounter@U2@@6B@ 10020348     U2Core:U2Core.dll
 0002:0000034c       __imp_?setReportingSupported@Task@U2@@UAEX_N@Z 1002034c     U2Core:U2Core.dll
 0002:00000350       __imp_?setReportingEnabled@Task@U2@@UAEX_N@Z 10020350     U2Core:U2Core.dll
 0002:00000354       __imp_?setNotificationReport@Task@U2@@UAEX_N@Z 10020354     U2Core:U2Core.dll
 0002:00000358       __imp_?setNoAutoDelete@Task@U2@@UAEX_N@Z 10020358     U2Core:U2Core.dll
 0002:0000035c       __imp_?setListenerForTask@ExternalToolSupportTask@U2@@MAEXPAVExternalToolRunTask@2@H@Z 1002035c     U2Core:U2Core.dll
 0002:00000360       __imp_?setListenerForHelper@ExternalToolSupportTask@U2@@MAEXPAVExternalToolRunTaskHelper@2@H@Z 10020360     U2Core:U2Core.dll
 0002:00000364       __imp_?setLastError@ExternalToolLogParser@U2@@MAEXABVQString@@@Z 10020364     U2Core:U2Core.dll
 0002:00000368       __imp_?setCollectChildrensWarningsFlag@Task@U2@@UAEX_N@Z 10020368     U2Core:U2Core.dll
 0002:0000036c       __imp_?run@Task@U2@@UAEXXZ 1002036c     U2Core:U2Core.dll
 0002:00000370       __imp_?run@ExternalToolRunTask@U2@@UAEXXZ 10020370     U2Core:U2Core.dll
 0002:00000374       __imp_?report@Task@U2@@UAE?AW4ReportResult@12@XZ 10020374     U2Core:U2Core.dll
 0002:00000378       __imp_?qt_metacast@TaskSignalMapper@U2@@UAEPAXPBD@Z 10020378     U2Core:U2Core.dll
 0002:0000037c       __imp_?qt_metacast@FailTask@U2@@UAEPAXPBD@Z 1002037c     U2Core:U2Core.dll
 0002:00000380       __imp_?qt_metacast@ExternalToolRunTask@U2@@UAEPAXPBD@Z 10020380     U2Core:U2Core.dll
 0002:00000384       __imp_?qt_metacast@ExternalToolLogParser@U2@@UAEPAXPBD@Z 10020384     U2Core:U2Core.dll
 0002:00000388       __imp_?qt_metacall@TaskSignalMapper@U2@@UAEHW4Call@QMetaObject@@HPAPAX@Z 10020388     U2Core:U2Core.dll
 0002:0000038c       __imp_?qt_metacall@FailTask@U2@@UAEHW4Call@QMetaObject@@HPAPAX@Z 1002038c     U2Core:U2Core.dll
 0002:00000390       __imp_?qt_metacall@ExternalToolRunTask@U2@@UAEHW4Call@QMetaObject@@HPAPAX@Z 10020390     U2Core:U2Core.dll
 0002:00000394       __imp_?qt_metacall@ExternalToolLogParser@U2@@UAEHW4Call@QMetaObject@@HPAPAX@Z 10020394     U2Core:U2Core.dll
 0002:00000398       __imp_?propagateSubtaskError@Task@U2@@UAE_NXZ 10020398     U2Core:U2Core.dll
 0002:0000039c       __imp_?processLine@ExternalToolLogParser@U2@@MAEXABVQString@@@Z 1002039c     U2Core:U2Core.dll
 0002:000003a0       __imp_?processErrLine@ExternalToolLogParser@U2@@MAEXABVQString@@@Z 100203a0     U2Core:U2Core.dll
 0002:000003a4       __imp_?prepare@Task@U2@@UAEXXZ 100203a4     U2Core:U2Core.dll
 0002:000003a8       __imp_?parseOutput@ExternalToolLogParser@U2@@UAEXABVQString@@@Z 100203a8     U2Core:U2Core.dll
 0002:000003ac       __imp_?parseErrOutput@ExternalToolLogParser@U2@@UAEXABVQString@@@Z 100203ac     U2Core:U2Core.dll
 0002:000003b0       __imp_?onSubTaskFinished@Task@U2@@MAE?AV?$QList@PAVTask@U2@@@@PAV12@@Z 100203b0     U2Core:U2Core.dll
 0002:000003b4       __imp_?metaObject@TaskSignalMapper@U2@@UBEPBUQMetaObject@@XZ 100203b4     U2Core:U2Core.dll
 0002:000003b8       __imp_?metaObject@FailTask@U2@@UBEPBUQMetaObject@@XZ 100203b8     U2Core:U2Core.dll
 0002:000003bc       __imp_?metaObject@ExternalToolRunTask@U2@@UBEPBUQMetaObject@@XZ 100203bc     U2Core:U2Core.dll
 0002:000003c0       __imp_?metaObject@ExternalToolLogParser@U2@@UBEPBUQMetaObject@@XZ 100203c0     U2Core:U2Core.dll
 0002:000003c4       __imp_?isTopLevelTask@Task@U2@@UBE_NXZ 100203c4     U2Core:U2Core.dll
 0002:000003c8       __imp_?isReportingSupported@Task@U2@@UBE_NXZ 100203c8     U2Core:U2Core.dll
 0002:000003cc       __imp_?isReportingEnabled@Task@U2@@UBE_NXZ 100203cc     U2Core:U2Core.dll
 0002:000003d0       __imp_?createWorkingDir@FileAndDirectoryUtils@U2@@SA?AVQString@@ABV3@H00@Z 100203d0     U2Core:U2Core.dll
 0002:000003d4       __imp_?hasWarning@Task@U2@@UBE_NXZ 100203d4     U2Core:U2Core.dll
 0002:000003d8       __imp_?hasSubtasksWithErrors@Task@U2@@UBE_NXZ 100203d8     U2Core:U2Core.dll
 0002:000003dc       __imp_?getWarnings@Task@U2@@UBE?AVQStringList@@XZ 100203dc     U2Core:U2Core.dll
 0002:000003e0       __imp_?getTopLevelParentTask@Task@U2@@UAEPAV12@XZ 100203e0     U2Core:U2Core.dll
 0002:000003e4       __imp_?getTaskId@Task@U2@@UBE_JXZ 100203e4     U2Core:U2Core.dll
 0002:000003e8       __imp_?getSubtaskWithErrors@Task@U2@@UBEPAV12@XZ 100203e8     U2Core:U2Core.dll
 0002:000003ec       __imp_?getProgress@ExternalToolLogParser@U2@@UAEHXZ 100203ec     U2Core:U2Core.dll
 0002:000003f0       __imp_?getParentTask@Task@U2@@UBEPAV12@XZ 100203f0     U2Core:U2Core.dll
 0002:000003f4       __imp_?getNumParallelSubtasks@Task@U2@@UBEHXZ 100203f4     U2Core:U2Core.dll
 0002:000003f8       __imp_?generateReport@Task@U2@@UBE?AVQString@@XZ 100203f8     U2Core:U2Core.dll
 0002:000003fc       __imp_?cleanup@Task@U2@@UAEXXZ 100203fc     U2Core:U2Core.dll
 0002:00000400       __imp_??1ExternalToolLogParser@U2@@UAE@XZ 10020400     U2Core:U2Core.dll
 0002:00000404       __imp_??0ExternalToolLogParser@U2@@QAE@_N@Z 10020404     U2Core:U2Core.dll
 0002:00000408       __imp_?addListeners@ExternalToolSupportTask@U2@@QAEXABV?$QList@PAVExternalToolListener@U2@@@@@Z 10020408     U2Core:U2Core.dll
 0002:0000040c       __imp_??1ExternalToolSupportTask@U2@@UAE@XZ 1002040c     U2Core:U2Core.dll
 0002:00000410       __imp_??0ExternalToolSupportTask@U2@@QAE@ABVQString@@V?$QFlags@W4TaskFlag@U2@@@@@Z 10020410     U2Core:U2Core.dll
 0002:00000414       __imp_??1ExternalToolRunTask@U2@@UAE@XZ 10020414     U2Core:U2Core.dll
 0002:00000418       __imp_??0ExternalToolRunTask@U2@@QAE@ABVQString@@ABVQStringList@@PAVExternalToolLogParser@1@010_N@Z 10020418     U2Core:U2Core.dll
 0002:0000041c       __imp_?runScript@ScriptTask@U2@@SA?AVQScriptValue@@PAVQScriptEngine@@ABV?$QMap@VQString@@VQScriptValue@@@@ABVQString@@AAVTaskStateInfo@2@@Z 1002041c     U2Core:U2Core.dll
 0002:00000420       __imp_??0TaskSignalMapper@U2@@QAE@PAVTask@1@@Z 10020420     U2Core:U2Core.dll
 0002:00000424       __imp_?required@L10N@U2@@SA?AVQString@@XZ 10020424     U2Core:U2Core.dll
 0002:00000428       __imp_??1FailTask@U2@@UAE@XZ 10020428     U2Core:U2Core.dll
 0002:0000042c       __imp_??0FailTask@U2@@QAE@ABVQString@@@Z 1002042c     U2Core:U2Core.dll
 0002:00000430       __imp_?setError@Task@U2@@QAEXABVQString@@@Z 10020430     U2Core:U2Core.dll
 0002:00000434       __imp_?hasError@Task@U2@@QBE_NXZ 10020434     U2Core:U2Core.dll
 0002:00000438       __imp_?addSubTask@Task@U2@@QAEXPAV12@@Z 10020438     U2Core:U2Core.dll
 0002:0000043c       __imp_??1TaskStateInfo@U2@@UAE@XZ 1002043c     U2Core:U2Core.dll
 0002:00000440       __imp_?setError@TaskStateInfo@U2@@UAEXABVQString@@@Z 10020440     U2Core:U2Core.dll
 0002:00000444       __imp_?getError@TaskStateInfo@U2@@UBE?AVQString@@XZ 10020444     U2Core:U2Core.dll
 0002:00000448       __imp_??0TaskStateInfo@U2@@QAE@XZ 10020448     U2Core:U2Core.dll
 0002:0000044c       __imp_?error@Logger@U2@@QAEXABVQString@@@Z 1002044c     U2Core:U2Core.dll
 0002:00000450       __imp_?trace@Logger@U2@@QAEXABVQString@@@Z 10020450     U2Core:U2Core.dll
 0002:00000454       __imp_??1Logger@U2@@UAE@XZ 10020454     U2Core:U2Core.dll
 0002:00000458       __imp_??0Logger@U2@@QAE@ABVQString@@@Z 10020458     U2Core:U2Core.dll
 0002:0000045c       __imp_?getDataPathByName@U2DataPathRegistry@U2@@QAEPAVU2DataPath@2@ABVQString@@@Z 1002045c     U2Core:U2Core.dll
 0002:00000460       __imp_?getPathByName@U2DataPath@U2@@QBE?AVQString@@ABV3@@Z 10020460     U2Core:U2Core.dll
 0002:00000464       __imp_?isValid@U2DataPath@U2@@QBE_NXZ 10020464     U2Core:U2Core.dll
 0002:00000468       __imp_?getPath@U2DataPath@U2@@QBEABVQString@@XZ 10020468     U2Core:U2Core.dll
 0002:0000046c       __imp_??1SimpleEventCounter@U2@@UAE@XZ 1002046c     U2Core:U2Core.dll
 0002:00000470       __imp_??0GReportableCounter@U2@@QAE@ABVQString@@0N@Z 10020470     U2Core:U2Core.dll
 0002:00000474       __imp_??1GCounter@U2@@UAE@XZ 10020474     U2Core:U2Core.dll
 0002:00000478       __imp_?rollFileName@GUrlUtils@U2@@SA?AVQString@@ABV3@0ABV?$QSet@VQString@@@@@Z 10020478     U2Core:U2Core.dll
 0002:0000047c       __imp_?ensureFileExt@GUrlUtils@U2@@SA?AVGUrl@2@ABV32@ABVQStringList@@@Z 1002047c     U2Core:U2Core.dll
 0002:00000480       __imp_?createDirectory@GUrlUtils@U2@@SA?AVQString@@ABV3@0AAVU2OpStatus@2@@Z 10020480     U2Core:U2Core.dll
 0002:00000484       __imp_??0U2OpStatusImpl@U2@@QAE@XZ 10020484     U2Core:U2Core.dll
 0002:00000488       __imp_?getError@U2OpStatusImpl@U2@@UBE?AVQString@@XZ 10020488     U2Core:U2Core.dll
 0002:0000048c       __imp_?getDataPathRegistry@AppContext@U2@@SAPAVU2DataPathRegistry@2@XZ 1002048c     U2Core:U2Core.dll
 0002:00000490       __imp_??1U2OpStatusImpl@U2@@UAE@XZ 10020490     U2Core:U2Core.dll
 0002:00000494       __imp_?tr@ExternalToolLogParser@U2@@SA?AVQString@@PBD0H@Z 10020494     U2Core:U2Core.dll
 0002:00000498       __imp_??0ExternalTool@U2@@QAE@VQString@@00@Z 10020498     U2Core:U2Core.dll
 0002:0000049c       __imp_??1ExternalTool@U2@@UAE@XZ 1002049c     U2Core:U2Core.dll
 0002:000004a0       __imp_?registerEntry@ExternalToolRegistry@U2@@QAE_NPAVExternalTool@2@@Z 100204a0     U2Core:U2Core.dll
 0002:000004a4       __imp_?unregisterEntry@ExternalToolRegistry@U2@@QAEXABVQString@@@Z 100204a4     U2Core:U2Core.dll
 0002:000004a8       __imp_?setToolkitDescription@ExternalToolRegistry@U2@@QAEXABVQString@@0@Z 100204a8     U2Core:U2Core.dll
 0002:000004ac       __imp_?getMainWindow@AppContext@U2@@SAPAVMainWindow@2@XZ 100204ac     U2Core:U2Core.dll
 0002:000004b0       __imp_?extractAdditionalParameters@ExternalTool@U2@@UAEXABVQString@@@Z 100204b0     U2Core:U2Core.dll
 0002:000004b4       __imp_?getAdditionalPaths@ExternalTool@U2@@UBE?AVQStringList@@XZ 100204b4     U2Core:U2Core.dll
 0002:000004b8       __imp_?getRunParameters@ExternalTool@U2@@UBE?AVQStringList@@XZ 100204b8     U2Core:U2Core.dll
 0002:000004bc       __imp_?getToolRunnerAdditionalOptions@ExternalTool@U2@@UBE?AVQStringList@@XZ 100204bc     U2Core:U2Core.dll
 0002:000004c0       __imp_?performAdditionalChecks@ExternalTool@U2@@UAEXABVQString@@@Z 100204c0     U2Core:U2Core.dll
 0002:000004c4       __imp_?getTestFramework@AppContext@U2@@SAPAVTestFramework@2@XZ 100204c4     U2Core:U2Core.dll
 0002:000004c8       __imp_?getExternalToolRegistry@AppContext@U2@@SAPAVExternalToolRegistry@2@XZ 100204c8     U2Core:U2Core.dll
 0002:000004cc       __imp_??0Plugin@U2@@QAE@ABVQString@@0_NW4PluginState@1@@Z 100204cc     U2Core:U2Core.dll
 0002:000004d0       __imp_??1Plugin@U2@@UAE@XZ 100204d0     U2Core:U2Core.dll
 0002:000004d4       __imp_?qt_metacast@Task@U2@@UAEPAXPBD@Z 100204d4     U2Core:U2Core.dll
 0002:000004d8       __imp_?qt_metacall@Task@U2@@UAEHW4Call@QMetaObject@@HPAPAX@Z 100204d8     U2Core:U2Core.dll
 0002:000004dc       __imp_?staticMetaObject@Task@U2@@2UQMetaObject@@B 100204dc     U2Core:U2Core.dll
 0002:000004e0       __imp_?qt_metacast@ExternalTool@U2@@UAEPAXPBD@Z 100204e0     U2Core:U2Core.dll
 0002:000004e4       __imp_?qt_metacall@ExternalTool@U2@@UAEHW4Call@QMetaObject@@HPAPAX@Z 100204e4     U2Core:U2Core.dll
 0002:000004e8       __imp_?staticMetaObject@ExternalTool@U2@@2UQMetaObject@@B 100204e8     U2Core:U2Core.dll
 0002:000004ec       __imp_?qt_metacast@Plugin@U2@@UAEPAXPBD@Z 100204ec     U2Core:U2Core.dll
 0002:000004f0       __imp_?qt_metacall@Plugin@U2@@UAEHW4Call@QMetaObject@@HPAPAX@Z 100204f0     U2Core:U2Core.dll
 0002:000004f4       __imp_?staticMetaObject@Plugin@U2@@2UQMetaObject@@B 100204f4     U2Core:U2Core.dll
 0002:000004f8       __imp_?isNotificationReport@Task@U2@@UBE_NXZ 100204f8     U2Core:U2Core.dll
 0002:000004fc       \177U2Core_NULL_THUNK_DATA 100204fc     U2Core:U2Core.dll
 0002:00000500       __imp_?qt_metacast@URLDelegate@U2@@UAEPAXPBD@Z 10020500     U2Designer:U2Designer.dll
 0002:00000504       __imp_?removeDelegate@DelegateEditor@U2@@UAEPAVPropertyDelegate@2@ABVQString@@@Z 10020504     U2Designer:U2Designer.dll
 0002:00000508       __imp_?setEditorData@ComboBoxDelegate@U2@@UBEXPAVQWidget@@ABVQModelIndex@@@Z 10020508     U2Designer:U2Designer.dll
 0002:0000050c       __imp_?setEditorData@URLDelegate@U2@@UBEXPAVQWidget@@ABVQModelIndex@@@Z 1002050c     U2Designer:U2Designer.dll
 0002:00000510       __imp_?setModelData@ComboBoxDelegate@U2@@UBEXPAVQWidget@@PAVQAbstractItemModel@@ABVQModelIndex@@@Z 10020510     U2Designer:U2Designer.dll
 0002:00000514       __imp_?setModelData@URLDelegate@U2@@UBEXPAVQWidget@@PAVQAbstractItemModel@@ABVQModelIndex@@@Z 10020514     U2Designer:U2Designer.dll
 0002:00000518       __imp_?type@URLDelegate@U2@@UBE?AW4Type@PropertyDelegate@2@XZ 10020518     U2Designer:U2Designer.dll
 0002:0000051c       __imp_?updateDelegate@DelegateEditor@U2@@UAEXABVQString@@@Z 1002051c     U2Designer:U2Designer.dll
 0002:00000520       __imp_?updateDelegates@DelegateEditor@U2@@UAEXXZ 10020520     U2Designer:U2Designer.dll
 0002:00000524       __imp_??0URLDelegate@U2@@QAE@ABVDelegateTags@1@ABVQString@@_N22PAVQObject@@22@Z 10020524     U2Designer:U2Designer.dll
 0002:00000528       __imp_??0SpinBoxDelegate@U2@@QAE@ABV?$QMap@VQString@@VQVariant@@@@PAVQObject@@@Z 10020528     U2Designer:U2Designer.dll
 0002:0000052c       __imp_??1SpinBoxDelegate@U2@@UAE@XZ 1002052c     U2Designer:U2Designer.dll
 0002:00000530       __imp_?clone@SpinBoxDelegate@U2@@UAEPAVPropertyDelegate@2@XZ 10020530     U2Designer:U2Designer.dll
 0002:00000534       __imp_?createEditor@SpinBoxDelegate@U2@@UBEPAVQWidget@@PAV3@ABVQStyleOptionViewItem@@ABVQModelIndex@@@Z 10020534     U2Designer:U2Designer.dll
 0002:00000538       __imp_?createWizardWidget@SpinBoxDelegate@U2@@UBEPAVPropertyWidget@2@AAVU2OpStatus@2@PAVQWidget@@@Z 10020538     U2Designer:U2Designer.dll
 0002:0000053c       __imp_?getDisplayValue@SpinBoxDelegate@U2@@UBE?AVQVariant@@ABV3@@Z 1002053c     U2Designer:U2Designer.dll
 0002:00000540       __imp_?getItems@SpinBoxDelegate@U2@@UBEXAAV?$QMap@VQString@@VQVariant@@@@@Z 10020540     U2Designer:U2Designer.dll
 0002:00000544       __imp_?metaObject@SpinBoxDelegate@U2@@UBEPBUQMetaObject@@XZ 10020544     U2Designer:U2Designer.dll
 0002:00000548       __imp_?qt_metacall@SpinBoxDelegate@U2@@UAEHW4Call@QMetaObject@@HPAPAX@Z 10020548     U2Designer:U2Designer.dll
 0002:0000054c       __imp_?qt_metacast@SpinBoxDelegate@U2@@UAEPAXPBD@Z 1002054c     U2Designer:U2Designer.dll
 0002:00000550       __imp_?setEditorData@SpinBoxDelegate@U2@@UBEXPAVQWidget@@ABVQModelIndex@@@Z 10020550     U2Designer:U2Designer.dll
 0002:00000554       __imp_?setModelData@SpinBoxDelegate@U2@@UBEXPAVQWidget@@PAVQAbstractItemModel@@ABVQModelIndex@@@Z 10020554     U2Designer:U2Designer.dll
 0002:00000558       __imp_??1DelegateEditor@U2@@UAE@XZ 10020558     U2Designer:U2Designer.dll
 0002:0000055c       __imp_??0URLDelegate@U2@@QAE@ABVDelegateTags@1@ABVQString@@ABV?$QFlags@W4Option@URLDelegate@U2@@@@PAVQObject@@@Z 1002055c     U2Designer:U2Designer.dll
 0002:00000560       __imp_??1URLDelegate@U2@@UAE@XZ 10020560     U2Designer:U2Designer.dll
 0002:00000564       __imp_??0ComboBoxDelegate@U2@@QAE@ABV?$QMap@VQString@@VQVariant@@@@PAVQObject@@@Z 10020564     U2Designer:U2Designer.dll
 0002:00000568       __imp_??1ComboBoxDelegate@U2@@UAE@XZ 10020568     U2Designer:U2Designer.dll
 0002:0000056c       __imp_?addDelegate@DelegateEditor@U2@@UAEXPAVPropertyDelegate@2@ABVQString@@@Z 1002056c     U2Designer:U2Designer.dll
 0002:00000570       __imp_?clone@ComboBoxDelegate@U2@@UAEPAVPropertyDelegate@2@XZ 10020570     U2Designer:U2Designer.dll
 0002:00000574       __imp_?clone@DelegateEditor@U2@@UAEPAVConfigurationEditor@2@XZ 10020574     U2Designer:U2Designer.dll
 0002:00000578       __imp_?clone@URLDelegate@U2@@UAEPAVPropertyDelegate@2@XZ 10020578     U2Designer:U2Designer.dll
 0002:0000057c       __imp_?commit@DelegateEditor@U2@@UAEXXZ 1002057c     U2Designer:U2Designer.dll
 0002:00000580       __imp_?createEditor@ComboBoxDelegate@U2@@UBEPAVQWidget@@PAV3@ABVQStyleOptionViewItem@@ABVQModelIndex@@@Z 10020580     U2Designer:U2Designer.dll
 0002:00000584       __imp_?createEditor@URLDelegate@U2@@UBEPAVQWidget@@PAV3@ABVQStyleOptionViewItem@@ABVQModelIndex@@@Z 10020584     U2Designer:U2Designer.dll
 0002:00000588       __imp_?createWizardWidget@ComboBoxDelegate@U2@@UBEPAVPropertyWidget@2@AAVU2OpStatus@2@PAVQWidget@@@Z 10020588     U2Designer:U2Designer.dll
 0002:0000058c       __imp_?createWizardWidget@URLDelegate@U2@@UBEPAVPropertyWidget@2@AAVU2OpStatus@2@PAVQWidget@@@Z 1002058c     U2Designer:U2Designer.dll
 0002:00000590       __imp_?getDelegate@DelegateEditor@U2@@UAEPAVPropertyDelegate@2@ABVQString@@@Z 10020590     U2Designer:U2Designer.dll
 0002:00000594       __imp_?getDisplayValue@ComboBoxDelegate@U2@@UBE?AVQVariant@@ABV3@@Z 10020594     U2Designer:U2Designer.dll
 0002:00000598       __imp_?getDisplayValue@URLDelegate@U2@@UBE?AVQVariant@@ABV3@@Z 10020598     U2Designer:U2Designer.dll
 0002:0000059c       __imp_?getItems@ComboBoxDelegate@U2@@UBEXAAV?$QMap@VQString@@VQVariant@@@@@Z 1002059c     U2Designer:U2Designer.dll
 0002:000005a0       __imp_?metaObject@ComboBoxDelegate@U2@@UBEPBUQMetaObject@@XZ 100205a0     U2Designer:U2Designer.dll
 0002:000005a4       __imp_?metaObject@DelegateEditor@U2@@UBEPBUQMetaObject@@XZ 100205a4     U2Designer:U2Designer.dll
 0002:000005a8       __imp_??0DelegateEditor@U2@@QAE@ABV?$QMap@VQString@@PAVPropertyDelegate@U2@@@@@Z 100205a8     U2Designer:U2Designer.dll
 0002:000005ac       __imp_?metaObject@URLDelegate@U2@@UBEPBUQMetaObject@@XZ 100205ac     U2Designer:U2Designer.dll
 0002:000005b0       __imp_?qt_metacall@ComboBoxDelegate@U2@@UAEHW4Call@QMetaObject@@HPAPAX@Z 100205b0     U2Designer:U2Designer.dll
 0002:000005b4       __imp_?qt_metacall@DelegateEditor@U2@@UAEHW4Call@QMetaObject@@HPAPAX@Z 100205b4     U2Designer:U2Designer.dll
 0002:000005b8       __imp_?qt_metacall@URLDelegate@U2@@UAEHW4Call@QMetaObject@@HPAPAX@Z 100205b8     U2Designer:U2Designer.dll
 0002:000005bc       __imp_?qt_metacast@ComboBoxDelegate@U2@@UAEPAXPBD@Z 100205bc     U2Designer:U2Designer.dll
 0002:000005c0       __imp_?qt_metacast@DelegateEditor@U2@@UAEPAXPBD@Z 100205c0     U2Designer:U2Designer.dll
 0002:000005c4       \177U2Designer_NULL_THUNK_DATA 100205c4     U2Designer:U2Designer.dll
 0002:000005c8       __imp_?prepareFileFilter@DialogUtils@U2@@SA?AVQString@@ABV3@ABVQStringList@@_N1@Z 100205c8     U2Gui:U2Gui.dll
 0002:000005cc       \177U2Gui_NULL_THUNK_DATA  100205cc     U2Gui:U2Gui.dll
 0002:000005d0       __imp_??1PropertyDelegate@U2@@UAE@XZ 100205d0     U2Lang:U2Lang.dll
 0002:000005d4       __imp_??0DelegateTags@U2@@QAE@PAVQObject@@@Z 100205d4     U2Lang:U2Lang.dll
 0002:000005d8       __imp_?set@DelegateTags@U2@@QAEXABVQString@@ABVQVariant@@@Z 100205d8     U2Lang:U2Lang.dll
 0002:000005dc       __imp_??1DelegateTags@U2@@UAE@XZ 100205dc     U2Lang:U2Lang.dll
 0002:000005e0       __imp_?getId@Actor@Workflow@U2@@QBE?AVQString@@XZ 100205e0     U2Lang:U2Lang.dll
 0002:000005e4       __imp_?getInputPorts@Actor@Workflow@U2@@QBE?AV?$QList@PAVPort@Workflow@U2@@@@XZ 100205e4     U2Lang:U2Lang.dll
 0002:000005e8       __imp_?getOutputPorts@Actor@Workflow@U2@@QBE?AV?$QList@PAVPort@Workflow@U2@@@@XZ 100205e8     U2Lang:U2Lang.dll
 0002:000005ec       __imp_??0Attribute@U2@@QAE@ABVDescriptor@1@V?$QExplicitlySharedDataPointer@VDataType@U2@@@@_NABVQVariant@@@Z 100205ec     U2Lang:U2Lang.dll
 0002:000005f0       __imp_?getScriptVars@AttributeScript@U2@@QBEABV?$QMap@VDescriptor@U2@@VQVariant@@@@XZ 100205f0     U2Lang:U2Lang.dll
 0002:000005f4       __imp_?getScriptText@AttributeScript@U2@@QBEABVQString@@XZ 100205f4     U2Lang:U2Lang.dll
 0002:000005f8       __imp_?isEmpty@AttributeScript@U2@@QBE_NXZ 100205f8     U2Lang:U2Lang.dll
 0002:000005fc       __imp_??1WorkflowScriptEngine@U2@@UAE@XZ 100205fc     U2Lang:U2Lang.dll
 0002:00000600       __imp_??0WorkflowScriptEngine@U2@@QAE@PAVWorkflowContext@Workflow@1@@Z 10020600     U2Lang:U2Lang.dll
 0002:00000604       __imp_?absolutePath@WorkflowContext@Workflow@U2@@QBE?AVQString@@ABV4@@Z 10020604     U2Lang:U2Lang.dll
 0002:00000608       __imp_?getMonitor@WorkflowContext@Workflow@U2@@QAEPAVWorkflowMonitor@23@XZ 10020608     U2Lang:U2Lang.dll
 0002:0000060c       __imp_?isOutUrlAttribute@RFSUtils@U2@@SA_NPAVAttribute@2@PAVActor@Workflow@2@AA_N@Z 1002060c     U2Lang:U2Lang.dll
 0002:00000610       __imp_??1MessageMetadata@U2@@QAE@XZ 10020610     U2Lang:U2Lang.dll
 0002:00000614       __imp_?getId@MessageMetadata@U2@@QBEHXZ 10020614     U2Lang:U2Lang.dll
 0002:00000618       __imp_??0MessageMetadata@U2@@QAE@ABVQString@@@Z 10020618     U2Lang:U2Lang.dll
 0002:0000061c       __imp_??0WorkflowNotification@U2@@QAE@ABV01@@Z 1002061c     U2Lang:U2Lang.dll
 0002:00000620       __imp_??1WorkflowNotification@U2@@QAE@XZ 10020620     U2Lang:U2Lang.dll
 0002:00000624       __imp_??0WorkflowNotification@U2@@QAE@ABVQString@@00@Z 10020624     U2Lang:U2Lang.dll
 0002:00000628       __imp_?initEngine@WorkflowScriptLibrary@U2@@SAXPAVWorkflowScriptEngine@2@@Z 10020628     U2Lang:U2Lang.dll
 0002:0000062c       __imp_??1MapDataType@U2@@UAE@XZ 1002062c     U2Lang:U2Lang.dll
 0002:00000630       __imp_??0MapDataType@U2@@QAE@ABVDescriptor@1@ABV?$QMap@VDescriptor@U2@@V?$QExplicitlySharedDataPointer@VDataType@U2@@@@@@@Z 10020630     U2Lang:U2Lang.dll
 0002:00000634       __imp_??0Descriptor@U2@@QAE@ABV01@@Z 10020634     U2Lang:U2Lang.dll
 0002:00000638       __imp_?getId@Descriptor@U2@@QBE?AVQString@@XZ 10020638     U2Lang:U2Lang.dll
 0002:0000063c       __imp_??1Descriptor@U2@@UAE@XZ 1002063c     U2Lang:U2Lang.dll
 0002:00000640       __imp_??0Descriptor@U2@@QAE@PBD@Z 10020640     U2Lang:U2Lang.dll
 0002:00000644       __imp_??0Descriptor@U2@@QAE@ABVQString@@@Z 10020644     U2Lang:U2Lang.dll
 0002:00000648       __imp_??0Descriptor@U2@@QAE@ABVQString@@00@Z 10020648     U2Lang:U2Lang.dll
 0002:0000064c       __imp_?put@MessageMetadataStorage@U2@@QAEXABVMessageMetadata@2@@Z 1002064c     U2Lang:U2Lang.dll
 0002:00000650       __imp_??1Attribute@U2@@UAE@XZ 10020650     U2Lang:U2Lang.dll
 0002:00000654       __imp_?getMetadataStorage@WorkflowContext@Workflow@U2@@QAEAAVMessageMetadataStorage@3@XZ 10020654     U2Lang:U2Lang.dll
 0002:00000658       __imp_?staticMetaObject@BaseWorker@LocalWorkflow@U2@@2UQMetaObject@@B 10020658     U2Lang:U2Lang.dll
 0002:0000065c       __imp_?qt_metacall@BaseWorker@LocalWorkflow@U2@@UAEHW4Call@QMetaObject@@HPAPAX@Z 1002065c     U2Lang:U2Lang.dll
 0002:00000660       __imp_?qt_metacast@BaseWorker@LocalWorkflow@U2@@UAEPAXPBD@Z 10020660     U2Lang:U2Lang.dll
 0002:00000664       __imp_?FILTER@DelegateTags@U2@@2VQString@@B 10020664     U2Lang:U2Lang.dll
 0002:00000668       __imp_?U2_INFO@WorkflowNotification@U2@@2VQString@@B 10020668     U2Lang:U2Lang.dll
 0002:0000066c       __imp_?valueChangingRelation@VisibilityRelation@U2@@UBE_NXZ 1002066c     U2Lang:U2Lang.dll
 0002:00000670       __imp_?validate@PortValidator@Workflow@U2@@UBE_NPBVConfiguration@3@AAV?$QList@VWorkflowNotification@U2@@@@@Z 10020670     U2Lang:U2Lang.dll
 0002:00000674       __imp_?validate@PairedReadsPortValidator@Workflow@U2@@UBE_NPBVIntegralBusPort@23@AAV?$QList@VWorkflowNotification@U2@@@@@Z 10020674     U2Lang:U2Lang.dll
 0002:00000678       __imp_?updateDelegateTags@AttributeRelation@U2@@UBEXABVQVariant@@PAVDelegateTags@2@@Z 10020678     U2Lang:U2Lang.dll
 0002:0000067c       __imp_?isSlotEnabled@SlotRelationDescriptor@U2@@UBE_NABVQVariant@@@Z 1002067c     U2Lang:U2Lang.dll
 0002:00000680       __imp_?getType@VisibilityRelation@U2@@UBE?AW4RelationType@2@XZ 10020680     U2Lang:U2Lang.dll
 0002:00000684       __imp_?getAffectResult@VisibilityRelation@U2@@UBE?AVQVariant@@ABV3@0PAVDelegateTags@2@1@Z 10020684     U2Lang:U2Lang.dll
 0002:00000688       __imp_?clone@VisibilityRelation@U2@@UBEPAV12@XZ 10020688     U2Lang:U2Lang.dll
 0002:0000068c       __imp_?clone@SlotRelationDescriptor@U2@@UBEPAV12@XZ 1002068c     U2Lang:U2Lang.dll
 0002:00000690       __imp_?getProducersOrUnset@PrompterBaseImpl@U2@@QAE?AVQString@@ABV3@0@Z 10020690     U2Lang:U2Lang.dll
 0002:00000694       __imp_?getParameter@PrompterBaseImpl@U2@@QAE?AVQVariant@@ABVQString@@@Z 10020694     U2Lang:U2Lang.dll
 0002:00000698       __imp_?reportError@BaseWorker@LocalWorkflow@U2@@IAEXABVQString@@@Z 10020698     U2Lang:U2Lang.dll
 0002:0000069c       __imp_?addInfo@WorkflowMonitor@Workflow@U2@@QAEXABVQString@@00@Z 1002069c     U2Lang:U2Lang.dll
 0002:000006a0       __imp_?getMetadataId@Message@Workflow@U2@@QBEHXZ 100206a0     U2Lang:U2Lang.dll
 0002:000006a4       __imp_?getData@Message@Workflow@U2@@QBE?AVQVariant@@XZ 100206a4     U2Lang:U2Lang.dll
 0002:000006a8       __imp_??1PairedReadsPortValidator@Workflow@U2@@UAE@XZ 100206a8     U2Lang:U2Lang.dll
 0002:000006ac       __imp_??0PairedReadsPortValidator@Workflow@U2@@QAE@ABVQString@@0@Z 100206ac     U2Lang:U2Lang.dll
 0002:000006b0       __imp_?BOOL_TYPE@BaseTypes@U2@@SA?AV?$QExplicitlySharedDataPointer@VDataType@U2@@@@XZ 100206b0     U2Lang:U2Lang.dll
 0002:000006b4       __imp_?setPortValidator@ActorPrototype@Workflow@U2@@QAEXABVQString@@PAVConfigurationValidator@3@@Z 100206b4     U2Lang:U2Lang.dll
 0002:000006b8       __imp_?addSlotRelation@Attribute@U2@@QAEXPAVSlotRelationDescriptor@2@@Z 100206b8     U2Lang:U2Lang.dll
 0002:000006bc       __imp_?addRelation@Attribute@U2@@QAEXPBVAttributeRelation@2@@Z 100206bc     U2Lang:U2Lang.dll
 0002:000006c0       __imp_??0Attribute@U2@@QAE@ABVDescriptor@1@V?$QExplicitlySharedDataPointer@VDataType@U2@@@@V?$QFlags@W4Flag@Attribute@U2@@@@ABVQVariant@@@Z 100206c0     U2Lang:U2Lang.dll
 0002:000006c4       __imp_??1SlotRelationDescriptor@U2@@UAE@XZ 100206c4     U2Lang:U2Lang.dll
 0002:000006c8       __imp_??0SlotRelationDescriptor@U2@@QAE@ABVQString@@0ABV?$QList@VQVariant@@@@@Z 100206c8     U2Lang:U2Lang.dll
 0002:000006cc       __imp_?workingDir@WorkflowContext@Workflow@U2@@QBE?AVQString@@XZ 100206cc     U2Lang:U2Lang.dll
 0002:000006d0       __imp_?get@MessageMetadataStorage@U2@@QBE?AVMessageMetadata@2@H@Z 100206d0     U2Lang:U2Lang.dll
 0002:000006d4       __imp_?getFileUrl@MessageMetadata@U2@@QBEABVQString@@XZ 100206d4     U2Lang:U2Lang.dll
 0002:000006d8       __imp_??1VisibilityRelation@U2@@UAE@XZ 100206d8     U2Lang:U2Lang.dll
 0002:000006dc       __imp_??0VisibilityRelation@U2@@QAE@ABVQString@@ABVQVariant@@_N@Z 100206dc     U2Lang:U2Lang.dll
 0002:000006e0       __imp_?ID@LocalDomainFactory@LocalWorkflow@U2@@2VQString@@B 100206e0     U2Lang:U2Lang.dll
 0002:000006e4       __imp_??_7ActorValidator@Workflow@U2@@6B@ 100206e4     U2Lang:U2Lang.dll
 0002:000006e8       __imp_??_7ConfigurationValidator@U2@@6B@ 100206e8     U2Lang:U2Lang.dll
 0002:000006ec       __imp_?PLACEHOLDER_TEXT@DelegateTags@U2@@2VQString@@B 100206ec     U2Lang:U2Lang.dll
 0002:000006f0       __imp_?U2_ERROR@WorkflowNotification@U2@@2VQString@@B 100206f0     U2Lang:U2Lang.dll
 0002:000006f4       __imp_?validate@Attribute@U2@@UAE_NAAV?$QList@VWorkflowNotification@U2@@@@@Z 100206f4     U2Lang:U2Lang.dll
 0002:000006f8       __imp_?validate@ActorValidator@Workflow@U2@@UBE_NPBVConfiguration@3@AAV?$QList@VWorkflowNotification@U2@@@@@Z 100206f8     U2Lang:U2Lang.dll
 0002:000006fc       __imp_?updateActorIds@Attribute@U2@@UAEXABV?$QMap@VQString@@V1@@@@Z 100206fc     U2Lang:U2Lang.dll
 0002:00000700       __imp_?update@PropertyDelegate@U2@@UAEXXZ 10020700     U2Lang:U2Lang.dll
 0002:00000704       __imp_?update@PrompterBaseImpl@U2@@UAEXABV?$QMap@VQString@@VQVariant@@@@@Z 10020704     U2Lang:U2Lang.dll
 0002:00000708       __imp_?unregisterEntry@?$IdRegistry@VDomainFactory@Workflow@U2@@@U2@@UAEPAVDomainFactory@Workflow@2@ABVQString@@@Z 10020708     U2Lang:U2Lang.dll
 0002:0000070c       __imp_?type@PropertyDelegate@U2@@UBE?AW4Type@12@XZ 1002070c     U2Lang:U2Lang.dll
 0002:00000710       __imp_?sl_actorModified@PrompterBaseImpl@U2@@MAEXXZ 10020710     U2Lang:U2Lang.dll
 0002:00000714       __imp_?setVisibleSlot@PortDescriptor@Workflow@U2@@UAEXABVQString@@_N@Z 10020714     U2Lang:U2Lang.dll
 0002:00000718       __imp_?setDone@BaseWorker@LocalWorkflow@U2@@UAEXXZ 10020718     U2Lang:U2Lang.dll
 0002:0000071c       __imp_?setDocumentation@Descriptor@U2@@UAEXABVQString@@@Z 1002071c     U2Lang:U2Lang.dll
 0002:00000720       __imp_?setDocumentation@ActorPrototype@Workflow@U2@@UAEXABVQString@@@Z 10020720     U2Lang:U2Lang.dll
 0002:00000724       __imp_?setDisplayName@Descriptor@U2@@UAEXABVQString@@@Z 10020724     U2Lang:U2Lang.dll
 0002:00000728       __imp_?setDisplayName@ActorPrototype@Workflow@U2@@UAEXABVQString@@@Z 10020728     U2Lang:U2Lang.dll
 0002:0000072c       __imp_?setAttributeValue@Attribute@U2@@UAEXABVQVariant@@@Z 1002072c     U2Lang:U2Lang.dll
 0002:00000730       __imp_?registerEntry@?$IdRegistry@VDomainFactory@Workflow@U2@@@U2@@UAE_NPAVDomainFactory@Workflow@2@@Z 10020730     U2Lang:U2Lang.dll
 0002:00000734       __imp_?qt_metacast@PrompterBaseImpl@U2@@UAEPAXPBD@Z 10020734     U2Lang:U2Lang.dll
 0002:00000738       __imp_?qt_metacast@ActorPrototype@Workflow@U2@@UAEPAXPBD@Z 10020738     U2Lang:U2Lang.dll
 0002:0000073c       __imp_?qt_metacall@PrompterBaseImpl@U2@@UAEHW4Call@QMetaObject@@HPAPAX@Z 1002073c     U2Lang:U2Lang.dll
 0002:00000740       __imp_?qt_metacall@ActorPrototype@Workflow@U2@@UAEHW4Call@QMetaObject@@HPAPAX@Z 10020740     U2Lang:U2Lang.dll
 0002:00000744       __imp_?metaObject@PrompterBaseImpl@U2@@UBEPBUQMetaObject@@XZ 10020744     U2Lang:U2Lang.dll
 0002:00000748       __imp_?metaObject@ActorPrototype@Workflow@U2@@UBEPBUQMetaObject@@XZ 10020748     U2Lang:U2Lang.dll
 0002:0000074c       __imp_?kind@MapDataType@U2@@UBE?AW4Kind@DataType@2@XZ 1002074c     U2Lang:U2Lang.dll
 0002:00000750       __imp_?isReady@BaseWorker@LocalWorkflow@U2@@UBE_NXZ 10020750     U2Lang:U2Lang.dll
 0002:00000754       __imp_?isEmpty@ConfigurationEditor@U2@@UBE_NXZ 10020754     U2Lang:U2Lang.dll
 0002:00000758       __imp_?isEmpty@Attribute@U2@@UBE_NXZ 10020758     U2Lang:U2Lang.dll
 0002:0000075c       __imp_?isDone@BaseWorker@LocalWorkflow@U2@@UBE_NXZ 1002075c     U2Lang:U2Lang.dll
 0002:00000760       __imp_?isDefaultValue@Attribute@U2@@UBE_NXZ 10020760     U2Lang:U2Lang.dll
 0002:00000764       __imp_?isAcceptableDrop@ActorPrototype@Workflow@U2@@UBE_NPBVQMimeData@@PAV?$QMap@VQString@@VQVariant@@@@@Z 10020764     U2Lang:U2Lang.dll
 0002:00000768       __imp_?getWidget@ConfigurationEditor@U2@@UAEPAVQWidget@@XZ 10020768     U2Lang:U2Lang.dll
 0002:0000076c       __imp_?getType@PortDescriptor@Workflow@U2@@UBE?AV?$QExplicitlySharedDataPointer@VDataType@U2@@@@XZ 1002076c     U2Lang:U2Lang.dll
 0002:00000770       __imp_?getOutputFiles@BaseWorker@LocalWorkflow@U2@@UAE?AVQStringList@@XZ 10020770     U2Lang:U2Lang.dll
 0002:00000774       __imp_?getMessageAndSetupScriptValues@BaseWorker@LocalWorkflow@U2@@UAE?AVMessage@Workflow@3@PAVCommunicationChannel@53@@Z 10020774     U2Lang:U2Lang.dll
 0002:00000778       __imp_?getItems@PropertyDelegate@U2@@UBEXAAV?$QMap@VQString@@VQVariant@@@@@Z 10020778     U2Lang:U2Lang.dll
 0002:0000077c       __imp_?getGroup@Attribute@U2@@UAE?AW4AttributeGroup@2@XZ 1002077c     U2Lang:U2Lang.dll
 0002:00000780       __imp_?getDefaultPureValue@Attribute@U2@@UBEABVQVariant@@XZ 10020780     U2Lang:U2Lang.dll
 0002:00000784       __imp_?getDatatypesMap@MapDataType@U2@@UBE?AV?$QMap@VDescriptor@U2@@V?$QExplicitlySharedDataPointer@VDataType@U2@@@@@@XZ 10020784     U2Lang:U2Lang.dll
 0002:00000788       __imp_?getDatatypeByDescriptor@MapDataType@U2@@UBE?AV?$QExplicitlySharedDataPointer@VDataType@U2@@@@ABVDescriptor@2@@Z 10020788     U2Lang:U2Lang.dll
 0002:0000078c       __imp_?getCommunication@BaseWorker@LocalWorkflow@U2@@UAEPAVCommunicationChannel@Workflow@3@ABVQString@@@Z 1002078c     U2Lang:U2Lang.dll
 0002:00000790       __imp_?getById@?$IdRegistry@VDomainFactory@Workflow@U2@@@U2@@UAEPAVDomainFactory@Workflow@2@ABVQString@@@Z 10020790     U2Lang:U2Lang.dll
 0002:00000794       __imp_?getAttributePureValue@Attribute@U2@@UBEABVQVariant@@XZ 10020794     U2Lang:U2Lang.dll
 0002:00000798       __imp_?getAllIds@?$IdRegistry@VDomainFactory@Workflow@U2@@@U2@@UBE?AV?$QList@VQString@@@@XZ 10020798     U2Lang:U2Lang.dll
 0002:0000079c       __imp_?getAllEntries@?$IdRegistry@VDomainFactory@Workflow@U2@@@U2@@UBE?AV?$QList@PAVDomainFactory@Workflow@U2@@@@XZ 1002079c     U2Lang:U2Lang.dll
 0002:000007a0       __imp_?getAllDescriptors@MapDataType@U2@@UBE?AV?$QList@VDescriptor@U2@@@@XZ 100207a0     U2Lang:U2Lang.dll
 0002:000007a4       __imp_?getActorId@BaseWorker@LocalWorkflow@U2@@UBE?AVQString@@XZ 100207a4     U2Lang:U2Lang.dll
 0002:000007a8       __imp_?destroy@DomainFactory@Workflow@U2@@UAEXPAVScheduler@23@PAVSchema@23@@Z 100207a8     U2Lang:U2Lang.dll
 0002:000007ac       __imp_?createScheduler@DomainFactory@Workflow@U2@@UAEPAVScheduler@23@PAVSchema@23@@Z 100207ac     U2Lang:U2Lang.dll
 0002:000007b0       __imp_?createPort@IntegralBusActorPrototype@Workflow@U2@@UAEPAVPort@23@ABVPortDescriptor@23@PAVActor@23@@Z 100207b0     U2Lang:U2Lang.dll
 0002:000007b4       __imp_?createInstance@ActorPrototype@Workflow@U2@@UAEPAVActor@23@ABVQString@@PAVAttributeScript@3@ABV?$QMap@VQString@@VQVariant@@@@@Z 100207b4     U2Lang:U2Lang.dll
 0002:000007b8       __imp_?createConnection@DomainFactory@Workflow@U2@@UAEPAVCommunicationChannel@23@PAVLink@23@@Z 100207b8     U2Lang:U2Lang.dll
 0002:000007bc       __imp_?clone@Attribute@U2@@UAEPAV12@XZ 100207bc     U2Lang:U2Lang.dll
 0002:000007c0       __imp_?canTaskBeCanceled@BaseWorker@LocalWorkflow@U2@@MBE_NPAVTask@3@@Z 100207c0     U2Lang:U2Lang.dll
 0002:000007c4       __imp_?addCommunication@BaseWorker@LocalWorkflow@U2@@UAE_NABVQString@@PAVCommunicationChannel@Workflow@3@@Z 100207c4     U2Lang:U2Lang.dll
 0002:000007c8       __imp_??1PrompterBaseImpl@U2@@UAE@XZ 100207c8     U2Lang:U2Lang.dll
 0002:000007cc       __imp_?getHyperlink@PrompterBaseImpl@U2@@SA?AVQString@@ABV3@0@Z 100207cc     U2Lang:U2Lang.dll
 0002:000007d0       __imp_?getURL@PrompterBaseImpl@U2@@QAE?AVQString@@ABV3@PA_N00@Z 100207d0     U2Lang:U2Lang.dll
 0002:000007d4       __imp_??0PrompterBaseImpl@U2@@QAE@PAVActor@Workflow@1@@Z 100207d4     U2Lang:U2Lang.dll
 0002:000007d8       __imp_?createLogListeners@BaseWorker@LocalWorkflow@U2@@QBE?AV?$QList@PAVExternalToolListener@U2@@@@H@Z 100207d8     U2Lang:U2Lang.dll
 0002:000007dc       __imp_??1BaseWorker@LocalWorkflow@U2@@UAE@XZ 100207dc     U2Lang:U2Lang.dll
 0002:000007e0       __imp_??0BaseWorker@LocalWorkflow@U2@@QAE@PAVActor@Workflow@2@_N@Z 100207e0     U2Lang:U2Lang.dll
 0002:000007e4       __imp_?getBusType@IntegralBus@Workflow@U2@@QBE?AV?$QExplicitlySharedDataPointer@VDataType@U2@@@@XZ 100207e4     U2Lang:U2Lang.dll
 0002:000007e8       __imp_?addOutputFile@WorkflowMonitor@Workflow@U2@@QAEXABVQString@@0_N@Z 100207e8     U2Lang:U2Lang.dll
 0002:000007ec       __imp_??1DomainFactory@Workflow@U2@@UAE@XZ 100207ec     U2Lang:U2Lang.dll
 0002:000007f0       __imp_??0DomainFactory@Workflow@U2@@QAE@ABVQString@@@Z 100207f0     U2Lang:U2Lang.dll
 0002:000007f4       __imp_??1Message@Workflow@U2@@QAE@XZ 100207f4     U2Lang:U2Lang.dll
 0002:000007f8       __imp_??0Message@Workflow@U2@@QAE@V?$QExplicitlySharedDataPointer@VDataType@U2@@@@ABVQVariant@@H@Z 100207f8     U2Lang:U2Lang.dll
 0002:000007fc       __imp_?getInstance@WorkflowEnv@Workflow@U2@@KAPAV123@XZ 100207fc     U2Lang:U2Lang.dll
 0002:00000800       __imp_?hasNext@DatasetFilesIterator@U2@@UAE_NXZ 10020800     U2Lang:U2Lang.dll
 0002:00000804       __imp_?getNextFile@DatasetFilesIterator@U2@@UAE?AVQString@@XZ 10020804     U2Lang:U2Lang.dll
 0002:00000808       __imp_??1DatasetFilesIterator@U2@@UAE@XZ 10020808     U2Lang:U2Lang.dll
 0002:0000080c       __imp_??0DatasetFilesIterator@U2@@QAE@ABV?$QList@VDataset@U2@@@@@Z 1002080c     U2Lang:U2Lang.dll
 0002:00000810       __imp_??1Dataset@U2@@QAE@XZ 10020810     U2Lang:U2Lang.dll
 0002:00000814       __imp_??0Dataset@U2@@QAE@ABV01@@Z 10020814     U2Lang:U2Lang.dll
 0002:00000818       __imp_?URL_DATASETS_TYPE@BaseTypes@U2@@SA?AV?$QExplicitlySharedDataPointer@VDataType@U2@@@@XZ 10020818     U2Lang:U2Lang.dll
 0002:0000081c       __imp_?NUM_TYPE@BaseTypes@U2@@SA?AV?$QExplicitlySharedDataPointer@VDataType@U2@@@@XZ 1002081c     U2Lang:U2Lang.dll
 0002:00000820       __imp_?STRING_TYPE@BaseTypes@U2@@SA?AV?$QExplicitlySharedDataPointer@VDataType@U2@@@@XZ 10020820     U2Lang:U2Lang.dll
 0002:00000824       __imp_?URL_SLOT@BaseSlots@Workflow@U2@@SA?BVDescriptor@3@XZ 10020824     U2Lang:U2Lang.dll
 0002:00000828       __imp_?unregisterProto@ActorPrototypeRegistry@Workflow@U2@@QAEPAVActorPrototype@23@ABVQString@@@Z 10020828     U2Lang:U2Lang.dll
 0002:0000082c       __imp_?registerProto@ActorPrototypeRegistry@Workflow@U2@@QAE_NABVDescriptor@3@PAVActorPrototype@23@@Z 1002082c     U2Lang:U2Lang.dll
 0002:00000830       __imp_?addExternalTool@ActorPrototype@Workflow@U2@@QAEXABVQString@@0@Z 10020830     U2Lang:U2Lang.dll
 0002:00000834       __imp_?setPrompter@ActorPrototype@Workflow@U2@@QAEXPAVPrompter@23@@Z 10020834     U2Lang:U2Lang.dll
 0002:00000838       __imp_?setValidator@ActorPrototype@Workflow@U2@@QAEXPAVConfigurationValidator@3@@Z 10020838     U2Lang:U2Lang.dll
 0002:0000083c       __imp_?setEditor@ActorPrototype@Workflow@U2@@QAEXPAVConfigurationEditor@3@@Z 1002083c     U2Lang:U2Lang.dll
 0002:00000840       __imp_??1ActorPrototype@Workflow@U2@@UAE@XZ 10020840     U2Lang:U2Lang.dll
 0002:00000844       __imp_??0ActorPrototype@Workflow@U2@@QAE@ABVDescriptor@2@ABV?$QList@PAVPortDescriptor@Workflow@U2@@@@ABV?$QList@PAVAttribute@U2@@@@@Z 10020844     U2Lang:U2Lang.dll
 0002:00000848       __imp_??1PortDescriptor@Workflow@U2@@UAE@XZ 10020848     U2Lang:U2Lang.dll
 0002:0000084c       __imp_??0PortDescriptor@Workflow@U2@@QAE@ABVDescriptor@2@V?$QExplicitlySharedDataPointer@VDataType@U2@@@@_N2I@Z 1002084c     U2Lang:U2Lang.dll
 0002:00000850       __imp_?staticMetaObject@PrompterBaseImpl@U2@@2UQMetaObject@@B 10020850     U2Lang:U2Lang.dll
 0002:00000854       \177U2Lang_NULL_THUNK_DATA 10020854     U2Lang:U2Lang.dll
 0002:00000858       __imp_?staticMetaObject@XMLTestFormat@U2@@2UQMetaObject@@B 10020858     U2Test:U2Test.dll
 0002:0000085c       __imp_??0XMLTestFactory@U2@@QAE@ABVQString@@@Z 1002085c     U2Test:U2Test.dll
 0002:00000860       __imp_??1XMLTestFactory@U2@@UAE@XZ 10020860     U2Test:U2Test.dll
 0002:00000864       __imp_??0XmlTest@U2@@QAE@ABVQString@@PAVGTest@1@PBVGTestEnvironment@1@V?$QFlags@W4TaskFlag@U2@@@@ABV?$QList@PAVGTest@U2@@@@@Z 10020864     U2Test:U2Test.dll
 0002:00000868       __imp_?checkNecessaryAttributeExistence@XmlTest@U2@@QAEXABVQDomElement@@ABVQString@@@Z 10020868     U2Test:U2Test.dll
 0002:0000086c       __imp_??1XmlTest@U2@@UAE@XZ 1002086c     U2Test:U2Test.dll
 0002:00000870       __imp_?replacePrefix@XMLTestUtils@U2@@SAXPBVGTestEnvironment@2@AAVQString@@@Z 10020870     U2Test:U2Test.dll
 0002:00000874       __imp_?metaObject@GTest@U2@@UBEPBUQMetaObject@@XZ 10020874     U2Test:U2Test.dll
 0002:00000878       __imp_?qt_metacall@GTest@U2@@UAEHW4Call@QMetaObject@@HPAPAX@Z 10020878     U2Test:U2Test.dll
 0002:0000087c       __imp_?qt_metacast@GTest@U2@@UAEPAXPBD@Z 1002087c     U2Test:U2Test.dll
 0002:00000880       __imp_?findFormat@GTestFormatRegistry@U2@@QAEPAVGTestFormat@2@ABVQString@@@Z 10020880     U2Test:U2Test.dll
 0002:00000884       \177U2Test_NULL_THUNK_DATA 10020884     U2Test:U2Test.dll
 0002:00000888       __imp_?getBaseFileNameWithSuffixes@NgsReadsClassificationUtils@U2@@SA?AVQString@@ABV3@ABVQStringList@@0_N@Z 10020888     ngs_reads_classification:ngs_reads_classification.dll
 0002:0000088c       __imp_??1DatabaseDelegate@LocalWorkflow@U2@@UAE@XZ 1002088c     ngs_reads_classification:ngs_reads_classification.dll
 0002:00000890       __imp_??0DatabaseDelegate@LocalWorkflow@U2@@QAE@ABVQString@@0ABV?$QList@U?$QPair@VQString@@V1@@@@@0_N@Z 10020890     ngs_reads_classification:ngs_reads_classification.dll
 0002:00000894       __imp_?TAXONOMY_CLASSIFICATION_TYPE@TaxonomySupport@LocalWorkflow@U2@@SA?AV?$QExplicitlySharedDataPointer@VDataType@U2@@@@XZ 10020894     ngs_reads_classification:ngs_reads_classification.dll
 0002:00000898       __imp_?TAXONOMY_CLASSIFICATION_SLOT@TaxonomySupport@LocalWorkflow@U2@@SA?BVDescriptor@3@XZ 10020898     ngs_reads_classification:ngs_reads_classification.dll
 0002:0000089c       __imp_?WORKFLOW_ELEMENTS_GROUP@NgsReadsClassificationPlugin@U2@@2VQString@@B 1002089c     ngs_reads_classification:ngs_reads_classification.dll
 0002:000008a0       __imp_?TAXON_TAXDUMP_ITEM_ID@NgsReadsClassificationPlugin@U2@@2VQString@@B 100208a0     ngs_reads_classification:ngs_reads_classification.dll
 0002:000008a4       __imp_?TAXON_NUCL_WGS_ACCESSION_2_TAXID_ITEM_ID@NgsReadsClassificationPlugin@U2@@2VQString@@B 100208a4     ngs_reads_classification:ngs_reads_classification.dll
 0002:000008a8       __imp_?TAXON_NUCL_GB_ACCESSION_2_TAXID_ITEM_ID@NgsReadsClassificationPlugin@U2@@2VQString@@B 100208a8     ngs_reads_classification:ngs_reads_classification.dll
 0002:000008ac       __imp_?TAXON_MERGED_ITEM_ID@NgsReadsClassificationPlugin@U2@@2VQString@@B 100208ac     ngs_reads_classification:ngs_reads_classification.dll
 0002:000008b0       __imp_?countClassified@NgsReadsClassificationUtils@U2@@SAHABV?$QMap@VQString@@I@@@Z 100208b0     ngs_reads_classification:ngs_reads_classification.dll
 0002:000008b4       __imp_?TAXON_NODES_ITEM_ID@NgsReadsClassificationPlugin@U2@@2VQString@@B 100208b4     ngs_reads_classification:ngs_reads_classification.dll
 0002:000008b8       __imp_?TAXONOMY_DATA_ID@NgsReadsClassificationPlugin@U2@@2VQString@@B 100208b8     ngs_reads_classification:ngs_reads_classification.dll
 0002:000008bc       __imp_?setModelData@GenomicLibraryDelegate@LocalWorkflow@U2@@UBEXPAVQWidget@@PAVQAbstractItemModel@@ABVQModelIndex@@@Z 100208bc     ngs_reads_classification:ngs_reads_classification.dll
 0002:000008c0       __imp_?setEditorData@GenomicLibraryDelegate@LocalWorkflow@U2@@UBEXPAVQWidget@@ABVQModelIndex@@@Z 100208c0     ngs_reads_classification:ngs_reads_classification.dll
 0002:000008c4       __imp_?qt_metacast@GenomicLibraryDelegate@LocalWorkflow@U2@@UAEPAXPBD@Z 100208c4     ngs_reads_classification:ngs_reads_classification.dll
 0002:000008c8       __imp_?qt_metacall@GenomicLibraryDelegate@LocalWorkflow@U2@@UAEHW4Call@QMetaObject@@HPAPAX@Z 100208c8     ngs_reads_classification:ngs_reads_classification.dll
 0002:000008cc       __imp_?metaObject@GenomicLibraryDelegate@LocalWorkflow@U2@@UBEPBUQMetaObject@@XZ 100208cc     ngs_reads_classification:ngs_reads_classification.dll
 0002:000008d0       __imp_?getDisplayValue@GenomicLibraryDelegate@LocalWorkflow@U2@@UBE?AVQVariant@@ABV4@@Z 100208d0     ngs_reads_classification:ngs_reads_classification.dll
 0002:000008d4       __imp_?createWizardWidget@GenomicLibraryDelegate@LocalWorkflow@U2@@UBEPAVPropertyWidget@3@AAVU2OpStatus@3@PAVQWidget@@@Z 100208d4     ngs_reads_classification:ngs_reads_classification.dll
 0002:000008d8       __imp_?createEditor@GenomicLibraryDelegate@LocalWorkflow@U2@@UBEPAVQWidget@@PAV4@ABVQStyleOptionViewItem@@ABVQModelIndex@@@Z 100208d8     ngs_reads_classification:ngs_reads_classification.dll
 0002:000008dc       __imp_?update@DatabaseDelegate@LocalWorkflow@U2@@UAEXXZ 100208dc     ngs_reads_classification:ngs_reads_classification.dll
 0002:000008e0       __imp_?CLARK_VIRAL_DATABASE_DATA_ID@NgsReadsClassificationPlugin@U2@@2VQString@@B 100208e0     ngs_reads_classification:ngs_reads_classification.dll
 0002:000008e4       __imp_?CLARK_VIRAL_DATABASE_ITEM_ID@NgsReadsClassificationPlugin@U2@@2VQString@@B 100208e4     ngs_reads_classification:ngs_reads_classification.dll
 0002:000008e8       __imp_?CLARK_BACTERIAL_VIRAL_DATABASE_DATA_ID@NgsReadsClassificationPlugin@U2@@2VQString@@B 100208e8     ngs_reads_classification:ngs_reads_classification.dll
 0002:000008ec       __imp_?CLARK_BACTERIAL_VIRAL_DATABASE_ITEM_ID@NgsReadsClassificationPlugin@U2@@2VQString@@B 100208ec     ngs_reads_classification:ngs_reads_classification.dll
 0002:000008f0       __imp_?REFSEQ_BACTERIAL_DATA_ID@NgsReadsClassificationPlugin@U2@@2VQString@@B 100208f0     ngs_reads_classification:ngs_reads_classification.dll
 0002:000008f4       __imp_?REFSEQ_VIRAL_DATA_ID@NgsReadsClassificationPlugin@U2@@2VQString@@B 100208f4     ngs_reads_classification:ngs_reads_classification.dll
 0002:000008f8       __imp_?WORKFLOW_CLASSIFY_TOOL_ID@NgsReadsClassificationPlugin@U2@@2VQString@@B 100208f8     ngs_reads_classification:ngs_reads_classification.dll
 0002:000008fc       __imp_?UNCLASSIFIED_ID@TaxonomyTree@LocalWorkflow@U2@@2IB 100208fc     ngs_reads_classification:ngs_reads_classification.dll
 0002:00000900       __imp_?TAXONOMY_CLASSIFICATION_SLOT_ID@TaxonomySupport@LocalWorkflow@U2@@2VQString@@B 10020900     ngs_reads_classification:ngs_reads_classification.dll
 0002:00000904       __imp_?CLASSIFICATION_SUFFIX@NgsReadsClassificationUtils@U2@@2VQString@@B 10020904     ngs_reads_classification:ngs_reads_classification.dll
 0002:00000908       __imp_?TAXON_NAMES_ITEM_ID@NgsReadsClassificationPlugin@U2@@2VQString@@B 10020908     ngs_reads_classification:ngs_reads_classification.dll
 0002:0000090c       __imp_?clone@GenomicLibraryDelegate@LocalWorkflow@U2@@UAEPAVPropertyDelegate@3@XZ 1002090c     ngs_reads_classification:ngs_reads_classification.dll
 0002:00000910       __imp_??0GenomicLibraryDelegate@LocalWorkflow@U2@@QAE@PAVQObject@@@Z 10020910     ngs_reads_classification:ngs_reads_classification.dll
 0002:00000914       \177ngs_reads_classification_NULL_THUNK_DATA 10020914     ngs_reads_classification:ngs_reads_classification.dll
 0002:00000918       ___xc_a                    10020918     MSVCRT:cinitexe.obj
 0002:00000b58       ___xc_z                    10020b58     MSVCRT:cinitexe.obj
 0002:00000b5c       ___xi_a                    10020b5c     MSVCRT:cinitexe.obj
 0002:00000b68       ___xi_z                    10020b68     MSVCRT:cinitexe.obj
 0002:00000ba8       ??_C@_00CNPNBAHC@?$AA@     10020ba8     ClarkBuildWorker.obj
 0002:00000bb0       ??_7error_category@std@@6B@ 10020bb0     ClarkBuildWorker.obj
 0002:00000bcc       ??_7_Generic_error_category@std@@6B@ 10020bcc     ClarkBuildWorker.obj
 0002:00000be4       ??_C@_07DCLBNMLN@generic?$AA@ 10020be4     ClarkBuildWorker.obj
 0002:00000bec       ??_C@_0O@BFJCFAAK@unknown?5error?$AA@ 10020bec     ClarkBuildWorker.obj
 0002:00000c00       ??_7_Iostream_error_category@std@@6B@ 10020c00     ClarkBuildWorker.obj
 0002:00000c18       ??_C@_08LLGCOLLL@iostream?$AA@ 10020c18     ClarkBuildWorker.obj
 0002:00000c24       ??_C@_0BG@PADBLCHM@iostream?5stream?5error?$AA@ 10020c24     ClarkBuildWorker.obj
 0002:00000c40       ??_7_System_error_category@std@@6B@ 10020c40     ClarkBuildWorker.obj
 0002:00000c58       ??_C@_06FHFOAHML@system?$AA@ 10020c58     ClarkBuildWorker.obj
 0002:00000c60       ??_C@_0L@JLHNEGIN@Algorithms?$AA@ 10020c60     ClarkBuildWorker.obj
 0002:00000c6c       ??_C@_07PGLPGHFC@Console?$AA@ 10020c6c     ClarkBuildWorker.obj
 0002:00000c74       ??_C@_0O@BOFHOPCF@Core?5Services?$AA@ 10020c74     ClarkBuildWorker.obj
 0002:00000c84       ??_C@_0N@PPADAKBM@Input?1Output?$AA@ 10020c84     ClarkBuildWorker.obj
 0002:00000c94       ??_C@_0M@KPPBKPKK@Performance?$AA@ 10020c94     ClarkBuildWorker.obj
 0002:00000ca0       ??_C@_07BFDHHBBI@Scripts?$AA@ 10020ca0     ClarkBuildWorker.obj
 0002:00000ca8       ??_C@_05EEGKELMG@Tasks?$AA@ 10020ca8     ClarkBuildWorker.obj
 0002:00000cb0       ??_C@_0P@NIIOBHGA@User?5Interface?$AA@ 10020cb0     ClarkBuildWorker.obj
 0002:00000cc0       ??_C@_0N@JINCGGMN@User?5Actions?$AA@ 10020cc0     ClarkBuildWorker.obj
 0002:00000cd4       ??_SFailTask@U2@@6B@       10020cd4     ClarkBuildWorker.obj
 0002:00000d64       ??_STaskSignalMapper@U2@@6B@ 10020d64     ClarkBuildWorker.obj
 0002:00000d94       ??_SDescriptor@U2@@6B@     10020d94     ClarkBuildWorker.obj
 0002:00000da4       ??_SMapDataType@U2@@6B@    10020da4     ClarkBuildWorker.obj
 0002:00000dc4       ??_SAttribute@U2@@6B@      10020dc4     ClarkBuildWorker.obj
 0002:00000df4       ??_C@_0BF@COKBMJP@Script?5task?5canceled?$AA@ 10020df4     ClarkBuildWorker.obj
 0002:00000e14       ??_SDelegateEditor@U2@@6B@ 10020e14     ClarkBuildWorker.obj
 0002:00000e6c       ??_SURLDelegate@U2@@6B@    10020e6c     ClarkBuildWorker.obj
 0002:00000eec       ??_SComboBoxDelegate@U2@@6B@ 10020eec     ClarkBuildWorker.obj
 0002:00000f6c       ??_SPortDescriptor@Workflow@U2@@6B@ 10020f6c     ClarkBuildWorker.obj
 0002:00000f80       ??_C@_0BD@FOHBGHEI@QList?$DMU2?3?3Dataset?$DO?$AA@ 10020f80     ClarkBuildWorker.obj
 0002:00000f98       ??_SIntegralBusActorPrototype@Workflow@U2@@6BQObject@@@ 10020f98     ClarkBuildWorker.obj
 0002:00000fd4       ??_SIntegralBusActorPrototype@Workflow@U2@@6BVisualDescriptor@2@@ 10020fd4     ClarkBuildWorker.obj
 0002:00000fe4       ??_SExternalToolRunTask@U2@@6B@ 10020fe4     ClarkBuildWorker.obj
 0002:00001074       ??_7ClarkBuildValidator@LocalWorkflow@U2@@6B@ 10021074     ClarkBuildWorker.obj
 0002:00001080       ??_C@_0BE@JJKHOKLC@ClarkBuildValidator?$AA@ 10021080     ClarkBuildWorker.obj
 0002:00001098       ??_7?$PrompterBase@VClarkBuildPrompter@LocalWorkflow@U2@@@U2@@6BActorDocument@Workflow@1@@ 10021098     ClarkBuildWorker.obj
 0002:000010e0       ??_7?$PrompterBase@VClarkBuildPrompter@LocalWorkflow@U2@@@U2@@6BPrompter@Workflow@1@@ 100210e0     ClarkBuildWorker.obj
 0002:000010ec       ??_7ClarkBuildPrompter@LocalWorkflow@U2@@6BActorDocument@Workflow@2@@ 100210ec     ClarkBuildWorker.obj
 0002:00001134       ??_7ClarkBuildPrompter@LocalWorkflow@U2@@6BPrompter@Workflow@2@@ 10021134     ClarkBuildWorker.obj
 0002:00001140       ??_7ClarkBuildWorker@LocalWorkflow@U2@@6BQObject@@@ 10021140     ClarkBuildWorker.obj
 0002:00001184       ??_7ClarkBuildWorker@LocalWorkflow@U2@@6BWorker@Workflow@2@@ 10021184     ClarkBuildWorker.obj
 0002:000011a0       ??_7ClarkBuildWorker@LocalWorkflow@U2@@6BCommunicationSubject@Workflow@2@@ 100211a0     ClarkBuildWorker.obj
 0002:000011b0       ??_7ClarkBuildWorkerFactory@LocalWorkflow@U2@@6B?$IdRegistry@VDomainFactory@Workflow@U2@@@2@@ 100211b0     ClarkBuildWorker.obj
 0002:000011dc       ??_7ClarkBuildWorkerFactory@LocalWorkflow@U2@@6BDescriptor@2@@ 100211dc     ClarkBuildWorker.obj
 0002:000011ec       ??_7ClarkBuildTask@LocalWorkflow@U2@@6B@ 100211ec     ClarkBuildWorker.obj
 0002:00001284       ??_SGenomicLibraryDelegate@LocalWorkflow@U2@@6B@ 10021284     ClarkBuildWorker.obj
 0002:00001300       ??_C@_0M@DAMPAGLL@clark?9build?$AA@ 10021300     ClarkBuildWorker.obj
 0002:0000130c       ??_C@_03KEJHNBPP@out?$AA@  1002130c     ClarkBuildWorker.obj
 0002:00001310       ??_C@_08PBOCEOLL@database?$AA@ 10021310     ClarkBuildWorker.obj
 0002:0000131c       ??_C@_0BA@GJNMLPPF@genomic?9library?$AA@ 1002131c     ClarkBuildWorker.obj
 0002:0000132c       ??_C@_0O@OOJIBHAK@taxonomy?9rank?$AA@ 1002132c     ClarkBuildWorker.obj
 0002:0000133c       ??_C@_0DP@GEFKKLJH@Taxonomy?5classification?5data?5fro@ 1002133c     ClarkBuildWorker.obj
 0002:00001380       ??_C@_0EL@ENMJCHGK@Taxonomy?5classification?5data?5fro@ 10021380     ClarkBuildWorker.obj
 0002:000013cc       ??_C@_0CM@NEMEONHO@Use?5custom?5data?5to?5build?5?$CF1?5CLAR@ 100213cc     ClarkBuildWorker.obj
 0002:000013f8       ??_C@_0LD@GKFMOAGM@Build?5a?5CLARK?5database?5from?5a?5se@ 100213f8     ClarkBuildWorker.obj
 0002:000014ac       ??_C@_0BF@MDPJABIP@Build?5CLARK?5Database?$AA@ 100214ac     ClarkBuildWorker.obj
 0002:000014c4       ??_C@_0CL@BIBEPGLJ@URL?5to?5the?5folder?5with?5the?5CLARK@ 100214c4     ClarkBuildWorker.obj
 0002:000014f0       ??_C@_0BG@GCKNDNLF@Output?5CLARK?5database?$AA@ 100214f0     ClarkBuildWorker.obj
 0002:00001508       ??_C@_0M@FOOCJNHH@Output?5URL?4?$AA@ 10021508     ClarkBuildWorker.obj
 0002:00001514       ??_C@_0L@OALCHELH@Output?5URL?$AA@ 10021514     ClarkBuildWorker.obj
 0002:00001520       ??_C@_0N@POIOLIAN@clark?4db?9url?$AA@ 10021520     ClarkBuildWorker.obj
 0002:00001530       ??_C@_0DK@DGGMNDLJ@A?5folder?5that?5should?5be?5used?5to?5@ 10021530     ClarkBuildWorker.obj
 0002:0000156c       ??_C@_08HDBDMMBI@Database?$AA@ 1002156c     ClarkBuildWorker.obj
 0002:00001578       ??_C@_0BCO@POALJIID@Genomes?5that?5should?5be?5used?5to?5b@ 10021578     ClarkBuildWorker.obj
 0002:000016a8       ??_C@_0BA@IPKMCDNP@Genomic?5library?$AA@ 100216a8     ClarkBuildWorker.obj
 0002:000016b8       ??_C@_0BEA@JBDPFGG@Set?5the?5taxonomy?5rank?5for?5the?5da@ 100216b8     ClarkBuildWorker.obj
 0002:000017f8       ??_C@_0O@JPGCHMAM@Taxonomy?5rank?$AA@ 100217f8     ClarkBuildWorker.obj
 0002:00001808       ??_C@_07CHJHAMJL@Species?$AA@ 10021808     ClarkBuildWorker.obj
 0002:00001810       ??_C@_05IAGDJMAL@Genus?$AA@ 10021810     ClarkBuildWorker.obj
 0002:00001818       ??_C@_06BOFMEHLD@Family?$AA@ 10021818     ClarkBuildWorker.obj
 0002:00001820       ??_C@_05NEHACHKB@Order?$AA@ 10021820     ClarkBuildWorker.obj
 0002:00001828       ??_C@_05EKAMNAII@Class?$AA@ 10021828     ClarkBuildWorker.obj
 0002:00001830       ??_C@_06KCLKDBFF@Phylum?$AA@ 10021830     ClarkBuildWorker.obj
 0002:00001838       ??_C@_0P@ODOEDNPN@clark?1database?$AA@ 10021838     ClarkBuildWorker.obj
 0002:00001848       ??_C@_0CK@IGBIANDN@Trying?5to?5recover?5from?5error?3?5?$CF1@ 10021848     ClarkBuildWorker.obj
 0002:00001874       ??_C@_0BK@LMMJOEHE@Port?5with?5id?5?8?$CF1?8?5is?5NULL?$AA@ 10021874     ClarkBuildWorker.obj
 0002:00001890       ??_C@_0BJ@KMJEHCJO@src?2ClarkBuildWorker?4cpp?$AA@ 10021890     ClarkBuildWorker.obj
 0002:000018ac       ??_C@_0DK@FGLPPHNF@Taxonomy?5classification?5data?5fro@ 100218ac     ClarkBuildWorker.obj
 0002:000018e8       ??_C@_0BJ@JJNIMNNJ@1sl_taskFinished?$CITask?5?$CK?$CJ?$AA@ 100218e8     ClarkBuildWorker.obj
 0002:00001904       ??_C@_0BJ@DHBKDAMN@2si_taskFinished?$CITask?5?$CK?$CJ?$AA@ 10021904     ClarkBuildWorker.obj
 0002:00001920       ??_C@_0BM@NNFFHGNB@Invalid?5task?5is?5encountered?$AA@ 10021920     ClarkBuildWorker.obj
 0002:0000193c       ??_C@_09DMOIMEE@Dataset?51?$AA@ 1002193c     ClarkBuildWorker.obj
 0002:00001948       ??_C@_0BF@LGOOHNFD@Built?5Clark?5database?$AA@ 10021948     ClarkBuildWorker.obj
 0002:00001960       ??_C@_0BF@KBLPOECO@Build?5Clark?5database?$AA@ 10021960     ClarkBuildWorker.obj
 0002:00001978       ??_C@_0P@JDHIOCJG@ClarkBuildTask?$AA@ 10021978     ClarkBuildWorker.obj
 0002:00001988       ??_C@_0CA@IIGHEGJE@CLARK?5database?5URL?5is?5undefined?$AA@ 10021988     ClarkBuildWorker.obj
 0002:000019a8       ??_C@_0BJ@OLOJDBFM@Taxdata?5URL?5is?5undefined?$AA@ 100219a8     ClarkBuildWorker.obj
 0002:000019c4       ??_C@_0BN@JEFIPCNJ@Genomic?5library?5set?5is?5empty?$AA@ 100219c4     ClarkBuildWorker.obj
 0002:000019e8       ??_C@_0KG@CAMJPKK@Failed?5to?5recognize?5the?5rank?4?5Pl@ 100219e8     ClarkBuildWorker.obj
 0002:00001a94       ??_7ClarkBuildLogParser@LocalWorkflow@U2@@6B@ 10021a94     ClarkBuildWorker.obj
 0002:00001adc       ??_C@_05BBAEEBBH@abort?$AA@ 10021adc     ClarkBuildWorker.obj
 0002:00001ae4       ??_C@_0M@GEPCFGAC@core?5dumped?$AA@ 10021ae4     ClarkBuildWorker.obj
 0002:00001af0       ??_C@_06EKNFNOKI@custom?$AA@ 10021af0     ClarkBuildWorker.obj
 0002:00001af8       ??_C@_08IAAECIGO@?1?4custom?$AA@ 10021af8     ClarkBuildWorker.obj
 0002:00001b04       ??_C@_0DC@GEFEMIEA@Failed?5to?5create?5folder?5for?5CLAR@ 10021b04     ClarkBuildWorker.obj
 0002:00001b38       ??_C@_01EEMJAFIK@?6?$AA@   10021b38     ClarkBuildWorker.obj
 0002:00001b3c       ??_C@_0BE@LGBLLFOL@1sl_actorModified?$CI?$CJ?$AA@ 10021b3c     ClarkBuildWorker.obj
 0002:00001b50       ??_C@_0BD@FGIDJNMI@2si_labelChanged?$CI?$CJ?$AA@ 10021b50     ClarkBuildWorker.obj
 0002:00001b64       ??_C@_0P@DIBOLHGA@2si_modified?$CI?$CJ?$AA@ 10021b64     ClarkBuildWorker.obj
 0002:00001b74       ??_C@_0BC@HBGBGNIM@2bindingChanged?$CI?$CJ?$AA@ 10021b74     ClarkBuildWorker.obj
 0002:00001b88       ??_C@_0BA@JFNIOLAK@string?5too?5long?$AA@ 10021b88     ClarkBuildWorker.obj
 0002:00001b98       ??_C@_0BI@CFPLBAOH@invalid?5string?5position?$AA@ 10021b98     ClarkBuildWorker.obj
 0002:00001bb0       __real@3ff0000000000000    10021bb0     ClarkBuildWorker.obj
 0002:00001bb8       ??_C@_07DLHCIBDH@default?$AA@ 10021bb8     ClarkClassifyWorker.obj
 0002:00001bc0       ??_C@_0CM@ICPJCNAJ@QtMetaTypePrivate?3?3QAssociativeI@ 10021bc0     ClarkClassifyWorker.obj
 0002:00001bf0       ??_SVisibilityRelation@U2@@6B@ 10021bf0     ClarkClassifyWorker.obj
 0002:00001c0c       ??_SSlotRelationDescriptor@U2@@6B@ 10021c0c     ClarkClassifyWorker.obj
 0002:00001c1c       ??_SSpinBoxDelegate@U2@@6B@ 10021c1c     ClarkClassifyWorker.obj
 0002:00001c9c       ??_SPairedReadsPortValidator@Workflow@U2@@6B@ 10021c9c     ClarkClassifyWorker.obj
 0002:00001ca8       ??_C@_0DA@ENPGIFBJ@U2?3?3LocalWorkflow?3?3TaxonomyClass@ 10021ca8     ClarkClassifyWorker.obj
 0002:00001cdc       ??_7?$PrompterBase@VClarkClassifyPrompter@LocalWorkflow@U2@@@U2@@6BActorDocument@Workflow@1@@ 10021cdc     ClarkClassifyWorker.obj
 0002:00001d24       ??_7?$PrompterBase@VClarkClassifyPrompter@LocalWorkflow@U2@@@U2@@6BPrompter@Workflow@1@@ 10021d24     ClarkClassifyWorker.obj
 0002:00001d30       ??_7ClarkClassifyPrompter@LocalWorkflow@U2@@6BActorDocument@Workflow@2@@ 10021d30     ClarkClassifyWorker.obj
 0002:00001d78       ??_7ClarkClassifyPrompter@LocalWorkflow@U2@@6BPrompter@Workflow@2@@ 10021d78     ClarkClassifyWorker.obj
 0002:00001d84       ??_7ClarkClassifyWorker@LocalWorkflow@U2@@6BQObject@@@ 10021d84     ClarkClassifyWorker.obj
 0002:00001dc8       ??_7ClarkClassifyWorker@LocalWorkflow@U2@@6BWorker@Workflow@2@@ 10021dc8     ClarkClassifyWorker.obj
 0002:00001de4       ??_7ClarkClassifyWorker@LocalWorkflow@U2@@6BCommunicationSubject@Workflow@2@@ 10021de4     ClarkClassifyWorker.obj
 0002:00001df4       ??_7ClarkClassifyValidator@LocalWorkflow@U2@@6B@ 10021df4     ClarkClassifyWorker.obj
 0002:00001e00       ??_C@_0BH@OBMBIJLA@ClarkClassifyValidator?$AA@ 10021e00     ClarkClassifyWorker.obj
 0002:00001e1c       ??_7ClarkClassifyWorkerFactory@LocalWorkflow@U2@@6B?$IdRegistry@VDomainFactory@Workflow@U2@@@2@@ 10021e1c     ClarkClassifyWorker.obj
 0002:00001e48       ??_7ClarkClassifyWorkerFactory@LocalWorkflow@U2@@6BDescriptor@2@@ 10021e48     ClarkClassifyWorker.obj
 0002:00001e58       ??_7ClarkLogParser@LocalWorkflow@U2@@6B@ 10021e58     ClarkClassifyWorker.obj
 0002:00001ea4       ??_7ClarkClassifyTask@LocalWorkflow@U2@@6B@ 10021ea4     ClarkClassifyWorker.obj
 0002:00001f3c       ??_SDatabaseDelegate@LocalWorkflow@U2@@6B@ 10021f3c     ClarkClassifyWorker.obj
 0002:00001fb8       ??_C@_0DP@HCLBAHHN@Classify?5sequences?5from?5?$DMu?$DO?$CF1?$DM?1u@ 10021fb8     ClarkClassifyWorker.obj
 0002:00001ff8       ??_C@_0EG@CCIHHMEA@Classify?5paired?9end?5reads?5from?5?$DM@ 10021ff8     ClarkClassifyWorker.obj
 0002:00002040       ??_C@_0CH@HBJABOBI@The?5database?5folder?5doesn?8t?5exis@ 10022040     ClarkClassifyWorker.obj
 0002:00002068       ??_C@_0M@HOAFHFBH@targets?4txt?$AA@ 10022068     ClarkClassifyWorker.obj
 0002:00002074       ??_C@_0BK@BKOIFCMH@?4custom?4fileToAccssnTaxID?$AA@ 10022074     ClarkClassifyWorker.obj
 0002:00002090       ??_C@_0BF@BPLGEKKM@?4custom?4fileToTaxIDs?$AA@ 10022090     ClarkClassifyWorker.obj
 0002:000020a8       ??_C@_01KMDKNFGN@?1?$AA@   100220a8     ClarkClassifyWorker.obj
 0002:000020ac       ??_C@_0CP@NMPMEACA@The?5mandatory?5database?5file?5does@ 100220ac     ClarkClassifyWorker.obj
 0002:000020e0       ??_C@_0GE@MNKFMMMF@Reference?5database?5for?5these?5CLA@ 100220e0     ClarkClassifyWorker.obj
 0002:00002144       ??_C@_0BF@CNHAAFPE@?$CK_m?$CF1_light_?$CF2?4tsk?4?$CK?$AA@ 10022144     ClarkClassifyWorker.obj
 0002:0000215c       ??_C@_0BG@OCHHLJI@?$CK_k?$CF1_t?$CK_s?$CK_m?$CF2?4tsk?4?$CK?$AA@ 1002215c     ClarkClassifyWorker.obj
 0002:00002174       ??_C@_0P@HCDCPDK@clark?9classify?$AA@ 10022174     ClarkClassifyWorker.obj
 0002:00002184       ??_C@_02LMMGJAGL@in?$AA@   10022184     ClarkClassifyWorker.obj
 0002:00002188       ??_C@_03DHKMCKDB@in2?$AA@  10022188     ClarkClassifyWorker.obj
 0002:0000218c       ??_C@_0L@LGHLPLD@reads?9url1?$AA@ 1002218c     ClarkClassifyWorker.obj
 0002:00002198       ??_C@_0L@CAEKOMHA@reads?9url2?$AA@ 10022198     ClarkClassifyWorker.obj
 0002:000021a4       ??_C@_0N@LEPPBDOM@tool?9variant?$AA@ 100221a4     ClarkClassifyWorker.obj
 0002:000021b4       ??_C@_0L@JDEFPCKN@output?9url?$AA@ 100221b4     ClarkClassifyWorker.obj
 0002:000021c0       ??_C@_08HFGIEONL@taxonomy?$AA@ 100221c0     ClarkClassifyWorker.obj
 0002:000021cc       ??_C@_08MPLDBMGC@k?9length?$AA@ 100221cc     ClarkClassifyWorker.obj
 0002:000021d8       ??_C@_0L@PAGBIALK@k?9min?9freq?$AA@ 100221d8     ClarkClassifyWorker.obj
 0002:000021e4       ??_C@_04GMGOKAFF@mode?$AA@ 100221e4     ClarkClassifyWorker.obj
 0002:000021ec       ??_C@_06CNBACIJO@factor?$AA@ 100221ec     ClarkClassifyWorker.obj
 0002:000021f4       ??_C@_03BOGADHLI@gap?$AA@  100221f4     ClarkClassifyWorker.obj
 0002:000021f8       ??_C@_0L@GOLAONFO@extend?9out?$AA@ 100221f8     ClarkClassifyWorker.obj
 0002:00002204       ??_C@_07GCEAJMEA@preload?$AA@ 10022204     ClarkClassifyWorker.obj
 0002:0000220c       ??_C@_07NFPADACG@threads?$AA@ 1002220c     ClarkClassifyWorker.obj
 0002:00002214       ??_C@_0BB@JKLNDIAA@sequencing?9reads?$AA@ 10022214     ClarkClassifyWorker.obj
 0002:00002228       ??_C@_0L@PCJLLKLK@single?9end?$AA@ 10022228     ClarkClassifyWorker.obj
 0002:00002234       ??_C@_0L@HGFAFILP@paired?9end?$AA@ 10022234     ClarkClassifyWorker.obj
 0002:00002240       ??_C@_05FOPMAJO@CLARK?$AA@ 10022240     ClarkClassifyWorker.obj
 0002:00002248       ??_C@_0BBK@MJDNBFJA@CLARK?5?$CICLAssifier?5based?5on?5Reduc@ 10022248     ClarkClassifyWorker.obj
 0002:00002364       ??_C@_0BO@PHEFLGFI@Classify?5Sequences?5with?5CLARK?$AA@ 10022364     ClarkClassifyWorker.obj
 0002:00002388       ??_C@_0BAF@MDCIJEPN@URL?$CIs?$CJ?5to?5FASTQ?5or?5FASTA?5file?$CIs?$CJ@ 10022388     ClarkClassifyWorker.obj
 0002:00002490       ??_C@_0BA@GLOOOALC@Input?5sequences?$AA@ 10022490     ClarkClassifyWorker.obj
 0002:000024a0       ??_C@_0EP@CDJOEIFJ@A?5map?5of?5sequence?5names?5with?5the@ 100224a0     ClarkClassifyWorker.obj
 0002:000024f0       ??_C@_0BF@PPKGPAJP@CLARK?5Classification?$AA@ 100224f0     ClarkClassifyWorker.obj
 0002:00002508       ??_C@_0N@JCLPICJJ@Input?5URL?51?4?$AA@ 10022508     ClarkClassifyWorker.obj
 0002:00002518       ??_C@_0M@LBNKAPAD@Input?5URL?51?$AA@ 10022518     ClarkClassifyWorker.obj
 0002:00002524       ??_C@_0N@JAPJDMMA@Input?5URL?52?4?$AA@ 10022524     ClarkClassifyWorker.obj
 0002:00002534       ??_C@_0M@JKPHFMMA@Input?5URL?52?$AA@ 10022534     ClarkClassifyWorker.obj
 0002:00002540       ??_C@_0M@IPENIMN@clark?4input?$AA@ 10022540     ClarkClassifyWorker.obj
 0002:0000254c       ??_C@_0N@GHNDANIA@clark?4output?$AA@ 1002254c     ClarkClassifyWorker.obj
 0002:00002560       ??_C@_0BKG@KKPIMLEG@Use?5CLARK?9l?5on?5workstations?5with@ 10022560     ClarkClassifyWorker.obj
 0002:00002708       ??_C@_0BE@BANMMFJF@Classification?5tool?$AA@ 10022708     ClarkClassifyWorker.obj
 0002:00002720       ??_C@_0OF@LCIJJFJL@A?5path?5to?5the?5folder?5with?5the?5CL@ 10022720     ClarkClassifyWorker.obj
 0002:00002808       ??_C@_0BO@FKBHNKFL@Specify?5the?5output?5file?5name?4?$AA@ 10022808     ClarkClassifyWorker.obj
 0002:00002828       ??_C@_0M@LEIJPAKP@Output?5file?$AA@ 10022828     ClarkClassifyWorker.obj
 0002:00002838       ??_C@_0CBB@NMHMIGLJ@Set?5the?5k?9mer?5length?5?$CI?9k?$CJ?4?$DMbr?$DO?$DMb@ 10022838     ClarkClassifyWorker.obj
 0002:00002a4c       ??_C@_0N@MNPMEPKA@K?9mer?5length?$AA@ 10022a4c     ClarkClassifyWorker.obj
 0002:00002a60       ??_C@_0MM@NICHJFGC@Minimum?5of?5k?9mer?5frequency?1occur@ 10022a60     ClarkClassifyWorker.obj
 0002:00002b2c       ??_C@_0BI@KNMOCBHI@Minimum?5k?9mer?5frequency?$AA@ 10022b2c     ClarkClassifyWorker.obj
 0002:00002b48       ??_C@_0BDC@PIIPGGO@Set?5the?5mode?5of?5the?5execution?5?$CI?9@ 10022b48     ClarkClassifyWorker.obj
 0002:00002c7c       ??_C@_04KNKPIPFB@Mode?$AA@ 10022c7c     ClarkClassifyWorker.obj
 0002:00002c88       ??_C@_0BFN@IKBKIOBK@Sample?5factor?5value?5?$CI?9s?$CJ?4?$DMbr?$DO?$DMbr@ 10022c88     ClarkClassifyWorker.obj
 0002:00002de8       ??_C@_0BG@DPIIMBJE@Sampling?5factor?5value?$AA@ 10022de8     ClarkClassifyWorker.obj
 0002:00002e00       ??_C@_0MG@NFAOFLIH@?$CCGap?$CC?5or?5number?5of?5non?9overlappi@ 10022e00     ClarkClassifyWorker.obj
 0002:00002ec8       ??_C@_03LOFCJIIG@Gap?$AA@  10022ec8     ClarkClassifyWorker.obj
 0002:00002ecc       ??_C@_0DN@FEHEOMLB@Request?5an?5extended?5output?5for?5t@ 10022ecc     ClarkClassifyWorker.obj
 0002:00002f0c       ??_C@_0BA@NIOFKLLM@Extended?5output?$AA@ 10022f0c     ClarkClassifyWorker.obj
 0002:00002f20       ??_C@_0BCG@GIEBFBOK@Request?5the?5loading?5of?5database?5@ 10022f20     ClarkClassifyWorker.obj
 0002:00003048       ??_C@_0BK@MBNCKPDD@Load?5database?5into?5memory?$AA@ 10023048     ClarkClassifyWorker.obj
 0002:00003068       ??_C@_0JF@MLAICDGO@Use?5multiple?5threads?5for?5the?5cla@ 10023068     ClarkClassifyWorker.obj
 0002:00003100       ??_C@_0BC@GJADDMKB@Number?5of?5threads?$AA@ 10023100     ClarkClassifyWorker.obj
 0002:00003118       ??_C@_0BIC@MFFKKPNE@To?5classify?5single?9end?5?$CISE?$CJ?5read@ 10023118     ClarkClassifyWorker.obj
 0002:0000329c       ??_C@_0L@DNPNCLBE@Input?5data?$AA@ 1002329c     ClarkClassifyWorker.obj
 0002:000032a8       ??_C@_0CA@BBFPBJKD@Classify?5tool?4?5Hidden?5attribute?$AA@ 100232a8     ClarkClassifyWorker.obj
 0002:000032c8       ??_C@_0BE@IHKBOJBH@SE?5reads?5or?5contigs?$AA@ 100232c8     ClarkClassifyWorker.obj
 0002:000032dc       ??_C@_08BKAKNCGK@PE?5reads?$AA@ 100232dc     ClarkClassifyWorker.obj
 0002:000032e8       ??_C@_07INHLJBND@CLARK?9l?$AA@ 100232e8     ClarkClassifyWorker.obj
 0002:000032f0       ??_C@_04LBDCJOFB@Auto?$AA@ 100232f0     ClarkClassifyWorker.obj
 0002:000032f8       ??_C@_03NIPKHAHH@csv?$AA@  100232f8     ClarkClassifyWorker.obj
 0002:000032fc       ??_C@_03NFABLNAL@CSV?$AA@  100232fc     ClarkClassifyWorker.obj
 0002:00003300       ??_C@_0N@KLHJANBO@clark?1output?$AA@ 10023300     ClarkClassifyWorker.obj
 0002:00003310       ??_C@_07CCOEHHFD@minimum?$AA@ 10023310     ClarkClassifyWorker.obj
 0002:00003318       ??_C@_07MEIENILC@maximum?$AA@ 10023318     ClarkClassifyWorker.obj
 0002:00003320       ??_C@_07MCAEODGB@Default?$AA@ 10023320     ClarkClassifyWorker.obj
 0002:00003328       ??_C@_04DKAKODEK@Full?$AA@ 10023328     ClarkClassifyWorker.obj
 0002:00003330       ??_C@_07PCEKDHDA@Express?$AA@ 10023330     ClarkClassifyWorker.obj
 0002:00003338       ??_C@_0BM@HEBJANCE@src?2ClarkClassifyWorker?4cpp?$AA@ 10023338     ClarkClassifyWorker.obj
 0002:00003358       ??_C@_0GE@EOBHNCHI@Unrecognized?5mode?5of?5execution?0?5@ 10023358     ClarkClassifyWorker.obj
 0002:000033bc       ??_C@_01IDAFKMJL@_?$AA@    100233bc     ClarkClassifyWorker.obj
 0002:000033c0       ??_C@_0N@GGPNLDAE@CLARK_?$CF1?4txt?$AA@ 100233c0     ClarkClassifyWorker.obj
 0002:000033d0       ??_C@_0CI@OHPCOEJH@CLARK?5worker?5is?5done?5as?5input?5ha@ 100233d0     ClarkClassifyWorker.obj
 0002:000033f8       ??_C@_0CC@CIANJNIC@CLARK?5produced?5classification?3?5?$CF@ 100233f8     ClarkClassifyWorker.obj
 0002:0000341c       ??_C@_0DF@GPCBDEIK@There?5were?5?$CF1?5input?5reads?0?5?$CF2?5re@ 1002341c     ClarkClassifyWorker.obj
 0002:00003454       ??_C@_0DD@LBOIMHHF@There?5is?5not?5enough?5memory?5?$CIRAM?$CJ@ 10023454     ClarkClassifyWorker.obj
 0002:00003488       ??_C@_0P@MKKIMBGC@std?3?3bad_alloc?$AA@ 10023488     ClarkClassifyWorker.obj
 0002:00003498       ??_C@_0HD@LPPMPLCO@CLARK?5process?5crashed?4?5It?5might?5@ 10023498     ClarkClassifyWorker.obj
 0002:0000350c       ??_C@_0BA@LNFPFBFA@Process?5crashed?$AA@ 1002350c     ClarkClassifyWorker.obj
 0002:0000351c       ??_C@_0L@GNIMMKCC@Object_ID?0?$AA@ 1002351c     ClarkClassifyWorker.obj
 0002:00003528       ??_C@_0EF@FIKGPPDN@?0Length?0Gamma?01st_assignment?0sco@ 10023528     ClarkClassifyWorker.obj
 0002:00003570       ??_C@_0BK@FGNLAOAM@Classify?5reads?5with?5Clark?$AA@ 10023570     ClarkClassifyWorker.obj
 0002:0000358c       ??_C@_0BC@CJEJDGNB@ClarkClassifyTask?$AA@ 1002358c     ClarkClassifyWorker.obj
 0002:000035a0       ??_C@_0BD@HKKHAEBH@Reads?5URL?5is?5empty?$AA@ 100235a0     ClarkClassifyWorker.obj
 0002:000035b4       ??_C@_0CD@JOFCEKPL@Classification?5report?5URL?5is?5emp@ 100235b4     ClarkClassifyWorker.obj
 0002:000035d8       ??_C@_0BM@KEDPLHAD@Clark?5database?5URL?5is?5empty?$AA@ 100235d8     ClarkClassifyWorker.obj
 0002:000035f8       ??_C@_0EK@LLKFAAGC@Unsupported?5CLARK?5variant?4?5Only?5@ 100235f8     ClarkClassifyWorker.obj
 0002:00003644       ??_C@_02KEDOHJFP@?9D?$AA@  10023644     ClarkClassifyWorker.obj
 0002:00003648       ??_C@_02OOPMGLAO@?9T?$AA@  10023648     ClarkClassifyWorker.obj
 0002:0000364c       ??_C@_0N@JOKKGLDK@?1targets?4txt?$AA@ 1002364c     ClarkClassifyWorker.obj
 0002:0000365c       ??_C@_04EBGNMJBD@?4csv?$AA@ 1002365c     ClarkClassifyWorker.obj
 0002:00003664       ??_C@_02LIKGMMII@?9R?$AA@  10023664     ClarkClassifyWorker.obj
 0002:00003668       ??_C@_02IKJAKOAK@?9P?$AA@  10023668     ClarkClassifyWorker.obj
 0002:0000366c       ??_C@_02EHMKKAJE@?9O?$AA@  1002366c     ClarkClassifyWorker.obj
 0002:00003670       ??_C@_02DEDJNJGL@?9s?$AA@  10023670     ClarkClassifyWorker.obj
 0002:00003674       ??_C@_02LGCCEBDC@?9k?$AA@  10023674     ClarkClassifyWorker.obj
 0002:00003678       ??_C@_02BKJHAODO@?9g?$AA@  10023678     ClarkClassifyWorker.obj
 0002:0000367c       ??_C@_02HLHIEPKM@?9t?$AA@  1002367c     ClarkClassifyWorker.obj
 0002:00003680       ??_C@_02OAHIOGLE@?9m?$AA@  10023680     ClarkClassifyWorker.obj
 0002:00003684       ??_C@_02MLFFLFHH@?9n?$AA@  10023684     ClarkClassifyWorker.obj
 0002:00003688       ??_C@_05CCCDJNKM@?9?9ldm?$AA@ 10023688     ClarkClassifyWorker.obj
 0002:00003690       ??_C@_0L@JHEHCOKM@?9?9extended?$AA@ 10023690     ClarkClassifyWorker.obj
 0002:0000369c       ??_C@_0CG@IHMCOLO@Cannot?5open?5classification?5repor@ 1002369c     ClarkClassifyWorker.obj
 0002:000036c4       ??_C@_0CM@MENMIJBK@Failed?5to?5recognize?5CLARK?5report@ 100236c4     ClarkClassifyWorker.obj
 0002:000036f0       ??_C@_0BI@NOBALKO@Broken?5CLARK?5report?3?5?$CF1?$AA@ 100236f0     ClarkClassifyWorker.obj
 0002:00003708       ??_C@_0CC@OIFCJADE@Found?5CLARK?5classification?3?5?$CF1?$DN?$CF@ 10023708     ClarkClassifyWorker.obj
 0002:0000372c       ??_C@_02JDNIPIGD@NA?$AA@   1002372c     ClarkClassifyWorker.obj
 0002:00003730       ??_C@_0EO@GBJCHADO@Duplicate?5sequence?5name?5?8?$CF1?8?5hav@ 10023730     ClarkClassifyWorker.obj
 0002:00003780       ??_C@_05OEPGNJB@light?$AA@ 10023780     ClarkClassifyWorker.obj
 0002:0000378c       ??_7?$AbstractId@H@U2@@6B@ 1002378c     ClarkSupport.obj
 0002:00003798       ??_7AbstractInt32Id@U2@@6B@ 10023798     ClarkSupport.obj
 0002:000037a4       ??_7ServiceType@U2@@6B@    100237a4     ClarkSupport.obj
 0002:000037b0       ??_7ClarkSupport@U2@@6B@   100237b0     ClarkSupport.obj
 0002:000037f0       ??_C@_0M@CHKIFHIJ@USUPP_CLARK?$AA@ 100237f0     ClarkSupport.obj
 0002:000037fc       ??_C@_0O@CEGCKJHJ@USUPP_CLARK_L?$AA@ 100237fc     ClarkSupport.obj
 0002:0000380c       ??_C@_0L@EPDEEDAB@builddb?4sh?$AA@ 1002380c     ClarkSupport.obj
 0002:00003818       ??_C@_0BF@HMINPMPB@USUPP_CLARK_BUILD_DB?$AA@ 10023818     ClarkSupport.obj
 0002:00003830       ??_C@_0P@JNOAALJI@getAccssnTaxID?$AA@ 10023830     ClarkSupport.obj
 0002:00003840       ??_C@_0BO@OPPHNFJO@USUPP_CLARK_GET_ACCSSN_TAX_ID?$AA@ 10023840     ClarkSupport.obj
 0002:00003860       ??_C@_0O@JPHPEPAE@getTargetsDef?$AA@ 10023860     ClarkSupport.obj
 0002:00003870       ??_C@_0BM@PMHNLKAP@USUPP_CLARK_GET_TARGETS_DEF?$AA@ 10023870     ClarkSupport.obj
 0002:0000388c       ??_C@_0BD@HMPNOCCM@getfilesToTaxNodes?$AA@ 1002388c     ClarkSupport.obj
 0002:000038a0       ??_C@_0CD@BHJGBOPP@USUPP_CLARK_GET_FILES_TO_TAX_NOD@ 100238a0     ClarkSupport.obj
 0002:000038c4       ??_C@_0CK@PGMKKHJF@?3external_tool_support?1images?1cm@ 100238c4     ClarkSupport.obj
 0002:000038f0       ??_C@_0CP@NPHMHKIL@?3external_tool_support?1images?1cm@ 100238f0     ClarkSupport.obj
 0002:00003920       ??_C@_0CP@MJGNLKEC@?3external_tool_support?1images?1cm@ 10023920     ClarkSupport.obj
 0002:00003950       ??_C@_04JLMDILM@?4exe?$AA@ 10023950     ClarkSupport.obj
 0002:00003958       ??_C@_0BE@OCGEGONF@UGENE?9customized?5?4?$CK?$AA@ 10023958     ClarkSupport.obj
 0002:00003970       ??_C@_0NC@KJDPMHIF@One?5of?5the?5classifiers?5from?5the?5@ 10023970     ClarkSupport.obj
 0002:00003a44       ??_C@_0CA@NGDNOCBN@Version?3?5?$CI?2d?$CL?2?4?2d?$CL?2?4?$DP?2d?$CK?2?4?$DP?2d?$CK?$CJ?$AA@ 10023a44     ClarkSupport.obj
 0002:00003a68       ??_C@_0BAE@MJBDAKJK@One?5of?5the?5classifiers?5from?5the?5@ 10023a68     ClarkSupport.obj
 0002:00003b6c       ??_C@_0BH@MHOGNJHA@UGENE?9customized?5CLARK?$AA@ 10023b6c     ClarkSupport.obj
 0002:00003b88       ??_C@_0HE@KMGMHAML@Used?5to?5set?5up?5metagenomic?5datab@ 10023b88     ClarkSupport.obj
 0002:00003c00       ??_7ClarkSupportPlugin@U2@@6B@ 10023c00     ClarkSupportPlugin.obj
 0002:00003c2c       ??_C@_0BM@CHNLCOME@CLARK?5external?5tool?5support?$AA@ 10023c2c     ClarkSupportPlugin.obj
 0002:00003c48       ??_C@_0HB@OGGNGKFE@The?5plugin?5supports?5CLARK?3?5fast?0@ 10023c48     ClarkSupportPlugin.obj
 0002:00003cbc       ??_C@_03PEIMBJDE@XML?$AA@  10023cbc     ClarkSupportPlugin.obj
 0002:00003cc0       ??_C@_0BL@GJGHLAEA@Can?8t?5find?5XML?5test?5format?$AA@ 10023cc0     ClarkSupportPlugin.obj
 0002:00003cdc       ??_C@_0BL@BBNEONPO@src?2ClarkSupportPlugin?4cpp?$AA@ 10023cdc     ClarkSupportPlugin.obj
 0002:00003cfc       ??_7?$GAutoDeleteList@VXMLTestFactory@U2@@@U2@@6B@ 10023cfc     ClarkSupportPlugin.obj
 0002:00003d2c       ??_7GTest_CompareClarkDatabaseMetafilesFactory@GTest_CompareClarkDatabaseMetafiles@U2@@6B@ 10023d2c     ClarkTests.obj
 0002:00003d38       ??_7GTest_CompareClarkDatabaseMetafiles@U2@@6B@ 10023d38     ClarkTests.obj
 0002:00003dc4       ??_C@_0CB@DJKPMFOI@clark?9compare?9database?9metafiles@ 10023dc4     ClarkTests.obj
 0002:00003de8       ??_C@_09JKBPIPPI@database1?$AA@ 10023de8     ClarkTests.obj
 0002:00003df4       ??_C@_09LBDCNMDL@database2?$AA@ 10023df4     ClarkTests.obj
 0002:00003e00       ??_C@_0BD@FJKPMDBK@database1?9prefixes?$AA@ 10023e00     ClarkTests.obj
 0002:00003e14       ??_C@_0BD@MAENKFBL@database2?9prefixes?$AA@ 10023e14     ClarkTests.obj
 0002:00003e28       ??_C@_0L@NDIHKJJP@?$CB?$EA?$CD$?$CF?$FO?$CG?$CK?$CI?$CJ?$AA@ 10023e28     ClarkTests.obj
 0002:00003e34       ??_C@_07FOGHKONL@?4custom?$AA@ 10023e34     ClarkTests.obj
 0002:00003e3c       ??_C@_0BB@FNPMLJID@?4custom_rejected?$AA@ 10023e3c     ClarkTests.obj
 0002:00003e50       ??_C@_0BD@BDCAHIJD@files_excluded?4txt?$AA@ 10023e50     ClarkTests.obj
 0002:00003e64       ??_C@_01ICJEACDI@?$DL?$AA@ 10023e64     ClarkTests.obj
 0002:00003e68       ??_C@_0BI@CDCDOFNJ@Database?51?5URL?5is?5empty?$AA@ 10023e68     ClarkTests.obj
 0002:00003e80       ??_C@_0BI@DCFOIPKA@Database?52?5URL?5is?5empty?$AA@ 10023e80     ClarkTests.obj
 0002:00003e98       ??_C@_0BP@MJCAHKMH@Database?51?5doesn?8t?5exist?3?5?8?$CF1?8?$AA@ 10023e98     ClarkTests.obj
 0002:00003eb8       ??_C@_0CE@HNDDFPH@Database?51?5is?5not?5a?5directory?3?5?8@ 10023eb8     ClarkTests.obj
 0002:00003edc       ??_C@_0BP@PAFINHIH@Database?52?5doesn?8t?5exist?3?5?8?$CF1?8?$AA@ 10023edc     ClarkTests.obj
 0002:00003efc       ??_C@_0CE@LEEHBIDE@Database?52?5is?5not?5a?5directory?3?5?8@ 10023efc     ClarkTests.obj
 0002:00003f20       ??_C@_0CF@IGNNBJOP@Can?8t?5open?5metafile?5?8?$CF1?8?5for?5rea@ 10023f20     ClarkTests.obj
 0002:00003f48       ??_C@_0DK@CBLHBMPH@Metafiles?5?8?$CF1?8?5and?5?8?$CF2?8?5differs?5@ 10023f48     ClarkTests.obj
 0002:00003f84       ??_C@_0DH@JPFOPGOK@Metafiles?5?8?$CF1?8?5and?5?8?$CF2?8?5have?5dif@ 10023f84     ClarkTests.obj
 0002:00004430       ?value@?$integral_constant@_N$0A@@std@@2_NB 10024430     MSVCRT:ti_inst.obj
 0002:00004431       ?value@?$integral_constant@_N$00@std@@2_NB 10024431     MSVCRT:ti_inst.obj
 0002:00004438       ??_7type_info@@6B@         10024438     MSVCRT:ti_inst.obj
 0002:0000443c       __pRawDllMain              1002443c     MSVCRT:crtdll.obj
 0002:0000443c       __pDefaultRawDllMain       1002443c     MSVCRT:crtdll.obj
 0002:00004448       ?ProcessDetach@NativeDll@<CrtImplementationDetails>@@0IB 10024448     MSVCRT:initsect.obj
 0002:0000444c       ?ProcessAttach@NativeDll@<CrtImplementationDetails>@@0IB 1002444c     MSVCRT:initsect.obj
 0002:00004450       ?ThreadAttach@NativeDll@<CrtImplementationDetails>@@0IB 10024450     MSVCRT:initsect.obj
 0002:00004454       ?ThreadDetach@NativeDll@<CrtImplementationDetails>@@0IB 10024454     MSVCRT:initsect.obj
 0002:00004458       ?ProcessVerifier@NativeDll@<CrtImplementationDetails>@@0IB 10024458     MSVCRT:initsect.obj
 0002:00004460       __load_config_used         10024460     MSVCRT:loadcfg.obj
 0002:0000451c       ??_R4error_category@std@@6B@ 1002451c     ClarkBuildWorker.obj
 0002:00004530       ??_R3error_category@std@@8 10024530     ClarkBuildWorker.obj
 0002:00004540       ??_R2error_category@std@@8 10024540     ClarkBuildWorker.obj
 0002:00004548       ??_R1A@?0A@EA@error_category@std@@8 10024548     ClarkBuildWorker.obj
 0002:00004564       ??_R4_Generic_error_category@std@@6B@ 10024564     ClarkBuildWorker.obj
 0002:00004578       ??_R3_Generic_error_category@std@@8 10024578     ClarkBuildWorker.obj
 0002:00004588       ??_R2_Generic_error_category@std@@8 10024588     ClarkBuildWorker.obj
 0002:00004594       ??_R1A@?0A@EA@_Generic_error_category@std@@8 10024594     ClarkBuildWorker.obj
 0002:000045b0       ??_R4_Iostream_error_category@std@@6B@ 100245b0     ClarkBuildWorker.obj
 0002:000045c4       ??_R3_Iostream_error_category@std@@8 100245c4     ClarkBuildWorker.obj
 0002:000045d4       ??_R2_Iostream_error_category@std@@8 100245d4     ClarkBuildWorker.obj
 0002:000045e4       ??_R1A@?0A@EA@_Iostream_error_category@std@@8 100245e4     ClarkBuildWorker.obj
 0002:00004600       ??_R4_System_error_category@std@@6B@ 10024600     ClarkBuildWorker.obj
 0002:00004614       ??_R3_System_error_category@std@@8 10024614     ClarkBuildWorker.obj
 0002:00004624       ??_R2_System_error_category@std@@8 10024624     ClarkBuildWorker.obj
 0002:00004634       ??_R1A@?0A@EA@_System_error_category@std@@8 10024634     ClarkBuildWorker.obj
 0002:00004650       ??_R1A@?0A@EA@QObject@@8   10024650     ClarkBuildWorker.obj
 0002:0000466c       ??_R3QObject@@8            1002466c     ClarkBuildWorker.obj
 0002:0000467c       ??_R2QObject@@8            1002467c     ClarkBuildWorker.obj
 0002:00004684       ??_R4FailTask@U2@@6B@      10024684     ClarkBuildWorker.obj
 0002:00004698       ??_R3FailTask@U2@@8        10024698     ClarkBuildWorker.obj
 0002:000046a8       ??_R2FailTask@U2@@8        100246a8     ClarkBuildWorker.obj
 0002:000046b8       ??_R1A@?0A@EA@FailTask@U2@@8 100246b8     ClarkBuildWorker.obj
 0002:000046d4       ??_R1A@?0A@EA@Task@U2@@8   100246d4     ClarkBuildWorker.obj
 0002:000046f0       ??_R3Task@U2@@8            100246f0     ClarkBuildWorker.obj
 0002:00004700       ??_R2Task@U2@@8            10024700     ClarkBuildWorker.obj
 0002:0000470c       ??_R4TaskSignalMapper@U2@@6B@ 1002470c     ClarkBuildWorker.obj
 0002:00004720       ??_R3TaskSignalMapper@U2@@8 10024720     ClarkBuildWorker.obj
 0002:00004730       ??_R2TaskSignalMapper@U2@@8 10024730     ClarkBuildWorker.obj
 0002:0000473c       ??_R1A@?0A@EA@TaskSignalMapper@U2@@8 1002473c     ClarkBuildWorker.obj
 0002:00004758       ??_R4Descriptor@U2@@6B@    10024758     ClarkBuildWorker.obj
 0002:0000476c       ??_R3Descriptor@U2@@8      1002476c     ClarkBuildWorker.obj
 0002:0000477c       ??_R2Descriptor@U2@@8      1002477c     ClarkBuildWorker.obj
 0002:00004784       ??_R1A@?0A@EA@Descriptor@U2@@8 10024784     ClarkBuildWorker.obj
 0002:000047a0       ??_R4MapDataType@U2@@6B@   100247a0     ClarkBuildWorker.obj
 0002:000047b4       ??_R3MapDataType@U2@@8     100247b4     ClarkBuildWorker.obj
 0002:000047c4       ??_R2MapDataType@U2@@8     100247c4     ClarkBuildWorker.obj
 0002:000047d8       ??_R1A@?0A@EA@MapDataType@U2@@8 100247d8     ClarkBuildWorker.obj
 0002:000047f4       ??_R1A@?0A@EA@DataType@U2@@8 100247f4     ClarkBuildWorker.obj
 0002:00004810       ??_R3DataType@U2@@8        10024810     ClarkBuildWorker.obj
 0002:00004820       ??_R2DataType@U2@@8        10024820     ClarkBuildWorker.obj
 0002:00004830       ??_R1BA@?0A@EA@QSharedData@@8 10024830     ClarkBuildWorker.obj
 0002:0000484c       ??_R3QSharedData@@8        1002484c     ClarkBuildWorker.obj
 0002:0000485c       ??_R2QSharedData@@8        1002485c     ClarkBuildWorker.obj
 0002:00004864       ??_R1A@?0A@EA@QSharedData@@8 10024864     ClarkBuildWorker.obj
 0002:00004880       ??_R4Attribute@U2@@6B@     10024880     ClarkBuildWorker.obj
 0002:00004894       ??_R3Attribute@U2@@8       10024894     ClarkBuildWorker.obj
 0002:000048a4       ??_R2Attribute@U2@@8       100248a4     ClarkBuildWorker.obj
 0002:000048b0       ??_R1A@?0A@EA@Attribute@U2@@8 100248b0     ClarkBuildWorker.obj
 0002:000048cc       ??_R3ConfigurationEditor@U2@@8 100248cc     ClarkBuildWorker.obj
 0002:000048dc       ??_R2ConfigurationEditor@U2@@8 100248dc     ClarkBuildWorker.obj
 0002:000048e8       ??_R1A@?0A@EA@ConfigurationEditor@U2@@8 100248e8     ClarkBuildWorker.obj
 0002:00004904       ??_R4DelegateEditor@U2@@6B@ 10024904     ClarkBuildWorker.obj
 0002:00004918       ??_R3DelegateEditor@U2@@8  10024918     ClarkBuildWorker.obj
 0002:00004928       ??_R2DelegateEditor@U2@@8  10024928     ClarkBuildWorker.obj
 0002:00004938       ??_R1A@?0A@EA@DelegateEditor@U2@@8 10024938     ClarkBuildWorker.obj
 0002:00004954       ??_R4URLDelegate@U2@@6B@   10024954     ClarkBuildWorker.obj
 0002:00004968       ??_R3URLDelegate@U2@@8     10024968     ClarkBuildWorker.obj
 0002:00004978       ??_R2URLDelegate@U2@@8     10024978     ClarkBuildWorker.obj
 0002:00004990       ??_R1A@?0A@EA@URLDelegate@U2@@8 10024990     ClarkBuildWorker.obj
 0002:000049ac       ??_R1A@?0A@EA@PropertyDelegate@U2@@8 100249ac     ClarkBuildWorker.obj
 0002:000049c8       ??_R3PropertyDelegate@U2@@8 100249c8     ClarkBuildWorker.obj
 0002:000049d8       ??_R2PropertyDelegate@U2@@8 100249d8     ClarkBuildWorker.obj
 0002:000049ec       ??_R1A@?0A@EA@QItemDelegate@@8 100249ec     ClarkBuildWorker.obj
 0002:00004a08       ??_R3QItemDelegate@@8      10024a08     ClarkBuildWorker.obj
 0002:00004a18       ??_R2QItemDelegate@@8      10024a18     ClarkBuildWorker.obj
 0002:00004a28       ??_R1A@?0A@EA@QAbstractItemDelegate@@8 10024a28     ClarkBuildWorker.obj
 0002:00004a44       ??_R3QAbstractItemDelegate@@8 10024a44     ClarkBuildWorker.obj
 0002:00004a54       ??_R2QAbstractItemDelegate@@8 10024a54     ClarkBuildWorker.obj
 0002:00004a60       ??_R4ComboBoxDelegate@U2@@6B@ 10024a60     ClarkBuildWorker.obj
 0002:00004a74       ??_R3ComboBoxDelegate@U2@@8 10024a74     ClarkBuildWorker.obj
 0002:00004a84       ??_R2ComboBoxDelegate@U2@@8 10024a84     ClarkBuildWorker.obj
 0002:00004a9c       ??_R1A@?0A@EA@ComboBoxDelegate@U2@@8 10024a9c     ClarkBuildWorker.obj
 0002:00004ab8       ??_R4PortDescriptor@Workflow@U2@@6B@ 10024ab8     ClarkBuildWorker.obj
 0002:00004acc       ??_R3PortDescriptor@Workflow@U2@@8 10024acc     ClarkBuildWorker.obj
 0002:00004adc       ??_R2PortDescriptor@Workflow@U2@@8 10024adc     ClarkBuildWorker.obj
 0002:00004ae8       ??_R1A@?0A@EA@PortDescriptor@Workflow@U2@@8 10024ae8     ClarkBuildWorker.obj
 0002:00004b04       ??_R17?0A@EA@Descriptor@U2@@8 10024b04     ClarkBuildWorker.obj
 0002:00004b20       ??_R4IntegralBusActorPrototype@Workflow@U2@@6BQObject@@@ 10024b20     ClarkBuildWorker.obj
 0002:00004b34       ??_R3IntegralBusActorPrototype@Workflow@U2@@8 10024b34     ClarkBuildWorker.obj
 0002:00004b44       ??_R2IntegralBusActorPrototype@Workflow@U2@@8 10024b44     ClarkBuildWorker.obj
 0002:00004b5c       ??_R1A@?0A@EA@IntegralBusActorPrototype@Workflow@U2@@8 10024b5c     ClarkBuildWorker.obj
 0002:00004b78       ??_R1A@?0A@EA@ActorPrototype@Workflow@U2@@8 10024b78     ClarkBuildWorker.obj
 0002:00004b94       ??_R3ActorPrototype@Workflow@U2@@8 10024b94     ClarkBuildWorker.obj
 0002:00004ba4       ??_R2ActorPrototype@Workflow@U2@@8 10024ba4     ClarkBuildWorker.obj
 0002:00004bb8       ??_R17?0A@EA@VisualDescriptor@U2@@8 10024bb8     ClarkBuildWorker.obj
 0002:00004bd4       ??_R3VisualDescriptor@U2@@8 10024bd4     ClarkBuildWorker.obj
 0002:00004be4       ??_R2VisualDescriptor@U2@@8 10024be4     ClarkBuildWorker.obj
 0002:00004bf0       ??_R1A@?0A@EA@VisualDescriptor@U2@@8 10024bf0     ClarkBuildWorker.obj
 0002:00004c0c       ??_R4IntegralBusActorPrototype@Workflow@U2@@6BVisualDescriptor@2@@ 10024c0c     ClarkBuildWorker.obj
 0002:00004c20       ??_R4ExternalToolRunTask@U2@@6B@ 10024c20     ClarkBuildWorker.obj
 0002:00004c34       ??_R3ExternalToolRunTask@U2@@8 10024c34     ClarkBuildWorker.obj
 0002:00004c44       ??_R2ExternalToolRunTask@U2@@8 10024c44     ClarkBuildWorker.obj
 0002:00004c54       ??_R1A@?0A@EA@ExternalToolRunTask@U2@@8 10024c54     ClarkBuildWorker.obj
 0002:00004c70       ??_R4ClarkBuildValidator@LocalWorkflow@U2@@6B@ 10024c70     ClarkBuildWorker.obj
 0002:00004c84       ??_R3ClarkBuildValidator@LocalWorkflow@U2@@8 10024c84     ClarkBuildWorker.obj
 0002:00004c94       ??_R2ClarkBuildValidator@LocalWorkflow@U2@@8 10024c94     ClarkBuildWorker.obj
 0002:00004ca4       ??_R1A@?0A@EA@ClarkBuildValidator@LocalWorkflow@U2@@8 10024ca4     ClarkBuildWorker.obj
 0002:00004cc0       ??_R1A@?0A@EA@ActorValidator@Workflow@U2@@8 10024cc0     ClarkBuildWorker.obj
 0002:00004cdc       ??_R3ActorValidator@Workflow@U2@@8 10024cdc     ClarkBuildWorker.obj
 0002:00004cec       ??_R2ActorValidator@Workflow@U2@@8 10024cec     ClarkBuildWorker.obj
 0002:00004cf8       ??_R1A@?0A@EA@ConfigurationValidator@U2@@8 10024cf8     ClarkBuildWorker.obj
 0002:00004d14       ??_R3ConfigurationValidator@U2@@8 10024d14     ClarkBuildWorker.obj
 0002:00004d24       ??_R2ConfigurationValidator@U2@@8 10024d24     ClarkBuildWorker.obj
 0002:00004d2c       ??_R4ClarkBuildPrompter@LocalWorkflow@U2@@6BActorDocument@Workflow@2@@ 10024d2c     ClarkBuildWorker.obj
 0002:00004d40       ??_R3ClarkBuildPrompter@LocalWorkflow@U2@@8 10024d40     ClarkBuildWorker.obj
 0002:00004d50       ??_R2ClarkBuildPrompter@LocalWorkflow@U2@@8 10024d50     ClarkBuildWorker.obj
 0002:00004d70       ??_R1A@?0A@EA@ClarkBuildPrompter@LocalWorkflow@U2@@8 10024d70     ClarkBuildWorker.obj
 0002:00004d8c       ??_R1A@?0A@EA@?$PrompterBase@VClarkBuildPrompter@LocalWorkflow@U2@@@U2@@8 10024d8c     ClarkBuildWorker.obj
 0002:00004da8       ??_R3?$PrompterBase@VClarkBuildPrompter@LocalWorkflow@U2@@@U2@@8 10024da8     ClarkBuildWorker.obj
 0002:00004db8       ??_R2?$PrompterBase@VClarkBuildPrompter@LocalWorkflow@U2@@@U2@@8 10024db8     ClarkBuildWorker.obj
 0002:00004dd4       ??_R1A@?0A@EA@PrompterBaseImpl@U2@@8 10024dd4     ClarkBuildWorker.obj
 0002:00004df0       ??_R3PrompterBaseImpl@U2@@8 10024df0     ClarkBuildWorker.obj
 0002:00004e00       ??_R2PrompterBaseImpl@U2@@8 10024e00     ClarkBuildWorker.obj
 0002:00004e18       ??_R1A@?0A@EA@ActorDocument@Workflow@U2@@8 10024e18     ClarkBuildWorker.obj
 0002:00004e34       ??_R3ActorDocument@Workflow@U2@@8 10024e34     ClarkBuildWorker.obj
 0002:00004e44       ??_R2ActorDocument@Workflow@U2@@8 10024e44     ClarkBuildWorker.obj
 0002:00004e54       ??_R1A@?0A@EA@QTextDocument@@8 10024e54     ClarkBuildWorker.obj
 0002:00004e70       ??_R3QTextDocument@@8      10024e70     ClarkBuildWorker.obj
 0002:00004e80       ??_R2QTextDocument@@8      10024e80     ClarkBuildWorker.obj
 0002:00004e8c       ??_R1M@?0A@EA@Prompter@Workflow@U2@@8 10024e8c     ClarkBuildWorker.obj
 0002:00004ea8       ??_R3Prompter@Workflow@U2@@8 10024ea8     ClarkBuildWorker.obj
 0002:00004eb8       ??_R2Prompter@Workflow@U2@@8 10024eb8     ClarkBuildWorker.obj
 0002:00004ec0       ??_R1A@?0A@EA@Prompter@Workflow@U2@@8 10024ec0     ClarkBuildWorker.obj
 0002:00004edc       ??_R4ClarkBuildPrompter@LocalWorkflow@U2@@6BPrompter@Workflow@2@@ 10024edc     ClarkBuildWorker.obj
 0002:00004ef0       ??_R4?$PrompterBase@VClarkBuildPrompter@LocalWorkflow@U2@@@U2@@6BActorDocument@Workflow@1@@ 10024ef0     ClarkBuildWorker.obj
 0002:00004f04       ??_R4?$PrompterBase@VClarkBuildPrompter@LocalWorkflow@U2@@@U2@@6BPrompter@Workflow@1@@ 10024f04     ClarkBuildWorker.obj
 0002:00004f18       ??_R4ClarkBuildWorker@LocalWorkflow@U2@@6BQObject@@@ 10024f18     ClarkBuildWorker.obj
 0002:00004f2c       ??_R3ClarkBuildWorker@LocalWorkflow@U2@@8 10024f2c     ClarkBuildWorker.obj
 0002:00004f3c       ??_R2ClarkBuildWorker@LocalWorkflow@U2@@8 10024f3c     ClarkBuildWorker.obj
 0002:00004f54       ??_R1A@?0A@EA@ClarkBuildWorker@LocalWorkflow@U2@@8 10024f54     ClarkBuildWorker.obj
 0002:00004f70       ??_R1A@?0A@EA@BaseWorker@LocalWorkflow@U2@@8 10024f70     ClarkBuildWorker.obj
 0002:00004f8c       ??_R3BaseWorker@LocalWorkflow@U2@@8 10024f8c     ClarkBuildWorker.obj
 0002:00004f9c       ??_R2BaseWorker@LocalWorkflow@U2@@8 10024f9c     ClarkBuildWorker.obj
 0002:00004fb0       ??_R17?0A@EA@Worker@Workflow@U2@@8 10024fb0     ClarkBuildWorker.obj
 0002:00004fcc       ??_R3Worker@Workflow@U2@@8 10024fcc     ClarkBuildWorker.obj
 0002:00004fdc       ??_R2Worker@Workflow@U2@@8 10024fdc     ClarkBuildWorker.obj
 0002:00004fe4       ??_R1A@?0A@EA@Worker@Workflow@U2@@8 10024fe4     ClarkBuildWorker.obj
 0002:00005000       ??_R1BA@?0A@EA@CommunicationSubject@Workflow@U2@@8 10025000     ClarkBuildWorker.obj
 0002:0000501c       ??_R3CommunicationSubject@Workflow@U2@@8 1002501c     ClarkBuildWorker.obj
 0002:0000502c       ??_R2CommunicationSubject@Workflow@U2@@8 1002502c     ClarkBuildWorker.obj
 0002:00005034       ??_R1A@?0A@EA@CommunicationSubject@Workflow@U2@@8 10025034     ClarkBuildWorker.obj
 0002:00005050       ??_R4ClarkBuildWorker@LocalWorkflow@U2@@6BWorker@Workflow@2@@ 10025050     ClarkBuildWorker.obj
 0002:00005064       ??_R4ClarkBuildWorker@LocalWorkflow@U2@@6BCommunicationSubject@Workflow@2@@ 10025064     ClarkBuildWorker.obj
 0002:00005078       ??_R4ClarkBuildWorkerFactory@LocalWorkflow@U2@@6B?$IdRegistry@VDomainFactory@Workflow@U2@@@2@@ 10025078     ClarkBuildWorker.obj
 0002:0000508c       ??_R3ClarkBuildWorkerFactory@LocalWorkflow@U2@@8 1002508c     ClarkBuildWorker.obj
 0002:0000509c       ??_R2ClarkBuildWorkerFactory@LocalWorkflow@U2@@8 1002509c     ClarkBuildWorker.obj
 0002:000050b0       ??_R1A@?0A@EA@ClarkBuildWorkerFactory@LocalWorkflow@U2@@8 100250b0     ClarkBuildWorker.obj
 0002:000050cc       ??_R1A@?0A@EA@DomainFactory@Workflow@U2@@8 100250cc     ClarkBuildWorker.obj
 0002:000050e8       ??_R3DomainFactory@Workflow@U2@@8 100250e8     ClarkBuildWorker.obj
 0002:000050f8       ??_R2DomainFactory@Workflow@U2@@8 100250f8     ClarkBuildWorker.obj
 0002:00005108       ??_R1A@?0A@EA@?$IdRegistry@VDomainFactory@Workflow@U2@@@U2@@8 10025108     ClarkBuildWorker.obj
 0002:00005124       ??_R3?$IdRegistry@VDomainFactory@Workflow@U2@@@U2@@8 10025124     ClarkBuildWorker.obj
 0002:00005134       ??_R2?$IdRegistry@VDomainFactory@Workflow@U2@@@U2@@8 10025134     ClarkBuildWorker.obj
 0002:0000513c       ??_R4ClarkBuildWorkerFactory@LocalWorkflow@U2@@6BDescriptor@2@@ 1002513c     ClarkBuildWorker.obj
 0002:00005150       ??_R4ClarkBuildTask@LocalWorkflow@U2@@6B@ 10025150     ClarkBuildWorker.obj
 0002:00005164       ??_R3ClarkBuildTask@LocalWorkflow@U2@@8 10025164     ClarkBuildWorker.obj
 0002:00005174       ??_R2ClarkBuildTask@LocalWorkflow@U2@@8 10025174     ClarkBuildWorker.obj
 0002:00005188       ??_R1A@?0A@EA@ClarkBuildTask@LocalWorkflow@U2@@8 10025188     ClarkBuildWorker.obj
 0002:000051a4       ??_R1A@?0A@EA@ExternalToolSupportTask@U2@@8 100251a4     ClarkBuildWorker.obj
 0002:000051c0       ??_R3ExternalToolSupportTask@U2@@8 100251c0     ClarkBuildWorker.obj
 0002:000051d0       ??_R2ExternalToolSupportTask@U2@@8 100251d0     ClarkBuildWorker.obj
 0002:000051e0       ??_R4GenomicLibraryDelegate@LocalWorkflow@U2@@6B@ 100251e0     ClarkBuildWorker.obj
 0002:000051f4       ??_R3GenomicLibraryDelegate@LocalWorkflow@U2@@8 100251f4     ClarkBuildWorker.obj
 0002:00005204       ??_R2GenomicLibraryDelegate@LocalWorkflow@U2@@8 10025204     ClarkBuildWorker.obj
 0002:0000521c       ??_R1A@?0A@EA@GenomicLibraryDelegate@LocalWorkflow@U2@@8 1002521c     ClarkBuildWorker.obj
 0002:00005238       ??_R4ClarkBuildLogParser@LocalWorkflow@U2@@6B@ 10025238     ClarkBuildWorker.obj
 0002:0000524c       ??_R3ClarkBuildLogParser@LocalWorkflow@U2@@8 1002524c     ClarkBuildWorker.obj
 0002:0000525c       ??_R2ClarkBuildLogParser@LocalWorkflow@U2@@8 1002525c     ClarkBuildWorker.obj
 0002:0000526c       ??_R1A@?0A@EA@ClarkBuildLogParser@LocalWorkflow@U2@@8 1002526c     ClarkBuildWorker.obj
 0002:00005288       ??_R1A@?0A@EA@ExternalToolLogParser@U2@@8 10025288     ClarkBuildWorker.obj
 0002:000052a4       ??_R3ExternalToolLogParser@U2@@8 100252a4     ClarkBuildWorker.obj
 0002:000052b4       ??_R2ExternalToolLogParser@U2@@8 100252b4     ClarkBuildWorker.obj
 0002:000052c0       ??_R4VisibilityRelation@U2@@6B@ 100252c0     ClarkClassifyWorker.obj
 0002:000052d4       ??_R3VisibilityRelation@U2@@8 100252d4     ClarkClassifyWorker.obj
 0002:000052e4       ??_R2VisibilityRelation@U2@@8 100252e4     ClarkClassifyWorker.obj
 0002:000052f0       ??_R1A@?0A@EA@VisibilityRelation@U2@@8 100252f0     ClarkClassifyWorker.obj
 0002:0000530c       ??_R1A@?0A@EA@AttributeRelation@U2@@8 1002530c     ClarkClassifyWorker.obj
 0002:00005328       ??_R3AttributeRelation@U2@@8 10025328     ClarkClassifyWorker.obj
 0002:00005338       ??_R2AttributeRelation@U2@@8 10025338     ClarkClassifyWorker.obj
 0002:00005340       ??_R4SlotRelationDescriptor@U2@@6B@ 10025340     ClarkClassifyWorker.obj
 0002:00005354       ??_R3SlotRelationDescriptor@U2@@8 10025354     ClarkClassifyWorker.obj
 0002:00005364       ??_R2SlotRelationDescriptor@U2@@8 10025364     ClarkClassifyWorker.obj
 0002:0000536c       ??_R1A@?0A@EA@SlotRelationDescriptor@U2@@8 1002536c     ClarkClassifyWorker.obj
 0002:00005388       ??_R4SpinBoxDelegate@U2@@6B@ 10025388     ClarkClassifyWorker.obj
 0002:0000539c       ??_R3SpinBoxDelegate@U2@@8 1002539c     ClarkClassifyWorker.obj
 0002:000053ac       ??_R2SpinBoxDelegate@U2@@8 100253ac     ClarkClassifyWorker.obj
 0002:000053c4       ??_R1A@?0A@EA@SpinBoxDelegate@U2@@8 100253c4     ClarkClassifyWorker.obj
 0002:000053e0       ??_R4PairedReadsPortValidator@Workflow@U2@@6B@ 100253e0     ClarkClassifyWorker.obj
 0002:000053f4       ??_R3PairedReadsPortValidator@Workflow@U2@@8 100253f4     ClarkClassifyWorker.obj
 0002:00005404       ??_R2PairedReadsPortValidator@Workflow@U2@@8 10025404     ClarkClassifyWorker.obj
 0002:00005414       ??_R1A@?0A@EA@PairedReadsPortValidator@Workflow@U2@@8 10025414     ClarkClassifyWorker.obj
 0002:00005430       ??_R1A@?0A@EA@PortValidator@Workflow@U2@@8 10025430     ClarkClassifyWorker.obj
 0002:0000544c       ??_R3PortValidator@Workflow@U2@@8 1002544c     ClarkClassifyWorker.obj
 0002:0000545c       ??_R2PortValidator@Workflow@U2@@8 1002545c     ClarkClassifyWorker.obj
 0002:00005468       ??_R4ClarkClassifyPrompter@LocalWorkflow@U2@@6BActorDocument@Workflow@2@@ 10025468     ClarkClassifyWorker.obj
 0002:0000547c       ??_R3ClarkClassifyPrompter@LocalWorkflow@U2@@8 1002547c     ClarkClassifyWorker.obj
 0002:0000548c       ??_R2ClarkClassifyPrompter@LocalWorkflow@U2@@8 1002548c     ClarkClassifyWorker.obj
 0002:000054ac       ??_R1A@?0A@EA@ClarkClassifyPrompter@LocalWorkflow@U2@@8 100254ac     ClarkClassifyWorker.obj
 0002:000054c8       ??_R1A@?0A@EA@?$PrompterBase@VClarkClassifyPrompter@LocalWorkflow@U2@@@U2@@8 100254c8     ClarkClassifyWorker.obj
 0002:000054e4       ??_R3?$PrompterBase@VClarkClassifyPrompter@LocalWorkflow@U2@@@U2@@8 100254e4     ClarkClassifyWorker.obj
 0002:000054f4       ??_R2?$PrompterBase@VClarkClassifyPrompter@LocalWorkflow@U2@@@U2@@8 100254f4     ClarkClassifyWorker.obj
 0002:00005510       ??_R4ClarkClassifyPrompter@LocalWorkflow@U2@@6BPrompter@Workflow@2@@ 10025510     ClarkClassifyWorker.obj
 0002:00005524       ??_R4?$PrompterBase@VClarkClassifyPrompter@LocalWorkflow@U2@@@U2@@6BActorDocument@Workflow@1@@ 10025524     ClarkClassifyWorker.obj
 0002:00005538       ??_R4?$PrompterBase@VClarkClassifyPrompter@LocalWorkflow@U2@@@U2@@6BPrompter@Workflow@1@@ 10025538     ClarkClassifyWorker.obj
 0002:0000554c       ??_R4ClarkClassifyWorker@LocalWorkflow@U2@@6BQObject@@@ 1002554c     ClarkClassifyWorker.obj
 0002:00005560       ??_R3ClarkClassifyWorker@LocalWorkflow@U2@@8 10025560     ClarkClassifyWorker.obj
 0002:00005570       ??_R2ClarkClassifyWorker@LocalWorkflow@U2@@8 10025570     ClarkClassifyWorker.obj
 0002:00005588       ??_R1A@?0A@EA@ClarkClassifyWorker@LocalWorkflow@U2@@8 10025588     ClarkClassifyWorker.obj
 0002:000055a4       ??_R4ClarkClassifyWorker@LocalWorkflow@U2@@6BWorker@Workflow@2@@ 100255a4     ClarkClassifyWorker.obj
 0002:000055b8       ??_R4ClarkClassifyWorker@LocalWorkflow@U2@@6BCommunicationSubject@Workflow@2@@ 100255b8     ClarkClassifyWorker.obj
 0002:000055cc       ??_R4ClarkClassifyValidator@LocalWorkflow@U2@@6B@ 100255cc     ClarkClassifyWorker.obj
 0002:000055e0       ??_R3ClarkClassifyValidator@LocalWorkflow@U2@@8 100255e0     ClarkClassifyWorker.obj
 0002:000055f0       ??_R2ClarkClassifyValidator@LocalWorkflow@U2@@8 100255f0     ClarkClassifyWorker.obj
 0002:00005600       ??_R1A@?0A@EA@ClarkClassifyValidator@LocalWorkflow@U2@@8 10025600     ClarkClassifyWorker.obj
 0002:0000561c       ??_R4ClarkClassifyWorkerFactory@LocalWorkflow@U2@@6B?$IdRegistry@VDomainFactory@Workflow@U2@@@2@@ 1002561c     ClarkClassifyWorker.obj
 0002:00005630       ??_R3ClarkClassifyWorkerFactory@LocalWorkflow@U2@@8 10025630     ClarkClassifyWorker.obj
 0002:00005640       ??_R2ClarkClassifyWorkerFactory@LocalWorkflow@U2@@8 10025640     ClarkClassifyWorker.obj
 0002:00005654       ??_R1A@?0A@EA@ClarkClassifyWorkerFactory@LocalWorkflow@U2@@8 10025654     ClarkClassifyWorker.obj
 0002:00005670       ??_R4ClarkClassifyWorkerFactory@LocalWorkflow@U2@@6BDescriptor@2@@ 10025670     ClarkClassifyWorker.obj
 0002:00005684       ??_R4ClarkLogParser@LocalWorkflow@U2@@6B@ 10025684     ClarkClassifyWorker.obj
 0002:00005698       ??_R3ClarkLogParser@LocalWorkflow@U2@@8 10025698     ClarkClassifyWorker.obj
 0002:000056a8       ??_R2ClarkLogParser@LocalWorkflow@U2@@8 100256a8     ClarkClassifyWorker.obj
 0002:000056b8       ??_R1A@?0A@EA@ClarkLogParser@LocalWorkflow@U2@@8 100256b8     ClarkClassifyWorker.obj
 0002:000056d4       ??_R4ClarkClassifyTask@LocalWorkflow@U2@@6B@ 100256d4     ClarkClassifyWorker.obj
 0002:000056e8       ??_R3ClarkClassifyTask@LocalWorkflow@U2@@8 100256e8     ClarkClassifyWorker.obj
 0002:000056f8       ??_R2ClarkClassifyTask@LocalWorkflow@U2@@8 100256f8     ClarkClassifyWorker.obj
 0002:0000570c       ??_R1A@?0A@EA@ClarkClassifyTask@LocalWorkflow@U2@@8 1002570c     ClarkClassifyWorker.obj
 0002:00005728       ??_R4DatabaseDelegate@LocalWorkflow@U2@@6B@ 10025728     ClarkClassifyWorker.obj
 0002:0000573c       ??_R3DatabaseDelegate@LocalWorkflow@U2@@8 1002573c     ClarkClassifyWorker.obj
 0002:0000574c       ??_R2DatabaseDelegate@LocalWorkflow@U2@@8 1002574c     ClarkClassifyWorker.obj
 0002:00005768       ??_R1A@?0A@EA@DatabaseDelegate@LocalWorkflow@U2@@8 10025768     ClarkClassifyWorker.obj
 0002:00005784       ??_R4AbstractInt32Id@U2@@6B@ 10025784     ClarkSupport.obj
 0002:00005798       ??_R3AbstractInt32Id@U2@@8 10025798     ClarkSupport.obj
 0002:000057a8       ??_R2AbstractInt32Id@U2@@8 100257a8     ClarkSupport.obj
 0002:000057b4       ??_R1A@?0A@EA@AbstractInt32Id@U2@@8 100257b4     ClarkSupport.obj
 0002:000057d0       ??_R1A@?0A@EA@?$AbstractId@H@U2@@8 100257d0     ClarkSupport.obj
 0002:000057ec       ??_R3?$AbstractId@H@U2@@8  100257ec     ClarkSupport.obj
 0002:000057fc       ??_R2?$AbstractId@H@U2@@8  100257fc     ClarkSupport.obj
 0002:00005804       ??_R4?$AbstractId@H@U2@@6B@ 10025804     ClarkSupport.obj
 0002:00005818       ??_R4ServiceType@U2@@6B@   10025818     ClarkSupport.obj
 0002:0000582c       ??_R3ServiceType@U2@@8     1002582c     ClarkSupport.obj
 0002:0000583c       ??_R2ServiceType@U2@@8     1002583c     ClarkSupport.obj
 0002:0000584c       ??_R1A@?0A@EA@ServiceType@U2@@8 1002584c     ClarkSupport.obj
 0002:00005868       ??_R4ClarkSupport@U2@@6B@  10025868     ClarkSupport.obj
 0002:0000587c       ??_R3ClarkSupport@U2@@8    1002587c     ClarkSupport.obj
 0002:0000588c       ??_R2ClarkSupport@U2@@8    1002588c     ClarkSupport.obj
 0002:0000589c       ??_R1A@?0A@EA@ClarkSupport@U2@@8 1002589c     ClarkSupport.obj
 0002:000058b8       ??_R1A@?0A@EA@ExternalTool@U2@@8 100258b8     ClarkSupport.obj
 0002:000058d4       ??_R3ExternalTool@U2@@8    100258d4     ClarkSupport.obj
 0002:000058e4       ??_R2ExternalTool@U2@@8    100258e4     ClarkSupport.obj
 0002:000058f0       ??_R4ClarkSupportPlugin@U2@@6B@ 100258f0     ClarkSupportPlugin.obj
 0002:00005904       ??_R3ClarkSupportPlugin@U2@@8 10025904     ClarkSupportPlugin.obj
 0002:00005914       ??_R2ClarkSupportPlugin@U2@@8 10025914     ClarkSupportPlugin.obj
 0002:00005924       ??_R1A@?0A@EA@ClarkSupportPlugin@U2@@8 10025924     ClarkSupportPlugin.obj
 0002:00005940       ??_R1A@?0A@EA@Plugin@U2@@8 10025940     ClarkSupportPlugin.obj
 0002:0000595c       ??_R3Plugin@U2@@8          1002595c     ClarkSupportPlugin.obj
 0002:0000596c       ??_R2Plugin@U2@@8          1002596c     ClarkSupportPlugin.obj
 0002:00005978       ??_R4?$GAutoDeleteList@VXMLTestFactory@U2@@@U2@@6B@ 10025978     ClarkSupportPlugin.obj
 0002:0000598c       ??_R3?$GAutoDeleteList@VXMLTestFactory@U2@@@U2@@8 1002598c     ClarkSupportPlugin.obj
 0002:0000599c       ??_R2?$GAutoDeleteList@VXMLTestFactory@U2@@@U2@@8 1002599c     ClarkSupportPlugin.obj
 0002:000059a8       ??_R1A@?0A@EA@?$GAutoDeleteList@VXMLTestFactory@U2@@@U2@@8 100259a8     ClarkSupportPlugin.obj
 0002:000059c4       ??_R1A@?0A@EA@XmlTest@U2@@8 100259c4     ClarkTests.obj
 0002:000059e0       ??_R3XmlTest@U2@@8         100259e0     ClarkTests.obj
 0002:000059f0       ??_R2XmlTest@U2@@8         100259f0     ClarkTests.obj
 0002:00005a04       ??_R1A@?0A@EA@GTest@U2@@8  10025a04     ClarkTests.obj
 0002:00005a20       ??_R3GTest@U2@@8           10025a20     ClarkTests.obj
 0002:00005a30       ??_R2GTest@U2@@8           10025a30     ClarkTests.obj
 0002:00005a40       ??_R1A@?0A@EA@XMLTestFactory@U2@@8 10025a40     ClarkTests.obj
 0002:00005a5c       ??_R3XMLTestFactory@U2@@8  10025a5c     ClarkTests.obj
 0002:00005a6c       ??_R2XMLTestFactory@U2@@8  10025a6c     ClarkTests.obj
 0002:00005a74       ??_R4GTest_CompareClarkDatabaseMetafiles@U2@@6B@ 10025a74     ClarkTests.obj
 0002:00005a88       ??_R3GTest_CompareClarkDatabaseMetafiles@U2@@8 10025a88     ClarkTests.obj
 0002:00005a98       ??_R2GTest_CompareClarkDatabaseMetafiles@U2@@8 10025a98     ClarkTests.obj
 0002:00005ab0       ??_R1A@?0A@EA@GTest_CompareClarkDatabaseMetafiles@U2@@8 10025ab0     ClarkTests.obj
 0002:00005acc       ??_R4GTest_CompareClarkDatabaseMetafilesFactory@GTest_CompareClarkDatabaseMetafiles@U2@@6B@ 10025acc     ClarkTests.obj
 0002:00005ae0       ??_R3GTest_CompareClarkDatabaseMetafilesFactory@GTest_CompareClarkDatabaseMetafiles@U2@@8 10025ae0     ClarkTests.obj
 0002:00005af0       ??_R2GTest_CompareClarkDatabaseMetafilesFactory@GTest_CompareClarkDatabaseMetafiles@U2@@8 10025af0     ClarkTests.obj
 0002:00005afc       ??_R1A@?0A@EA@GTest_CompareClarkDatabaseMetafilesFactory@GTest_CompareClarkDatabaseMetafiles@U2@@8 10025afc     ClarkTests.obj
 0002:00005b18       ??_R4type_info@@6B@        10025b18     MSVCRT:ti_inst.obj
 0002:00005b2c       ??_R3type_info@@8          10025b2c     MSVCRT:ti_inst.obj
 0002:00005b3c       ??_R2type_info@@8          10025b3c     MSVCRT:ti_inst.obj
 0002:00005b44       ??_R1A@?0A@EA@type_info@@8 10025b44     MSVCRT:ti_inst.obj
 0002:00005b60       ___safe_se_handler_table   10025b60     <linker-defined>
 0002:00005e5c       ___rtc_iaa                 10025e5c     MSVCRT:initsect.obj
 0002:00005e60       ___rtc_izz                 10025e60     MSVCRT:initsect.obj
 0002:00005e64       ___rtc_taa                 10025e64     MSVCRT:initsect.obj
 0002:00005e68       ___rtc_tzz                 10025e68     MSVCRT:initsect.obj
 0002:0000a748       __IMPORT_DESCRIPTOR_U2Core 1002a748     U2Core:U2Core.dll
 0002:0000a75c       __IMPORT_DESCRIPTOR_U2Gui  1002a75c     U2Gui:U2Gui.dll
 0002:0000a770       __IMPORT_DESCRIPTOR_U2Test 1002a770     U2Test:U2Test.dll
 0002:0000a784       __IMPORT_DESCRIPTOR_U2Lang 1002a784     U2Lang:U2Lang.dll
 0002:0000a798       __IMPORT_DESCRIPTOR_U2Designer 1002a798     U2Designer:U2Designer.dll
 0002:0000a7ac       __IMPORT_DESCRIPTOR_ngs_reads_classification 1002a7ac     ngs_reads_classification:ngs_reads_classification.dll
 0002:0000a7c0       __IMPORT_DESCRIPTOR_Qt5Widgets 1002a7c0     Qt5Widgets:Qt5Widgets.dll
 0002:0000a7d4       __IMPORT_DESCRIPTOR_Qt5Gui 1002a7d4     Qt5Gui:Qt5Gui.dll
 0002:0000a7e8       __IMPORT_DESCRIPTOR_Qt5Script 1002a7e8     Qt5Script:Qt5Script.dll
 0002:0000a7fc       __IMPORT_DESCRIPTOR_Qt5Xml 1002a7fc     Qt5Xml:Qt5Xml.dll
 0002:0000a810       __IMPORT_DESCRIPTOR_Qt5Core 1002a810     Qt5Core:Qt5Core.dll
 0002:0000a824       __IMPORT_DESCRIPTOR_MSVCP120 1002a824     msvcprt:MSVCP120.dll
 0002:0000a838       __IMPORT_DESCRIPTOR_MSVCR120 1002a838     MSVCRT:MSVCR120.dll
 0002:0000a84c       __IMPORT_DESCRIPTOR_KERNEL32 1002a84c     kernel32:KERNEL32.dll
 0002:0000a860       __NULL_IMPORT_DESCRIPTOR   1002a860     U2Core:U2Core.dll
 0003:00000000       ?_Generic_object@?$_Error_objects@H@std@@2V_Generic_error_category@2@A 10033000     ClarkBuildWorker.obj
 0003:00000004       ?_Iostream_object@?$_Error_objects@H@std@@2V_Iostream_error_category@2@A 10033004     ClarkBuildWorker.obj
 0003:00000008       ?_System_object@?$_Error_objects@H@std@@2V_System_error_category@2@A 10033008     ClarkBuildWorker.obj
 0003:00000074       ?staticMetaObject@ClarkBuildPrompter@LocalWorkflow@U2@@2UQMetaObject@@B 10033074     moc_ClarkBuildWorker.obj
 0003:0000008c       ?staticMetaObject@ClarkBuildWorker@LocalWorkflow@U2@@2UQMetaObject@@B 1003308c     moc_ClarkBuildWorker.obj
 0003:000000a4       ?staticMetaObject@ClarkBuildTask@LocalWorkflow@U2@@2UQMetaObject@@B 100330a4     moc_ClarkBuildWorker.obj
 0003:000000bc       ?staticMetaObject@ClarkClassifyPrompter@LocalWorkflow@U2@@2UQMetaObject@@B 100330bc     moc_ClarkClassifyWorker.obj
 0003:000000d4       ?staticMetaObject@ClarkClassifyWorker@LocalWorkflow@U2@@2UQMetaObject@@B 100330d4     moc_ClarkClassifyWorker.obj
 0003:000000ec       ?staticMetaObject@ClarkClassifyTask@LocalWorkflow@U2@@2UQMetaObject@@B 100330ec     moc_ClarkClassifyWorker.obj
 0003:00000104       ?staticMetaObject@ClarkSupport@U2@@2UQMetaObject@@B 10033104     moc_ClarkSupport.obj
 0003:0000011c       ?staticMetaObject@ClarkSupportPlugin@U2@@2UQMetaObject@@B 1003311c     moc_ClarkSupportPlugin.obj
 0003:00000134       ___security_cookie         10033134     MSVCRT:gs_cookie.obj
 0003:00000138       ___security_cookie_complement 10033138     MSVCRT:gs_cookie.obj
 0003:00000140       ___native_dllmain_reason   10033140     MSVCRT:natstart.obj
 0003:00000148       ??_R0?AVerror_category@std@@@8 10033148     ClarkBuildWorker.obj
 0003:0000016c       ??_R0?AV_Generic_error_category@std@@@8 1003316c     ClarkBuildWorker.obj
 0003:00000198       ??_R0?AV_Iostream_error_category@std@@@8 10033198     ClarkBuildWorker.obj
 0003:000001c4       ??_R0?AV_System_error_category@std@@@8 100331c4     ClarkBuildWorker.obj
 0003:000001f0       ??_R0?AVQObject@@@8        100331f0     ClarkBuildWorker.obj
 0003:00000208       ??_R0?AVFailTask@U2@@@8    10033208     ClarkBuildWorker.obj
 0003:00000224       ??_R0?AVTask@U2@@@8        10033224     ClarkBuildWorker.obj
 0003:0000023c       ??_R0?AVTaskSignalMapper@U2@@@8 1003323c     ClarkBuildWorker.obj
 0003:00000260       ??_R0?AVDescriptor@U2@@@8  10033260     ClarkBuildWorker.obj
 0003:0000027c       ??_R0?AVMapDataType@U2@@@8 1003327c     ClarkBuildWorker.obj
 0003:0000029c       ??_R0?AVDataType@U2@@@8    1003329c     ClarkBuildWorker.obj
 0003:000002b8       ??_R0?AVQSharedData@@@8    100332b8     ClarkBuildWorker.obj
 0003:000002d4       ??_R0?AVAttribute@U2@@@8   100332d4     ClarkBuildWorker.obj
 0003:000002f0       ??_R0?AVConfigurationEditor@U2@@@8 100332f0     ClarkBuildWorker.obj
 0003:00000318       ??_R0?AVDelegateEditor@U2@@@8 10033318     ClarkBuildWorker.obj
 0003:00000338       ??_R0?AVURLDelegate@U2@@@8 10033338     ClarkBuildWorker.obj
 0003:00000358       ??_R0?AVPropertyDelegate@U2@@@8 10033358     ClarkBuildWorker.obj
 0003:0000037c       ??_R0?AVQItemDelegate@@@8  1003337c     ClarkBuildWorker.obj
 0003:00000398       ??_R0?AVQAbstractItemDelegate@@@8 10033398     ClarkBuildWorker.obj
 0003:000003bc       ??_R0?AVComboBoxDelegate@U2@@@8 100333bc     ClarkBuildWorker.obj
 0003:000003e0       ??_R0?AVPortDescriptor@Workflow@U2@@@8 100333e0     ClarkBuildWorker.obj
 0003:0000040c       ??_R0?AVIntegralBusActorPrototype@Workflow@U2@@@8 1003340c     ClarkBuildWorker.obj
 0003:00000440       ??_R0?AVActorPrototype@Workflow@U2@@@8 10033440     ClarkBuildWorker.obj
 0003:0000046c       ??_R0?AVVisualDescriptor@U2@@@8 1003346c     ClarkBuildWorker.obj
 0003:00000490       ??_R0?AVExternalToolRunTask@U2@@@8 10033490     ClarkBuildWorker.obj
 0003:000004b8       ??_R0?AVClarkBuildValidator@LocalWorkflow@U2@@@8 100334b8     ClarkBuildWorker.obj
 0003:000004ec       ??_R0?AVActorValidator@Workflow@U2@@@8 100334ec     ClarkBuildWorker.obj
 0003:00000518       ??_R0?AVConfigurationValidator@U2@@@8 10033518     ClarkBuildWorker.obj
 0003:00000540       ??_R0?AVClarkBuildPrompter@LocalWorkflow@U2@@@8 10033540     ClarkBuildWorker.obj
 0003:00000578       ??_R0?AV?$PrompterBase@VClarkBuildPrompter@LocalWorkflow@U2@@@U2@@@8 10033578     ClarkBuildWorker.obj
 0003:000005c0       ??_R0?AVPrompterBaseImpl@U2@@@8 100335c0     ClarkBuildWorker.obj
 0003:000005e4       ??_R0?AVActorDocument@Workflow@U2@@@8 100335e4     ClarkBuildWorker.obj
 0003:0000060c       ??_R0?AVQTextDocument@@@8  1003360c     ClarkBuildWorker.obj
 0003:00000628       ??_R0?AVPrompter@Workflow@U2@@@8 10033628     ClarkBuildWorker.obj
 0003:0000064c       ??_R0?AVClarkBuildWorker@LocalWorkflow@U2@@@8 1003364c     ClarkBuildWorker.obj
 0003:0000067c       ??_R0?AVBaseWorker@LocalWorkflow@U2@@@8 1003367c     ClarkBuildWorker.obj
 0003:000006a8       ??_R0?AVWorker@Workflow@U2@@@8 100336a8     ClarkBuildWorker.obj
 0003:000006cc       ??_R0?AVCommunicationSubject@Workflow@U2@@@8 100336cc     ClarkBuildWorker.obj
 0003:000006fc       ??_R0?AVClarkBuildWorkerFactory@LocalWorkflow@U2@@@8 100336fc     ClarkBuildWorker.obj
 0003:00000734       ??_R0?AVDomainFactory@Workflow@U2@@@8 10033734     ClarkBuildWorker.obj
 0003:0000075c       ??_R0?AV?$IdRegistry@VDomainFactory@Workflow@U2@@@U2@@@8 1003375c     ClarkBuildWorker.obj
 0003:00000798       ??_R0?AVClarkBuildTask@LocalWorkflow@U2@@@8 10033798     ClarkBuildWorker.obj
 0003:000007c8       ??_R0?AVExternalToolSupportTask@U2@@@8 100337c8     ClarkBuildWorker.obj
 0003:000007f4       ??_R0?AVGenomicLibraryDelegate@LocalWorkflow@U2@@@8 100337f4     ClarkBuildWorker.obj
 0003:0000082c       ??_R0?AVClarkBuildLogParser@LocalWorkflow@U2@@@8 1003382c     ClarkBuildWorker.obj
 0003:00000860       ??_R0?AVExternalToolLogParser@U2@@@8 10033860     ClarkBuildWorker.obj
 0003:00000888       ??_R0?AVVisibilityRelation@U2@@@8 10033888     ClarkClassifyWorker.obj
 0003:000008ac       ??_R0?AVAttributeRelation@U2@@@8 100338ac     ClarkClassifyWorker.obj
 0003:000008d0       ??_R0?AVSlotRelationDescriptor@U2@@@8 100338d0     ClarkClassifyWorker.obj
 0003:000008f8       ??_R0?AVSpinBoxDelegate@U2@@@8 100338f8     ClarkClassifyWorker.obj
 0003:0000091c       ??_R0?AVPairedReadsPortValidator@Workflow@U2@@@8 1003391c     ClarkClassifyWorker.obj
 0003:00000950       ??_R0?AVPortValidator@Workflow@U2@@@8 10033950     ClarkClassifyWorker.obj
 0003:00000978       ??_R0?AVClarkClassifyPrompter@LocalWorkflow@U2@@@8 10033978     ClarkClassifyWorker.obj
 0003:000009b0       ??_R0?AV?$PrompterBase@VClarkClassifyPrompter@LocalWorkflow@U2@@@U2@@@8 100339b0     ClarkClassifyWorker.obj
 0003:000009fc       ??_R0?AVClarkClassifyWorker@LocalWorkflow@U2@@@8 100339fc     ClarkClassifyWorker.obj
 0003:00000a30       ??_R0?AVClarkClassifyValidator@LocalWorkflow@U2@@@8 10033a30     ClarkClassifyWorker.obj
 0003:00000a68       ??_R0?AVClarkClassifyWorkerFactory@LocalWorkflow@U2@@@8 10033a68     ClarkClassifyWorker.obj
 0003:00000aa4       ??_R0?AVClarkLogParser@LocalWorkflow@U2@@@8 10033aa4     ClarkClassifyWorker.obj
 0003:00000ad4       ??_R0?AVClarkClassifyTask@LocalWorkflow@U2@@@8 10033ad4     ClarkClassifyWorker.obj
 0003:00000b08       ??_R0?AVDatabaseDelegate@LocalWorkflow@U2@@@8 10033b08     ClarkClassifyWorker.obj
 0003:00000b38       ??_R0?AVAbstractInt32Id@U2@@@8 10033b38     ClarkSupport.obj
 0003:00000b5c       ??_R0?AV?$AbstractId@H@U2@@@8 10033b5c     ClarkSupport.obj
 0003:00000b7c       ??_R0?AVServiceType@U2@@@8 10033b7c     ClarkSupport.obj
 0003:00000b9c       ??_R0?AVClarkSupport@U2@@@8 10033b9c     ClarkSupport.obj
 0003:00000bbc       ??_R0?AVExternalTool@U2@@@8 10033bbc     ClarkSupport.obj
 0003:00000bdc       ??_R0?AVClarkSupportPlugin@U2@@@8 10033bdc     ClarkSupportPlugin.obj
 0003:00000c00       ??_R0?AVPlugin@U2@@@8      10033c00     ClarkSupportPlugin.obj
 0003:00000c18       ??_R0?AV?$GAutoDeleteList@VXMLTestFactory@U2@@@U2@@@8 10033c18     ClarkSupportPlugin.obj
 0003:00000c50       ??_R0?AVXmlTest@U2@@@8     10033c50     ClarkTests.obj
 0003:00000c6c       ??_R0?AVGTest@U2@@@8       10033c6c     ClarkTests.obj
 0003:00000c84       ??_R0?AVXMLTestFactory@U2@@@8 10033c84     ClarkTests.obj
 0003:00000ca4       ??_R0?AVGTest_CompareClarkDatabaseMetafiles@U2@@@8 10033ca4     ClarkTests.obj
 0003:00000ce0       ??_R0?AVGTest_CompareClarkDatabaseMetafilesFactory@GTest_CompareClarkDatabaseMetafiles@U2@@@8 10033ce0     ClarkTests.obj
 0003:00000d40       ??_R0?AVtype_info@@@8      10033d40     MSVCRT:ti_inst.obj
 0003:00000da0       ?wellKnownErrors@ClarkBuildLogParser@LocalWorkflow@U2@@0VQStringList@@B 10033da0     ClarkBuildWorker.obj
 0003:00000db8       ?ACTOR_ID@ClarkBuildWorkerFactory@LocalWorkflow@U2@@0VQString@@B 10033db8     ClarkBuildWorker.obj
 0003:00000dbc       ?id@?$num_put@DV?$back_insert_iterator@V?$basic_string@DU?$char_traits@D@std@@V?$allocator@D@2@@std@@@std@@@std@@2V0locale@2@A 10033dbc     ClarkBuildWorker.obj
 0003:00000dc0       ?id@?$num_put@_WV?$back_insert_iterator@V?$basic_string@_WU?$char_traits@_W@std@@V?$allocator@_W@2@@std@@@std@@@std@@2V0locale@2@A 10033dc0     ClarkBuildWorker.obj
 0003:00000dc4       ?metatype_id@?1??qt_metatype_id@?$QMetaTypeId@V?$QList@VDataset@U2@@@@@@SAHXZ@4V?$QBasicAtomicInteger@H@@A 10033dc4     ClarkBuildWorker.obj
 0003:00000dfc       ?INPUT_SLOT@ClarkClassifyWorkerFactory@LocalWorkflow@U2@@2VQString@@B 10033dfc     ClarkClassifyWorker.obj
 0003:00000e00       ?OUTPUT_URL@ClarkClassifyWorkerFactory@LocalWorkflow@U2@@2VQString@@B 10033e00     ClarkClassifyWorker.obj
 0003:00000e04       ?FACTOR@ClarkClassifyWorkerFactory@LocalWorkflow@U2@@2VQString@@B 10033e04     ClarkClassifyWorker.obj
 0003:00000e08       ?NUM_THREADS@ClarkClassifyWorkerFactory@LocalWorkflow@U2@@2VQString@@B 10033e08     ClarkClassifyWorker.obj
 0003:00000e0c       ?WORKFLOW_CLASSIFY_TOOL_CLARK@ClarkClassifyWorkerFactory@LocalWorkflow@U2@@2VQString@@B 10033e0c     ClarkClassifyWorker.obj
 0003:00000e38       ?ACTOR_ID@ClarkClassifyWorkerFactory@LocalWorkflow@U2@@2VQString@@B 10033e38     ClarkClassifyWorker.obj
 0003:00000e3c       ?DB_URL@ClarkClassifyWorkerFactory@LocalWorkflow@U2@@2VQString@@B 10033e3c     ClarkClassifyWorker.obj
 0003:00000e40       ?MODE@ClarkClassifyWorkerFactory@LocalWorkflow@U2@@2VQString@@B 10033e40     ClarkClassifyWorker.obj
 0003:00000e44       ?TOOL_DEFAULT@ClarkClassifySettings@LocalWorkflow@U2@@2VQString@@B 10033e44     ClarkClassifyWorker.obj
 0003:00000e48       ?TOOL_LIGHT@ClarkClassifySettings@LocalWorkflow@U2@@2VQString@@B 10033e48     ClarkClassifyWorker.obj
 0003:00000e4c       ?wellKnownErrors@ClarkLogParser@LocalWorkflow@U2@@0V?$QMap@VQString@@V1@@@B 10033e4c     ClarkClassifyWorker.obj
 0003:00000e64       ?EXTEND_OUT@ClarkClassifyWorkerFactory@LocalWorkflow@U2@@2VQString@@B 10033e64     ClarkClassifyWorker.obj
 0003:00000e68       ?TAXONOMY@ClarkClassifyWorkerFactory@LocalWorkflow@U2@@2VQString@@B 10033e68     ClarkClassifyWorker.obj
 0003:00000e6c       ?K_LENGTH@ClarkClassifyWorkerFactory@LocalWorkflow@U2@@2VQString@@B 10033e6c     ClarkClassifyWorker.obj
 0003:00000e70       ?PAIRED_INPUT_PORT@ClarkClassifyWorkerFactory@LocalWorkflow@U2@@2VQString@@B 10033e70     ClarkClassifyWorker.obj
 0003:00000e7c       ?INPUT_PORT@ClarkClassifyWorkerFactory@LocalWorkflow@U2@@2VQString@@B 10033e7c     ClarkClassifyWorker.obj
 0003:00000e80       ?K_MIN_FREQ@ClarkClassifyWorkerFactory@LocalWorkflow@U2@@2VQString@@B 10033e80     ClarkClassifyWorker.obj
 0003:00000e84       ?SEQUENCING_READS@ClarkClassifyWorkerFactory@LocalWorkflow@U2@@2VQString@@B 10033e84     ClarkClassifyWorker.obj
 0003:00000e90       ?DB_TO_RAM@ClarkClassifyWorkerFactory@LocalWorkflow@U2@@2VQString@@B 10033e90     ClarkClassifyWorker.obj
 0003:00000e94       ?TOOL_VARIANT@ClarkClassifyWorkerFactory@LocalWorkflow@U2@@2VQString@@B 10033e94     ClarkClassifyWorker.obj
 0003:00000e98       ?SINGLE_END@ClarkClassifyWorkerFactory@LocalWorkflow@U2@@2VQString@@B 10033e98     ClarkClassifyWorker.obj
 0003:00000e9c       ?OUTPUT_PORT@ClarkClassifyWorkerFactory@LocalWorkflow@U2@@2VQString@@B 10033e9c     ClarkClassifyWorker.obj
 0003:00000ea0       ?TAXONOMY_RANK@ClarkClassifyWorkerFactory@LocalWorkflow@U2@@2VQString@@B 10033ea0     ClarkClassifyWorker.obj
 0003:00000ea4       ?GAP@ClarkClassifyWorkerFactory@LocalWorkflow@U2@@2VQString@@B 10033ea4     ClarkClassifyWorker.obj
 0003:00000ea8       ?PAIRED_INPUT_SLOT@ClarkClassifyWorkerFactory@LocalWorkflow@U2@@2VQString@@B 10033ea8     ClarkClassifyWorker.obj
 0003:00000eac       ?PAIRED_END@ClarkClassifyWorkerFactory@LocalWorkflow@U2@@2VQString@@B 10033eac     ClarkClassifyWorker.obj
 0003:00000eb0       ?metatype_id@?1??qt_metatype_id@?$QMetaTypeId@VQAssociativeIterableImpl@QtMetaTypePrivate@@@@SAHXZ@4V?$QBasicAtomicInteger@H@@A 10033eb0     ClarkClassifyWorker.obj
 0003:00000eb4       ?metatype_id@?1??qt_metatype_id@?$QMetaTypeId@V?$QMap@VQString@@I@@@@SAHXZ@4V?$QBasicAtomicInteger@H@@A 10033eb4     ClarkClassifyWorker.obj
 0003:00000ee4       ?f@?4??registerConverter@?$AssociativeValueTypeIsMetaType@V?$QMap@VQString@@I@@$00@QtPrivate@@SA_NH@Z@4U?$ConverterFunctor@V?$QMap@VQString@@I@@VQAssociativeIterableImpl@QtMetaTypePrivate@@U?$QAssociativeIterableConvertFunctor@V?$QMap@VQString@@I@@@3@@3@B 10033ee4     ClarkClassifyWorker.obj
 0003:00000eec       ??_B?4??registerConverter@?$AssociativeValueTypeIsMetaType@V?$QMap@VQString@@I@@$00@QtPrivate@@SA_NH@Z@54 10033eec     ClarkClassifyWorker.obj
 0003:00000ef4       ?ET_CLARK_GET_FILES_TO_TAX_NODES@ClarkSupport@U2@@2VQString@@B 10033ef4     ClarkSupport.obj
 0003:00000f00       ?CLARK_GROUP@ClarkSupport@U2@@2VQString@@B 10033f00     ClarkSupport.obj
 0003:00000f0c       ?ET_CLARK_GET_ACCSSN_TAX_ID_ID@ClarkSupport@U2@@2VQString@@B 10033f0c     ClarkSupport.obj
 0003:00000f18       ?ET_CLARK_L_ID@ClarkSupport@U2@@2VQString@@B 10033f18     ClarkSupport.obj
 0003:00000f24       ?ET_CLARK_BUILD_SCRIPT_ID@ClarkSupport@U2@@2VQString@@B 10033f24     ClarkSupport.obj
 0003:00000f40       ?ET_CLARK@ClarkSupport@U2@@2VQString@@B 10033f40     ClarkSupport.obj
 0003:00000f44       ?ET_CLARK_ID@ClarkSupport@U2@@2VQString@@B 10033f44     ClarkSupport.obj
 0003:00000f50       ?ET_CLARK_GET_ACCSSN_TAX_ID@ClarkSupport@U2@@2VQString@@B 10033f50     ClarkSupport.obj
 0003:00000f54       ?ET_CLARK_BUILD_SCRIPT@ClarkSupport@U2@@2VQString@@B 10033f54     ClarkSupport.obj
 0003:00000f58       ?ET_CLARK_L@ClarkSupport@U2@@2VQString@@B 10033f58     ClarkSupport.obj
 0003:00000f5c       ?ET_CLARK_GET_TARGETS_DEF@ClarkSupport@U2@@2VQString@@B 10033f5c     ClarkSupport.obj
 0003:00000f68       ?ET_CLARK_GET_FILES_TO_TAX_NODES_ID@ClarkSupport@U2@@2VQString@@B 10033f68     ClarkSupport.obj
 0003:00000f6c       ?ET_CLARK_GET_TARGETS_DEF_ID@ClarkSupport@U2@@2VQString@@B 10033f6c     ClarkSupport.obj
 0003:00000f94       ?PLUGIN_DESCRIPRION@ClarkSupportPlugin@U2@@2VQString@@B 10033f94     ClarkSupportPlugin.obj
 0003:00000fa0       ?PLUGIN_NAME@ClarkSupportPlugin@U2@@2VQString@@B 10033fa0     ClarkSupportPlugin.obj
 0003:00000fd8       ?DATABASE_METAFILES@GTest_CompareClarkDatabaseMetafiles@U2@@0VQStringList@@B 10033fd8     ClarkTests.obj
 0003:00000ff4       ?DATABASE2@GTest_CompareClarkDatabaseMetafiles@U2@@0VQString@@B 10033ff4     ClarkTests.obj
 0003:00001008       ?DATABASE_PREFIX_PLACEHOLDER@GTest_CompareClarkDatabaseMetafiles@U2@@0VQString@@B 10034008     ClarkTests.obj
 0003:0000101c       ?DATABASE1@GTest_CompareClarkDatabaseMetafiles@U2@@0VQString@@B 1003401c     ClarkTests.obj
 0003:00001020       ?PREFIXES_SEPARATOR@GTest_CompareClarkDatabaseMetafiles@U2@@0VQString@@B 10034020     ClarkTests.obj
 0003:00001024       ?DATABASE1_PREFIXES@GTest_CompareClarkDatabaseMetafiles@U2@@0VQString@@B 10034024     ClarkTests.obj
 0003:00001028       ?DATABASE2_PREFIXES@GTest_CompareClarkDatabaseMetafiles@U2@@0VQString@@B 10034028     ClarkTests.obj
 0003:00001078       ?metatype_id@?1??qt_metatype_id@?$QMetaTypeIdQObject@PAVTask@U2@@$00@@SAHXZ@4V?$QBasicAtomicInteger@H@@A 10034078     moc_ClarkBuildWorker.obj
 0003:000013f8       ?__type_info_root_node@@3U__type_info_node@@A 100343f8     MSVCRT:tncleanup.obj
 0003:00001400       ___native_startup_lock     10034400     <common>
 0003:00001404       ___native_startup_state    10034404     <common>
 0003:00001408       ___dyn_tls_init_callback   10034408     <common>
 0003:0000140c       ___onexitend               1003440c     <common>
 0003:00001410       ___onexitbegin             10034410     <common>

 entry point at        0001:00018d40

 Static symbols

 0000:fffc5000       .debug$S                   10000000     MSVCRT:MSVCR120.dll
 0000:fffc5000       .debug$S                   10000000     MSVCRT:MSVCR120.dll
 0000:fffc5000       .debug$S                   10000000     MSVCRT:MSVCR120.dll
 0000:fffc5000       .debug$S                   10000000     MSVCRT:MSVCR120.dll
 0000:fffc5000       .debug$S                   10000000     MSVCRT:MSVCR120.dll
 0000:fffc5000       .debug$S                   10000000     MSVCRT:MSVCR120.dll
 0000:fffc5000       .debug$S                   10000000     MSVCRT:MSVCR120.dll
 0000:fffc5000       .debug$S                   10000000     MSVCRT:MSVCR120.dll
 0000:fffc5000       .debug$S                   10000000     MSVCRT:MSVCR120.dll
 0001:fffff000       __unwindfunclet$?createNode@?$QMapData@VQString@@VQVariant@@@@QAEPAU?$QMapNode@VQString@@VQVariant@@@@ABVQString@@ABVQVariant@@PAU2@_N@Z$4 10000000 f   ClarkClassifyWorker.obj
 0001:fffff000       __unwindfunclet$?createNode@?$QMapData@VQString@@VQScriptValue@@@@QAEPAU?$QMapNode@VQString@@VQScriptValue@@@@ABVQString@@ABVQScriptValue@@PAU2@_N@Z$4 10000000 f   ClarkClassifyWorker.obj
 0000:fffc5000       .debug$S                   10000000     MSVCRT:MSVCR120.dll
 0001:fffff000       __unwindfunclet$?createNode@?$QMapData@VDescriptor@U2@@V?$QExplicitlySharedDataPointer@VDataType@U2@@@@@@QAEPAU?$QMapNode@VDescriptor@U2@@V?$QExplicitlySharedDataPointer@VDataType@U2@@@@@@ABVDescriptor@U2@@ABV?$QExplicitlySharedDataPointer@VDataType@U2@@@@PAU2@_N@Z$4 10000000 f   ClarkClassifyWorker.obj
 0000:fffc5000       .debug$S                   10000000     MSVCRT:MSVCR120.dll
 0001:fffff000       __unwindfunclet$?createNode@?$QMapData@VQString@@PAVPropertyDelegate@U2@@@@QAEPAU?$QMapNode@VQString@@PAVPropertyDelegate@U2@@@@ABVQString@@ABQAVPropertyDelegate@U2@@PAU2@_N@Z$4 10000000 f   ClarkClassifyWorker.obj
 0000:fffc5000       .debug$S                   10000000     MSVCRT:MSVCR120.dll
 0001:fffff000       __ehhandler$?_Copy@?$basic_string@DU?$char_traits@D@std@@V?$allocator@D@2@@std@@QAEXII@Z 10000000 f   moc_ClarkSupportPlugin.obj
 0001:fffff000       __ehhandler$??0?$QList@PAVPort@Workflow@U2@@@@QAE@ABV0@@Z 10000000 f   ClarkClassifyWorker.obj
 0001:fffff000       __unwindfunclet$?metaType@?$QVariantValueHelper@VQString@@@QtPrivate@@SA?AVQString@@ABVQVariant@@@Z$0 10000000 f   ClarkClassifyWorker.obj
 0002:fffe0000       __catchsym$?_Copy@?$basic_string@DU?$char_traits@D@std@@V?$allocator@D@2@@std@@QAEXII@Z$5 10000000     ClarkClassifyWorker.obj
 0002:fffe0000       __unwindtable$??H@YA?BVQString@@ABV0@PBD@Z 10000000     ClarkClassifyWorker.obj
 0002:fffe0000       __catchsym$??0?$QList@VQString@@@@QAE@ABV0@@Z$2 10000000     ClarkClassifyWorker.obj
 0002:fffe0000       __catchsym$?append@?$QList@VQString@@@@QAEXABVQString@@@Z$13 10000000     ClarkClassifyWorker.obj
 0002:fffe0000       __catchsym$?_Copy@?$basic_string@DU?$char_traits@D@std@@V?$allocator@D@2@@std@@QAEXII@Z$5 10000000     moc_ClarkSupportPlugin.obj
 0000:fffc5000       .debug$S                   10000000     MSVCRT:MSVCR120.dll
 0000:fffc5000       .debug$S                   10000000     MSVCRT:MSVCR120.dll
 0000:fffc5000       .debug$S                   10000000     MSVCRT:MSVCR120.dll
 0000:fffc5000       .debug$S                   10000000     MSVCRT:MSVCR120.dll
 0000:fffc5000       .debug$S                   10000000     MSVCRT:MSVCR120.dll
 0002:fffe0000       ?_Generic_object$initializer$@?$_Error_objects@H@std@@2P6AXXZA 10000000     moc_ClarkSupportPlugin.obj
 0002:fffe0000       ?_Iostream_object$initializer$@?$_Error_objects@H@std@@2P6AXXZA 10000000     moc_ClarkSupportPlugin.obj
 0002:fffe0000       ?_System_object$initializer$@?$_Error_objects@H@std@@2P6AXXZA 10000000     moc_ClarkSupportPlugin.obj
 0000:fffc5000       .debug$S                   10000000     MSVCRT:MSVCR120.dll
 0000:fffc5000       .debug$S                   10000000     MSVCRT:MSVCR120.dll
 0002:fffe0000       __catchsym$?detach_helper_grow@?$QList@VQString@@@@AAEPAUNode@1@HH@Z$5 10000000     ClarkClassifyWorker.obj
 0002:fffe0000       __unwindtable$?node_construct@?$QList@VQString@@@@AAEXPAUNode@1@ABVQString@@@Z 10000000     ClarkClassifyWorker.obj
 0000:fffc5000       .debug$S                   10000000     MSVCRT:MSVCR120.dll
 0002:fffe0000       __catchsym$?node_copy@?$QList@VQString@@@@AAEXPAUNode@1@00@Z$6 10000000     ClarkClassifyWorker.obj
 0000:fffc5000       .debug$S                   10000000     MSVCRT:MSVCR120.dll
 0002:fffe0000       __unwindtable$??A?$QMap@VQString@@VQVariant@@@@QAEAAVQVariant@@ABVQString@@@Z 10000000     ClarkClassifyWorker.obj
 0000:fffc5000       .debug$S                   10000000     MSVCRT:MSVCR120.dll
 0001:fffff000       __ehhandler$?_Copy@?$basic_string@DU?$char_traits@D@std@@V?$allocator@D@2@@std@@QAEXII@Z 10000000 f   moc_ClarkSupport.obj
 0002:fffe0000       __unwindtable$??A?$QMap@VQString@@VQScriptValue@@@@QAEAAVQScriptValue@@ABVQString@@@Z 10000000     ClarkClassifyWorker.obj
 0002:fffe0000       __catchsym$??0?$QList@VDescriptor@U2@@@@QAE@ABV0@@Z$2 10000000     ClarkClassifyWorker.obj
 0002:fffe0000       __catchsym$?append@?$QList@VDescriptor@U2@@@@QAEXABVDescriptor@U2@@@Z$9 10000000     ClarkClassifyWorker.obj
 0002:fffe0000       __catchsym$?detach_helper_grow@?$QList@VDescriptor@U2@@@@AAEPAUNode@1@HH@Z$5 10000000     ClarkClassifyWorker.obj
 0002:fffe0000       __catchsym$?detach_helper@?$QList@VDescriptor@U2@@@@AAEXH@Z$2 10000000     ClarkClassifyWorker.obj
 0002:fffe0000       __unwindtable$?node_construct@?$QList@VDescriptor@U2@@@@AAEXPAUNode@1@ABVDescriptor@U2@@@Z 10000000     ClarkClassifyWorker.obj
 0002:fffe0000       __catchsym$?_Copy@?$basic_string@DU?$char_traits@D@std@@V?$allocator@D@2@@std@@QAEXII@Z$5 10000000     moc_ClarkSupport.obj
 0000:fffc5000       .debug$S                   10000000     MSVCRT:MSVCR120.dll
 0000:fffc5000       .debug$S                   10000000     MSVCRT:MSVCR120.dll
 0000:fffc5000       .debug$S                   10000000     MSVCRT:MSVCR120.dll
 0000:fffc5000       .debug$S                   10000000     MSVCRT:MSVCR120.dll
 0002:fffe0000       __catchsym$?node_copy@?$QList@VDescriptor@U2@@@@AAEXPAUNode@1@00@Z$6 10000000     ClarkClassifyWorker.obj
 0002:fffe0000       ?_Generic_object$initializer$@?$_Error_objects@H@std@@2P6AXXZA 10000000     moc_ClarkSupport.obj
 0002:fffe0000       ?_Iostream_object$initializer$@?$_Error_objects@H@std@@2P6AXXZA 10000000     moc_ClarkSupport.obj
 0002:fffe0000       ?_System_object$initializer$@?$_Error_objects@H@std@@2P6AXXZA 10000000     moc_ClarkSupport.obj
 0002:fffe0000       __unwindtable$??A?$QMap@VDescriptor@U2@@V?$QExplicitlySharedDataPointer@VDataType@U2@@@@@@QAEAAV?$QExplicitlySharedDataPointer@VDataType@U2@@@@ABVDescriptor@U2@@@Z 10000000     ClarkClassifyWorker.obj
 0002:fffe0000       __unwindtable$?uniqueKeys@?$QMap@VDescriptor@U2@@VQVariant@@@@QBE?AV?$QList@VDescriptor@U2@@@@XZ 10000000     ClarkClassifyWorker.obj
 0002:fffe0000       __ehfuncinfo$??$getAttributeValue@VQString@@@Attribute@U2@@QBE?AVQString@@PAVWorkflowContext@Workflow@1@@Z 10000000     ClarkClassifyWorker.obj
 0000:fffc5000       .debug$S                   10000000     msvcprt:MSVCP120.dll
 0000:fffc5000       .debug$S                   10000000     msvcprt:MSVCP120.dll
 0000:fffc5000       .debug$S                   10000000     msvcprt:MSVCP120.dll
 0002:fffe0000       __ehfuncinfo$??$getAttributeValue@H@Attribute@U2@@QBEHPAVWorkflowContext@Workflow@1@@Z 10000000     ClarkClassifyWorker.obj
 0000:fffc5000       .debug$S                   10000000     msvcprt:MSVCP120.dll
 0002:fffe0000       __catchsym$?append@?$QList@PAVAttribute@U2@@@@QAEXABQAVAttribute@U2@@@Z$6 10000000     ClarkClassifyWorker.obj
 0000:fffc5000       .debug$S                   10000000     msvcprt:MSVCP120.dll
 0002:fffe0000       __catchsym$?detach_helper_grow@?$QList@PAVAttribute@U2@@@@AAEPAUNode@1@HH@Z$5 10000000     ClarkClassifyWorker.obj
 0000:fffc5000       .debug$S                   10000000     kernel32:KERNEL32.dll
 0002:fffe0000       __catchsym$?append@?$QList@PAVPortDescriptor@Workflow@U2@@@@QAEXABQAVPortDescriptor@Workflow@U2@@@Z$6 10000000     ClarkClassifyWorker.obj
 0000:fffc5000       .debug$S                   10000000     kernel32:KERNEL32.dll
 0002:fffe0000       __catchsym$?detach_helper_grow@?$QList@PAVPortDescriptor@Workflow@U2@@@@AAEPAUNode@1@HH@Z$5 10000000     ClarkClassifyWorker.obj
 0000:fffc5000       .debug$S                   10000000     kernel32:KERNEL32.dll
 0002:fffe0000       __catchsym$?append@?$QList@VWorkflowNotification@U2@@@@QAEXABVWorkflowNotification@U2@@@Z$11 10000000     ClarkClassifyWorker.obj
 0000:fffc5000       .debug$S                   10000000     kernel32:KERNEL32.dll
 0002:fffe0000       __catchsym$?detach_helper_grow@?$QList@VWorkflowNotification@U2@@@@AAEPAUNode@1@HH@Z$5 10000000     ClarkClassifyWorker.obj
 0000:fffc5000       .debug$S                   10000000     kernel32:KERNEL32.dll
 0002:fffe0000       __unwindtable$?node_construct@?$QList@VWorkflowNotification@U2@@@@AAEXPAUNode@1@ABVWorkflowNotification@U2@@@Z 10000000     ClarkClassifyWorker.obj
 0000:fffc5000       .debug$S                   10000000     kernel32:KERNEL32.dll
 0002:fffe0000       __catchsym$?node_copy@?$QList@VWorkflowNotification@U2@@@@AAEXPAUNode@1@00@Z$6 10000000     ClarkClassifyWorker.obj
 0000:fffc5000       .debug$S                   10000000     kernel32:KERNEL32.dll
 0002:fffe0000       __unwindtable$??$getValue@VQString@@@BaseWorker@LocalWorkflow@U2@@IBE?AVQString@@ABV3@@Z 10000000     ClarkClassifyWorker.obj
 0002:fffe0000       __catchsym$?createNode@?$QMapData@VQString@@VQVariant@@@@QAEPAU?$QMapNode@VQString@@VQVariant@@@@ABVQString@@ABVQVariant@@PAU2@_N@Z$7 10000000     ClarkClassifyWorker.obj
 0002:fffe0000       __catchsym$?createNode@?$QMapData@VQString@@VQScriptValue@@@@QAEPAU?$QMapNode@VQString@@VQScriptValue@@@@ABVQString@@ABVQScriptValue@@PAU2@_N@Z$7 10000000     ClarkClassifyWorker.obj
 0002:fffe0000       __catchsym$?createNode@?$QMapData@VDescriptor@U2@@V?$QExplicitlySharedDataPointer@VDataType@U2@@@@@@QAEPAU?$QMapNode@VDescriptor@U2@@V?$QExplicitlySharedDataPointer@VDataType@U2@@@@@@ABVDescriptor@U2@@ABV?$QExplicitlySharedDataPointer@VDataType@U2@@@@PAU2@_N@Z$6 10000000     ClarkClassifyWorker.obj
 0000:fffc5000       .debug$S                   10000000     kernel32:KERNEL32.dll
 0002:fffe0000       __catchsym$?createNode@?$QMapData@VQString@@PAVPropertyDelegate@U2@@@@QAEPAU?$QMapNode@VQString@@PAVPropertyDelegate@U2@@@@ABVQString@@ABQAVPropertyDelegate@U2@@PAU2@_N@Z$5 10000000     ClarkClassifyWorker.obj
 0000:fffc5000       .debug$S                   10000000     kernel32:KERNEL32.dll
 0002:fffe0000       __catchsym$??0?$QList@PAVPort@Workflow@U2@@@@QAE@ABV0@@Z$2 10000000     ClarkClassifyWorker.obj
 0000:fffc5000       .debug$S                   10000000     Qt5Core:Qt5Core.dll
 0001:fffff000       __ehhandler$?_Copy@?$basic_string@DU?$char_traits@D@std@@V?$allocator@D@2@@std@@QAEXII@Z 10000000 f   moc_ClarkClassifyWorker.obj
 0002:fffe0000       __unwindtable$?metaType@?$QVariantValueHelper@VQString@@@QtPrivate@@SA?AVQString@@ABVQVariant@@@Z 10000000     ClarkClassifyWorker.obj
 0002:fffe0000       ?_Generic_object$initializer$@?$_Error_objects@H@std@@2P6AXXZA 10000000     ClarkClassifyWorker.obj
 0000:fffc5000       .debug$S                   10000000     Qt5Core:Qt5Core.dll
 0000:fffc5000       .debug$S                   10000000     Qt5Core:Qt5Core.dll
 0000:fffc5000       .debug$S                   10000000     Qt5Core:Qt5Core.dll
 0000:fffc5000       .debug$S                   10000000     Qt5Core:Qt5Core.dll
 0000:fffc5000       .debug$S                   10000000     Qt5Core:Qt5Core.dll
 0000:fffc5000       .debug$S                   10000000     Qt5Core:Qt5Core.dll
 0000:fffc5000       .debug$S                   10000000     Qt5Core:Qt5Core.dll
 0000:fffc5000       .debug$S                   10000000     Qt5Core:Qt5Core.dll
 0000:fffc5000       .debug$S                   10000000     Qt5Core:Qt5Core.dll
 0000:fffc5000       .debug$S                   10000000     Qt5Core:Qt5Core.dll
 0000:fffc5000       .debug$S                   10000000     Qt5Core:Qt5Core.dll
 0000:fffc5000       .debug$S                   10000000     Qt5Core:Qt5Core.dll
 0000:fffc5000       .debug$S                   10000000     Qt5Core:Qt5Core.dll
 0000:fffc5000       .debug$S                   10000000     Qt5Core:Qt5Core.dll
 0000:fffc5000       .debug$S                   10000000     Qt5Core:Qt5Core.dll
 0000:fffc5000       .debug$S                   10000000     Qt5Core:Qt5Core.dll
 0000:fffc5000       .debug$S                   10000000     Qt5Core:Qt5Core.dll
 0000:fffc5000       .debug$S                   10000000     Qt5Core:Qt5Core.dll
 0002:fffe0000       ?_Iostream_object$initializer$@?$_Error_objects@H@std@@2P6AXXZA 10000000     ClarkClassifyWorker.obj
 0001:fffff000       __unwindfunclet$?qt_metatype_id@?$QMetaTypeIdQObject@PAVTask@U2@@$00@@SAHXZ$0 10000000 f   moc_ClarkClassifyWorker.obj
 0002:fffe0000       ?_System_object$initializer$@?$_Error_objects@H@std@@2P6AXXZA 10000000     ClarkClassifyWorker.obj
 0001:fffff000       __unwindfunclet$??$getValue@VQString@@@BaseWorker@LocalWorkflow@U2@@IBE?AVQString@@ABV3@@Z$0 10000000 f   ClarkClassifyWorker.obj
 0001:fffff000       __unwindfunclet$?node_copy@?$QList@VWorkflowNotification@U2@@@@AAEXPAUNode@1@00@Z$4 10000000 f   ClarkClassifyWorker.obj
 0001:fffff000       __unwindfunclet$?node_construct@?$QList@VWorkflowNotification@U2@@@@AAEXPAUNode@1@ABVWorkflowNotification@U2@@@Z$0 10000000 f   ClarkClassifyWorker.obj
 0002:fffe0000       __catchsym$?_Copy@?$basic_string@DU?$char_traits@D@std@@V?$allocator@D@2@@std@@QAEXII@Z$5 10000000     moc_ClarkClassifyWorker.obj
 0000:fffc5000       .debug$S                   10000000     Qt5Core:Qt5Core.dll
 0000:fffc5000       .debug$S                   10000000     Qt5Core:Qt5Core.dll
 0000:fffc5000       .debug$S                   10000000     Qt5Core:Qt5Core.dll
 0000:fffc5000       .debug$S                   10000000     Qt5Core:Qt5Core.dll
 0000:fffc5000       .debug$S                   10000000     Qt5Core:Qt5Core.dll
 0000:fffc5000       .debug$S                   10000000     Qt5Core:Qt5Core.dll
 0000:fffc5000       .debug$S                   10000000     Qt5Core:Qt5Core.dll
 0000:fffc5000       .debug$S                   10000000     Qt5Core:Qt5Core.dll
 0000:fffc5000       .debug$S                   10000000     Qt5Core:Qt5Core.dll
 0000:fffc5000       .debug$S                   10000000     Qt5Core:Qt5Core.dll
 0000:fffc5000       .debug$S                   10000000     Qt5Core:Qt5Core.dll
 0000:fffc5000       .debug$S                   10000000     Qt5Core:Qt5Core.dll
 0000:fffc5000       .debug$S                   10000000     Qt5Core:Qt5Core.dll
 0000:fffc5000       .debug$S                   10000000     Qt5Core:Qt5Core.dll
 0000:fffc5000       .debug$S                   10000000     Qt5Core:Qt5Core.dll
 0000:fffc5000       .debug$S                   10000000     Qt5Core:Qt5Core.dll
 0000:fffc5000       .debug$S                   10000000     Qt5Core:Qt5Core.dll
 0000:fffc5000       .debug$S                   10000000     Qt5Core:Qt5Core.dll
 0001:fffff000       __ehhandler$?detach_helper_grow@?$QList@VWorkflowNotification@U2@@@@AAEPAUNode@1@HH@Z 10000000 f   ClarkClassifyWorker.obj
 0002:fffe0000       __unwindtable$?qt_metatype_id@?$QMetaTypeIdQObject@PAVTask@U2@@$00@@SAHXZ 10000000     moc_ClarkClassifyWorker.obj
 0000:fffc5000       .debug$S                   10000000     Qt5Core:Qt5Core.dll
 0000:fffc5000       .debug$S                   10000000     Qt5Core:Qt5Core.dll
 0000:fffc5000       .debug$S                   10000000     Qt5Core:Qt5Core.dll
 0000:fffc5000       .debug$S                   10000000     Qt5Core:Qt5Core.dll
 0000:fffc5000       .debug$S                   10000000     Qt5Core:Qt5Core.dll
 0000:fffc5000       .debug$S                   10000000     Qt5Core:Qt5Core.dll
 0000:fffc5000       .debug$S                   10000000     Qt5Core:Qt5Core.dll
 0000:fffc5000       .debug$S                   10000000     Qt5Core:Qt5Core.dll
 0000:fffc5000       .debug$S                   10000000     Qt5Core:Qt5Core.dll
 0000:fffc5000       .debug$S                   10000000     Qt5Core:Qt5Core.dll
 0000:fffc5000       .debug$S                   10000000     Qt5Core:Qt5Core.dll
 0000:fffc5000       .debug$S                   10000000     Qt5Core:Qt5Core.dll
 0000:fffc5000       .debug$S                   10000000     Qt5Core:Qt5Core.dll
 0000:fffc5000       .debug$S                   10000000     Qt5Core:Qt5Core.dll
 0000:fffc5000       .debug$S                   10000000     Qt5Core:Qt5Core.dll
 0000:fffc5000       .debug$S                   10000000     Qt5Core:Qt5Core.dll
 0000:fffc5000       .debug$S                   10000000     Qt5Core:Qt5Core.dll
 0000:fffc5000       .debug$S                   10000000     Qt5Core:Qt5Core.dll
 0000:fffc5000       .debug$S                   10000000     Qt5Core:Qt5Core.dll
 0000:fffc5000       .debug$S                   10000000     Qt5Core:Qt5Core.dll
 0000:fffc5000       .debug$S                   10000000     Qt5Core:Qt5Core.dll
 0000:fffc5000       .debug$S                   10000000     Qt5Core:Qt5Core.dll
 0000:fffc5000       .debug$S                   10000000     Qt5Core:Qt5Core.dll
 0000:fffc5000       .debug$S                   10000000     Qt5Core:Qt5Core.dll
 0000:fffc5000       .debug$S                   10000000     Qt5Core:Qt5Core.dll
 0002:fffe0000       ?_Generic_object$initializer$@?$_Error_objects@H@std@@2P6AXXZA 10000000     moc_ClarkClassifyWorker.obj
 0002:fffe0000       ?_Iostream_object$initializer$@?$_Error_objects@H@std@@2P6AXXZA 10000000     moc_ClarkClassifyWorker.obj
 0002:fffe0000       ?_System_object$initializer$@?$_Error_objects@H@std@@2P6AXXZA 10000000     moc_ClarkClassifyWorker.obj
 0000:fffc5000       .debug$S                   10000000     Qt5Core:Qt5Core.dll
 0000:fffc5000       .debug$S                   10000000     Qt5Core:Qt5Core.dll
 0000:fffc5000       .debug$S                   10000000     Qt5Core:Qt5Core.dll
 0000:fffc5000       .debug$S                   10000000     Qt5Core:Qt5Core.dll
 0000:fffc5000       .debug$S                   10000000     Qt5Core:Qt5Core.dll
 0000:fffc5000       .debug$S                   10000000     Qt5Core:Qt5Core.dll
 0001:fffff000       __unwindfunclet$?append@?$QList@VWorkflowNotification@U2@@@@QAEXABVWorkflowNotification@U2@@@Z$6 10000000 f   ClarkClassifyWorker.obj
 0000:fffc5000       .debug$S                   10000000     Qt5Core:Qt5Core.dll
 0001:fffff000       __ehhandler$?detach_helper_grow@?$QList@PAVPortDescriptor@Workflow@U2@@@@AAEPAUNode@1@HH@Z 10000000 f   ClarkClassifyWorker.obj
 0000:fffc5000       .debug$S                   10000000     Qt5Core:Qt5Core.dll
 0001:fffff000       __ehhandler$?append@?$QList@PAVPortDescriptor@Workflow@U2@@@@QAEXABQAVPortDescriptor@Workflow@U2@@@Z 10000000 f   ClarkClassifyWorker.obj
 0000:fffc5000       .debug$S                   10000000     Qt5Core:Qt5Core.dll
 0001:fffff000       __ehhandler$?detach_helper_grow@?$QList@PAVAttribute@U2@@@@AAEPAUNode@1@HH@Z 10000000 f   ClarkClassifyWorker.obj
 0000:fffc5000       .debug$S                   10000000     Qt5Core:Qt5Core.dll
 0001:fffff000       __ehhandler$?append@?$QList@PAVAttribute@U2@@@@QAEXABQAVAttribute@U2@@@Z 10000000 f   ClarkClassifyWorker.obj
 0000:fffc5000       .debug$S                   10000000     Qt5Core:Qt5Core.dll
 0001:fffff000       __unwindfunclet$??$getAttributeValue@H@Attribute@U2@@QBEHPAVWorkflowContext@Workflow@1@@Z$0 10000000 f   ClarkClassifyWorker.obj
 0000:fffc5000       .debug$S                   10000000     Qt5Core:Qt5Core.dll
 0001:fffff000       __unwindfunclet$??$getAttributeValue@VQString@@@Attribute@U2@@QBE?AVQString@@PAVWorkflowContext@Workflow@1@@Z$0 10000000 f   ClarkClassifyWorker.obj
 0000:fffc5000       .debug$S                   10000000     Qt5Core:Qt5Core.dll
 0001:fffff000       __unwindfunclet$?uniqueKeys@?$QMap@VDescriptor@U2@@VQVariant@@@@QBE?AV?$QList@VDescriptor@U2@@@@XZ$1 10000000 f   ClarkClassifyWorker.obj
 0000:fffc5000       .debug$S                   10000000     Qt5Core:Qt5Core.dll
 0001:fffff000       __unwindfunclet$??A?$QMap@VDescriptor@U2@@V?$QExplicitlySharedDataPointer@VDataType@U2@@@@@@QAEAAV?$QExplicitlySharedDataPointer@VDataType@U2@@@@ABVDescriptor@U2@@@Z$0 10000000 f   ClarkClassifyWorker.obj
 0000:fffc5000       .debug$S                   10000000     Qt5Core:Qt5Core.dll
 0001:fffff000       __unwindfunclet$?node_copy@?$QList@VDescriptor@U2@@@@AAEXPAUNode@1@00@Z$4 10000000 f   ClarkClassifyWorker.obj
 0001:fffff000       __unwindfunclet$?node_construct@?$QList@VDescriptor@U2@@@@AAEXPAUNode@1@ABVDescriptor@U2@@@Z$0 10000000 f   ClarkClassifyWorker.obj
 0001:fffff000       __ehhandler$?detach_helper@?$QList@VDescriptor@U2@@@@AAEXH@Z 10000000 f   ClarkClassifyWorker.obj
 0001:fffff000       __ehhandler$?detach_helper_grow@?$QList@VDescriptor@U2@@@@AAEPAUNode@1@HH@Z 10000000 f   ClarkClassifyWorker.obj
 0000:fffc5000       .debug$S                   10000000     Qt5Core:Qt5Core.dll
 0001:fffff000       __unwindfunclet$?append@?$QList@VDescriptor@U2@@@@QAEXABVDescriptor@U2@@@Z$6 10000000 f   ClarkClassifyWorker.obj
 0000:fffc5000       .debug$S                   10000000     Qt5Core:Qt5Core.dll
 0001:fffff000       __ehhandler$??0?$QList@VDescriptor@U2@@@@QAE@ABV0@@Z 10000000 f   ClarkClassifyWorker.obj
 0000:fffc5000       .debug$S                   10000000     Qt5Core:Qt5Core.dll
 0001:fffff000       __ehhandler$?_Copy@?$basic_string@DU?$char_traits@D@std@@V?$allocator@D@2@@std@@QAEXII@Z 10000000 f   moc_ClarkBuildWorker.obj
 0001:fffff000       __unwindfunclet$??A?$QMap@VQString@@VQScriptValue@@@@QAEAAVQScriptValue@@ABVQString@@@Z$0 10000000 f   ClarkClassifyWorker.obj
 0001:fffff000       __unwindfunclet$??A?$QMap@VQString@@VQVariant@@@@QAEAAVQVariant@@ABVQString@@@Z$0 10000000 f   ClarkClassifyWorker.obj
 0000:fffc5000       .debug$S                   10000000     Qt5Core:Qt5Core.dll
 0000:fffc5000       .debug$S                   10000000     Qt5Core:Qt5Core.dll
 0000:fffc5000       .debug$S                   10000000     Qt5Core:Qt5Core.dll
 0000:fffc5000       .debug$S                   10000000     Qt5Core:Qt5Core.dll
 0000:fffc5000       .debug$S                   10000000     Qt5Core:Qt5Core.dll
 0000:fffc5000       .debug$S                   10000000     Qt5Core:Qt5Core.dll
 0000:fffc5000       .debug$S                   10000000     Qt5Core:Qt5Core.dll
 0000:fffc5000       .debug$S                   10000000     Qt5Core:Qt5Core.dll
 0000:fffc5000       .debug$S                   10000000     Qt5Core:Qt5Core.dll
 0000:fffc5000       .debug$S                   10000000     Qt5Core:Qt5Core.dll
 0000:fffc5000       .debug$S                   10000000     Qt5Core:Qt5Core.dll
 0000:fffc5000       .debug$S                   10000000     Qt5Core:Qt5Core.dll
 0000:fffc5000       .debug$S                   10000000     Qt5Core:Qt5Core.dll
 0000:fffc5000       .debug$S                   10000000     Qt5Core:Qt5Core.dll
 0000:fffc5000       .debug$S                   10000000     Qt5Core:Qt5Core.dll
 0000:fffc5000       .debug$S                   10000000     Qt5Core:Qt5Core.dll
 0000:fffc5000       .debug$S                   10000000     Qt5Core:Qt5Core.dll
 0000:fffc5000       .debug$S                   10000000     Qt5Core:Qt5Core.dll
 0000:fffc5000       .debug$S                   10000000     Qt5Core:Qt5Core.dll
 0000:fffc5000       .debug$S                   10000000     Qt5Core:Qt5Core.dll
 0001:fffff000       __unwindfunclet$?node_copy@?$QList@VQString@@@@AAEXPAUNode@1@00@Z$5 10000000 f   ClarkClassifyWorker.obj
 0001:fffff000       __unwindfunclet$?node_construct@?$QList@VQString@@@@AAEXPAUNode@1@ABVQString@@@Z$1 10000000 f   ClarkClassifyWorker.obj
 0001:fffff000       __ehhandler$?detach_helper_grow@?$QList@VQString@@@@AAEPAUNode@1@HH@Z 10000000 f   ClarkClassifyWorker.obj
 0001:fffff000       __unwindfunclet$?append@?$QList@VQString@@@@QAEXABVQString@@@Z$7 10000000 f   ClarkClassifyWorker.obj
 0002:fffe0000       __catchsym$?_Copy@?$basic_string@DU?$char_traits@D@std@@V?$allocator@D@2@@std@@QAEXII@Z$5 10000000     moc_ClarkBuildWorker.obj
 0000:fffc5000       .debug$S                   10000000     Qt5Core:Qt5Core.dll
 0000:fffc5000       .debug$S                   10000000     Qt5Core:Qt5Core.dll
 0000:fffc5000       .debug$S                   10000000     Qt5Core:Qt5Core.dll
 0000:fffc5000       .debug$S                   10000000     Qt5Core:Qt5Core.dll
 0000:fffc5000       .debug$S                   10000000     Qt5Core:Qt5Core.dll
 0000:fffc5000       .debug$S                   10000000     Qt5Core:Qt5Core.dll
 0000:fffc5000       .debug$S                   10000000     Qt5Core:Qt5Core.dll
 0000:fffc5000       .debug$S                   10000000     Qt5Core:Qt5Core.dll
 0000:fffc5000       .debug$S                   10000000     Qt5Core:Qt5Core.dll
 0000:fffc5000       .debug$S                   10000000     Qt5Core:Qt5Core.dll
 0000:fffc5000       .debug$S                   10000000     Qt5Core:Qt5Core.dll
 0000:fffc5000       .debug$S                   10000000     Qt5Core:Qt5Core.dll
 0000:fffc5000       .debug$S                   10000000     Qt5Core:Qt5Core.dll
 0000:fffc5000       .debug$S                   10000000     Qt5Core:Qt5Core.dll
 0000:fffc5000       .debug$S                   10000000     Qt5Core:Qt5Core.dll
 0000:fffc5000       .debug$S                   10000000     Qt5Core:Qt5Core.dll
 0000:fffc5000       .debug$S                   10000000     Qt5Core:Qt5Core.dll
 0000:fffc5000       .debug$S                   10000000     Qt5Core:Qt5Core.dll
 0000:fffc5000       .debug$S                   10000000     Qt5Core:Qt5Core.dll
 0000:fffc5000       .debug$S                   10000000     Qt5Core:Qt5Core.dll
 0000:fffc5000       .debug$S                   10000000     Qt5Core:Qt5Core.dll
 0000:fffc5000       .debug$S                   10000000     Qt5Core:Qt5Core.dll
 0000:fffc5000       .debug$S                   10000000     Qt5Core:Qt5Core.dll
 0000:fffc5000       .debug$S                   10000000     Qt5Core:Qt5Core.dll
 0000:fffc5000       .debug$S                   10000000     Qt5Core:Qt5Core.dll
 0000:fffc5000       .debug$S                   10000000     Qt5Core:Qt5Core.dll
 0000:fffc5000       .debug$S                   10000000     Qt5Xml:Qt5Xml.dll
 0000:fffc5000       .debug$S                   10000000     Qt5Script:Qt5Script.dll
 0000:fffc5000       .debug$S                   10000000     Qt5Script:Qt5Script.dll
 0000:fffc5000       .debug$S                   10000000     Qt5Script:Qt5Script.dll
 0000:fffc5000       .debug$S                   10000000     Qt5Script:Qt5Script.dll
 0000:fffc5000       .debug$S                   10000000     Qt5Script:Qt5Script.dll
 0000:fffc5000       .debug$S                   10000000     Qt5Script:Qt5Script.dll
 0000:fffc5000       .debug$S                   10000000     Qt5Script:Qt5Script.dll
 0000:fffc5000       .debug$S                   10000000     Qt5Script:Qt5Script.dll
 0000:fffc5000       .debug$S                   10000000     Qt5Script:Qt5Script.dll
 0000:fffc5000       .debug$S                   10000000     Qt5Script:Qt5Script.dll
 0000:fffc5000       .debug$S                   10000000     Qt5Gui:Qt5Gui.dll
 0000:fffc5000       .debug$S                   10000000     Qt5Gui:Qt5Gui.dll
 0000:fffc5000       .debug$S                   10000000     Qt5Gui:Qt5Gui.dll
 0000:fffc5000       .debug$S                   10000000     Qt5Gui:Qt5Gui.dll
 0000:fffc5000       .debug$S                   10000000     Qt5Gui:Qt5Gui.dll
 0000:fffc5000       .debug$S                   10000000     Qt5Gui:Qt5Gui.dll
 0000:fffc5000       .debug$S                   10000000     Qt5Widgets:Qt5Widgets.dll
 0000:fffc5000       .debug$S                   10000000     Qt5Widgets:Qt5Widgets.dll
 0002:fffe0000       ?_Generic_object$initializer$@?$_Error_objects@H@std@@2P6AXXZA 10000000     moc_ClarkBuildWorker.obj
 0002:fffe0000       ?_Iostream_object$initializer$@?$_Error_objects@H@std@@2P6AXXZA 10000000     moc_ClarkBuildWorker.obj
 0002:fffe0000       ?_System_object$initializer$@?$_Error_objects@H@std@@2P6AXXZA 10000000     moc_ClarkBuildWorker.obj
 0001:fffff000       __ehhandler$??0?$QList@VQString@@@@QAE@ABV0@@Z 10000000 f   ClarkClassifyWorker.obj
 0000:fffc5000       .debug$S                   10000000     Qt5Widgets:Qt5Widgets.dll
 0001:fffff000       __unwindfunclet$??H@YA?BVQString@@ABV0@PBD@Z$0 10000000 f   ClarkClassifyWorker.obj
 0000:fffc5000       .debug$S                   10000000     Qt5Widgets:Qt5Widgets.dll
 0001:fffff000       __ehhandler$?_Copy@?$basic_string@DU?$char_traits@D@std@@V?$allocator@D@2@@std@@QAEXII@Z 10000000 f   ClarkClassifyWorker.obj
 0000:fffc5000       .debug$S                   10000000     Qt5Widgets:Qt5Widgets.dll
 0002:fffe0000       ?_System_object$initializer$@?$_Error_objects@H@std@@2P6AXXZA 10000000     ClarkSupport.obj
 0000:fffc5000       .debug$S                   10000000     Qt5Widgets:Qt5Widgets.dll
 0002:fffe0000       ?_Iostream_object$initializer$@?$_Error_objects@H@std@@2P6AXXZA 10000000     ClarkSupport.obj
 0000:fffc5000       .debug$S                   10000000     Qt5Widgets:Qt5Widgets.dll
 0002:fffe0000       ?_Generic_object$initializer$@?$_Error_objects@H@std@@2P6AXXZA 10000000     ClarkSupport.obj
 0000:fffc5000       .debug$S                   10000000     Qt5Widgets:Qt5Widgets.dll
 0002:fffe0000       __unwindtable$??H@YA?BVQString@@ABV0@PBD@Z 10000000     ClarkSupport.obj
 0000:fffc5000       .debug$S                   10000000     Qt5Widgets:Qt5Widgets.dll
 0002:fffe0000       __catchsym$?_Copy@?$basic_string@DU?$char_traits@D@std@@V?$allocator@D@2@@std@@QAEXII@Z$5 10000000     ClarkSupport.obj
 0000:fffc5000       .debug$S                   10000000     Qt5Widgets:Qt5Widgets.dll
 0000:fffc5000       .debug$S                   10000000     U2Core:U2Core.dll
 0000:fffc5000       .debug$S                   10000000     Qt5Widgets:Qt5Widgets.dll
 0000:fffc5000       .debug$S                   10000000     U2Core:U2Core.dll
 0000:fffc5000       .debug$S                   10000000     Qt5Widgets:Qt5Widgets.dll
 0000:fffc5000       .debug$S                   10000000     U2Core:U2Core.dll
 0000:fffc5000       .debug$S                   10000000     ngs_reads_classification:ngs_reads_classification.dll
 0000:fffc5000       .debug$S                   10000000     U2Core:U2Core.dll
 0000:fffc5000       .debug$S                   10000000     ngs_reads_classification:ngs_reads_classification.dll
 0000:fffc5000       .debug$S                   10000000     U2Core:U2Core.dll
 0000:fffc5000       .debug$S                   10000000     ngs_reads_classification:ngs_reads_classification.dll
 0000:fffc5000       .debug$S                   10000000     U2Core:U2Core.dll
 0000:fffc5000       .debug$S                   10000000     ngs_reads_classification:ngs_reads_classification.dll
 0000:fffc5000       .debug$S                   10000000     U2Core:U2Core.dll
 0000:fffc5000       .debug$S                   10000000     ngs_reads_classification:ngs_reads_classification.dll
 0000:fffc5000       .debug$S                   10000000     U2Core:U2Core.dll
 0000:fffc5000       .debug$S                   10000000     ngs_reads_classification:ngs_reads_classification.dll
 0000:fffc5000       .debug$S                   10000000     U2Core:U2Core.dll
 0000:fffc5000       .debug$S                   10000000     ngs_reads_classification:ngs_reads_classification.dll
 0000:fffc5000       .debug$S                   10000000     U2Core:U2Core.dll
 0000:fffc5000       .debug$S                   10000000     ngs_reads_classification:ngs_reads_classification.dll
 0000:fffc5000       .debug$S                   10000000     U2Core:U2Core.dll
 0000:fffc5000       .debug$S                   10000000     ngs_reads_classification:ngs_reads_classification.dll
 0001:fffff000       __ehhandler$?_Copy@?$basic_string@DU?$char_traits@D@std@@V?$allocator@D@2@@std@@QAEXII@Z 10000000 f   ClarkTests.obj
 0000:fffc5000       .debug$S                   10000000     U2Core:U2Core.dll
 0000:fffc5000       .debug$S                   10000000     U2Core:U2Core.dll
 0000:fffc5000       .debug$S                   10000000     U2Core:U2Core.dll
 0001:fffff000       __unwindfunclet$??H@YA?BVQString@@ABV0@0@Z$0 10000000 f   ClarkTests.obj
 0000:fffc5000       .debug$S                   10000000     U2Core:U2Core.dll
 0001:fffff000       __unwindfunclet$??H@YA?BVQString@@ABV0@PBD@Z$0 10000000 f   ClarkTests.obj
 0000:fffc5000       .debug$S                   10000000     U2Core:U2Core.dll
 0001:fffff000       __ehhandler$??0?$QList@VQString@@@@QAE@ABV0@@Z 10000000 f   ClarkTests.obj
 0000:fffc5000       .debug$S                   10000000     U2Core:U2Core.dll
 0000:fffc5000       .debug$S                   10000000     U2Core:U2Core.dll
 0000:fffc5000       .debug$S                   10000000     U2Core:U2Core.dll
 0000:fffc5000       .debug$S                   10000000     U2Core:U2Core.dll
 0001:fffff000       __unwindfunclet$?append@?$QList@VQString@@@@QAEXABVQString@@@Z$7 10000000 f   ClarkTests.obj
 0000:fffc5000       .debug$S                   10000000     U2Core:U2Core.dll
 0001:fffff000       __ehhandler$?detach_helper_grow@?$QList@VQString@@@@AAEPAUNode@1@HH@Z 10000000 f   ClarkTests.obj
 0000:fffc5000       .debug$S                   10000000     U2Core:U2Core.dll
 0000:fffc5000       .debug$S                   10000000     U2Core:U2Core.dll
 0001:fffff000       __ehhandler$?detach_helper@?$QList@VQString@@@@AAEXH@Z 10000000 f   ClarkTests.obj
 0000:fffc5000       .debug$S                   10000000     U2Core:U2Core.dll
 0000:fffc5000       .debug$S                   10000000     U2Core:U2Core.dll
 0001:fffff000       __unwindfunclet$?node_construct@?$QList@VQString@@@@AAEXPAUNode@1@ABVQString@@@Z$1 10000000 f   ClarkTests.obj
 0000:fffc5000       .debug$S                   10000000     U2Core:U2Core.dll
 0000:fffc5000       .debug$S                   10000000     U2Core:U2Core.dll
 0001:fffff000       __unwindfunclet$?node_copy@?$QList@VQString@@@@AAEXPAUNode@1@00@Z$5 10000000 f   ClarkTests.obj
 0000:fffc5000       .debug$S                   10000000     ngs_reads_classification:ngs_reads_classification.dll
 0000:fffc5000       .debug$S                   10000000     ngs_reads_classification:ngs_reads_classification.dll
 0000:fffc5000       .debug$S                   10000000     ngs_reads_classification:ngs_reads_classification.dll
 0000:fffc5000       .debug$S                   10000000     ngs_reads_classification:ngs_reads_classification.dll
 0000:fffc5000       .debug$S                   10000000     ngs_reads_classification:ngs_reads_classification.dll
 0000:fffc5000       .debug$S                   10000000     ngs_reads_classification:ngs_reads_classification.dll
 0000:fffc5000       .debug$S                   10000000     ngs_reads_classification:ngs_reads_classification.dll
 0000:fffc5000       .debug$S                   10000000     ngs_reads_classification:ngs_reads_classification.dll
 0000:fffc5000       .debug$S                   10000000     ngs_reads_classification:ngs_reads_classification.dll
 0000:fffc5000       .debug$S                   10000000     ngs_reads_classification:ngs_reads_classification.dll
 0000:fffc5000       .debug$S                   10000000     ngs_reads_classification:ngs_reads_classification.dll
 0000:fffc5000       .debug$S                   10000000     ngs_reads_classification:ngs_reads_classification.dll
 0000:fffc5000       .debug$S                   10000000     ngs_reads_classification:ngs_reads_classification.dll
 0000:fffc5000       .debug$S                   10000000     ngs_reads_classification:ngs_reads_classification.dll
 0000:fffc5000       .debug$S                   10000000     ngs_reads_classification:ngs_reads_classification.dll
 0000:fffc5000       .debug$S                   10000000     ngs_reads_classification:ngs_reads_classification.dll
 0000:fffc5000       .debug$S                   10000000     ngs_reads_classification:ngs_reads_classification.dll
 0000:fffc5000       .debug$S                   10000000     ngs_reads_classification:ngs_reads_classification.dll
 0000:fffc5000       .debug$S                   10000000     ngs_reads_classification:ngs_reads_classification.dll
 0000:fffc5000       .debug$S                   10000000     ngs_reads_classification:ngs_reads_classification.dll
 0000:fffc5000       .debug$S                   10000000     ngs_reads_classification:ngs_reads_classification.dll
 0000:fffc5000       .debug$S                   10000000     ngs_reads_classification:ngs_reads_classification.dll
 0000:fffc5000       .debug$S                   10000000     ngs_reads_classification:ngs_reads_classification.dll
 0000:fffc5000       .debug$S                   10000000     ngs_reads_classification:ngs_reads_classification.dll
 0000:fffc5000       .debug$S                   10000000     ngs_reads_classification:ngs_reads_classification.dll
 0000:fffc5000       .debug$S                   10000000     ngs_reads_classification:ngs_reads_classification.dll
 0000:fffc5000       .debug$S                   10000000     U2Designer:U2Designer.dll
 0000:fffc5000       .debug$S                   10000000     U2Designer:U2Designer.dll
 0000:fffc5000       .debug$S                   10000000     U2Designer:U2Designer.dll
 0000:fffc5000       .debug$S                   10000000     U2Designer:U2Designer.dll
 0000:fffc5000       .debug$S                   10000000     U2Designer:U2Designer.dll
 0000:fffc5000       .debug$S                   10000000     U2Designer:U2Designer.dll
 0000:fffc5000       .debug$S                   10000000     U2Designer:U2Designer.dll
 0000:fffc5000       .debug$S                   10000000     U2Designer:U2Designer.dll
 0000:fffc5000       .debug$S                   10000000     U2Designer:U2Designer.dll
 0000:fffc5000       .debug$S                   10000000     U2Designer:U2Designer.dll
 0000:fffc5000       .debug$S                   10000000     U2Designer:U2Designer.dll
 0000:fffc5000       .debug$S                   10000000     U2Designer:U2Designer.dll
 0000:fffc5000       .debug$S                   10000000     U2Designer:U2Designer.dll
 0000:fffc5000       .debug$S                   10000000     U2Designer:U2Designer.dll
 0000:fffc5000       .debug$S                   10000000     U2Designer:U2Designer.dll
 0000:fffc5000       .debug$S                   10000000     U2Designer:U2Designer.dll
 0000:fffc5000       .debug$S                   10000000     U2Designer:U2Designer.dll
 0000:fffc5000       .debug$S                   10000000     U2Designer:U2Designer.dll
 0000:fffc5000       .debug$S                   10000000     U2Designer:U2Designer.dll
 0000:fffc5000       .debug$S                   10000000     U2Designer:U2Designer.dll
 0000:fffc5000       .debug$S                   10000000     U2Designer:U2Designer.dll
 0000:fffc5000       .debug$S                   10000000     U2Designer:U2Designer.dll
 0000:fffc5000       .debug$S                   10000000     U2Designer:U2Designer.dll
 0000:fffc5000       .debug$S                   10000000     U2Designer:U2Designer.dll
 0000:fffc5000       .debug$S                   10000000     U2Designer:U2Designer.dll
 0000:fffc5000       .debug$S                   10000000     U2Designer:U2Designer.dll
 0000:fffc5000       .debug$S                   10000000     U2Designer:U2Designer.dll
 0000:fffc5000       .debug$S                   10000000     U2Designer:U2Designer.dll
 0000:fffc5000       .debug$S                   10000000     U2Designer:U2Designer.dll
 0000:fffc5000       .debug$S                   10000000     U2Designer:U2Designer.dll
 0000:fffc5000       .debug$S                   10000000     U2Designer:U2Designer.dll
 0000:fffc5000       .debug$S                   10000000     U2Designer:U2Designer.dll
 0000:fffc5000       .debug$S                   10000000     U2Designer:U2Designer.dll
 0000:fffc5000       .debug$S                   10000000     U2Designer:U2Designer.dll
 0000:fffc5000       .debug$S                   10000000     U2Designer:U2Designer.dll
 0000:fffc5000       .debug$S                   10000000     U2Designer:U2Designer.dll
 0000:fffc5000       .debug$S                   10000000     U2Designer:U2Designer.dll
 0000:fffc5000       .debug$S                   10000000     U2Designer:U2Designer.dll
 0000:fffc5000       .debug$S                   10000000     U2Designer:U2Designer.dll
 0000:fffc5000       .debug$S                   10000000     U2Designer:U2Designer.dll
 0000:fffc5000       .debug$S                   10000000     U2Designer:U2Designer.dll
 0000:fffc5000       .debug$S                   10000000     U2Designer:U2Designer.dll
 0000:fffc5000       .debug$S                   10000000     U2Designer:U2Designer.dll
 0000:fffc5000       .debug$S                   10000000     U2Designer:U2Designer.dll
 0000:fffc5000       .debug$S                   10000000     U2Designer:U2Designer.dll
 0000:fffc5000       .debug$S                   10000000     U2Designer:U2Designer.dll
 0000:fffc5000       .debug$S                   10000000     U2Designer:U2Designer.dll
 0000:fffc5000       .debug$S                   10000000     U2Designer:U2Designer.dll
 0000:fffc5000       .debug$S                   10000000     U2Designer:U2Designer.dll
 0000:fffc5000       .debug$S                   10000000     U2Lang:U2Lang.dll
 0000:fffc5000       .debug$S                   10000000     U2Lang:U2Lang.dll
 0000:fffc5000       .debug$S                   10000000     U2Lang:U2Lang.dll
 0000:fffc5000       .debug$S                   10000000     U2Lang:U2Lang.dll
 0000:fffc5000       .debug$S                   10000000     U2Lang:U2Lang.dll
 0000:fffc5000       .debug$S                   10000000     U2Lang:U2Lang.dll
 0000:fffc5000       .debug$S                   10000000     U2Lang:U2Lang.dll
 0000:fffc5000       .debug$S                   10000000     U2Lang:U2Lang.dll
 0000:fffc5000       .debug$S                   10000000     U2Lang:U2Lang.dll
 0000:fffc5000       .debug$S                   10000000     U2Lang:U2Lang.dll
 0000:fffc5000       .debug$S                   10000000     U2Lang:U2Lang.dll
 0000:fffc5000       .debug$S                   10000000     U2Lang:U2Lang.dll
 0000:fffc5000       .debug$S                   10000000     U2Lang:U2Lang.dll
 0000:fffc5000       .debug$S                   10000000     U2Lang:U2Lang.dll
 0000:fffc5000       .debug$S                   10000000     U2Lang:U2Lang.dll
 0000:fffc5000       .debug$S                   10000000     U2Lang:U2Lang.dll
 0000:fffc5000       .debug$S                   10000000     U2Lang:U2Lang.dll
 0000:fffc5000       .debug$S                   10000000     U2Lang:U2Lang.dll
 0000:fffc5000       .debug$S                   10000000     U2Lang:U2Lang.dll
 0000:fffc5000       .debug$S                   10000000     U2Lang:U2Lang.dll
 0000:fffc5000       .debug$S                   10000000     U2Lang:U2Lang.dll
 0000:fffc5000       .debug$S                   10000000     U2Lang:U2Lang.dll
 0000:fffc5000       .debug$S                   10000000     U2Lang:U2Lang.dll
 0000:fffc5000       .debug$S                   10000000     U2Lang:U2Lang.dll
 0000:fffc5000       .debug$S                   10000000     U2Lang:U2Lang.dll
 0000:fffc5000       .debug$S                   10000000     U2Lang:U2Lang.dll
 0000:fffc5000       .debug$S                   10000000     U2Lang:U2Lang.dll
 0000:fffc5000       .debug$S                   10000000     U2Lang:U2Lang.dll
 0000:fffc5000       .debug$S                   10000000     U2Lang:U2Lang.dll
 0000:fffc5000       .debug$S                   10000000     U2Lang:U2Lang.dll
 0000:fffc5000       .debug$S                   10000000     U2Lang:U2Lang.dll
 0000:fffc5000       .debug$S                   10000000     U2Lang:U2Lang.dll
 0000:fffc5000       .debug$S                   10000000     U2Core:U2Core.dll
 0000:fffc5000       .debug$S                   10000000     U2Lang:U2Lang.dll
 0000:fffc5000       .debug$S                   10000000     U2Core:U2Core.dll
 0000:fffc5000       .debug$S                   10000000     U2Core:U2Core.dll
 0000:fffc5000       .debug$S                   10000000     U2Lang:U2Lang.dll
 0001:fffff000       __unwindfunclet$??H@YA?BVQString@@ABV0@PBD@Z$0 10000000 f   ClarkSupport.obj
 0001:fffff000       __ehhandler$?_Copy@?$basic_string@DU?$char_traits@D@std@@V?$allocator@D@2@@std@@QAEXII@Z 10000000 f   ClarkSupport.obj
 0000:fffc5000       .debug$S                   10000000     U2Core:U2Core.dll
 0000:fffc5000       .debug$S                   10000000     U2Core:U2Core.dll
 0000:fffc5000       .debug$S                   10000000     U2Core:U2Core.dll
 0002:fffe0000       __catchsym$?_Copy@?$basic_string@DU?$char_traits@D@std@@V?$allocator@D@2@@std@@QAEXII@Z$5 10000000     ClarkTests.obj
 0000:fffc5000       .debug$S                   10000000     U2Core:U2Core.dll
 0002:fffe0000       __unwindtable$??H@YA?BVQString@@ABV0@0@Z 10000000     ClarkTests.obj
 0000:fffc5000       .debug$S                   10000000     U2Core:U2Core.dll
 0002:fffe0000       __unwindtable$??H@YA?BVQString@@ABV0@PBD@Z 10000000     ClarkTests.obj
 0000:fffc5000       .debug$S                   10000000     U2Core:U2Core.dll
 0000:fffc5000       .debug$S                   10000000     U2Core:U2Core.dll
 0000:fffc5000       .debug$S                   10000000     U2Core:U2Core.dll
 0002:fffe0000       __catchsym$??0?$QList@VQString@@@@QAE@ABV0@@Z$2 10000000     ClarkTests.obj
 0000:fffc5000       .debug$S                   10000000     U2Core:U2Core.dll
 0000:fffc5000       .debug$S                   10000000     U2Core:U2Core.dll
 0000:fffc5000       .debug$S                   10000000     U2Core:U2Core.dll
 0000:fffc5000       .debug$S                   10000000     U2Core:U2Core.dll
 0002:fffe0000       __catchsym$?append@?$QList@VQString@@@@QAEXABVQString@@@Z$13 10000000     ClarkTests.obj
 0000:fffc5000       .debug$S                   10000000     U2Core:U2Core.dll
 0000:fffc5000       .debug$S                   10000000     U2Core:U2Core.dll
 0000:fffc5000       .debug$S                   10000000     U2Core:U2Core.dll
 0000:fffc5000       .debug$S                   10000000     U2Core:U2Core.dll
 0002:fffe0000       __catchsym$?detach_helper_grow@?$QList@VQString@@@@AAEPAUNode@1@HH@Z$5 10000000     ClarkTests.obj
 0000:fffc5000       .debug$S                   10000000     U2Core:U2Core.dll
 0000:fffc5000       .debug$S                   10000000     U2Core:U2Core.dll
 0000:fffc5000       .debug$S                   10000000     U2Core:U2Core.dll
 0002:fffe0000       __catchsym$?detach_helper@?$QList@VQString@@@@AAEXH@Z$2 10000000     ClarkTests.obj
 0000:fffc5000       .debug$S                   10000000     U2Core:U2Core.dll
 0002:fffe0000       __unwindtable$?node_construct@?$QList@VQString@@@@AAEXPAUNode@1@ABVQString@@@Z 10000000     ClarkTests.obj
 0000:fffc5000       .debug$S                   10000000     U2Core:U2Core.dll
 0000:fffc5000       .debug$S                   10000000     U2Core:U2Core.dll
 0000:fffc5000       .debug$S                   10000000     U2Core:U2Core.dll
 0002:fffe0000       __catchsym$?node_copy@?$QList@VQString@@@@AAEXPAUNode@1@00@Z$6 10000000     ClarkTests.obj
 0000:fffc5000       .debug$S                   10000000     U2Lang:U2Lang.dll
 0000:fffc5000       .debug$S                   10000000     U2Lang:U2Lang.dll
 0000:fffc5000       .debug$S                   10000000     U2Lang:U2Lang.dll
 0000:fffc5000       .debug$S                   10000000     U2Lang:U2Lang.dll
 0000:fffc5000       .debug$S                   10000000     U2Lang:U2Lang.dll
 0000:fffc5000       .debug$S                   10000000     U2Lang:U2Lang.dll
 0000:fffc5000       .debug$S                   10000000     U2Lang:U2Lang.dll
 0000:fffc5000       .debug$S                   10000000     U2Lang:U2Lang.dll
 0000:fffc5000       .debug$S                   10000000     U2Lang:U2Lang.dll
 0000:fffc5000       .debug$S                   10000000     U2Lang:U2Lang.dll
 0000:fffc5000       .debug$S                   10000000     U2Lang:U2Lang.dll
 0000:fffc5000       .debug$S                   10000000     U2Lang:U2Lang.dll
 0000:fffc5000       .debug$S                   10000000     U2Lang:U2Lang.dll
 0000:fffc5000       .debug$S                   10000000     U2Lang:U2Lang.dll
 0000:fffc5000       .debug$S                   10000000     U2Lang:U2Lang.dll
 0000:fffc5000       .debug$S                   10000000     U2Lang:U2Lang.dll
 0000:fffc5000       .debug$S                   10000000     U2Lang:U2Lang.dll
 0000:fffc5000       .debug$S                   10000000     U2Lang:U2Lang.dll
 0000:fffc5000       .debug$S                   10000000     U2Lang:U2Lang.dll
 0000:fffc5000       .debug$S                   10000000     U2Lang:U2Lang.dll
 0000:fffc5000       .debug$S                   10000000     U2Lang:U2Lang.dll
 0000:fffc5000       .debug$S                   10000000     U2Lang:U2Lang.dll
 0000:fffc5000       .debug$S                   10000000     U2Lang:U2Lang.dll
 0000:fffc5000       .debug$S                   10000000     U2Lang:U2Lang.dll
 0000:fffc5000       .debug$S                   10000000     U2Lang:U2Lang.dll
 0000:fffc5000       .debug$S                   10000000     U2Lang:U2Lang.dll
 0000:fffc5000       .debug$S                   10000000     U2Lang:U2Lang.dll
 0000:fffc5000       .debug$S                   10000000     U2Lang:U2Lang.dll
 0000:fffc5000       .debug$S                   10000000     U2Lang:U2Lang.dll
 0000:fffc5000       .debug$S                   10000000     U2Lang:U2Lang.dll
 0000:fffc5000       .debug$S                   10000000     U2Lang:U2Lang.dll
 0000:fffc5000       .debug$S                   10000000     U2Lang:U2Lang.dll
 0000:fffc5000       .debug$S                   10000000     U2Lang:U2Lang.dll
 0000:fffc5000       .debug$S                   10000000     U2Lang:U2Lang.dll
 0000:fffc5000       .debug$S                   10000000     U2Lang:U2Lang.dll
 0000:fffc5000       .debug$S                   10000000     U2Lang:U2Lang.dll
 0000:fffc5000       .debug$S                   10000000     U2Lang:U2Lang.dll
 0000:fffc5000       .debug$S                   10000000     U2Lang:U2Lang.dll
 0000:fffc5000       .debug$S                   10000000     U2Lang:U2Lang.dll
 0000:fffc5000       .debug$S                   10000000     U2Lang:U2Lang.dll
 0000:fffc5000       .debug$S                   10000000     U2Lang:U2Lang.dll
 0000:fffc5000       .debug$S                   10000000     U2Lang:U2Lang.dll
 0000:fffc5000       .debug$S                   10000000     U2Lang:U2Lang.dll
 0000:fffc5000       .debug$S                   10000000     U2Lang:U2Lang.dll
 0000:fffc5000       .debug$S                   10000000     U2Lang:U2Lang.dll
 0000:fffc5000       .debug$S                   10000000     U2Lang:U2Lang.dll
 0000:fffc5000       .debug$S                   10000000     U2Lang:U2Lang.dll
 0000:fffc5000       .debug$S                   10000000     U2Lang:U2Lang.dll
 0000:fffc5000       .debug$S                   10000000     U2Lang:U2Lang.dll
 0000:fffc5000       .debug$S                   10000000     U2Lang:U2Lang.dll
 0000:fffc5000       .debug$S                   10000000     U2Lang:U2Lang.dll
 0000:fffc5000       .debug$S                   10000000     U2Lang:U2Lang.dll
 0000:fffc5000       .debug$S                   10000000     U2Lang:U2Lang.dll
 0000:fffc5000       .debug$S                   10000000     U2Lang:U2Lang.dll
 0000:fffc5000       .debug$S                   10000000     U2Lang:U2Lang.dll
 0000:fffc5000       .debug$S                   10000000     U2Lang:U2Lang.dll
 0000:fffc5000       .debug$S                   10000000     U2Lang:U2Lang.dll
 0000:fffc5000       .debug$S                   10000000     U2Lang:U2Lang.dll
 0000:fffc5000       .debug$S                   10000000     U2Lang:U2Lang.dll
 0000:fffc5000       .debug$S                   10000000     U2Lang:U2Lang.dll
 0000:fffc5000       .debug$S                   10000000     U2Lang:U2Lang.dll
 0000:fffc5000       .debug$S                   10000000     U2Lang:U2Lang.dll
 0000:fffc5000       .debug$S                   10000000     U2Lang:U2Lang.dll
 0000:fffc5000       .debug$S                   10000000     U2Lang:U2Lang.dll
 0000:fffc5000       .debug$S                   10000000     U2Lang:U2Lang.dll
 0000:fffc5000       .debug$S                   10000000     U2Lang:U2Lang.dll
 0000:fffc5000       .debug$S                   10000000     U2Lang:U2Lang.dll
 0000:fffc5000       .debug$S                   10000000     U2Lang:U2Lang.dll
 0000:fffc5000       .debug$S                   10000000     U2Lang:U2Lang.dll
 0000:fffc5000       .debug$S                   10000000     U2Lang:U2Lang.dll
 0000:fffc5000       .debug$S                   10000000     U2Lang:U2Lang.dll
 0000:fffc5000       .debug$S                   10000000     U2Lang:U2Lang.dll
 0000:fffc5000       .debug$S                   10000000     U2Lang:U2Lang.dll
 0000:fffc5000       .debug$S                   10000000     U2Lang:U2Lang.dll
 0000:fffc5000       .debug$S                   10000000     U2Lang:U2Lang.dll
 0000:fffc5000       .debug$S                   10000000     U2Lang:U2Lang.dll
 0000:fffc5000       .debug$S                   10000000     U2Lang:U2Lang.dll
 0000:fffc5000       .debug$S                   10000000     U2Lang:U2Lang.dll
 0002:fffe0000       ?_Generic_object$initializer$@?$_Error_objects@H@std@@2P6AXXZA 10000000     ClarkTests.obj
 0002:fffe0000       ?_Iostream_object$initializer$@?$_Error_objects@H@std@@2P6AXXZA 10000000     ClarkTests.obj
 0002:fffe0000       ?_System_object$initializer$@?$_Error_objects@H@std@@2P6AXXZA 10000000     ClarkTests.obj
 0000:fffc5000       .debug$S                   10000000     U2Core:U2Core.dll
 0000:fffc5000       .debug$S                   10000000     U2Lang:U2Lang.dll
 0000:fffc5000       .debug$S                   10000000     U2Core:U2Core.dll
 0000:fffc5000       .debug$S                   10000000     U2Lang:U2Lang.dll
 0000:fffc5000       .debug$S                   10000000     U2Core:U2Core.dll
 0000:fffc5000       .debug$S                   10000000     U2Lang:U2Lang.dll
 0000:fffc5000       .debug$S                   10000000     U2Core:U2Core.dll
 0000:fffc5000       .debug$S                   10000000     U2Lang:U2Lang.dll
 0000:fffc5000       .debug$S                   10000000     U2Core:U2Core.dll
 0000:fffc5000       .debug$S                   10000000     U2Lang:U2Lang.dll
 0000:fffc5000       .debug$S                   10000000     U2Core:U2Core.dll
 0000:fffc5000       .debug$S                   10000000     U2Lang:U2Lang.dll
 0000:fffc5000       .debug$S                   10000000     U2Core:U2Core.dll
 0000:fffc5000       .debug$S                   10000000     U2Lang:U2Lang.dll
 0000:fffc5000       .debug$S                   10000000     U2Core:U2Core.dll
 0000:fffc5000       .debug$S                   10000000     U2Lang:U2Lang.dll
 0000:fffc5000       .debug$S                   10000000     U2Core:U2Core.dll
 0000:fffc5000       .debug$S                   10000000     U2Lang:U2Lang.dll
 0000:fffc5000       .debug$S                   10000000     U2Core:U2Core.dll
 0000:fffc5000       .debug$S                   10000000     U2Lang:U2Lang.dll
 0000:fffc5000       .debug$S                   10000000     U2Core:U2Core.dll
 0000:fffc5000       .debug$S                   10000000     U2Lang:U2Lang.dll
 0000:fffc5000       .debug$S                   10000000     U2Core:U2Core.dll
 0000:fffc5000       .debug$S                   10000000     U2Lang:U2Lang.dll
 0000:fffc5000       .debug$S                   10000000     U2Core:U2Core.dll
 0000:fffc5000       .debug$S                   10000000     U2Lang:U2Lang.dll
 0000:fffc5000       .debug$S                   10000000     U2Core:U2Core.dll
 0000:fffc5000       .debug$S                   10000000     U2Lang:U2Lang.dll
 0001:fffff000       __ehhandler$?_Copy@?$basic_string@DU?$char_traits@D@std@@V?$allocator@D@2@@std@@QAEXII@Z 10000000 f   ClarkSupportPlugin.obj
 0000:fffc5000       .debug$S                   10000000     U2Core:U2Core.dll
 0002:fffe0000       ?_System_object$initializer$@?$_Error_objects@H@std@@2P6AXXZA 10000000     ClarkSupportPlugin.obj
 0000:fffc5000       .debug$S                   10000000     U2Lang:U2Lang.dll
 0000:fffc5000       .debug$S                   10000000     U2Lang:U2Lang.dll
 0000:fffc5000       .debug$S                   10000000     U2Lang:U2Lang.dll
 0000:fffc5000       .debug$S                   10000000     U2Lang:U2Lang.dll
 0000:fffc5000       .debug$S                   10000000     U2Lang:U2Lang.dll
 0000:fffc5000       .debug$S                   10000000     U2Lang:U2Lang.dll
 0000:fffc5000       .debug$S                   10000000     U2Lang:U2Lang.dll
 0000:fffc5000       .debug$S                   10000000     U2Lang:U2Lang.dll
 0000:fffc5000       .debug$S                   10000000     U2Lang:U2Lang.dll
 0000:fffc5000       .debug$S                   10000000     U2Lang:U2Lang.dll
 0000:fffc5000       .debug$S                   10000000     U2Lang:U2Lang.dll
 0000:fffc5000       .debug$S                   10000000     U2Lang:U2Lang.dll
 0000:fffc5000       .debug$S                   10000000     U2Lang:U2Lang.dll
 0000:fffc5000       .debug$S                   10000000     U2Lang:U2Lang.dll
 0000:fffc5000       .debug$S                   10000000     U2Lang:U2Lang.dll
 0000:fffc5000       .debug$S                   10000000     U2Lang:U2Lang.dll
 0000:fffc5000       .debug$S                   10000000     U2Lang:U2Lang.dll
 0000:fffc5000       .debug$S                   10000000     U2Lang:U2Lang.dll
 0000:fffc5000       .debug$S                   10000000     U2Lang:U2Lang.dll
 0000:fffc5000       .debug$S                   10000000     U2Lang:U2Lang.dll
 0000:fffc5000       .debug$S                   10000000     U2Lang:U2Lang.dll
 0000:fffc5000       .debug$S                   10000000     U2Lang:U2Lang.dll
 0000:fffc5000       .debug$S                   10000000     U2Lang:U2Lang.dll
 0000:fffc5000       .debug$S                   10000000     U2Lang:U2Lang.dll
 0000:fffc5000       .debug$S                   10000000     U2Lang:U2Lang.dll
 0000:fffc5000       .debug$S                   10000000     U2Lang:U2Lang.dll
 0000:fffc5000       .debug$S                   10000000     U2Lang:U2Lang.dll
 0000:fffc5000       .debug$S                   10000000     U2Lang:U2Lang.dll
 0000:fffc5000       .debug$S                   10000000     U2Lang:U2Lang.dll
 0000:fffc5000       .debug$S                   10000000     U2Lang:U2Lang.dll
 0000:fffc5000       .debug$S                   10000000     U2Lang:U2Lang.dll
 0000:fffc5000       .debug$S                   10000000     U2Lang:U2Lang.dll
 0000:fffc5000       .debug$S                   10000000     U2Lang:U2Lang.dll
 0000:fffc5000       .debug$S                   10000000     U2Lang:U2Lang.dll
 0000:fffc5000       .debug$S                   10000000     U2Lang:U2Lang.dll
 0000:fffc5000       .debug$S                   10000000     U2Test:U2Test.dll
 0000:fffc5000       .debug$S                   10000000     U2Test:U2Test.dll
 0000:fffc5000       .debug$S                   10000000     U2Test:U2Test.dll
 0000:fffc5000       .debug$S                   10000000     U2Test:U2Test.dll
 0000:fffc5000       .debug$S                   10000000     U2Test:U2Test.dll
 0000:fffc5000       .debug$S                   10000000     U2Test:U2Test.dll
 0000:fffc5000       .debug$S                   10000000     U2Test:U2Test.dll
 0000:fffc5000       .debug$S                   10000000     U2Test:U2Test.dll
 0002:fffe0000       ?_Iostream_object$initializer$@?$_Error_objects@H@std@@2P6AXXZA 10000000     ClarkSupportPlugin.obj
 0002:fffe0000       ?_Generic_object$initializer$@?$_Error_objects@H@std@@2P6AXXZA 10000000     ClarkSupportPlugin.obj
 0000:fffc5000       .debug$S                   10000000     U2Core:U2Core.dll
 0000:fffc5000       .debug$S                   10000000     U2Core:U2Core.dll
 0000:fffc5000       .debug$S                   10000000     U2Core:U2Core.dll
 0002:fffe0000       __catchsym$?_Copy@?$basic_string@DU?$char_traits@D@std@@V?$allocator@D@2@@std@@QAEXII@Z$5 10000000     ClarkSupportPlugin.obj
 0000:fffc5000       .debug$S                   10000000     U2Test:U2Test.dll
 0000:fffc5000       .debug$S                   10000000     U2Test:U2Test.dll
 0000:fffc5000       .debug$S                   10000000     U2Test:U2Test.dll
 0000:fffc5000       .debug$S                   10000000     U2Gui:U2Gui.dll
 0000:fffc5000       .debug$S                   10000000     U2Core:U2Core.dll
 0000:fffc5000       .debug$S                   10000000     U2Core:U2Core.dll
 0000:fffc5000       .debug$S                   10000000     U2Core:U2Core.dll
 0000:fffc5000       .debug$S                   10000000     U2Core:U2Core.dll
 0000:fffc5000       .debug$S                   10000000     U2Core:U2Core.dll
 0000:fffc5000       .debug$S                   10000000     U2Core:U2Core.dll
 0000:fffc5000       .debug$S                   10000000     U2Core:U2Core.dll
 0000:fffc5000       .debug$S                   10000000     U2Core:U2Core.dll
 0000:fffc5000       .debug$S                   10000000     U2Core:U2Core.dll
 0000:fffc5000       .debug$S                   10000000     U2Core:U2Core.dll
 0000:fffc5000       .debug$S                   10000000     U2Core:U2Core.dll
 0000:fffc5000       .debug$S                   10000000     U2Core:U2Core.dll
 0000:fffc5000       .debug$S                   10000000     U2Core:U2Core.dll
 0000:fffc5000       .debug$S                   10000000     U2Core:U2Core.dll
 0000:fffc5000       .debug$S                   10000000     U2Core:U2Core.dll
 0000:fffc5000       .debug$S                   10000000     U2Core:U2Core.dll
 0000:fffc5000       .debug$S                   10000000     U2Core:U2Core.dll
 0000:fffc5000       .debug$S                   10000000     U2Core:U2Core.dll
 0000:fffc5000       .debug$S                   10000000     U2Core:U2Core.dll
 0000:fffc5000       .debug$S                   10000000     U2Core:U2Core.dll
 0000:fffc5000       .debug$S                   10000000     U2Core:U2Core.dll
 0000:fffc5000       .debug$S                   10000000     U2Core:U2Core.dll
 0000:fffc5000       .debug$S                   10000000     U2Core:U2Core.dll
 0000:fffc5000       .debug$S                   10000000     U2Core:U2Core.dll
 0000:fffc5000       .debug$S                   10000000     U2Core:U2Core.dll
 0000:fffc5000       .debug$S                   10000000     U2Core:U2Core.dll
 0000:fffc5000       .debug$S                   10000000     U2Core:U2Core.dll
 0000:fffc5000       .debug$S                   10000000     U2Core:U2Core.dll
 0000:fffc5000       .debug$S                   10000000     U2Core:U2Core.dll
 0000:fffc5000       .debug$S                   10000000     U2Core:U2Core.dll
 0000:fffc5000       .debug$S                   10000000     U2Core:U2Core.dll
 0000:fffc5000       .debug$S                   10000000     U2Core:U2Core.dll
 0000:fffc5000       .debug$S                   10000000     U2Core:U2Core.dll
 0000:fffc5000       .debug$S                   10000000     U2Core:U2Core.dll
 0000:fffc5000       .debug$S                   10000000     U2Core:U2Core.dll
 0000:fffc5000       .debug$S                   10000000     U2Core:U2Core.dll
 0000:fffc5000       .debug$S                   10000000     U2Core:U2Core.dll
 0000:fffc5000       .debug$S                   10000000     U2Core:U2Core.dll
 0000:fffc5000       .debug$S                   10000000     U2Core:U2Core.dll
 0000:fffc5000       .debug$S                   10000000     U2Core:U2Core.dll
 0000:fffc5000       .debug$S                   10000000     U2Core:U2Core.dll
 0000:fffc5000       .debug$S                   10000000     U2Core:U2Core.dll
 0000:fffc5000       .debug$S                   10000000     U2Core:U2Core.dll
 0000:fffc5000       .debug$S                   10000000     U2Core:U2Core.dll
 0000:fffc5000       .debug$S                   10000000     U2Core:U2Core.dll
 0002:fffe0008       __ehfuncinfo$??A?$QMap@VQString@@VQScriptValue@@@@QAEAAVQScriptValue@@ABVQString@@@Z 10000008     ClarkClassifyWorker.obj
 0002:fffe0008       __ehfuncinfo$?uniqueKeys@?$QMap@VDescriptor@U2@@VQVariant@@@@QBE?AV?$QList@VDescriptor@U2@@@@XZ 10000008     ClarkClassifyWorker.obj
 0002:fffe0008       __ehfuncinfo$??A?$QMap@VDescriptor@U2@@V?$QExplicitlySharedDataPointer@VDataType@U2@@@@@@QAEAAV?$QExplicitlySharedDataPointer@VDataType@U2@@@@ABVDescriptor@U2@@@Z 10000008     ClarkClassifyWorker.obj
 0002:fffe0008       __ehfuncinfo$??H@YA?BVQString@@ABV0@0@Z 10000008     ClarkTests.obj
 0002:fffe0008       __ehfuncinfo$??A?$QMap@VQString@@VQVariant@@@@QAEAAVQVariant@@ABVQString@@@Z 10000008     ClarkClassifyWorker.obj
 0001:fffff008       __ehhandler$??A?$QMap@VDescriptor@U2@@V?$QExplicitlySharedDataPointer@VDataType@U2@@@@@@QAEAAV?$QExplicitlySharedDataPointer@VDataType@U2@@@@ABVDescriptor@U2@@@Z 10000008 f   ClarkClassifyWorker.obj
 0002:fffe0008       __ehfuncinfo$?qt_metatype_id@?$QMetaTypeIdQObject@PAVTask@U2@@$00@@SAHXZ 10000008     moc_ClarkClassifyWorker.obj
 0001:fffff009       __ehhandler$??A?$QMap@VQString@@VQVariant@@@@QAEAAVQVariant@@ABVQString@@@Z 10000009 f   ClarkClassifyWorker.obj
 0001:fffff009       __unwindfunclet$??$getAttributeValue@H@Attribute@U2@@QBEHPAVWorkflowContext@Workflow@1@@Z$1 10000009 f   ClarkClassifyWorker.obj
 0001:fffff009       __ehhandler$??A?$QMap@VQString@@VQScriptValue@@@@QAEAAVQScriptValue@@ABVQString@@@Z 10000009 f   ClarkClassifyWorker.obj
 0001:fffff009       __ehhandler$?qt_metatype_id@?$QMetaTypeIdQObject@PAVTask@U2@@$00@@SAHXZ 10000009 f   moc_ClarkClassifyWorker.obj
 0001:fffff00b       __ehhandler$?node_copy@?$QList@VWorkflowNotification@U2@@@@AAEXPAUNode@1@00@Z 1000000b f   ClarkClassifyWorker.obj
 0001:fffff00b       __ehhandler$?node_copy@?$QList@VDescriptor@U2@@@@AAEXPAUNode@1@00@Z 1000000b f   ClarkClassifyWorker.obj
 0001:fffff00b       __ehhandler$?append@?$QList@VDescriptor@U2@@@@QAEXABVDescriptor@U2@@@Z 1000000b f   ClarkClassifyWorker.obj
 0001:fffff00b       __ehhandler$?node_construct@?$QList@VDescriptor@U2@@@@AAEXPAUNode@1@ABVDescriptor@U2@@@Z 1000000b f   ClarkClassifyWorker.obj
 0001:fffff00b       __ehhandler$?node_construct@?$QList@VWorkflowNotification@U2@@@@AAEXPAUNode@1@ABVWorkflowNotification@U2@@@Z 1000000b f   ClarkClassifyWorker.obj
 0001:fffff00b       __ehhandler$?append@?$QList@VWorkflowNotification@U2@@@@QAEXABVWorkflowNotification@U2@@@Z 1000000b f   ClarkClassifyWorker.obj
 0002:fffe0010       __catchsym$?detach_helper_grow@?$QList@VQString@@@@AAEPAUNode@1@HH@Z$4 10000010     ClarkClassifyWorker.obj
 0002:fffe0010       __ehfuncinfo$?node_construct@?$QList@VQString@@@@AAEXPAUNode@1@ABVQString@@@Z 10000010     ClarkClassifyWorker.obj
 0002:fffe0010       __tryblocktable$?node_copy@?$QList@VQString@@@@AAEXPAUNode@1@00@Z 10000010     ClarkClassifyWorker.obj
 0002:fffe0010       __catchsym$?_Copy@?$basic_string@DU?$char_traits@D@std@@V?$allocator@D@2@@std@@QAEXII@Z$4 10000010     moc_ClarkSupportPlugin.obj
 0002:fffe0010       __catchsym$?append@?$QList@VQString@@@@QAEXABVQString@@@Z$12 10000010     ClarkClassifyWorker.obj
 0002:fffe0010       __unwindtable$??0?$QList@VDescriptor@U2@@@@QAE@ABV0@@Z 10000010     ClarkClassifyWorker.obj
 0002:fffe0010       __catchsym$?_Copy@?$basic_string@DU?$char_traits@D@std@@V?$allocator@D@2@@std@@QAEXII@Z$4 10000010     ClarkTests.obj
 0002:fffe0010       __ehfuncinfo$??H@YA?BVQString@@ABV0@PBD@Z 10000010     ClarkClassifyWorker.obj
 0002:fffe0010       __catchsym$?append@?$QList@VDescriptor@U2@@@@QAEXABVDescriptor@U2@@@Z$8 10000010     ClarkClassifyWorker.obj
 0002:fffe0010       __catchsym$?_Copy@?$basic_string@DU?$char_traits@D@std@@V?$allocator@D@2@@std@@QAEXII@Z$4 10000010     moc_ClarkBuildWorker.obj
 0002:fffe0010       __catchsym$?detach_helper_grow@?$QList@VDescriptor@U2@@@@AAEPAUNode@1@HH@Z$4 10000010     ClarkClassifyWorker.obj
 0002:fffe0010       __catchsym$?_Copy@?$basic_string@DU?$char_traits@D@std@@V?$allocator@D@2@@std@@QAEXII@Z$4 10000010     ClarkClassifyWorker.obj
 0002:fffe0010       __unwindtable$?detach_helper@?$QList@VDescriptor@U2@@@@AAEXH@Z 10000010     ClarkClassifyWorker.obj
 0002:fffe0010       __ehfuncinfo$??H@YA?BVQString@@ABV0@PBD@Z 10000010     ClarkTests.obj
 0002:fffe0010       __ehfuncinfo$?node_construct@?$QList@VDescriptor@U2@@@@AAEXPAUNode@1@ABVDescriptor@U2@@@Z 10000010     ClarkClassifyWorker.obj
 0002:fffe0010       __catchsym$?_Copy@?$basic_string@DU?$char_traits@D@std@@V?$allocator@D@2@@std@@QAEXII@Z$4 10000010     moc_ClarkSupport.obj
 0002:fffe0010       __tryblocktable$?node_copy@?$QList@VDescriptor@U2@@@@AAEXPAUNode@1@00@Z 10000010     ClarkClassifyWorker.obj
 0002:fffe0010       __ehfuncinfo$??H@YA?BVQString@@ABV0@PBD@Z 10000010     ClarkSupport.obj
 0002:fffe0010       __catchsym$?_Copy@?$basic_string@DU?$char_traits@D@std@@V?$allocator@D@2@@std@@QAEXII@Z$4 10000010     ClarkSupport.obj
 0002:fffe0010       __tryblocktable$?append@?$QList@PAVAttribute@U2@@@@QAEXABQAVAttribute@U2@@@Z 10000010     ClarkClassifyWorker.obj
 0002:fffe0010       __tryblocktable$?node_copy@?$QList@VQString@@@@AAEXPAUNode@1@00@Z 10000010     ClarkTests.obj
 0002:fffe0010       __catchsym$?_Copy@?$basic_string@DU?$char_traits@D@std@@V?$allocator@D@2@@std@@QAEXII@Z$4 10000010     moc_ClarkClassifyWorker.obj
 0002:fffe0010       __catchsym$?detach_helper_grow@?$QList@PAVAttribute@U2@@@@AAEPAUNode@1@HH@Z$4 10000010     ClarkClassifyWorker.obj
 0002:fffe0010       __tryblocktable$?append@?$QList@PAVPortDescriptor@Workflow@U2@@@@QAEXABQAVPortDescriptor@Workflow@U2@@@Z 10000010     ClarkClassifyWorker.obj
 0002:fffe0010       __unwindtable$??0?$QList@VQString@@@@QAE@ABV0@@Z 10000010     ClarkClassifyWorker.obj
 0002:fffe0010       __catchsym$?detach_helper_grow@?$QList@PAVPortDescriptor@Workflow@U2@@@@AAEPAUNode@1@HH@Z$4 10000010     ClarkClassifyWorker.obj
 0002:fffe0010       __ehfuncinfo$?node_construct@?$QList@VQString@@@@AAEXPAUNode@1@ABVQString@@@Z 10000010     ClarkTests.obj
 0002:fffe0010       __unwindtable$??0?$QList@VQString@@@@QAE@ABV0@@Z 10000010     ClarkTests.obj
 0002:fffe0010       __catchsym$?_Copy@?$basic_string@DU?$char_traits@D@std@@V?$allocator@D@2@@std@@QAEXII@Z$4 10000010     ClarkSupportPlugin.obj
 0002:fffe0010       __catchsym$?append@?$QList@VWorkflowNotification@U2@@@@QAEXABVWorkflowNotification@U2@@@Z$10 10000010     ClarkClassifyWorker.obj
 0002:fffe0010       __unwindtable$?detach_helper@?$QList@VQString@@@@AAEXH@Z 10000010     ClarkTests.obj
 0002:fffe0010       __ehfuncinfo$?metaType@?$QVariantValueHelper@VQString@@@QtPrivate@@SA?AVQString@@ABVQVariant@@@Z 10000010     ClarkClassifyWorker.obj
 0002:fffe0010       __catchsym$?detach_helper_grow@?$QList@VWorkflowNotification@U2@@@@AAEPAUNode@1@HH@Z$4 10000010     ClarkClassifyWorker.obj
 0002:fffe0010       __ehfuncinfo$?node_construct@?$QList@VWorkflowNotification@U2@@@@AAEXPAUNode@1@ABVWorkflowNotification@U2@@@Z 10000010     ClarkClassifyWorker.obj
 0002:fffe0010       __catchsym$?detach_helper_grow@?$QList@VQString@@@@AAEPAUNode@1@HH@Z$4 10000010     ClarkTests.obj
 0002:fffe0010       __tryblocktable$?node_copy@?$QList@VWorkflowNotification@U2@@@@AAEXPAUNode@1@00@Z 10000010     ClarkClassifyWorker.obj
 0002:fffe0010       __ehfuncinfo$??$getValue@VQString@@@BaseWorker@LocalWorkflow@U2@@IBE?AVQString@@ABV3@@Z 10000010     ClarkClassifyWorker.obj
 0002:fffe0010       __unwindtable$??0?$QList@PAVPort@Workflow@U2@@@@QAE@ABV0@@Z 10000010     ClarkClassifyWorker.obj
 0002:fffe0010       __tryblocktable$?createNode@?$QMapData@VQString@@PAVPropertyDelegate@U2@@@@QAEPAU?$QMapNode@VQString@@PAVPropertyDelegate@U2@@@@ABVQString@@ABQAVPropertyDelegate@U2@@PAU2@_N@Z 10000010     ClarkClassifyWorker.obj
 0002:fffe0010       __catchsym$?createNode@?$QMapData@VQString@@VQVariant@@@@QAEPAU?$QMapNode@VQString@@VQVariant@@@@ABVQString@@ABVQVariant@@PAU2@_N@Z$6 10000010     ClarkClassifyWorker.obj
 0002:fffe0010       __tryblocktable$?createNode@?$QMapData@VDescriptor@U2@@V?$QExplicitlySharedDataPointer@VDataType@U2@@@@@@QAEPAU?$QMapNode@VDescriptor@U2@@V?$QExplicitlySharedDataPointer@VDataType@U2@@@@@@ABVDescriptor@U2@@ABV?$QExplicitlySharedDataPointer@VDataType@U2@@@@PAU2@_N@Z 10000010     ClarkClassifyWorker.obj
 0002:fffe0010       __catchsym$?createNode@?$QMapData@VQString@@VQScriptValue@@@@QAEPAU?$QMapNode@VQString@@VQScriptValue@@@@ABVQString@@ABVQScriptValue@@PAU2@_N@Z$6 10000010     ClarkClassifyWorker.obj
 0002:fffe0010       __catchsym$?append@?$QList@VQString@@@@QAEXABVQString@@@Z$12 10000010     ClarkTests.obj
 0001:fffff011       __ehhandler$?node_copy@?$QList@VQString@@@@AAEXPAUNode@1@00@Z 10000011 f   ClarkTests.obj
 0001:fffff011       __unwindfunclet$??$getAttributeValue@H@Attribute@U2@@QBEHPAVWorkflowContext@Workflow@1@@Z$2 10000011 f   ClarkClassifyWorker.obj
 0001:fffff011       __ehhandler$?node_copy@?$QList@VQString@@@@AAEXPAUNode@1@00@Z 10000011 f   ClarkClassifyWorker.obj
 0001:fffff011       __ehhandler$?node_construct@?$QList@VQString@@@@AAEXPAUNode@1@ABVQString@@@Z 10000011 f   ClarkClassifyWorker.obj
 0001:fffff011       __unwindfunclet$?append@?$QList@VQString@@@@QAEXABVQString@@@Z$11 10000011 f   ClarkClassifyWorker.obj
 0001:fffff011       __unwindfunclet$?append@?$QList@VQString@@@@QAEXABVQString@@@Z$11 10000011 f   ClarkTests.obj
 0001:fffff011       __ehhandler$?node_construct@?$QList@VQString@@@@AAEXPAUNode@1@ABVQString@@@Z 10000011 f   ClarkTests.obj
 0001:fffff014       __ehhandler$?createNode@?$QMapData@VDescriptor@U2@@V?$QExplicitlySharedDataPointer@VDataType@U2@@@@@@QAEPAU?$QMapNode@VDescriptor@U2@@V?$QExplicitlySharedDataPointer@VDataType@U2@@@@@@ABVDescriptor@U2@@ABV?$QExplicitlySharedDataPointer@VDataType@U2@@@@PAU2@_N@Z 10000014 f   ClarkClassifyWorker.obj
 0001:fffff014       __ehhandler$?createNode@?$QMapData@VQString@@PAVPropertyDelegate@U2@@@@QAEPAU?$QMapNode@VQString@@PAVPropertyDelegate@U2@@@@ABVQString@@ABQAVPropertyDelegate@U2@@PAU2@_N@Z 10000014 f   ClarkClassifyWorker.obj
 0001:fffff014       __unwindfunclet$?createNode@?$QMapData@VQString@@VQScriptValue@@@@QAEPAU?$QMapNode@VQString@@VQScriptValue@@@@ABVQString@@ABVQScriptValue@@PAU2@_N@Z$5 10000014 f   ClarkClassifyWorker.obj
 0001:fffff014       __unwindfunclet$?createNode@?$QMapData@VQString@@VQVariant@@@@QAEPAU?$QMapNode@VQString@@VQVariant@@@@ABVQString@@ABVQVariant@@PAU2@_N@Z$5 10000014 f   ClarkClassifyWorker.obj
 0001:fffff019       __ehhandler$?uniqueKeys@?$QMap@VDescriptor@U2@@VQVariant@@@@QBE?AV?$QList@VDescriptor@U2@@@@XZ 10000019 f   ClarkClassifyWorker.obj
 0001:fffff019       __unwindfunclet$??$getAttributeValue@H@Attribute@U2@@QBEHPAVWorkflowContext@Workflow@1@@Z$3 10000019 f   ClarkClassifyWorker.obj
 0001:fffff01a       __unwindfunclet$??H@YA?BVQString@@ABV0@PBD@Z$1 1000001a f   ClarkSupport.obj
 0001:fffff01a       __unwindfunclet$??H@YA?BVQString@@ABV0@PBD@Z$1 1000001a f   ClarkClassifyWorker.obj
 0001:fffff01a       __unwindfunclet$??$getAttributeValue@VQString@@@Attribute@U2@@QBE?AVQString@@PAVWorkflowContext@Workflow@1@@Z$1 1000001a f   ClarkClassifyWorker.obj
 0001:fffff01a       __ehhandler$??H@YA?BVQString@@ABV0@0@Z 1000001a f   ClarkTests.obj
 0001:fffff01a       __unwindfunclet$??H@YA?BVQString@@ABV0@PBD@Z$1 1000001a f   ClarkTests.obj
 0001:fffff01a       __unwindfunclet$??$getValue@VQString@@@BaseWorker@LocalWorkflow@U2@@IBE?AVQString@@ABV3@@Z$1 1000001a f   ClarkClassifyWorker.obj
 0001:fffff01a       __unwindfunclet$?metaType@?$QVariantValueHelper@VQString@@@QtPrivate@@SA?AVQString@@ABVQVariant@@@Z$1 1000001a f   ClarkClassifyWorker.obj
 0002:fffe0020       __unwindtable$?detach_helper_grow@?$QList@VQString@@@@AAEPAUNode@1@HH@Z 10000020     ClarkClassifyWorker.obj
 0002:fffe0020       __unwindtable$?_Copy@?$basic_string@DU?$char_traits@D@std@@V?$allocator@D@2@@std@@QAEXII@Z 10000020     ClarkTests.obj
 0002:fffe0020       __tryblocktable$??0?$QList@VDescriptor@U2@@@@QAE@ABV0@@Z 10000020     ClarkClassifyWorker.obj
 0002:fffe0020       __ehfuncinfo$?append@?$QList@VDescriptor@U2@@@@QAEXABVDescriptor@U2@@@Z 10000020     ClarkClassifyWorker.obj
 0002:fffe0020       __unwindtable$?detach_helper_grow@?$QList@VDescriptor@U2@@@@AAEPAUNode@1@HH@Z 10000020     ClarkClassifyWorker.obj
 0002:fffe0020       __tryblocktable$??0?$QList@VQString@@@@QAE@ABV0@@Z 10000020     ClarkClassifyWorker.obj
 0002:fffe0020       __unwindtable$?_Copy@?$basic_string@DU?$char_traits@D@std@@V?$allocator@D@2@@std@@QAEXII@Z 10000020     moc_ClarkSupportPlugin.obj
 0002:fffe0020       __unwindtable$?_Copy@?$basic_string@DU?$char_traits@D@std@@V?$allocator@D@2@@std@@QAEXII@Z 10000020     moc_ClarkSupport.obj
 0002:fffe0020       __unwindtable$?_Copy@?$basic_string@DU?$char_traits@D@std@@V?$allocator@D@2@@std@@QAEXII@Z 10000020     ClarkClassifyWorker.obj
 0002:fffe0020       __tryblocktable$?detach_helper@?$QList@VDescriptor@U2@@@@AAEXH@Z 10000020     ClarkClassifyWorker.obj
 0002:fffe0020       __unwindtable$?detach_helper_grow@?$QList@PAVAttribute@U2@@@@AAEPAUNode@1@HH@Z 10000020     ClarkClassifyWorker.obj
 0002:fffe0020       __unwindtable$?detach_helper_grow@?$QList@PAVPortDescriptor@Workflow@U2@@@@AAEPAUNode@1@HH@Z 10000020     ClarkClassifyWorker.obj
 0002:fffe0020       __unwindtable$?_Copy@?$basic_string@DU?$char_traits@D@std@@V?$allocator@D@2@@std@@QAEXII@Z 10000020     moc_ClarkClassifyWorker.obj
 0002:fffe0020       __ehfuncinfo$?append@?$QList@VWorkflowNotification@U2@@@@QAEXABVWorkflowNotification@U2@@@Z 10000020     ClarkClassifyWorker.obj
 0002:fffe0020       __tryblocktable$??0?$QList@VQString@@@@QAE@ABV0@@Z 10000020     ClarkTests.obj
 0002:fffe0020       __unwindtable$?_Copy@?$basic_string@DU?$char_traits@D@std@@V?$allocator@D@2@@std@@QAEXII@Z 10000020     moc_ClarkBuildWorker.obj
 0002:fffe0020       __tryblocktable$?detach_helper@?$QList@VQString@@@@AAEXH@Z 10000020     ClarkTests.obj
 0002:fffe0020       __ehfuncinfo$?append@?$QList@VQString@@@@QAEXABVQString@@@Z 10000020     ClarkTests.obj
 0002:fffe0020       __unwindtable$?detach_helper_grow@?$QList@VWorkflowNotification@U2@@@@AAEPAUNode@1@HH@Z 10000020     ClarkClassifyWorker.obj
 0002:fffe0020       __tryblocktable$??0?$QList@PAVPort@Workflow@U2@@@@QAE@ABV0@@Z 10000020     ClarkClassifyWorker.obj
 0002:fffe0020       __ehfuncinfo$?createNode@?$QMapData@VQString@@VQVariant@@@@QAEPAU?$QMapNode@VQString@@VQVariant@@@@ABVQString@@ABVQVariant@@PAU2@_N@Z 10000020     ClarkClassifyWorker.obj
 0002:fffe0020       __unwindtable$?_Copy@?$basic_string@DU?$char_traits@D@std@@V?$allocator@D@2@@std@@QAEXII@Z 10000020     ClarkSupportPlugin.obj
 0002:fffe0020       __unwindtable$?detach_helper_grow@?$QList@VQString@@@@AAEPAUNode@1@HH@Z 10000020     ClarkTests.obj
 0002:fffe0020       __ehfuncinfo$?append@?$QList@VQString@@@@QAEXABVQString@@@Z 10000020     ClarkClassifyWorker.obj
 0002:fffe0020       __ehfuncinfo$?createNode@?$QMapData@VQString@@VQScriptValue@@@@QAEPAU?$QMapNode@VQString@@VQScriptValue@@@@ABVQString@@ABVQScriptValue@@PAU2@_N@Z 10000020     ClarkClassifyWorker.obj
 0002:fffe0020       __unwindtable$?_Copy@?$basic_string@DU?$char_traits@D@std@@V?$allocator@D@2@@std@@QAEXII@Z 10000020     ClarkSupport.obj
 0001:fffff021       __unwindfunclet$??$getAttributeValue@H@Attribute@U2@@QBEHPAVWorkflowContext@Workflow@1@@Z$4 10000021 f   ClarkClassifyWorker.obj
 0001:fffff022       __ehhandler$?append@?$QList@VQString@@@@QAEXABVQString@@@Z 10000022 f   ClarkTests.obj
 0001:fffff022       __ehhandler$?append@?$QList@VQString@@@@QAEXABVQString@@@Z 10000022 f   ClarkClassifyWorker.obj
 0001:fffff023       __ehhandler$??H@YA?BVQString@@ABV0@PBD@Z 10000023 f   ClarkSupport.obj
 0001:fffff023       __ehhandler$??$getValue@VQString@@@BaseWorker@LocalWorkflow@U2@@IBE?AVQString@@ABV3@@Z 10000023 f   ClarkClassifyWorker.obj
 0001:fffff023       __ehhandler$??H@YA?BVQString@@ABV0@PBD@Z 10000023 f   ClarkClassifyWorker.obj
 0001:fffff023       __ehhandler$?metaType@?$QVariantValueHelper@VQString@@@QtPrivate@@SA?AVQString@@ABVQVariant@@@Z 10000023 f   ClarkClassifyWorker.obj
 0001:fffff023       __unwindfunclet$??$getAttributeValue@VQString@@@Attribute@U2@@QBE?AVQString@@PAVWorkflowContext@Workflow@1@@Z$2 10000023 f   ClarkClassifyWorker.obj
 0001:fffff023       __ehhandler$??H@YA?BVQString@@ABV0@PBD@Z 10000023 f   ClarkTests.obj
 0002:fffe0024       __ehfuncinfo$?node_copy@?$QList@VQString@@@@AAEXPAUNode@1@00@Z 10000024     ClarkTests.obj
 0002:fffe0024       __ehfuncinfo$?append@?$QList@PAVAttribute@U2@@@@QAEXABQAVAttribute@U2@@@Z 10000024     ClarkClassifyWorker.obj
 0002:fffe0024       __unwindtable$??$getAttributeValue@H@Attribute@U2@@QBEHPAVWorkflowContext@Workflow@1@@Z 10000024     ClarkClassifyWorker.obj
 0002:fffe0024       __unwindtable$??$getAttributeValue@VQString@@@Attribute@U2@@QBE?AVQString@@PAVWorkflowContext@Workflow@1@@Z 10000024     ClarkClassifyWorker.obj
 0002:fffe0024       __ehfuncinfo$?append@?$QList@PAVPortDescriptor@Workflow@U2@@@@QAEXABQAVPortDescriptor@Workflow@U2@@@Z 10000024     ClarkClassifyWorker.obj
 0002:fffe0024       __ehfuncinfo$?node_copy@?$QList@VWorkflowNotification@U2@@@@AAEXPAUNode@1@00@Z 10000024     ClarkClassifyWorker.obj
 0002:fffe0024       __ehfuncinfo$?createNode@?$QMapData@VQString@@PAVPropertyDelegate@U2@@@@QAEPAU?$QMapNode@VQString@@PAVPropertyDelegate@U2@@@@ABVQString@@ABQAVPropertyDelegate@U2@@PAU2@_N@Z 10000024     ClarkClassifyWorker.obj
 0002:fffe0024       __ehfuncinfo$?node_copy@?$QList@VQString@@@@AAEXPAUNode@1@00@Z 10000024     ClarkClassifyWorker.obj
 0002:fffe0024       __ehfuncinfo$?createNode@?$QMapData@VDescriptor@U2@@V?$QExplicitlySharedDataPointer@VDataType@U2@@@@@@QAEPAU?$QMapNode@VDescriptor@U2@@V?$QExplicitlySharedDataPointer@VDataType@U2@@@@@@ABVDescriptor@U2@@ABV?$QExplicitlySharedDataPointer@VDataType@U2@@@@PAU2@_N@Z 10000024     ClarkClassifyWorker.obj
 0002:fffe0024       __ehfuncinfo$?node_copy@?$QList@VDescriptor@U2@@@@AAEXPAUNode@1@00@Z 10000024     ClarkClassifyWorker.obj
 0001:fffff028       __ehhandler$?createNode@?$QMapData@VQString@@VQVariant@@@@QAEPAU?$QMapNode@VQString@@VQVariant@@@@ABVQString@@ABVQVariant@@PAU2@_N@Z 10000028 f   ClarkClassifyWorker.obj
 0001:fffff028       __ehhandler$?createNode@?$QMapData@VQString@@VQScriptValue@@@@QAEPAU?$QMapNode@VQString@@VQScriptValue@@@@ABVQString@@ABVQScriptValue@@PAU2@_N@Z 10000028 f   ClarkClassifyWorker.obj
 0001:fffff02a       __unwindfunclet$??$getAttributeValue@H@Attribute@U2@@QBEHPAVWorkflowContext@Workflow@1@@Z$5 1000002a f   ClarkClassifyWorker.obj
 0001:fffff02b       __unwindfunclet$??$getAttributeValue@VQString@@@Attribute@U2@@QBE?AVQString@@PAVWorkflowContext@Workflow@1@@Z$3 1000002b f   ClarkClassifyWorker.obj
 0001:fffff033       __unwindfunclet$??$getAttributeValue@VQString@@@Attribute@U2@@QBE?AVQString@@PAVWorkflowContext@Workflow@1@@Z$4 10000033 f   ClarkClassifyWorker.obj
 0001:fffff033       __unwindfunclet$??$getAttributeValue@H@Attribute@U2@@QBEHPAVWorkflowContext@Workflow@1@@Z$6 10000033 f   ClarkClassifyWorker.obj
 0002:fffe0034       __ehfuncinfo$??0?$QList@VQString@@@@QAE@ABV0@@Z 10000034     ClarkClassifyWorker.obj
 0002:fffe0034       __ehfuncinfo$??0?$QList@VQString@@@@QAE@ABV0@@Z 10000034     ClarkTests.obj
 0002:fffe0034       __ehfuncinfo$??0?$QList@PAVPort@Workflow@U2@@@@QAE@ABV0@@Z 10000034     ClarkClassifyWorker.obj
 0002:fffe0034       __ehfuncinfo$?detach_helper@?$QList@VQString@@@@AAEXH@Z 10000034     ClarkTests.obj
 0002:fffe0034       __ehfuncinfo$??0?$QList@VDescriptor@U2@@@@QAE@ABV0@@Z 10000034     ClarkClassifyWorker.obj
 0002:fffe0034       __ehfuncinfo$?detach_helper@?$QList@VDescriptor@U2@@@@AAEXH@Z 10000034     ClarkClassifyWorker.obj
 0001:fffff03b       __unwindfunclet$??$getAttributeValue@VQString@@@Attribute@U2@@QBE?AVQString@@PAVWorkflowContext@Workflow@1@@Z$5 1000003b f   ClarkClassifyWorker.obj
 0001:fffff03c       __unwindfunclet$??$getAttributeValue@H@Attribute@U2@@QBEHPAVWorkflowContext@Workflow@1@@Z$7 1000003c f   ClarkClassifyWorker.obj
 0002:fffe0040       __ehfuncinfo$?detach_helper_grow@?$QList@VQString@@@@AAEPAUNode@1@HH@Z 10000040     ClarkClassifyWorker.obj
 0002:fffe0040       __ehfuncinfo$?_Copy@?$basic_string@DU?$char_traits@D@std@@V?$allocator@D@2@@std@@QAEXII@Z 10000040     ClarkSupport.obj
 0002:fffe0040       __ehfuncinfo$?detach_helper_grow@?$QList@VDescriptor@U2@@@@AAEPAUNode@1@HH@Z 10000040     ClarkClassifyWorker.obj
 0002:fffe0040       __ehfuncinfo$?detach_helper_grow@?$QList@VWorkflowNotification@U2@@@@AAEPAUNode@1@HH@Z 10000040     ClarkClassifyWorker.obj
 0002:fffe0040       __ehfuncinfo$?_Copy@?$basic_string@DU?$char_traits@D@std@@V?$allocator@D@2@@std@@QAEXII@Z 10000040     ClarkTests.obj
 0002:fffe0040       __ehfuncinfo$?_Copy@?$basic_string@DU?$char_traits@D@std@@V?$allocator@D@2@@std@@QAEXII@Z 10000040     moc_ClarkSupport.obj
 0002:fffe0040       __ehfuncinfo$?_Copy@?$basic_string@DU?$char_traits@D@std@@V?$allocator@D@2@@std@@QAEXII@Z 10000040     moc_ClarkClassifyWorker.obj
 0002:fffe0040       __ehfuncinfo$?detach_helper_grow@?$QList@VQString@@@@AAEPAUNode@1@HH@Z 10000040     ClarkTests.obj
 0002:fffe0040       __ehfuncinfo$?detach_helper_grow@?$QList@PAVPortDescriptor@Workflow@U2@@@@AAEPAUNode@1@HH@Z 10000040     ClarkClassifyWorker.obj
 0002:fffe0040       __ehfuncinfo$?_Copy@?$basic_string@DU?$char_traits@D@std@@V?$allocator@D@2@@std@@QAEXII@Z 10000040     moc_ClarkSupportPlugin.obj
 0002:fffe0040       __ehfuncinfo$?_Copy@?$basic_string@DU?$char_traits@D@std@@V?$allocator@D@2@@std@@QAEXII@Z 10000040     ClarkClassifyWorker.obj
 0002:fffe0040       __ehfuncinfo$?_Copy@?$basic_string@DU?$char_traits@D@std@@V?$allocator@D@2@@std@@QAEXII@Z 10000040     ClarkSupportPlugin.obj
 0002:fffe0040       __ehfuncinfo$?_Copy@?$basic_string@DU?$char_traits@D@std@@V?$allocator@D@2@@std@@QAEXII@Z 10000040     moc_ClarkBuildWorker.obj
 0002:fffe0040       __ehfuncinfo$?detach_helper_grow@?$QList@PAVAttribute@U2@@@@AAEPAUNode@1@HH@Z 10000040     ClarkClassifyWorker.obj
 0002:fffe0044       __tryblocktable$?append@?$QList@VQString@@@@QAEXABVQString@@@Z 10000044     ClarkTests.obj
 0001:fffff044       __unwindfunclet$??$getAttributeValue@VQString@@@Attribute@U2@@QBE?AVQString@@PAVWorkflowContext@Workflow@1@@Z$6 10000044 f   ClarkClassifyWorker.obj
 0002:fffe0044       __tryblocktable$?createNode@?$QMapData@VQString@@VQScriptValue@@@@QAEPAU?$QMapNode@VQString@@VQScriptValue@@@@ABVQString@@ABVQScriptValue@@PAU2@_N@Z 10000044     ClarkClassifyWorker.obj
 0002:fffe0044       __tryblocktable$?createNode@?$QMapData@VQString@@VQVariant@@@@QAEPAU?$QMapNode@VQString@@VQVariant@@@@ABVQString@@ABVQVariant@@PAU2@_N@Z 10000044     ClarkClassifyWorker.obj
 0002:fffe0044       __tryblocktable$?append@?$QList@VWorkflowNotification@U2@@@@QAEXABVWorkflowNotification@U2@@@Z 10000044     ClarkClassifyWorker.obj
 0002:fffe0044       __tryblocktable$?append@?$QList@VDescriptor@U2@@@@QAEXABVDescriptor@U2@@@Z 10000044     ClarkClassifyWorker.obj
 0002:fffe0044       __tryblocktable$?append@?$QList@VQString@@@@QAEXABVQString@@@Z 10000044     ClarkClassifyWorker.obj
 0001:fffff045       __unwindfunclet$??$getAttributeValue@H@Attribute@U2@@QBEHPAVWorkflowContext@Workflow@1@@Z$8 10000045 f   ClarkClassifyWorker.obj
 0002:fffe0048       __unwindtable$?append@?$QList@PAVAttribute@U2@@@@QAEXABQAVAttribute@U2@@@Z 10000048     ClarkClassifyWorker.obj
 0002:fffe0048       __unwindtable$?node_copy@?$QList@VDescriptor@U2@@@@AAEXPAUNode@1@00@Z 10000048     ClarkClassifyWorker.obj
 0002:fffe0048       __unwindtable$?node_copy@?$QList@VQString@@@@AAEXPAUNode@1@00@Z 10000048     ClarkClassifyWorker.obj
 0002:fffe0048       __unwindtable$?createNode@?$QMapData@VDescriptor@U2@@V?$QExplicitlySharedDataPointer@VDataType@U2@@@@@@QAEPAU?$QMapNode@VDescriptor@U2@@V?$QExplicitlySharedDataPointer@VDataType@U2@@@@@@ABVDescriptor@U2@@ABV?$QExplicitlySharedDataPointer@VDataType@U2@@@@PAU2@_N@Z 10000048     ClarkClassifyWorker.obj
 0002:fffe0048       __unwindtable$?createNode@?$QMapData@VQString@@PAVPropertyDelegate@U2@@@@QAEPAU?$QMapNode@VQString@@PAVPropertyDelegate@U2@@@@ABVQString@@ABQAVPropertyDelegate@U2@@PAU2@_N@Z 10000048     ClarkClassifyWorker.obj
 0002:fffe0048       __unwindtable$?append@?$QList@PAVPortDescriptor@Workflow@U2@@@@QAEXABQAVPortDescriptor@Workflow@U2@@@Z 10000048     ClarkClassifyWorker.obj
 0002:fffe0048       __unwindtable$?node_copy@?$QList@VQString@@@@AAEXPAUNode@1@00@Z 10000048     ClarkTests.obj
 0002:fffe0048       __unwindtable$?node_copy@?$QList@VWorkflowNotification@U2@@@@AAEXPAUNode@1@00@Z 10000048     ClarkClassifyWorker.obj
 0001:fffff04d       __unwindfunclet$??$getAttributeValue@VQString@@@Attribute@U2@@QBE?AVQString@@PAVWorkflowContext@Workflow@1@@Z$7 1000004d f   ClarkClassifyWorker.obj
 0001:fffff04e       __unwindfunclet$??$getAttributeValue@H@Attribute@U2@@QBEHPAVWorkflowContext@Workflow@1@@Z$9 1000004e f   ClarkClassifyWorker.obj
 0001:fffff056       __unwindfunclet$??$getAttributeValue@VQString@@@Attribute@U2@@QBE?AVQString@@PAVWorkflowContext@Workflow@1@@Z$8 10000056 f   ClarkClassifyWorker.obj
 0001:fffff057       __unwindfunclet$??$getAttributeValue@H@Attribute@U2@@QBEHPAVWorkflowContext@Workflow@1@@Z$10 10000057 f   ClarkClassifyWorker.obj
 0001:fffff05f       __unwindfunclet$??$getAttributeValue@VQString@@@Attribute@U2@@QBE?AVQString@@PAVWorkflowContext@Workflow@1@@Z$9 1000005f f   ClarkClassifyWorker.obj
 0001:fffff060       __unwindfunclet$??$getAttributeValue@H@Attribute@U2@@QBEHPAVWorkflowContext@Workflow@1@@Z$11 10000060 f   ClarkClassifyWorker.obj
 0001:fffff062       __catch$?node_copy@?$QList@VQString@@@@AAEXPAUNode@1@00@Z$2 10000062 f   ClarkClassifyWorker.obj
 0001:fffff062       __catch$?node_copy@?$QList@VQString@@@@AAEXPAUNode@1@00@Z$2 10000062 f   ClarkTests.obj
 0002:fffe0064       __tryblocktable$?detach_helper_grow@?$QList@PAVAttribute@U2@@@@AAEPAUNode@1@HH@Z 10000064     ClarkClassifyWorker.obj
 0002:fffe0064       __tryblocktable$?_Copy@?$basic_string@DU?$char_traits@D@std@@V?$allocator@D@2@@std@@QAEXII@Z 10000064     ClarkSupport.obj
 0002:fffe0064       __tryblocktable$?detach_helper_grow@?$QList@VDescriptor@U2@@@@AAEPAUNode@1@HH@Z 10000064     ClarkClassifyWorker.obj
 0002:fffe0064       __tryblocktable$?_Copy@?$basic_string@DU?$char_traits@D@std@@V?$allocator@D@2@@std@@QAEXII@Z 10000064     moc_ClarkSupportPlugin.obj
 0002:fffe0064       __tryblocktable$?detach_helper_grow@?$QList@VQString@@@@AAEPAUNode@1@HH@Z 10000064     ClarkClassifyWorker.obj
 0002:fffe0064       __tryblocktable$?_Copy@?$basic_string@DU?$char_traits@D@std@@V?$allocator@D@2@@std@@QAEXII@Z 10000064     moc_ClarkBuildWorker.obj
 0002:fffe0064       __tryblocktable$?detach_helper_grow@?$QList@VWorkflowNotification@U2@@@@AAEPAUNode@1@HH@Z 10000064     ClarkClassifyWorker.obj
 0002:fffe0064       __tryblocktable$?_Copy@?$basic_string@DU?$char_traits@D@std@@V?$allocator@D@2@@std@@QAEXII@Z 10000064     ClarkClassifyWorker.obj
 0002:fffe0064       __tryblocktable$?_Copy@?$basic_string@DU?$char_traits@D@std@@V?$allocator@D@2@@std@@QAEXII@Z 10000064     moc_ClarkClassifyWorker.obj
 0002:fffe0064       __tryblocktable$?_Copy@?$basic_string@DU?$char_traits@D@std@@V?$allocator@D@2@@std@@QAEXII@Z 10000064     ClarkSupportPlugin.obj
 0002:fffe0064       __tryblocktable$?_Copy@?$basic_string@DU?$char_traits@D@std@@V?$allocator@D@2@@std@@QAEXII@Z 10000064     moc_ClarkSupport.obj
 0002:fffe0064       __tryblocktable$?detach_helper_grow@?$QList@PAVPortDescriptor@Workflow@U2@@@@AAEPAUNode@1@HH@Z 10000064     ClarkClassifyWorker.obj
 0002:fffe0064       __tryblocktable$?detach_helper_grow@?$QList@VQString@@@@AAEPAUNode@1@HH@Z 10000064     ClarkTests.obj
 0002:fffe0064       __tryblocktable$?_Copy@?$basic_string@DU?$char_traits@D@std@@V?$allocator@D@2@@std@@QAEXII@Z 10000064     ClarkTests.obj
 0001:fffff068       __unwindfunclet$??$getAttributeValue@VQString@@@Attribute@U2@@QBE?AVQString@@PAVWorkflowContext@Workflow@1@@Z$10 10000068 f   ClarkClassifyWorker.obj
 0001:fffff069       __ehhandler$??$getAttributeValue@H@Attribute@U2@@QBEHPAVWorkflowContext@Workflow@1@@Z 10000069 f   ClarkClassifyWorker.obj
 0002:fffe006c       __unwindtable$?append@?$QList@VDescriptor@U2@@@@QAEXABVDescriptor@U2@@@Z 1000006c     ClarkClassifyWorker.obj
 0002:fffe006c       __unwindtable$?append@?$QList@VWorkflowNotification@U2@@@@QAEXABVWorkflowNotification@U2@@@Z 1000006c     ClarkClassifyWorker.obj
 0002:fffe006c       __unwindtable$?append@?$QList@VQString@@@@QAEXABVQString@@@Z 1000006c     ClarkTests.obj
 0002:fffe006c       __unwindtable$?createNode@?$QMapData@VQString@@VQScriptValue@@@@QAEPAU?$QMapNode@VQString@@VQScriptValue@@@@ABVQString@@ABVQScriptValue@@PAU2@_N@Z 1000006c     ClarkClassifyWorker.obj
 0002:fffe006c       __unwindtable$?createNode@?$QMapData@VQString@@VQVariant@@@@QAEPAU?$QMapNode@VQString@@VQVariant@@@@ABVQString@@ABVQVariant@@PAU2@_N@Z 1000006c     ClarkClassifyWorker.obj
 0002:fffe006c       __unwindtable$?append@?$QList@VQString@@@@QAEXABVQString@@@Z 1000006c     ClarkClassifyWorker.obj
 0001:fffff071       __unwindfunclet$??$getAttributeValue@VQString@@@Attribute@U2@@QBE?AVQString@@PAVWorkflowContext@Workflow@1@@Z$11 10000071 f   ClarkClassifyWorker.obj
 0001:fffff07a       __unwindfunclet$??$getAttributeValue@VQString@@@Attribute@U2@@QBE?AVQString@@PAVWorkflowContext@Workflow@1@@Z$12 1000007a f   ClarkClassifyWorker.obj
 0001:fffff07d       __catch$?append@?$QList@VQString@@@@QAEXABVQString@@@Z$0 1000007d f   ClarkTests.obj
 0001:fffff07d       __catch$?append@?$QList@VQString@@@@QAEXABVQString@@@Z$0 1000007d f   ClarkClassifyWorker.obj
 0001:fffff07e       __catch$?node_copy@?$QList@VWorkflowNotification@U2@@@@AAEXPAUNode@1@00@Z$0 1000007e f   ClarkClassifyWorker.obj
 0001:fffff083       __ehhandler$??$getAttributeValue@VQString@@@Attribute@U2@@QBE?AVQString@@PAVWorkflowContext@Workflow@1@@Z 10000083 f   ClarkClassifyWorker.obj
 0001:fffff085       __catch$?node_copy@?$QList@VDescriptor@U2@@@@AAEXPAUNode@1@00@Z$0 10000085 f   ClarkClassifyWorker.obj
 0001:fffff085       __catch$?createNode@?$QMapData@VQString@@PAVPropertyDelegate@U2@@@@QAEPAU?$QMapNode@VQString@@PAVPropertyDelegate@U2@@@@ABVQString@@ABQAVPropertyDelegate@U2@@PAU2@_N@Z$2 10000085 f   ClarkClassifyWorker.obj
 0001:fffff085       __catch$?append@?$QList@PAVAttribute@U2@@@@QAEXABQAVAttribute@U2@@@Z$4 10000085 f   ClarkClassifyWorker.obj
 0001:fffff085       __catch$?append@?$QList@PAVPortDescriptor@Workflow@U2@@@@QAEXABQAVPortDescriptor@Workflow@U2@@@Z$4 10000085 f   ClarkClassifyWorker.obj
 0001:fffff08e       __catch$?createNode@?$QMapData@VQString@@VQScriptValue@@@@QAEPAU?$QMapNode@VQString@@VQScriptValue@@@@ABVQString@@ABVQScriptValue@@PAU2@_N@Z$0 1000008e f   ClarkClassifyWorker.obj
 0001:fffff08e       __catch$?createNode@?$QMapData@VQString@@VQVariant@@@@QAEPAU?$QMapNode@VQString@@VQVariant@@@@ABVQString@@ABVQVariant@@PAU2@_N@Z$0 1000008e f   ClarkClassifyWorker.obj
 0001:fffff096       __catch$?_Copy@?$basic_string@DU?$char_traits@D@std@@V?$allocator@D@2@@std@@QAEXII@Z$0 10000096 f   moc_ClarkBuildWorker.obj
 0001:fffff096       __catch$?_Copy@?$basic_string@DU?$char_traits@D@std@@V?$allocator@D@2@@std@@QAEXII@Z$0 10000096 f   ClarkSupport.obj
 0001:fffff096       __catch$?_Copy@?$basic_string@DU?$char_traits@D@std@@V?$allocator@D@2@@std@@QAEXII@Z$0 10000096 f   ClarkSupportPlugin.obj
 0001:fffff096       __catch$?_Copy@?$basic_string@DU?$char_traits@D@std@@V?$allocator@D@2@@std@@QAEXII@Z$0 10000096 f   ClarkClassifyWorker.obj
 0001:fffff096       __catch$?_Copy@?$basic_string@DU?$char_traits@D@std@@V?$allocator@D@2@@std@@QAEXII@Z$0 10000096 f   moc_ClarkSupport.obj
 0001:fffff096       __catch$?_Copy@?$basic_string@DU?$char_traits@D@std@@V?$allocator@D@2@@std@@QAEXII@Z$0 10000096 f   moc_ClarkClassifyWorker.obj
 0001:fffff096       __catch$?_Copy@?$basic_string@DU?$char_traits@D@std@@V?$allocator@D@2@@std@@QAEXII@Z$0 10000096 f   ClarkTests.obj
 0001:fffff096       __catch$?_Copy@?$basic_string@DU?$char_traits@D@std@@V?$allocator@D@2@@std@@QAEXII@Z$0 10000096 f   moc_ClarkSupportPlugin.obj
 0001:fffff09d       __catch$?createNode@?$QMapData@VDescriptor@U2@@V?$QExplicitlySharedDataPointer@VDataType@U2@@@@@@QAEPAU?$QMapNode@VDescriptor@U2@@V?$QExplicitlySharedDataPointer@VDataType@U2@@@@@@ABVDescriptor@U2@@ABV?$QExplicitlySharedDataPointer@VDataType@U2@@@@PAU2@_N@Z$2 1000009d f   ClarkClassifyWorker.obj
 0001:fffff09e       __catch$??0?$QList@PAVPort@Workflow@U2@@@@QAE@ABV0@@Z$0 1000009e f   ClarkClassifyWorker.obj
 0001:fffff09e       __catch$??0?$QList@VQString@@@@QAE@ABV0@@Z$0 1000009e f   ClarkTests.obj
 0001:fffff09e       __catch$??0?$QList@VQString@@@@QAE@ABV0@@Z$0 1000009e f   ClarkClassifyWorker.obj
 0001:fffff09e       __catch$??0?$QList@VDescriptor@U2@@@@QAE@ABV0@@Z$0 1000009e f   ClarkClassifyWorker.obj
 0001:fffff0a0       __catch$?append@?$QList@VWorkflowNotification@U2@@@@QAEXABVWorkflowNotification@U2@@@Z$2 100000a0 f   ClarkClassifyWorker.obj
 0001:fffff0a0       __catch$?append@?$QList@VWorkflowNotification@U2@@@@QAEXABVWorkflowNotification@U2@@@Z$0 100000a0 f   ClarkClassifyWorker.obj
 0001:fffff0a3       __catch$?createNode@?$QMapData@VQString@@VQScriptValue@@@@QAEPAU?$QMapNode@VQString@@VQScriptValue@@@@ABVQString@@ABVQScriptValue@@PAU2@_N@Z$2 100000a3 f   ClarkClassifyWorker.obj
 0001:fffff0a3       __catch$?createNode@?$QMapData@VQString@@VQVariant@@@@QAEPAU?$QMapNode@VQString@@VQVariant@@@@ABVQString@@ABVQVariant@@PAU2@_N@Z$2 100000a3 f   ClarkClassifyWorker.obj
 0001:fffff0aa       __catch$?detach_helper@?$QList@VDescriptor@U2@@@@AAEXH@Z$0 100000aa f   ClarkClassifyWorker.obj
 0001:fffff0ac       __catch$?append@?$QList@VDescriptor@U2@@@@QAEXABVDescriptor@U2@@@Z$0 100000ac f   ClarkClassifyWorker.obj
 0001:fffff0ac       __catch$?append@?$QList@VDescriptor@U2@@@@QAEXABVDescriptor@U2@@@Z$2 100000ac f   ClarkClassifyWorker.obj
 0001:fffff0ce       __catch$?append@?$QList@VQString@@@@QAEXABVQString@@@Z$4 100000ce f   ClarkClassifyWorker.obj
 0001:fffff0ce       __catch$?append@?$QList@VQString@@@@QAEXABVQString@@@Z$4 100000ce f   ClarkTests.obj
 0001:fffff0d1       __catch$?detach_helper@?$QList@VQString@@@@AAEXH@Z$0 100000d1 f   ClarkTests.obj
 0001:fffff0d3       __catch$?_Copy@?$basic_string@DU?$char_traits@D@std@@V?$allocator@D@2@@std@@QAEXII@Z$1 100000d3 f   moc_ClarkSupport.obj
 0001:fffff0d3       __catch$?_Copy@?$basic_string@DU?$char_traits@D@std@@V?$allocator@D@2@@std@@QAEXII@Z$1 100000d3 f   moc_ClarkClassifyWorker.obj
 0001:fffff0d3       __catch$?_Copy@?$basic_string@DU?$char_traits@D@std@@V?$allocator@D@2@@std@@QAEXII@Z$1 100000d3 f   ClarkSupport.obj
 0001:fffff0d3       __catch$?_Copy@?$basic_string@DU?$char_traits@D@std@@V?$allocator@D@2@@std@@QAEXII@Z$1 100000d3 f   ClarkClassifyWorker.obj
 0001:fffff0d3       __catch$?_Copy@?$basic_string@DU?$char_traits@D@std@@V?$allocator@D@2@@std@@QAEXII@Z$1 100000d3 f   moc_ClarkSupportPlugin.obj
 0001:fffff0d3       __catch$?_Copy@?$basic_string@DU?$char_traits@D@std@@V?$allocator@D@2@@std@@QAEXII@Z$1 100000d3 f   ClarkTests.obj
 0001:fffff0d3       __catch$?_Copy@?$basic_string@DU?$char_traits@D@std@@V?$allocator@D@2@@std@@QAEXII@Z$1 100000d3 f   ClarkSupportPlugin.obj
 0001:fffff0d3       __catch$?_Copy@?$basic_string@DU?$char_traits@D@std@@V?$allocator@D@2@@std@@QAEXII@Z$1 100000d3 f   moc_ClarkBuildWorker.obj
 0001:fffff0ef       __catch$?detach_helper_grow@?$QList@VDescriptor@U2@@@@AAEPAUNode@1@HH@Z$2 100000ef f   ClarkClassifyWorker.obj
 0001:fffff0ef       __catch$?detach_helper_grow@?$QList@VWorkflowNotification@U2@@@@AAEPAUNode@1@HH@Z$2 100000ef f   ClarkClassifyWorker.obj
 0001:fffff0f1       __catch$?detach_helper_grow@?$QList@PAVPortDescriptor@Workflow@U2@@@@AAEPAUNode@1@HH@Z$2 100000f1 f   ClarkClassifyWorker.obj
 0001:fffff0f1       __catch$?detach_helper_grow@?$QList@PAVPortDescriptor@Workflow@U2@@@@AAEPAUNode@1@HH@Z$0 100000f1 f   ClarkClassifyWorker.obj
 0001:fffff0f1       __catch$?detach_helper_grow@?$QList@PAVAttribute@U2@@@@AAEPAUNode@1@HH@Z$2 100000f1 f   ClarkClassifyWorker.obj
 0001:fffff0f1       __catch$?detach_helper_grow@?$QList@PAVAttribute@U2@@@@AAEPAUNode@1@HH@Z$0 100000f1 f   ClarkClassifyWorker.obj
 0001:fffff11e       __catch$?detach_helper_grow@?$QList@VQString@@@@AAEPAUNode@1@HH@Z$2 1000011e f   ClarkTests.obj
 0001:fffff11e       __catch$?detach_helper_grow@?$QList@VQString@@@@AAEPAUNode@1@HH@Z$2 1000011e f   ClarkClassifyWorker.obj
 0001:fffff12a       __catch$?detach_helper_grow@?$QList@VDescriptor@U2@@@@AAEPAUNode@1@HH@Z$0 1000012a f   ClarkClassifyWorker.obj
 0001:fffff12a       __catch$?detach_helper_grow@?$QList@VWorkflowNotification@U2@@@@AAEPAUNode@1@HH@Z$0 1000012a f   ClarkClassifyWorker.obj
 0001:fffff159       __catch$?detach_helper_grow@?$QList@VQString@@@@AAEPAUNode@1@HH@Z$0 10000159 f   ClarkClassifyWorker.obj
 0001:fffff159       __catch$?detach_helper_grow@?$QList@VQString@@@@AAEPAUNode@1@HH@Z$0 10000159 f   ClarkTests.obj
 0001:00000000       ??__E?ACTOR_ID@ClarkBuildWorkerFactory@LocalWorkflow@U2@@0VQString@@B@@YAXXZ 10001000 f   ClarkBuildWorker.obj
 0001:00000020       ??__E?_Generic_object@?$_Error_objects@H@std@@2V_Generic_error_category@2@A@@YAXXZ 10001020 f   ClarkBuildWorker.obj
 0001:00000030       ??__E?_Iostream_object@?$_Error_objects@H@std@@2V_Iostream_error_category@2@A@@YAXXZ 10001030 f   ClarkBuildWorker.obj
 0001:00000040       ??__E?_System_object@?$_Error_objects@H@std@@2V_System_error_category@2@A@@YAXXZ 10001040 f   ClarkBuildWorker.obj
 0001:00000050       ??__E?wellKnownErrors@ClarkBuildLogParser@LocalWorkflow@U2@@0VQStringList@@B@@YAXXZ 10001050 f   ClarkBuildWorker.obj
 0001:00000120       ??__EDB_URL@LocalWorkflow@U2@@YAXXZ 10001120 f   ClarkBuildWorker.obj
 0001:00000140       ??__EGENOMIC_LIBRARY@LocalWorkflow@U2@@YAXXZ 10001140 f   ClarkBuildWorker.obj
 0001:00000160       ??__EOUTPUT_PORT@LocalWorkflow@U2@@YAXXZ 10001160 f   ClarkBuildWorker.obj
 0001:00000180       ??__ETAXONOMY_RANK@LocalWorkflow@U2@@YAXXZ 10001180 f   ClarkBuildWorker.obj
 0001:000001a0       ??__EalgoLog@U2@@YAXXZ     100011a0 f   ClarkBuildWorker.obj
 0001:00000220       ??__EcmdLog@U2@@YAXXZ      10001220 f   ClarkBuildWorker.obj
 0001:000002a0       ??__EcoreLog@U2@@YAXXZ     100012a0 f   ClarkBuildWorker.obj
 0001:00000320       ??__EioLog@U2@@YAXXZ       10001320 f   ClarkBuildWorker.obj
 0001:000003a0       ??__EperfLog@U2@@YAXXZ     100013a0 f   ClarkBuildWorker.obj
 0001:00000420       ??__EscriptLog@U2@@YAXXZ   10001420 f   ClarkBuildWorker.obj
 0001:000004a0       ??__EtaskLog@U2@@YAXXZ     100014a0 f   ClarkBuildWorker.obj
 0001:00000520       ??__EuiLog@U2@@YAXXZ       10001520 f   ClarkBuildWorker.obj
 0001:000005a0       ??__EuserActLog@U2@@YAXXZ  100015a0 f   ClarkBuildWorker.obj
 0001:00000620       ??__E?ACTOR_ID@ClarkClassifyWorkerFactory@LocalWorkflow@U2@@2VQString@@B@@YAXXZ 10001620 f   ClarkClassifyWorker.obj
 0001:00000640       ??__E?DB_TO_RAM@ClarkClassifyWorkerFactory@LocalWorkflow@U2@@2VQString@@B@@YAXXZ 10001640 f   ClarkClassifyWorker.obj
 0001:00000660       ??__E?DB_URL@ClarkClassifyWorkerFactory@LocalWorkflow@U2@@2VQString@@B@@YAXXZ 10001660 f   ClarkClassifyWorker.obj
 0001:00000680       ??__E?EXTEND_OUT@ClarkClassifyWorkerFactory@LocalWorkflow@U2@@2VQString@@B@@YAXXZ 10001680 f   ClarkClassifyWorker.obj
 0001:000006a0       ??__E?FACTOR@ClarkClassifyWorkerFactory@LocalWorkflow@U2@@2VQString@@B@@YAXXZ 100016a0 f   ClarkClassifyWorker.obj
 0001:000006c0       ??__E?GAP@ClarkClassifyWorkerFactory@LocalWorkflow@U2@@2VQString@@B@@YAXXZ 100016c0 f   ClarkClassifyWorker.obj
 0001:000006e0       ??__E?INPUT_PORT@ClarkClassifyWorkerFactory@LocalWorkflow@U2@@2VQString@@B@@YAXXZ 100016e0 f   ClarkClassifyWorker.obj
 0001:00000700       ??__E?INPUT_SLOT@ClarkClassifyWorkerFactory@LocalWorkflow@U2@@2VQString@@B@@YAXXZ 10001700 f   ClarkClassifyWorker.obj
 0001:00000720       ??__E?K_LENGTH@ClarkClassifyWorkerFactory@LocalWorkflow@U2@@2VQString@@B@@YAXXZ 10001720 f   ClarkClassifyWorker.obj
 0001:00000740       ??__E?K_MIN_FREQ@ClarkClassifyWorkerFactory@LocalWorkflow@U2@@2VQString@@B@@YAXXZ 10001740 f   ClarkClassifyWorker.obj
 0001:00000760       ??__E?MODE@ClarkClassifyWorkerFactory@LocalWorkflow@U2@@2VQString@@B@@YAXXZ 10001760 f   ClarkClassifyWorker.obj
 0001:00000780       ??__E?NUM_THREADS@ClarkClassifyWorkerFactory@LocalWorkflow@U2@@2VQString@@B@@YAXXZ 10001780 f   ClarkClassifyWorker.obj
 0001:000007a0       ??__E?OUTPUT_PORT@ClarkClassifyWorkerFactory@LocalWorkflow@U2@@2VQString@@B@@YAXXZ 100017a0 f   ClarkClassifyWorker.obj
 0001:000007c0       ??__E?OUTPUT_URL@ClarkClassifyWorkerFactory@LocalWorkflow@U2@@2VQString@@B@@YAXXZ 100017c0 f   ClarkClassifyWorker.obj
 0001:000007e0       ??__E?PAIRED_END@ClarkClassifyWorkerFactory@LocalWorkflow@U2@@2VQString@@B@@YAXXZ 100017e0 f   ClarkClassifyWorker.obj
 0001:00000800       ??__E?PAIRED_INPUT_PORT@ClarkClassifyWorkerFactory@LocalWorkflow@U2@@2VQString@@B@@YAXXZ 10001800 f   ClarkClassifyWorker.obj
 0001:00000820       ??__E?PAIRED_INPUT_SLOT@ClarkClassifyWorkerFactory@LocalWorkflow@U2@@2VQString@@B@@YAXXZ 10001820 f   ClarkClassifyWorker.obj
 0001:00000840       ??__E?SEQUENCING_READS@ClarkClassifyWorkerFactory@LocalWorkflow@U2@@2VQString@@B@@YAXXZ 10001840 f   ClarkClassifyWorker.obj
 0001:00000860       ??__E?SINGLE_END@ClarkClassifyWorkerFactory@LocalWorkflow@U2@@2VQString@@B@@YAXXZ 10001860 f   ClarkClassifyWorker.obj
 0001:00000880       ??__E?TAXONOMY@ClarkClassifyWorkerFactory@LocalWorkflow@U2@@2VQString@@B@@YAXXZ 10001880 f   ClarkClassifyWorker.obj
 0001:000008a0       ??__E?TAXONOMY_RANK@ClarkClassifyWorkerFactory@LocalWorkflow@U2@@2VQString@@B@@YAXXZ 100018a0 f   ClarkClassifyWorker.obj
 0001:000008c0       ??__E?TOOL_DEFAULT@ClarkClassifySettings@LocalWorkflow@U2@@2VQString@@B@@YAXXZ 100018c0 f   ClarkClassifyWorker.obj
 0001:000008e0       ??__E?TOOL_LIGHT@ClarkClassifySettings@LocalWorkflow@U2@@2VQString@@B@@YAXXZ 100018e0 f   ClarkClassifyWorker.obj
 0001:00000900       ??__E?TOOL_VARIANT@ClarkClassifyWorkerFactory@LocalWorkflow@U2@@2VQString@@B@@YAXXZ 10001900 f   ClarkClassifyWorker.obj
 0001:00000920       ??__E?WORKFLOW_CLASSIFY_TOOL_CLARK@ClarkClassifyWorkerFactory@LocalWorkflow@U2@@2VQString@@B@@YAXXZ 10001920 f   ClarkClassifyWorker.obj
 0001:00000940       ??__E?_Generic_object@?$_Error_objects@H@std@@2V_Generic_error_category@2@A@@YAXXZ 10001940 f   ClarkClassifyWorker.obj
 0001:00000950       ??__E?_Iostream_object@?$_Error_objects@H@std@@2V_Iostream_error_category@2@A@@YAXXZ 10001950 f   ClarkClassifyWorker.obj
 0001:00000960       ??__E?_System_object@?$_Error_objects@H@std@@2V_System_error_category@2@A@@YAXXZ 10001960 f   ClarkClassifyWorker.obj
 0001:00000970       ??__E?wellKnownErrors@ClarkLogParser@LocalWorkflow@U2@@0V?$QMap@VQString@@V1@@@B@@YAXXZ 10001970 f   ClarkClassifyWorker.obj
 0001:00000990       ??__EEXTENDED_REPORT_SUFFIX@LocalWorkflow@U2@@YAXXZ 10001990 f   ClarkClassifyWorker.obj
 0001:000009b0       ??__EREPORT_PREFIX@LocalWorkflow@U2@@YAXXZ 100019b0 f   ClarkClassifyWorker.obj
 0001:000009d0       ??__EalgoLog@U2@@YAXXZ     100019d0 f   ClarkClassifyWorker.obj
 0001:00000a50       ??__EcmdLog@U2@@YAXXZ      10001a50 f   ClarkClassifyWorker.obj
 0001:00000ad0       ??__EcoreLog@U2@@YAXXZ     10001ad0 f   ClarkClassifyWorker.obj
 0001:00000b50       ??__EioLog@U2@@YAXXZ       10001b50 f   ClarkClassifyWorker.obj
 0001:00000bd0       ??__EperfLog@U2@@YAXXZ     10001bd0 f   ClarkClassifyWorker.obj
 0001:00000c50       ??__EscriptLog@U2@@YAXXZ   10001c50 f   ClarkClassifyWorker.obj
 0001:00000cd0       ??__EtaskLog@U2@@YAXXZ     10001cd0 f   ClarkClassifyWorker.obj
 0001:00000d50       ??__EuiLog@U2@@YAXXZ       10001d50 f   ClarkClassifyWorker.obj
 0001:00000dd0       ??__EuserActLog@U2@@YAXXZ  10001dd0 f   ClarkClassifyWorker.obj
 0001:00000e50       ??__E?CLARK_GROUP@ClarkSupport@U2@@2VQString@@B@@YAXXZ 10001e50 f   ClarkSupport.obj
 0001:00000e70       ??__E?ET_CLARK@ClarkSupport@U2@@2VQString@@B@@YAXXZ 10001e70 f   ClarkSupport.obj
 0001:00000e90       ??__E?ET_CLARK_BUILD_SCRIPT@ClarkSupport@U2@@2VQString@@B@@YAXXZ 10001e90 f   ClarkSupport.obj
 0001:00000eb0       ??__E?ET_CLARK_BUILD_SCRIPT_ID@ClarkSupport@U2@@2VQString@@B@@YAXXZ 10001eb0 f   ClarkSupport.obj
 0001:00000ed0       ??__E?ET_CLARK_GET_ACCSSN_TAX_ID@ClarkSupport@U2@@2VQString@@B@@YAXXZ 10001ed0 f   ClarkSupport.obj
 0001:00000ef0       ??__E?ET_CLARK_GET_ACCSSN_TAX_ID_ID@ClarkSupport@U2@@2VQString@@B@@YAXXZ 10001ef0 f   ClarkSupport.obj
 0001:00000f10       ??__E?ET_CLARK_GET_FILES_TO_TAX_NODES@ClarkSupport@U2@@2VQString@@B@@YAXXZ 10001f10 f   ClarkSupport.obj
 0001:00000f30       ??__E?ET_CLARK_GET_FILES_TO_TAX_NODES_ID@ClarkSupport@U2@@2VQString@@B@@YAXXZ 10001f30 f   ClarkSupport.obj
 0001:00000f50       ??__E?ET_CLARK_GET_TARGETS_DEF@ClarkSupport@U2@@2VQString@@B@@YAXXZ 10001f50 f   ClarkSupport.obj
 0001:00000f70       ??__E?ET_CLARK_GET_TARGETS_DEF_ID@ClarkSupport@U2@@2VQString@@B@@YAXXZ 10001f70 f   ClarkSupport.obj
 0001:00000f90       ??__E?ET_CLARK_ID@ClarkSupport@U2@@2VQString@@B@@YAXXZ 10001f90 f   ClarkSupport.obj
 0001:00000fb0       ??__E?ET_CLARK_L@ClarkSupport@U2@@2VQString@@B@@YAXXZ 10001fb0 f   ClarkSupport.obj
 0001:00000fd0       ??__E?ET_CLARK_L_ID@ClarkSupport@U2@@2VQString@@B@@YAXXZ 10001fd0 f   ClarkSupport.obj
 0001:00000ff0       ??__E?_Generic_object@?$_Error_objects@H@std@@2V_Generic_error_category@2@A@@YAXXZ 10001ff0 f   ClarkSupport.obj
 0001:00001000       ??__E?_Iostream_object@?$_Error_objects@H@std@@2V_Iostream_error_category@2@A@@YAXXZ 10002000 f   ClarkSupport.obj
 0001:00001010       ??__E?_System_object@?$_Error_objects@H@std@@2V_System_error_category@2@A@@YAXXZ 10002010 f   ClarkSupport.obj
 0001:00001020       ??__EService_DNAExport@U2@@YAXXZ 10002020 f   ClarkSupport.obj
 0001:00001030       ??__EService_DNAGraphPack@U2@@YAXXZ 10002030 f   ClarkSupport.obj
 0001:00001040       ??__EService_ExternalToolSupport@U2@@YAXXZ 10002040 f   ClarkSupport.obj
 0001:00001050       ??__EService_GUITesting@U2@@YAXXZ 10002050 f   ClarkSupport.obj
 0001:00001060       ??__EService_MaxCoreServiceId@U2@@YAXXZ 10002060 f   ClarkSupport.obj
 0001:00001070       ??__EService_MinCoreServiceId@U2@@YAXXZ 10002070 f   ClarkSupport.obj
 0001:00001080       ??__EService_PluginViewer@U2@@YAXXZ 10002080 f   ClarkSupport.obj
 0001:00001090       ??__EService_Project@U2@@YAXXZ 10002090 f   ClarkSupport.obj
 0001:000010a0       ??__EService_ProjectView@U2@@YAXXZ 100020a0 f   ClarkSupport.obj
 0001:000010b0       ??__EService_QueryDesigner@U2@@YAXXZ 100020b0 f   ClarkSupport.obj
 0001:000010c0       ??__EService_ScriptRegistry@U2@@YAXXZ 100020c0 f   ClarkSupport.obj
 0001:000010d0       ??__EService_TestRunner@U2@@YAXXZ 100020d0 f   ClarkSupport.obj
 0001:000010e0       ??__EService_WorkflowDesigner@U2@@YAXXZ 100020e0 f   ClarkSupport.obj
 0001:000010f0       ??__EalgoLog@U2@@YAXXZ     100020f0 f   ClarkSupport.obj
 0001:00001170       ??__EcmdLog@U2@@YAXXZ      10002170 f   ClarkSupport.obj
 0001:000011f0       ??__EcoreLog@U2@@YAXXZ     100021f0 f   ClarkSupport.obj
 0001:00001270       ??__EioLog@U2@@YAXXZ       10002270 f   ClarkSupport.obj
 0001:000012f0       ??__EperfLog@U2@@YAXXZ     100022f0 f   ClarkSupport.obj
 0001:00001370       ??__EscriptLog@U2@@YAXXZ   10002370 f   ClarkSupport.obj
 0001:000013f0       ??__EtaskLog@U2@@YAXXZ     100023f0 f   ClarkSupport.obj
 0001:00001470       ??__EuiLog@U2@@YAXXZ       10002470 f   ClarkSupport.obj
 0001:000014f0       ??__EuserActLog@U2@@YAXXZ  100024f0 f   ClarkSupport.obj
 0001:00001570       ??__E?PLUGIN_DESCRIPRION@ClarkSupportPlugin@U2@@2VQString@@B@@YAXXZ 10002570 f   ClarkSupportPlugin.obj
 0001:000015a0       ??__E?PLUGIN_NAME@ClarkSupportPlugin@U2@@2VQString@@B@@YAXXZ 100025a0 f   ClarkSupportPlugin.obj
 0001:000015d0       ??__E?_Generic_object@?$_Error_objects@H@std@@2V_Generic_error_category@2@A@@YAXXZ 100025d0 f   ClarkSupportPlugin.obj
 0001:000015e0       ??__E?_Iostream_object@?$_Error_objects@H@std@@2V_Iostream_error_category@2@A@@YAXXZ 100025e0 f   ClarkSupportPlugin.obj
 0001:000015f0       ??__E?_System_object@?$_Error_objects@H@std@@2V_System_error_category@2@A@@YAXXZ 100025f0 f   ClarkSupportPlugin.obj
 0001:00001600       ??__EalgoLog@U2@@YAXXZ     10002600 f   ClarkSupportPlugin.obj
 0001:00001680       ??__EcmdLog@U2@@YAXXZ      10002680 f   ClarkSupportPlugin.obj
 0001:00001700       ??__EcoreLog@U2@@YAXXZ     10002700 f   ClarkSupportPlugin.obj
 0001:00001780       ??__EioLog@U2@@YAXXZ       10002780 f   ClarkSupportPlugin.obj
 0001:00001800       ??__EperfLog@U2@@YAXXZ     10002800 f   ClarkSupportPlugin.obj
 0001:00001880       ??__EscriptLog@U2@@YAXXZ   10002880 f   ClarkSupportPlugin.obj
 0001:00001900       ??__EtaskLog@U2@@YAXXZ     10002900 f   ClarkSupportPlugin.obj
 0001:00001980       ??__EuiLog@U2@@YAXXZ       10002980 f   ClarkSupportPlugin.obj
 0001:00001a00       ??__EuserActLog@U2@@YAXXZ  10002a00 f   ClarkSupportPlugin.obj
 0001:00001a80       ??__E?DATABASE1@GTest_CompareClarkDatabaseMetafiles@U2@@0VQString@@B@@YAXXZ 10002a80 f   ClarkTests.obj
 0001:00001aa0       ??__E?DATABASE1_PREFIXES@GTest_CompareClarkDatabaseMetafiles@U2@@0VQString@@B@@YAXXZ 10002aa0 f   ClarkTests.obj
 0001:00001ac0       ??__E?DATABASE2@GTest_CompareClarkDatabaseMetafiles@U2@@0VQString@@B@@YAXXZ 10002ac0 f   ClarkTests.obj
 0001:00001ae0       ??__E?DATABASE2_PREFIXES@GTest_CompareClarkDatabaseMetafiles@U2@@0VQString@@B@@YAXXZ 10002ae0 f   ClarkTests.obj
 0001:00001b00       ??__E?DATABASE_METAFILES@GTest_CompareClarkDatabaseMetafiles@U2@@0VQStringList@@B@@YAXXZ 10002b00 f   ClarkTests.obj
 0001:00001bf0       ??__E?DATABASE_PREFIX_PLACEHOLDER@GTest_CompareClarkDatabaseMetafiles@U2@@0VQString@@B@@YAXXZ 10002bf0 f   ClarkTests.obj
 0001:00001c10       ??__E?PREFIXES_SEPARATOR@GTest_CompareClarkDatabaseMetafiles@U2@@0VQString@@B@@YAXXZ 10002c10 f   ClarkTests.obj
 0001:00001c30       ??__E?_Generic_object@?$_Error_objects@H@std@@2V_Generic_error_category@2@A@@YAXXZ 10002c30 f   ClarkTests.obj
 0001:00001c40       ??__E?_Iostream_object@?$_Error_objects@H@std@@2V_Iostream_error_category@2@A@@YAXXZ 10002c40 f   ClarkTests.obj
 0001:00001c50       ??__E?_System_object@?$_Error_objects@H@std@@2V_System_error_category@2@A@@YAXXZ 10002c50 f   ClarkTests.obj
 0001:00001c60       ??__EalgoLog@U2@@YAXXZ     10002c60 f   ClarkTests.obj
 0001:00001ce0       ??__EcmdLog@U2@@YAXXZ      10002ce0 f   ClarkTests.obj
 0001:00001d60       ??__EcoreLog@U2@@YAXXZ     10002d60 f   ClarkTests.obj
 0001:00001de0       ??__EioLog@U2@@YAXXZ       10002de0 f   ClarkTests.obj
 0001:00001e60       ??__EperfLog@U2@@YAXXZ     10002e60 f   ClarkTests.obj
 0001:00001ee0       ??__EscriptLog@U2@@YAXXZ   10002ee0 f   ClarkTests.obj
 0001:00001f60       ??__EtaskLog@U2@@YAXXZ     10002f60 f   ClarkTests.obj
 0001:00001fe0       ??__EuiLog@U2@@YAXXZ       10002fe0 f   ClarkTests.obj
 0001:00002060       ??__EuserActLog@U2@@YAXXZ  10003060 f   ClarkTests.obj
 0001:000020e0       ??__E?_Generic_object@?$_Error_objects@H@std@@2V_Generic_error_category@2@A@@YAXXZ 100030e0 f   moc_ClarkBuildWorker.obj
 0001:000020f0       ??__E?_Iostream_object@?$_Error_objects@H@std@@2V_Iostream_error_category@2@A@@YAXXZ 100030f0 f   moc_ClarkBuildWorker.obj
 0001:00002100       ??__E?_System_object@?$_Error_objects@H@std@@2V_System_error_category@2@A@@YAXXZ 10003100 f   moc_ClarkBuildWorker.obj
 0001:00002110       ??__E?staticMetaObject@ClarkBuildPrompter@LocalWorkflow@U2@@2UQMetaObject@@B@@YAXXZ 10003110 f   moc_ClarkBuildWorker.obj
 0001:00002120       ??__E?staticMetaObject@ClarkBuildTask@LocalWorkflow@U2@@2UQMetaObject@@B@@YAXXZ 10003120 f   moc_ClarkBuildWorker.obj
 0001:00002130       ??__E?staticMetaObject@ClarkBuildWorker@LocalWorkflow@U2@@2UQMetaObject@@B@@YAXXZ 10003130 f   moc_ClarkBuildWorker.obj
 0001:00002140       ??__EalgoLog@U2@@YAXXZ     10003140 f   moc_ClarkBuildWorker.obj
 0001:000021c0       ??__EcmdLog@U2@@YAXXZ      100031c0 f   moc_ClarkBuildWorker.obj
 0001:00002240       ??__EcoreLog@U2@@YAXXZ     10003240 f   moc_ClarkBuildWorker.obj
 0001:000022c0       ??__EioLog@U2@@YAXXZ       100032c0 f   moc_ClarkBuildWorker.obj
 0001:00002340       ??__EperfLog@U2@@YAXXZ     10003340 f   moc_ClarkBuildWorker.obj
 0001:000023c0       ??__EscriptLog@U2@@YAXXZ   100033c0 f   moc_ClarkBuildWorker.obj
 0001:00002440       ??__EtaskLog@U2@@YAXXZ     10003440 f   moc_ClarkBuildWorker.obj
 0001:000024c0       ??__EuiLog@U2@@YAXXZ       100034c0 f   moc_ClarkBuildWorker.obj
 0001:00002540       ??__EuserActLog@U2@@YAXXZ  10003540 f   moc_ClarkBuildWorker.obj
 0001:000025c0       ??__E?_Generic_object@?$_Error_objects@H@std@@2V_Generic_error_category@2@A@@YAXXZ 100035c0 f   moc_ClarkClassifyWorker.obj
 0001:000025d0       ??__E?_Iostream_object@?$_Error_objects@H@std@@2V_Iostream_error_category@2@A@@YAXXZ 100035d0 f   moc_ClarkClassifyWorker.obj
 0001:000025e0       ??__E?_System_object@?$_Error_objects@H@std@@2V_System_error_category@2@A@@YAXXZ 100035e0 f   moc_ClarkClassifyWorker.obj
 0001:000025f0       ??__E?staticMetaObject@ClarkClassifyPrompter@LocalWorkflow@U2@@2UQMetaObject@@B@@YAXXZ 100035f0 f   moc_ClarkClassifyWorker.obj
 0001:00002600       ??__E?staticMetaObject@ClarkClassifyTask@LocalWorkflow@U2@@2UQMetaObject@@B@@YAXXZ 10003600 f   moc_ClarkClassifyWorker.obj
 0001:00002610       ??__E?staticMetaObject@ClarkClassifyWorker@LocalWorkflow@U2@@2UQMetaObject@@B@@YAXXZ 10003610 f   moc_ClarkClassifyWorker.obj
 0001:00002620       ??__EalgoLog@U2@@YAXXZ     10003620 f   moc_ClarkClassifyWorker.obj
 0001:000026a0       ??__EcmdLog@U2@@YAXXZ      100036a0 f   moc_ClarkClassifyWorker.obj
 0001:00002720       ??__EcoreLog@U2@@YAXXZ     10003720 f   moc_ClarkClassifyWorker.obj
 0001:000027a0       ??__EioLog@U2@@YAXXZ       100037a0 f   moc_ClarkClassifyWorker.obj
 0001:00002820       ??__EperfLog@U2@@YAXXZ     10003820 f   moc_ClarkClassifyWorker.obj
 0001:000028a0       ??__EscriptLog@U2@@YAXXZ   100038a0 f   moc_ClarkClassifyWorker.obj
 0001:00002920       ??__EtaskLog@U2@@YAXXZ     10003920 f   moc_ClarkClassifyWorker.obj
 0001:000029a0       ??__EuiLog@U2@@YAXXZ       100039a0 f   moc_ClarkClassifyWorker.obj
 0001:00002a20       ??__EuserActLog@U2@@YAXXZ  10003a20 f   moc_ClarkClassifyWorker.obj
 0001:00002aa0       ??__E?_Generic_object@?$_Error_objects@H@std@@2V_Generic_error_category@2@A@@YAXXZ 10003aa0 f   moc_ClarkSupport.obj
 0001:00002ab0       ??__E?_Iostream_object@?$_Error_objects@H@std@@2V_Iostream_error_category@2@A@@YAXXZ 10003ab0 f   moc_ClarkSupport.obj
 0001:00002ac0       ??__E?_System_object@?$_Error_objects@H@std@@2V_System_error_category@2@A@@YAXXZ 10003ac0 f   moc_ClarkSupport.obj
 0001:00002ad0       ??__E?staticMetaObject@ClarkSupport@U2@@2UQMetaObject@@B@@YAXXZ 10003ad0 f   moc_ClarkSupport.obj
 0001:00002ae0       ??__E?_Generic_object@?$_Error_objects@H@std@@2V_Generic_error_category@2@A@@YAXXZ 10003ae0 f   moc_ClarkSupportPlugin.obj
 0001:00002af0       ??__E?_Iostream_object@?$_Error_objects@H@std@@2V_Iostream_error_category@2@A@@YAXXZ 10003af0 f   moc_ClarkSupportPlugin.obj
 0001:00002b00       ??__E?_System_object@?$_Error_objects@H@std@@2V_System_error_category@2@A@@YAXXZ 10003b00 f   moc_ClarkSupportPlugin.obj
 0001:00002b10       ??__E?staticMetaObject@ClarkSupportPlugin@U2@@2UQMetaObject@@B@@YAXXZ 10003b10 f   moc_ClarkSupportPlugin.obj
 0001:00003b7e       __catch$??0?$QList@PAVPort@Workflow@U2@@@@QAE@ABV0@@Z$0 10004b7e f i ClarkBuildWorker.obj
 0001:00003c6e       __catch$??0?$QList@VDataset@U2@@@@QAE@ABV0@@Z$0 10004c6e f i ClarkBuildWorker.obj
 0001:00003d5e       __catch$??0?$QList@VDescriptor@U2@@@@QAE@ABV0@@Z$0 10004d5e f i ClarkBuildWorker.obj
 0001:00003e2e       __catch$??0?$QList@VQString@@@@QAE@ABV0@@Z$0 10004e2e f i ClarkBuildWorker.obj
 0001:00005786       __catch$?_Copy@?$basic_string@DU?$char_traits@D@std@@V?$allocator@D@2@@std@@QAEXII@Z$0 10006786 f i ClarkBuildWorker.obj
 0001:000057c3       __catch$?_Copy@?$basic_string@DU?$char_traits@D@std@@V?$allocator@D@2@@std@@QAEXII@Z$1 100067c3 f i ClarkBuildWorker.obj
 0001:00005ae5       __catch$?append@?$QList@PAVAttribute@U2@@@@QAEXABQAVAttribute@U2@@@Z$4 10006ae5 f i ClarkBuildWorker.obj
 0001:00005b75       __catch$?append@?$QList@PAVPortDescriptor@Workflow@U2@@@@QAEXABQAVPortDescriptor@Workflow@U2@@@Z$4 10006b75 f i ClarkBuildWorker.obj
 0001:00005c2c       __catch$?append@?$QList@VDescriptor@U2@@@@QAEXABVDescriptor@U2@@@Z$0 10006c2c f i ClarkBuildWorker.obj
 0001:00005c2c       __catch$?append@?$QList@VDescriptor@U2@@@@QAEXABVDescriptor@U2@@@Z$2 10006c2c f i ClarkBuildWorker.obj
 0001:00005ced       __catch$?append@?$QList@VQString@@@@QAEXABVQString@@@Z$0 10006ced f i ClarkBuildWorker.obj
 0001:00005d3e       __catch$?append@?$QList@VQString@@@@QAEXABVQString@@@Z$4 10006d3e f i ClarkBuildWorker.obj
 0001:00005e00       __catch$?append@?$QList@VWorkflowNotification@U2@@@@QAEXABVWorkflowNotification@U2@@@Z$2 10006e00 f i ClarkBuildWorker.obj
 0001:00005e00       __catch$?append@?$QList@VWorkflowNotification@U2@@@@QAEXABVWorkflowNotification@U2@@@Z$0 10006e00 f i ClarkBuildWorker.obj
 0001:000068ed       __catch$?createNode@?$QMapData@VDescriptor@U2@@V?$QExplicitlySharedDataPointer@VDataType@U2@@@@@@QAEPAU?$QMapNode@VDescriptor@U2@@V?$QExplicitlySharedDataPointer@VDataType@U2@@@@@@ABVDescriptor@U2@@ABV?$QExplicitlySharedDataPointer@VDataType@U2@@@@PAU2@_N@Z$2 100078ed f i ClarkBuildWorker.obj
 0001:00006995       __catch$?createNode@?$QMapData@VQString@@PAVPropertyDelegate@U2@@@@QAEPAU?$QMapNode@VQString@@PAVPropertyDelegate@U2@@@@ABVQString@@ABQAVPropertyDelegate@U2@@PAU2@_N@Z$2 10007995 f i ClarkBuildWorker.obj
 0001:00006a3e       __catch$?createNode@?$QMapData@VQString@@VQScriptValue@@@@QAEPAU?$QMapNode@VQString@@VQScriptValue@@@@ABVQString@@ABVQScriptValue@@PAU2@_N@Z$0 10007a3e f i ClarkBuildWorker.obj
 0001:00006a53       __catch$?createNode@?$QMapData@VQString@@VQScriptValue@@@@QAEPAU?$QMapNode@VQString@@VQScriptValue@@@@ABVQString@@ABVQScriptValue@@PAU2@_N@Z$2 10007a53 f i ClarkBuildWorker.obj
 0001:00006afe       __catch$?createNode@?$QMapData@VQString@@VQVariant@@@@QAEPAU?$QMapNode@VQString@@VQVariant@@@@ABVQString@@ABVQVariant@@PAU2@_N@Z$0 10007afe f i ClarkBuildWorker.obj
 0001:00006b13       __catch$?createNode@?$QMapData@VQString@@VQVariant@@@@QAEPAU?$QMapNode@VQString@@VQVariant@@@@ABVQString@@ABVQVariant@@PAU2@_N@Z$2 10007b13 f i ClarkBuildWorker.obj
 0001:0000717a       __catch$?detach_helper@?$QList@VDescriptor@U2@@@@AAEXH@Z$0 1000817a f i ClarkBuildWorker.obj
 0001:000074c1       __catch$?detach_helper_grow@?$QList@PAVAttribute@U2@@@@AAEPAUNode@1@HH@Z$2 100084c1 f i ClarkBuildWorker.obj
 0001:000074c1       __catch$?detach_helper_grow@?$QList@PAVAttribute@U2@@@@AAEPAUNode@1@HH@Z$0 100084c1 f i ClarkBuildWorker.obj
 0001:000075d1       __catch$?detach_helper_grow@?$QList@PAVPortDescriptor@Workflow@U2@@@@AAEPAUNode@1@HH@Z$2 100085d1 f i ClarkBuildWorker.obj
 0001:000075d1       __catch$?detach_helper_grow@?$QList@PAVPortDescriptor@Workflow@U2@@@@AAEPAUNode@1@HH@Z$0 100085d1 f i ClarkBuildWorker.obj
 0001:000076df       __catch$?detach_helper_grow@?$QList@VDescriptor@U2@@@@AAEPAUNode@1@HH@Z$2 100086df f i ClarkBuildWorker.obj
 0001:0000771a       __catch$?detach_helper_grow@?$QList@VDescriptor@U2@@@@AAEPAUNode@1@HH@Z$0 1000871a f i ClarkBuildWorker.obj
 0001:0000785e       __catch$?detach_helper_grow@?$QList@VQString@@@@AAEPAUNode@1@HH@Z$2 1000885e f i ClarkBuildWorker.obj
 0001:00007899       __catch$?detach_helper_grow@?$QList@VQString@@@@AAEPAUNode@1@HH@Z$0 10008899 f i ClarkBuildWorker.obj
 0001:000079af       __catch$?detach_helper_grow@?$QList@VWorkflowNotification@U2@@@@AAEPAUNode@1@HH@Z$2 100089af f i ClarkBuildWorker.obj
 0001:000079ea       __catch$?detach_helper_grow@?$QList@VWorkflowNotification@U2@@@@AAEPAUNode@1@HH@Z$0 100089ea f i ClarkBuildWorker.obj
 0001:00009aee       __catch$?node_copy@?$QList@VDataset@U2@@@@AAEXPAUNode@1@00@Z$0 1000aaee f i ClarkBuildWorker.obj
 0001:00009bc5       __catch$?node_copy@?$QList@VDescriptor@U2@@@@AAEXPAUNode@1@00@Z$0 1000abc5 f i ClarkBuildWorker.obj
 0001:00009c72       __catch$?node_copy@?$QList@VQString@@@@AAEXPAUNode@1@00@Z$2 1000ac72 f i ClarkBuildWorker.obj
 0001:00009d2e       __catch$?node_copy@?$QList@VWorkflowNotification@U2@@@@AAEXPAUNode@1@00@Z$0 1000ad2e f i ClarkBuildWorker.obj
 0001:0000d152       __catch$?append@?$QList@U?$QPair@VQString@@V1@@@@@QAEXABU?$QPair@VQString@@V1@@@@Z$0 1000e152 f i ClarkClassifyWorker.obj
 0001:0000d152       __catch$?append@?$QList@U?$QPair@VQString@@V1@@@@@QAEXABU?$QPair@VQString@@V1@@@@Z$2 1000e152 f i ClarkClassifyWorker.obj
 0001:0000d230       __catch$?append@?$QList@VQVariant@@@@QAEXABVQVariant@@@Z$2 1000e230 f i ClarkClassifyWorker.obj
 0001:0000d230       __catch$?append@?$QList@VQVariant@@@@QAEXABVQVariant@@@Z$0 1000e230 f i ClarkClassifyWorker.obj
 0001:0000dc75       __catch$?createNode@?$QMapData@VQString@@I@@QAEPAU?$QMapNode@VQString@@I@@ABVQString@@ABIPAU2@_N@Z$2 1000ec75 f i ClarkClassifyWorker.obj
 0001:0000dd1e       __catch$?createNode@?$QMapData@VQString@@V1@@@QAEPAU?$QMapNode@VQString@@V1@@@ABVQString@@0PAU2@_N@Z$0 1000ed1e f i ClarkClassifyWorker.obj
 0001:0000dd33       __catch$?createNode@?$QMapData@VQString@@V1@@@QAEPAU?$QMapNode@VQString@@V1@@@ABVQString@@0PAU2@_N@Z$2 1000ed33 f i ClarkClassifyWorker.obj
 0001:0000e101       __catch$?detach_helper@?$QList@VQString@@@@AAEXH@Z$0 1000f101 f i ClarkClassifyWorker.obj
 0001:0000e35c       __catch$?detach_helper_grow@?$QList@U?$QPair@VQString@@V1@@@@@AAEPAUNode@1@HH@Z$2 1000f35c f i ClarkClassifyWorker.obj
 0001:0000e397       __catch$?detach_helper_grow@?$QList@U?$QPair@VQString@@V1@@@@@AAEPAUNode@1@HH@Z$0 1000f397 f i ClarkClassifyWorker.obj
 0001:0000e4af       __catch$?detach_helper_grow@?$QList@VQVariant@@@@AAEPAUNode@1@HH@Z$2 1000f4af f i ClarkClassifyWorker.obj
 0001:0000e4ea       __catch$?detach_helper_grow@?$QList@VQVariant@@@@AAEPAUNode@1@HH@Z$0 1000f4ea f i ClarkClassifyWorker.obj
 0001:0001230b       __catch$?node_copy@?$QList@U?$QPair@VQString@@V1@@@@@AAEXPAUNode@1@00@Z$0 1001330b f i ClarkClassifyWorker.obj
 0001:000123ee       __catch$?node_copy@?$QList@VQVariant@@@@AAEXPAUNode@1@00@Z$0 100133ee f i ClarkClassifyWorker.obj
 0001:0001534e       __catch$??0?$QList@PAVXMLTestFactory@U2@@@@QAE@ABV0@@Z$0 1001634e f i ClarkSupportPlugin.obj
 0001:00016275       __catch$?append@?$QList@PAVXMLTestFactory@U2@@@@QAEXABQAVXMLTestFactory@U2@@@Z$4 10017275 f i ClarkTests.obj
 0001:0001649c       __catch$?detach_helper@?$QList@PAVXMLTestFactory@U2@@@@AAEXH@Z$0 1001749c f i ClarkTests.obj
 0001:000165b1       __catch$?detach_helper_grow@?$QList@PAVXMLTestFactory@U2@@@@AAEPAUNode@1@HH@Z$0 100175b1 f i ClarkTests.obj
 0001:000165b1       __catch$?detach_helper_grow@?$QList@PAVXMLTestFactory@U2@@@@AAEPAUNode@1@HH@Z$2 100175b1 f i ClarkTests.obj
 0001:00018a7f       ?ArrayUnwindFilter@@YAHPAU_EXCEPTION_POINTERS@@@Z 10019a7f f   MSVCRT:ehvecdtr.obj
 0001:00018af6       _pre_c_init                10019af6 f   MSVCRT:crtdll.obj
 0001:00018d63       ___DllMainCRTStartup       10019d63 f   MSVCRT:crtdll.obj
 0001:00018eb0       $$000000                   10019eb0     MSVCRT:sehprolg4.obj
 0001:00019530       __unwindfunclet$??$getAttributeValue@H@Attribute@U2@@QBEHPAVWorkflowContext@Workflow@1@@Z$0 1001a530 f   ClarkBuildWorker.obj
 0001:00019539       __unwindfunclet$??$getAttributeValue@H@Attribute@U2@@QBEHPAVWorkflowContext@Workflow@1@@Z$1 1001a539 f   ClarkBuildWorker.obj
 0001:00019541       __unwindfunclet$??$getAttributeValue@H@Attribute@U2@@QBEHPAVWorkflowContext@Workflow@1@@Z$2 1001a541 f   ClarkBuildWorker.obj
 0001:00019549       __unwindfunclet$??$getAttributeValue@H@Attribute@U2@@QBEHPAVWorkflowContext@Workflow@1@@Z$3 1001a549 f   ClarkBuildWorker.obj
 0001:00019551       __unwindfunclet$??$getAttributeValue@H@Attribute@U2@@QBEHPAVWorkflowContext@Workflow@1@@Z$4 1001a551 f   ClarkBuildWorker.obj
 0001:0001955a       __unwindfunclet$??$getAttributeValue@H@Attribute@U2@@QBEHPAVWorkflowContext@Workflow@1@@Z$5 1001a55a f   ClarkBuildWorker.obj
 0001:00019563       __unwindfunclet$??$getAttributeValue@H@Attribute@U2@@QBEHPAVWorkflowContext@Workflow@1@@Z$6 1001a563 f   ClarkBuildWorker.obj
 0001:0001956c       __unwindfunclet$??$getAttributeValue@H@Attribute@U2@@QBEHPAVWorkflowContext@Workflow@1@@Z$7 1001a56c f   ClarkBuildWorker.obj
 0001:00019575       __unwindfunclet$??$getAttributeValue@H@Attribute@U2@@QBEHPAVWorkflowContext@Workflow@1@@Z$8 1001a575 f   ClarkBuildWorker.obj
 0001:0001957e       __unwindfunclet$??$getAttributeValue@H@Attribute@U2@@QBEHPAVWorkflowContext@Workflow@1@@Z$9 1001a57e f   ClarkBuildWorker.obj
 0001:00019587       __unwindfunclet$??$getAttributeValue@H@Attribute@U2@@QBEHPAVWorkflowContext@Workflow@1@@Z$10 1001a587 f   ClarkBuildWorker.obj
 0001:00019590       __unwindfunclet$??$getAttributeValue@H@Attribute@U2@@QBEHPAVWorkflowContext@Workflow@1@@Z$11 1001a590 f   ClarkBuildWorker.obj
 0001:00019599       __ehhandler$??$getAttributeValue@H@Attribute@U2@@QBEHPAVWorkflowContext@Workflow@1@@Z 1001a599 f   ClarkBuildWorker.obj
 0001:000195c0       __unwindfunclet$??$getAttributeValue@VQString@@@Attribute@U2@@QBE?AVQString@@PAVWorkflowContext@Workflow@1@@Z$0 1001a5c0 f   ClarkBuildWorker.obj
 0001:000195da       __unwindfunclet$??$getAttributeValue@VQString@@@Attribute@U2@@QBE?AVQString@@PAVWorkflowContext@Workflow@1@@Z$1 1001a5da f   ClarkBuildWorker.obj
 0001:000195e3       __unwindfunclet$??$getAttributeValue@VQString@@@Attribute@U2@@QBE?AVQString@@PAVWorkflowContext@Workflow@1@@Z$2 1001a5e3 f   ClarkBuildWorker.obj
 0001:000195eb       __unwindfunclet$??$getAttributeValue@VQString@@@Attribute@U2@@QBE?AVQString@@PAVWorkflowContext@Workflow@1@@Z$3 1001a5eb f   ClarkBuildWorker.obj
 0001:000195f3       __unwindfunclet$??$getAttributeValue@VQString@@@Attribute@U2@@QBE?AVQString@@PAVWorkflowContext@Workflow@1@@Z$4 1001a5f3 f   ClarkBuildWorker.obj
 0001:000195fb       __unwindfunclet$??$getAttributeValue@VQString@@@Attribute@U2@@QBE?AVQString@@PAVWorkflowContext@Workflow@1@@Z$5 1001a5fb f   ClarkBuildWorker.obj
 0001:00019604       __unwindfunclet$??$getAttributeValue@VQString@@@Attribute@U2@@QBE?AVQString@@PAVWorkflowContext@Workflow@1@@Z$6 1001a604 f   ClarkBuildWorker.obj
 0001:0001960d       __unwindfunclet$??$getAttributeValue@VQString@@@Attribute@U2@@QBE?AVQString@@PAVWorkflowContext@Workflow@1@@Z$7 1001a60d f   ClarkBuildWorker.obj
 0001:00019616       __unwindfunclet$??$getAttributeValue@VQString@@@Attribute@U2@@QBE?AVQString@@PAVWorkflowContext@Workflow@1@@Z$8 1001a616 f   ClarkBuildWorker.obj
 0001:0001961f       __unwindfunclet$??$getAttributeValue@VQString@@@Attribute@U2@@QBE?AVQString@@PAVWorkflowContext@Workflow@1@@Z$9 1001a61f f   ClarkBuildWorker.obj
 0001:00019628       __unwindfunclet$??$getAttributeValue@VQString@@@Attribute@U2@@QBE?AVQString@@PAVWorkflowContext@Workflow@1@@Z$10 1001a628 f   ClarkBuildWorker.obj
 0001:00019631       __unwindfunclet$??$getAttributeValue@VQString@@@Attribute@U2@@QBE?AVQString@@PAVWorkflowContext@Workflow@1@@Z$11 1001a631 f   ClarkBuildWorker.obj
 0001:0001963a       __unwindfunclet$??$getAttributeValue@VQString@@@Attribute@U2@@QBE?AVQString@@PAVWorkflowContext@Workflow@1@@Z$12 1001a63a f   ClarkBuildWorker.obj
 0001:00019643       __ehhandler$??$getAttributeValue@VQString@@@Attribute@U2@@QBE?AVQString@@PAVWorkflowContext@Workflow@1@@Z 1001a643 f   ClarkBuildWorker.obj
 0001:00019670       __unwindfunclet$??$getValue@VQString@@@BaseWorker@LocalWorkflow@U2@@IBE?AVQString@@ABV3@@Z$0 1001a670 f   ClarkBuildWorker.obj
 0001:0001968a       __unwindfunclet$??$getValue@VQString@@@BaseWorker@LocalWorkflow@U2@@IBE?AVQString@@ABV3@@Z$1 1001a68a f   ClarkBuildWorker.obj
 0001:00019693       __ehhandler$??$getValue@VQString@@@BaseWorker@LocalWorkflow@U2@@IBE?AVQString@@ABV3@@Z 1001a693 f   ClarkBuildWorker.obj
 0001:000196b0       __unwindfunclet$??$qRegisterMetaType@V?$QList@VDataset@U2@@@@@@YAHPBDPAV?$QList@VDataset@U2@@@@W4DefinedType@?$MetaTypeDefinedHelper@V?$QList@VDataset@U2@@@@$00@QtPrivate@@@Z$0 1001a6b0 f   ClarkBuildWorker.obj
 0001:000196b9       __ehhandler$??$qRegisterMetaType@V?$QList@VDataset@U2@@@@@@YAHPBDPAV?$QList@VDataset@U2@@@@W4DefinedType@?$MetaTypeDefinedHelper@V?$QList@VDataset@U2@@@@$00@QtPrivate@@@Z 1001a6b9 f   ClarkBuildWorker.obj
 0001:000196e0       __ehhandler$??0?$QList@PAVPort@Workflow@U2@@@@QAE@ABV0@@Z 1001a6e0 f   ClarkBuildWorker.obj
 0001:00019700       __ehhandler$??0?$QList@VDataset@U2@@@@QAE@ABV0@@Z 1001a700 f   ClarkBuildWorker.obj
 0001:00019720       __ehhandler$??0?$QList@VDescriptor@U2@@@@QAE@ABV0@@Z 1001a720 f   ClarkBuildWorker.obj
 0001:00019740       __ehhandler$??0?$QList@VQString@@@@QAE@ABV0@@Z 1001a740 f   ClarkBuildWorker.obj
 0001:00019760       __unwindfunclet$??0ClarkBuildTask@LocalWorkflow@U2@@QAE@ABVQString@@ABVQStringList@@H0@Z$0 1001a760 f   ClarkBuildWorker.obj
 0001:00019769       __unwindfunclet$??0ClarkBuildTask@LocalWorkflow@U2@@QAE@ABVQString@@ABVQStringList@@H0@Z$1 1001a769 f   ClarkBuildWorker.obj
 0001:00019772       __unwindfunclet$??0ClarkBuildTask@LocalWorkflow@U2@@QAE@ABVQString@@ABVQStringList@@H0@Z$2 1001a772 f   ClarkBuildWorker.obj
 0001:00019781       __unwindfunclet$??0ClarkBuildTask@LocalWorkflow@U2@@QAE@ABVQString@@ABVQStringList@@H0@Z$3 1001a781 f   ClarkBuildWorker.obj
 0001:00019790       __unwindfunclet$??0ClarkBuildTask@LocalWorkflow@U2@@QAE@ABVQString@@ABVQStringList@@H0@Z$4 1001a790 f   ClarkBuildWorker.obj
 0001:0001979e       __unwindfunclet$??0ClarkBuildTask@LocalWorkflow@U2@@QAE@ABVQString@@ABVQStringList@@H0@Z$5 1001a79e f   ClarkBuildWorker.obj
 0001:000197ac       __unwindfunclet$??0ClarkBuildTask@LocalWorkflow@U2@@QAE@ABVQString@@ABVQStringList@@H0@Z$6 1001a7ac f   ClarkBuildWorker.obj
 0001:000197b5       __unwindfunclet$??0ClarkBuildTask@LocalWorkflow@U2@@QAE@ABVQString@@ABVQStringList@@H0@Z$7 1001a7b5 f   ClarkBuildWorker.obj
 0001:000197be       __unwindfunclet$??0ClarkBuildTask@LocalWorkflow@U2@@QAE@ABVQString@@ABVQStringList@@H0@Z$8 1001a7be f   ClarkBuildWorker.obj
 0001:000197c7       __unwindfunclet$??0ClarkBuildTask@LocalWorkflow@U2@@QAE@ABVQString@@ABVQStringList@@H0@Z$9 1001a7c7 f   ClarkBuildWorker.obj
 0001:000197d0       __unwindfunclet$??0ClarkBuildTask@LocalWorkflow@U2@@QAE@ABVQString@@ABVQStringList@@H0@Z$10 1001a7d0 f   ClarkBuildWorker.obj
 0001:000197d9       __unwindfunclet$??0ClarkBuildTask@LocalWorkflow@U2@@QAE@ABVQString@@ABVQStringList@@H0@Z$11 1001a7d9 f   ClarkBuildWorker.obj
 0001:000197e2       __unwindfunclet$??0ClarkBuildTask@LocalWorkflow@U2@@QAE@ABVQString@@ABVQStringList@@H0@Z$12 1001a7e2 f   ClarkBuildWorker.obj
 0001:000197eb       __ehhandler$??0ClarkBuildTask@LocalWorkflow@U2@@QAE@ABVQString@@ABVQStringList@@H0@Z 1001a7eb f   ClarkBuildWorker.obj
 0001:00019810       __unwindfunclet$??1ClarkBuildTask@LocalWorkflow@U2@@UAE@XZ$0 1001a810 f   ClarkBuildWorker.obj
 0001:00019819       __unwindfunclet$??1ClarkBuildTask@LocalWorkflow@U2@@UAE@XZ$1 1001a819 f   ClarkBuildWorker.obj
 0001:00019828       __unwindfunclet$??1ClarkBuildTask@LocalWorkflow@U2@@UAE@XZ$2 1001a828 f   ClarkBuildWorker.obj
 0001:00019837       __ehhandler$??1ClarkBuildTask@LocalWorkflow@U2@@UAE@XZ 1001a837 f   ClarkBuildWorker.obj
 0001:00019860       __unwindfunclet$??A?$QMap@VDescriptor@U2@@V?$QExplicitlySharedDataPointer@VDataType@U2@@@@@@QAEAAV?$QExplicitlySharedDataPointer@VDataType@U2@@@@ABVDescriptor@U2@@@Z$0 1001a860 f   ClarkBuildWorker.obj
 0001:00019868       __ehhandler$??A?$QMap@VDescriptor@U2@@V?$QExplicitlySharedDataPointer@VDataType@U2@@@@@@QAEAAV?$QExplicitlySharedDataPointer@VDataType@U2@@@@ABVDescriptor@U2@@@Z 1001a868 f   ClarkBuildWorker.obj
 0001:00019890       __unwindfunclet$??A?$QMap@VQString@@VQScriptValue@@@@QAEAAVQScriptValue@@ABVQString@@@Z$0 1001a890 f   ClarkBuildWorker.obj
 0001:00019899       __ehhandler$??A?$QMap@VQString@@VQScriptValue@@@@QAEAAVQScriptValue@@ABVQString@@@Z 1001a899 f   ClarkBuildWorker.obj
 0001:000198c0       __unwindfunclet$??A?$QMap@VQString@@VQVariant@@@@QAEAAVQVariant@@ABVQString@@@Z$0 1001a8c0 f   ClarkBuildWorker.obj
 0001:000198c9       __ehhandler$??A?$QMap@VQString@@VQVariant@@@@QAEAAVQVariant@@ABVQString@@@Z 1001a8c9 f   ClarkBuildWorker.obj
 0001:000198f0       __unwindfunclet$??H@YA?BVQString@@ABV0@PBD@Z$0 1001a8f0 f   ClarkBuildWorker.obj
 0001:0001990a       __unwindfunclet$??H@YA?BVQString@@ABV0@PBD@Z$1 1001a90a f   ClarkBuildWorker.obj
 0001:00019913       __ehhandler$??H@YA?BVQString@@ABV0@PBD@Z 1001a913 f   ClarkBuildWorker.obj
 0001:00019930       __unwindfunclet$??_GClarkBuildTask@LocalWorkflow@U2@@UAEPAXI@Z$0 1001a930 f   ClarkBuildWorker.obj
 0001:00019939       __unwindfunclet$??_GClarkBuildTask@LocalWorkflow@U2@@UAEPAXI@Z$1 1001a939 f   ClarkBuildWorker.obj
 0001:00019948       __unwindfunclet$??_GClarkBuildTask@LocalWorkflow@U2@@UAEPAXI@Z$2 1001a948 f   ClarkBuildWorker.obj
 0001:00019957       __ehhandler$??_GClarkBuildTask@LocalWorkflow@U2@@UAEPAXI@Z 1001a957 f   ClarkBuildWorker.obj
 0001:00019980       __unwindfunclet$??__E?wellKnownErrors@ClarkBuildLogParser@LocalWorkflow@U2@@0VQStringList@@B@@YAXXZ$0 1001a980 f   ClarkBuildWorker.obj
 0001:00019989       __unwindfunclet$??__E?wellKnownErrors@ClarkBuildLogParser@LocalWorkflow@U2@@0VQStringList@@B@@YAXXZ$1 1001a989 f   ClarkBuildWorker.obj
 0001:00019992       __unwindfunclet$??__E?wellKnownErrors@ClarkBuildLogParser@LocalWorkflow@U2@@0VQStringList@@B@@YAXXZ$2 1001a992 f   ClarkBuildWorker.obj
 0001:0001999a       __ehhandler$??__E?wellKnownErrors@ClarkBuildLogParser@LocalWorkflow@U2@@0VQStringList@@B@@YAXXZ 1001a99a f   ClarkBuildWorker.obj
 0001:000199c0       __unwindfunclet$??__EalgoLog@U2@@YAXXZ$0 1001a9c0 f   ClarkBuildWorker.obj
 0001:000199c9       __ehhandler$??__EalgoLog@U2@@YAXXZ 1001a9c9 f   ClarkBuildWorker.obj
 0001:000199f0       __unwindfunclet$??__EcmdLog@U2@@YAXXZ$0 1001a9f0 f   ClarkBuildWorker.obj
 0001:000199f9       __ehhandler$??__EcmdLog@U2@@YAXXZ 1001a9f9 f   ClarkBuildWorker.obj
 0001:00019a20       __unwindfunclet$??__EcoreLog@U2@@YAXXZ$0 1001aa20 f   ClarkBuildWorker.obj
 0001:00019a29       __ehhandler$??__EcoreLog@U2@@YAXXZ 1001aa29 f   ClarkBuildWorker.obj
 0001:00019a50       __unwindfunclet$??__EioLog@U2@@YAXXZ$0 1001aa50 f   ClarkBuildWorker.obj
 0001:00019a59       __ehhandler$??__EioLog@U2@@YAXXZ 1001aa59 f   ClarkBuildWorker.obj
 0001:00019a80       __unwindfunclet$??__EperfLog@U2@@YAXXZ$0 1001aa80 f   ClarkBuildWorker.obj
 0001:00019a89       __ehhandler$??__EperfLog@U2@@YAXXZ 1001aa89 f   ClarkBuildWorker.obj
 0001:00019ab0       __unwindfunclet$??__EscriptLog@U2@@YAXXZ$0 1001aab0 f   ClarkBuildWorker.obj
 0001:00019ab9       __ehhandler$??__EscriptLog@U2@@YAXXZ 1001aab9 f   ClarkBuildWorker.obj
 0001:00019ae0       __unwindfunclet$??__EtaskLog@U2@@YAXXZ$0 1001aae0 f   ClarkBuildWorker.obj
 0001:00019ae9       __ehhandler$??__EtaskLog@U2@@YAXXZ 1001aae9 f   ClarkBuildWorker.obj
 0001:00019b10       __unwindfunclet$??__EuiLog@U2@@YAXXZ$0 1001ab10 f   ClarkBuildWorker.obj
 0001:00019b19       __ehhandler$??__EuiLog@U2@@YAXXZ 1001ab19 f   ClarkBuildWorker.obj
 0001:00019b40       __unwindfunclet$??__EuserActLog@U2@@YAXXZ$0 1001ab40 f   ClarkBuildWorker.obj
 0001:00019b49       __ehhandler$??__EuserActLog@U2@@YAXXZ 1001ab49 f   ClarkBuildWorker.obj
 0001:00019b70       __unwindfunclet$?Construct@?$QMetaTypeFunctionHelper@V?$QList@VDataset@U2@@@@$00@QtMetaTypePrivate@@SAPAXPAXPBX@Z$0 1001ab70 f   ClarkBuildWorker.obj
 0001:00019b81       __ehhandler$?Construct@?$QMetaTypeFunctionHelper@V?$QList@VDataset@U2@@@@$00@QtMetaTypePrivate@@SAPAXPAXPBX@Z 1001ab81 f   ClarkBuildWorker.obj
 0001:00019ba0       __unwindfunclet$?Create@?$QMetaTypeFunctionHelper@V?$QList@VDataset@U2@@@@$00@QtMetaTypePrivate@@SAPAXPBX@Z$0 1001aba0 f   ClarkBuildWorker.obj
 0001:00019bab       __ehhandler$?Create@?$QMetaTypeFunctionHelper@V?$QList@VDataset@U2@@@@$00@QtMetaTypePrivate@@SAPAXPBX@Z 1001abab f   ClarkBuildWorker.obj
 0001:00019bd0       __ehhandler$?_Copy@?$basic_string@DU?$char_traits@D@std@@V?$allocator@D@2@@std@@QAEXII@Z 1001abd0 f   ClarkBuildWorker.obj
 0001:00019bf0       __ehhandler$?append@?$QList@PAVAttribute@U2@@@@QAEXABQAVAttribute@U2@@@Z 1001abf0 f   ClarkBuildWorker.obj
 0001:00019c10       __ehhandler$?append@?$QList@PAVPortDescriptor@Workflow@U2@@@@QAEXABQAVPortDescriptor@Workflow@U2@@@Z 1001ac10 f   ClarkBuildWorker.obj
 0001:00019c30       __unwindfunclet$?append@?$QList@VDescriptor@U2@@@@QAEXABVDescriptor@U2@@@Z$6 1001ac30 f   ClarkBuildWorker.obj
 0001:00019c3b       __ehhandler$?append@?$QList@VDescriptor@U2@@@@QAEXABVDescriptor@U2@@@Z 1001ac3b f   ClarkBuildWorker.obj
 0001:00019c60       __unwindfunclet$?append@?$QList@VQString@@@@QAEXABVQString@@@Z$7 1001ac60 f   ClarkBuildWorker.obj
 0001:00019c71       __unwindfunclet$?append@?$QList@VQString@@@@QAEXABVQString@@@Z$11 1001ac71 f   ClarkBuildWorker.obj
 0001:00019c82       __ehhandler$?append@?$QList@VQString@@@@QAEXABVQString@@@Z 1001ac82 f   ClarkBuildWorker.obj
 0001:00019ca0       __unwindfunclet$?append@?$QList@VWorkflowNotification@U2@@@@QAEXABVWorkflowNotification@U2@@@Z$6 1001aca0 f   ClarkBuildWorker.obj
 0001:00019cab       __ehhandler$?append@?$QList@VWorkflowNotification@U2@@@@QAEXABVWorkflowNotification@U2@@@Z 1001acab f   ClarkBuildWorker.obj
 0001:00019cd0       __unwindfunclet$?composeRichDoc@ClarkBuildPrompter@LocalWorkflow@U2@@MAE?AVQString@@XZ$0 1001acd0 f   ClarkBuildWorker.obj
 0001:00019cd9       __unwindfunclet$?composeRichDoc@ClarkBuildPrompter@LocalWorkflow@U2@@MAE?AVQString@@XZ$1 1001acd9 f   ClarkBuildWorker.obj
 0001:00019ce2       __unwindfunclet$?composeRichDoc@ClarkBuildPrompter@LocalWorkflow@U2@@MAE?AVQString@@XZ$2 1001ace2 f   ClarkBuildWorker.obj
 0001:00019ceb       __unwindfunclet$?composeRichDoc@ClarkBuildPrompter@LocalWorkflow@U2@@MAE?AVQString@@XZ$3 1001aceb f   ClarkBuildWorker.obj
 0001:00019cf4       __unwindfunclet$?composeRichDoc@ClarkBuildPrompter@LocalWorkflow@U2@@MAE?AVQString@@XZ$4 1001acf4 f   ClarkBuildWorker.obj
 0001:00019cfd       __unwindfunclet$?composeRichDoc@ClarkBuildPrompter@LocalWorkflow@U2@@MAE?AVQString@@XZ$5 1001acfd f   ClarkBuildWorker.obj
 0001:00019d17       __ehhandler$?composeRichDoc@ClarkBuildPrompter@LocalWorkflow@U2@@MAE?AVQString@@XZ 1001ad17 f   ClarkBuildWorker.obj
 0001:00019d40       __unwindfunclet$?createDescription@?$PrompterBase@VClarkBuildPrompter@LocalWorkflow@U2@@@U2@@UAEPAVActorDocument@Workflow@2@PAVActor@42@@Z$0 1001ad40 f   ClarkBuildWorker.obj
 0001:00019d4b       __unwindfunclet$?createDescription@?$PrompterBase@VClarkBuildPrompter@LocalWorkflow@U2@@@U2@@UAEPAVActorDocument@Workflow@2@PAVActor@42@@Z$3 1001ad4b f   ClarkBuildWorker.obj
 0001:00019d53       __unwindfunclet$?createDescription@?$PrompterBase@VClarkBuildPrompter@LocalWorkflow@U2@@@U2@@UAEPAVActorDocument@Workflow@2@PAVActor@42@@Z$4 1001ad53 f   ClarkBuildWorker.obj
 0001:00019d5b       __unwindfunclet$?createDescription@?$PrompterBase@VClarkBuildPrompter@LocalWorkflow@U2@@@U2@@UAEPAVActorDocument@Workflow@2@PAVActor@42@@Z$6 1001ad5b f   ClarkBuildWorker.obj
 0001:00019d63       __unwindfunclet$?createDescription@?$PrompterBase@VClarkBuildPrompter@LocalWorkflow@U2@@@U2@@UAEPAVActorDocument@Workflow@2@PAVActor@42@@Z$7 1001ad63 f   ClarkBuildWorker.obj
 0001:00019d6b       __ehhandler$?createDescription@?$PrompterBase@VClarkBuildPrompter@LocalWorkflow@U2@@@U2@@UAEPAVActorDocument@Workflow@2@PAVActor@42@@Z 1001ad6b f   ClarkBuildWorker.obj
 0001:00019d90       __unwindfunclet$?createNode@?$QMapData@VDescriptor@U2@@V?$QExplicitlySharedDataPointer@VDataType@U2@@@@@@QAEPAU?$QMapNode@VDescriptor@U2@@V?$QExplicitlySharedDataPointer@VDataType@U2@@@@@@ABVDescriptor@U2@@ABV?$QExplicitlySharedDataPointer@VDataType@U2@@@@PAU2@_N@Z$4 1001ad90 f   ClarkBuildWorker.obj
 0001:00019da4       __ehhandler$?createNode@?$QMapData@VDescriptor@U2@@V?$QExplicitlySharedDataPointer@VDataType@U2@@@@@@QAEPAU?$QMapNode@VDescriptor@U2@@V?$QExplicitlySharedDataPointer@VDataType@U2@@@@@@ABVDescriptor@U2@@ABV?$QExplicitlySharedDataPointer@VDataType@U2@@@@PAU2@_N@Z 1001ada4 f   ClarkBuildWorker.obj
 0001:00019dc0       __unwindfunclet$?createNode@?$QMapData@VQString@@PAVPropertyDelegate@U2@@@@QAEPAU?$QMapNode@VQString@@PAVPropertyDelegate@U2@@@@ABVQString@@ABQAVPropertyDelegate@U2@@PAU2@_N@Z$4 1001adc0 f   ClarkBuildWorker.obj
 0001:00019dd4       __ehhandler$?createNode@?$QMapData@VQString@@PAVPropertyDelegate@U2@@@@QAEPAU?$QMapNode@VQString@@PAVPropertyDelegate@U2@@@@ABVQString@@ABQAVPropertyDelegate@U2@@PAU2@_N@Z 1001add4 f   ClarkBuildWorker.obj
 0001:00019df0       __unwindfunclet$?createNode@?$QMapData@VQString@@VQScriptValue@@@@QAEPAU?$QMapNode@VQString@@VQScriptValue@@@@ABVQString@@ABVQScriptValue@@PAU2@_N@Z$4 1001adf0 f   ClarkBuildWorker.obj
 0001:00019e04       __unwindfunclet$?createNode@?$QMapData@VQString@@VQScriptValue@@@@QAEPAU?$QMapNode@VQString@@VQScriptValue@@@@ABVQString@@ABVQScriptValue@@PAU2@_N@Z$5 1001ae04 f   ClarkBuildWorker.obj
 0001:00019e18       __ehhandler$?createNode@?$QMapData@VQString@@VQScriptValue@@@@QAEPAU?$QMapNode@VQString@@VQScriptValue@@@@ABVQString@@ABVQScriptValue@@PAU2@_N@Z 1001ae18 f   ClarkBuildWorker.obj
 0001:00019e40       __unwindfunclet$?createNode@?$QMapData@VQString@@VQVariant@@@@QAEPAU?$QMapNode@VQString@@VQVariant@@@@ABVQString@@ABVQVariant@@PAU2@_N@Z$4 1001ae40 f   ClarkBuildWorker.obj
 0001:00019e54       __unwindfunclet$?createNode@?$QMapData@VQString@@VQVariant@@@@QAEPAU?$QMapNode@VQString@@VQVariant@@@@ABVQString@@ABVQVariant@@PAU2@_N@Z$5 1001ae54 f   ClarkBuildWorker.obj
 0001:00019e68       __ehhandler$?createNode@?$QMapData@VQString@@VQVariant@@@@QAEPAU?$QMapNode@VQString@@VQVariant@@@@ABVQString@@ABVQVariant@@PAU2@_N@Z 1001ae68 f   ClarkBuildWorker.obj
 0001:00019e90       __unwindfunclet$?createWorker@ClarkBuildWorkerFactory@LocalWorkflow@U2@@UAEPAVWorker@Workflow@3@PAVActor@53@@Z$0 1001ae90 f   ClarkBuildWorker.obj
 0001:00019e9b       __ehhandler$?createWorker@ClarkBuildWorkerFactory@LocalWorkflow@U2@@UAEPAVWorker@Workflow@3@PAVActor@53@@Z 1001ae9b f   ClarkBuildWorker.obj
 0001:00019ec0       __ehhandler$?detach_helper@?$QList@VDescriptor@U2@@@@AAEXH@Z 1001aec0 f   ClarkBuildWorker.obj
 0001:00019ee0       __ehhandler$?detach_helper_grow@?$QList@PAVAttribute@U2@@@@AAEPAUNode@1@HH@Z 1001aee0 f   ClarkBuildWorker.obj
 0001:00019f00       __ehhandler$?detach_helper_grow@?$QList@PAVPortDescriptor@Workflow@U2@@@@AAEPAUNode@1@HH@Z 1001af00 f   ClarkBuildWorker.obj
 0001:00019f20       __ehhandler$?detach_helper_grow@?$QList@VDescriptor@U2@@@@AAEPAUNode@1@HH@Z 1001af20 f   ClarkBuildWorker.obj
 0001:00019f40       __ehhandler$?detach_helper_grow@?$QList@VQString@@@@AAEPAUNode@1@HH@Z 1001af40 f   ClarkBuildWorker.obj
 0001:00019f60       __ehhandler$?detach_helper_grow@?$QList@VWorkflowNotification@U2@@@@AAEPAUNode@1@HH@Z 1001af60 f   ClarkBuildWorker.obj
 0001:00019f80       __unwindfunclet$?getArguments@ClarkBuildTask@LocalWorkflow@U2@@AAE?AVQStringList@@XZ$0 1001af80 f   ClarkBuildWorker.obj
 0001:00019f99       __unwindfunclet$?getArguments@ClarkBuildTask@LocalWorkflow@U2@@AAE?AVQStringList@@XZ$1 1001af99 f   ClarkBuildWorker.obj
 0001:00019fa2       __unwindfunclet$?getArguments@ClarkBuildTask@LocalWorkflow@U2@@AAE?AVQStringList@@XZ$2 1001afa2 f   ClarkBuildWorker.obj
 0001:00019fab       __ehhandler$?getArguments@ClarkBuildTask@LocalWorkflow@U2@@AAE?AVQStringList@@XZ 1001afab f   ClarkBuildWorker.obj
 0001:00019fd0       __unwindfunclet$?init@ClarkBuildWorker@LocalWorkflow@U2@@MAEXXZ$0 1001afd0 f   ClarkBuildWorker.obj
 0001:00019fd9       __unwindfunclet$?init@ClarkBuildWorker@LocalWorkflow@U2@@MAEXXZ$1 1001afd9 f   ClarkBuildWorker.obj
 0001:00019fe2       __unwindfunclet$?init@ClarkBuildWorker@LocalWorkflow@U2@@MAEXXZ$2 1001afe2 f   ClarkBuildWorker.obj
 0001:00019feb       __unwindfunclet$?init@ClarkBuildWorker@LocalWorkflow@U2@@MAEXXZ$3 1001afeb f   ClarkBuildWorker.obj
 0001:00019ff4       __unwindfunclet$?init@ClarkBuildWorker@LocalWorkflow@U2@@MAEXXZ$4 1001aff4 f   ClarkBuildWorker.obj
 0001:00019ffd       __unwindfunclet$?init@ClarkBuildWorker@LocalWorkflow@U2@@MAEXXZ$5 1001affd f   ClarkBuildWorker.obj
 0001:0001a006       __unwindfunclet$?init@ClarkBuildWorker@LocalWorkflow@U2@@MAEXXZ$6 1001b006 f   ClarkBuildWorker.obj
 0001:0001a00f       __ehhandler$?init@ClarkBuildWorker@LocalWorkflow@U2@@MAEXXZ 1001b00f f   ClarkBuildWorker.obj
 0001:0001a030       __unwindfunclet$?init@ClarkBuildWorkerFactory@LocalWorkflow@U2@@SAXXZ$0 1001b030 f   ClarkBuildWorker.obj
 0001:0001a039       __unwindfunclet$?init@ClarkBuildWorkerFactory@LocalWorkflow@U2@@SAXXZ$1 1001b039 f   ClarkBuildWorker.obj
 0001:0001a042       __unwindfunclet$?init@ClarkBuildWorkerFactory@LocalWorkflow@U2@@SAXXZ$2 1001b042 f   ClarkBuildWorker.obj
 0001:0001a04e       __unwindfunclet$?init@ClarkBuildWorkerFactory@LocalWorkflow@U2@@SAXXZ$3 1001b04e f   ClarkBuildWorker.obj
 0001:0001a056       __unwindfunclet$?init@ClarkBuildWorkerFactory@LocalWorkflow@U2@@SAXXZ$4 1001b056 f   ClarkBuildWorker.obj
 0001:0001a05f       __unwindfunclet$?init@ClarkBuildWorkerFactory@LocalWorkflow@U2@@SAXXZ$5 1001b05f f   ClarkBuildWorker.obj
 0001:0001a068       __unwindfunclet$?init@ClarkBuildWorkerFactory@LocalWorkflow@U2@@SAXXZ$6 1001b068 f   ClarkBuildWorker.obj
 0001:0001a071       __unwindfunclet$?init@ClarkBuildWorkerFactory@LocalWorkflow@U2@@SAXXZ$7 1001b071 f   ClarkBuildWorker.obj
 0001:0001a07a       __unwindfunclet$?init@ClarkBuildWorkerFactory@LocalWorkflow@U2@@SAXXZ$8 1001b07a f   ClarkBuildWorker.obj
 0001:0001a083       __unwindfunclet$?init@ClarkBuildWorkerFactory@LocalWorkflow@U2@@SAXXZ$9 1001b083 f   ClarkBuildWorker.obj
 0001:0001a08c       __unwindfunclet$?init@ClarkBuildWorkerFactory@LocalWorkflow@U2@@SAXXZ$10 1001b08c f   ClarkBuildWorker.obj
 0001:0001a095       __unwindfunclet$?init@ClarkBuildWorkerFactory@LocalWorkflow@U2@@SAXXZ$11 1001b095 f   ClarkBuildWorker.obj
 0001:0001a0a1       __unwindfunclet$?init@ClarkBuildWorkerFactory@LocalWorkflow@U2@@SAXXZ$12 1001b0a1 f   ClarkBuildWorker.obj
 0001:0001a0a9       __unwindfunclet$?init@ClarkBuildWorkerFactory@LocalWorkflow@U2@@SAXXZ$13 1001b0a9 f   ClarkBuildWorker.obj
 0001:0001a0b1       __unwindfunclet$?init@ClarkBuildWorkerFactory@LocalWorkflow@U2@@SAXXZ$14 1001b0b1 f   ClarkBuildWorker.obj
 0001:0001a0bc       __unwindfunclet$?init@ClarkBuildWorkerFactory@LocalWorkflow@U2@@SAXXZ$15 1001b0bc f   ClarkBuildWorker.obj
 0001:0001a0c7       __unwindfunclet$?init@ClarkBuildWorkerFactory@LocalWorkflow@U2@@SAXXZ$16 1001b0c7 f   ClarkBuildWorker.obj
 0001:0001a0e1       __unwindfunclet$?init@ClarkBuildWorkerFactory@LocalWorkflow@U2@@SAXXZ$18 1001b0e1 f   ClarkBuildWorker.obj
 0001:0001a0e9       __unwindfunclet$?init@ClarkBuildWorkerFactory@LocalWorkflow@U2@@SAXXZ$19 1001b0e9 f   ClarkBuildWorker.obj
 0001:0001a0f2       __unwindfunclet$?init@ClarkBuildWorkerFactory@LocalWorkflow@U2@@SAXXZ$20 1001b0f2 f   ClarkBuildWorker.obj
 0001:0001a0fb       __unwindfunclet$?init@ClarkBuildWorkerFactory@LocalWorkflow@U2@@SAXXZ$21 1001b0fb f   ClarkBuildWorker.obj
 0001:0001a104       __unwindfunclet$?init@ClarkBuildWorkerFactory@LocalWorkflow@U2@@SAXXZ$22 1001b104 f   ClarkBuildWorker.obj
 0001:0001a10d       __unwindfunclet$?init@ClarkBuildWorkerFactory@LocalWorkflow@U2@@SAXXZ$23 1001b10d f   ClarkBuildWorker.obj
 0001:0001a116       __unwindfunclet$?init@ClarkBuildWorkerFactory@LocalWorkflow@U2@@SAXXZ$24 1001b116 f   ClarkBuildWorker.obj
 0001:0001a11f       __unwindfunclet$?init@ClarkBuildWorkerFactory@LocalWorkflow@U2@@SAXXZ$25 1001b11f f   ClarkBuildWorker.obj
 0001:0001a128       __unwindfunclet$?init@ClarkBuildWorkerFactory@LocalWorkflow@U2@@SAXXZ$26 1001b128 f   ClarkBuildWorker.obj
 0001:0001a131       __unwindfunclet$?init@ClarkBuildWorkerFactory@LocalWorkflow@U2@@SAXXZ$27 1001b131 f   ClarkBuildWorker.obj
 0001:0001a13d       __unwindfunclet$?init@ClarkBuildWorkerFactory@LocalWorkflow@U2@@SAXXZ$28 1001b13d f   ClarkBuildWorker.obj
 0001:0001a148       __unwindfunclet$?init@ClarkBuildWorkerFactory@LocalWorkflow@U2@@SAXXZ$29 1001b148 f   ClarkBuildWorker.obj
 0001:0001a162       __unwindfunclet$?init@ClarkBuildWorkerFactory@LocalWorkflow@U2@@SAXXZ$31 1001b162 f   ClarkBuildWorker.obj
 0001:0001a16d       __unwindfunclet$?init@ClarkBuildWorkerFactory@LocalWorkflow@U2@@SAXXZ$32 1001b16d f   ClarkBuildWorker.obj
 0001:0001a187       __unwindfunclet$?init@ClarkBuildWorkerFactory@LocalWorkflow@U2@@SAXXZ$34 1001b187 f   ClarkBuildWorker.obj
 0001:0001a192       __unwindfunclet$?init@ClarkBuildWorkerFactory@LocalWorkflow@U2@@SAXXZ$35 1001b192 f   ClarkBuildWorker.obj
 0001:0001a1ac       __unwindfunclet$?init@ClarkBuildWorkerFactory@LocalWorkflow@U2@@SAXXZ$37 1001b1ac f   ClarkBuildWorker.obj
 0001:0001a1b4       __unwindfunclet$?init@ClarkBuildWorkerFactory@LocalWorkflow@U2@@SAXXZ$38 1001b1b4 f   ClarkBuildWorker.obj
 0001:0001a1bc       __unwindfunclet$?init@ClarkBuildWorkerFactory@LocalWorkflow@U2@@SAXXZ$39 1001b1bc f   ClarkBuildWorker.obj
 0001:0001a1c5       __unwindfunclet$?init@ClarkBuildWorkerFactory@LocalWorkflow@U2@@SAXXZ$40 1001b1c5 f   ClarkBuildWorker.obj
 0001:0001a1ce       __unwindfunclet$?init@ClarkBuildWorkerFactory@LocalWorkflow@U2@@SAXXZ$41 1001b1ce f   ClarkBuildWorker.obj
 0001:0001a1d7       __unwindfunclet$?init@ClarkBuildWorkerFactory@LocalWorkflow@U2@@SAXXZ$42 1001b1d7 f   ClarkBuildWorker.obj
 0001:0001a1e0       __unwindfunclet$?init@ClarkBuildWorkerFactory@LocalWorkflow@U2@@SAXXZ$43 1001b1e0 f   ClarkBuildWorker.obj
 0001:0001a1e9       __unwindfunclet$?init@ClarkBuildWorkerFactory@LocalWorkflow@U2@@SAXXZ$44 1001b1e9 f   ClarkBuildWorker.obj
 0001:0001a1f2       __unwindfunclet$?init@ClarkBuildWorkerFactory@LocalWorkflow@U2@@SAXXZ$45 1001b1f2 f   ClarkBuildWorker.obj
 0001:0001a1fb       __unwindfunclet$?init@ClarkBuildWorkerFactory@LocalWorkflow@U2@@SAXXZ$46 1001b1fb f   ClarkBuildWorker.obj
 0001:0001a204       __unwindfunclet$?init@ClarkBuildWorkerFactory@LocalWorkflow@U2@@SAXXZ$47 1001b204 f   ClarkBuildWorker.obj
 0001:0001a20d       __unwindfunclet$?init@ClarkBuildWorkerFactory@LocalWorkflow@U2@@SAXXZ$48 1001b20d f   ClarkBuildWorker.obj
 0001:0001a216       __unwindfunclet$?init@ClarkBuildWorkerFactory@LocalWorkflow@U2@@SAXXZ$49 1001b216 f   ClarkBuildWorker.obj
 0001:0001a21f       __unwindfunclet$?init@ClarkBuildWorkerFactory@LocalWorkflow@U2@@SAXXZ$50 1001b21f f   ClarkBuildWorker.obj
 0001:0001a228       __unwindfunclet$?init@ClarkBuildWorkerFactory@LocalWorkflow@U2@@SAXXZ$51 1001b228 f   ClarkBuildWorker.obj
 0001:0001a233       __unwindfunclet$?init@ClarkBuildWorkerFactory@LocalWorkflow@U2@@SAXXZ$52 1001b233 f   ClarkBuildWorker.obj
 0001:0001a23c       __unwindfunclet$?init@ClarkBuildWorkerFactory@LocalWorkflow@U2@@SAXXZ$53 1001b23c f   ClarkBuildWorker.obj
 0001:0001a245       __unwindfunclet$?init@ClarkBuildWorkerFactory@LocalWorkflow@U2@@SAXXZ$54 1001b245 f   ClarkBuildWorker.obj
 0001:0001a24e       __unwindfunclet$?init@ClarkBuildWorkerFactory@LocalWorkflow@U2@@SAXXZ$55 1001b24e f   ClarkBuildWorker.obj
 0001:0001a259       __unwindfunclet$?init@ClarkBuildWorkerFactory@LocalWorkflow@U2@@SAXXZ$56 1001b259 f   ClarkBuildWorker.obj
 0001:0001a273       __unwindfunclet$?init@ClarkBuildWorkerFactory@LocalWorkflow@U2@@SAXXZ$57 1001b273 f   ClarkBuildWorker.obj
 0001:0001a27e       __unwindfunclet$?init@ClarkBuildWorkerFactory@LocalWorkflow@U2@@SAXXZ$58 1001b27e f   ClarkBuildWorker.obj
 0001:0001a289       __unwindfunclet$?init@ClarkBuildWorkerFactory@LocalWorkflow@U2@@SAXXZ$59 1001b289 f   ClarkBuildWorker.obj
 0001:0001a294       __unwindfunclet$?init@ClarkBuildWorkerFactory@LocalWorkflow@U2@@SAXXZ$60 1001b294 f   ClarkBuildWorker.obj
 0001:0001a29f       __unwindfunclet$?init@ClarkBuildWorkerFactory@LocalWorkflow@U2@@SAXXZ$61 1001b29f f   ClarkBuildWorker.obj
 0001:0001a2a8       __unwindfunclet$?init@ClarkBuildWorkerFactory@LocalWorkflow@U2@@SAXXZ$62 1001b2a8 f   ClarkBuildWorker.obj
 0001:0001a2b1       __unwindfunclet$?init@ClarkBuildWorkerFactory@LocalWorkflow@U2@@SAXXZ$63 1001b2b1 f   ClarkBuildWorker.obj
 0001:0001a2ba       __unwindfunclet$?init@ClarkBuildWorkerFactory@LocalWorkflow@U2@@SAXXZ$64 1001b2ba f   ClarkBuildWorker.obj
 0001:0001a2c3       __unwindfunclet$?init@ClarkBuildWorkerFactory@LocalWorkflow@U2@@SAXXZ$65 1001b2c3 f   ClarkBuildWorker.obj
 0001:0001a2cc       __unwindfunclet$?init@ClarkBuildWorkerFactory@LocalWorkflow@U2@@SAXXZ$66 1001b2cc f   ClarkBuildWorker.obj
 0001:0001a2d7       __ehhandler$?init@ClarkBuildWorkerFactory@LocalWorkflow@U2@@SAXXZ 1001b2d7 f   ClarkBuildWorker.obj
 0001:0001a300       __unwindfunclet$?isError@ClarkBuildLogParser@LocalWorkflow@U2@@EBE_NABVQString@@@Z$0 1001b300 f   ClarkBuildWorker.obj
 0001:0001a308       __ehhandler$?isError@ClarkBuildLogParser@LocalWorkflow@U2@@EBE_NABVQString@@@Z 1001b308 f   ClarkBuildWorker.obj
 0001:0001a330       __unwindfunclet$?metaType@?$QVariantValueHelper@V?$QList@VDataset@U2@@@@@QtPrivate@@SA?AV?$QList@VDataset@U2@@@@ABVQVariant@@@Z$0 1001b330 f   ClarkBuildWorker.obj
 0001:0001a349       __unwindfunclet$?metaType@?$QVariantValueHelper@V?$QList@VDataset@U2@@@@@QtPrivate@@SA?AV?$QList@VDataset@U2@@@@ABVQVariant@@@Z$1 1001b349 f   ClarkBuildWorker.obj
 0001:0001a351       __ehhandler$?metaType@?$QVariantValueHelper@V?$QList@VDataset@U2@@@@@QtPrivate@@SA?AV?$QList@VDataset@U2@@@@ABVQVariant@@@Z 1001b351 f   ClarkBuildWorker.obj
 0001:0001a370       __unwindfunclet$?metaType@?$QVariantValueHelper@VQString@@@QtPrivate@@SA?AVQString@@ABVQVariant@@@Z$0 1001b370 f   ClarkBuildWorker.obj
 0001:0001a38a       __unwindfunclet$?metaType@?$QVariantValueHelper@VQString@@@QtPrivate@@SA?AVQString@@ABVQVariant@@@Z$1 1001b38a f   ClarkBuildWorker.obj
 0001:0001a393       __ehhandler$?metaType@?$QVariantValueHelper@VQString@@@QtPrivate@@SA?AVQString@@ABVQVariant@@@Z 1001b393 f   ClarkBuildWorker.obj
 0001:0001a3b0       __unwindfunclet$?node_construct@?$QList@VDescriptor@U2@@@@AAEXPAUNode@1@ABVDescriptor@U2@@@Z$0 1001b3b0 f   ClarkBuildWorker.obj
 0001:0001a3bb       __ehhandler$?node_construct@?$QList@VDescriptor@U2@@@@AAEXPAUNode@1@ABVDescriptor@U2@@@Z 1001b3bb f   ClarkBuildWorker.obj
 0001:0001a3e0       __unwindfunclet$?node_construct@?$QList@VQString@@@@AAEXPAUNode@1@ABVQString@@@Z$1 1001b3e0 f   ClarkBuildWorker.obj
 0001:0001a3f1       __ehhandler$?node_construct@?$QList@VQString@@@@AAEXPAUNode@1@ABVQString@@@Z 1001b3f1 f   ClarkBuildWorker.obj
 0001:0001a410       __unwindfunclet$?node_construct@?$QList@VWorkflowNotification@U2@@@@AAEXPAUNode@1@ABVWorkflowNotification@U2@@@Z$0 1001b410 f   ClarkBuildWorker.obj
 0001:0001a41b       __ehhandler$?node_construct@?$QList@VWorkflowNotification@U2@@@@AAEXPAUNode@1@ABVWorkflowNotification@U2@@@Z 1001b41b f   ClarkBuildWorker.obj
 0001:0001a440       __unwindfunclet$?node_copy@?$QList@VDataset@U2@@@@AAEXPAUNode@1@00@Z$4 1001b440 f   ClarkBuildWorker.obj
 0001:0001a44b       __ehhandler$?node_copy@?$QList@VDataset@U2@@@@AAEXPAUNode@1@00@Z 1001b44b f   ClarkBuildWorker.obj
 0001:0001a470       __unwindfunclet$?node_copy@?$QList@VDescriptor@U2@@@@AAEXPAUNode@1@00@Z$4 1001b470 f   ClarkBuildWorker.obj
 0001:0001a47b       __ehhandler$?node_copy@?$QList@VDescriptor@U2@@@@AAEXPAUNode@1@00@Z 1001b47b f   ClarkBuildWorker.obj
 0001:0001a4a0       __unwindfunclet$?node_copy@?$QList@VQString@@@@AAEXPAUNode@1@00@Z$5 1001b4a0 f   ClarkBuildWorker.obj
 0001:0001a4b1       __ehhandler$?node_copy@?$QList@VQString@@@@AAEXPAUNode@1@00@Z 1001b4b1 f   ClarkBuildWorker.obj
 0001:0001a4d0       __unwindfunclet$?node_copy@?$QList@VWorkflowNotification@U2@@@@AAEXPAUNode@1@00@Z$4 1001b4d0 f   ClarkBuildWorker.obj
 0001:0001a4db       __ehhandler$?node_copy@?$QList@VWorkflowNotification@U2@@@@AAEXPAUNode@1@00@Z 1001b4db f   ClarkBuildWorker.obj
 0001:0001a500       __unwindfunclet$?prepare@ClarkBuildTask@LocalWorkflow@U2@@EAEXXZ$0 1001b500 f   ClarkBuildWorker.obj
 0001:0001a509       __unwindfunclet$?prepare@ClarkBuildTask@LocalWorkflow@U2@@EAEXXZ$1 1001b509 f   ClarkBuildWorker.obj
 0001:0001a512       __unwindfunclet$?prepare@ClarkBuildTask@LocalWorkflow@U2@@EAEXXZ$2 1001b512 f   ClarkBuildWorker.obj
 0001:0001a51b       __unwindfunclet$?prepare@ClarkBuildTask@LocalWorkflow@U2@@EAEXXZ$3 1001b51b f   ClarkBuildWorker.obj
 0001:0001a524       __unwindfunclet$?prepare@ClarkBuildTask@LocalWorkflow@U2@@EAEXXZ$4 1001b524 f   ClarkBuildWorker.obj
 0001:0001a52d       __unwindfunclet$?prepare@ClarkBuildTask@LocalWorkflow@U2@@EAEXXZ$5 1001b52d f   ClarkBuildWorker.obj
 0001:0001a536       __unwindfunclet$?prepare@ClarkBuildTask@LocalWorkflow@U2@@EAEXXZ$6 1001b536 f   ClarkBuildWorker.obj
 0001:0001a53f       __unwindfunclet$?prepare@ClarkBuildTask@LocalWorkflow@U2@@EAEXXZ$7 1001b53f f   ClarkBuildWorker.obj
 0001:0001a548       __unwindfunclet$?prepare@ClarkBuildTask@LocalWorkflow@U2@@EAEXXZ$8 1001b548 f   ClarkBuildWorker.obj
 0001:0001a551       __unwindfunclet$?prepare@ClarkBuildTask@LocalWorkflow@U2@@EAEXXZ$9 1001b551 f   ClarkBuildWorker.obj
 0001:0001a55a       __unwindfunclet$?prepare@ClarkBuildTask@LocalWorkflow@U2@@EAEXXZ$10 1001b55a f   ClarkBuildWorker.obj
 0001:0001a563       __unwindfunclet$?prepare@ClarkBuildTask@LocalWorkflow@U2@@EAEXXZ$11 1001b563 f   ClarkBuildWorker.obj
 0001:0001a56c       __unwindfunclet$?prepare@ClarkBuildTask@LocalWorkflow@U2@@EAEXXZ$12 1001b56c f   ClarkBuildWorker.obj
 0001:0001a577       __unwindfunclet$?prepare@ClarkBuildTask@LocalWorkflow@U2@@EAEXXZ$13 1001b577 f   ClarkBuildWorker.obj
 0001:0001a591       __unwindfunclet$?prepare@ClarkBuildTask@LocalWorkflow@U2@@EAEXXZ$14 1001b591 f   ClarkBuildWorker.obj
 0001:0001a59c       __unwindfunclet$?prepare@ClarkBuildTask@LocalWorkflow@U2@@EAEXXZ$15 1001b59c f   ClarkBuildWorker.obj
 0001:0001a5b6       __unwindfunclet$?prepare@ClarkBuildTask@LocalWorkflow@U2@@EAEXXZ$16 1001b5b6 f   ClarkBuildWorker.obj
 0001:0001a5cf       __unwindfunclet$?prepare@ClarkBuildTask@LocalWorkflow@U2@@EAEXXZ$17 1001b5cf f   ClarkBuildWorker.obj
 0001:0001a5e8       __unwindfunclet$?prepare@ClarkBuildTask@LocalWorkflow@U2@@EAEXXZ$18 1001b5e8 f   ClarkBuildWorker.obj
 0001:0001a5f0       __ehhandler$?prepare@ClarkBuildTask@LocalWorkflow@U2@@EAEXXZ 1001b5f0 f   ClarkBuildWorker.obj
 0001:0001a610       __unwindfunclet$?qt_metatype_id@?$QMetaTypeId@V?$QList@VDataset@U2@@@@@@SAHXZ$0 1001b610 f   ClarkBuildWorker.obj
 0001:0001a619       __ehhandler$?qt_metatype_id@?$QMetaTypeId@V?$QList@VDataset@U2@@@@@@SAHXZ 1001b619 f   ClarkBuildWorker.obj
 0001:0001a640       __unwindfunclet$?sl_taskFinished@ClarkBuildWorker@LocalWorkflow@U2@@AAEXPAVTask@3@@Z$0 1001b640 f   ClarkBuildWorker.obj
 0001:0001a649       __unwindfunclet$?sl_taskFinished@ClarkBuildWorker@LocalWorkflow@U2@@AAEXPAVTask@3@@Z$1 1001b649 f   ClarkBuildWorker.obj
 0001:0001a652       __unwindfunclet$?sl_taskFinished@ClarkBuildWorker@LocalWorkflow@U2@@AAEXPAVTask@3@@Z$2 1001b652 f   ClarkBuildWorker.obj
 0001:0001a65b       __unwindfunclet$?sl_taskFinished@ClarkBuildWorker@LocalWorkflow@U2@@AAEXPAVTask@3@@Z$3 1001b65b f   ClarkBuildWorker.obj
 0001:0001a664       __unwindfunclet$?sl_taskFinished@ClarkBuildWorker@LocalWorkflow@U2@@AAEXPAVTask@3@@Z$4 1001b664 f   ClarkBuildWorker.obj
 0001:0001a66d       __unwindfunclet$?sl_taskFinished@ClarkBuildWorker@LocalWorkflow@U2@@AAEXPAVTask@3@@Z$5 1001b66d f   ClarkBuildWorker.obj
 0001:0001a676       __unwindfunclet$?sl_taskFinished@ClarkBuildWorker@LocalWorkflow@U2@@AAEXPAVTask@3@@Z$6 1001b676 f   ClarkBuildWorker.obj
 0001:0001a67f       __unwindfunclet$?sl_taskFinished@ClarkBuildWorker@LocalWorkflow@U2@@AAEXPAVTask@3@@Z$7 1001b67f f   ClarkBuildWorker.obj
 0001:0001a688       __unwindfunclet$?sl_taskFinished@ClarkBuildWorker@LocalWorkflow@U2@@AAEXPAVTask@3@@Z$8 1001b688 f   ClarkBuildWorker.obj
 0001:0001a691       __unwindfunclet$?sl_taskFinished@ClarkBuildWorker@LocalWorkflow@U2@@AAEXPAVTask@3@@Z$9 1001b691 f   ClarkBuildWorker.obj
 0001:0001a699       __unwindfunclet$?sl_taskFinished@ClarkBuildWorker@LocalWorkflow@U2@@AAEXPAVTask@3@@Z$10 1001b699 f   ClarkBuildWorker.obj
 0001:0001a6a2       __unwindfunclet$?sl_taskFinished@ClarkBuildWorker@LocalWorkflow@U2@@AAEXPAVTask@3@@Z$11 1001b6a2 f   ClarkBuildWorker.obj
 0001:0001a6ab       __unwindfunclet$?sl_taskFinished@ClarkBuildWorker@LocalWorkflow@U2@@AAEXPAVTask@3@@Z$12 1001b6ab f   ClarkBuildWorker.obj
 0001:0001a6b4       __unwindfunclet$?sl_taskFinished@ClarkBuildWorker@LocalWorkflow@U2@@AAEXPAVTask@3@@Z$13 1001b6b4 f   ClarkBuildWorker.obj
 0001:0001a6bd       __unwindfunclet$?sl_taskFinished@ClarkBuildWorker@LocalWorkflow@U2@@AAEXPAVTask@3@@Z$15 1001b6bd f   ClarkBuildWorker.obj
 0001:0001a6c6       __unwindfunclet$?sl_taskFinished@ClarkBuildWorker@LocalWorkflow@U2@@AAEXPAVTask@3@@Z$16 1001b6c6 f   ClarkBuildWorker.obj
 0001:0001a6cf       __unwindfunclet$?sl_taskFinished@ClarkBuildWorker@LocalWorkflow@U2@@AAEXPAVTask@3@@Z$17 1001b6cf f   ClarkBuildWorker.obj
 0001:0001a6d8       __ehhandler$?sl_taskFinished@ClarkBuildWorker@LocalWorkflow@U2@@AAEXPAVTask@3@@Z 1001b6d8 f   ClarkBuildWorker.obj
 0001:0001a700       __unwindfunclet$?tick@ClarkBuildWorker@LocalWorkflow@U2@@MAEPAVTask@3@XZ$0 1001b700 f   ClarkBuildWorker.obj
 0001:0001a709       __unwindfunclet$?tick@ClarkBuildWorker@LocalWorkflow@U2@@MAEPAVTask@3@XZ$1 1001b709 f   ClarkBuildWorker.obj
 0001:0001a711       __unwindfunclet$?tick@ClarkBuildWorker@LocalWorkflow@U2@@MAEPAVTask@3@XZ$4 1001b711 f   ClarkBuildWorker.obj
 0001:0001a71a       __unwindfunclet$?tick@ClarkBuildWorker@LocalWorkflow@U2@@MAEPAVTask@3@XZ$5 1001b71a f   ClarkBuildWorker.obj
 0001:0001a722       __unwindfunclet$?tick@ClarkBuildWorker@LocalWorkflow@U2@@MAEPAVTask@3@XZ$6 1001b722 f   ClarkBuildWorker.obj
 0001:0001a72b       __unwindfunclet$?tick@ClarkBuildWorker@LocalWorkflow@U2@@MAEPAVTask@3@XZ$7 1001b72b f   ClarkBuildWorker.obj
 0001:0001a734       __unwindfunclet$?tick@ClarkBuildWorker@LocalWorkflow@U2@@MAEPAVTask@3@XZ$8 1001b734 f   ClarkBuildWorker.obj
 0001:0001a73f       __unwindfunclet$?tick@ClarkBuildWorker@LocalWorkflow@U2@@MAEPAVTask@3@XZ$9 1001b73f f   ClarkBuildWorker.obj
 0001:0001a747       __unwindfunclet$?tick@ClarkBuildWorker@LocalWorkflow@U2@@MAEPAVTask@3@XZ$10 1001b747 f   ClarkBuildWorker.obj
 0001:0001a752       __unwindfunclet$?tick@ClarkBuildWorker@LocalWorkflow@U2@@MAEPAVTask@3@XZ$2 1001b752 f   ClarkBuildWorker.obj
 0001:0001a75d       __unwindfunclet$?tick@ClarkBuildWorker@LocalWorkflow@U2@@MAEPAVTask@3@XZ$3 1001b75d f   ClarkBuildWorker.obj
 0001:0001a777       __ehhandler$?tick@ClarkBuildWorker@LocalWorkflow@U2@@MAEPAVTask@3@XZ 1001b777 f   ClarkBuildWorker.obj
 0001:0001a7a0       __unwindfunclet$?uniqueKeys@?$QMap@VDescriptor@U2@@VQVariant@@@@QBE?AV?$QList@VDescriptor@U2@@@@XZ$1 1001b7a0 f   ClarkBuildWorker.obj
 0001:0001a7b9       __ehhandler$?uniqueKeys@?$QMap@VDescriptor@U2@@VQVariant@@@@QBE?AV?$QList@VDescriptor@U2@@@@XZ 1001b7b9 f   ClarkBuildWorker.obj
 0001:0001a7e0       __unwindfunclet$?validateTaxonomy@ClarkBuildValidator@LocalWorkflow@U2@@ABE_NPBVActor@Workflow@3@AAV?$QList@VWorkflowNotification@U2@@@@@Z$3 1001b7e0 f   ClarkBuildWorker.obj
 0001:0001a7e9       __unwindfunclet$?validateTaxonomy@ClarkBuildValidator@LocalWorkflow@U2@@ABE_NPBVActor@Workflow@3@AAV?$QList@VWorkflowNotification@U2@@@@@Z$4 1001b7e9 f   ClarkBuildWorker.obj
 0001:0001a7f2       __unwindfunclet$?validateTaxonomy@ClarkBuildValidator@LocalWorkflow@U2@@ABE_NPBVActor@Workflow@3@AAV?$QList@VWorkflowNotification@U2@@@@@Z$5 1001b7f2 f   ClarkBuildWorker.obj
 0001:0001a7fb       __unwindfunclet$?validateTaxonomy@ClarkBuildValidator@LocalWorkflow@U2@@ABE_NPBVActor@Workflow@3@AAV?$QList@VWorkflowNotification@U2@@@@@Z$6 1001b7fb f   ClarkBuildWorker.obj
 0001:0001a804       __unwindfunclet$?validateTaxonomy@ClarkBuildValidator@LocalWorkflow@U2@@ABE_NPBVActor@Workflow@3@AAV?$QList@VWorkflowNotification@U2@@@@@Z$7 1001b804 f   ClarkBuildWorker.obj
 0001:0001a80d       __unwindfunclet$?validateTaxonomy@ClarkBuildValidator@LocalWorkflow@U2@@ABE_NPBVActor@Workflow@3@AAV?$QList@VWorkflowNotification@U2@@@@@Z$8 1001b80d f   ClarkBuildWorker.obj
 0001:0001a816       __unwindfunclet$?validateTaxonomy@ClarkBuildValidator@LocalWorkflow@U2@@ABE_NPBVActor@Workflow@3@AAV?$QList@VWorkflowNotification@U2@@@@@Z$9 1001b816 f   ClarkBuildWorker.obj
 0001:0001a81f       __unwindfunclet$?validateTaxonomy@ClarkBuildValidator@LocalWorkflow@U2@@ABE_NPBVActor@Workflow@3@AAV?$QList@VWorkflowNotification@U2@@@@@Z$10 1001b81f f   ClarkBuildWorker.obj
 0001:0001a828       __unwindfunclet$?validateTaxonomy@ClarkBuildValidator@LocalWorkflow@U2@@ABE_NPBVActor@Workflow@3@AAV?$QList@VWorkflowNotification@U2@@@@@Z$11 1001b828 f   ClarkBuildWorker.obj
 0001:0001a831       __unwindfunclet$?validateTaxonomy@ClarkBuildValidator@LocalWorkflow@U2@@ABE_NPBVActor@Workflow@3@AAV?$QList@VWorkflowNotification@U2@@@@@Z$12 1001b831 f   ClarkBuildWorker.obj
 0001:0001a83a       __unwindfunclet$?validateTaxonomy@ClarkBuildValidator@LocalWorkflow@U2@@ABE_NPBVActor@Workflow@3@AAV?$QList@VWorkflowNotification@U2@@@@@Z$13 1001b83a f   ClarkBuildWorker.obj
 0001:0001a843       __unwindfunclet$?validateTaxonomy@ClarkBuildValidator@LocalWorkflow@U2@@ABE_NPBVActor@Workflow@3@AAV?$QList@VWorkflowNotification@U2@@@@@Z$14 1001b843 f   ClarkBuildWorker.obj
 0001:0001a84c       __unwindfunclet$?validateTaxonomy@ClarkBuildValidator@LocalWorkflow@U2@@ABE_NPBVActor@Workflow@3@AAV?$QList@VWorkflowNotification@U2@@@@@Z$15 1001b84c f   ClarkBuildWorker.obj
 0001:0001a855       __unwindfunclet$?validateTaxonomy@ClarkBuildValidator@LocalWorkflow@U2@@ABE_NPBVActor@Workflow@3@AAV?$QList@VWorkflowNotification@U2@@@@@Z$16 1001b855 f   ClarkBuildWorker.obj
 0001:0001a85e       __unwindfunclet$?validateTaxonomy@ClarkBuildValidator@LocalWorkflow@U2@@ABE_NPBVActor@Workflow@3@AAV?$QList@VWorkflowNotification@U2@@@@@Z$17 1001b85e f   ClarkBuildWorker.obj
 0001:0001a867       __unwindfunclet$?validateTaxonomy@ClarkBuildValidator@LocalWorkflow@U2@@ABE_NPBVActor@Workflow@3@AAV?$QList@VWorkflowNotification@U2@@@@@Z$18 1001b867 f   ClarkBuildWorker.obj
 0001:0001a870       __unwindfunclet$?validateTaxonomy@ClarkBuildValidator@LocalWorkflow@U2@@ABE_NPBVActor@Workflow@3@AAV?$QList@VWorkflowNotification@U2@@@@@Z$19 1001b870 f   ClarkBuildWorker.obj
 0001:0001a879       __unwindfunclet$?validateTaxonomy@ClarkBuildValidator@LocalWorkflow@U2@@ABE_NPBVActor@Workflow@3@AAV?$QList@VWorkflowNotification@U2@@@@@Z$20 1001b879 f   ClarkBuildWorker.obj
 0001:0001a882       __unwindfunclet$?validateTaxonomy@ClarkBuildValidator@LocalWorkflow@U2@@ABE_NPBVActor@Workflow@3@AAV?$QList@VWorkflowNotification@U2@@@@@Z$21 1001b882 f   ClarkBuildWorker.obj
 0001:0001a88b       __unwindfunclet$?validateTaxonomy@ClarkBuildValidator@LocalWorkflow@U2@@ABE_NPBVActor@Workflow@3@AAV?$QList@VWorkflowNotification@U2@@@@@Z$22 1001b88b f   ClarkBuildWorker.obj
 0001:0001a894       __unwindfunclet$?validateTaxonomy@ClarkBuildValidator@LocalWorkflow@U2@@ABE_NPBVActor@Workflow@3@AAV?$QList@VWorkflowNotification@U2@@@@@Z$23 1001b894 f   ClarkBuildWorker.obj
 0001:0001a89d       __unwindfunclet$?validateTaxonomy@ClarkBuildValidator@LocalWorkflow@U2@@ABE_NPBVActor@Workflow@3@AAV?$QList@VWorkflowNotification@U2@@@@@Z$24 1001b89d f   ClarkBuildWorker.obj
 0001:0001a8a6       __unwindfunclet$?validateTaxonomy@ClarkBuildValidator@LocalWorkflow@U2@@ABE_NPBVActor@Workflow@3@AAV?$QList@VWorkflowNotification@U2@@@@@Z$0 1001b8a6 f   ClarkBuildWorker.obj
 0001:0001a8af       __unwindfunclet$?validateTaxonomy@ClarkBuildValidator@LocalWorkflow@U2@@ABE_NPBVActor@Workflow@3@AAV?$QList@VWorkflowNotification@U2@@@@@Z$1 1001b8af f   ClarkBuildWorker.obj
 0001:0001a8b8       __unwindfunclet$?validateTaxonomy@ClarkBuildValidator@LocalWorkflow@U2@@ABE_NPBVActor@Workflow@3@AAV?$QList@VWorkflowNotification@U2@@@@@Z$2 1001b8b8 f   ClarkBuildWorker.obj
 0001:0001a8c1       __ehhandler$?validateTaxonomy@ClarkBuildValidator@LocalWorkflow@U2@@ABE_NPBVActor@Workflow@3@AAV?$QList@VWorkflowNotification@U2@@@@@Z 1001b8c1 f   ClarkBuildWorker.obj
 0001:0001a8e0       __unwindfunclet$??$qRegisterMetaType@V?$QMap@VQString@@I@@@@YAHPBDPAV?$QMap@VQString@@I@@W4DefinedType@?$MetaTypeDefinedHelper@V?$QMap@VQString@@I@@$00@QtPrivate@@@Z$0 1001b8e0 f   ClarkClassifyWorker.obj
 0001:0001a8e9       __ehhandler$??$qRegisterMetaType@V?$QMap@VQString@@I@@@@YAHPBDPAV?$QMap@VQString@@I@@W4DefinedType@?$MetaTypeDefinedHelper@V?$QMap@VQString@@I@@$00@QtPrivate@@@Z 1001b8e9 f   ClarkClassifyWorker.obj
 0001:0001a910       __unwindfunclet$??$qRegisterMetaType@VQAssociativeIterableImpl@QtMetaTypePrivate@@@@YAHPBDPAVQAssociativeIterableImpl@QtMetaTypePrivate@@W4DefinedType@?$MetaTypeDefinedHelper@VQAssociativeIterableImpl@QtMetaTypePrivate@@$00@QtPrivate@@@Z$0 1001b910 f   ClarkClassifyWorker.obj
 0001:0001a919       __ehhandler$??$qRegisterMetaType@VQAssociativeIterableImpl@QtMetaTypePrivate@@@@YAHPBDPAVQAssociativeIterableImpl@QtMetaTypePrivate@@W4DefinedType@?$MetaTypeDefinedHelper@VQAssociativeIterableImpl@QtMetaTypePrivate@@$00@QtPrivate@@@Z 1001b919 f   ClarkClassifyWorker.obj
 0001:0001a940       __unwindfunclet$??0?$QPair@VQString@@V1@@@QAE@ABU0@@Z$0 1001b940 f   ClarkClassifyWorker.obj
 0001:0001a949       __ehhandler$??0?$QPair@VQString@@V1@@@QAE@ABU0@@Z 1001b949 f   ClarkClassifyWorker.obj
 0001:0001a970       __unwindfunclet$??0?$QPair@VQString@@V1@@@QAE@ABVQString@@0@Z$0 1001b970 f   ClarkClassifyWorker.obj
 0001:0001a979       __ehhandler$??0?$QPair@VQString@@V1@@@QAE@ABVQString@@0@Z 1001b979 f   ClarkClassifyWorker.obj
 0001:0001a9a0       __unwindfunclet$??0ClarkClassifySettings@LocalWorkflow@U2@@QAE@ABV012@@Z$0 1001b9a0 f   ClarkClassifyWorker.obj
 0001:0001a9a9       __ehhandler$??0ClarkClassifySettings@LocalWorkflow@U2@@QAE@ABV012@@Z 1001b9a9 f   ClarkClassifyWorker.obj
 0001:0001a9d0       __unwindfunclet$??0ClarkClassifySettings@LocalWorkflow@U2@@QAE@XZ$0 1001b9d0 f   ClarkClassifyWorker.obj
 0001:0001a9d9       __ehhandler$??0ClarkClassifySettings@LocalWorkflow@U2@@QAE@XZ 1001b9d9 f   ClarkClassifyWorker.obj
 0001:0001aa00       __unwindfunclet$??0ClarkClassifyTask@LocalWorkflow@U2@@QAE@ABVClarkClassifySettings@12@ABVQString@@11@Z$0 1001ba00 f   ClarkClassifyWorker.obj
 0001:0001aa09       __unwindfunclet$??0ClarkClassifyTask@LocalWorkflow@U2@@QAE@ABVClarkClassifySettings@12@ABVQString@@11@Z$1 1001ba09 f   ClarkClassifyWorker.obj
 0001:0001aa12       __unwindfunclet$??0ClarkClassifyTask@LocalWorkflow@U2@@QAE@ABVClarkClassifySettings@12@ABVQString@@11@Z$14 1001ba12 f   ClarkClassifyWorker.obj
 0001:0001aa1b       __unwindfunclet$??0ClarkClassifyTask@LocalWorkflow@U2@@QAE@ABVClarkClassifySettings@12@ABVQString@@11@Z$2 1001ba1b f   ClarkClassifyWorker.obj
 0001:0001aa29       __unwindfunclet$??0ClarkClassifyTask@LocalWorkflow@U2@@QAE@ABVClarkClassifySettings@12@ABVQString@@11@Z$3 1001ba29 f   ClarkClassifyWorker.obj
 0001:0001aa38       __unwindfunclet$??0ClarkClassifyTask@LocalWorkflow@U2@@QAE@ABVClarkClassifySettings@12@ABVQString@@11@Z$4 1001ba38 f   ClarkClassifyWorker.obj
 0001:0001aa47       __unwindfunclet$??0ClarkClassifyTask@LocalWorkflow@U2@@QAE@ABVClarkClassifySettings@12@ABVQString@@11@Z$5 1001ba47 f   ClarkClassifyWorker.obj
 0001:0001aa56       __unwindfunclet$??0ClarkClassifyTask@LocalWorkflow@U2@@QAE@ABVClarkClassifySettings@12@ABVQString@@11@Z$6 1001ba56 f   ClarkClassifyWorker.obj
 0001:0001aa64       __unwindfunclet$??0ClarkClassifyTask@LocalWorkflow@U2@@QAE@ABVClarkClassifySettings@12@ABVQString@@11@Z$7 1001ba64 f   ClarkClassifyWorker.obj
 0001:0001aa72       __unwindfunclet$??0ClarkClassifyTask@LocalWorkflow@U2@@QAE@ABVClarkClassifySettings@12@ABVQString@@11@Z$8 1001ba72 f   ClarkClassifyWorker.obj
 0001:0001aa7b       __unwindfunclet$??0ClarkClassifyTask@LocalWorkflow@U2@@QAE@ABVClarkClassifySettings@12@ABVQString@@11@Z$9 1001ba7b f   ClarkClassifyWorker.obj
 0001:0001aa84       __unwindfunclet$??0ClarkClassifyTask@LocalWorkflow@U2@@QAE@ABVClarkClassifySettings@12@ABVQString@@11@Z$10 1001ba84 f   ClarkClassifyWorker.obj
 0001:0001aa8d       __unwindfunclet$??0ClarkClassifyTask@LocalWorkflow@U2@@QAE@ABVClarkClassifySettings@12@ABVQString@@11@Z$11 1001ba8d f   ClarkClassifyWorker.obj
 0001:0001aa96       __unwindfunclet$??0ClarkClassifyTask@LocalWorkflow@U2@@QAE@ABVClarkClassifySettings@12@ABVQString@@11@Z$12 1001ba96 f   ClarkClassifyWorker.obj
 0001:0001aa9f       __unwindfunclet$??0ClarkClassifyTask@LocalWorkflow@U2@@QAE@ABVClarkClassifySettings@12@ABVQString@@11@Z$13 1001ba9f f   ClarkClassifyWorker.obj
 0001:0001aaa8       __ehhandler$??0ClarkClassifyTask@LocalWorkflow@U2@@QAE@ABVClarkClassifySettings@12@ABVQString@@11@Z 1001baa8 f   ClarkClassifyWorker.obj
 0001:0001aad0       __unwindfunclet$??0ClarkClassifyWorker@LocalWorkflow@U2@@QAE@PAVActor@Workflow@2@@Z$0 1001bad0 f   ClarkClassifyWorker.obj
 0001:0001aad9       __unwindfunclet$??0ClarkClassifyWorker@LocalWorkflow@U2@@QAE@PAVActor@Workflow@2@@Z$2 1001bad9 f   ClarkClassifyWorker.obj
 0001:0001aae2       __ehhandler$??0ClarkClassifyWorker@LocalWorkflow@U2@@QAE@PAVActor@Workflow@2@@Z 1001bae2 f   ClarkClassifyWorker.obj
 0001:0001ab00       __unwindfunclet$??0QStringList@@QAE@ABVQString@@@Z$0 1001bb00 f   ClarkClassifyWorker.obj
 0001:0001ab08       __ehhandler$??0QStringList@@QAE@ABVQString@@@Z 1001bb08 f   ClarkClassifyWorker.obj
 0001:0001ab30       __unwindfunclet$??1?$QPair@VQString@@V1@@@QAE@XZ$0 1001bb30 f   ClarkClassifyWorker.obj
 0001:0001ab39       __ehhandler$??1?$QPair@VQString@@V1@@@QAE@XZ 1001bb39 f   ClarkClassifyWorker.obj
 0001:0001ab60       __unwindfunclet$??1ClarkClassifySettings@LocalWorkflow@U2@@QAE@XZ$0 1001bb60 f   ClarkClassifyWorker.obj
 0001:0001ab69       __ehhandler$??1ClarkClassifySettings@LocalWorkflow@U2@@QAE@XZ 1001bb69 f   ClarkClassifyWorker.obj
 0001:0001ab90       __unwindfunclet$??1ClarkClassifyTask@LocalWorkflow@U2@@UAE@XZ$0 1001bb90 f   ClarkClassifyWorker.obj
 0001:0001ab99       __unwindfunclet$??1ClarkClassifyTask@LocalWorkflow@U2@@UAE@XZ$1 1001bb99 f   ClarkClassifyWorker.obj
 0001:0001aba7       __unwindfunclet$??1ClarkClassifyTask@LocalWorkflow@U2@@UAE@XZ$2 1001bba7 f   ClarkClassifyWorker.obj
 0001:0001abb6       __unwindfunclet$??1ClarkClassifyTask@LocalWorkflow@U2@@UAE@XZ$3 1001bbb6 f   ClarkClassifyWorker.obj
 0001:0001abc5       __unwindfunclet$??1ClarkClassifyTask@LocalWorkflow@U2@@UAE@XZ$4 1001bbc5 f   ClarkClassifyWorker.obj
 0001:0001abd4       __unwindfunclet$??1ClarkClassifyTask@LocalWorkflow@U2@@UAE@XZ$6 1001bbd4 f   ClarkClassifyWorker.obj
 0001:0001abdd       __ehhandler$??1ClarkClassifyTask@LocalWorkflow@U2@@UAE@XZ 1001bbdd f   ClarkClassifyWorker.obj
 0001:0001ac00       __unwindfunclet$??1ClarkClassifyWorker@LocalWorkflow@U2@@UAE@XZ$0 1001bc00 f   ClarkClassifyWorker.obj
 0001:0001ac09       __unwindfunclet$??1ClarkClassifyWorker@LocalWorkflow@U2@@UAE@XZ$2 1001bc09 f   ClarkClassifyWorker.obj
 0001:0001ac12       __ehhandler$??1ClarkClassifyWorker@LocalWorkflow@U2@@UAE@XZ 1001bc12 f   ClarkClassifyWorker.obj
 0001:0001ac30       __unwindfunclet$??H@YA?BVQString@@ABV0@0@Z$0 1001bc30 f   ClarkClassifyWorker.obj
 0001:0001ac4a       __ehhandler$??H@YA?BVQString@@ABV0@0@Z 1001bc4a f   ClarkClassifyWorker.obj
 0001:0001ac70       __unwindfunclet$??_G?$QPair@VQString@@V1@@@QAEPAXI@Z$0 1001bc70 f   ClarkClassifyWorker.obj
 0001:0001ac79       __ehhandler$??_G?$QPair@VQString@@V1@@@QAEPAXI@Z 1001bc79 f   ClarkClassifyWorker.obj
 0001:0001aca0       __unwindfunclet$??_GClarkClassifyWorker@LocalWorkflow@U2@@UAEPAXI@Z$0 1001bca0 f   ClarkClassifyWorker.obj
 0001:0001aca9       __unwindfunclet$??_GClarkClassifyWorker@LocalWorkflow@U2@@UAEPAXI@Z$2 1001bca9 f   ClarkClassifyWorker.obj
 0001:0001acb2       __ehhandler$??_GClarkClassifyWorker@LocalWorkflow@U2@@UAEPAXI@Z 1001bcb2 f   ClarkClassifyWorker.obj
 0001:0001acd0       __unwindfunclet$??__EalgoLog@U2@@YAXXZ$0 1001bcd0 f   ClarkClassifyWorker.obj
 0001:0001acd9       __ehhandler$??__EalgoLog@U2@@YAXXZ 1001bcd9 f   ClarkClassifyWorker.obj
 0001:0001ad00       __unwindfunclet$??__EcmdLog@U2@@YAXXZ$0 1001bd00 f   ClarkClassifyWorker.obj
 0001:0001ad09       __ehhandler$??__EcmdLog@U2@@YAXXZ 1001bd09 f   ClarkClassifyWorker.obj
 0001:0001ad30       __unwindfunclet$??__EcoreLog@U2@@YAXXZ$0 1001bd30 f   ClarkClassifyWorker.obj
 0001:0001ad39       __ehhandler$??__EcoreLog@U2@@YAXXZ 1001bd39 f   ClarkClassifyWorker.obj
 0001:0001ad60       __unwindfunclet$??__EioLog@U2@@YAXXZ$0 1001bd60 f   ClarkClassifyWorker.obj
 0001:0001ad69       __ehhandler$??__EioLog@U2@@YAXXZ 1001bd69 f   ClarkClassifyWorker.obj
 0001:0001ad90       __unwindfunclet$??__EperfLog@U2@@YAXXZ$0 1001bd90 f   ClarkClassifyWorker.obj
 0001:0001ad99       __ehhandler$??__EperfLog@U2@@YAXXZ 1001bd99 f   ClarkClassifyWorker.obj
 0001:0001adc0       __unwindfunclet$??__EscriptLog@U2@@YAXXZ$0 1001bdc0 f   ClarkClassifyWorker.obj
 0001:0001adc9       __ehhandler$??__EscriptLog@U2@@YAXXZ 1001bdc9 f   ClarkClassifyWorker.obj
 0001:0001adf0       __unwindfunclet$??__EtaskLog@U2@@YAXXZ$0 1001bdf0 f   ClarkClassifyWorker.obj
 0001:0001adf9       __ehhandler$??__EtaskLog@U2@@YAXXZ 1001bdf9 f   ClarkClassifyWorker.obj
 0001:0001ae20       __unwindfunclet$??__EuiLog@U2@@YAXXZ$0 1001be20 f   ClarkClassifyWorker.obj
 0001:0001ae29       __ehhandler$??__EuiLog@U2@@YAXXZ 1001be29 f   ClarkClassifyWorker.obj
 0001:0001ae50       __unwindfunclet$??__EuserActLog@U2@@YAXXZ$0 1001be50 f   ClarkClassifyWorker.obj
 0001:0001ae59       __ehhandler$??__EuserActLog@U2@@YAXXZ 1001be59 f   ClarkClassifyWorker.obj
 0001:0001ae80       __unwindfunclet$?Construct@?$QMetaTypeFunctionHelper@V?$QMap@VQString@@I@@$00@QtMetaTypePrivate@@SAPAXPAXPBX@Z$0 1001be80 f   ClarkClassifyWorker.obj
 0001:0001ae91       __ehhandler$?Construct@?$QMetaTypeFunctionHelper@V?$QMap@VQString@@I@@$00@QtMetaTypePrivate@@SAPAXPAXPBX@Z 1001be91 f   ClarkClassifyWorker.obj
 0001:0001aeb0       __unwindfunclet$?Create@?$QMetaTypeFunctionHelper@V?$QMap@VQString@@I@@$00@QtMetaTypePrivate@@SAPAXPBX@Z$0 1001beb0 f   ClarkClassifyWorker.obj
 0001:0001aebb       __ehhandler$?Create@?$QMetaTypeFunctionHelper@V?$QMap@VQString@@I@@$00@QtMetaTypePrivate@@SAPAXPBX@Z 1001bebb f   ClarkClassifyWorker.obj
 0001:0001aee0       __ehhandler$?append@?$QList@U?$QPair@VQString@@V1@@@@@QAEXABU?$QPair@VQString@@V1@@@@Z 1001bee0 f   ClarkClassifyWorker.obj
 0001:0001af00       __unwindfunclet$?append@?$QList@VQVariant@@@@QAEXABVQVariant@@@Z$6 1001bf00 f   ClarkClassifyWorker.obj
 0001:0001af0b       __ehhandler$?append@?$QList@VQVariant@@@@QAEXABVQVariant@@@Z 1001bf0b f   ClarkClassifyWorker.obj
 0001:0001af30       __unwindfunclet$?checkRefseqAvailability@ClarkClassifyValidator@LocalWorkflow@U2@@ABE_NPBVActor@Workflow@3@AAV?$QList@VWorkflowNotification@U2@@@@ABVQString@@@Z$0 1001bf30 f   ClarkClassifyWorker.obj
 0001:0001af39       __unwindfunclet$?checkRefseqAvailability@ClarkClassifyValidator@LocalWorkflow@U2@@ABE_NPBVActor@Workflow@3@AAV?$QList@VWorkflowNotification@U2@@@@ABVQString@@@Z$1 1001bf39 f   ClarkClassifyWorker.obj
 0001:0001af42       __unwindfunclet$?checkRefseqAvailability@ClarkClassifyValidator@LocalWorkflow@U2@@ABE_NPBVActor@Workflow@3@AAV?$QList@VWorkflowNotification@U2@@@@ABVQString@@@Z$2 1001bf42 f   ClarkClassifyWorker.obj
 0001:0001af4b       __ehhandler$?checkRefseqAvailability@ClarkClassifyValidator@LocalWorkflow@U2@@ABE_NPBVActor@Workflow@3@AAV?$QList@VWorkflowNotification@U2@@@@ABVQString@@@Z 1001bf4b f   ClarkClassifyWorker.obj
 0001:0001af70       __unwindfunclet$?composeRichDoc@ClarkClassifyPrompter@LocalWorkflow@U2@@MAE?AVQString@@XZ$0 1001bf70 f   ClarkClassifyWorker.obj
 0001:0001af79       __unwindfunclet$?composeRichDoc@ClarkClassifyPrompter@LocalWorkflow@U2@@MAE?AVQString@@XZ$1 1001bf79 f   ClarkClassifyWorker.obj
 0001:0001af82       __unwindfunclet$?composeRichDoc@ClarkClassifyPrompter@LocalWorkflow@U2@@MAE?AVQString@@XZ$2 1001bf82 f   ClarkClassifyWorker.obj
 0001:0001af8b       __unwindfunclet$?composeRichDoc@ClarkClassifyPrompter@LocalWorkflow@U2@@MAE?AVQString@@XZ$3 1001bf8b f   ClarkClassifyWorker.obj
 0001:0001af94       __unwindfunclet$?composeRichDoc@ClarkClassifyPrompter@LocalWorkflow@U2@@MAE?AVQString@@XZ$4 1001bf94 f   ClarkClassifyWorker.obj
 0001:0001af9d       __unwindfunclet$?composeRichDoc@ClarkClassifyPrompter@LocalWorkflow@U2@@MAE?AVQString@@XZ$5 1001bf9d f   ClarkClassifyWorker.obj
 0001:0001afa6       __unwindfunclet$?composeRichDoc@ClarkClassifyPrompter@LocalWorkflow@U2@@MAE?AVQString@@XZ$6 1001bfa6 f   ClarkClassifyWorker.obj
 0001:0001afaf       __unwindfunclet$?composeRichDoc@ClarkClassifyPrompter@LocalWorkflow@U2@@MAE?AVQString@@XZ$7 1001bfaf f   ClarkClassifyWorker.obj
 0001:0001afb8       __unwindfunclet$?composeRichDoc@ClarkClassifyPrompter@LocalWorkflow@U2@@MAE?AVQString@@XZ$8 1001bfb8 f   ClarkClassifyWorker.obj
 0001:0001afc1       __unwindfunclet$?composeRichDoc@ClarkClassifyPrompter@LocalWorkflow@U2@@MAE?AVQString@@XZ$9 1001bfc1 f   ClarkClassifyWorker.obj
 0001:0001afdb       __unwindfunclet$?composeRichDoc@ClarkClassifyPrompter@LocalWorkflow@U2@@MAE?AVQString@@XZ$10 1001bfdb f   ClarkClassifyWorker.obj
 0001:0001afe4       __unwindfunclet$?composeRichDoc@ClarkClassifyPrompter@LocalWorkflow@U2@@MAE?AVQString@@XZ$11 1001bfe4 f   ClarkClassifyWorker.obj
 0001:0001afed       __unwindfunclet$?composeRichDoc@ClarkClassifyPrompter@LocalWorkflow@U2@@MAE?AVQString@@XZ$12 1001bfed f   ClarkClassifyWorker.obj
 0001:0001aff6       __ehhandler$?composeRichDoc@ClarkClassifyPrompter@LocalWorkflow@U2@@MAE?AVQString@@XZ 1001bff6 f   ClarkClassifyWorker.obj
 0001:0001b020       __unwindfunclet$?createDescription@?$PrompterBase@VClarkClassifyPrompter@LocalWorkflow@U2@@@U2@@UAEPAVActorDocument@Workflow@2@PAVActor@42@@Z$0 1001c020 f   ClarkClassifyWorker.obj
 0001:0001b02b       __unwindfunclet$?createDescription@?$PrompterBase@VClarkClassifyPrompter@LocalWorkflow@U2@@@U2@@UAEPAVActorDocument@Workflow@2@PAVActor@42@@Z$3 1001c02b f   ClarkClassifyWorker.obj
 0001:0001b033       __unwindfunclet$?createDescription@?$PrompterBase@VClarkClassifyPrompter@LocalWorkflow@U2@@@U2@@UAEPAVActorDocument@Workflow@2@PAVActor@42@@Z$4 1001c033 f   ClarkClassifyWorker.obj
 0001:0001b03b       __unwindfunclet$?createDescription@?$PrompterBase@VClarkClassifyPrompter@LocalWorkflow@U2@@@U2@@UAEPAVActorDocument@Workflow@2@PAVActor@42@@Z$6 1001c03b f   ClarkClassifyWorker.obj
 0001:0001b043       __unwindfunclet$?createDescription@?$PrompterBase@VClarkClassifyPrompter@LocalWorkflow@U2@@@U2@@UAEPAVActorDocument@Workflow@2@PAVActor@42@@Z$7 1001c043 f   ClarkClassifyWorker.obj
 0001:0001b04b       __ehhandler$?createDescription@?$PrompterBase@VClarkClassifyPrompter@LocalWorkflow@U2@@@U2@@UAEPAVActorDocument@Workflow@2@PAVActor@42@@Z 1001c04b f   ClarkClassifyWorker.obj
 0001:0001b070       __unwindfunclet$?createNode@?$QMapData@VQString@@I@@QAEPAU?$QMapNode@VQString@@I@@ABVQString@@ABIPAU2@_N@Z$4 1001c070 f   ClarkClassifyWorker.obj
 0001:0001b084       __ehhandler$?createNode@?$QMapData@VQString@@I@@QAEPAU?$QMapNode@VQString@@I@@ABVQString@@ABIPAU2@_N@Z 1001c084 f   ClarkClassifyWorker.obj
 0001:0001b0a0       __unwindfunclet$?createNode@?$QMapData@VQString@@V1@@@QAEPAU?$QMapNode@VQString@@V1@@@ABVQString@@0PAU2@_N@Z$4 1001c0a0 f   ClarkClassifyWorker.obj
 0001:0001b0b4       __unwindfunclet$?createNode@?$QMapData@VQString@@V1@@@QAEPAU?$QMapNode@VQString@@V1@@@ABVQString@@0PAU2@_N@Z$5 1001c0b4 f   ClarkClassifyWorker.obj
 0001:0001b0c8       __ehhandler$?createNode@?$QMapData@VQString@@V1@@@QAEPAU?$QMapNode@VQString@@V1@@@ABVQString@@0PAU2@_N@Z 1001c0c8 f   ClarkClassifyWorker.obj
 0001:0001b0f0       __unwindfunclet$?createWorker@ClarkClassifyWorkerFactory@LocalWorkflow@U2@@UAEPAVWorker@Workflow@3@PAVActor@53@@Z$0 1001c0f0 f   ClarkClassifyWorker.obj
 0001:0001b0fb       __ehhandler$?createWorker@ClarkClassifyWorkerFactory@LocalWorkflow@U2@@UAEPAVWorker@Workflow@3@PAVActor@53@@Z 1001c0fb f   ClarkClassifyWorker.obj
 0001:0001b120       __ehhandler$?detach_helper@?$QList@VQString@@@@AAEXH@Z 1001c120 f   ClarkClassifyWorker.obj
 0001:0001b140       __ehhandler$?detach_helper_grow@?$QList@U?$QPair@VQString@@V1@@@@@AAEPAUNode@1@HH@Z 1001c140 f   ClarkClassifyWorker.obj
 0001:0001b160       __ehhandler$?detach_helper_grow@?$QList@VQVariant@@@@AAEPAUNode@1@HH@Z 1001c160 f   ClarkClassifyWorker.obj
 0001:0001b180       __unwindfunclet$?getArguments@ClarkClassifyTask@LocalWorkflow@U2@@AAE?AVQStringList@@XZ$0 1001c180 f   ClarkClassifyWorker.obj
 0001:0001b199       __unwindfunclet$?getArguments@ClarkClassifyTask@LocalWorkflow@U2@@AAE?AVQStringList@@XZ$1 1001c199 f   ClarkClassifyWorker.obj
 0001:0001b1a2       __unwindfunclet$?getArguments@ClarkClassifyTask@LocalWorkflow@U2@@AAE?AVQStringList@@XZ$2 1001c1a2 f   ClarkClassifyWorker.obj
 0001:0001b1ab       __unwindfunclet$?getArguments@ClarkClassifyTask@LocalWorkflow@U2@@AAE?AVQStringList@@XZ$3 1001c1ab f   ClarkClassifyWorker.obj
 0001:0001b1b4       __unwindfunclet$?getArguments@ClarkClassifyTask@LocalWorkflow@U2@@AAE?AVQStringList@@XZ$4 1001c1b4 f   ClarkClassifyWorker.obj
 0001:0001b1bd       __unwindfunclet$?getArguments@ClarkClassifyTask@LocalWorkflow@U2@@AAE?AVQStringList@@XZ$5 1001c1bd f   ClarkClassifyWorker.obj
 0001:0001b1c6       __unwindfunclet$?getArguments@ClarkClassifyTask@LocalWorkflow@U2@@AAE?AVQStringList@@XZ$6 1001c1c6 f   ClarkClassifyWorker.obj
 0001:0001b1cf       __unwindfunclet$?getArguments@ClarkClassifyTask@LocalWorkflow@U2@@AAE?AVQStringList@@XZ$7 1001c1cf f   ClarkClassifyWorker.obj
 0001:0001b1d8       __unwindfunclet$?getArguments@ClarkClassifyTask@LocalWorkflow@U2@@AAE?AVQStringList@@XZ$8 1001c1d8 f   ClarkClassifyWorker.obj
 0001:0001b1e1       __unwindfunclet$?getArguments@ClarkClassifyTask@LocalWorkflow@U2@@AAE?AVQStringList@@XZ$9 1001c1e1 f   ClarkClassifyWorker.obj
 0001:0001b1ea       __unwindfunclet$?getArguments@ClarkClassifyTask@LocalWorkflow@U2@@AAE?AVQStringList@@XZ$10 1001c1ea f   ClarkClassifyWorker.obj
 0001:0001b1f3       __unwindfunclet$?getArguments@ClarkClassifyTask@LocalWorkflow@U2@@AAE?AVQStringList@@XZ$11 1001c1f3 f   ClarkClassifyWorker.obj
 0001:0001b1fc       __unwindfunclet$?getArguments@ClarkClassifyTask@LocalWorkflow@U2@@AAE?AVQStringList@@XZ$12 1001c1fc f   ClarkClassifyWorker.obj
 0001:0001b205       __unwindfunclet$?getArguments@ClarkClassifyTask@LocalWorkflow@U2@@AAE?AVQStringList@@XZ$13 1001c205 f   ClarkClassifyWorker.obj
 0001:0001b20e       __unwindfunclet$?getArguments@ClarkClassifyTask@LocalWorkflow@U2@@AAE?AVQStringList@@XZ$14 1001c20e f   ClarkClassifyWorker.obj
 0001:0001b217       __unwindfunclet$?getArguments@ClarkClassifyTask@LocalWorkflow@U2@@AAE?AVQStringList@@XZ$15 1001c217 f   ClarkClassifyWorker.obj
 0001:0001b220       __unwindfunclet$?getArguments@ClarkClassifyTask@LocalWorkflow@U2@@AAE?AVQStringList@@XZ$16 1001c220 f   ClarkClassifyWorker.obj
 0001:0001b229       __unwindfunclet$?getArguments@ClarkClassifyTask@LocalWorkflow@U2@@AAE?AVQStringList@@XZ$17 1001c229 f   ClarkClassifyWorker.obj
 0001:0001b232       __unwindfunclet$?getArguments@ClarkClassifyTask@LocalWorkflow@U2@@AAE?AVQStringList@@XZ$18 1001c232 f   ClarkClassifyWorker.obj
 0001:0001b23b       __unwindfunclet$?getArguments@ClarkClassifyTask@LocalWorkflow@U2@@AAE?AVQStringList@@XZ$19 1001c23b f   ClarkClassifyWorker.obj
 0001:0001b244       __unwindfunclet$?getArguments@ClarkClassifyTask@LocalWorkflow@U2@@AAE?AVQStringList@@XZ$20 1001c244 f   ClarkClassifyWorker.obj
 0001:0001b24d       __unwindfunclet$?getArguments@ClarkClassifyTask@LocalWorkflow@U2@@AAE?AVQStringList@@XZ$21 1001c24d f   ClarkClassifyWorker.obj
 0001:0001b256       __unwindfunclet$?getArguments@ClarkClassifyTask@LocalWorkflow@U2@@AAE?AVQStringList@@XZ$22 1001c256 f   ClarkClassifyWorker.obj
 0001:0001b25f       __unwindfunclet$?getArguments@ClarkClassifyTask@LocalWorkflow@U2@@AAE?AVQStringList@@XZ$23 1001c25f f   ClarkClassifyWorker.obj
 0001:0001b268       __unwindfunclet$?getArguments@ClarkClassifyTask@LocalWorkflow@U2@@AAE?AVQStringList@@XZ$24 1001c268 f   ClarkClassifyWorker.obj
 0001:0001b271       __unwindfunclet$?getArguments@ClarkClassifyTask@LocalWorkflow@U2@@AAE?AVQStringList@@XZ$25 1001c271 f   ClarkClassifyWorker.obj
 0001:0001b27a       __unwindfunclet$?getArguments@ClarkClassifyTask@LocalWorkflow@U2@@AAE?AVQStringList@@XZ$26 1001c27a f   ClarkClassifyWorker.obj
 0001:0001b283       __unwindfunclet$?getArguments@ClarkClassifyTask@LocalWorkflow@U2@@AAE?AVQStringList@@XZ$27 1001c283 f   ClarkClassifyWorker.obj
 0001:0001b28c       __unwindfunclet$?getArguments@ClarkClassifyTask@LocalWorkflow@U2@@AAE?AVQStringList@@XZ$28 1001c28c f   ClarkClassifyWorker.obj
 0001:0001b295       __ehhandler$?getArguments@ClarkClassifyTask@LocalWorkflow@U2@@AAE?AVQStringList@@XZ 1001c295 f   ClarkClassifyWorker.obj
 0001:0001b2b0       __unwindfunclet$?init@ClarkClassifyWorker@LocalWorkflow@U2@@MAEXXZ$0 1001c2b0 f   ClarkClassifyWorker.obj
 0001:0001b2b9       __unwindfunclet$?init@ClarkClassifyWorker@LocalWorkflow@U2@@MAEXXZ$1 1001c2b9 f   ClarkClassifyWorker.obj
 0001:0001b2c2       __unwindfunclet$?init@ClarkClassifyWorker@LocalWorkflow@U2@@MAEXXZ$2 1001c2c2 f   ClarkClassifyWorker.obj
 0001:0001b2cb       __unwindfunclet$?init@ClarkClassifyWorker@LocalWorkflow@U2@@MAEXXZ$3 1001c2cb f   ClarkClassifyWorker.obj
 0001:0001b2d4       __unwindfunclet$?init@ClarkClassifyWorker@LocalWorkflow@U2@@MAEXXZ$4 1001c2d4 f   ClarkClassifyWorker.obj
 0001:0001b2dd       __unwindfunclet$?init@ClarkClassifyWorker@LocalWorkflow@U2@@MAEXXZ$5 1001c2dd f   ClarkClassifyWorker.obj
 0001:0001b2e6       __unwindfunclet$?init@ClarkClassifyWorker@LocalWorkflow@U2@@MAEXXZ$6 1001c2e6 f   ClarkClassifyWorker.obj
 0001:0001b2ef       __unwindfunclet$?init@ClarkClassifyWorker@LocalWorkflow@U2@@MAEXXZ$7 1001c2ef f   ClarkClassifyWorker.obj
 0001:0001b2f8       __unwindfunclet$?init@ClarkClassifyWorker@LocalWorkflow@U2@@MAEXXZ$8 1001c2f8 f   ClarkClassifyWorker.obj
 0001:0001b301       __unwindfunclet$?init@ClarkClassifyWorker@LocalWorkflow@U2@@MAEXXZ$9 1001c301 f   ClarkClassifyWorker.obj
 0001:0001b30a       __unwindfunclet$?init@ClarkClassifyWorker@LocalWorkflow@U2@@MAEXXZ$10 1001c30a f   ClarkClassifyWorker.obj
 0001:0001b313       __unwindfunclet$?init@ClarkClassifyWorker@LocalWorkflow@U2@@MAEXXZ$11 1001c313 f   ClarkClassifyWorker.obj
 0001:0001b31c       __unwindfunclet$?init@ClarkClassifyWorker@LocalWorkflow@U2@@MAEXXZ$12 1001c31c f   ClarkClassifyWorker.obj
 0001:0001b325       __unwindfunclet$?init@ClarkClassifyWorker@LocalWorkflow@U2@@MAEXXZ$13 1001c325 f   ClarkClassifyWorker.obj
 0001:0001b32e       __unwindfunclet$?init@ClarkClassifyWorker@LocalWorkflow@U2@@MAEXXZ$14 1001c32e f   ClarkClassifyWorker.obj
 0001:0001b337       __unwindfunclet$?init@ClarkClassifyWorker@LocalWorkflow@U2@@MAEXXZ$15 1001c337 f   ClarkClassifyWorker.obj
 0001:0001b340       __unwindfunclet$?init@ClarkClassifyWorker@LocalWorkflow@U2@@MAEXXZ$16 1001c340 f   ClarkClassifyWorker.obj
 0001:0001b349       __unwindfunclet$?init@ClarkClassifyWorker@LocalWorkflow@U2@@MAEXXZ$17 1001c349 f   ClarkClassifyWorker.obj
 0001:0001b352       __unwindfunclet$?init@ClarkClassifyWorker@LocalWorkflow@U2@@MAEXXZ$18 1001c352 f   ClarkClassifyWorker.obj
 0001:0001b35b       __unwindfunclet$?init@ClarkClassifyWorker@LocalWorkflow@U2@@MAEXXZ$19 1001c35b f   ClarkClassifyWorker.obj
 0001:0001b364       __ehhandler$?init@ClarkClassifyWorker@LocalWorkflow@U2@@MAEXXZ 1001c364 f   ClarkClassifyWorker.obj
 0001:0001b380       __unwindfunclet$?init@ClarkClassifyWorkerFactory@LocalWorkflow@U2@@SAXXZ$0 1001c380 f   ClarkClassifyWorker.obj
 0001:0001b38c       __unwindfunclet$?init@ClarkClassifyWorkerFactory@LocalWorkflow@U2@@SAXXZ$1 1001c38c f   ClarkClassifyWorker.obj
 0001:0001b398       __unwindfunclet$?init@ClarkClassifyWorkerFactory@LocalWorkflow@U2@@SAXXZ$2 1001c398 f   ClarkClassifyWorker.obj
 0001:0001b3a4       __unwindfunclet$?init@ClarkClassifyWorkerFactory@LocalWorkflow@U2@@SAXXZ$3 1001c3a4 f   ClarkClassifyWorker.obj
 0001:0001b3ac       __unwindfunclet$?init@ClarkClassifyWorkerFactory@LocalWorkflow@U2@@SAXXZ$4 1001c3ac f   ClarkClassifyWorker.obj
 0001:0001b3b5       __unwindfunclet$?init@ClarkClassifyWorkerFactory@LocalWorkflow@U2@@SAXXZ$5 1001c3b5 f   ClarkClassifyWorker.obj
 0001:0001b3be       __unwindfunclet$?init@ClarkClassifyWorkerFactory@LocalWorkflow@U2@@SAXXZ$6 1001c3be f   ClarkClassifyWorker.obj
 0001:0001b3c7       __unwindfunclet$?init@ClarkClassifyWorkerFactory@LocalWorkflow@U2@@SAXXZ$7 1001c3c7 f   ClarkClassifyWorker.obj
 0001:0001b3d0       __unwindfunclet$?init@ClarkClassifyWorkerFactory@LocalWorkflow@U2@@SAXXZ$8 1001c3d0 f   ClarkClassifyWorker.obj
 0001:0001b3d9       __unwindfunclet$?init@ClarkClassifyWorkerFactory@LocalWorkflow@U2@@SAXXZ$9 1001c3d9 f   ClarkClassifyWorker.obj
 0001:0001b3e5       __unwindfunclet$?init@ClarkClassifyWorkerFactory@LocalWorkflow@U2@@SAXXZ$10 1001c3e5 f   ClarkClassifyWorker.obj
 0001:0001b3ee       __unwindfunclet$?init@ClarkClassifyWorkerFactory@LocalWorkflow@U2@@SAXXZ$11 1001c3ee f   ClarkClassifyWorker.obj
 0001:0001b3f7       __unwindfunclet$?init@ClarkClassifyWorkerFactory@LocalWorkflow@U2@@SAXXZ$12 1001c3f7 f   ClarkClassifyWorker.obj
 0001:0001b403       __unwindfunclet$?init@ClarkClassifyWorkerFactory@LocalWorkflow@U2@@SAXXZ$13 1001c403 f   ClarkClassifyWorker.obj
 0001:0001b40c       __unwindfunclet$?init@ClarkClassifyWorkerFactory@LocalWorkflow@U2@@SAXXZ$14 1001c40c f   ClarkClassifyWorker.obj
 0001:0001b415       __unwindfunclet$?init@ClarkClassifyWorkerFactory@LocalWorkflow@U2@@SAXXZ$15 1001c415 f   ClarkClassifyWorker.obj
 0001:0001b421       __unwindfunclet$?init@ClarkClassifyWorkerFactory@LocalWorkflow@U2@@SAXXZ$16 1001c421 f   ClarkClassifyWorker.obj
 0001:0001b429       __unwindfunclet$?init@ClarkClassifyWorkerFactory@LocalWorkflow@U2@@SAXXZ$17 1001c429 f   ClarkClassifyWorker.obj
 0001:0001b431       __unwindfunclet$?init@ClarkClassifyWorkerFactory@LocalWorkflow@U2@@SAXXZ$18 1001c431 f   ClarkClassifyWorker.obj
 0001:0001b439       __unwindfunclet$?init@ClarkClassifyWorkerFactory@LocalWorkflow@U2@@SAXXZ$19 1001c439 f   ClarkClassifyWorker.obj
 0001:0001b444       __unwindfunclet$?init@ClarkClassifyWorkerFactory@LocalWorkflow@U2@@SAXXZ$20 1001c444 f   ClarkClassifyWorker.obj
 0001:0001b44f       __unwindfunclet$?init@ClarkClassifyWorkerFactory@LocalWorkflow@U2@@SAXXZ$21 1001c44f f   ClarkClassifyWorker.obj
 0001:0001b46c       __unwindfunclet$?init@ClarkClassifyWorkerFactory@LocalWorkflow@U2@@SAXXZ$23 1001c46c f   ClarkClassifyWorker.obj
 0001:0001b474       __unwindfunclet$?init@ClarkClassifyWorkerFactory@LocalWorkflow@U2@@SAXXZ$24 1001c474 f   ClarkClassifyWorker.obj
 0001:0001b47c       __unwindfunclet$?init@ClarkClassifyWorkerFactory@LocalWorkflow@U2@@SAXXZ$25 1001c47c f   ClarkClassifyWorker.obj
 0001:0001b485       __unwindfunclet$?init@ClarkClassifyWorkerFactory@LocalWorkflow@U2@@SAXXZ$26 1001c485 f   ClarkClassifyWorker.obj
 0001:0001b490       __unwindfunclet$?init@ClarkClassifyWorkerFactory@LocalWorkflow@U2@@SAXXZ$27 1001c490 f   ClarkClassifyWorker.obj
 0001:0001b49b       __unwindfunclet$?init@ClarkClassifyWorkerFactory@LocalWorkflow@U2@@SAXXZ$28 1001c49b f   ClarkClassifyWorker.obj
 0001:0001b4b8       __unwindfunclet$?init@ClarkClassifyWorkerFactory@LocalWorkflow@U2@@SAXXZ$30 1001c4b8 f   ClarkClassifyWorker.obj
 0001:0001b4c0       __unwindfunclet$?init@ClarkClassifyWorkerFactory@LocalWorkflow@U2@@SAXXZ$31 1001c4c0 f   ClarkClassifyWorker.obj
 0001:0001b4c9       __unwindfunclet$?init@ClarkClassifyWorkerFactory@LocalWorkflow@U2@@SAXXZ$32 1001c4c9 f   ClarkClassifyWorker.obj
 0001:0001b4d2       __unwindfunclet$?init@ClarkClassifyWorkerFactory@LocalWorkflow@U2@@SAXXZ$33 1001c4d2 f   ClarkClassifyWorker.obj
 0001:0001b4db       __unwindfunclet$?init@ClarkClassifyWorkerFactory@LocalWorkflow@U2@@SAXXZ$34 1001c4db f   ClarkClassifyWorker.obj
 0001:0001b4e4       __unwindfunclet$?init@ClarkClassifyWorkerFactory@LocalWorkflow@U2@@SAXXZ$35 1001c4e4 f   ClarkClassifyWorker.obj
 0001:0001b4ed       __unwindfunclet$?init@ClarkClassifyWorkerFactory@LocalWorkflow@U2@@SAXXZ$36 1001c4ed f   ClarkClassifyWorker.obj
 0001:0001b4f9       __unwindfunclet$?init@ClarkClassifyWorkerFactory@LocalWorkflow@U2@@SAXXZ$37 1001c4f9 f   ClarkClassifyWorker.obj
 0001:0001b502       __unwindfunclet$?init@ClarkClassifyWorkerFactory@LocalWorkflow@U2@@SAXXZ$38 1001c502 f   ClarkClassifyWorker.obj
 0001:0001b50b       __unwindfunclet$?init@ClarkClassifyWorkerFactory@LocalWorkflow@U2@@SAXXZ$39 1001c50b f   ClarkClassifyWorker.obj
 0001:0001b517       __unwindfunclet$?init@ClarkClassifyWorkerFactory@LocalWorkflow@U2@@SAXXZ$40 1001c517 f   ClarkClassifyWorker.obj
 0001:0001b520       __unwindfunclet$?init@ClarkClassifyWorkerFactory@LocalWorkflow@U2@@SAXXZ$41 1001c520 f   ClarkClassifyWorker.obj
 0001:0001b529       __unwindfunclet$?init@ClarkClassifyWorkerFactory@LocalWorkflow@U2@@SAXXZ$42 1001c529 f   ClarkClassifyWorker.obj
 0001:0001b535       __unwindfunclet$?init@ClarkClassifyWorkerFactory@LocalWorkflow@U2@@SAXXZ$43 1001c535 f   ClarkClassifyWorker.obj
 0001:0001b541       __unwindfunclet$?init@ClarkClassifyWorkerFactory@LocalWorkflow@U2@@SAXXZ$44 1001c541 f   ClarkClassifyWorker.obj
 0001:0001b54d       __unwindfunclet$?init@ClarkClassifyWorkerFactory@LocalWorkflow@U2@@SAXXZ$45 1001c54d f   ClarkClassifyWorker.obj
 0001:0001b559       __unwindfunclet$?init@ClarkClassifyWorkerFactory@LocalWorkflow@U2@@SAXXZ$46 1001c559 f   ClarkClassifyWorker.obj
 0001:0001b565       __unwindfunclet$?init@ClarkClassifyWorkerFactory@LocalWorkflow@U2@@SAXXZ$47 1001c565 f   ClarkClassifyWorker.obj
 0001:0001b571       __unwindfunclet$?init@ClarkClassifyWorkerFactory@LocalWorkflow@U2@@SAXXZ$48 1001c571 f   ClarkClassifyWorker.obj
 0001:0001b57d       __unwindfunclet$?init@ClarkClassifyWorkerFactory@LocalWorkflow@U2@@SAXXZ$49 1001c57d f   ClarkClassifyWorker.obj
 0001:0001b589       __unwindfunclet$?init@ClarkClassifyWorkerFactory@LocalWorkflow@U2@@SAXXZ$50 1001c589 f   ClarkClassifyWorker.obj
 0001:0001b595       __unwindfunclet$?init@ClarkClassifyWorkerFactory@LocalWorkflow@U2@@SAXXZ$51 1001c595 f   ClarkClassifyWorker.obj
 0001:0001b5a1       __unwindfunclet$?init@ClarkClassifyWorkerFactory@LocalWorkflow@U2@@SAXXZ$52 1001c5a1 f   ClarkClassifyWorker.obj
 0001:0001b5ad       __unwindfunclet$?init@ClarkClassifyWorkerFactory@LocalWorkflow@U2@@SAXXZ$53 1001c5ad f   ClarkClassifyWorker.obj
 0001:0001b5b9       __unwindfunclet$?init@ClarkClassifyWorkerFactory@LocalWorkflow@U2@@SAXXZ$54 1001c5b9 f   ClarkClassifyWorker.obj
 0001:0001b5c5       __unwindfunclet$?init@ClarkClassifyWorkerFactory@LocalWorkflow@U2@@SAXXZ$55 1001c5c5 f   ClarkClassifyWorker.obj
 0001:0001b5d1       __unwindfunclet$?init@ClarkClassifyWorkerFactory@LocalWorkflow@U2@@SAXXZ$56 1001c5d1 f   ClarkClassifyWorker.obj
 0001:0001b5dd       __unwindfunclet$?init@ClarkClassifyWorkerFactory@LocalWorkflow@U2@@SAXXZ$57 1001c5dd f   ClarkClassifyWorker.obj
 0001:0001b5e9       __unwindfunclet$?init@ClarkClassifyWorkerFactory@LocalWorkflow@U2@@SAXXZ$58 1001c5e9 f   ClarkClassifyWorker.obj
 0001:0001b5f5       __unwindfunclet$?init@ClarkClassifyWorkerFactory@LocalWorkflow@U2@@SAXXZ$59 1001c5f5 f   ClarkClassifyWorker.obj
 0001:0001b601       __unwindfunclet$?init@ClarkClassifyWorkerFactory@LocalWorkflow@U2@@SAXXZ$60 1001c601 f   ClarkClassifyWorker.obj
 0001:0001b60d       __unwindfunclet$?init@ClarkClassifyWorkerFactory@LocalWorkflow@U2@@SAXXZ$61 1001c60d f   ClarkClassifyWorker.obj
 0001:0001b619       __unwindfunclet$?init@ClarkClassifyWorkerFactory@LocalWorkflow@U2@@SAXXZ$62 1001c619 f   ClarkClassifyWorker.obj
 0001:0001b625       __unwindfunclet$?init@ClarkClassifyWorkerFactory@LocalWorkflow@U2@@SAXXZ$63 1001c625 f   ClarkClassifyWorker.obj
 0001:0001b631       __unwindfunclet$?init@ClarkClassifyWorkerFactory@LocalWorkflow@U2@@SAXXZ$64 1001c631 f   ClarkClassifyWorker.obj
 0001:0001b63d       __unwindfunclet$?init@ClarkClassifyWorkerFactory@LocalWorkflow@U2@@SAXXZ$65 1001c63d f   ClarkClassifyWorker.obj
 0001:0001b649       __unwindfunclet$?init@ClarkClassifyWorkerFactory@LocalWorkflow@U2@@SAXXZ$66 1001c649 f   ClarkClassifyWorker.obj
 0001:0001b655       __unwindfunclet$?init@ClarkClassifyWorkerFactory@LocalWorkflow@U2@@SAXXZ$67 1001c655 f   ClarkClassifyWorker.obj
 0001:0001b65e       __unwindfunclet$?init@ClarkClassifyWorkerFactory@LocalWorkflow@U2@@SAXXZ$68 1001c65e f   ClarkClassifyWorker.obj
 0001:0001b66a       __unwindfunclet$?init@ClarkClassifyWorkerFactory@LocalWorkflow@U2@@SAXXZ$69 1001c66a f   ClarkClassifyWorker.obj
 0001:0001b675       __unwindfunclet$?init@ClarkClassifyWorkerFactory@LocalWorkflow@U2@@SAXXZ$70 1001c675 f   ClarkClassifyWorker.obj
 0001:0001b68f       __unwindfunclet$?init@ClarkClassifyWorkerFactory@LocalWorkflow@U2@@SAXXZ$72 1001c68f f   ClarkClassifyWorker.obj
 0001:0001b69a       __unwindfunclet$?init@ClarkClassifyWorkerFactory@LocalWorkflow@U2@@SAXXZ$73 1001c69a f   ClarkClassifyWorker.obj
 0001:0001b6b4       __unwindfunclet$?init@ClarkClassifyWorkerFactory@LocalWorkflow@U2@@SAXXZ$74 1001c6b4 f   ClarkClassifyWorker.obj
 0001:0001b6cd       __unwindfunclet$?init@ClarkClassifyWorkerFactory@LocalWorkflow@U2@@SAXXZ$75 1001c6cd f   ClarkClassifyWorker.obj
 0001:0001b6d8       __unwindfunclet$?init@ClarkClassifyWorkerFactory@LocalWorkflow@U2@@SAXXZ$76 1001c6d8 f   ClarkClassifyWorker.obj
 0001:0001b6f2       __unwindfunclet$?init@ClarkClassifyWorkerFactory@LocalWorkflow@U2@@SAXXZ$78 1001c6f2 f   ClarkClassifyWorker.obj
 0001:0001b6fb       __unwindfunclet$?init@ClarkClassifyWorkerFactory@LocalWorkflow@U2@@SAXXZ$79 1001c6fb f   ClarkClassifyWorker.obj
 0001:0001b704       __unwindfunclet$?init@ClarkClassifyWorkerFactory@LocalWorkflow@U2@@SAXXZ$80 1001c704 f   ClarkClassifyWorker.obj
 0001:0001b70d       __unwindfunclet$?init@ClarkClassifyWorkerFactory@LocalWorkflow@U2@@SAXXZ$81 1001c70d f   ClarkClassifyWorker.obj
 0001:0001b718       __unwindfunclet$?init@ClarkClassifyWorkerFactory@LocalWorkflow@U2@@SAXXZ$82 1001c718 f   ClarkClassifyWorker.obj
 0001:0001b732       __unwindfunclet$?init@ClarkClassifyWorkerFactory@LocalWorkflow@U2@@SAXXZ$84 1001c732 f   ClarkClassifyWorker.obj
 0001:0001b73d       __unwindfunclet$?init@ClarkClassifyWorkerFactory@LocalWorkflow@U2@@SAXXZ$85 1001c73d f   ClarkClassifyWorker.obj
 0001:0001b75c       __unwindfunclet$?init@ClarkClassifyWorkerFactory@LocalWorkflow@U2@@SAXXZ$87 1001c75c f   ClarkClassifyWorker.obj
 0001:0001b767       __unwindfunclet$?init@ClarkClassifyWorkerFactory@LocalWorkflow@U2@@SAXXZ$88 1001c767 f   ClarkClassifyWorker.obj
 0001:0001b786       __unwindfunclet$?init@ClarkClassifyWorkerFactory@LocalWorkflow@U2@@SAXXZ$89 1001c786 f   ClarkClassifyWorker.obj
 0001:0001b791       __unwindfunclet$?init@ClarkClassifyWorkerFactory@LocalWorkflow@U2@@SAXXZ$90 1001c791 f   ClarkClassifyWorker.obj
 0001:0001b7b0       __unwindfunclet$?init@ClarkClassifyWorkerFactory@LocalWorkflow@U2@@SAXXZ$92 1001c7b0 f   ClarkClassifyWorker.obj
 0001:0001b7bb       __unwindfunclet$?init@ClarkClassifyWorkerFactory@LocalWorkflow@U2@@SAXXZ$93 1001c7bb f   ClarkClassifyWorker.obj
 0001:0001b7da       __unwindfunclet$?init@ClarkClassifyWorkerFactory@LocalWorkflow@U2@@SAXXZ$95 1001c7da f   ClarkClassifyWorker.obj
 0001:0001b7e5       __unwindfunclet$?init@ClarkClassifyWorkerFactory@LocalWorkflow@U2@@SAXXZ$96 1001c7e5 f   ClarkClassifyWorker.obj
 0001:0001b804       __unwindfunclet$?init@ClarkClassifyWorkerFactory@LocalWorkflow@U2@@SAXXZ$98 1001c804 f   ClarkClassifyWorker.obj
 0001:0001b80f       __unwindfunclet$?init@ClarkClassifyWorkerFactory@LocalWorkflow@U2@@SAXXZ$99 1001c80f f   ClarkClassifyWorker.obj
 0001:0001b82e       __unwindfunclet$?init@ClarkClassifyWorkerFactory@LocalWorkflow@U2@@SAXXZ$100 1001c82e f   ClarkClassifyWorker.obj
 0001:0001b839       __unwindfunclet$?init@ClarkClassifyWorkerFactory@LocalWorkflow@U2@@SAXXZ$101 1001c839 f   ClarkClassifyWorker.obj
 0001:0001b858       __unwindfunclet$?init@ClarkClassifyWorkerFactory@LocalWorkflow@U2@@SAXXZ$103 1001c858 f   ClarkClassifyWorker.obj
 0001:0001b863       __unwindfunclet$?init@ClarkClassifyWorkerFactory@LocalWorkflow@U2@@SAXXZ$104 1001c863 f   ClarkClassifyWorker.obj
 0001:0001b882       __unwindfunclet$?init@ClarkClassifyWorkerFactory@LocalWorkflow@U2@@SAXXZ$105 1001c882 f   ClarkClassifyWorker.obj
 0001:0001b88d       __unwindfunclet$?init@ClarkClassifyWorkerFactory@LocalWorkflow@U2@@SAXXZ$106 1001c88d f   ClarkClassifyWorker.obj
 0001:0001b8ac       __unwindfunclet$?init@ClarkClassifyWorkerFactory@LocalWorkflow@U2@@SAXXZ$108 1001c8ac f   ClarkClassifyWorker.obj
 0001:0001b8b7       __unwindfunclet$?init@ClarkClassifyWorkerFactory@LocalWorkflow@U2@@SAXXZ$109 1001c8b7 f   ClarkClassifyWorker.obj
 0001:0001b8d6       __unwindfunclet$?init@ClarkClassifyWorkerFactory@LocalWorkflow@U2@@SAXXZ$110 1001c8d6 f   ClarkClassifyWorker.obj
 0001:0001b8e1       __unwindfunclet$?init@ClarkClassifyWorkerFactory@LocalWorkflow@U2@@SAXXZ$111 1001c8e1 f   ClarkClassifyWorker.obj
 0001:0001b900       __unwindfunclet$?init@ClarkClassifyWorkerFactory@LocalWorkflow@U2@@SAXXZ$113 1001c900 f   ClarkClassifyWorker.obj
 0001:0001b90b       __unwindfunclet$?init@ClarkClassifyWorkerFactory@LocalWorkflow@U2@@SAXXZ$114 1001c90b f   ClarkClassifyWorker.obj
 0001:0001b92a       __unwindfunclet$?init@ClarkClassifyWorkerFactory@LocalWorkflow@U2@@SAXXZ$116 1001c92a f   ClarkClassifyWorker.obj
 0001:0001b935       __unwindfunclet$?init@ClarkClassifyWorkerFactory@LocalWorkflow@U2@@SAXXZ$117 1001c935 f   ClarkClassifyWorker.obj
 0001:0001b954       __unwindfunclet$?init@ClarkClassifyWorkerFactory@LocalWorkflow@U2@@SAXXZ$119 1001c954 f   ClarkClassifyWorker.obj
 0001:0001b95f       __unwindfunclet$?init@ClarkClassifyWorkerFactory@LocalWorkflow@U2@@SAXXZ$120 1001c95f f   ClarkClassifyWorker.obj
 0001:0001b97e       __unwindfunclet$?init@ClarkClassifyWorkerFactory@LocalWorkflow@U2@@SAXXZ$122 1001c97e f   ClarkClassifyWorker.obj
 0001:0001b986       __unwindfunclet$?init@ClarkClassifyWorkerFactory@LocalWorkflow@U2@@SAXXZ$123 1001c986 f   ClarkClassifyWorker.obj
 0001:0001b98e       __unwindfunclet$?init@ClarkClassifyWorkerFactory@LocalWorkflow@U2@@SAXXZ$124 1001c98e f   ClarkClassifyWorker.obj
 0001:0001b997       __unwindfunclet$?init@ClarkClassifyWorkerFactory@LocalWorkflow@U2@@SAXXZ$125 1001c997 f   ClarkClassifyWorker.obj
 0001:0001b9a0       __unwindfunclet$?init@ClarkClassifyWorkerFactory@LocalWorkflow@U2@@SAXXZ$126 1001c9a0 f   ClarkClassifyWorker.obj
 0001:0001b9ac       __unwindfunclet$?init@ClarkClassifyWorkerFactory@LocalWorkflow@U2@@SAXXZ$127 1001c9ac f   ClarkClassifyWorker.obj
 0001:0001b9b5       __unwindfunclet$?init@ClarkClassifyWorkerFactory@LocalWorkflow@U2@@SAXXZ$128 1001c9b5 f   ClarkClassifyWorker.obj
 0001:0001b9c0       __unwindfunclet$?init@ClarkClassifyWorkerFactory@LocalWorkflow@U2@@SAXXZ$129 1001c9c0 f   ClarkClassifyWorker.obj
 0001:0001b9c8       __unwindfunclet$?init@ClarkClassifyWorkerFactory@LocalWorkflow@U2@@SAXXZ$130 1001c9c8 f   ClarkClassifyWorker.obj
 0001:0001b9d1       __unwindfunclet$?init@ClarkClassifyWorkerFactory@LocalWorkflow@U2@@SAXXZ$131 1001c9d1 f   ClarkClassifyWorker.obj
 0001:0001b9da       __unwindfunclet$?init@ClarkClassifyWorkerFactory@LocalWorkflow@U2@@SAXXZ$132 1001c9da f   ClarkClassifyWorker.obj
 0001:0001b9e6       __unwindfunclet$?init@ClarkClassifyWorkerFactory@LocalWorkflow@U2@@SAXXZ$133 1001c9e6 f   ClarkClassifyWorker.obj
 0001:0001b9ef       __unwindfunclet$?init@ClarkClassifyWorkerFactory@LocalWorkflow@U2@@SAXXZ$134 1001c9ef f   ClarkClassifyWorker.obj
 0001:0001b9fa       __unwindfunclet$?init@ClarkClassifyWorkerFactory@LocalWorkflow@U2@@SAXXZ$135 1001c9fa f   ClarkClassifyWorker.obj
 0001:0001ba06       __unwindfunclet$?init@ClarkClassifyWorkerFactory@LocalWorkflow@U2@@SAXXZ$136 1001ca06 f   ClarkClassifyWorker.obj
 0001:0001ba0f       __unwindfunclet$?init@ClarkClassifyWorkerFactory@LocalWorkflow@U2@@SAXXZ$137 1001ca0f f   ClarkClassifyWorker.obj
 0001:0001ba18       __unwindfunclet$?init@ClarkClassifyWorkerFactory@LocalWorkflow@U2@@SAXXZ$138 1001ca18 f   ClarkClassifyWorker.obj
 0001:0001ba21       __unwindfunclet$?init@ClarkClassifyWorkerFactory@LocalWorkflow@U2@@SAXXZ$139 1001ca21 f   ClarkClassifyWorker.obj
 0001:0001ba29       __unwindfunclet$?init@ClarkClassifyWorkerFactory@LocalWorkflow@U2@@SAXXZ$196 1001ca29 f   ClarkClassifyWorker.obj
 0001:0001ba31       __unwindfunclet$?init@ClarkClassifyWorkerFactory@LocalWorkflow@U2@@SAXXZ$140 1001ca31 f   ClarkClassifyWorker.obj
 0001:0001ba39       __unwindfunclet$?init@ClarkClassifyWorkerFactory@LocalWorkflow@U2@@SAXXZ$141 1001ca39 f   ClarkClassifyWorker.obj
 0001:0001ba42       __unwindfunclet$?init@ClarkClassifyWorkerFactory@LocalWorkflow@U2@@SAXXZ$142 1001ca42 f   ClarkClassifyWorker.obj
 0001:0001ba4b       __unwindfunclet$?init@ClarkClassifyWorkerFactory@LocalWorkflow@U2@@SAXXZ$143 1001ca4b f   ClarkClassifyWorker.obj
 0001:0001ba56       __unwindfunclet$?init@ClarkClassifyWorkerFactory@LocalWorkflow@U2@@SAXXZ$144 1001ca56 f   ClarkClassifyWorker.obj
 0001:0001ba75       __unwindfunclet$?init@ClarkClassifyWorkerFactory@LocalWorkflow@U2@@SAXXZ$145 1001ca75 f   ClarkClassifyWorker.obj
 0001:0001ba7d       __unwindfunclet$?init@ClarkClassifyWorkerFactory@LocalWorkflow@U2@@SAXXZ$146 1001ca7d f   ClarkClassifyWorker.obj
 0001:0001ba86       __unwindfunclet$?init@ClarkClassifyWorkerFactory@LocalWorkflow@U2@@SAXXZ$147 1001ca86 f   ClarkClassifyWorker.obj
 0001:0001ba8f       __unwindfunclet$?init@ClarkClassifyWorkerFactory@LocalWorkflow@U2@@SAXXZ$148 1001ca8f f   ClarkClassifyWorker.obj
 0001:0001ba98       __unwindfunclet$?init@ClarkClassifyWorkerFactory@LocalWorkflow@U2@@SAXXZ$149 1001ca98 f   ClarkClassifyWorker.obj
 0001:0001baa1       __unwindfunclet$?init@ClarkClassifyWorkerFactory@LocalWorkflow@U2@@SAXXZ$150 1001caa1 f   ClarkClassifyWorker.obj
 0001:0001baac       __unwindfunclet$?init@ClarkClassifyWorkerFactory@LocalWorkflow@U2@@SAXXZ$151 1001caac f   ClarkClassifyWorker.obj
 0001:0001bab4       __unwindfunclet$?init@ClarkClassifyWorkerFactory@LocalWorkflow@U2@@SAXXZ$152 1001cab4 f   ClarkClassifyWorker.obj
 0001:0001babd       __unwindfunclet$?init@ClarkClassifyWorkerFactory@LocalWorkflow@U2@@SAXXZ$153 1001cabd f   ClarkClassifyWorker.obj
 0001:0001bac6       __unwindfunclet$?init@ClarkClassifyWorkerFactory@LocalWorkflow@U2@@SAXXZ$154 1001cac6 f   ClarkClassifyWorker.obj
 0001:0001bacf       __unwindfunclet$?init@ClarkClassifyWorkerFactory@LocalWorkflow@U2@@SAXXZ$155 1001cacf f   ClarkClassifyWorker.obj
 0001:0001bad8       __unwindfunclet$?init@ClarkClassifyWorkerFactory@LocalWorkflow@U2@@SAXXZ$156 1001cad8 f   ClarkClassifyWorker.obj
 0001:0001bae3       __unwindfunclet$?init@ClarkClassifyWorkerFactory@LocalWorkflow@U2@@SAXXZ$157 1001cae3 f   ClarkClassifyWorker.obj
 0001:0001baeb       __unwindfunclet$?init@ClarkClassifyWorkerFactory@LocalWorkflow@U2@@SAXXZ$158 1001caeb f   ClarkClassifyWorker.obj
 0001:0001baf4       __unwindfunclet$?init@ClarkClassifyWorkerFactory@LocalWorkflow@U2@@SAXXZ$159 1001caf4 f   ClarkClassifyWorker.obj
 0001:0001bafd       __unwindfunclet$?init@ClarkClassifyWorkerFactory@LocalWorkflow@U2@@SAXXZ$160 1001cafd f   ClarkClassifyWorker.obj
 0001:0001bb09       __unwindfunclet$?init@ClarkClassifyWorkerFactory@LocalWorkflow@U2@@SAXXZ$161 1001cb09 f   ClarkClassifyWorker.obj
 0001:0001bb12       __unwindfunclet$?init@ClarkClassifyWorkerFactory@LocalWorkflow@U2@@SAXXZ$162 1001cb12 f   ClarkClassifyWorker.obj
 0001:0001bb1e       __unwindfunclet$?init@ClarkClassifyWorkerFactory@LocalWorkflow@U2@@SAXXZ$163 1001cb1e f   ClarkClassifyWorker.obj
 0001:0001bb27       __unwindfunclet$?init@ClarkClassifyWorkerFactory@LocalWorkflow@U2@@SAXXZ$164 1001cb27 f   ClarkClassifyWorker.obj
 0001:0001bb32       __unwindfunclet$?init@ClarkClassifyWorkerFactory@LocalWorkflow@U2@@SAXXZ$165 1001cb32 f   ClarkClassifyWorker.obj
 0001:0001bb3a       __unwindfunclet$?init@ClarkClassifyWorkerFactory@LocalWorkflow@U2@@SAXXZ$166 1001cb3a f   ClarkClassifyWorker.obj
 0001:0001bb43       __unwindfunclet$?init@ClarkClassifyWorkerFactory@LocalWorkflow@U2@@SAXXZ$167 1001cb43 f   ClarkClassifyWorker.obj
 0001:0001bb4c       __unwindfunclet$?init@ClarkClassifyWorkerFactory@LocalWorkflow@U2@@SAXXZ$168 1001cb4c f   ClarkClassifyWorker.obj
 0001:0001bb55       __unwindfunclet$?init@ClarkClassifyWorkerFactory@LocalWorkflow@U2@@SAXXZ$169 1001cb55 f   ClarkClassifyWorker.obj
 0001:0001bb5e       __unwindfunclet$?init@ClarkClassifyWorkerFactory@LocalWorkflow@U2@@SAXXZ$170 1001cb5e f   ClarkClassifyWorker.obj
 0001:0001bb69       __unwindfunclet$?init@ClarkClassifyWorkerFactory@LocalWorkflow@U2@@SAXXZ$171 1001cb69 f   ClarkClassifyWorker.obj
 0001:0001bb71       __unwindfunclet$?init@ClarkClassifyWorkerFactory@LocalWorkflow@U2@@SAXXZ$172 1001cb71 f   ClarkClassifyWorker.obj
 0001:0001bb7a       __unwindfunclet$?init@ClarkClassifyWorkerFactory@LocalWorkflow@U2@@SAXXZ$173 1001cb7a f   ClarkClassifyWorker.obj
 0001:0001bb83       __unwindfunclet$?init@ClarkClassifyWorkerFactory@LocalWorkflow@U2@@SAXXZ$174 1001cb83 f   ClarkClassifyWorker.obj
 0001:0001bb8c       __unwindfunclet$?init@ClarkClassifyWorkerFactory@LocalWorkflow@U2@@SAXXZ$175 1001cb8c f   ClarkClassifyWorker.obj
 0001:0001bb95       __unwindfunclet$?init@ClarkClassifyWorkerFactory@LocalWorkflow@U2@@SAXXZ$176 1001cb95 f   ClarkClassifyWorker.obj
 0001:0001bba0       __unwindfunclet$?init@ClarkClassifyWorkerFactory@LocalWorkflow@U2@@SAXXZ$177 1001cba0 f   ClarkClassifyWorker.obj
 0001:0001bba8       __unwindfunclet$?init@ClarkClassifyWorkerFactory@LocalWorkflow@U2@@SAXXZ$178 1001cba8 f   ClarkClassifyWorker.obj
 0001:0001bbb1       __unwindfunclet$?init@ClarkClassifyWorkerFactory@LocalWorkflow@U2@@SAXXZ$179 1001cbb1 f   ClarkClassifyWorker.obj
 0001:0001bbba       __unwindfunclet$?init@ClarkClassifyWorkerFactory@LocalWorkflow@U2@@SAXXZ$180 1001cbba f   ClarkClassifyWorker.obj
 0001:0001bbc3       __unwindfunclet$?init@ClarkClassifyWorkerFactory@LocalWorkflow@U2@@SAXXZ$181 1001cbc3 f   ClarkClassifyWorker.obj
 0001:0001bbcc       __unwindfunclet$?init@ClarkClassifyWorkerFactory@LocalWorkflow@U2@@SAXXZ$182 1001cbcc f   ClarkClassifyWorker.obj
 0001:0001bbd7       __unwindfunclet$?init@ClarkClassifyWorkerFactory@LocalWorkflow@U2@@SAXXZ$183 1001cbd7 f   ClarkClassifyWorker.obj
 0001:0001bbdf       __unwindfunclet$?init@ClarkClassifyWorkerFactory@LocalWorkflow@U2@@SAXXZ$199 1001cbdf f   ClarkClassifyWorker.obj
 0001:0001bbe8       __unwindfunclet$?init@ClarkClassifyWorkerFactory@LocalWorkflow@U2@@SAXXZ$184 1001cbe8 f   ClarkClassifyWorker.obj
 0001:0001bbf0       __unwindfunclet$?init@ClarkClassifyWorkerFactory@LocalWorkflow@U2@@SAXXZ$201 1001cbf0 f   ClarkClassifyWorker.obj
 0001:0001bbf9       __unwindfunclet$?init@ClarkClassifyWorkerFactory@LocalWorkflow@U2@@SAXXZ$203 1001cbf9 f   ClarkClassifyWorker.obj
 0001:0001bc05       __unwindfunclet$?init@ClarkClassifyWorkerFactory@LocalWorkflow@U2@@SAXXZ$185 1001cc05 f   ClarkClassifyWorker.obj
 0001:0001bc10       __unwindfunclet$?init@ClarkClassifyWorkerFactory@LocalWorkflow@U2@@SAXXZ$205 1001cc10 f   ClarkClassifyWorker.obj
 0001:0001bc1c       __unwindfunclet$?init@ClarkClassifyWorkerFactory@LocalWorkflow@U2@@SAXXZ$186 1001cc1c f   ClarkClassifyWorker.obj
 0001:0001bc27       __unwindfunclet$?init@ClarkClassifyWorkerFactory@LocalWorkflow@U2@@SAXXZ$187 1001cc27 f   ClarkClassifyWorker.obj
 0001:0001bc46       __unwindfunclet$?init@ClarkClassifyWorkerFactory@LocalWorkflow@U2@@SAXXZ$188 1001cc46 f   ClarkClassifyWorker.obj
 0001:0001bc51       __unwindfunclet$?init@ClarkClassifyWorkerFactory@LocalWorkflow@U2@@SAXXZ$189 1001cc51 f   ClarkClassifyWorker.obj
 0001:0001bc5c       __unwindfunclet$?init@ClarkClassifyWorkerFactory@LocalWorkflow@U2@@SAXXZ$190 1001cc5c f   ClarkClassifyWorker.obj
 0001:0001bc67       __unwindfunclet$?init@ClarkClassifyWorkerFactory@LocalWorkflow@U2@@SAXXZ$191 1001cc67 f   ClarkClassifyWorker.obj
 0001:0001bc72       __unwindfunclet$?init@ClarkClassifyWorkerFactory@LocalWorkflow@U2@@SAXXZ$192 1001cc72 f   ClarkClassifyWorker.obj
 0001:0001bc7b       __unwindfunclet$?init@ClarkClassifyWorkerFactory@LocalWorkflow@U2@@SAXXZ$193 1001cc7b f   ClarkClassifyWorker.obj
 0001:0001bc84       __unwindfunclet$?init@ClarkClassifyWorkerFactory@LocalWorkflow@U2@@SAXXZ$194 1001cc84 f   ClarkClassifyWorker.obj
 0001:0001bc8d       __unwindfunclet$?init@ClarkClassifyWorkerFactory@LocalWorkflow@U2@@SAXXZ$195 1001cc8d f   ClarkClassifyWorker.obj
 0001:0001bc98       __ehhandler$?init@ClarkClassifyWorkerFactory@LocalWorkflow@U2@@SAXXZ 1001cc98 f   ClarkClassifyWorker.obj
 0001:0001bcc0       __unwindfunclet$?initWellKnownErrors@ClarkLogParser@LocalWorkflow@U2@@CA?AV?$QMap@VQString@@V1@@@XZ$0 1001ccc0 f   ClarkClassifyWorker.obj
 0001:0001bcd9       __unwindfunclet$?initWellKnownErrors@ClarkLogParser@LocalWorkflow@U2@@CA?AV?$QMap@VQString@@V1@@@XZ$1 1001ccd9 f   ClarkClassifyWorker.obj
 0001:0001bce2       __unwindfunclet$?initWellKnownErrors@ClarkLogParser@LocalWorkflow@U2@@CA?AV?$QMap@VQString@@V1@@@XZ$2 1001cce2 f   ClarkClassifyWorker.obj
 0001:0001bceb       __unwindfunclet$?initWellKnownErrors@ClarkLogParser@LocalWorkflow@U2@@CA?AV?$QMap@VQString@@V1@@@XZ$3 1001cceb f   ClarkClassifyWorker.obj
 0001:0001bcf4       __unwindfunclet$?initWellKnownErrors@ClarkLogParser@LocalWorkflow@U2@@CA?AV?$QMap@VQString@@V1@@@XZ$4 1001ccf4 f   ClarkClassifyWorker.obj
 0001:0001bcfd       __ehhandler$?initWellKnownErrors@ClarkLogParser@LocalWorkflow@U2@@CA?AV?$QMap@VQString@@V1@@@XZ 1001ccfd f   ClarkClassifyWorker.obj
 0001:0001bd20       __unwindfunclet$?isDatabaseAlreadyBuilt@ClarkClassifyValidator@LocalWorkflow@U2@@ABE_NPBVActor@Workflow@3@@Z$0 1001cd20 f   ClarkClassifyWorker.obj
 0001:0001bd29       __unwindfunclet$?isDatabaseAlreadyBuilt@ClarkClassifyValidator@LocalWorkflow@U2@@ABE_NPBVActor@Workflow@3@@Z$1 1001cd29 f   ClarkClassifyWorker.obj
 0001:0001bd31       __unwindfunclet$?isDatabaseAlreadyBuilt@ClarkClassifyValidator@LocalWorkflow@U2@@ABE_NPBVActor@Workflow@3@@Z$2 1001cd31 f   ClarkClassifyWorker.obj
 0001:0001bd3a       __unwindfunclet$?isDatabaseAlreadyBuilt@ClarkClassifyValidator@LocalWorkflow@U2@@ABE_NPBVActor@Workflow@3@@Z$3 1001cd3a f   ClarkClassifyWorker.obj
 0001:0001bd43       __unwindfunclet$?isDatabaseAlreadyBuilt@ClarkClassifyValidator@LocalWorkflow@U2@@ABE_NPBVActor@Workflow@3@@Z$4 1001cd43 f   ClarkClassifyWorker.obj
 0001:0001bd4c       __unwindfunclet$?isDatabaseAlreadyBuilt@ClarkClassifyValidator@LocalWorkflow@U2@@ABE_NPBVActor@Workflow@3@@Z$5 1001cd4c f   ClarkClassifyWorker.obj
 0001:0001bd55       __unwindfunclet$?isDatabaseAlreadyBuilt@ClarkClassifyValidator@LocalWorkflow@U2@@ABE_NPBVActor@Workflow@3@@Z$6 1001cd55 f   ClarkClassifyWorker.obj
 0001:0001bd5e       __unwindfunclet$?isDatabaseAlreadyBuilt@ClarkClassifyValidator@LocalWorkflow@U2@@ABE_NPBVActor@Workflow@3@@Z$7 1001cd5e f   ClarkClassifyWorker.obj
 0001:0001bd67       __unwindfunclet$?isDatabaseAlreadyBuilt@ClarkClassifyValidator@LocalWorkflow@U2@@ABE_NPBVActor@Workflow@3@@Z$8 1001cd67 f   ClarkClassifyWorker.obj
 0001:0001bd70       __unwindfunclet$?isDatabaseAlreadyBuilt@ClarkClassifyValidator@LocalWorkflow@U2@@ABE_NPBVActor@Workflow@3@@Z$9 1001cd70 f   ClarkClassifyWorker.obj
 0001:0001bd79       __unwindfunclet$?isDatabaseAlreadyBuilt@ClarkClassifyValidator@LocalWorkflow@U2@@ABE_NPBVActor@Workflow@3@@Z$10 1001cd79 f   ClarkClassifyWorker.obj
 0001:0001bd82       __unwindfunclet$?isDatabaseAlreadyBuilt@ClarkClassifyValidator@LocalWorkflow@U2@@ABE_NPBVActor@Workflow@3@@Z$11 1001cd82 f   ClarkClassifyWorker.obj
 0001:0001bd8a       __ehhandler$?isDatabaseAlreadyBuilt@ClarkClassifyValidator@LocalWorkflow@U2@@ABE_NPBVActor@Workflow@3@@Z 1001cd8a f   ClarkClassifyWorker.obj
 0001:0001bdb0       __unwindfunclet$?isError@ClarkLogParser@LocalWorkflow@U2@@EBE_NABVQString@@@Z$0 1001cdb0 f   ClarkClassifyWorker.obj
 0001:0001bdb8       __unwindfunclet$?isError@ClarkLogParser@LocalWorkflow@U2@@EBE_NABVQString@@@Z$1 1001cdb8 f   ClarkClassifyWorker.obj
 0001:0001bdc0       __ehhandler$?isError@ClarkLogParser@LocalWorkflow@U2@@EBE_NABVQString@@@Z 1001cdc0 f   ClarkClassifyWorker.obj
 0001:0001bde0       __unwindfunclet$?keys@?$QMap@VQString@@V1@@@QBE?AV?$QList@VQString@@@@XZ$0 1001cde0 f   ClarkClassifyWorker.obj
 0001:0001bdf9       __ehhandler$?keys@?$QMap@VQString@@V1@@@QBE?AV?$QList@VQString@@@@XZ 1001cdf9 f   ClarkClassifyWorker.obj
 0001:0001be20       __unwindfunclet$?node_construct@?$QList@U?$QPair@VQString@@V1@@@@@AAEXPAUNode@1@ABU?$QPair@VQString@@V1@@@@Z$0 1001ce20 f   ClarkClassifyWorker.obj
 0001:0001be2b       __unwindfunclet$?node_construct@?$QList@U?$QPair@VQString@@V1@@@@@AAEXPAUNode@1@ABU?$QPair@VQString@@V1@@@@Z$2 1001ce2b f   ClarkClassifyWorker.obj
 0001:0001be34       __ehhandler$?node_construct@?$QList@U?$QPair@VQString@@V1@@@@@AAEXPAUNode@1@ABU?$QPair@VQString@@V1@@@@Z 1001ce34 f   ClarkClassifyWorker.obj
 0001:0001be50       __unwindfunclet$?node_construct@?$QList@VQVariant@@@@AAEXPAUNode@1@ABVQVariant@@@Z$0 1001ce50 f   ClarkClassifyWorker.obj
 0001:0001be5b       __ehhandler$?node_construct@?$QList@VQVariant@@@@AAEXPAUNode@1@ABVQVariant@@@Z 1001ce5b f   ClarkClassifyWorker.obj
 0001:0001be80       __unwindfunclet$?node_copy@?$QList@U?$QPair@VQString@@V1@@@@@AAEXPAUNode@1@00@Z$4 1001ce80 f   ClarkClassifyWorker.obj
 0001:0001be8b       __unwindfunclet$?node_copy@?$QList@U?$QPair@VQString@@V1@@@@@AAEXPAUNode@1@00@Z$6 1001ce8b f   ClarkClassifyWorker.obj
 0001:0001be94       __unwindfunclet$?node_copy@?$QList@U?$QPair@VQString@@V1@@@@@AAEXPAUNode@1@00@Z$8 1001ce94 f   ClarkClassifyWorker.obj
 0001:0001be9d       __ehhandler$?node_copy@?$QList@U?$QPair@VQString@@V1@@@@@AAEXPAUNode@1@00@Z 1001ce9d f   ClarkClassifyWorker.obj
 0001:0001bec0       __unwindfunclet$?node_copy@?$QList@VQVariant@@@@AAEXPAUNode@1@00@Z$4 1001cec0 f   ClarkClassifyWorker.obj
 0001:0001becb       __ehhandler$?node_copy@?$QList@VQVariant@@@@AAEXPAUNode@1@00@Z 1001cecb f   ClarkClassifyWorker.obj
 0001:0001bef0       __unwindfunclet$?node_destruct@?$QList@U?$QPair@VQString@@V1@@@@@AAEXPAUNode@1@0@Z$0 1001cef0 f   ClarkClassifyWorker.obj
 0001:0001bef9       __ehhandler$?node_destruct@?$QList@U?$QPair@VQString@@V1@@@@@AAEXPAUNode@1@0@Z 1001cef9 f   ClarkClassifyWorker.obj
 0001:0001bf20       __unwindfunclet$?node_destruct@?$QList@U?$QPair@VQString@@V1@@@@@AAEXPAUNode@1@@Z$0 1001cf20 f   ClarkClassifyWorker.obj
 0001:0001bf29       __ehhandler$?node_destruct@?$QList@U?$QPair@VQString@@V1@@@@@AAEXPAUNode@1@@Z 1001cf29 f   ClarkClassifyWorker.obj
 0001:0001bf50       __unwindfunclet$?prepare@ClarkClassifyTask@LocalWorkflow@U2@@EAEXXZ$0 1001cf50 f   ClarkClassifyWorker.obj
 0001:0001bf59       __unwindfunclet$?prepare@ClarkClassifyTask@LocalWorkflow@U2@@EAEXXZ$2 1001cf59 f   ClarkClassifyWorker.obj
 0001:0001bf64       __unwindfunclet$?prepare@ClarkClassifyTask@LocalWorkflow@U2@@EAEXXZ$3 1001cf64 f   ClarkClassifyWorker.obj
 0001:0001bf6f       __unwindfunclet$?prepare@ClarkClassifyTask@LocalWorkflow@U2@@EAEXXZ$1 1001cf6f f   ClarkClassifyWorker.obj
 0001:0001bf78       __unwindfunclet$?prepare@ClarkClassifyTask@LocalWorkflow@U2@@EAEXXZ$4 1001cf78 f   ClarkClassifyWorker.obj
 0001:0001bf92       __unwindfunclet$?prepare@ClarkClassifyTask@LocalWorkflow@U2@@EAEXXZ$5 1001cf92 f   ClarkClassifyWorker.obj
 0001:0001bfab       __unwindfunclet$?prepare@ClarkClassifyTask@LocalWorkflow@U2@@EAEXXZ$6 1001cfab f   ClarkClassifyWorker.obj
 0001:0001bfc4       __unwindfunclet$?prepare@ClarkClassifyTask@LocalWorkflow@U2@@EAEXXZ$7 1001cfc4 f   ClarkClassifyWorker.obj
 0001:0001bfcc       __ehhandler$?prepare@ClarkClassifyTask@LocalWorkflow@U2@@EAEXXZ 1001cfcc f   ClarkClassifyWorker.obj
 0001:0001bff0       __unwindfunclet$?qt_metatype_id@?$QMetaTypeId@V?$QMap@VQString@@I@@@@SAHXZ$0 1001cff0 f   ClarkClassifyWorker.obj
 0001:0001bff9       __ehhandler$?qt_metatype_id@?$QMetaTypeId@V?$QMap@VQString@@I@@@@SAHXZ 1001cff9 f   ClarkClassifyWorker.obj
 0001:0001c020       __unwindfunclet$?qt_metatype_id@?$QMetaTypeId@VQAssociativeIterableImpl@QtMetaTypePrivate@@@@SAHXZ$0 1001d020 f   ClarkClassifyWorker.obj
 0001:0001c029       __ehhandler$?qt_metatype_id@?$QMetaTypeId@VQAssociativeIterableImpl@QtMetaTypePrivate@@@@SAHXZ 1001d029 f   ClarkClassifyWorker.obj
 0001:0001c050       __unwindfunclet$?run@ClarkClassifyTask@LocalWorkflow@U2@@EAEXXZ$0 1001d050 f   ClarkClassifyWorker.obj
 0001:0001c059       __unwindfunclet$?run@ClarkClassifyTask@LocalWorkflow@U2@@EAEXXZ$1 1001d059 f   ClarkClassifyWorker.obj
 0001:0001c062       __unwindfunclet$?run@ClarkClassifyTask@LocalWorkflow@U2@@EAEXXZ$2 1001d062 f   ClarkClassifyWorker.obj
 0001:0001c06b       __unwindfunclet$?run@ClarkClassifyTask@LocalWorkflow@U2@@EAEXXZ$3 1001d06b f   ClarkClassifyWorker.obj
 0001:0001c074       __unwindfunclet$?run@ClarkClassifyTask@LocalWorkflow@U2@@EAEXXZ$4 1001d074 f   ClarkClassifyWorker.obj
 0001:0001c07d       __unwindfunclet$?run@ClarkClassifyTask@LocalWorkflow@U2@@EAEXXZ$5 1001d07d f   ClarkClassifyWorker.obj
 0001:0001c086       __unwindfunclet$?run@ClarkClassifyTask@LocalWorkflow@U2@@EAEXXZ$6 1001d086 f   ClarkClassifyWorker.obj
 0001:0001c08f       __unwindfunclet$?run@ClarkClassifyTask@LocalWorkflow@U2@@EAEXXZ$7 1001d08f f   ClarkClassifyWorker.obj
 0001:0001c098       __unwindfunclet$?run@ClarkClassifyTask@LocalWorkflow@U2@@EAEXXZ$8 1001d098 f   ClarkClassifyWorker.obj
 0001:0001c0a1       __unwindfunclet$?run@ClarkClassifyTask@LocalWorkflow@U2@@EAEXXZ$9 1001d0a1 f   ClarkClassifyWorker.obj
 0001:0001c0aa       __unwindfunclet$?run@ClarkClassifyTask@LocalWorkflow@U2@@EAEXXZ$10 1001d0aa f   ClarkClassifyWorker.obj
 0001:0001c0b2       __unwindfunclet$?run@ClarkClassifyTask@LocalWorkflow@U2@@EAEXXZ$13 1001d0b2 f   ClarkClassifyWorker.obj
 0001:0001c0bb       __unwindfunclet$?run@ClarkClassifyTask@LocalWorkflow@U2@@EAEXXZ$14 1001d0bb f   ClarkClassifyWorker.obj
 0001:0001c0c4       __unwindfunclet$?run@ClarkClassifyTask@LocalWorkflow@U2@@EAEXXZ$15 1001d0c4 f   ClarkClassifyWorker.obj
 0001:0001c0cd       __unwindfunclet$?run@ClarkClassifyTask@LocalWorkflow@U2@@EAEXXZ$16 1001d0cd f   ClarkClassifyWorker.obj
 0001:0001c0d6       __unwindfunclet$?run@ClarkClassifyTask@LocalWorkflow@U2@@EAEXXZ$17 1001d0d6 f   ClarkClassifyWorker.obj
 0001:0001c0df       __unwindfunclet$?run@ClarkClassifyTask@LocalWorkflow@U2@@EAEXXZ$20 1001d0df f   ClarkClassifyWorker.obj
 0001:0001c0e8       __unwindfunclet$?run@ClarkClassifyTask@LocalWorkflow@U2@@EAEXXZ$21 1001d0e8 f   ClarkClassifyWorker.obj
 0001:0001c0f1       __unwindfunclet$?run@ClarkClassifyTask@LocalWorkflow@U2@@EAEXXZ$18 1001d0f1 f   ClarkClassifyWorker.obj
 0001:0001c0fa       __unwindfunclet$?run@ClarkClassifyTask@LocalWorkflow@U2@@EAEXXZ$19 1001d0fa f   ClarkClassifyWorker.obj
 0001:0001c103       __unwindfunclet$?run@ClarkClassifyTask@LocalWorkflow@U2@@EAEXXZ$11 1001d103 f   ClarkClassifyWorker.obj
 0001:0001c10c       __unwindfunclet$?run@ClarkClassifyTask@LocalWorkflow@U2@@EAEXXZ$12 1001d10c f   ClarkClassifyWorker.obj
 0001:0001c115       __ehhandler$?run@ClarkClassifyTask@LocalWorkflow@U2@@EAEXXZ 1001d115 f   ClarkClassifyWorker.obj
 0001:0001c130       __unwindfunclet$?setLastError@ClarkLogParser@LocalWorkflow@U2@@EAEXABVQString@@@Z$0 1001d130 f   ClarkClassifyWorker.obj
 0001:0001c139       __unwindfunclet$?setLastError@ClarkLogParser@LocalWorkflow@U2@@EAEXABVQString@@@Z$1 1001d139 f   ClarkClassifyWorker.obj
 0001:0001c141       __unwindfunclet$?setLastError@ClarkLogParser@LocalWorkflow@U2@@EAEXABVQString@@@Z$2 1001d141 f   ClarkClassifyWorker.obj
 0001:0001c149       __unwindfunclet$?setLastError@ClarkLogParser@LocalWorkflow@U2@@EAEXABVQString@@@Z$3 1001d149 f   ClarkClassifyWorker.obj
 0001:0001c152       __ehhandler$?setLastError@ClarkLogParser@LocalWorkflow@U2@@EAEXABVQString@@@Z 1001d152 f   ClarkClassifyWorker.obj
 0001:0001c170       __unwindfunclet$?sl_taskFinished@ClarkClassifyWorker@LocalWorkflow@U2@@AAEXPAVTask@3@@Z$0 1001d170 f   ClarkClassifyWorker.obj
 0001:0001c179       __unwindfunclet$?sl_taskFinished@ClarkClassifyWorker@LocalWorkflow@U2@@AAEXPAVTask@3@@Z$1 1001d179 f   ClarkClassifyWorker.obj
 0001:0001c182       __unwindfunclet$?sl_taskFinished@ClarkClassifyWorker@LocalWorkflow@U2@@AAEXPAVTask@3@@Z$2 1001d182 f   ClarkClassifyWorker.obj
 0001:0001c18b       __unwindfunclet$?sl_taskFinished@ClarkClassifyWorker@LocalWorkflow@U2@@AAEXPAVTask@3@@Z$3 1001d18b f   ClarkClassifyWorker.obj
 0001:0001c194       __unwindfunclet$?sl_taskFinished@ClarkClassifyWorker@LocalWorkflow@U2@@AAEXPAVTask@3@@Z$4 1001d194 f   ClarkClassifyWorker.obj
 0001:0001c19d       __unwindfunclet$?sl_taskFinished@ClarkClassifyWorker@LocalWorkflow@U2@@AAEXPAVTask@3@@Z$5 1001d19d f   ClarkClassifyWorker.obj
 0001:0001c1a6       __unwindfunclet$?sl_taskFinished@ClarkClassifyWorker@LocalWorkflow@U2@@AAEXPAVTask@3@@Z$6 1001d1a6 f   ClarkClassifyWorker.obj
 0001:0001c1af       __unwindfunclet$?sl_taskFinished@ClarkClassifyWorker@LocalWorkflow@U2@@AAEXPAVTask@3@@Z$7 1001d1af f   ClarkClassifyWorker.obj
 0001:0001c1b8       __unwindfunclet$?sl_taskFinished@ClarkClassifyWorker@LocalWorkflow@U2@@AAEXPAVTask@3@@Z$8 1001d1b8 f   ClarkClassifyWorker.obj
 0001:0001c1c1       __unwindfunclet$?sl_taskFinished@ClarkClassifyWorker@LocalWorkflow@U2@@AAEXPAVTask@3@@Z$9 1001d1c1 f   ClarkClassifyWorker.obj
 0001:0001c1c9       __unwindfunclet$?sl_taskFinished@ClarkClassifyWorker@LocalWorkflow@U2@@AAEXPAVTask@3@@Z$10 1001d1c9 f   ClarkClassifyWorker.obj
 0001:0001c1d2       __unwindfunclet$?sl_taskFinished@ClarkClassifyWorker@LocalWorkflow@U2@@AAEXPAVTask@3@@Z$11 1001d1d2 f   ClarkClassifyWorker.obj
 0001:0001c1db       __unwindfunclet$?sl_taskFinished@ClarkClassifyWorker@LocalWorkflow@U2@@AAEXPAVTask@3@@Z$13 1001d1db f   ClarkClassifyWorker.obj
 0001:0001c1e4       __unwindfunclet$?sl_taskFinished@ClarkClassifyWorker@LocalWorkflow@U2@@AAEXPAVTask@3@@Z$14 1001d1e4 f   ClarkClassifyWorker.obj
 0001:0001c1ed       __unwindfunclet$?sl_taskFinished@ClarkClassifyWorker@LocalWorkflow@U2@@AAEXPAVTask@3@@Z$15 1001d1ed f   ClarkClassifyWorker.obj
 0001:0001c1f6       __unwindfunclet$?sl_taskFinished@ClarkClassifyWorker@LocalWorkflow@U2@@AAEXPAVTask@3@@Z$16 1001d1f6 f   ClarkClassifyWorker.obj
 0001:0001c1ff       __unwindfunclet$?sl_taskFinished@ClarkClassifyWorker@LocalWorkflow@U2@@AAEXPAVTask@3@@Z$17 1001d1ff f   ClarkClassifyWorker.obj
 0001:0001c208       __unwindfunclet$?sl_taskFinished@ClarkClassifyWorker@LocalWorkflow@U2@@AAEXPAVTask@3@@Z$18 1001d208 f   ClarkClassifyWorker.obj
 0001:0001c211       __unwindfunclet$?sl_taskFinished@ClarkClassifyWorker@LocalWorkflow@U2@@AAEXPAVTask@3@@Z$19 1001d211 f   ClarkClassifyWorker.obj
 0001:0001c21a       __unwindfunclet$?sl_taskFinished@ClarkClassifyWorker@LocalWorkflow@U2@@AAEXPAVTask@3@@Z$20 1001d21a f   ClarkClassifyWorker.obj
 0001:0001c223       __ehhandler$?sl_taskFinished@ClarkClassifyWorker@LocalWorkflow@U2@@AAEXPAVTask@3@@Z 1001d223 f   ClarkClassifyWorker.obj
 0001:0001c240       __unwindfunclet$?tick@ClarkClassifyWorker@LocalWorkflow@U2@@MAEPAVTask@3@XZ$0 1001d240 f   ClarkClassifyWorker.obj
 0001:0001c24c       __unwindfunclet$?tick@ClarkClassifyWorker@LocalWorkflow@U2@@MAEPAVTask@3@XZ$1 1001d24c f   ClarkClassifyWorker.obj
 0001:0001c258       __unwindfunclet$?tick@ClarkClassifyWorker@LocalWorkflow@U2@@MAEPAVTask@3@XZ$2 1001d258 f   ClarkClassifyWorker.obj
 0001:0001c260       __unwindfunclet$?tick@ClarkClassifyWorker@LocalWorkflow@U2@@MAEPAVTask@3@XZ$3 1001d260 f   ClarkClassifyWorker.obj
 0001:0001c269       __unwindfunclet$?tick@ClarkClassifyWorker@LocalWorkflow@U2@@MAEPAVTask@3@XZ$4 1001d269 f   ClarkClassifyWorker.obj
 0001:0001c272       __unwindfunclet$?tick@ClarkClassifyWorker@LocalWorkflow@U2@@MAEPAVTask@3@XZ$5 1001d272 f   ClarkClassifyWorker.obj
 0001:0001c27e       __unwindfunclet$?tick@ClarkClassifyWorker@LocalWorkflow@U2@@MAEPAVTask@3@XZ$6 1001d27e f   ClarkClassifyWorker.obj
 0001:0001c287       __unwindfunclet$?tick@ClarkClassifyWorker@LocalWorkflow@U2@@MAEPAVTask@3@XZ$7 1001d287 f   ClarkClassifyWorker.obj
 0001:0001c290       __unwindfunclet$?tick@ClarkClassifyWorker@LocalWorkflow@U2@@MAEPAVTask@3@XZ$8 1001d290 f   ClarkClassifyWorker.obj
 0001:0001c299       __unwindfunclet$?tick@ClarkClassifyWorker@LocalWorkflow@U2@@MAEPAVTask@3@XZ$9 1001d299 f   ClarkClassifyWorker.obj
 0001:0001c2a2       __unwindfunclet$?tick@ClarkClassifyWorker@LocalWorkflow@U2@@MAEPAVTask@3@XZ$10 1001d2a2 f   ClarkClassifyWorker.obj
 0001:0001c2ab       __unwindfunclet$?tick@ClarkClassifyWorker@LocalWorkflow@U2@@MAEPAVTask@3@XZ$11 1001d2ab f   ClarkClassifyWorker.obj
 0001:0001c2b4       __unwindfunclet$?tick@ClarkClassifyWorker@LocalWorkflow@U2@@MAEPAVTask@3@XZ$12 1001d2b4 f   ClarkClassifyWorker.obj
 0001:0001c2bd       __unwindfunclet$?tick@ClarkClassifyWorker@LocalWorkflow@U2@@MAEPAVTask@3@XZ$13 1001d2bd f   ClarkClassifyWorker.obj
 0001:0001c2c8       __unwindfunclet$?tick@ClarkClassifyWorker@LocalWorkflow@U2@@MAEPAVTask@3@XZ$14 1001d2c8 f   ClarkClassifyWorker.obj
 0001:0001c2e2       __unwindfunclet$?tick@ClarkClassifyWorker@LocalWorkflow@U2@@MAEPAVTask@3@XZ$15 1001d2e2 f   ClarkClassifyWorker.obj
 0001:0001c2eb       __unwindfunclet$?tick@ClarkClassifyWorker@LocalWorkflow@U2@@MAEPAVTask@3@XZ$16 1001d2eb f   ClarkClassifyWorker.obj
 0001:0001c2f7       __unwindfunclet$?tick@ClarkClassifyWorker@LocalWorkflow@U2@@MAEPAVTask@3@XZ$17 1001d2f7 f   ClarkClassifyWorker.obj
 0001:0001c300       __unwindfunclet$?tick@ClarkClassifyWorker@LocalWorkflow@U2@@MAEPAVTask@3@XZ$18 1001d300 f   ClarkClassifyWorker.obj
 0001:0001c31a       __unwindfunclet$?tick@ClarkClassifyWorker@LocalWorkflow@U2@@MAEPAVTask@3@XZ$19 1001d31a f   ClarkClassifyWorker.obj
 0001:0001c334       __unwindfunclet$?tick@ClarkClassifyWorker@LocalWorkflow@U2@@MAEPAVTask@3@XZ$20 1001d334 f   ClarkClassifyWorker.obj
 0001:0001c34e       __unwindfunclet$?tick@ClarkClassifyWorker@LocalWorkflow@U2@@MAEPAVTask@3@XZ$21 1001d34e f   ClarkClassifyWorker.obj
 0001:0001c368       __unwindfunclet$?tick@ClarkClassifyWorker@LocalWorkflow@U2@@MAEPAVTask@3@XZ$22 1001d368 f   ClarkClassifyWorker.obj
 0001:0001c381       __unwindfunclet$?tick@ClarkClassifyWorker@LocalWorkflow@U2@@MAEPAVTask@3@XZ$23 1001d381 f   ClarkClassifyWorker.obj
 0001:0001c39b       __unwindfunclet$?tick@ClarkClassifyWorker@LocalWorkflow@U2@@MAEPAVTask@3@XZ$24 1001d39b f   ClarkClassifyWorker.obj
 0001:0001c3a4       __unwindfunclet$?tick@ClarkClassifyWorker@LocalWorkflow@U2@@MAEPAVTask@3@XZ$25 1001d3a4 f   ClarkClassifyWorker.obj
 0001:0001c3ad       __unwindfunclet$?tick@ClarkClassifyWorker@LocalWorkflow@U2@@MAEPAVTask@3@XZ$26 1001d3ad f   ClarkClassifyWorker.obj
 0001:0001c3b6       __unwindfunclet$?tick@ClarkClassifyWorker@LocalWorkflow@U2@@MAEPAVTask@3@XZ$27 1001d3b6 f   ClarkClassifyWorker.obj
 0001:0001c3bf       __unwindfunclet$?tick@ClarkClassifyWorker@LocalWorkflow@U2@@MAEPAVTask@3@XZ$29 1001d3bf f   ClarkClassifyWorker.obj
 0001:0001c3c8       __unwindfunclet$?tick@ClarkClassifyWorker@LocalWorkflow@U2@@MAEPAVTask@3@XZ$30 1001d3c8 f   ClarkClassifyWorker.obj
 0001:0001c3d1       __unwindfunclet$?tick@ClarkClassifyWorker@LocalWorkflow@U2@@MAEPAVTask@3@XZ$45 1001d3d1 f   ClarkClassifyWorker.obj
 0001:0001c3d9       __unwindfunclet$?tick@ClarkClassifyWorker@LocalWorkflow@U2@@MAEPAVTask@3@XZ$31 1001d3d9 f   ClarkClassifyWorker.obj
 0001:0001c3e1       __unwindfunclet$?tick@ClarkClassifyWorker@LocalWorkflow@U2@@MAEPAVTask@3@XZ$32 1001d3e1 f   ClarkClassifyWorker.obj
 0001:0001c3ea       __unwindfunclet$?tick@ClarkClassifyWorker@LocalWorkflow@U2@@MAEPAVTask@3@XZ$33 1001d3ea f   ClarkClassifyWorker.obj
 0001:0001c3f3       __unwindfunclet$?tick@ClarkClassifyWorker@LocalWorkflow@U2@@MAEPAVTask@3@XZ$34 1001d3f3 f   ClarkClassifyWorker.obj
 0001:0001c3fb       __unwindfunclet$?tick@ClarkClassifyWorker@LocalWorkflow@U2@@MAEPAVTask@3@XZ$35 1001d3fb f   ClarkClassifyWorker.obj
 0001:0001c404       __unwindfunclet$?tick@ClarkClassifyWorker@LocalWorkflow@U2@@MAEPAVTask@3@XZ$36 1001d404 f   ClarkClassifyWorker.obj
 0001:0001c40d       __unwindfunclet$?tick@ClarkClassifyWorker@LocalWorkflow@U2@@MAEPAVTask@3@XZ$37 1001d40d f   ClarkClassifyWorker.obj
 0001:0001c415       __unwindfunclet$?tick@ClarkClassifyWorker@LocalWorkflow@U2@@MAEPAVTask@3@XZ$38 1001d415 f   ClarkClassifyWorker.obj
 0001:0001c41e       __unwindfunclet$?tick@ClarkClassifyWorker@LocalWorkflow@U2@@MAEPAVTask@3@XZ$39 1001d41e f   ClarkClassifyWorker.obj
 0001:0001c429       __unwindfunclet$?tick@ClarkClassifyWorker@LocalWorkflow@U2@@MAEPAVTask@3@XZ$40 1001d429 f   ClarkClassifyWorker.obj
 0001:0001c431       __unwindfunclet$?tick@ClarkClassifyWorker@LocalWorkflow@U2@@MAEPAVTask@3@XZ$41 1001d431 f   ClarkClassifyWorker.obj
 0001:0001c43c       __unwindfunclet$?tick@ClarkClassifyWorker@LocalWorkflow@U2@@MAEPAVTask@3@XZ$43 1001d43c f   ClarkClassifyWorker.obj
 0001:0001c445       __ehhandler$?tick@ClarkClassifyWorker@LocalWorkflow@U2@@MAEPAVTask@3@XZ 1001d445 f   ClarkClassifyWorker.obj
 0001:0001c470       __unwindfunclet$?validateDatabase@ClarkClassifyValidator@LocalWorkflow@U2@@ABE_NPBVActor@Workflow@3@AAV?$QList@VWorkflowNotification@U2@@@@@Z$0 1001d470 f   ClarkClassifyWorker.obj
 0001:0001c479       __unwindfunclet$?validateDatabase@ClarkClassifyValidator@LocalWorkflow@U2@@ABE_NPBVActor@Workflow@3@AAV?$QList@VWorkflowNotification@U2@@@@@Z$1 1001d479 f   ClarkClassifyWorker.obj
 0001:0001c482       __unwindfunclet$?validateDatabase@ClarkClassifyValidator@LocalWorkflow@U2@@ABE_NPBVActor@Workflow@3@AAV?$QList@VWorkflowNotification@U2@@@@@Z$2 1001d482 f   ClarkClassifyWorker.obj
 0001:0001c48b       __unwindfunclet$?validateDatabase@ClarkClassifyValidator@LocalWorkflow@U2@@ABE_NPBVActor@Workflow@3@AAV?$QList@VWorkflowNotification@U2@@@@@Z$3 1001d48b f   ClarkClassifyWorker.obj
 0001:0001c494       __unwindfunclet$?validateDatabase@ClarkClassifyValidator@LocalWorkflow@U2@@ABE_NPBVActor@Workflow@3@AAV?$QList@VWorkflowNotification@U2@@@@@Z$4 1001d494 f   ClarkClassifyWorker.obj
 0001:0001c49d       __unwindfunclet$?validateDatabase@ClarkClassifyValidator@LocalWorkflow@U2@@ABE_NPBVActor@Workflow@3@AAV?$QList@VWorkflowNotification@U2@@@@@Z$5 1001d49d f   ClarkClassifyWorker.obj
 0001:0001c4a6       __unwindfunclet$?validateDatabase@ClarkClassifyValidator@LocalWorkflow@U2@@ABE_NPBVActor@Workflow@3@AAV?$QList@VWorkflowNotification@U2@@@@@Z$6 1001d4a6 f   ClarkClassifyWorker.obj
 0001:0001c4af       __unwindfunclet$?validateDatabase@ClarkClassifyValidator@LocalWorkflow@U2@@ABE_NPBVActor@Workflow@3@AAV?$QList@VWorkflowNotification@U2@@@@@Z$7 1001d4af f   ClarkClassifyWorker.obj
 0001:0001c4b8       __unwindfunclet$?validateDatabase@ClarkClassifyValidator@LocalWorkflow@U2@@ABE_NPBVActor@Workflow@3@AAV?$QList@VWorkflowNotification@U2@@@@@Z$8 1001d4b8 f   ClarkClassifyWorker.obj
 0001:0001c4c1       __unwindfunclet$?validateDatabase@ClarkClassifyValidator@LocalWorkflow@U2@@ABE_NPBVActor@Workflow@3@AAV?$QList@VWorkflowNotification@U2@@@@@Z$9 1001d4c1 f   ClarkClassifyWorker.obj
 0001:0001c4c9       __unwindfunclet$?validateDatabase@ClarkClassifyValidator@LocalWorkflow@U2@@ABE_NPBVActor@Workflow@3@AAV?$QList@VWorkflowNotification@U2@@@@@Z$10 1001d4c9 f   ClarkClassifyWorker.obj
 0001:0001c4d1       __unwindfunclet$?validateDatabase@ClarkClassifyValidator@LocalWorkflow@U2@@ABE_NPBVActor@Workflow@3@AAV?$QList@VWorkflowNotification@U2@@@@@Z$11 1001d4d1 f   ClarkClassifyWorker.obj
 0001:0001c4d9       __unwindfunclet$?validateDatabase@ClarkClassifyValidator@LocalWorkflow@U2@@ABE_NPBVActor@Workflow@3@AAV?$QList@VWorkflowNotification@U2@@@@@Z$12 1001d4d9 f   ClarkClassifyWorker.obj
 0001:0001c4e1       __unwindfunclet$?validateDatabase@ClarkClassifyValidator@LocalWorkflow@U2@@ABE_NPBVActor@Workflow@3@AAV?$QList@VWorkflowNotification@U2@@@@@Z$13 1001d4e1 f   ClarkClassifyWorker.obj
 0001:0001c4ea       __unwindfunclet$?validateDatabase@ClarkClassifyValidator@LocalWorkflow@U2@@ABE_NPBVActor@Workflow@3@AAV?$QList@VWorkflowNotification@U2@@@@@Z$14 1001d4ea f   ClarkClassifyWorker.obj
 0001:0001c4f3       __unwindfunclet$?validateDatabase@ClarkClassifyValidator@LocalWorkflow@U2@@ABE_NPBVActor@Workflow@3@AAV?$QList@VWorkflowNotification@U2@@@@@Z$15 1001d4f3 f   ClarkClassifyWorker.obj
 0001:0001c4fc       __unwindfunclet$?validateDatabase@ClarkClassifyValidator@LocalWorkflow@U2@@ABE_NPBVActor@Workflow@3@AAV?$QList@VWorkflowNotification@U2@@@@@Z$16 1001d4fc f   ClarkClassifyWorker.obj
 0001:0001c504       __unwindfunclet$?validateDatabase@ClarkClassifyValidator@LocalWorkflow@U2@@ABE_NPBVActor@Workflow@3@AAV?$QList@VWorkflowNotification@U2@@@@@Z$17 1001d504 f   ClarkClassifyWorker.obj
 0001:0001c50d       __unwindfunclet$?validateDatabase@ClarkClassifyValidator@LocalWorkflow@U2@@ABE_NPBVActor@Workflow@3@AAV?$QList@VWorkflowNotification@U2@@@@@Z$18 1001d50d f   ClarkClassifyWorker.obj
 0001:0001c516       __unwindfunclet$?validateDatabase@ClarkClassifyValidator@LocalWorkflow@U2@@ABE_NPBVActor@Workflow@3@AAV?$QList@VWorkflowNotification@U2@@@@@Z$19 1001d516 f   ClarkClassifyWorker.obj
 0001:0001c51f       __unwindfunclet$?validateDatabase@ClarkClassifyValidator@LocalWorkflow@U2@@ABE_NPBVActor@Workflow@3@AAV?$QList@VWorkflowNotification@U2@@@@@Z$20 1001d51f f   ClarkClassifyWorker.obj
 0001:0001c528       __ehhandler$?validateDatabase@ClarkClassifyValidator@LocalWorkflow@U2@@ABE_NPBVActor@Workflow@3@AAV?$QList@VWorkflowNotification@U2@@@@@Z 1001d528 f   ClarkClassifyWorker.obj
 0001:0001c550       __unwindfunclet$?validateRefseqAvailability@ClarkClassifyValidator@LocalWorkflow@U2@@ABE_NPBVActor@Workflow@3@AAV?$QList@VWorkflowNotification@U2@@@@@Z$0 1001d550 f   ClarkClassifyWorker.obj
 0001:0001c559       __unwindfunclet$?validateRefseqAvailability@ClarkClassifyValidator@LocalWorkflow@U2@@ABE_NPBVActor@Workflow@3@AAV?$QList@VWorkflowNotification@U2@@@@@Z$1 1001d559 f   ClarkClassifyWorker.obj
 0001:0001c562       __unwindfunclet$?validateRefseqAvailability@ClarkClassifyValidator@LocalWorkflow@U2@@ABE_NPBVActor@Workflow@3@AAV?$QList@VWorkflowNotification@U2@@@@@Z$2 1001d562 f   ClarkClassifyWorker.obj
 0001:0001c56b       __ehhandler$?validateRefseqAvailability@ClarkClassifyValidator@LocalWorkflow@U2@@ABE_NPBVActor@Workflow@3@AAV?$QList@VWorkflowNotification@U2@@@@@Z 1001d56b f   ClarkClassifyWorker.obj
 0001:0001c590       __unwindfunclet$??0ClarkSupport@U2@@QAE@ABVQString@@00@Z$0 1001d590 f   ClarkSupport.obj
 0001:0001c599       __unwindfunclet$??0ClarkSupport@U2@@QAE@ABVQString@@00@Z$1 1001d599 f   ClarkSupport.obj
 0001:0001c5a2       __unwindfunclet$??0ClarkSupport@U2@@QAE@ABVQString@@00@Z$3 1001d5a2 f   ClarkSupport.obj
 0001:0001c5ab       __unwindfunclet$??0ClarkSupport@U2@@QAE@ABVQString@@00@Z$4 1001d5ab f   ClarkSupport.obj
 0001:0001c5b4       __unwindfunclet$??0ClarkSupport@U2@@QAE@ABVQString@@00@Z$5 1001d5b4 f   ClarkSupport.obj
 0001:0001c5bd       __unwindfunclet$??0ClarkSupport@U2@@QAE@ABVQString@@00@Z$6 1001d5bd f   ClarkSupport.obj
 0001:0001c5c6       __unwindfunclet$??0ClarkSupport@U2@@QAE@ABVQString@@00@Z$7 1001d5c6 f   ClarkSupport.obj
 0001:0001c5cf       __unwindfunclet$??0ClarkSupport@U2@@QAE@ABVQString@@00@Z$8 1001d5cf f   ClarkSupport.obj
 0001:0001c5d8       __unwindfunclet$??0ClarkSupport@U2@@QAE@ABVQString@@00@Z$9 1001d5d8 f   ClarkSupport.obj
 0001:0001c5e1       __unwindfunclet$??0ClarkSupport@U2@@QAE@ABVQString@@00@Z$10 1001d5e1 f   ClarkSupport.obj
 0001:0001c5ea       __unwindfunclet$??0ClarkSupport@U2@@QAE@ABVQString@@00@Z$11 1001d5ea f   ClarkSupport.obj
 0001:0001c5f3       __unwindfunclet$??0ClarkSupport@U2@@QAE@ABVQString@@00@Z$12 1001d5f3 f   ClarkSupport.obj
 0001:0001c5fc       __unwindfunclet$??0ClarkSupport@U2@@QAE@ABVQString@@00@Z$13 1001d5fc f   ClarkSupport.obj
 0001:0001c605       __unwindfunclet$??0ClarkSupport@U2@@QAE@ABVQString@@00@Z$14 1001d605 f   ClarkSupport.obj
 0001:0001c60e       __unwindfunclet$??0ClarkSupport@U2@@QAE@ABVQString@@00@Z$15 1001d60e f   ClarkSupport.obj
 0001:0001c617       __unwindfunclet$??0ClarkSupport@U2@@QAE@ABVQString@@00@Z$16 1001d617 f   ClarkSupport.obj
 0001:0001c620       __unwindfunclet$??0ClarkSupport@U2@@QAE@ABVQString@@00@Z$17 1001d620 f   ClarkSupport.obj
 0001:0001c629       __unwindfunclet$??0ClarkSupport@U2@@QAE@ABVQString@@00@Z$18 1001d629 f   ClarkSupport.obj
 0001:0001c632       __ehhandler$??0ClarkSupport@U2@@QAE@ABVQString@@00@Z 1001d632 f   ClarkSupport.obj
 0001:0001c650       __unwindfunclet$??H@YA?BVQString@@PBDABV0@@Z$0 1001d650 f   ClarkSupport.obj
 0001:0001c66a       __ehhandler$??H@YA?BVQString@@PBDABV0@@Z 1001d66a f   ClarkSupport.obj
 0001:0001c690       __unwindfunclet$??__EalgoLog@U2@@YAXXZ$0 1001d690 f   ClarkSupport.obj
 0001:0001c699       __ehhandler$??__EalgoLog@U2@@YAXXZ 1001d699 f   ClarkSupport.obj
 0001:0001c6c0       __unwindfunclet$??__EcmdLog@U2@@YAXXZ$0 1001d6c0 f   ClarkSupport.obj
 0001:0001c6c9       __ehhandler$??__EcmdLog@U2@@YAXXZ 1001d6c9 f   ClarkSupport.obj
 0001:0001c6f0       __unwindfunclet$??__EcoreLog@U2@@YAXXZ$0 1001d6f0 f   ClarkSupport.obj
 0001:0001c6f9       __ehhandler$??__EcoreLog@U2@@YAXXZ 1001d6f9 f   ClarkSupport.obj
 0001:0001c720       __unwindfunclet$??__EioLog@U2@@YAXXZ$0 1001d720 f   ClarkSupport.obj
 0001:0001c729       __ehhandler$??__EioLog@U2@@YAXXZ 1001d729 f   ClarkSupport.obj
 0001:0001c750       __unwindfunclet$??__EperfLog@U2@@YAXXZ$0 1001d750 f   ClarkSupport.obj
 0001:0001c759       __ehhandler$??__EperfLog@U2@@YAXXZ 1001d759 f   ClarkSupport.obj
 0001:0001c780       __unwindfunclet$??__EscriptLog@U2@@YAXXZ$0 1001d780 f   ClarkSupport.obj
 0001:0001c789       __ehhandler$??__EscriptLog@U2@@YAXXZ 1001d789 f   ClarkSupport.obj
 0001:0001c7b0       __unwindfunclet$??__EtaskLog@U2@@YAXXZ$0 1001d7b0 f   ClarkSupport.obj
 0001:0001c7b9       __ehhandler$??__EtaskLog@U2@@YAXXZ 1001d7b9 f   ClarkSupport.obj
 0001:0001c7e0       __unwindfunclet$??__EuiLog@U2@@YAXXZ$0 1001d7e0 f   ClarkSupport.obj
 0001:0001c7e9       __ehhandler$??__EuiLog@U2@@YAXXZ 1001d7e9 f   ClarkSupport.obj
 0001:0001c810       __unwindfunclet$??__EuserActLog@U2@@YAXXZ$0 1001d810 f   ClarkSupport.obj
 0001:0001c819       __ehhandler$??__EuserActLog@U2@@YAXXZ 1001d819 f   ClarkSupport.obj
 0001:0001c840       __unwindfunclet$?registerTools@ClarkSupport@U2@@SAXPAVExternalToolRegistry@2@@Z$0 1001d840 f   ClarkSupport.obj
 0001:0001c84b       __unwindfunclet$?registerTools@ClarkSupport@U2@@SAXPAVExternalToolRegistry@2@@Z$1 1001d84b f   ClarkSupport.obj
 0001:0001c865       __unwindfunclet$?registerTools@ClarkSupport@U2@@SAXPAVExternalToolRegistry@2@@Z$2 1001d865 f   ClarkSupport.obj
 0001:0001c870       __unwindfunclet$?registerTools@ClarkSupport@U2@@SAXPAVExternalToolRegistry@2@@Z$3 1001d870 f   ClarkSupport.obj
 0001:0001c88a       __unwindfunclet$?registerTools@ClarkSupport@U2@@SAXPAVExternalToolRegistry@2@@Z$4 1001d88a f   ClarkSupport.obj
 0001:0001c895       __unwindfunclet$?registerTools@ClarkSupport@U2@@SAXPAVExternalToolRegistry@2@@Z$5 1001d895 f   ClarkSupport.obj
 0001:0001c8af       __unwindfunclet$?registerTools@ClarkSupport@U2@@SAXPAVExternalToolRegistry@2@@Z$6 1001d8af f   ClarkSupport.obj
 0001:0001c8ba       __unwindfunclet$?registerTools@ClarkSupport@U2@@SAXPAVExternalToolRegistry@2@@Z$7 1001d8ba f   ClarkSupport.obj
 0001:0001c8d4       __unwindfunclet$?registerTools@ClarkSupport@U2@@SAXPAVExternalToolRegistry@2@@Z$8 1001d8d4 f   ClarkSupport.obj
 0001:0001c8df       __unwindfunclet$?registerTools@ClarkSupport@U2@@SAXPAVExternalToolRegistry@2@@Z$9 1001d8df f   ClarkSupport.obj
 0001:0001c8f9       __unwindfunclet$?registerTools@ClarkSupport@U2@@SAXPAVExternalToolRegistry@2@@Z$10 1001d8f9 f   ClarkSupport.obj
 0001:0001c904       __unwindfunclet$?registerTools@ClarkSupport@U2@@SAXPAVExternalToolRegistry@2@@Z$11 1001d904 f   ClarkSupport.obj
 0001:0001c91e       __unwindfunclet$?registerTools@ClarkSupport@U2@@SAXPAVExternalToolRegistry@2@@Z$12 1001d91e f   ClarkSupport.obj
 0001:0001c927       __ehhandler$?registerTools@ClarkSupport@U2@@SAXPAVExternalToolRegistry@2@@Z 1001d927 f   ClarkSupport.obj
 0001:0001c950       __ehhandler$??0?$QList@PAVXMLTestFactory@U2@@@@QAE@ABV0@@Z 1001d950 f   ClarkSupportPlugin.obj
 0001:0001c970       __unwindfunclet$??0ClarkSupportPlugin@U2@@QAE@XZ$0 1001d970 f   ClarkSupportPlugin.obj
 0001:0001c979       __unwindfunclet$??0ClarkSupportPlugin@U2@@QAE@XZ$1 1001d979 f   ClarkSupportPlugin.obj
 0001:0001c982       __unwindfunclet$??0ClarkSupportPlugin@U2@@QAE@XZ$2 1001d982 f   ClarkSupportPlugin.obj
 0001:0001c98b       __unwindfunclet$??0ClarkSupportPlugin@U2@@QAE@XZ$3 1001d98b f   ClarkSupportPlugin.obj
 0001:0001c994       __unwindfunclet$??0ClarkSupportPlugin@U2@@QAE@XZ$4 1001d994 f   ClarkSupportPlugin.obj
 0001:0001c99d       __unwindfunclet$??0ClarkSupportPlugin@U2@@QAE@XZ$5 1001d99d f   ClarkSupportPlugin.obj
 0001:0001c9a6       __unwindfunclet$??0ClarkSupportPlugin@U2@@QAE@XZ$6 1001d9a6 f   ClarkSupportPlugin.obj
 0001:0001c9af       __unwindfunclet$??0ClarkSupportPlugin@U2@@QAE@XZ$7 1001d9af f   ClarkSupportPlugin.obj
 0001:0001c9b8       __unwindfunclet$??0ClarkSupportPlugin@U2@@QAE@XZ$8 1001d9b8 f   ClarkSupportPlugin.obj
 0001:0001c9c3       __unwindfunclet$??0ClarkSupportPlugin@U2@@QAE@XZ$10 1001d9c3 f   ClarkSupportPlugin.obj
 0001:0001c9cb       __ehhandler$??0ClarkSupportPlugin@U2@@QAE@XZ 1001d9cb f   ClarkSupportPlugin.obj
 0001:0001c9f0       __unwindfunclet$??1?$GAutoDeleteList@VXMLTestFactory@U2@@@U2@@UAE@XZ$0 1001d9f0 f   ClarkSupportPlugin.obj
 0001:0001c9f9       __unwindfunclet$??1?$GAutoDeleteList@VXMLTestFactory@U2@@@U2@@UAE@XZ$1 1001d9f9 f   ClarkSupportPlugin.obj
 0001:0001ca04       __ehhandler$??1?$GAutoDeleteList@VXMLTestFactory@U2@@@U2@@UAE@XZ 1001da04 f   ClarkSupportPlugin.obj
 0001:0001ca20       __unwindfunclet$??1ClarkSupportPlugin@U2@@UAE@XZ$0 1001da20 f   ClarkSupportPlugin.obj
 0001:0001ca29       __unwindfunclet$??1ClarkSupportPlugin@U2@@UAE@XZ$1 1001da29 f   ClarkSupportPlugin.obj
 0001:0001ca32       __unwindfunclet$??1ClarkSupportPlugin@U2@@UAE@XZ$2 1001da32 f   ClarkSupportPlugin.obj
 0001:0001ca3b       __unwindfunclet$??1ClarkSupportPlugin@U2@@UAE@XZ$3 1001da3b f   ClarkSupportPlugin.obj
 0001:0001ca44       __unwindfunclet$??1ClarkSupportPlugin@U2@@UAE@XZ$4 1001da44 f   ClarkSupportPlugin.obj
 0001:0001ca4d       __unwindfunclet$??1ClarkSupportPlugin@U2@@UAE@XZ$5 1001da4d f   ClarkSupportPlugin.obj
 0001:0001ca56       __unwindfunclet$??1ClarkSupportPlugin@U2@@UAE@XZ$6 1001da56 f   ClarkSupportPlugin.obj
 0001:0001ca5f       __unwindfunclet$??1ClarkSupportPlugin@U2@@UAE@XZ$7 1001da5f f   ClarkSupportPlugin.obj
 0001:0001ca68       __unwindfunclet$??1ClarkSupportPlugin@U2@@UAE@XZ$8 1001da68 f   ClarkSupportPlugin.obj
 0001:0001ca70       __ehhandler$??1ClarkSupportPlugin@U2@@UAE@XZ 1001da70 f   ClarkSupportPlugin.obj
 0001:0001ca90       __unwindfunclet$??__EalgoLog@U2@@YAXXZ$0 1001da90 f   ClarkSupportPlugin.obj
 0001:0001ca99       __ehhandler$??__EalgoLog@U2@@YAXXZ 1001da99 f   ClarkSupportPlugin.obj
 0001:0001cac0       __unwindfunclet$??__EcmdLog@U2@@YAXXZ$0 1001dac0 f   ClarkSupportPlugin.obj
 0001:0001cac9       __ehhandler$??__EcmdLog@U2@@YAXXZ 1001dac9 f   ClarkSupportPlugin.obj
 0001:0001caf0       __unwindfunclet$??__EcoreLog@U2@@YAXXZ$0 1001daf0 f   ClarkSupportPlugin.obj
 0001:0001caf9       __ehhandler$??__EcoreLog@U2@@YAXXZ 1001daf9 f   ClarkSupportPlugin.obj
 0001:0001cb20       __unwindfunclet$??__EioLog@U2@@YAXXZ$0 1001db20 f   ClarkSupportPlugin.obj
 0001:0001cb29       __ehhandler$??__EioLog@U2@@YAXXZ 1001db29 f   ClarkSupportPlugin.obj
 0001:0001cb50       __unwindfunclet$??__EperfLog@U2@@YAXXZ$0 1001db50 f   ClarkSupportPlugin.obj
 0001:0001cb59       __ehhandler$??__EperfLog@U2@@YAXXZ 1001db59 f   ClarkSupportPlugin.obj
 0001:0001cb80       __unwindfunclet$??__EscriptLog@U2@@YAXXZ$0 1001db80 f   ClarkSupportPlugin.obj
 0001:0001cb89       __ehhandler$??__EscriptLog@U2@@YAXXZ 1001db89 f   ClarkSupportPlugin.obj
 0001:0001cbb0       __unwindfunclet$??__EtaskLog@U2@@YAXXZ$0 1001dbb0 f   ClarkSupportPlugin.obj
 0001:0001cbb9       __ehhandler$??__EtaskLog@U2@@YAXXZ 1001dbb9 f   ClarkSupportPlugin.obj
 0001:0001cbe0       __unwindfunclet$??__EuiLog@U2@@YAXXZ$0 1001dbe0 f   ClarkSupportPlugin.obj
 0001:0001cbe9       __ehhandler$??__EuiLog@U2@@YAXXZ 1001dbe9 f   ClarkSupportPlugin.obj
 0001:0001cc10       __unwindfunclet$??__EuserActLog@U2@@YAXXZ$0 1001dc10 f   ClarkSupportPlugin.obj
 0001:0001cc19       __ehhandler$??__EuserActLog@U2@@YAXXZ 1001dc19 f   ClarkSupportPlugin.obj
 0001:0001cc40       __unwindfunclet$??0GTest_CompareClarkDatabaseMetafiles@U2@@QAE@PAVXMLTestFormat@1@ABVQString@@PAVGTest@1@PBVGTestEnvironment@1@ABV?$QList@PAVGTest@U2@@@@ABVQDomElement@@@Z$0 1001dc40 f   ClarkTests.obj
 0001:0001cc49       __unwindfunclet$??0GTest_CompareClarkDatabaseMetafiles@U2@@QAE@PAVXMLTestFormat@1@ABVQString@@PAVGTest@1@PBVGTestEnvironment@1@ABV?$QList@PAVGTest@U2@@@@ABVQDomElement@@@Z$1 1001dc49 f   ClarkTests.obj
 0001:0001cc58       __unwindfunclet$??0GTest_CompareClarkDatabaseMetafiles@U2@@QAE@PAVXMLTestFormat@1@ABVQString@@PAVGTest@1@PBVGTestEnvironment@1@ABV?$QList@PAVGTest@U2@@@@ABVQDomElement@@@Z$2 1001dc58 f   ClarkTests.obj
 0001:0001cc67       __unwindfunclet$??0GTest_CompareClarkDatabaseMetafiles@U2@@QAE@PAVXMLTestFormat@1@ABVQString@@PAVGTest@1@PBVGTestEnvironment@1@ABV?$QList@PAVGTest@U2@@@@ABVQDomElement@@@Z$3 1001dc67 f   ClarkTests.obj
 0001:0001cc75       __unwindfunclet$??0GTest_CompareClarkDatabaseMetafiles@U2@@QAE@PAVXMLTestFormat@1@ABVQString@@PAVGTest@1@PBVGTestEnvironment@1@ABV?$QList@PAVGTest@U2@@@@ABVQDomElement@@@Z$4 1001dc75 f   ClarkTests.obj
 0001:0001cc83       __ehhandler$??0GTest_CompareClarkDatabaseMetafiles@U2@@QAE@PAVXMLTestFormat@1@ABVQString@@PAVGTest@1@PBVGTestEnvironment@1@ABV?$QList@PAVGTest@U2@@@@ABVQDomElement@@@Z 1001dc83 f   ClarkTests.obj
 0001:0001cca0       __unwindfunclet$??0GTest_CompareClarkDatabaseMetafilesFactory@GTest_CompareClarkDatabaseMetafiles@U2@@QAE@XZ$0 1001dca0 f   ClarkTests.obj
 0001:0001cca9       __unwindfunclet$??0GTest_CompareClarkDatabaseMetafilesFactory@GTest_CompareClarkDatabaseMetafiles@U2@@QAE@XZ$1 1001dca9 f   ClarkTests.obj
 0001:0001ccb2       __ehhandler$??0GTest_CompareClarkDatabaseMetafilesFactory@GTest_CompareClarkDatabaseMetafiles@U2@@QAE@XZ 1001dcb2 f   ClarkTests.obj
 0001:0001ccd0       __unwindfunclet$??1GTest_CompareClarkDatabaseMetafiles@U2@@UAE@XZ$0 1001dcd0 f   ClarkTests.obj
 0001:0001ccd9       __unwindfunclet$??1GTest_CompareClarkDatabaseMetafiles@U2@@UAE@XZ$1 1001dcd9 f   ClarkTests.obj
 0001:0001cce8       __unwindfunclet$??1GTest_CompareClarkDatabaseMetafiles@U2@@UAE@XZ$2 1001dce8 f   ClarkTests.obj
 0001:0001ccf7       __unwindfunclet$??1GTest_CompareClarkDatabaseMetafiles@U2@@UAE@XZ$3 1001dcf7 f   ClarkTests.obj
 0001:0001cd05       __ehhandler$??1GTest_CompareClarkDatabaseMetafiles@U2@@UAE@XZ 1001dd05 f   ClarkTests.obj
 0001:0001cd20       __unwindfunclet$??_GGTest_CompareClarkDatabaseMetafiles@U2@@UAEPAXI@Z$0 1001dd20 f   ClarkTests.obj
 0001:0001cd29       __unwindfunclet$??_GGTest_CompareClarkDatabaseMetafiles@U2@@UAEPAXI@Z$1 1001dd29 f   ClarkTests.obj
 0001:0001cd38       __unwindfunclet$??_GGTest_CompareClarkDatabaseMetafiles@U2@@UAEPAXI@Z$2 1001dd38 f   ClarkTests.obj
 0001:0001cd47       __unwindfunclet$??_GGTest_CompareClarkDatabaseMetafiles@U2@@UAEPAXI@Z$3 1001dd47 f   ClarkTests.obj
 0001:0001cd55       __ehhandler$??_GGTest_CompareClarkDatabaseMetafiles@U2@@UAEPAXI@Z 1001dd55 f   ClarkTests.obj
 0001:0001cd70       __unwindfunclet$??__E?DATABASE_METAFILES@GTest_CompareClarkDatabaseMetafiles@U2@@0VQStringList@@B@@YAXXZ$0 1001dd70 f   ClarkTests.obj
 0001:0001cd79       __unwindfunclet$??__E?DATABASE_METAFILES@GTest_CompareClarkDatabaseMetafiles@U2@@0VQStringList@@B@@YAXXZ$1 1001dd79 f   ClarkTests.obj
 0001:0001cd82       __unwindfunclet$??__E?DATABASE_METAFILES@GTest_CompareClarkDatabaseMetafiles@U2@@0VQStringList@@B@@YAXXZ$2 1001dd82 f   ClarkTests.obj
 0001:0001cd8b       __unwindfunclet$??__E?DATABASE_METAFILES@GTest_CompareClarkDatabaseMetafiles@U2@@0VQStringList@@B@@YAXXZ$3 1001dd8b f   ClarkTests.obj
 0001:0001cd94       __unwindfunclet$??__E?DATABASE_METAFILES@GTest_CompareClarkDatabaseMetafiles@U2@@0VQStringList@@B@@YAXXZ$4 1001dd94 f   ClarkTests.obj
 0001:0001cd9d       __unwindfunclet$??__E?DATABASE_METAFILES@GTest_CompareClarkDatabaseMetafiles@U2@@0VQStringList@@B@@YAXXZ$6 1001dd9d f   ClarkTests.obj
 0001:0001cdb1       __ehhandler$??__E?DATABASE_METAFILES@GTest_CompareClarkDatabaseMetafiles@U2@@0VQStringList@@B@@YAXXZ 1001ddb1 f   ClarkTests.obj
 0001:0001cde0       __unwindfunclet$??__EalgoLog@U2@@YAXXZ$0 1001dde0 f   ClarkTests.obj
 0001:0001cde9       __ehhandler$??__EalgoLog@U2@@YAXXZ 1001dde9 f   ClarkTests.obj
 0001:0001ce10       __unwindfunclet$??__EcmdLog@U2@@YAXXZ$0 1001de10 f   ClarkTests.obj
 0001:0001ce19       __ehhandler$??__EcmdLog@U2@@YAXXZ 1001de19 f   ClarkTests.obj
 0001:0001ce40       __unwindfunclet$??__EcoreLog@U2@@YAXXZ$0 1001de40 f   ClarkTests.obj
 0001:0001ce49       __ehhandler$??__EcoreLog@U2@@YAXXZ 1001de49 f   ClarkTests.obj
 0001:0001ce70       __unwindfunclet$??__EioLog@U2@@YAXXZ$0 1001de70 f   ClarkTests.obj
 0001:0001ce79       __ehhandler$??__EioLog@U2@@YAXXZ 1001de79 f   ClarkTests.obj
 0001:0001cea0       __unwindfunclet$??__EperfLog@U2@@YAXXZ$0 1001dea0 f   ClarkTests.obj
 0001:0001cea9       __ehhandler$??__EperfLog@U2@@YAXXZ 1001dea9 f   ClarkTests.obj
 0001:0001ced0       __unwindfunclet$??__EscriptLog@U2@@YAXXZ$0 1001ded0 f   ClarkTests.obj
 0001:0001ced9       __ehhandler$??__EscriptLog@U2@@YAXXZ 1001ded9 f   ClarkTests.obj
 0001:0001cf00       __unwindfunclet$??__EtaskLog@U2@@YAXXZ$0 1001df00 f   ClarkTests.obj
 0001:0001cf09       __ehhandler$??__EtaskLog@U2@@YAXXZ 1001df09 f   ClarkTests.obj
 0001:0001cf30       __unwindfunclet$??__EuiLog@U2@@YAXXZ$0 1001df30 f   ClarkTests.obj
 0001:0001cf39       __ehhandler$??__EuiLog@U2@@YAXXZ 1001df39 f   ClarkTests.obj
 0001:0001cf60       __unwindfunclet$??__EuserActLog@U2@@YAXXZ$0 1001df60 f   ClarkTests.obj
 0001:0001cf69       __ehhandler$??__EuserActLog@U2@@YAXXZ 1001df69 f   ClarkTests.obj
 0001:0001cf90       __ehhandler$?append@?$QList@PAVXMLTestFactory@U2@@@@QAEXABQAVXMLTestFactory@U2@@@Z 1001df90 f   ClarkTests.obj
 0001:0001cfb0       __unwindfunclet$?createFactory@GTest_CompareClarkDatabaseMetafiles@U2@@SAPAVXMLTestFactory@2@XZ$0 1001dfb0 f   ClarkTests.obj
 0001:0001cfbb       __unwindfunclet$?createFactory@GTest_CompareClarkDatabaseMetafiles@U2@@SAPAVXMLTestFactory@2@XZ$1 1001dfbb f   ClarkTests.obj
 0001:0001cfc4       __unwindfunclet$?createFactory@GTest_CompareClarkDatabaseMetafiles@U2@@SAPAVXMLTestFactory@2@XZ$2 1001dfc4 f   ClarkTests.obj
 0001:0001cfcd       __ehhandler$?createFactory@GTest_CompareClarkDatabaseMetafiles@U2@@SAPAVXMLTestFactory@2@XZ 1001dfcd f   ClarkTests.obj
 0001:0001cff0       __unwindfunclet$?createTest@GTest_CompareClarkDatabaseMetafilesFactory@GTest_CompareClarkDatabaseMetafiles@U2@@UAEPAVGTest@3@PAVXMLTestFormat@3@ABVQString@@PAV43@PBVGTestEnvironment@3@ABV?$QList@PAVGTest@U2@@@@ABVQDomElement@@@Z$0 1001dff0 f   ClarkTests.obj
 0001:0001cffb       __ehhandler$?createTest@GTest_CompareClarkDatabaseMetafilesFactory@GTest_CompareClarkDatabaseMetafiles@U2@@UAEPAVGTest@3@PAVXMLTestFormat@3@ABVQString@@PAV43@PBVGTestEnvironment@3@ABV?$QList@PAVGTest@U2@@@@ABVQDomElement@@@Z 1001dffb f   ClarkTests.obj
 0001:0001d020       __ehhandler$?detach_helper@?$QList@PAVXMLTestFactory@U2@@@@AAEXH@Z 1001e020 f   ClarkTests.obj
 0001:0001d040       __ehhandler$?detach_helper_grow@?$QList@PAVXMLTestFactory@U2@@@@AAEPAUNode@1@HH@Z 1001e040 f   ClarkTests.obj
 0001:0001d060       __unwindfunclet$?init@GTest_CompareClarkDatabaseMetafiles@U2@@QAEXPAVXMLTestFormat@2@ABVQDomElement@@@Z$0 1001e060 f   ClarkTests.obj
 0001:0001d069       __unwindfunclet$?init@GTest_CompareClarkDatabaseMetafiles@U2@@QAEXPAVXMLTestFormat@2@ABVQDomElement@@@Z$1 1001e069 f   ClarkTests.obj
 0001:0001d072       __unwindfunclet$?init@GTest_CompareClarkDatabaseMetafiles@U2@@QAEXPAVXMLTestFormat@2@ABVQDomElement@@@Z$2 1001e072 f   ClarkTests.obj
 0001:0001d07b       __unwindfunclet$?init@GTest_CompareClarkDatabaseMetafiles@U2@@QAEXPAVXMLTestFormat@2@ABVQDomElement@@@Z$3 1001e07b f   ClarkTests.obj
 0001:0001d084       __unwindfunclet$?init@GTest_CompareClarkDatabaseMetafiles@U2@@QAEXPAVXMLTestFormat@2@ABVQDomElement@@@Z$4 1001e084 f   ClarkTests.obj
 0001:0001d08d       __unwindfunclet$?init@GTest_CompareClarkDatabaseMetafiles@U2@@QAEXPAVXMLTestFormat@2@ABVQDomElement@@@Z$5 1001e08d f   ClarkTests.obj
 0001:0001d096       __unwindfunclet$?init@GTest_CompareClarkDatabaseMetafiles@U2@@QAEXPAVXMLTestFormat@2@ABVQDomElement@@@Z$6 1001e096 f   ClarkTests.obj
 0001:0001d09f       __unwindfunclet$?init@GTest_CompareClarkDatabaseMetafiles@U2@@QAEXPAVXMLTestFormat@2@ABVQDomElement@@@Z$7 1001e09f f   ClarkTests.obj
 0001:0001d0a8       __unwindfunclet$?init@GTest_CompareClarkDatabaseMetafiles@U2@@QAEXPAVXMLTestFormat@2@ABVQDomElement@@@Z$8 1001e0a8 f   ClarkTests.obj
 0001:0001d0b0       __unwindfunclet$?init@GTest_CompareClarkDatabaseMetafiles@U2@@QAEXPAVXMLTestFormat@2@ABVQDomElement@@@Z$9 1001e0b0 f   ClarkTests.obj
 0001:0001d0b8       __unwindfunclet$?init@GTest_CompareClarkDatabaseMetafiles@U2@@QAEXPAVXMLTestFormat@2@ABVQDomElement@@@Z$10 1001e0b8 f   ClarkTests.obj
 0001:0001d0c1       __unwindfunclet$?init@GTest_CompareClarkDatabaseMetafiles@U2@@QAEXPAVXMLTestFormat@2@ABVQDomElement@@@Z$11 1001e0c1 f   ClarkTests.obj
 0001:0001d0ca       __unwindfunclet$?init@GTest_CompareClarkDatabaseMetafiles@U2@@QAEXPAVXMLTestFormat@2@ABVQDomElement@@@Z$12 1001e0ca f   ClarkTests.obj
 0001:0001d0d3       __unwindfunclet$?init@GTest_CompareClarkDatabaseMetafiles@U2@@QAEXPAVXMLTestFormat@2@ABVQDomElement@@@Z$13 1001e0d3 f   ClarkTests.obj
 0001:0001d0db       __unwindfunclet$?init@GTest_CompareClarkDatabaseMetafiles@U2@@QAEXPAVXMLTestFormat@2@ABVQDomElement@@@Z$14 1001e0db f   ClarkTests.obj
 0001:0001d0e3       __unwindfunclet$?init@GTest_CompareClarkDatabaseMetafiles@U2@@QAEXPAVXMLTestFormat@2@ABVQDomElement@@@Z$15 1001e0e3 f   ClarkTests.obj
 0001:0001d0ec       __ehhandler$?init@GTest_CompareClarkDatabaseMetafiles@U2@@QAEXPAVXMLTestFormat@2@ABVQDomElement@@@Z 1001e0ec f   ClarkTests.obj
 0001:0001d110       __unwindfunclet$?report@GTest_CompareClarkDatabaseMetafiles@U2@@EAE?AW4ReportResult@Task@2@XZ$0 1001e110 f   ClarkTests.obj
 0001:0001d119       __unwindfunclet$?report@GTest_CompareClarkDatabaseMetafiles@U2@@EAE?AW4ReportResult@Task@2@XZ$1 1001e119 f   ClarkTests.obj
 0001:0001d122       __unwindfunclet$?report@GTest_CompareClarkDatabaseMetafiles@U2@@EAE?AW4ReportResult@Task@2@XZ$2 1001e122 f   ClarkTests.obj
 0001:0001d12b       __unwindfunclet$?report@GTest_CompareClarkDatabaseMetafiles@U2@@EAE?AW4ReportResult@Task@2@XZ$3 1001e12b f   ClarkTests.obj
 0001:0001d134       __unwindfunclet$?report@GTest_CompareClarkDatabaseMetafiles@U2@@EAE?AW4ReportResult@Task@2@XZ$4 1001e134 f   ClarkTests.obj
 0001:0001d13d       __unwindfunclet$?report@GTest_CompareClarkDatabaseMetafiles@U2@@EAE?AW4ReportResult@Task@2@XZ$5 1001e13d f   ClarkTests.obj
 0001:0001d146       __unwindfunclet$?report@GTest_CompareClarkDatabaseMetafiles@U2@@EAE?AW4ReportResult@Task@2@XZ$6 1001e146 f   ClarkTests.obj
 0001:0001d14f       __unwindfunclet$?report@GTest_CompareClarkDatabaseMetafiles@U2@@EAE?AW4ReportResult@Task@2@XZ$7 1001e14f f   ClarkTests.obj
 0001:0001d158       __unwindfunclet$?report@GTest_CompareClarkDatabaseMetafiles@U2@@EAE?AW4ReportResult@Task@2@XZ$8 1001e158 f   ClarkTests.obj
 0001:0001d161       __unwindfunclet$?report@GTest_CompareClarkDatabaseMetafiles@U2@@EAE?AW4ReportResult@Task@2@XZ$9 1001e161 f   ClarkTests.obj
 0001:0001d16a       __unwindfunclet$?report@GTest_CompareClarkDatabaseMetafiles@U2@@EAE?AW4ReportResult@Task@2@XZ$10 1001e16a f   ClarkTests.obj
 0001:0001d172       __unwindfunclet$?report@GTest_CompareClarkDatabaseMetafiles@U2@@EAE?AW4ReportResult@Task@2@XZ$11 1001e172 f   ClarkTests.obj
 0001:0001d17b       __unwindfunclet$?report@GTest_CompareClarkDatabaseMetafiles@U2@@EAE?AW4ReportResult@Task@2@XZ$12 1001e17b f   ClarkTests.obj
 0001:0001d184       __unwindfunclet$?report@GTest_CompareClarkDatabaseMetafiles@U2@@EAE?AW4ReportResult@Task@2@XZ$13 1001e184 f   ClarkTests.obj
 0001:0001d18d       __unwindfunclet$?report@GTest_CompareClarkDatabaseMetafiles@U2@@EAE?AW4ReportResult@Task@2@XZ$17 1001e18d f   ClarkTests.obj
 0001:0001d196       __unwindfunclet$?report@GTest_CompareClarkDatabaseMetafiles@U2@@EAE?AW4ReportResult@Task@2@XZ$18 1001e196 f   ClarkTests.obj
 0001:0001d1a2       __unwindfunclet$?report@GTest_CompareClarkDatabaseMetafiles@U2@@EAE?AW4ReportResult@Task@2@XZ$19 1001e1a2 f   ClarkTests.obj
 0001:0001d1ab       __unwindfunclet$?report@GTest_CompareClarkDatabaseMetafiles@U2@@EAE?AW4ReportResult@Task@2@XZ$20 1001e1ab f   ClarkTests.obj
 0001:0001d1b4       __unwindfunclet$?report@GTest_CompareClarkDatabaseMetafiles@U2@@EAE?AW4ReportResult@Task@2@XZ$24 1001e1b4 f   ClarkTests.obj
 0001:0001d1bd       __unwindfunclet$?report@GTest_CompareClarkDatabaseMetafiles@U2@@EAE?AW4ReportResult@Task@2@XZ$25 1001e1bd f   ClarkTests.obj
 0001:0001d1c6       __unwindfunclet$?report@GTest_CompareClarkDatabaseMetafiles@U2@@EAE?AW4ReportResult@Task@2@XZ$26 1001e1c6 f   ClarkTests.obj
 0001:0001d1d1       __unwindfunclet$?report@GTest_CompareClarkDatabaseMetafiles@U2@@EAE?AW4ReportResult@Task@2@XZ$27 1001e1d1 f   ClarkTests.obj
 0001:0001d1da       __unwindfunclet$?report@GTest_CompareClarkDatabaseMetafiles@U2@@EAE?AW4ReportResult@Task@2@XZ$28 1001e1da f   ClarkTests.obj
 0001:0001d1e2       __unwindfunclet$?report@GTest_CompareClarkDatabaseMetafiles@U2@@EAE?AW4ReportResult@Task@2@XZ$29 1001e1e2 f   ClarkTests.obj
 0001:0001d1eb       __unwindfunclet$?report@GTest_CompareClarkDatabaseMetafiles@U2@@EAE?AW4ReportResult@Task@2@XZ$30 1001e1eb f   ClarkTests.obj
 0001:0001d1f4       __unwindfunclet$?report@GTest_CompareClarkDatabaseMetafiles@U2@@EAE?AW4ReportResult@Task@2@XZ$31 1001e1f4 f   ClarkTests.obj
 0001:0001d1fd       __unwindfunclet$?report@GTest_CompareClarkDatabaseMetafiles@U2@@EAE?AW4ReportResult@Task@2@XZ$32 1001e1fd f   ClarkTests.obj
 0001:0001d206       __unwindfunclet$?report@GTest_CompareClarkDatabaseMetafiles@U2@@EAE?AW4ReportResult@Task@2@XZ$33 1001e206 f   ClarkTests.obj
 0001:0001d212       __unwindfunclet$?report@GTest_CompareClarkDatabaseMetafiles@U2@@EAE?AW4ReportResult@Task@2@XZ$34 1001e212 f   ClarkTests.obj
 0001:0001d21e       __unwindfunclet$?report@GTest_CompareClarkDatabaseMetafiles@U2@@EAE?AW4ReportResult@Task@2@XZ$35 1001e21e f   ClarkTests.obj
 0001:0001d227       __unwindfunclet$?report@GTest_CompareClarkDatabaseMetafiles@U2@@EAE?AW4ReportResult@Task@2@XZ$36 1001e227 f   ClarkTests.obj
 0001:0001d230       __unwindfunclet$?report@GTest_CompareClarkDatabaseMetafiles@U2@@EAE?AW4ReportResult@Task@2@XZ$37 1001e230 f   ClarkTests.obj
 0001:0001d239       __unwindfunclet$?report@GTest_CompareClarkDatabaseMetafiles@U2@@EAE?AW4ReportResult@Task@2@XZ$21 1001e239 f   ClarkTests.obj
 0001:0001d242       __unwindfunclet$?report@GTest_CompareClarkDatabaseMetafiles@U2@@EAE?AW4ReportResult@Task@2@XZ$22 1001e242 f   ClarkTests.obj
 0001:0001d24b       __unwindfunclet$?report@GTest_CompareClarkDatabaseMetafiles@U2@@EAE?AW4ReportResult@Task@2@XZ$23 1001e24b f   ClarkTests.obj
 0001:0001d254       __unwindfunclet$?report@GTest_CompareClarkDatabaseMetafiles@U2@@EAE?AW4ReportResult@Task@2@XZ$14 1001e254 f   ClarkTests.obj
 0001:0001d25d       __unwindfunclet$?report@GTest_CompareClarkDatabaseMetafiles@U2@@EAE?AW4ReportResult@Task@2@XZ$15 1001e25d f   ClarkTests.obj
 0001:0001d266       __unwindfunclet$?report@GTest_CompareClarkDatabaseMetafiles@U2@@EAE?AW4ReportResult@Task@2@XZ$16 1001e266 f   ClarkTests.obj
 0001:0001d26f       __ehhandler$?report@GTest_CompareClarkDatabaseMetafiles@U2@@EAE?AW4ReportResult@Task@2@XZ 1001e26f f   ClarkTests.obj
 0001:0001d290       __unwindfunclet$??__EalgoLog@U2@@YAXXZ$0 1001e290 f   moc_ClarkBuildWorker.obj
 0001:0001d299       __ehhandler$??__EalgoLog@U2@@YAXXZ 1001e299 f   moc_ClarkBuildWorker.obj
 0001:0001d2c0       __unwindfunclet$??__EcmdLog@U2@@YAXXZ$0 1001e2c0 f   moc_ClarkBuildWorker.obj
 0001:0001d2c9       __ehhandler$??__EcmdLog@U2@@YAXXZ 1001e2c9 f   moc_ClarkBuildWorker.obj
 0001:0001d2f0       __unwindfunclet$??__EcoreLog@U2@@YAXXZ$0 1001e2f0 f   moc_ClarkBuildWorker.obj
 0001:0001d2f9       __ehhandler$??__EcoreLog@U2@@YAXXZ 1001e2f9 f   moc_ClarkBuildWorker.obj
 0001:0001d320       __unwindfunclet$??__EioLog@U2@@YAXXZ$0 1001e320 f   moc_ClarkBuildWorker.obj
 0001:0001d329       __ehhandler$??__EioLog@U2@@YAXXZ 1001e329 f   moc_ClarkBuildWorker.obj
 0001:0001d350       __unwindfunclet$??__EperfLog@U2@@YAXXZ$0 1001e350 f   moc_ClarkBuildWorker.obj
 0001:0001d359       __ehhandler$??__EperfLog@U2@@YAXXZ 1001e359 f   moc_ClarkBuildWorker.obj
 0001:0001d380       __unwindfunclet$??__EscriptLog@U2@@YAXXZ$0 1001e380 f   moc_ClarkBuildWorker.obj
 0001:0001d389       __ehhandler$??__EscriptLog@U2@@YAXXZ 1001e389 f   moc_ClarkBuildWorker.obj
 0001:0001d3b0       __unwindfunclet$??__EtaskLog@U2@@YAXXZ$0 1001e3b0 f   moc_ClarkBuildWorker.obj
 0001:0001d3b9       __ehhandler$??__EtaskLog@U2@@YAXXZ 1001e3b9 f   moc_ClarkBuildWorker.obj
 0001:0001d3e0       __unwindfunclet$??__EuiLog@U2@@YAXXZ$0 1001e3e0 f   moc_ClarkBuildWorker.obj
 0001:0001d3e9       __ehhandler$??__EuiLog@U2@@YAXXZ 1001e3e9 f   moc_ClarkBuildWorker.obj
 0001:0001d410       __unwindfunclet$??__EuserActLog@U2@@YAXXZ$0 1001e410 f   moc_ClarkBuildWorker.obj
 0001:0001d419       __ehhandler$??__EuserActLog@U2@@YAXXZ 1001e419 f   moc_ClarkBuildWorker.obj
 0001:0001d440       __unwindfunclet$?qt_metatype_id@?$QMetaTypeIdQObject@PAVTask@U2@@$00@@SAHXZ$0 1001e440 f   moc_ClarkBuildWorker.obj
 0001:0001d449       __ehhandler$?qt_metatype_id@?$QMetaTypeIdQObject@PAVTask@U2@@$00@@SAHXZ 1001e449 f   moc_ClarkBuildWorker.obj
 0001:0001d470       __unwindfunclet$??__EalgoLog@U2@@YAXXZ$0 1001e470 f   moc_ClarkClassifyWorker.obj
 0001:0001d479       __ehhandler$??__EalgoLog@U2@@YAXXZ 1001e479 f   moc_ClarkClassifyWorker.obj
 0001:0001d4a0       __unwindfunclet$??__EcmdLog@U2@@YAXXZ$0 1001e4a0 f   moc_ClarkClassifyWorker.obj
 0001:0001d4a9       __ehhandler$??__EcmdLog@U2@@YAXXZ 1001e4a9 f   moc_ClarkClassifyWorker.obj
 0001:0001d4d0       __unwindfunclet$??__EcoreLog@U2@@YAXXZ$0 1001e4d0 f   moc_ClarkClassifyWorker.obj
 0001:0001d4d9       __ehhandler$??__EcoreLog@U2@@YAXXZ 1001e4d9 f   moc_ClarkClassifyWorker.obj
 0001:0001d500       __unwindfunclet$??__EioLog@U2@@YAXXZ$0 1001e500 f   moc_ClarkClassifyWorker.obj
 0001:0001d509       __ehhandler$??__EioLog@U2@@YAXXZ 1001e509 f   moc_ClarkClassifyWorker.obj
 0001:0001d530       __unwindfunclet$??__EperfLog@U2@@YAXXZ$0 1001e530 f   moc_ClarkClassifyWorker.obj
 0001:0001d539       __ehhandler$??__EperfLog@U2@@YAXXZ 1001e539 f   moc_ClarkClassifyWorker.obj
 0001:0001d560       __unwindfunclet$??__EscriptLog@U2@@YAXXZ$0 1001e560 f   moc_ClarkClassifyWorker.obj
 0001:0001d569       __ehhandler$??__EscriptLog@U2@@YAXXZ 1001e569 f   moc_ClarkClassifyWorker.obj
 0001:0001d590       __unwindfunclet$??__EtaskLog@U2@@YAXXZ$0 1001e590 f   moc_ClarkClassifyWorker.obj
 0001:0001d599       __ehhandler$??__EtaskLog@U2@@YAXXZ 1001e599 f   moc_ClarkClassifyWorker.obj
 0001:0001d5c0       __unwindfunclet$??__EuiLog@U2@@YAXXZ$0 1001e5c0 f   moc_ClarkClassifyWorker.obj
 0001:0001d5c9       __ehhandler$??__EuiLog@U2@@YAXXZ 1001e5c9 f   moc_ClarkClassifyWorker.obj
 0001:0001d5f0       __unwindfunclet$??__EuserActLog@U2@@YAXXZ$0 1001e5f0 f   moc_ClarkClassifyWorker.obj
 0001:0001d5f9       __ehhandler$??__EuserActLog@U2@@YAXXZ 1001e5f9 f   moc_ClarkClassifyWorker.obj
 0001:0001d620       ??__F?ACTOR_ID@ClarkBuildWorkerFactory@LocalWorkflow@U2@@0VQString@@B@@YAXXZ 1001e620 f   ClarkBuildWorker.obj
 0001:0001d630       ??__F?_Generic_object@?$_Error_objects@H@std@@2V_Generic_error_category@2@A@@YAXXZ 1001e630 f   ClarkBuildWorker.obj
 0001:0001d640       ??__F?_Iostream_object@?$_Error_objects@H@std@@2V_Iostream_error_category@2@A@@YAXXZ 1001e640 f   ClarkBuildWorker.obj
 0001:0001d650       ??__F?_System_object@?$_Error_objects@H@std@@2V_System_error_category@2@A@@YAXXZ 1001e650 f   ClarkBuildWorker.obj
 0001:0001d660       ??__F?wellKnownErrors@ClarkBuildLogParser@LocalWorkflow@U2@@0VQStringList@@B@@YAXXZ 1001e660 f   ClarkBuildWorker.obj
 0001:0001d670       ??__FDB_URL@LocalWorkflow@U2@@YAXXZ 1001e670 f   ClarkBuildWorker.obj
 0001:0001d680       ??__FGENOMIC_LIBRARY@LocalWorkflow@U2@@YAXXZ 1001e680 f   ClarkBuildWorker.obj
 0001:0001d690       ??__FOUTPUT_PORT@LocalWorkflow@U2@@YAXXZ 1001e690 f   ClarkBuildWorker.obj
 0001:0001d6a0       ??__FTAXONOMY_RANK@LocalWorkflow@U2@@YAXXZ 1001e6a0 f   ClarkBuildWorker.obj
 0001:0001d6b0       ??__FalgoLog@U2@@YAXXZ     1001e6b0 f   ClarkBuildWorker.obj
 0001:0001d6c0       ??__FcmdLog@U2@@YAXXZ      1001e6c0 f   ClarkBuildWorker.obj
 0001:0001d6d0       ??__FcoreLog@U2@@YAXXZ     1001e6d0 f   ClarkBuildWorker.obj
 0001:0001d6e0       ??__Fcvar@?1???0ClarkBuildTask@LocalWorkflow@U2@@QAE@ABVQString@@ABVQStringList@@H0@Z@YAXXZ 1001e6e0 f   ClarkBuildWorker.obj
 0001:0001d6f0       ??__FioLog@U2@@YAXXZ       1001e6f0 f   ClarkBuildWorker.obj
 0001:0001d700       ??__FperfLog@U2@@YAXXZ     1001e700 f   ClarkBuildWorker.obj
 0001:0001d710       ??__FscriptLog@U2@@YAXXZ   1001e710 f   ClarkBuildWorker.obj
 0001:0001d720       ??__FtaskLog@U2@@YAXXZ     1001e720 f   ClarkBuildWorker.obj
 0001:0001d730       ??__FuiLog@U2@@YAXXZ       1001e730 f   ClarkBuildWorker.obj
 0001:0001d740       ??__FuserActLog@U2@@YAXXZ  1001e740 f   ClarkBuildWorker.obj
 0001:0001d750       ??__F?ACTOR_ID@ClarkClassifyWorkerFactory@LocalWorkflow@U2@@2VQString@@B@@YAXXZ 1001e750 f   ClarkClassifyWorker.obj
 0001:0001d760       ??__F?DB_TO_RAM@ClarkClassifyWorkerFactory@LocalWorkflow@U2@@2VQString@@B@@YAXXZ 1001e760 f   ClarkClassifyWorker.obj
 0001:0001d770       ??__F?DB_URL@ClarkClassifyWorkerFactory@LocalWorkflow@U2@@2VQString@@B@@YAXXZ 1001e770 f   ClarkClassifyWorker.obj
 0001:0001d780       ??__F?EXTEND_OUT@ClarkClassifyWorkerFactory@LocalWorkflow@U2@@2VQString@@B@@YAXXZ 1001e780 f   ClarkClassifyWorker.obj
 0001:0001d790       ??__F?FACTOR@ClarkClassifyWorkerFactory@LocalWorkflow@U2@@2VQString@@B@@YAXXZ 1001e790 f   ClarkClassifyWorker.obj
 0001:0001d7a0       ??__F?GAP@ClarkClassifyWorkerFactory@LocalWorkflow@U2@@2VQString@@B@@YAXXZ 1001e7a0 f   ClarkClassifyWorker.obj
 0001:0001d7b0       ??__F?INPUT_PORT@ClarkClassifyWorkerFactory@LocalWorkflow@U2@@2VQString@@B@@YAXXZ 1001e7b0 f   ClarkClassifyWorker.obj
 0001:0001d7c0       ??__F?INPUT_SLOT@ClarkClassifyWorkerFactory@LocalWorkflow@U2@@2VQString@@B@@YAXXZ 1001e7c0 f   ClarkClassifyWorker.obj
 0001:0001d7d0       ??__F?K_LENGTH@ClarkClassifyWorkerFactory@LocalWorkflow@U2@@2VQString@@B@@YAXXZ 1001e7d0 f   ClarkClassifyWorker.obj
 0001:0001d7e0       ??__F?K_MIN_FREQ@ClarkClassifyWorkerFactory@LocalWorkflow@U2@@2VQString@@B@@YAXXZ 1001e7e0 f   ClarkClassifyWorker.obj
 0001:0001d7f0       ??__F?MODE@ClarkClassifyWorkerFactory@LocalWorkflow@U2@@2VQString@@B@@YAXXZ 1001e7f0 f   ClarkClassifyWorker.obj
 0001:0001d800       ??__F?NUM_THREADS@ClarkClassifyWorkerFactory@LocalWorkflow@U2@@2VQString@@B@@YAXXZ 1001e800 f   ClarkClassifyWorker.obj
 0001:0001d810       ??__F?OUTPUT_PORT@ClarkClassifyWorkerFactory@LocalWorkflow@U2@@2VQString@@B@@YAXXZ 1001e810 f   ClarkClassifyWorker.obj
 0001:0001d820       ??__F?OUTPUT_URL@ClarkClassifyWorkerFactory@LocalWorkflow@U2@@2VQString@@B@@YAXXZ 1001e820 f   ClarkClassifyWorker.obj
 0001:0001d830       ??__F?PAIRED_END@ClarkClassifyWorkerFactory@LocalWorkflow@U2@@2VQString@@B@@YAXXZ 1001e830 f   ClarkClassifyWorker.obj
 0001:0001d840       ??__F?PAIRED_INPUT_PORT@ClarkClassifyWorkerFactory@LocalWorkflow@U2@@2VQString@@B@@YAXXZ 1001e840 f   ClarkClassifyWorker.obj
 0001:0001d850       ??__F?PAIRED_INPUT_SLOT@ClarkClassifyWorkerFactory@LocalWorkflow@U2@@2VQString@@B@@YAXXZ 1001e850 f   ClarkClassifyWorker.obj
 0001:0001d860       ??__F?SEQUENCING_READS@ClarkClassifyWorkerFactory@LocalWorkflow@U2@@2VQString@@B@@YAXXZ 1001e860 f   ClarkClassifyWorker.obj
 0001:0001d870       ??__F?SINGLE_END@ClarkClassifyWorkerFactory@LocalWorkflow@U2@@2VQString@@B@@YAXXZ 1001e870 f   ClarkClassifyWorker.obj
 0001:0001d880       ??__F?TAXONOMY@ClarkClassifyWorkerFactory@LocalWorkflow@U2@@2VQString@@B@@YAXXZ 1001e880 f   ClarkClassifyWorker.obj
 0001:0001d890       ??__F?TAXONOMY_RANK@ClarkClassifyWorkerFactory@LocalWorkflow@U2@@2VQString@@B@@YAXXZ 1001e890 f   ClarkClassifyWorker.obj
 0001:0001d8a0       ??__F?TOOL_DEFAULT@ClarkClassifySettings@LocalWorkflow@U2@@2VQString@@B@@YAXXZ 1001e8a0 f   ClarkClassifyWorker.obj
 0001:0001d8b0       ??__F?TOOL_LIGHT@ClarkClassifySettings@LocalWorkflow@U2@@2VQString@@B@@YAXXZ 1001e8b0 f   ClarkClassifyWorker.obj
 0001:0001d8c0       ??__F?TOOL_VARIANT@ClarkClassifyWorkerFactory@LocalWorkflow@U2@@2VQString@@B@@YAXXZ 1001e8c0 f   ClarkClassifyWorker.obj
 0001:0001d8d0       ??__F?WORKFLOW_CLASSIFY_TOOL_CLARK@ClarkClassifyWorkerFactory@LocalWorkflow@U2@@2VQString@@B@@YAXXZ 1001e8d0 f   ClarkClassifyWorker.obj
 0001:0001d8e0       ??__F?_Generic_object@?$_Error_objects@H@std@@2V_Generic_error_category@2@A@@YAXXZ 1001e8e0 f   ClarkClassifyWorker.obj
 0001:0001d8f0       ??__F?_Iostream_object@?$_Error_objects@H@std@@2V_Iostream_error_category@2@A@@YAXXZ 1001e8f0 f   ClarkClassifyWorker.obj
 0001:0001d900       ??__F?_System_object@?$_Error_objects@H@std@@2V_System_error_category@2@A@@YAXXZ 1001e900 f   ClarkClassifyWorker.obj
 0001:0001d910       ??__F?wellKnownErrors@ClarkLogParser@LocalWorkflow@U2@@0V?$QMap@VQString@@V1@@@B@@YAXXZ 1001e910 f   ClarkClassifyWorker.obj
 0001:0001d960       ??__FEXTENDED_REPORT_SUFFIX@LocalWorkflow@U2@@YAXXZ 1001e960 f   ClarkClassifyWorker.obj
 0001:0001d970       ??__FREPORT_PREFIX@LocalWorkflow@U2@@YAXXZ 1001e970 f   ClarkClassifyWorker.obj
 0001:0001d980       ??__FalgoLog@U2@@YAXXZ     1001e980 f   ClarkClassifyWorker.obj
 0001:0001d990       ??__FcmdLog@U2@@YAXXZ      1001e990 f   ClarkClassifyWorker.obj
 0001:0001d9a0       ??__FcoreLog@U2@@YAXXZ     1001e9a0 f   ClarkClassifyWorker.obj
 0001:0001d9b0       ??__Fcvar@?1???0ClarkClassifyTask@LocalWorkflow@U2@@QAE@ABVClarkClassifySettings@12@ABVQString@@11@Z@YAXXZ 1001e9b0 f   ClarkClassifyWorker.obj
 0001:0001d9e0       ??__FioLog@U2@@YAXXZ       1001e9e0 f   ClarkClassifyWorker.obj
 0001:0001d9f0       ??__FperfLog@U2@@YAXXZ     1001e9f0 f   ClarkClassifyWorker.obj
 0001:0001da00       ??__FscriptLog@U2@@YAXXZ   1001ea00 f   ClarkClassifyWorker.obj
 0001:0001da10       ??__FtaskLog@U2@@YAXXZ     1001ea10 f   ClarkClassifyWorker.obj
 0001:0001da20       ??__FuiLog@U2@@YAXXZ       1001ea20 f   ClarkClassifyWorker.obj
 0001:0001da30       ??__FuserActLog@U2@@YAXXZ  1001ea30 f   ClarkClassifyWorker.obj
 0001:0001da40       ??__F?CLARK_GROUP@ClarkSupport@U2@@2VQString@@B@@YAXXZ 1001ea40 f   ClarkSupport.obj
 0001:0001da50       ??__F?ET_CLARK@ClarkSupport@U2@@2VQString@@B@@YAXXZ 1001ea50 f   ClarkSupport.obj
 0001:0001da60       ??__F?ET_CLARK_BUILD_SCRIPT@ClarkSupport@U2@@2VQString@@B@@YAXXZ 1001ea60 f   ClarkSupport.obj
 0001:0001da70       ??__F?ET_CLARK_BUILD_SCRIPT_ID@ClarkSupport@U2@@2VQString@@B@@YAXXZ 1001ea70 f   ClarkSupport.obj
 0001:0001da80       ??__F?ET_CLARK_GET_ACCSSN_TAX_ID@ClarkSupport@U2@@2VQString@@B@@YAXXZ 1001ea80 f   ClarkSupport.obj
 0001:0001da90       ??__F?ET_CLARK_GET_ACCSSN_TAX_ID_ID@ClarkSupport@U2@@2VQString@@B@@YAXXZ 1001ea90 f   ClarkSupport.obj
 0001:0001daa0       ??__F?ET_CLARK_GET_FILES_TO_TAX_NODES@ClarkSupport@U2@@2VQString@@B@@YAXXZ 1001eaa0 f   ClarkSupport.obj
 0001:0001dab0       ??__F?ET_CLARK_GET_FILES_TO_TAX_NODES_ID@ClarkSupport@U2@@2VQString@@B@@YAXXZ 1001eab0 f   ClarkSupport.obj
 0001:0001dac0       ??__F?ET_CLARK_GET_TARGETS_DEF@ClarkSupport@U2@@2VQString@@B@@YAXXZ 1001eac0 f   ClarkSupport.obj
 0001:0001dad0       ??__F?ET_CLARK_GET_TARGETS_DEF_ID@ClarkSupport@U2@@2VQString@@B@@YAXXZ 1001ead0 f   ClarkSupport.obj
 0001:0001dae0       ??__F?ET_CLARK_ID@ClarkSupport@U2@@2VQString@@B@@YAXXZ 1001eae0 f   ClarkSupport.obj
 0001:0001daf0       ??__F?ET_CLARK_L@ClarkSupport@U2@@2VQString@@B@@YAXXZ 1001eaf0 f   ClarkSupport.obj
 0001:0001db00       ??__F?ET_CLARK_L_ID@ClarkSupport@U2@@2VQString@@B@@YAXXZ 1001eb00 f   ClarkSupport.obj
 0001:0001db10       ??__F?_Generic_object@?$_Error_objects@H@std@@2V_Generic_error_category@2@A@@YAXXZ 1001eb10 f   ClarkSupport.obj
 0001:0001db20       ??__F?_Iostream_object@?$_Error_objects@H@std@@2V_Iostream_error_category@2@A@@YAXXZ 1001eb20 f   ClarkSupport.obj
 0001:0001db30       ??__F?_System_object@?$_Error_objects@H@std@@2V_System_error_category@2@A@@YAXXZ 1001eb30 f   ClarkSupport.obj
 0001:0001db40       ??__FService_DNAExport@U2@@YAXXZ 1001eb40 f   ClarkSupport.obj
 0001:0001db50       ??__FService_DNAGraphPack@U2@@YAXXZ 1001eb50 f   ClarkSupport.obj
 0001:0001db60       ??__FService_ExternalToolSupport@U2@@YAXXZ 1001eb60 f   ClarkSupport.obj
 0001:0001db70       ??__FService_GUITesting@U2@@YAXXZ 1001eb70 f   ClarkSupport.obj
 0001:0001db80       ??__FService_MaxCoreServiceId@U2@@YAXXZ 1001eb80 f   ClarkSupport.obj
 0001:0001db90       ??__FService_MinCoreServiceId@U2@@YAXXZ 1001eb90 f   ClarkSupport.obj
 0001:0001dba0       ??__FService_PluginViewer@U2@@YAXXZ 1001eba0 f   ClarkSupport.obj
 0001:0001dbb0       ??__FService_Project@U2@@YAXXZ 1001ebb0 f   ClarkSupport.obj
 0001:0001dbc0       ??__FService_ProjectView@U2@@YAXXZ 1001ebc0 f   ClarkSupport.obj
 0001:0001dbd0       ??__FService_QueryDesigner@U2@@YAXXZ 1001ebd0 f   ClarkSupport.obj
 0001:0001dbe0       ??__FService_ScriptRegistry@U2@@YAXXZ 1001ebe0 f   ClarkSupport.obj
 0001:0001dbf0       ??__FService_TestRunner@U2@@YAXXZ 1001ebf0 f   ClarkSupport.obj
 0001:0001dc00       ??__FService_WorkflowDesigner@U2@@YAXXZ 1001ec00 f   ClarkSupport.obj
 0001:0001dc10       ??__FalgoLog@U2@@YAXXZ     1001ec10 f   ClarkSupport.obj
 0001:0001dc20       ??__FcmdLog@U2@@YAXXZ      1001ec20 f   ClarkSupport.obj
 0001:0001dc30       ??__FcoreLog@U2@@YAXXZ     1001ec30 f   ClarkSupport.obj
 0001:0001dc40       ??__FioLog@U2@@YAXXZ       1001ec40 f   ClarkSupport.obj
 0001:0001dc50       ??__FperfLog@U2@@YAXXZ     1001ec50 f   ClarkSupport.obj
 0001:0001dc60       ??__FscriptLog@U2@@YAXXZ   1001ec60 f   ClarkSupport.obj
 0001:0001dc70       ??__FtaskLog@U2@@YAXXZ     1001ec70 f   ClarkSupport.obj
 0001:0001dc80       ??__FuiLog@U2@@YAXXZ       1001ec80 f   ClarkSupport.obj
 0001:0001dc90       ??__FuserActLog@U2@@YAXXZ  1001ec90 f   ClarkSupport.obj
 0001:0001dca0       ??__F?PLUGIN_DESCRIPRION@ClarkSupportPlugin@U2@@2VQString@@B@@YAXXZ 1001eca0 f   ClarkSupportPlugin.obj
 0001:0001dcb0       ??__F?PLUGIN_NAME@ClarkSupportPlugin@U2@@2VQString@@B@@YAXXZ 1001ecb0 f   ClarkSupportPlugin.obj
 0001:0001dcc0       ??__F?_Generic_object@?$_Error_objects@H@std@@2V_Generic_error_category@2@A@@YAXXZ 1001ecc0 f   ClarkSupportPlugin.obj
 0001:0001dcd0       ??__F?_Iostream_object@?$_Error_objects@H@std@@2V_Iostream_error_category@2@A@@YAXXZ 1001ecd0 f   ClarkSupportPlugin.obj
 0001:0001dce0       ??__F?_System_object@?$_Error_objects@H@std@@2V_System_error_category@2@A@@YAXXZ 1001ece0 f   ClarkSupportPlugin.obj
 0001:0001dcf0       ??__FalgoLog@U2@@YAXXZ     1001ecf0 f   ClarkSupportPlugin.obj
 0001:0001dd00       ??__FcmdLog@U2@@YAXXZ      1001ed00 f   ClarkSupportPlugin.obj
 0001:0001dd10       ??__FcoreLog@U2@@YAXXZ     1001ed10 f   ClarkSupportPlugin.obj
 0001:0001dd20       ??__FioLog@U2@@YAXXZ       1001ed20 f   ClarkSupportPlugin.obj
 0001:0001dd30       ??__FperfLog@U2@@YAXXZ     1001ed30 f   ClarkSupportPlugin.obj
 0001:0001dd40       ??__FscriptLog@U2@@YAXXZ   1001ed40 f   ClarkSupportPlugin.obj
 0001:0001dd50       ??__FtaskLog@U2@@YAXXZ     1001ed50 f   ClarkSupportPlugin.obj
 0001:0001dd60       ??__FuiLog@U2@@YAXXZ       1001ed60 f   ClarkSupportPlugin.obj
 0001:0001dd70       ??__FuserActLog@U2@@YAXXZ  1001ed70 f   ClarkSupportPlugin.obj
 0001:0001dd80       ??__F?DATABASE1@GTest_CompareClarkDatabaseMetafiles@U2@@0VQString@@B@@YAXXZ 1001ed80 f   ClarkTests.obj
 0001:0001dd90       ??__F?DATABASE1_PREFIXES@GTest_CompareClarkDatabaseMetafiles@U2@@0VQString@@B@@YAXXZ 1001ed90 f   ClarkTests.obj
 0001:0001dda0       ??__F?DATABASE2@GTest_CompareClarkDatabaseMetafiles@U2@@0VQString@@B@@YAXXZ 1001eda0 f   ClarkTests.obj
 0001:0001ddb0       ??__F?DATABASE2_PREFIXES@GTest_CompareClarkDatabaseMetafiles@U2@@0VQString@@B@@YAXXZ 1001edb0 f   ClarkTests.obj
 0001:0001ddc0       ??__F?DATABASE_METAFILES@GTest_CompareClarkDatabaseMetafiles@U2@@0VQStringList@@B@@YAXXZ 1001edc0 f   ClarkTests.obj
 0001:0001ddd0       ??__F?DATABASE_PREFIX_PLACEHOLDER@GTest_CompareClarkDatabaseMetafiles@U2@@0VQString@@B@@YAXXZ 1001edd0 f   ClarkTests.obj
 0001:0001dde0       ??__F?PREFIXES_SEPARATOR@GTest_CompareClarkDatabaseMetafiles@U2@@0VQString@@B@@YAXXZ 1001ede0 f   ClarkTests.obj
 0001:0001ddf0       ??__F?_Generic_object@?$_Error_objects@H@std@@2V_Generic_error_category@2@A@@YAXXZ 1001edf0 f   ClarkTests.obj
 0001:0001de00       ??__F?_Iostream_object@?$_Error_objects@H@std@@2V_Iostream_error_category@2@A@@YAXXZ 1001ee00 f   ClarkTests.obj
 0001:0001de10       ??__F?_System_object@?$_Error_objects@H@std@@2V_System_error_category@2@A@@YAXXZ 1001ee10 f   ClarkTests.obj
 0001:0001de20       ??__FalgoLog@U2@@YAXXZ     1001ee20 f   ClarkTests.obj
 0001:0001de30       ??__FcmdLog@U2@@YAXXZ      1001ee30 f   ClarkTests.obj
 0001:0001de40       ??__FcoreLog@U2@@YAXXZ     1001ee40 f   ClarkTests.obj
 0001:0001de50       ??__FioLog@U2@@YAXXZ       1001ee50 f   ClarkTests.obj
 0001:0001de60       ??__FperfLog@U2@@YAXXZ     1001ee60 f   ClarkTests.obj
 0001:0001de70       ??__FscriptLog@U2@@YAXXZ   1001ee70 f   ClarkTests.obj
 0001:0001de80       ??__FtaskLog@U2@@YAXXZ     1001ee80 f   ClarkTests.obj
 0001:0001de90       ??__FuiLog@U2@@YAXXZ       1001ee90 f   ClarkTests.obj
 0001:0001dea0       ??__FuserActLog@U2@@YAXXZ  1001eea0 f   ClarkTests.obj
 0001:0001deb0       ??__F?_Generic_object@?$_Error_objects@H@std@@2V_Generic_error_category@2@A@@YAXXZ 1001eeb0 f   moc_ClarkBuildWorker.obj
 0001:0001dec0       ??__F?_Iostream_object@?$_Error_objects@H@std@@2V_Iostream_error_category@2@A@@YAXXZ 1001eec0 f   moc_ClarkBuildWorker.obj
 0001:0001ded0       ??__F?_System_object@?$_Error_objects@H@std@@2V_System_error_category@2@A@@YAXXZ 1001eed0 f   moc_ClarkBuildWorker.obj
 0001:0001dee0       ??__FalgoLog@U2@@YAXXZ     1001eee0 f   moc_ClarkBuildWorker.obj
 0001:0001def0       ??__FcmdLog@U2@@YAXXZ      1001eef0 f   moc_ClarkBuildWorker.obj
 0001:0001df00       ??__FcoreLog@U2@@YAXXZ     1001ef00 f   moc_ClarkBuildWorker.obj
 0001:0001df10       ??__FioLog@U2@@YAXXZ       1001ef10 f   moc_ClarkBuildWorker.obj
 0001:0001df20       ??__FperfLog@U2@@YAXXZ     1001ef20 f   moc_ClarkBuildWorker.obj
 0001:0001df30       ??__FscriptLog@U2@@YAXXZ   1001ef30 f   moc_ClarkBuildWorker.obj
 0001:0001df40       ??__FtaskLog@U2@@YAXXZ     1001ef40 f   moc_ClarkBuildWorker.obj
 0001:0001df50       ??__FuiLog@U2@@YAXXZ       1001ef50 f   moc_ClarkBuildWorker.obj
 0001:0001df60       ??__FuserActLog@U2@@YAXXZ  1001ef60 f   moc_ClarkBuildWorker.obj
 0001:0001df70       ??__F?_Generic_object@?$_Error_objects@H@std@@2V_Generic_error_category@2@A@@YAXXZ 1001ef70 f   moc_ClarkClassifyWorker.obj
 0001:0001df80       ??__F?_Iostream_object@?$_Error_objects@H@std@@2V_Iostream_error_category@2@A@@YAXXZ 1001ef80 f   moc_ClarkClassifyWorker.obj
 0001:0001df90       ??__F?_System_object@?$_Error_objects@H@std@@2V_System_error_category@2@A@@YAXXZ 1001ef90 f   moc_ClarkClassifyWorker.obj
 0001:0001dfa0       ??__FalgoLog@U2@@YAXXZ     1001efa0 f   moc_ClarkClassifyWorker.obj
 0001:0001dfb0       ??__FcmdLog@U2@@YAXXZ      1001efb0 f   moc_ClarkClassifyWorker.obj
 0001:0001dfc0       ??__FcoreLog@U2@@YAXXZ     1001efc0 f   moc_ClarkClassifyWorker.obj
 0001:0001dfd0       ??__FioLog@U2@@YAXXZ       1001efd0 f   moc_ClarkClassifyWorker.obj
 0001:0001dfe0       ??__FperfLog@U2@@YAXXZ     1001efe0 f   moc_ClarkClassifyWorker.obj
 0001:0001dff0       ??__FscriptLog@U2@@YAXXZ   1001eff0 f   moc_ClarkClassifyWorker.obj
 0001:0001e000       ??__FtaskLog@U2@@YAXXZ     1001f000 f   moc_ClarkClassifyWorker.obj
 0001:0001e010       ??__FuiLog@U2@@YAXXZ       1001f010 f   moc_ClarkClassifyWorker.obj
 0001:0001e020       ??__FuserActLog@U2@@YAXXZ  1001f020 f   moc_ClarkClassifyWorker.obj
 0001:0001e030       ??__F?_Generic_object@?$_Error_objects@H@std@@2V_Generic_error_category@2@A@@YAXXZ 1001f030 f   moc_ClarkSupport.obj
 0001:0001e040       ??__F?_Iostream_object@?$_Error_objects@H@std@@2V_Iostream_error_category@2@A@@YAXXZ 1001f040 f   moc_ClarkSupport.obj
 0001:0001e050       ??__F?_System_object@?$_Error_objects@H@std@@2V_System_error_category@2@A@@YAXXZ 1001f050 f   moc_ClarkSupport.obj
 0001:0001e060       ??__F?_Generic_object@?$_Error_objects@H@std@@2V_Generic_error_category@2@A@@YAXXZ 1001f060 f   moc_ClarkSupportPlugin.obj
 0001:0001e070       ??__F?_Iostream_object@?$_Error_objects@H@std@@2V_Iostream_error_category@2@A@@YAXXZ 1001f070 f   moc_ClarkSupportPlugin.obj
 0001:0001e080       ??__F?_System_object@?$_Error_objects@H@std@@2V_System_error_category@2@A@@YAXXZ 1001f080 f   moc_ClarkSupportPlugin.obj
 0002:0000091c       _algoLog$initializer$      1002091c     ClarkBuildWorker.obj
 0002:00000920       _cmdLog$initializer$       10020920     ClarkBuildWorker.obj
 0002:00000924       _coreLog$initializer$      10020924     ClarkBuildWorker.obj
 0002:00000928       _ioLog$initializer$        10020928     ClarkBuildWorker.obj
 0002:0000092c       _perfLog$initializer$      1002092c     ClarkBuildWorker.obj
 0002:00000930       _scriptLog$initializer$    10020930     ClarkBuildWorker.obj
 0002:00000934       _taskLog$initializer$      10020934     ClarkBuildWorker.obj
 0002:00000938       _uiLog$initializer$        10020938     ClarkBuildWorker.obj
 0002:0000093c       _userActLog$initializer$   1002093c     ClarkBuildWorker.obj
 0002:00000940       ?ACTOR_ID$initializer$@ClarkBuildWorkerFactory@LocalWorkflow@U2@@0P6AXXZA 10020940     ClarkBuildWorker.obj
 0002:00000944       _OUTPUT_PORT$initializer$  10020944     ClarkBuildWorker.obj
 0002:00000948       _DB_URL$initializer$       10020948     ClarkBuildWorker.obj
 0002:0000094c       _GENOMIC_LIBRARY$initializer$ 1002094c     ClarkBuildWorker.obj
 0002:00000950       _TAXONOMY_RANK$initializer$ 10020950     ClarkBuildWorker.obj
 0002:00000954       ?wellKnownErrors$initializer$@ClarkBuildLogParser@LocalWorkflow@U2@@0P6AXXZA 10020954     ClarkBuildWorker.obj
 0002:00000958       ?_Generic_object$initializer$@?$_Error_objects@H@std@@2P6AXXZA 10020958     ClarkBuildWorker.obj
 0002:0000095c       ?_Iostream_object$initializer$@?$_Error_objects@H@std@@2P6AXXZA 1002095c     ClarkBuildWorker.obj
 0002:00000960       ?_System_object$initializer$@?$_Error_objects@H@std@@2P6AXXZA 10020960     ClarkBuildWorker.obj
 0002:00000964       _algoLog$initializer$      10020964     ClarkClassifyWorker.obj
 0002:00000968       _cmdLog$initializer$       10020968     ClarkClassifyWorker.obj
 0002:0000096c       _coreLog$initializer$      1002096c     ClarkClassifyWorker.obj
 0002:00000970       _ioLog$initializer$        10020970     ClarkClassifyWorker.obj
 0002:00000974       _perfLog$initializer$      10020974     ClarkClassifyWorker.obj
 0002:00000978       _scriptLog$initializer$    10020978     ClarkClassifyWorker.obj
 0002:0000097c       _taskLog$initializer$      1002097c     ClarkClassifyWorker.obj
 0002:00000980       _uiLog$initializer$        10020980     ClarkClassifyWorker.obj
 0002:00000984       _userActLog$initializer$   10020984     ClarkClassifyWorker.obj
 0002:00000988       ?ACTOR_ID$initializer$@ClarkClassifyWorkerFactory@LocalWorkflow@U2@@2P6AXXZA 10020988     ClarkClassifyWorker.obj
 0002:0000098c       ?INPUT_PORT$initializer$@ClarkClassifyWorkerFactory@LocalWorkflow@U2@@2P6AXXZA 1002098c     ClarkClassifyWorker.obj
 0002:00000990       ?PAIRED_INPUT_PORT$initializer$@ClarkClassifyWorkerFactory@LocalWorkflow@U2@@2P6AXXZA 10020990     ClarkClassifyWorker.obj
 0002:00000994       ?INPUT_SLOT$initializer$@ClarkClassifyWorkerFactory@LocalWorkflow@U2@@2P6AXXZA 10020994     ClarkClassifyWorker.obj
 0002:00000998       ?PAIRED_INPUT_SLOT$initializer$@ClarkClassifyWorkerFactory@LocalWorkflow@U2@@2P6AXXZA 10020998     ClarkClassifyWorker.obj
 0002:0000099c       ?OUTPUT_PORT$initializer$@ClarkClassifyWorkerFactory@LocalWorkflow@U2@@2P6AXXZA 1002099c     ClarkClassifyWorker.obj
 0002:000009a0       ?TOOL_VARIANT$initializer$@ClarkClassifyWorkerFactory@LocalWorkflow@U2@@2P6AXXZA 100209a0     ClarkClassifyWorker.obj
 0002:000009a4       ?DB_URL$initializer$@ClarkClassifyWorkerFactory@LocalWorkflow@U2@@2P6AXXZA 100209a4     ClarkClassifyWorker.obj
 0002:000009a8       ?OUTPUT_URL$initializer$@ClarkClassifyWorkerFactory@LocalWorkflow@U2@@2P6AXXZA 100209a8     ClarkClassifyWorker.obj
 0002:000009ac       ?TAXONOMY$initializer$@ClarkClassifyWorkerFactory@LocalWorkflow@U2@@2P6AXXZA 100209ac     ClarkClassifyWorker.obj
 0002:000009b0       ?TAXONOMY_RANK$initializer$@ClarkClassifyWorkerFactory@LocalWorkflow@U2@@2P6AXXZA 100209b0     ClarkClassifyWorker.obj
 0002:000009b4       ?K_LENGTH$initializer$@ClarkClassifyWorkerFactory@LocalWorkflow@U2@@2P6AXXZA 100209b4     ClarkClassifyWorker.obj
 0002:000009b8       ?K_MIN_FREQ$initializer$@ClarkClassifyWorkerFactory@LocalWorkflow@U2@@2P6AXXZA 100209b8     ClarkClassifyWorker.obj
 0002:000009bc       ?MODE$initializer$@ClarkClassifyWorkerFactory@LocalWorkflow@U2@@2P6AXXZA 100209bc     ClarkClassifyWorker.obj
 0002:000009c0       ?FACTOR$initializer$@ClarkClassifyWorkerFactory@LocalWorkflow@U2@@2P6AXXZA 100209c0     ClarkClassifyWorker.obj
 0002:000009c4       ?GAP$initializer$@ClarkClassifyWorkerFactory@LocalWorkflow@U2@@2P6AXXZA 100209c4     ClarkClassifyWorker.obj
 0002:000009c8       ?EXTEND_OUT$initializer$@ClarkClassifyWorkerFactory@LocalWorkflow@U2@@2P6AXXZA 100209c8     ClarkClassifyWorker.obj
 0002:000009cc       ?DB_TO_RAM$initializer$@ClarkClassifyWorkerFactory@LocalWorkflow@U2@@2P6AXXZA 100209cc     ClarkClassifyWorker.obj
 0002:000009d0       ?NUM_THREADS$initializer$@ClarkClassifyWorkerFactory@LocalWorkflow@U2@@2P6AXXZA 100209d0     ClarkClassifyWorker.obj
 0002:000009d4       ?SEQUENCING_READS$initializer$@ClarkClassifyWorkerFactory@LocalWorkflow@U2@@2P6AXXZA 100209d4     ClarkClassifyWorker.obj
 0002:000009d8       ?SINGLE_END$initializer$@ClarkClassifyWorkerFactory@LocalWorkflow@U2@@2P6AXXZA 100209d8     ClarkClassifyWorker.obj
 0002:000009dc       ?PAIRED_END$initializer$@ClarkClassifyWorkerFactory@LocalWorkflow@U2@@2P6AXXZA 100209dc     ClarkClassifyWorker.obj
 0002:000009e0       ?WORKFLOW_CLASSIFY_TOOL_CLARK$initializer$@ClarkClassifyWorkerFactory@LocalWorkflow@U2@@2P6AXXZA 100209e0     ClarkClassifyWorker.obj
 0002:000009e4       ?wellKnownErrors$initializer$@ClarkLogParser@LocalWorkflow@U2@@0P6AXXZA 100209e4     ClarkClassifyWorker.obj
 0002:000009e8       _REPORT_PREFIX$initializer$ 100209e8     ClarkClassifyWorker.obj
 0002:000009ec       _EXTENDED_REPORT_SUFFIX$initializer$ 100209ec     ClarkClassifyWorker.obj
 0002:000009f0       ?TOOL_DEFAULT$initializer$@ClarkClassifySettings@LocalWorkflow@U2@@2P6AXXZA 100209f0     ClarkClassifyWorker.obj
 0002:000009f4       ?TOOL_LIGHT$initializer$@ClarkClassifySettings@LocalWorkflow@U2@@2P6AXXZA 100209f4     ClarkClassifyWorker.obj
 0002:000009f8       _algoLog$initializer$      100209f8     ClarkSupport.obj
 0002:000009fc       _cmdLog$initializer$       100209fc     ClarkSupport.obj
 0002:00000a00       _coreLog$initializer$      10020a00     ClarkSupport.obj
 0002:00000a04       _ioLog$initializer$        10020a04     ClarkSupport.obj
 0002:00000a08       _perfLog$initializer$      10020a08     ClarkSupport.obj
 0002:00000a0c       _scriptLog$initializer$    10020a0c     ClarkSupport.obj
 0002:00000a10       _taskLog$initializer$      10020a10     ClarkSupport.obj
 0002:00000a14       _uiLog$initializer$        10020a14     ClarkSupport.obj
 0002:00000a18       _userActLog$initializer$   10020a18     ClarkSupport.obj
 0002:00000a1c       _Service_PluginViewer$initializer$ 10020a1c     ClarkSupport.obj
 0002:00000a20       _Service_Project$initializer$ 10020a20     ClarkSupport.obj
 0002:00000a24       _Service_ProjectView$initializer$ 10020a24     ClarkSupport.obj
 0002:00000a28       _Service_DNAGraphPack$initializer$ 10020a28     ClarkSupport.obj
 0002:00000a2c       _Service_DNAExport$initializer$ 10020a2c     ClarkSupport.obj
 0002:00000a30       _Service_TestRunner$initializer$ 10020a30     ClarkSupport.obj
 0002:00000a34       _Service_ScriptRegistry$initializer$ 10020a34     ClarkSupport.obj
 0002:00000a38       _Service_ExternalToolSupport$initializer$ 10020a38     ClarkSupport.obj
 0002:00000a3c       _Service_GUITesting$initializer$ 10020a3c     ClarkSupport.obj
 0002:00000a40       _Service_WorkflowDesigner$initializer$ 10020a40     ClarkSupport.obj
 0002:00000a44       _Service_QueryDesigner$initializer$ 10020a44     ClarkSupport.obj
 0002:00000a48       _Service_MinCoreServiceId$initializer$ 10020a48     ClarkSupport.obj
 0002:00000a4c       _Service_MaxCoreServiceId$initializer$ 10020a4c     ClarkSupport.obj
 0002:00000a50       ?CLARK_GROUP$initializer$@ClarkSupport@U2@@2P6AXXZA 10020a50     ClarkSupport.obj
 0002:00000a54       ?ET_CLARK$initializer$@ClarkSupport@U2@@2P6AXXZA 10020a54     ClarkSupport.obj
 0002:00000a58       ?ET_CLARK_ID$initializer$@ClarkSupport@U2@@2P6AXXZA 10020a58     ClarkSupport.obj
 0002:00000a5c       ?ET_CLARK_L$initializer$@ClarkSupport@U2@@2P6AXXZA 10020a5c     ClarkSupport.obj
 0002:00000a60       ?ET_CLARK_L_ID$initializer$@ClarkSupport@U2@@2P6AXXZA 10020a60     ClarkSupport.obj
 0002:00000a64       ?ET_CLARK_BUILD_SCRIPT$initializer$@ClarkSupport@U2@@2P6AXXZA 10020a64     ClarkSupport.obj
 0002:00000a68       ?ET_CLARK_BUILD_SCRIPT_ID$initializer$@ClarkSupport@U2@@2P6AXXZA 10020a68     ClarkSupport.obj
 0002:00000a6c       ?ET_CLARK_GET_ACCSSN_TAX_ID$initializer$@ClarkSupport@U2@@2P6AXXZA 10020a6c     ClarkSupport.obj
 0002:00000a70       ?ET_CLARK_GET_ACCSSN_TAX_ID_ID$initializer$@ClarkSupport@U2@@2P6AXXZA 10020a70     ClarkSupport.obj
 0002:00000a74       ?ET_CLARK_GET_TARGETS_DEF$initializer$@ClarkSupport@U2@@2P6AXXZA 10020a74     ClarkSupport.obj
 0002:00000a78       ?ET_CLARK_GET_TARGETS_DEF_ID$initializer$@ClarkSupport@U2@@2P6AXXZA 10020a78     ClarkSupport.obj
 0002:00000a7c       ?ET_CLARK_GET_FILES_TO_TAX_NODES$initializer$@ClarkSupport@U2@@2P6AXXZA 10020a7c     ClarkSupport.obj
 0002:00000a80       ?ET_CLARK_GET_FILES_TO_TAX_NODES_ID$initializer$@ClarkSupport@U2@@2P6AXXZA 10020a80     ClarkSupport.obj
 0002:00000a84       _algoLog$initializer$      10020a84     ClarkSupportPlugin.obj
 0002:00000a88       _cmdLog$initializer$       10020a88     ClarkSupportPlugin.obj
 0002:00000a8c       _coreLog$initializer$      10020a8c     ClarkSupportPlugin.obj
 0002:00000a90       _ioLog$initializer$        10020a90     ClarkSupportPlugin.obj
 0002:00000a94       _perfLog$initializer$      10020a94     ClarkSupportPlugin.obj
 0002:00000a98       _scriptLog$initializer$    10020a98     ClarkSupportPlugin.obj
 0002:00000a9c       _taskLog$initializer$      10020a9c     ClarkSupportPlugin.obj
 0002:00000aa0       _uiLog$initializer$        10020aa0     ClarkSupportPlugin.obj
 0002:00000aa4       _userActLog$initializer$   10020aa4     ClarkSupportPlugin.obj
 0002:00000aa8       ?PLUGIN_NAME$initializer$@ClarkSupportPlugin@U2@@2P6AXXZA 10020aa8     ClarkSupportPlugin.obj
 0002:00000aac       ?PLUGIN_DESCRIPRION$initializer$@ClarkSupportPlugin@U2@@2P6AXXZA 10020aac     ClarkSupportPlugin.obj
 0002:00000ab0       _algoLog$initializer$      10020ab0     ClarkTests.obj
 0002:00000ab4       _cmdLog$initializer$       10020ab4     ClarkTests.obj
 0002:00000ab8       _coreLog$initializer$      10020ab8     ClarkTests.obj
 0002:00000abc       _ioLog$initializer$        10020abc     ClarkTests.obj
 0002:00000ac0       _perfLog$initializer$      10020ac0     ClarkTests.obj
 0002:00000ac4       _scriptLog$initializer$    10020ac4     ClarkTests.obj
 0002:00000ac8       _taskLog$initializer$      10020ac8     ClarkTests.obj
 0002:00000acc       _uiLog$initializer$        10020acc     ClarkTests.obj
 0002:00000ad0       _userActLog$initializer$   10020ad0     ClarkTests.obj
 0002:00000ad4       ?DATABASE1$initializer$@GTest_CompareClarkDatabaseMetafiles@U2@@0P6AXXZA 10020ad4     ClarkTests.obj
 0002:00000ad8       ?DATABASE2$initializer$@GTest_CompareClarkDatabaseMetafiles@U2@@0P6AXXZA 10020ad8     ClarkTests.obj
 0002:00000adc       ?DATABASE1_PREFIXES$initializer$@GTest_CompareClarkDatabaseMetafiles@U2@@0P6AXXZA 10020adc     ClarkTests.obj
 0002:00000ae0       ?DATABASE2_PREFIXES$initializer$@GTest_CompareClarkDatabaseMetafiles@U2@@0P6AXXZA 10020ae0     ClarkTests.obj
 0002:00000ae4       ?DATABASE_PREFIX_PLACEHOLDER$initializer$@GTest_CompareClarkDatabaseMetafiles@U2@@0P6AXXZA 10020ae4     ClarkTests.obj
 0002:00000ae8       ?DATABASE_METAFILES$initializer$@GTest_CompareClarkDatabaseMetafiles@U2@@0P6AXXZA 10020ae8     ClarkTests.obj
 0002:00000aec       ?PREFIXES_SEPARATOR$initializer$@GTest_CompareClarkDatabaseMetafiles@U2@@0P6AXXZA 10020aec     ClarkTests.obj
 0002:00000af0       _algoLog$initializer$      10020af0     moc_ClarkBuildWorker.obj
 0002:00000af4       _cmdLog$initializer$       10020af4     moc_ClarkBuildWorker.obj
 0002:00000af8       _coreLog$initializer$      10020af8     moc_ClarkBuildWorker.obj
 0002:00000afc       _ioLog$initializer$        10020afc     moc_ClarkBuildWorker.obj
 0002:00000b00       _perfLog$initializer$      10020b00     moc_ClarkBuildWorker.obj
 0002:00000b04       _scriptLog$initializer$    10020b04     moc_ClarkBuildWorker.obj
 0002:00000b08       _taskLog$initializer$      10020b08     moc_ClarkBuildWorker.obj
 0002:00000b0c       _uiLog$initializer$        10020b0c     moc_ClarkBuildWorker.obj
 0002:00000b10       _userActLog$initializer$   10020b10     moc_ClarkBuildWorker.obj
 0002:00000b14       ?staticMetaObject$initializer$@ClarkBuildPrompter@LocalWorkflow@U2@@2P6AXXZA 10020b14     moc_ClarkBuildWorker.obj
 0002:00000b18       ?staticMetaObject$initializer$@ClarkBuildWorker@LocalWorkflow@U2@@2P6AXXZA 10020b18     moc_ClarkBuildWorker.obj
 0002:00000b1c       ?staticMetaObject$initializer$@ClarkBuildTask@LocalWorkflow@U2@@2P6AXXZA 10020b1c     moc_ClarkBuildWorker.obj
 0002:00000b20       _algoLog$initializer$      10020b20     moc_ClarkClassifyWorker.obj
 0002:00000b24       _cmdLog$initializer$       10020b24     moc_ClarkClassifyWorker.obj
 0002:00000b28       _coreLog$initializer$      10020b28     moc_ClarkClassifyWorker.obj
 0002:00000b2c       _ioLog$initializer$        10020b2c     moc_ClarkClassifyWorker.obj
 0002:00000b30       _perfLog$initializer$      10020b30     moc_ClarkClassifyWorker.obj
 0002:00000b34       _scriptLog$initializer$    10020b34     moc_ClarkClassifyWorker.obj
 0002:00000b38       _taskLog$initializer$      10020b38     moc_ClarkClassifyWorker.obj
 0002:00000b3c       _uiLog$initializer$        10020b3c     moc_ClarkClassifyWorker.obj
 0002:00000b40       _userActLog$initializer$   10020b40     moc_ClarkClassifyWorker.obj
 0002:00000b44       ?staticMetaObject$initializer$@ClarkClassifyPrompter@LocalWorkflow@U2@@2P6AXXZA 10020b44     moc_ClarkClassifyWorker.obj
 0002:00000b48       ?staticMetaObject$initializer$@ClarkClassifyWorker@LocalWorkflow@U2@@2P6AXXZA 10020b48     moc_ClarkClassifyWorker.obj
 0002:00000b4c       ?staticMetaObject$initializer$@ClarkClassifyTask@LocalWorkflow@U2@@2P6AXXZA 10020b4c     moc_ClarkClassifyWorker.obj
 0002:00000b50       ?staticMetaObject$initializer$@ClarkSupport@U2@@2P6AXXZA 10020b50     moc_ClarkSupport.obj
 0002:00000b54       ?staticMetaObject$initializer$@ClarkSupportPlugin@U2@@2P6AXXZA 10020b54     moc_ClarkSupportPlugin.obj
 0002:00000b60       _pcinit                    10020b60     MSVCRT:crtdll.obj
 0002:00000b64       _pinit                     10020b64     MSVCRT:atonexit.obj
 0002:00003fc0       _qt_meta_stringdata_U2__LocalWorkflow__ClarkBuildPrompter 10023fc0     moc_ClarkBuildWorker.obj
 0002:00003ff8       _qt_meta_data_U2__LocalWorkflow__ClarkBuildPrompter 10023ff8     moc_ClarkBuildWorker.obj
 0002:00004034       _qt_meta_stringdata_U2__LocalWorkflow__ClarkBuildTask 10024034     moc_ClarkBuildWorker.obj
 0002:00004068       _qt_meta_stringdata_U2__LocalWorkflow__ClarkBuildWorker 10024068     moc_ClarkBuildWorker.obj
 0002:000040f8       _qt_meta_data_U2__LocalWorkflow__ClarkBuildWorker 100240f8     moc_ClarkBuildWorker.obj
 0002:00004154       _qt_meta_data_U2__LocalWorkflow__ClarkBuildTask 10024154     moc_ClarkBuildWorker.obj
 0002:00004190       _qt_meta_stringdata_U2__LocalWorkflow__ClarkClassifyPrompter 10024190     moc_ClarkClassifyWorker.obj
 0002:000041cc       _qt_meta_data_U2__LocalWorkflow__ClarkClassifyPrompter 100241cc     moc_ClarkClassifyWorker.obj
 0002:00004208       _qt_meta_stringdata_U2__LocalWorkflow__ClarkClassifyWorker 10024208     moc_ClarkClassifyWorker.obj
 0002:0000429c       _qt_meta_data_U2__LocalWorkflow__ClarkClassifyTask 1002429c     moc_ClarkClassifyWorker.obj
 0002:000042d8       _qt_meta_data_U2__LocalWorkflow__ClarkClassifyWorker 100242d8     moc_ClarkClassifyWorker.obj
 0002:00004334       _qt_meta_stringdata_U2__LocalWorkflow__ClarkClassifyTask 10024334     moc_ClarkClassifyWorker.obj
 0002:0000436c       _qt_meta_stringdata_U2__ClarkSupport 1002436c     moc_ClarkSupport.obj
 0002:00004390       _qt_meta_data_U2__ClarkSupport 10024390     moc_ClarkSupport.obj
 0002:000043cc       _qt_meta_stringdata_U2__ClarkSupportPlugin 100243cc     moc_ClarkSupportPlugin.obj
 0002:000043f4       _qt_meta_data_U2__ClarkSupportPlugin 100243f4     moc_ClarkSupportPlugin.obj
 0002:00004440       _GS_ExceptionPointers      10024440     MSVCRT:gs_report.obj
 0002:00005e70       __catchsym$?_Copy@?$basic_string@DU?$char_traits@D@std@@V?$allocator@D@2@@std@@QAEXII@Z$5 10025e70     ClarkBuildWorker.obj
 0002:00005e80       __catchsym$?_Copy@?$basic_string@DU?$char_traits@D@std@@V?$allocator@D@2@@std@@QAEXII@Z$4 10025e80     ClarkBuildWorker.obj
 0002:00005e90       __unwindtable$?_Copy@?$basic_string@DU?$char_traits@D@std@@V?$allocator@D@2@@std@@QAEXII@Z 10025e90     ClarkBuildWorker.obj
 0002:00005eb0       __ehfuncinfo$?_Copy@?$basic_string@DU?$char_traits@D@std@@V?$allocator@D@2@@std@@QAEXII@Z 10025eb0     ClarkBuildWorker.obj
 0002:00005ed4       __tryblocktable$?_Copy@?$basic_string@DU?$char_traits@D@std@@V?$allocator@D@2@@std@@QAEXII@Z 10025ed4     ClarkBuildWorker.obj
 0002:00005efc       __unwindtable$??H@YA?BVQString@@ABV0@PBD@Z 10025efc     ClarkBuildWorker.obj
 0002:00005f0c       __ehfuncinfo$??H@YA?BVQString@@ABV0@PBD@Z 10025f0c     ClarkBuildWorker.obj
 0002:00005f30       __catchsym$??0?$QList@VQString@@@@QAE@ABV0@@Z$2 10025f30     ClarkBuildWorker.obj
 0002:00005f40       __unwindtable$??0?$QList@VQString@@@@QAE@ABV0@@Z 10025f40     ClarkBuildWorker.obj
 0002:00005f50       __tryblocktable$??0?$QList@VQString@@@@QAE@ABV0@@Z 10025f50     ClarkBuildWorker.obj
 0002:00005f64       __ehfuncinfo$??0?$QList@VQString@@@@QAE@ABV0@@Z 10025f64     ClarkBuildWorker.obj
 0002:00005f88       __catchsym$?append@?$QList@VQString@@@@QAEXABVQString@@@Z$13 10025f88     ClarkBuildWorker.obj
 0002:00005f98       __catchsym$?append@?$QList@VQString@@@@QAEXABVQString@@@Z$12 10025f98     ClarkBuildWorker.obj
 0002:00005fa8       __ehfuncinfo$?append@?$QList@VQString@@@@QAEXABVQString@@@Z 10025fa8     ClarkBuildWorker.obj
 0002:00005fcc       __tryblocktable$?append@?$QList@VQString@@@@QAEXABVQString@@@Z 10025fcc     ClarkBuildWorker.obj
 0002:00005ff4       __unwindtable$?append@?$QList@VQString@@@@QAEXABVQString@@@Z 10025ff4     ClarkBuildWorker.obj
 0002:00006054       __catchsym$?detach_helper_grow@?$QList@VQString@@@@AAEPAUNode@1@HH@Z$5 10026054     ClarkBuildWorker.obj
 0002:00006064       __catchsym$?detach_helper_grow@?$QList@VQString@@@@AAEPAUNode@1@HH@Z$4 10026064     ClarkBuildWorker.obj
 0002:00006074       __unwindtable$?detach_helper_grow@?$QList@VQString@@@@AAEPAUNode@1@HH@Z 10026074     ClarkBuildWorker.obj
 0002:00006094       __ehfuncinfo$?detach_helper_grow@?$QList@VQString@@@@AAEPAUNode@1@HH@Z 10026094     ClarkBuildWorker.obj
 0002:000060b8       __tryblocktable$?detach_helper_grow@?$QList@VQString@@@@AAEPAUNode@1@HH@Z 100260b8     ClarkBuildWorker.obj
 0002:000060e0       __unwindtable$?node_construct@?$QList@VQString@@@@AAEXPAUNode@1@ABVQString@@@Z 100260e0     ClarkBuildWorker.obj
 0002:000060f0       __ehfuncinfo$?node_construct@?$QList@VQString@@@@AAEXPAUNode@1@ABVQString@@@Z 100260f0     ClarkBuildWorker.obj
 0002:00006114       __catchsym$?node_copy@?$QList@VQString@@@@AAEXPAUNode@1@00@Z$6 10026114     ClarkBuildWorker.obj
 0002:00006124       __tryblocktable$?node_copy@?$QList@VQString@@@@AAEXPAUNode@1@00@Z 10026124     ClarkBuildWorker.obj
 0002:00006138       __ehfuncinfo$?node_copy@?$QList@VQString@@@@AAEXPAUNode@1@00@Z 10026138     ClarkBuildWorker.obj
 0002:0000615c       __unwindtable$?node_copy@?$QList@VQString@@@@AAEXPAUNode@1@00@Z 1002615c     ClarkBuildWorker.obj
 0002:0000618c       __unwindtable$??A?$QMap@VQString@@VQVariant@@@@QAEAAVQVariant@@ABVQString@@@Z 1002618c     ClarkBuildWorker.obj
 0002:00006194       __ehfuncinfo$??A?$QMap@VQString@@VQVariant@@@@QAEAAVQVariant@@ABVQString@@@Z 10026194     ClarkBuildWorker.obj
 0002:000061b8       __unwindtable$??__EalgoLog@U2@@YAXXZ 100261b8     ClarkBuildWorker.obj
 0002:000061c0       __ehfuncinfo$??__EalgoLog@U2@@YAXXZ 100261c0     ClarkBuildWorker.obj
 0002:000061e4       __unwindtable$??__EcmdLog@U2@@YAXXZ 100261e4     ClarkBuildWorker.obj
 0002:000061ec       __ehfuncinfo$??__EcmdLog@U2@@YAXXZ 100261ec     ClarkBuildWorker.obj
 0002:00006210       __unwindtable$??__EcoreLog@U2@@YAXXZ 10026210     ClarkBuildWorker.obj
 0002:00006218       __ehfuncinfo$??__EcoreLog@U2@@YAXXZ 10026218     ClarkBuildWorker.obj
 0002:0000623c       __unwindtable$??__EioLog@U2@@YAXXZ 1002623c     ClarkBuildWorker.obj
 0002:00006244       __ehfuncinfo$??__EioLog@U2@@YAXXZ 10026244     ClarkBuildWorker.obj
 0002:00006268       __unwindtable$??__EperfLog@U2@@YAXXZ 10026268     ClarkBuildWorker.obj
 0002:00006270       __ehfuncinfo$??__EperfLog@U2@@YAXXZ 10026270     ClarkBuildWorker.obj
 0002:00006294       __unwindtable$??__EscriptLog@U2@@YAXXZ 10026294     ClarkBuildWorker.obj
 0002:0000629c       __ehfuncinfo$??__EscriptLog@U2@@YAXXZ 1002629c     ClarkBuildWorker.obj
 0002:000062c0       __unwindtable$??__EtaskLog@U2@@YAXXZ 100262c0     ClarkBuildWorker.obj
 0002:000062c8       __ehfuncinfo$??__EtaskLog@U2@@YAXXZ 100262c8     ClarkBuildWorker.obj
 0002:000062ec       __unwindtable$??__EuiLog@U2@@YAXXZ 100262ec     ClarkBuildWorker.obj
 0002:000062f4       __ehfuncinfo$??__EuiLog@U2@@YAXXZ 100262f4     ClarkBuildWorker.obj
 0002:00006318       __unwindtable$??__EuserActLog@U2@@YAXXZ 10026318     ClarkBuildWorker.obj
 0002:00006320       __ehfuncinfo$??__EuserActLog@U2@@YAXXZ 10026320     ClarkBuildWorker.obj
 0002:00006344       __unwindtable$??A?$QMap@VQString@@VQScriptValue@@@@QAEAAVQScriptValue@@ABVQString@@@Z 10026344     ClarkBuildWorker.obj
 0002:0000634c       __ehfuncinfo$??A?$QMap@VQString@@VQScriptValue@@@@QAEAAVQScriptValue@@ABVQString@@@Z 1002634c     ClarkBuildWorker.obj
 0002:00006370       __catchsym$??0?$QList@VDescriptor@U2@@@@QAE@ABV0@@Z$2 10026370     ClarkBuildWorker.obj
 0002:00006380       __unwindtable$??0?$QList@VDescriptor@U2@@@@QAE@ABV0@@Z 10026380     ClarkBuildWorker.obj
 0002:00006390       __tryblocktable$??0?$QList@VDescriptor@U2@@@@QAE@ABV0@@Z 10026390     ClarkBuildWorker.obj
 0002:000063a4       __ehfuncinfo$??0?$QList@VDescriptor@U2@@@@QAE@ABV0@@Z 100263a4     ClarkBuildWorker.obj
 0002:000063c8       __catchsym$?append@?$QList@VDescriptor@U2@@@@QAEXABVDescriptor@U2@@@Z$9 100263c8     ClarkBuildWorker.obj
 0002:000063d8       __catchsym$?append@?$QList@VDescriptor@U2@@@@QAEXABVDescriptor@U2@@@Z$8 100263d8     ClarkBuildWorker.obj
 0002:000063e8       __ehfuncinfo$?append@?$QList@VDescriptor@U2@@@@QAEXABVDescriptor@U2@@@Z 100263e8     ClarkBuildWorker.obj
 0002:0000640c       __tryblocktable$?append@?$QList@VDescriptor@U2@@@@QAEXABVDescriptor@U2@@@Z 1002640c     ClarkBuildWorker.obj
 0002:00006434       __unwindtable$?append@?$QList@VDescriptor@U2@@@@QAEXABVDescriptor@U2@@@Z 10026434     ClarkBuildWorker.obj
 0002:00006474       __catchsym$?detach_helper_grow@?$QList@VDescriptor@U2@@@@AAEPAUNode@1@HH@Z$5 10026474     ClarkBuildWorker.obj
 0002:00006484       __catchsym$?detach_helper_grow@?$QList@VDescriptor@U2@@@@AAEPAUNode@1@HH@Z$4 10026484     ClarkBuildWorker.obj
 0002:00006494       __unwindtable$?detach_helper_grow@?$QList@VDescriptor@U2@@@@AAEPAUNode@1@HH@Z 10026494     ClarkBuildWorker.obj
 0002:000064b4       __ehfuncinfo$?detach_helper_grow@?$QList@VDescriptor@U2@@@@AAEPAUNode@1@HH@Z 100264b4     ClarkBuildWorker.obj
 0002:000064d8       __tryblocktable$?detach_helper_grow@?$QList@VDescriptor@U2@@@@AAEPAUNode@1@HH@Z 100264d8     ClarkBuildWorker.obj
 0002:00006500       __catchsym$?detach_helper@?$QList@VDescriptor@U2@@@@AAEXH@Z$2 10026500     ClarkBuildWorker.obj
 0002:00006510       __unwindtable$?detach_helper@?$QList@VDescriptor@U2@@@@AAEXH@Z 10026510     ClarkBuildWorker.obj
 0002:00006520       __tryblocktable$?detach_helper@?$QList@VDescriptor@U2@@@@AAEXH@Z 10026520     ClarkBuildWorker.obj
 0002:00006534       __ehfuncinfo$?detach_helper@?$QList@VDescriptor@U2@@@@AAEXH@Z 10026534     ClarkBuildWorker.obj
 0002:00006558       __unwindtable$?node_construct@?$QList@VDescriptor@U2@@@@AAEXPAUNode@1@ABVDescriptor@U2@@@Z 10026558     ClarkBuildWorker.obj
 0002:00006568       __ehfuncinfo$?node_construct@?$QList@VDescriptor@U2@@@@AAEXPAUNode@1@ABVDescriptor@U2@@@Z 10026568     ClarkBuildWorker.obj
 0002:0000658c       __catchsym$?node_copy@?$QList@VDescriptor@U2@@@@AAEXPAUNode@1@00@Z$6 1002658c     ClarkBuildWorker.obj
 0002:0000659c       __tryblocktable$?node_copy@?$QList@VDescriptor@U2@@@@AAEXPAUNode@1@00@Z 1002659c     ClarkBuildWorker.obj
 0002:000065b0       __ehfuncinfo$?node_copy@?$QList@VDescriptor@U2@@@@AAEXPAUNode@1@00@Z 100265b0     ClarkBuildWorker.obj
 0002:000065d4       __unwindtable$?node_copy@?$QList@VDescriptor@U2@@@@AAEXPAUNode@1@00@Z 100265d4     ClarkBuildWorker.obj
 0002:00006604       __unwindtable$??A?$QMap@VDescriptor@U2@@V?$QExplicitlySharedDataPointer@VDataType@U2@@@@@@QAEAAV?$QExplicitlySharedDataPointer@VDataType@U2@@@@ABVDescriptor@U2@@@Z 10026604     ClarkBuildWorker.obj
 0002:0000660c       __ehfuncinfo$??A?$QMap@VDescriptor@U2@@V?$QExplicitlySharedDataPointer@VDataType@U2@@@@@@QAEAAV?$QExplicitlySharedDataPointer@VDataType@U2@@@@ABVDescriptor@U2@@@Z 1002660c     ClarkBuildWorker.obj
 0002:00006630       __unwindtable$?uniqueKeys@?$QMap@VDescriptor@U2@@VQVariant@@@@QBE?AV?$QList@VDescriptor@U2@@@@XZ 10026630     ClarkBuildWorker.obj
 0002:00006638       __ehfuncinfo$?uniqueKeys@?$QMap@VDescriptor@U2@@VQVariant@@@@QBE?AV?$QList@VDescriptor@U2@@@@XZ 10026638     ClarkBuildWorker.obj
 0002:0000665c       __ehfuncinfo$??$getAttributeValue@VQString@@@Attribute@U2@@QBE?AVQString@@PAVWorkflowContext@Workflow@1@@Z 1002665c     ClarkBuildWorker.obj
 0002:00006680       __unwindtable$??$getAttributeValue@VQString@@@Attribute@U2@@QBE?AVQString@@PAVWorkflowContext@Workflow@1@@Z 10026680     ClarkBuildWorker.obj
 0002:000066f0       __ehfuncinfo$??$getAttributeValue@H@Attribute@U2@@QBEHPAVWorkflowContext@Workflow@1@@Z 100266f0     ClarkBuildWorker.obj
 0002:00006714       __unwindtable$??$getAttributeValue@H@Attribute@U2@@QBEHPAVWorkflowContext@Workflow@1@@Z 10026714     ClarkBuildWorker.obj
 0002:0000677c       __catchsym$?append@?$QList@PAVAttribute@U2@@@@QAEXABQAVAttribute@U2@@@Z$6 1002677c     ClarkBuildWorker.obj
 0002:0000678c       __tryblocktable$?append@?$QList@PAVAttribute@U2@@@@QAEXABQAVAttribute@U2@@@Z 1002678c     ClarkBuildWorker.obj
 0002:000067a0       __ehfuncinfo$?append@?$QList@PAVAttribute@U2@@@@QAEXABQAVAttribute@U2@@@Z 100267a0     ClarkBuildWorker.obj
 0002:000067c4       __unwindtable$?append@?$QList@PAVAttribute@U2@@@@QAEXABQAVAttribute@U2@@@Z 100267c4     ClarkBuildWorker.obj
 0002:000067f4       __catchsym$?detach_helper_grow@?$QList@PAVAttribute@U2@@@@AAEPAUNode@1@HH@Z$5 100267f4     ClarkBuildWorker.obj
 0002:00006804       __catchsym$?detach_helper_grow@?$QList@PAVAttribute@U2@@@@AAEPAUNode@1@HH@Z$4 10026804     ClarkBuildWorker.obj
 0002:00006814       __unwindtable$?detach_helper_grow@?$QList@PAVAttribute@U2@@@@AAEPAUNode@1@HH@Z 10026814     ClarkBuildWorker.obj
 0002:00006834       __ehfuncinfo$?detach_helper_grow@?$QList@PAVAttribute@U2@@@@AAEPAUNode@1@HH@Z 10026834     ClarkBuildWorker.obj
 0002:00006858       __tryblocktable$?detach_helper_grow@?$QList@PAVAttribute@U2@@@@AAEPAUNode@1@HH@Z 10026858     ClarkBuildWorker.obj
 0002:00006880       __catchsym$?append@?$QList@PAVPortDescriptor@Workflow@U2@@@@QAEXABQAVPortDescriptor@Workflow@U2@@@Z$6 10026880     ClarkBuildWorker.obj
 0002:00006890       __tryblocktable$?append@?$QList@PAVPortDescriptor@Workflow@U2@@@@QAEXABQAVPortDescriptor@Workflow@U2@@@Z 10026890     ClarkBuildWorker.obj
 0002:000068a4       __ehfuncinfo$?append@?$QList@PAVPortDescriptor@Workflow@U2@@@@QAEXABQAVPortDescriptor@Workflow@U2@@@Z 100268a4     ClarkBuildWorker.obj
 0002:000068c8       __unwindtable$?append@?$QList@PAVPortDescriptor@Workflow@U2@@@@QAEXABQAVPortDescriptor@Workflow@U2@@@Z 100268c8     ClarkBuildWorker.obj
 0002:000068f8       __catchsym$?detach_helper_grow@?$QList@PAVPortDescriptor@Workflow@U2@@@@AAEPAUNode@1@HH@Z$5 100268f8     ClarkBuildWorker.obj
 0002:00006908       __catchsym$?detach_helper_grow@?$QList@PAVPortDescriptor@Workflow@U2@@@@AAEPAUNode@1@HH@Z$4 10026908     ClarkBuildWorker.obj
 0002:00006918       __unwindtable$?detach_helper_grow@?$QList@PAVPortDescriptor@Workflow@U2@@@@AAEPAUNode@1@HH@Z 10026918     ClarkBuildWorker.obj
 0002:00006938       __ehfuncinfo$?detach_helper_grow@?$QList@PAVPortDescriptor@Workflow@U2@@@@AAEPAUNode@1@HH@Z 10026938     ClarkBuildWorker.obj
 0002:0000695c       __tryblocktable$?detach_helper_grow@?$QList@PAVPortDescriptor@Workflow@U2@@@@AAEPAUNode@1@HH@Z 1002695c     ClarkBuildWorker.obj
 0002:00006984       __catchsym$??0?$QList@VDataset@U2@@@@QAE@ABV0@@Z$2 10026984     ClarkBuildWorker.obj
 0002:00006994       __unwindtable$??0?$QList@VDataset@U2@@@@QAE@ABV0@@Z 10026994     ClarkBuildWorker.obj
 0002:000069a4       __tryblocktable$??0?$QList@VDataset@U2@@@@QAE@ABV0@@Z 100269a4     ClarkBuildWorker.obj
 0002:000069b8       __ehfuncinfo$??0?$QList@VDataset@U2@@@@QAE@ABV0@@Z 100269b8     ClarkBuildWorker.obj
 0002:000069dc       __catchsym$?node_copy@?$QList@VDataset@U2@@@@AAEXPAUNode@1@00@Z$6 100269dc     ClarkBuildWorker.obj
 0002:000069ec       __tryblocktable$?node_copy@?$QList@VDataset@U2@@@@AAEXPAUNode@1@00@Z 100269ec     ClarkBuildWorker.obj
 0002:00006a00       __ehfuncinfo$?node_copy@?$QList@VDataset@U2@@@@AAEXPAUNode@1@00@Z 10026a00     ClarkBuildWorker.obj
 0002:00006a24       __unwindtable$?node_copy@?$QList@VDataset@U2@@@@AAEXPAUNode@1@00@Z 10026a24     ClarkBuildWorker.obj
 0002:00006a54       __unwindtable$?qt_metatype_id@?$QMetaTypeId@V?$QList@VDataset@U2@@@@@@SAHXZ 10026a54     ClarkBuildWorker.obj
 0002:00006a5c       __ehfuncinfo$?qt_metatype_id@?$QMetaTypeId@V?$QList@VDataset@U2@@@@@@SAHXZ 10026a5c     ClarkBuildWorker.obj
 0002:00006a80       __unwindtable$??$qRegisterMetaType@V?$QList@VDataset@U2@@@@@@YAHPBDPAV?$QList@VDataset@U2@@@@W4DefinedType@?$MetaTypeDefinedHelper@V?$QList@VDataset@U2@@@@$00@QtPrivate@@@Z 10026a80     ClarkBuildWorker.obj
 0002:00006a88       __ehfuncinfo$??$qRegisterMetaType@V?$QList@VDataset@U2@@@@@@YAHPBDPAV?$QList@VDataset@U2@@@@W4DefinedType@?$MetaTypeDefinedHelper@V?$QList@VDataset@U2@@@@$00@QtPrivate@@@Z 10026a88     ClarkBuildWorker.obj
 0002:00006aac       __catchsym$?append@?$QList@VWorkflowNotification@U2@@@@QAEXABVWorkflowNotification@U2@@@Z$11 10026aac     ClarkBuildWorker.obj
 0002:00006abc       __catchsym$?append@?$QList@VWorkflowNotification@U2@@@@QAEXABVWorkflowNotification@U2@@@Z$10 10026abc     ClarkBuildWorker.obj
 0002:00006acc       __ehfuncinfo$?append@?$QList@VWorkflowNotification@U2@@@@QAEXABVWorkflowNotification@U2@@@Z 10026acc     ClarkBuildWorker.obj
 0002:00006af0       __tryblocktable$?append@?$QList@VWorkflowNotification@U2@@@@QAEXABVWorkflowNotification@U2@@@Z 10026af0     ClarkBuildWorker.obj
 0002:00006b18       __unwindtable$?append@?$QList@VWorkflowNotification@U2@@@@QAEXABVWorkflowNotification@U2@@@Z 10026b18     ClarkBuildWorker.obj
 0002:00006b68       __catchsym$?detach_helper_grow@?$QList@VWorkflowNotification@U2@@@@AAEPAUNode@1@HH@Z$5 10026b68     ClarkBuildWorker.obj
 0002:00006b78       __catchsym$?detach_helper_grow@?$QList@VWorkflowNotification@U2@@@@AAEPAUNode@1@HH@Z$4 10026b78     ClarkBuildWorker.obj
 0002:00006b88       __unwindtable$?detach_helper_grow@?$QList@VWorkflowNotification@U2@@@@AAEPAUNode@1@HH@Z 10026b88     ClarkBuildWorker.obj
 0002:00006ba8       __ehfuncinfo$?detach_helper_grow@?$QList@VWorkflowNotification@U2@@@@AAEPAUNode@1@HH@Z 10026ba8     ClarkBuildWorker.obj
 0002:00006bcc       __tryblocktable$?detach_helper_grow@?$QList@VWorkflowNotification@U2@@@@AAEPAUNode@1@HH@Z 10026bcc     ClarkBuildWorker.obj
 0002:00006bf4       __unwindtable$?node_construct@?$QList@VWorkflowNotification@U2@@@@AAEXPAUNode@1@ABVWorkflowNotification@U2@@@Z 10026bf4     ClarkBuildWorker.obj
 0002:00006c04       __ehfuncinfo$?node_construct@?$QList@VWorkflowNotification@U2@@@@AAEXPAUNode@1@ABVWorkflowNotification@U2@@@Z 10026c04     ClarkBuildWorker.obj
 0002:00006c28       __catchsym$?node_copy@?$QList@VWorkflowNotification@U2@@@@AAEXPAUNode@1@00@Z$6 10026c28     ClarkBuildWorker.obj
 0002:00006c38       __tryblocktable$?node_copy@?$QList@VWorkflowNotification@U2@@@@AAEXPAUNode@1@00@Z 10026c38     ClarkBuildWorker.obj
 0002:00006c4c       __ehfuncinfo$?node_copy@?$QList@VWorkflowNotification@U2@@@@AAEXPAUNode@1@00@Z 10026c4c     ClarkBuildWorker.obj
 0002:00006c70       __unwindtable$?node_copy@?$QList@VWorkflowNotification@U2@@@@AAEXPAUNode@1@00@Z 10026c70     ClarkBuildWorker.obj
 0002:00006ca0       __unwindtable$??$getValue@VQString@@@BaseWorker@LocalWorkflow@U2@@IBE?AVQString@@ABV3@@Z 10026ca0     ClarkBuildWorker.obj
 0002:00006cb0       __ehfuncinfo$??$getValue@VQString@@@BaseWorker@LocalWorkflow@U2@@IBE?AVQString@@ABV3@@Z 10026cb0     ClarkBuildWorker.obj
 0002:00006cd4       __ehfuncinfo$?validateTaxonomy@ClarkBuildValidator@LocalWorkflow@U2@@ABE_NPBVActor@Workflow@3@AAV?$QList@VWorkflowNotification@U2@@@@@Z 10026cd4     ClarkBuildWorker.obj
 0002:00006cf8       __unwindtable$?validateTaxonomy@ClarkBuildValidator@LocalWorkflow@U2@@ABE_NPBVActor@Workflow@3@AAV?$QList@VWorkflowNotification@U2@@@@@Z 10026cf8     ClarkBuildWorker.obj
 0002:00006dc0       __ehfuncinfo$?createDescription@?$PrompterBase@VClarkBuildPrompter@LocalWorkflow@U2@@@U2@@UAEPAVActorDocument@Workflow@2@PAVActor@42@@Z 10026dc0     ClarkBuildWorker.obj
 0002:00006de4       __unwindtable$?createDescription@?$PrompterBase@VClarkBuildPrompter@LocalWorkflow@U2@@@U2@@UAEPAVActorDocument@Workflow@2@PAVActor@42@@Z 10026de4     ClarkBuildWorker.obj
 0002:00006e1c       __ehfuncinfo$?composeRichDoc@ClarkBuildPrompter@LocalWorkflow@U2@@MAE?AVQString@@XZ 10026e1c     ClarkBuildWorker.obj
 0002:00006e40       __unwindtable$?composeRichDoc@ClarkBuildPrompter@LocalWorkflow@U2@@MAE?AVQString@@XZ 10026e40     ClarkBuildWorker.obj
 0002:00006e70       __ehfuncinfo$?init@ClarkBuildWorker@LocalWorkflow@U2@@MAEXXZ 10026e70     ClarkBuildWorker.obj
 0002:00006e94       __unwindtable$?init@ClarkBuildWorker@LocalWorkflow@U2@@MAEXXZ 10026e94     ClarkBuildWorker.obj
 0002:00006ecc       __ehfuncinfo$?tick@ClarkBuildWorker@LocalWorkflow@U2@@MAEPAVTask@3@XZ 10026ecc     ClarkBuildWorker.obj
 0002:00006ef0       __unwindtable$?tick@ClarkBuildWorker@LocalWorkflow@U2@@MAEPAVTask@3@XZ 10026ef0     ClarkBuildWorker.obj
 0002:00006f50       __ehfuncinfo$?sl_taskFinished@ClarkBuildWorker@LocalWorkflow@U2@@AAEXPAVTask@3@@Z 10026f50     ClarkBuildWorker.obj
 0002:00006f74       __unwindtable$?sl_taskFinished@ClarkBuildWorker@LocalWorkflow@U2@@AAEXPAVTask@3@@Z 10026f74     ClarkBuildWorker.obj
 0002:00007004       __ehfuncinfo$?init@ClarkBuildWorkerFactory@LocalWorkflow@U2@@SAXXZ 10027004     ClarkBuildWorker.obj
 0002:00007028       __unwindtable$?init@ClarkBuildWorkerFactory@LocalWorkflow@U2@@SAXXZ 10027028     ClarkBuildWorker.obj
 0002:000072c0       __unwindtable$?createWorker@ClarkBuildWorkerFactory@LocalWorkflow@U2@@UAEPAVWorker@Workflow@3@PAVActor@53@@Z 100272c0     ClarkBuildWorker.obj
 0002:000072c8       __ehfuncinfo$?createWorker@ClarkBuildWorkerFactory@LocalWorkflow@U2@@UAEPAVWorker@Workflow@3@PAVActor@53@@Z 100272c8     ClarkBuildWorker.obj
 0002:000072ec       __ehfuncinfo$??0ClarkBuildTask@LocalWorkflow@U2@@QAE@ABVQString@@ABVQStringList@@H0@Z 100272ec     ClarkBuildWorker.obj
 0002:00007310       __unwindtable$??0ClarkBuildTask@LocalWorkflow@U2@@QAE@ABVQString@@ABVQStringList@@H0@Z 10027310     ClarkBuildWorker.obj
 0002:00007380       __ehfuncinfo$?prepare@ClarkBuildTask@LocalWorkflow@U2@@EAEXXZ 10027380     ClarkBuildWorker.obj
 0002:000073a4       __unwindtable$?prepare@ClarkBuildTask@LocalWorkflow@U2@@EAEXXZ 100273a4     ClarkBuildWorker.obj
 0002:0000747c       __unwindtable$?getArguments@ClarkBuildTask@LocalWorkflow@U2@@AAE?AVQStringList@@XZ 1002747c     ClarkBuildWorker.obj
 0002:00007494       __ehfuncinfo$?getArguments@ClarkBuildTask@LocalWorkflow@U2@@AAE?AVQStringList@@XZ 10027494     ClarkBuildWorker.obj
 0002:000074b8       __unwindtable$??1ClarkBuildTask@LocalWorkflow@U2@@UAE@XZ 100274b8     ClarkBuildWorker.obj
 0002:000074d0       __ehfuncinfo$??1ClarkBuildTask@LocalWorkflow@U2@@UAE@XZ 100274d0     ClarkBuildWorker.obj
 0002:000074f4       __unwindtable$??_GClarkBuildTask@LocalWorkflow@U2@@UAEPAXI@Z 100274f4     ClarkBuildWorker.obj
 0002:0000750c       __ehfuncinfo$??_GClarkBuildTask@LocalWorkflow@U2@@UAEPAXI@Z 1002750c     ClarkBuildWorker.obj
 0002:00007530       __unwindtable$?isError@ClarkBuildLogParser@LocalWorkflow@U2@@EBE_NABVQString@@@Z 10027530     ClarkBuildWorker.obj
 0002:00007538       __ehfuncinfo$?isError@ClarkBuildLogParser@LocalWorkflow@U2@@EBE_NABVQString@@@Z 10027538     ClarkBuildWorker.obj
 0002:0000755c       __unwindtable$??__E?wellKnownErrors@ClarkBuildLogParser@LocalWorkflow@U2@@0VQStringList@@B@@YAXXZ 1002755c     ClarkBuildWorker.obj
 0002:00007574       __ehfuncinfo$??__E?wellKnownErrors@ClarkBuildLogParser@LocalWorkflow@U2@@0VQStringList@@B@@YAXXZ 10027574     ClarkBuildWorker.obj
 0002:00007598       __catchsym$?createNode@?$QMapData@VQString@@VQVariant@@@@QAEPAU?$QMapNode@VQString@@VQVariant@@@@ABVQString@@ABVQVariant@@PAU2@_N@Z$7 10027598     ClarkBuildWorker.obj
 0002:000075a8       __catchsym$?createNode@?$QMapData@VQString@@VQVariant@@@@QAEPAU?$QMapNode@VQString@@VQVariant@@@@ABVQString@@ABVQVariant@@PAU2@_N@Z$6 100275a8     ClarkBuildWorker.obj
 0002:000075b8       __ehfuncinfo$?createNode@?$QMapData@VQString@@VQVariant@@@@QAEPAU?$QMapNode@VQString@@VQVariant@@@@ABVQString@@ABVQVariant@@PAU2@_N@Z 100275b8     ClarkBuildWorker.obj
 0002:000075dc       __tryblocktable$?createNode@?$QMapData@VQString@@VQVariant@@@@QAEPAU?$QMapNode@VQString@@VQVariant@@@@ABVQString@@ABVQVariant@@PAU2@_N@Z 100275dc     ClarkBuildWorker.obj
 0002:00007604       __unwindtable$?createNode@?$QMapData@VQString@@VQVariant@@@@QAEPAU?$QMapNode@VQString@@VQVariant@@@@ABVQString@@ABVQVariant@@PAU2@_N@Z 10027604     ClarkBuildWorker.obj
 0002:00007634       __catchsym$?createNode@?$QMapData@VQString@@VQScriptValue@@@@QAEPAU?$QMapNode@VQString@@VQScriptValue@@@@ABVQString@@ABVQScriptValue@@PAU2@_N@Z$7 10027634     ClarkBuildWorker.obj
 0002:00007644       __catchsym$?createNode@?$QMapData@VQString@@VQScriptValue@@@@QAEPAU?$QMapNode@VQString@@VQScriptValue@@@@ABVQString@@ABVQScriptValue@@PAU2@_N@Z$6 10027644     ClarkBuildWorker.obj
 0002:00007654       __ehfuncinfo$?createNode@?$QMapData@VQString@@VQScriptValue@@@@QAEPAU?$QMapNode@VQString@@VQScriptValue@@@@ABVQString@@ABVQScriptValue@@PAU2@_N@Z 10027654     ClarkBuildWorker.obj
 0002:00007678       __tryblocktable$?createNode@?$QMapData@VQString@@VQScriptValue@@@@QAEPAU?$QMapNode@VQString@@VQScriptValue@@@@ABVQString@@ABVQScriptValue@@PAU2@_N@Z 10027678     ClarkBuildWorker.obj
 0002:000076a0       __unwindtable$?createNode@?$QMapData@VQString@@VQScriptValue@@@@QAEPAU?$QMapNode@VQString@@VQScriptValue@@@@ABVQString@@ABVQScriptValue@@PAU2@_N@Z 100276a0     ClarkBuildWorker.obj
 0002:000076d0       __catchsym$?createNode@?$QMapData@VDescriptor@U2@@V?$QExplicitlySharedDataPointer@VDataType@U2@@@@@@QAEPAU?$QMapNode@VDescriptor@U2@@V?$QExplicitlySharedDataPointer@VDataType@U2@@@@@@ABVDescriptor@U2@@ABV?$QExplicitlySharedDataPointer@VDataType@U2@@@@PAU2@_N@Z$6 100276d0     ClarkBuildWorker.obj
 0002:000076e0       __tryblocktable$?createNode@?$QMapData@VDescriptor@U2@@V?$QExplicitlySharedDataPointer@VDataType@U2@@@@@@QAEPAU?$QMapNode@VDescriptor@U2@@V?$QExplicitlySharedDataPointer@VDataType@U2@@@@@@ABVDescriptor@U2@@ABV?$QExplicitlySharedDataPointer@VDataType@U2@@@@PAU2@_N@Z 100276e0     ClarkBuildWorker.obj
 0002:000076f4       __ehfuncinfo$?createNode@?$QMapData@VDescriptor@U2@@V?$QExplicitlySharedDataPointer@VDataType@U2@@@@@@QAEPAU?$QMapNode@VDescriptor@U2@@V?$QExplicitlySharedDataPointer@VDataType@U2@@@@@@ABVDescriptor@U2@@ABV?$QExplicitlySharedDataPointer@VDataType@U2@@@@PAU2@_N@Z 100276f4     ClarkBuildWorker.obj
 0002:00007718       __unwindtable$?createNode@?$QMapData@VDescriptor@U2@@V?$QExplicitlySharedDataPointer@VDataType@U2@@@@@@QAEPAU?$QMapNode@VDescriptor@U2@@V?$QExplicitlySharedDataPointer@VDataType@U2@@@@@@ABVDescriptor@U2@@ABV?$QExplicitlySharedDataPointer@VDataType@U2@@@@PAU2@_N@Z 10027718     ClarkBuildWorker.obj
 0002:00007740       __catchsym$?createNode@?$QMapData@VQString@@PAVPropertyDelegate@U2@@@@QAEPAU?$QMapNode@VQString@@PAVPropertyDelegate@U2@@@@ABVQString@@ABQAVPropertyDelegate@U2@@PAU2@_N@Z$5 10027740     ClarkBuildWorker.obj
 0002:00007750       __tryblocktable$?createNode@?$QMapData@VQString@@PAVPropertyDelegate@U2@@@@QAEPAU?$QMapNode@VQString@@PAVPropertyDelegate@U2@@@@ABVQString@@ABQAVPropertyDelegate@U2@@PAU2@_N@Z 10027750     ClarkBuildWorker.obj
 0002:00007764       __ehfuncinfo$?createNode@?$QMapData@VQString@@PAVPropertyDelegate@U2@@@@QAEPAU?$QMapNode@VQString@@PAVPropertyDelegate@U2@@@@ABVQString@@ABQAVPropertyDelegate@U2@@PAU2@_N@Z 10027764     ClarkBuildWorker.obj
 0002:00007788       __unwindtable$?createNode@?$QMapData@VQString@@PAVPropertyDelegate@U2@@@@QAEPAU?$QMapNode@VQString@@PAVPropertyDelegate@U2@@@@ABVQString@@ABQAVPropertyDelegate@U2@@PAU2@_N@Z 10027788     ClarkBuildWorker.obj
 0002:000077b0       __catchsym$??0?$QList@PAVPort@Workflow@U2@@@@QAE@ABV0@@Z$2 100277b0     ClarkBuildWorker.obj
 0002:000077c0       __unwindtable$??0?$QList@PAVPort@Workflow@U2@@@@QAE@ABV0@@Z 100277c0     ClarkBuildWorker.obj
 0002:000077d0       __tryblocktable$??0?$QList@PAVPort@Workflow@U2@@@@QAE@ABV0@@Z 100277d0     ClarkBuildWorker.obj
 0002:000077e4       __ehfuncinfo$??0?$QList@PAVPort@Workflow@U2@@@@QAE@ABV0@@Z 100277e4     ClarkBuildWorker.obj
 0002:00007808       __unwindtable$?metaType@?$QVariantValueHelper@VQString@@@QtPrivate@@SA?AVQString@@ABVQVariant@@@Z 10027808     ClarkBuildWorker.obj
 0002:00007818       __ehfuncinfo$?metaType@?$QVariantValueHelper@VQString@@@QtPrivate@@SA?AVQString@@ABVQVariant@@@Z 10027818     ClarkBuildWorker.obj
 0002:0000783c       __unwindtable$?Create@?$QMetaTypeFunctionHelper@V?$QList@VDataset@U2@@@@$00@QtMetaTypePrivate@@SAPAXPBX@Z 1002783c     ClarkBuildWorker.obj
 0002:00007844       __ehfuncinfo$?Create@?$QMetaTypeFunctionHelper@V?$QList@VDataset@U2@@@@$00@QtMetaTypePrivate@@SAPAXPBX@Z 10027844     ClarkBuildWorker.obj
 0002:00007868       __unwindtable$?Construct@?$QMetaTypeFunctionHelper@V?$QList@VDataset@U2@@@@$00@QtMetaTypePrivate@@SAPAXPAXPBX@Z 10027868     ClarkBuildWorker.obj
 0002:00007870       __ehfuncinfo$?Construct@?$QMetaTypeFunctionHelper@V?$QList@VDataset@U2@@@@$00@QtMetaTypePrivate@@SAPAXPAXPBX@Z 10027870     ClarkBuildWorker.obj
 0002:00007894       __unwindtable$?metaType@?$QVariantValueHelper@V?$QList@VDataset@U2@@@@@QtPrivate@@SA?AV?$QList@VDataset@U2@@@@ABVQVariant@@@Z 10027894     ClarkBuildWorker.obj
 0002:000078a4       __ehfuncinfo$?metaType@?$QVariantValueHelper@V?$QList@VDataset@U2@@@@@QtPrivate@@SA?AV?$QList@VDataset@U2@@@@ABVQVariant@@@Z 100278a4     ClarkBuildWorker.obj
 0002:000078c8       __unwindtable$??H@YA?BVQString@@ABV0@0@Z 100278c8     ClarkClassifyWorker.obj
 0002:000078d0       __ehfuncinfo$??H@YA?BVQString@@ABV0@0@Z 100278d0     ClarkClassifyWorker.obj
 0002:000078f4       __unwindtable$?qt_metatype_id@?$QMetaTypeId@VQAssociativeIterableImpl@QtMetaTypePrivate@@@@SAHXZ 100278f4     ClarkClassifyWorker.obj
 0002:000078fc       __ehfuncinfo$?qt_metatype_id@?$QMetaTypeId@VQAssociativeIterableImpl@QtMetaTypePrivate@@@@SAHXZ 100278fc     ClarkClassifyWorker.obj
 0002:00007920       __unwindtable$??$qRegisterMetaType@VQAssociativeIterableImpl@QtMetaTypePrivate@@@@YAHPBDPAVQAssociativeIterableImpl@QtMetaTypePrivate@@W4DefinedType@?$MetaTypeDefinedHelper@VQAssociativeIterableImpl@QtMetaTypePrivate@@$00@QtPrivate@@@Z 10027920     ClarkClassifyWorker.obj
 0002:00007928       __ehfuncinfo$??$qRegisterMetaType@VQAssociativeIterableImpl@QtMetaTypePrivate@@@@YAHPBDPAVQAssociativeIterableImpl@QtMetaTypePrivate@@W4DefinedType@?$MetaTypeDefinedHelper@VQAssociativeIterableImpl@QtMetaTypePrivate@@$00@QtPrivate@@@Z 10027928     ClarkClassifyWorker.obj
 0002:0000794c       __catchsym$?detach_helper@?$QList@VQString@@@@AAEXH@Z$2 1002794c     ClarkClassifyWorker.obj
 0002:0000795c       __unwindtable$?detach_helper@?$QList@VQString@@@@AAEXH@Z 1002795c     ClarkClassifyWorker.obj
 0002:0000796c       __tryblocktable$?detach_helper@?$QList@VQString@@@@AAEXH@Z 1002796c     ClarkClassifyWorker.obj
 0002:00007980       __ehfuncinfo$?detach_helper@?$QList@VQString@@@@AAEXH@Z 10027980     ClarkClassifyWorker.obj
 0002:000079a4       __unwindtable$??0QStringList@@QAE@ABVQString@@@Z 100279a4     ClarkClassifyWorker.obj
 0002:000079ac       __ehfuncinfo$??0QStringList@@QAE@ABVQString@@@Z 100279ac     ClarkClassifyWorker.obj
 0002:000079d0       __catchsym$?append@?$QList@VQVariant@@@@QAEXABVQVariant@@@Z$11 100279d0     ClarkClassifyWorker.obj
 0002:000079e0       __catchsym$?append@?$QList@VQVariant@@@@QAEXABVQVariant@@@Z$10 100279e0     ClarkClassifyWorker.obj
 0002:000079f0       __ehfuncinfo$?append@?$QList@VQVariant@@@@QAEXABVQVariant@@@Z 100279f0     ClarkClassifyWorker.obj
 0002:00007a14       __tryblocktable$?append@?$QList@VQVariant@@@@QAEXABVQVariant@@@Z 10027a14     ClarkClassifyWorker.obj
 0002:00007a3c       __unwindtable$?append@?$QList@VQVariant@@@@QAEXABVQVariant@@@Z 10027a3c     ClarkClassifyWorker.obj
 0002:00007a8c       __catchsym$?detach_helper_grow@?$QList@VQVariant@@@@AAEPAUNode@1@HH@Z$5 10027a8c     ClarkClassifyWorker.obj
 0002:00007a9c       __catchsym$?detach_helper_grow@?$QList@VQVariant@@@@AAEPAUNode@1@HH@Z$4 10027a9c     ClarkClassifyWorker.obj
 0002:00007aac       __unwindtable$?detach_helper_grow@?$QList@VQVariant@@@@AAEPAUNode@1@HH@Z 10027aac     ClarkClassifyWorker.obj
 0002:00007acc       __ehfuncinfo$?detach_helper_grow@?$QList@VQVariant@@@@AAEPAUNode@1@HH@Z 10027acc     ClarkClassifyWorker.obj
 0002:00007af0       __tryblocktable$?detach_helper_grow@?$QList@VQVariant@@@@AAEPAUNode@1@HH@Z 10027af0     ClarkClassifyWorker.obj
 0002:00007b18       __unwindtable$?node_construct@?$QList@VQVariant@@@@AAEXPAUNode@1@ABVQVariant@@@Z 10027b18     ClarkClassifyWorker.obj
 0002:00007b28       __ehfuncinfo$?node_construct@?$QList@VQVariant@@@@AAEXPAUNode@1@ABVQVariant@@@Z 10027b28     ClarkClassifyWorker.obj
 0002:00007b4c       __catchsym$?node_copy@?$QList@VQVariant@@@@AAEXPAUNode@1@00@Z$6 10027b4c     ClarkClassifyWorker.obj
 0002:00007b5c       __tryblocktable$?node_copy@?$QList@VQVariant@@@@AAEXPAUNode@1@00@Z 10027b5c     ClarkClassifyWorker.obj
 0002:00007b70       __ehfuncinfo$?node_copy@?$QList@VQVariant@@@@AAEXPAUNode@1@00@Z 10027b70     ClarkClassifyWorker.obj
 0002:00007b94       __unwindtable$?node_copy@?$QList@VQVariant@@@@AAEXPAUNode@1@00@Z 10027b94     ClarkClassifyWorker.obj
 0002:00007bc4       __unwindtable$??__EalgoLog@U2@@YAXXZ 10027bc4     ClarkClassifyWorker.obj
 0002:00007bcc       __ehfuncinfo$??__EalgoLog@U2@@YAXXZ 10027bcc     ClarkClassifyWorker.obj
 0002:00007bf0       __unwindtable$??__EcmdLog@U2@@YAXXZ 10027bf0     ClarkClassifyWorker.obj
 0002:00007bf8       __ehfuncinfo$??__EcmdLog@U2@@YAXXZ 10027bf8     ClarkClassifyWorker.obj
 0002:00007c1c       __unwindtable$??__EcoreLog@U2@@YAXXZ 10027c1c     ClarkClassifyWorker.obj
 0002:00007c24       __ehfuncinfo$??__EcoreLog@U2@@YAXXZ 10027c24     ClarkClassifyWorker.obj
 0002:00007c48       __unwindtable$??__EioLog@U2@@YAXXZ 10027c48     ClarkClassifyWorker.obj
 0002:00007c50       __ehfuncinfo$??__EioLog@U2@@YAXXZ 10027c50     ClarkClassifyWorker.obj
 0002:00007c74       __unwindtable$??__EperfLog@U2@@YAXXZ 10027c74     ClarkClassifyWorker.obj
 0002:00007c7c       __ehfuncinfo$??__EperfLog@U2@@YAXXZ 10027c7c     ClarkClassifyWorker.obj
 0002:00007ca0       __unwindtable$??__EscriptLog@U2@@YAXXZ 10027ca0     ClarkClassifyWorker.obj
 0002:00007ca8       __ehfuncinfo$??__EscriptLog@U2@@YAXXZ 10027ca8     ClarkClassifyWorker.obj
 0002:00007ccc       __unwindtable$??__EtaskLog@U2@@YAXXZ 10027ccc     ClarkClassifyWorker.obj
 0002:00007cd4       __ehfuncinfo$??__EtaskLog@U2@@YAXXZ 10027cd4     ClarkClassifyWorker.obj
 0002:00007cf8       __unwindtable$??__EuiLog@U2@@YAXXZ 10027cf8     ClarkClassifyWorker.obj
 0002:00007d00       __ehfuncinfo$??__EuiLog@U2@@YAXXZ 10027d00     ClarkClassifyWorker.obj
 0002:00007d24       __unwindtable$??__EuserActLog@U2@@YAXXZ 10027d24     ClarkClassifyWorker.obj
 0002:00007d2c       __ehfuncinfo$??__EuserActLog@U2@@YAXXZ 10027d2c     ClarkClassifyWorker.obj
 0002:00007d50       __unwindtable$?keys@?$QMap@VQString@@V1@@@QBE?AV?$QList@VQString@@@@XZ 10027d50     ClarkClassifyWorker.obj
 0002:00007d58       __ehfuncinfo$?keys@?$QMap@VQString@@V1@@@QBE?AV?$QList@VQString@@@@XZ 10027d58     ClarkClassifyWorker.obj
 0002:00007d7c       __unwindtable$??0?$QPair@VQString@@V1@@@QAE@ABVQString@@0@Z 10027d7c     ClarkClassifyWorker.obj
 0002:00007d84       __ehfuncinfo$??0?$QPair@VQString@@V1@@@QAE@ABVQString@@0@Z 10027d84     ClarkClassifyWorker.obj
 0002:00007da8       __unwindtable$??1?$QPair@VQString@@V1@@@QAE@XZ 10027da8     ClarkClassifyWorker.obj
 0002:00007db0       __ehfuncinfo$??1?$QPair@VQString@@V1@@@QAE@XZ 10027db0     ClarkClassifyWorker.obj
 0002:00007dd4       __unwindtable$??0?$QPair@VQString@@V1@@@QAE@ABU0@@Z 10027dd4     ClarkClassifyWorker.obj
 0002:00007ddc       __ehfuncinfo$??0?$QPair@VQString@@V1@@@QAE@ABU0@@Z 10027ddc     ClarkClassifyWorker.obj
 0002:00007e00       __unwindtable$??_G?$QPair@VQString@@V1@@@QAEPAXI@Z 10027e00     ClarkClassifyWorker.obj
 0002:00007e08       __ehfuncinfo$??_G?$QPair@VQString@@V1@@@QAEPAXI@Z 10027e08     ClarkClassifyWorker.obj
 0002:00007e2c       __unwindtable$?qt_metatype_id@?$QMetaTypeId@V?$QMap@VQString@@I@@@@SAHXZ 10027e2c     ClarkClassifyWorker.obj
 0002:00007e34       __ehfuncinfo$?qt_metatype_id@?$QMetaTypeId@V?$QMap@VQString@@I@@@@SAHXZ 10027e34     ClarkClassifyWorker.obj
 0002:00007e58       __unwindtable$??$qRegisterMetaType@V?$QMap@VQString@@I@@@@YAHPBDPAV?$QMap@VQString@@I@@W4DefinedType@?$MetaTypeDefinedHelper@V?$QMap@VQString@@I@@$00@QtPrivate@@@Z 10027e58     ClarkClassifyWorker.obj
 0002:00007e60       __ehfuncinfo$??$qRegisterMetaType@V?$QMap@VQString@@I@@@@YAHPBDPAV?$QMap@VQString@@I@@W4DefinedType@?$MetaTypeDefinedHelper@V?$QMap@VQString@@I@@$00@QtPrivate@@@Z 10027e60     ClarkClassifyWorker.obj
 0002:00007e84       __unwindtable$??0ClarkClassifySettings@LocalWorkflow@U2@@QAE@XZ 10027e84     ClarkClassifyWorker.obj
 0002:00007e8c       __ehfuncinfo$??0ClarkClassifySettings@LocalWorkflow@U2@@QAE@XZ 10027e8c     ClarkClassifyWorker.obj
 0002:00007eb0       __unwindtable$??1ClarkClassifySettings@LocalWorkflow@U2@@QAE@XZ 10027eb0     ClarkClassifyWorker.obj
 0002:00007eb8       __ehfuncinfo$??1ClarkClassifySettings@LocalWorkflow@U2@@QAE@XZ 10027eb8     ClarkClassifyWorker.obj
 0002:00007edc       __unwindtable$??0ClarkClassifySettings@LocalWorkflow@U2@@QAE@ABV012@@Z 10027edc     ClarkClassifyWorker.obj
 0002:00007ee4       __ehfuncinfo$??0ClarkClassifySettings@LocalWorkflow@U2@@QAE@ABV012@@Z 10027ee4     ClarkClassifyWorker.obj
 0002:00007f08       __ehfuncinfo$?createDescription@?$PrompterBase@VClarkClassifyPrompter@LocalWorkflow@U2@@@U2@@UAEPAVActorDocument@Workflow@2@PAVActor@42@@Z 10027f08     ClarkClassifyWorker.obj
 0002:00007f2c       __unwindtable$?createDescription@?$PrompterBase@VClarkClassifyPrompter@LocalWorkflow@U2@@@U2@@UAEPAVActorDocument@Workflow@2@PAVActor@42@@Z 10027f2c     ClarkClassifyWorker.obj
 0002:00007f64       __ehfuncinfo$?composeRichDoc@ClarkClassifyPrompter@LocalWorkflow@U2@@MAE?AVQString@@XZ 10027f64     ClarkClassifyWorker.obj
 0002:00007f88       __unwindtable$?composeRichDoc@ClarkClassifyPrompter@LocalWorkflow@U2@@MAE?AVQString@@XZ 10027f88     ClarkClassifyWorker.obj
 0002:00008008       __unwindtable$??0ClarkClassifyWorker@LocalWorkflow@U2@@QAE@PAVActor@Workflow@2@@Z 10028008     ClarkClassifyWorker.obj
 0002:00008018       __ehfuncinfo$??0ClarkClassifyWorker@LocalWorkflow@U2@@QAE@PAVActor@Workflow@2@@Z 10028018     ClarkClassifyWorker.obj
 0002:0000803c       __ehfuncinfo$?init@ClarkClassifyWorker@LocalWorkflow@U2@@MAEXXZ 1002803c     ClarkClassifyWorker.obj
 0002:00008060       __unwindtable$?init@ClarkClassifyWorker@LocalWorkflow@U2@@MAEXXZ 10028060     ClarkClassifyWorker.obj
 0002:00008100       __ehfuncinfo$?tick@ClarkClassifyWorker@LocalWorkflow@U2@@MAEPAVTask@3@XZ 10028100     ClarkClassifyWorker.obj
 0002:00008124       __unwindtable$?tick@ClarkClassifyWorker@LocalWorkflow@U2@@MAEPAVTask@3@XZ 10028124     ClarkClassifyWorker.obj
 0002:000082ac       __ehfuncinfo$?sl_taskFinished@ClarkClassifyWorker@LocalWorkflow@U2@@AAEXPAVTask@3@@Z 100282ac     ClarkClassifyWorker.obj
 0002:000082d0       __unwindtable$?sl_taskFinished@ClarkClassifyWorker@LocalWorkflow@U2@@AAEXPAVTask@3@@Z 100282d0     ClarkClassifyWorker.obj
 0002:00008370       __unwindtable$??1ClarkClassifyWorker@LocalWorkflow@U2@@UAE@XZ 10028370     ClarkClassifyWorker.obj
 0002:00008380       __ehfuncinfo$??1ClarkClassifyWorker@LocalWorkflow@U2@@UAE@XZ 10028380     ClarkClassifyWorker.obj
 0002:000083a4       __unwindtable$??_GClarkClassifyWorker@LocalWorkflow@U2@@UAEPAXI@Z 100283a4     ClarkClassifyWorker.obj
 0002:000083b4       __ehfuncinfo$??_GClarkClassifyWorker@LocalWorkflow@U2@@UAEPAXI@Z 100283b4     ClarkClassifyWorker.obj
 0002:000083d8       __ehfuncinfo$?validateDatabase@ClarkClassifyValidator@LocalWorkflow@U2@@ABE_NPBVActor@Workflow@3@AAV?$QList@VWorkflowNotification@U2@@@@@Z 100283d8     ClarkClassifyWorker.obj
 0002:000083fc       __unwindtable$?validateDatabase@ClarkClassifyValidator@LocalWorkflow@U2@@ABE_NPBVActor@Workflow@3@AAV?$QList@VWorkflowNotification@U2@@@@@Z 100283fc     ClarkClassifyWorker.obj
 0002:000084cc       __unwindtable$?validateRefseqAvailability@ClarkClassifyValidator@LocalWorkflow@U2@@ABE_NPBVActor@Workflow@3@AAV?$QList@VWorkflowNotification@U2@@@@@Z 100284cc     ClarkClassifyWorker.obj
 0002:000084e4       __ehfuncinfo$?validateRefseqAvailability@ClarkClassifyValidator@LocalWorkflow@U2@@ABE_NPBVActor@Workflow@3@AAV?$QList@VWorkflowNotification@U2@@@@@Z 100284e4     ClarkClassifyWorker.obj
 0002:00008508       __unwindtable$?checkRefseqAvailability@ClarkClassifyValidator@LocalWorkflow@U2@@ABE_NPBVActor@Workflow@3@AAV?$QList@VWorkflowNotification@U2@@@@ABVQString@@@Z 10028508     ClarkClassifyWorker.obj
 0002:00008520       __ehfuncinfo$?checkRefseqAvailability@ClarkClassifyValidator@LocalWorkflow@U2@@ABE_NPBVActor@Workflow@3@AAV?$QList@VWorkflowNotification@U2@@@@ABVQString@@@Z 10028520     ClarkClassifyWorker.obj
 0002:00008544       __ehfuncinfo$?isDatabaseAlreadyBuilt@ClarkClassifyValidator@LocalWorkflow@U2@@ABE_NPBVActor@Workflow@3@@Z 10028544     ClarkClassifyWorker.obj
 0002:00008568       __unwindtable$?isDatabaseAlreadyBuilt@ClarkClassifyValidator@LocalWorkflow@U2@@ABE_NPBVActor@Workflow@3@@Z 10028568     ClarkClassifyWorker.obj
 0002:000085d0       __ehfuncinfo$?init@ClarkClassifyWorkerFactory@LocalWorkflow@U2@@SAXXZ 100285d0     ClarkClassifyWorker.obj
 0002:000085f4       __unwindtable$?init@ClarkClassifyWorkerFactory@LocalWorkflow@U2@@SAXXZ 100285f4     ClarkClassifyWorker.obj
 0002:00008da4       __unwindtable$?createWorker@ClarkClassifyWorkerFactory@LocalWorkflow@U2@@UAEPAVWorker@Workflow@3@PAVActor@53@@Z 10028da4     ClarkClassifyWorker.obj
 0002:00008dac       __ehfuncinfo$?createWorker@ClarkClassifyWorkerFactory@LocalWorkflow@U2@@UAEPAVWorker@Workflow@3@PAVActor@53@@Z 10028dac     ClarkClassifyWorker.obj
 0002:00008dd0       __unwindtable$?isError@ClarkLogParser@LocalWorkflow@U2@@EBE_NABVQString@@@Z 10028dd0     ClarkClassifyWorker.obj
 0002:00008de8       __ehfuncinfo$?isError@ClarkLogParser@LocalWorkflow@U2@@EBE_NABVQString@@@Z 10028de8     ClarkClassifyWorker.obj
 0002:00008e0c       __ehfuncinfo$?setLastError@ClarkLogParser@LocalWorkflow@U2@@EAEXABVQString@@@Z 10028e0c     ClarkClassifyWorker.obj
 0002:00008e30       __unwindtable$?setLastError@ClarkLogParser@LocalWorkflow@U2@@EAEXABVQString@@@Z 10028e30     ClarkClassifyWorker.obj
 0002:00008e58       __ehfuncinfo$?initWellKnownErrors@ClarkLogParser@LocalWorkflow@U2@@CA?AV?$QMap@VQString@@V1@@@XZ 10028e58     ClarkClassifyWorker.obj
 0002:00008e7c       __unwindtable$?initWellKnownErrors@ClarkLogParser@LocalWorkflow@U2@@CA?AV?$QMap@VQString@@V1@@@XZ 10028e7c     ClarkClassifyWorker.obj
 0002:00008ea4       __ehfuncinfo$??0ClarkClassifyTask@LocalWorkflow@U2@@QAE@ABVClarkClassifySettings@12@ABVQString@@11@Z 10028ea4     ClarkClassifyWorker.obj
 0002:00008ec8       __unwindtable$??0ClarkClassifyTask@LocalWorkflow@U2@@QAE@ABVClarkClassifySettings@12@ABVQString@@11@Z 10028ec8     ClarkClassifyWorker.obj
 0002:00008f48       __ehfuncinfo$?prepare@ClarkClassifyTask@LocalWorkflow@U2@@EAEXXZ 10028f48     ClarkClassifyWorker.obj
 0002:00008f6c       __unwindtable$?prepare@ClarkClassifyTask@LocalWorkflow@U2@@EAEXXZ 10028f6c     ClarkClassifyWorker.obj
 0002:00008fdc       __ehfuncinfo$?run@ClarkClassifyTask@LocalWorkflow@U2@@EAEXXZ 10028fdc     ClarkClassifyWorker.obj
 0002:00009000       __unwindtable$?run@ClarkClassifyTask@LocalWorkflow@U2@@EAEXXZ 10029000     ClarkClassifyWorker.obj
 0002:000090c0       __ehfuncinfo$?getArguments@ClarkClassifyTask@LocalWorkflow@U2@@AAE?AVQStringList@@XZ 100290c0     ClarkClassifyWorker.obj
 0002:000090e4       __unwindtable$?getArguments@ClarkClassifyTask@LocalWorkflow@U2@@AAE?AVQStringList@@XZ 100290e4     ClarkClassifyWorker.obj
 0002:000091cc       __ehfuncinfo$??1ClarkClassifyTask@LocalWorkflow@U2@@UAE@XZ 100291cc     ClarkClassifyWorker.obj
 0002:000091f0       __unwindtable$??1ClarkClassifyTask@LocalWorkflow@U2@@UAE@XZ 100291f0     ClarkClassifyWorker.obj
 0002:00009220       __catchsym$?append@?$QList@U?$QPair@VQString@@V1@@@@@QAEXABU?$QPair@VQString@@V1@@@@Z$7 10029220     ClarkClassifyWorker.obj
 0002:00009230       __catchsym$?append@?$QList@U?$QPair@VQString@@V1@@@@@QAEXABU?$QPair@VQString@@V1@@@@Z$6 10029230     ClarkClassifyWorker.obj
 0002:00009240       __ehfuncinfo$?append@?$QList@U?$QPair@VQString@@V1@@@@@QAEXABU?$QPair@VQString@@V1@@@@Z 10029240     ClarkClassifyWorker.obj
 0002:00009264       __tryblocktable$?append@?$QList@U?$QPair@VQString@@V1@@@@@QAEXABU?$QPair@VQString@@V1@@@@Z 10029264     ClarkClassifyWorker.obj
 0002:0000928c       __unwindtable$?append@?$QList@U?$QPair@VQString@@V1@@@@@QAEXABU?$QPair@VQString@@V1@@@@Z 1002928c     ClarkClassifyWorker.obj
 0002:000092bc       __catchsym$?detach_helper_grow@?$QList@U?$QPair@VQString@@V1@@@@@AAEPAUNode@1@HH@Z$5 100292bc     ClarkClassifyWorker.obj
 0002:000092cc       __catchsym$?detach_helper_grow@?$QList@U?$QPair@VQString@@V1@@@@@AAEPAUNode@1@HH@Z$4 100292cc     ClarkClassifyWorker.obj
 0002:000092dc       __unwindtable$?detach_helper_grow@?$QList@U?$QPair@VQString@@V1@@@@@AAEPAUNode@1@HH@Z 100292dc     ClarkClassifyWorker.obj
 0002:000092fc       __ehfuncinfo$?detach_helper_grow@?$QList@U?$QPair@VQString@@V1@@@@@AAEPAUNode@1@HH@Z 100292fc     ClarkClassifyWorker.obj
 0002:00009320       __tryblocktable$?detach_helper_grow@?$QList@U?$QPair@VQString@@V1@@@@@AAEPAUNode@1@HH@Z 10029320     ClarkClassifyWorker.obj
 0002:00009348       __unwindtable$?node_construct@?$QList@U?$QPair@VQString@@V1@@@@@AAEXPAUNode@1@ABU?$QPair@VQString@@V1@@@@Z 10029348     ClarkClassifyWorker.obj
 0002:00009368       __ehfuncinfo$?node_construct@?$QList@U?$QPair@VQString@@V1@@@@@AAEXPAUNode@1@ABU?$QPair@VQString@@V1@@@@Z 10029368     ClarkClassifyWorker.obj
 0002:0000938c       __unwindtable$?node_destruct@?$QList@U?$QPair@VQString@@V1@@@@@AAEXPAUNode@1@@Z 1002938c     ClarkClassifyWorker.obj
 0002:0000939c       __ehfuncinfo$?node_destruct@?$QList@U?$QPair@VQString@@V1@@@@@AAEXPAUNode@1@@Z 1002939c     ClarkClassifyWorker.obj
 0002:000093c0       __catchsym$?node_copy@?$QList@U?$QPair@VQString@@V1@@@@@AAEXPAUNode@1@00@Z$14 100293c0     ClarkClassifyWorker.obj
 0002:000093d0       __tryblocktable$?node_copy@?$QList@U?$QPair@VQString@@V1@@@@@AAEXPAUNode@1@00@Z 100293d0     ClarkClassifyWorker.obj
 0002:000093e4       __ehfuncinfo$?node_copy@?$QList@U?$QPair@VQString@@V1@@@@@AAEXPAUNode@1@00@Z 100293e4     ClarkClassifyWorker.obj
 0002:00009408       __unwindtable$?node_copy@?$QList@U?$QPair@VQString@@V1@@@@@AAEXPAUNode@1@00@Z 10029408     ClarkClassifyWorker.obj
 0002:00009458       __unwindtable$?node_destruct@?$QList@U?$QPair@VQString@@V1@@@@@AAEXPAUNode@1@0@Z 10029458     ClarkClassifyWorker.obj
 0002:00009468       __ehfuncinfo$?node_destruct@?$QList@U?$QPair@VQString@@V1@@@@@AAEXPAUNode@1@0@Z 10029468     ClarkClassifyWorker.obj
 0002:0000948c       __catchsym$?createNode@?$QMapData@VQString@@V1@@@QAEPAU?$QMapNode@VQString@@V1@@@ABVQString@@0PAU2@_N@Z$7 1002948c     ClarkClassifyWorker.obj
 0002:0000949c       __catchsym$?createNode@?$QMapData@VQString@@V1@@@QAEPAU?$QMapNode@VQString@@V1@@@ABVQString@@0PAU2@_N@Z$6 1002949c     ClarkClassifyWorker.obj
 0002:000094ac       __ehfuncinfo$?createNode@?$QMapData@VQString@@V1@@@QAEPAU?$QMapNode@VQString@@V1@@@ABVQString@@0PAU2@_N@Z 100294ac     ClarkClassifyWorker.obj
 0002:000094d0       __tryblocktable$?createNode@?$QMapData@VQString@@V1@@@QAEPAU?$QMapNode@VQString@@V1@@@ABVQString@@0PAU2@_N@Z 100294d0     ClarkClassifyWorker.obj
 0002:000094f8       __unwindtable$?createNode@?$QMapData@VQString@@V1@@@QAEPAU?$QMapNode@VQString@@V1@@@ABVQString@@0PAU2@_N@Z 100294f8     ClarkClassifyWorker.obj
 0002:00009528       __catchsym$?createNode@?$QMapData@VQString@@I@@QAEPAU?$QMapNode@VQString@@I@@ABVQString@@ABIPAU2@_N@Z$5 10029528     ClarkClassifyWorker.obj
 0002:00009538       __tryblocktable$?createNode@?$QMapData@VQString@@I@@QAEPAU?$QMapNode@VQString@@I@@ABVQString@@ABIPAU2@_N@Z 10029538     ClarkClassifyWorker.obj
 0002:0000954c       __ehfuncinfo$?createNode@?$QMapData@VQString@@I@@QAEPAU?$QMapNode@VQString@@I@@ABVQString@@ABIPAU2@_N@Z 1002954c     ClarkClassifyWorker.obj
 0002:00009570       __unwindtable$?createNode@?$QMapData@VQString@@I@@QAEPAU?$QMapNode@VQString@@I@@ABVQString@@ABIPAU2@_N@Z 10029570     ClarkClassifyWorker.obj
 0002:00009598       __unwindtable$?Create@?$QMetaTypeFunctionHelper@V?$QMap@VQString@@I@@$00@QtMetaTypePrivate@@SAPAXPBX@Z 10029598     ClarkClassifyWorker.obj
 0002:000095a0       __ehfuncinfo$?Create@?$QMetaTypeFunctionHelper@V?$QMap@VQString@@I@@$00@QtMetaTypePrivate@@SAPAXPBX@Z 100295a0     ClarkClassifyWorker.obj
 0002:000095c4       __unwindtable$?Construct@?$QMetaTypeFunctionHelper@V?$QMap@VQString@@I@@$00@QtMetaTypePrivate@@SAPAXPAXPBX@Z 100295c4     ClarkClassifyWorker.obj
 0002:000095cc       __ehfuncinfo$?Construct@?$QMetaTypeFunctionHelper@V?$QMap@VQString@@I@@$00@QtMetaTypePrivate@@SAPAXPAXPBX@Z 100295cc     ClarkClassifyWorker.obj
 0002:000095f0       __unwindtable$??H@YA?BVQString@@PBDABV0@@Z 100295f0     ClarkSupport.obj
 0002:000095f8       __ehfuncinfo$??H@YA?BVQString@@PBDABV0@@Z 100295f8     ClarkSupport.obj
 0002:0000961c       __ehfuncinfo$??0ClarkSupport@U2@@QAE@ABVQString@@00@Z 1002961c     ClarkSupport.obj
 0002:00009640       __unwindtable$??0ClarkSupport@U2@@QAE@ABVQString@@00@Z 10029640     ClarkSupport.obj
 0002:000096d0       __ehfuncinfo$?registerTools@ClarkSupport@U2@@SAXPAVExternalToolRegistry@2@@Z 100296d0     ClarkSupport.obj
 0002:000096f4       __unwindtable$?registerTools@ClarkSupport@U2@@SAXPAVExternalToolRegistry@2@@Z 100296f4     ClarkSupport.obj
 0002:0000978c       __unwindtable$??__EalgoLog@U2@@YAXXZ 1002978c     ClarkSupport.obj
 0002:00009794       __ehfuncinfo$??__EalgoLog@U2@@YAXXZ 10029794     ClarkSupport.obj
 0002:000097b8       __unwindtable$??__EcmdLog@U2@@YAXXZ 100297b8     ClarkSupport.obj
 0002:000097c0       __ehfuncinfo$??__EcmdLog@U2@@YAXXZ 100297c0     ClarkSupport.obj
 0002:000097e4       __unwindtable$??__EcoreLog@U2@@YAXXZ 100297e4     ClarkSupport.obj
 0002:000097ec       __ehfuncinfo$??__EcoreLog@U2@@YAXXZ 100297ec     ClarkSupport.obj
 0002:00009810       __unwindtable$??__EioLog@U2@@YAXXZ 10029810     ClarkSupport.obj
 0002:00009818       __ehfuncinfo$??__EioLog@U2@@YAXXZ 10029818     ClarkSupport.obj
 0002:0000983c       __unwindtable$??__EperfLog@U2@@YAXXZ 1002983c     ClarkSupport.obj
 0002:00009844       __ehfuncinfo$??__EperfLog@U2@@YAXXZ 10029844     ClarkSupport.obj
 0002:00009868       __unwindtable$??__EscriptLog@U2@@YAXXZ 10029868     ClarkSupport.obj
 0002:00009870       __ehfuncinfo$??__EscriptLog@U2@@YAXXZ 10029870     ClarkSupport.obj
 0002:00009894       __unwindtable$??__EtaskLog@U2@@YAXXZ 10029894     ClarkSupport.obj
 0002:0000989c       __ehfuncinfo$??__EtaskLog@U2@@YAXXZ 1002989c     ClarkSupport.obj
 0002:000098c0       __unwindtable$??__EuiLog@U2@@YAXXZ 100298c0     ClarkSupport.obj
 0002:000098c8       __ehfuncinfo$??__EuiLog@U2@@YAXXZ 100298c8     ClarkSupport.obj
 0002:000098ec       __unwindtable$??__EuserActLog@U2@@YAXXZ 100298ec     ClarkSupport.obj
 0002:000098f4       __ehfuncinfo$??__EuserActLog@U2@@YAXXZ 100298f4     ClarkSupport.obj
 0002:00009918       __unwindtable$??__EalgoLog@U2@@YAXXZ 10029918     ClarkSupportPlugin.obj
 0002:00009920       __ehfuncinfo$??__EalgoLog@U2@@YAXXZ 10029920     ClarkSupportPlugin.obj
 0002:00009944       __unwindtable$??__EcmdLog@U2@@YAXXZ 10029944     ClarkSupportPlugin.obj
 0002:0000994c       __ehfuncinfo$??__EcmdLog@U2@@YAXXZ 1002994c     ClarkSupportPlugin.obj
 0002:00009970       __unwindtable$??__EcoreLog@U2@@YAXXZ 10029970     ClarkSupportPlugin.obj
 0002:00009978       __ehfuncinfo$??__EcoreLog@U2@@YAXXZ 10029978     ClarkSupportPlugin.obj
 0002:0000999c       __unwindtable$??__EioLog@U2@@YAXXZ 1002999c     ClarkSupportPlugin.obj
 0002:000099a4       __ehfuncinfo$??__EioLog@U2@@YAXXZ 100299a4     ClarkSupportPlugin.obj
 0002:000099c8       __unwindtable$??__EperfLog@U2@@YAXXZ 100299c8     ClarkSupportPlugin.obj
 0002:000099d0       __ehfuncinfo$??__EperfLog@U2@@YAXXZ 100299d0     ClarkSupportPlugin.obj
 0002:000099f4       __unwindtable$??__EscriptLog@U2@@YAXXZ 100299f4     ClarkSupportPlugin.obj
 0002:000099fc       __ehfuncinfo$??__EscriptLog@U2@@YAXXZ 100299fc     ClarkSupportPlugin.obj
 0002:00009a20       __unwindtable$??__EtaskLog@U2@@YAXXZ 10029a20     ClarkSupportPlugin.obj
 0002:00009a28       __ehfuncinfo$??__EtaskLog@U2@@YAXXZ 10029a28     ClarkSupportPlugin.obj
 0002:00009a4c       __unwindtable$??__EuiLog@U2@@YAXXZ 10029a4c     ClarkSupportPlugin.obj
 0002:00009a54       __ehfuncinfo$??__EuiLog@U2@@YAXXZ 10029a54     ClarkSupportPlugin.obj
 0002:00009a78       __unwindtable$??__EuserActLog@U2@@YAXXZ 10029a78     ClarkSupportPlugin.obj
 0002:00009a80       __ehfuncinfo$??__EuserActLog@U2@@YAXXZ 10029a80     ClarkSupportPlugin.obj
 0002:00009aa4       __ehfuncinfo$??0ClarkSupportPlugin@U2@@QAE@XZ 10029aa4     ClarkSupportPlugin.obj
 0002:00009ac8       __unwindtable$??0ClarkSupportPlugin@U2@@QAE@XZ 10029ac8     ClarkSupportPlugin.obj
 0002:00009b18       __ehfuncinfo$??1ClarkSupportPlugin@U2@@UAE@XZ 10029b18     ClarkSupportPlugin.obj
 0002:00009b3c       __unwindtable$??1ClarkSupportPlugin@U2@@UAE@XZ 10029b3c     ClarkSupportPlugin.obj
 0002:00009b84       __unwindtable$??1?$GAutoDeleteList@VXMLTestFactory@U2@@@U2@@UAE@XZ 10029b84     ClarkSupportPlugin.obj
 0002:00009b94       __ehfuncinfo$??1?$GAutoDeleteList@VXMLTestFactory@U2@@@U2@@UAE@XZ 10029b94     ClarkSupportPlugin.obj
 0002:00009bb8       __catchsym$??0?$QList@PAVXMLTestFactory@U2@@@@QAE@ABV0@@Z$2 10029bb8     ClarkSupportPlugin.obj
 0002:00009bc8       __unwindtable$??0?$QList@PAVXMLTestFactory@U2@@@@QAE@ABV0@@Z 10029bc8     ClarkSupportPlugin.obj
 0002:00009bd8       __tryblocktable$??0?$QList@PAVXMLTestFactory@U2@@@@QAE@ABV0@@Z 10029bd8     ClarkSupportPlugin.obj
 0002:00009bec       __ehfuncinfo$??0?$QList@PAVXMLTestFactory@U2@@@@QAE@ABV0@@Z 10029bec     ClarkSupportPlugin.obj
 0002:00009c10       __unwindtable$??__EalgoLog@U2@@YAXXZ 10029c10     ClarkTests.obj
 0002:00009c18       __ehfuncinfo$??__EalgoLog@U2@@YAXXZ 10029c18     ClarkTests.obj
 0002:00009c3c       __unwindtable$??__EcmdLog@U2@@YAXXZ 10029c3c     ClarkTests.obj
 0002:00009c44       __ehfuncinfo$??__EcmdLog@U2@@YAXXZ 10029c44     ClarkTests.obj
 0002:00009c68       __unwindtable$??__EcoreLog@U2@@YAXXZ 10029c68     ClarkTests.obj
 0002:00009c70       __ehfuncinfo$??__EcoreLog@U2@@YAXXZ 10029c70     ClarkTests.obj
 0002:00009c94       __unwindtable$??__EioLog@U2@@YAXXZ 10029c94     ClarkTests.obj
 0002:00009c9c       __ehfuncinfo$??__EioLog@U2@@YAXXZ 10029c9c     ClarkTests.obj
 0002:00009cc0       __unwindtable$??__EperfLog@U2@@YAXXZ 10029cc0     ClarkTests.obj
 0002:00009cc8       __ehfuncinfo$??__EperfLog@U2@@YAXXZ 10029cc8     ClarkTests.obj
 0002:00009cec       __unwindtable$??__EscriptLog@U2@@YAXXZ 10029cec     ClarkTests.obj
 0002:00009cf4       __ehfuncinfo$??__EscriptLog@U2@@YAXXZ 10029cf4     ClarkTests.obj
 0002:00009d18       __unwindtable$??__EtaskLog@U2@@YAXXZ 10029d18     ClarkTests.obj
 0002:00009d20       __ehfuncinfo$??__EtaskLog@U2@@YAXXZ 10029d20     ClarkTests.obj
 0002:00009d44       __unwindtable$??__EuiLog@U2@@YAXXZ 10029d44     ClarkTests.obj
 0002:00009d4c       __ehfuncinfo$??__EuiLog@U2@@YAXXZ 10029d4c     ClarkTests.obj
 0002:00009d70       __unwindtable$??__EuserActLog@U2@@YAXXZ 10029d70     ClarkTests.obj
 0002:00009d78       __ehfuncinfo$??__EuserActLog@U2@@YAXXZ 10029d78     ClarkTests.obj
 0002:00009d9c       __ehfuncinfo$??0GTest_CompareClarkDatabaseMetafiles@U2@@QAE@PAVXMLTestFormat@1@ABVQString@@PAVGTest@1@PBVGTestEnvironment@1@ABV?$QList@PAVGTest@U2@@@@ABVQDomElement@@@Z 10029d9c     ClarkTests.obj
 0002:00009dc0       __unwindtable$??0GTest_CompareClarkDatabaseMetafiles@U2@@QAE@PAVXMLTestFormat@1@ABVQString@@PAVGTest@1@PBVGTestEnvironment@1@ABV?$QList@PAVGTest@U2@@@@ABVQDomElement@@@Z 10029dc0     ClarkTests.obj
 0002:00009de8       __ehfuncinfo$?init@GTest_CompareClarkDatabaseMetafiles@U2@@QAEXPAVXMLTestFormat@2@ABVQDomElement@@@Z 10029de8     ClarkTests.obj
 0002:00009e0c       __unwindtable$?init@GTest_CompareClarkDatabaseMetafiles@U2@@QAEXPAVXMLTestFormat@2@ABVQDomElement@@@Z 10029e0c     ClarkTests.obj
 0002:00009ebc       __unwindtable$??0GTest_CompareClarkDatabaseMetafilesFactory@GTest_CompareClarkDatabaseMetafiles@U2@@QAE@XZ 10029ebc     ClarkTests.obj
 0002:00009ed4       __ehfuncinfo$??0GTest_CompareClarkDatabaseMetafilesFactory@GTest_CompareClarkDatabaseMetafiles@U2@@QAE@XZ 10029ed4     ClarkTests.obj
 0002:00009ef8       __unwindtable$?createTest@GTest_CompareClarkDatabaseMetafilesFactory@GTest_CompareClarkDatabaseMetafiles@U2@@UAEPAVGTest@3@PAVXMLTestFormat@3@ABVQString@@PAV43@PBVGTestEnvironment@3@ABV?$QList@PAVGTest@U2@@@@ABVQDomElement@@@Z 10029ef8     ClarkTests.obj
 0002:00009f00       __ehfuncinfo$?createTest@GTest_CompareClarkDatabaseMetafilesFactory@GTest_CompareClarkDatabaseMetafiles@U2@@UAEPAVGTest@3@PAVXMLTestFormat@3@ABVQString@@PAV43@PBVGTestEnvironment@3@ABV?$QList@PAVGTest@U2@@@@ABVQDomElement@@@Z 10029f00     ClarkTests.obj
 0002:00009f24       __unwindtable$?createFactory@GTest_CompareClarkDatabaseMetafiles@U2@@SAPAVXMLTestFactory@2@XZ 10029f24     ClarkTests.obj
 0002:00009f44       __ehfuncinfo$?createFactory@GTest_CompareClarkDatabaseMetafiles@U2@@SAPAVXMLTestFactory@2@XZ 10029f44     ClarkTests.obj
 0002:00009f68       __ehfuncinfo$?report@GTest_CompareClarkDatabaseMetafiles@U2@@EAE?AW4ReportResult@Task@2@XZ 10029f68     ClarkTests.obj
 0002:00009f8c       __unwindtable$?report@GTest_CompareClarkDatabaseMetafiles@U2@@EAE?AW4ReportResult@Task@2@XZ 10029f8c     ClarkTests.obj
 0002:0000a0cc       __unwindtable$??1GTest_CompareClarkDatabaseMetafiles@U2@@UAE@XZ 1002a0cc     ClarkTests.obj
 0002:0000a0ec       __ehfuncinfo$??1GTest_CompareClarkDatabaseMetafiles@U2@@UAE@XZ 1002a0ec     ClarkTests.obj
 0002:0000a110       __unwindtable$??_GGTest_CompareClarkDatabaseMetafiles@U2@@UAEPAXI@Z 1002a110     ClarkTests.obj
 0002:0000a130       __ehfuncinfo$??_GGTest_CompareClarkDatabaseMetafiles@U2@@UAEPAXI@Z 1002a130     ClarkTests.obj
 0002:0000a154       __ehfuncinfo$??__E?DATABASE_METAFILES@GTest_CompareClarkDatabaseMetafiles@U2@@0VQStringList@@B@@YAXXZ 1002a154     ClarkTests.obj
 0002:0000a178       __unwindtable$??__E?DATABASE_METAFILES@GTest_CompareClarkDatabaseMetafiles@U2@@0VQStringList@@B@@YAXXZ 1002a178     ClarkTests.obj
 0002:0000a1a8       __catchsym$?append@?$QList@PAVXMLTestFactory@U2@@@@QAEXABQAVXMLTestFactory@U2@@@Z$6 1002a1a8     ClarkTests.obj
 0002:0000a1b8       __tryblocktable$?append@?$QList@PAVXMLTestFactory@U2@@@@QAEXABQAVXMLTestFactory@U2@@@Z 1002a1b8     ClarkTests.obj
 0002:0000a1cc       __ehfuncinfo$?append@?$QList@PAVXMLTestFactory@U2@@@@QAEXABQAVXMLTestFactory@U2@@@Z 1002a1cc     ClarkTests.obj
 0002:0000a1f0       __unwindtable$?append@?$QList@PAVXMLTestFactory@U2@@@@QAEXABQAVXMLTestFactory@U2@@@Z 1002a1f0     ClarkTests.obj
 0002:0000a220       __catchsym$?detach_helper_grow@?$QList@PAVXMLTestFactory@U2@@@@AAEPAUNode@1@HH@Z$5 1002a220     ClarkTests.obj
 0002:0000a230       __catchsym$?detach_helper_grow@?$QList@PAVXMLTestFactory@U2@@@@AAEPAUNode@1@HH@Z$4 1002a230     ClarkTests.obj
 0002:0000a240       __unwindtable$?detach_helper_grow@?$QList@PAVXMLTestFactory@U2@@@@AAEPAUNode@1@HH@Z 1002a240     ClarkTests.obj
 0002:0000a260       __ehfuncinfo$?detach_helper_grow@?$QList@PAVXMLTestFactory@U2@@@@AAEPAUNode@1@HH@Z 1002a260     ClarkTests.obj
 0002:0000a284       __tryblocktable$?detach_helper_grow@?$QList@PAVXMLTestFactory@U2@@@@AAEPAUNode@1@HH@Z 1002a284     ClarkTests.obj
 0002:0000a2ac       __catchsym$?detach_helper@?$QList@PAVXMLTestFactory@U2@@@@AAEXH@Z$2 1002a2ac     ClarkTests.obj
 0002:0000a2bc       __unwindtable$?detach_helper@?$QList@PAVXMLTestFactory@U2@@@@AAEXH@Z 1002a2bc     ClarkTests.obj
 0002:0000a2cc       __tryblocktable$?detach_helper@?$QList@PAVXMLTestFactory@U2@@@@AAEXH@Z 1002a2cc     ClarkTests.obj
 0002:0000a2e0       __ehfuncinfo$?detach_helper@?$QList@PAVXMLTestFactory@U2@@@@AAEXH@Z 1002a2e0     ClarkTests.obj
 0002:0000a304       __unwindtable$??__EalgoLog@U2@@YAXXZ 1002a304     moc_ClarkBuildWorker.obj
 0002:0000a30c       __ehfuncinfo$??__EalgoLog@U2@@YAXXZ 1002a30c     moc_ClarkBuildWorker.obj
 0002:0000a330       __unwindtable$??__EcmdLog@U2@@YAXXZ 1002a330     moc_ClarkBuildWorker.obj
 0002:0000a338       __ehfuncinfo$??__EcmdLog@U2@@YAXXZ 1002a338     moc_ClarkBuildWorker.obj
 0002:0000a35c       __unwindtable$??__EcoreLog@U2@@YAXXZ 1002a35c     moc_ClarkBuildWorker.obj
 0002:0000a364       __ehfuncinfo$??__EcoreLog@U2@@YAXXZ 1002a364     moc_ClarkBuildWorker.obj
 0002:0000a388       __unwindtable$??__EioLog@U2@@YAXXZ 1002a388     moc_ClarkBuildWorker.obj
 0002:0000a390       __ehfuncinfo$??__EioLog@U2@@YAXXZ 1002a390     moc_ClarkBuildWorker.obj
 0002:0000a3b4       __unwindtable$??__EperfLog@U2@@YAXXZ 1002a3b4     moc_ClarkBuildWorker.obj
 0002:0000a3bc       __ehfuncinfo$??__EperfLog@U2@@YAXXZ 1002a3bc     moc_ClarkBuildWorker.obj
 0002:0000a3e0       __unwindtable$??__EscriptLog@U2@@YAXXZ 1002a3e0     moc_ClarkBuildWorker.obj
 0002:0000a3e8       __ehfuncinfo$??__EscriptLog@U2@@YAXXZ 1002a3e8     moc_ClarkBuildWorker.obj
 0002:0000a40c       __unwindtable$??__EtaskLog@U2@@YAXXZ 1002a40c     moc_ClarkBuildWorker.obj
 0002:0000a414       __ehfuncinfo$??__EtaskLog@U2@@YAXXZ 1002a414     moc_ClarkBuildWorker.obj
 0002:0000a438       __unwindtable$??__EuiLog@U2@@YAXXZ 1002a438     moc_ClarkBuildWorker.obj
 0002:0000a440       __ehfuncinfo$??__EuiLog@U2@@YAXXZ 1002a440     moc_ClarkBuildWorker.obj
 0002:0000a464       __unwindtable$??__EuserActLog@U2@@YAXXZ 1002a464     moc_ClarkBuildWorker.obj
 0002:0000a46c       __ehfuncinfo$??__EuserActLog@U2@@YAXXZ 1002a46c     moc_ClarkBuildWorker.obj
 0002:0000a490       __unwindtable$?qt_metatype_id@?$QMetaTypeIdQObject@PAVTask@U2@@$00@@SAHXZ 1002a490     moc_ClarkBuildWorker.obj
 0002:0000a498       __ehfuncinfo$?qt_metatype_id@?$QMetaTypeIdQObject@PAVTask@U2@@$00@@SAHXZ 1002a498     moc_ClarkBuildWorker.obj
 0002:0000a4bc       __unwindtable$??__EalgoLog@U2@@YAXXZ 1002a4bc     moc_ClarkClassifyWorker.obj
 0002:0000a4c4       __ehfuncinfo$??__EalgoLog@U2@@YAXXZ 1002a4c4     moc_ClarkClassifyWorker.obj
 0002:0000a4e8       __unwindtable$??__EcmdLog@U2@@YAXXZ 1002a4e8     moc_ClarkClassifyWorker.obj
 0002:0000a4f0       __ehfuncinfo$??__EcmdLog@U2@@YAXXZ 1002a4f0     moc_ClarkClassifyWorker.obj
 0002:0000a514       __unwindtable$??__EcoreLog@U2@@YAXXZ 1002a514     moc_ClarkClassifyWorker.obj
 0002:0000a51c       __ehfuncinfo$??__EcoreLog@U2@@YAXXZ 1002a51c     moc_ClarkClassifyWorker.obj
 0002:0000a540       __unwindtable$??__EioLog@U2@@YAXXZ 1002a540     moc_ClarkClassifyWorker.obj
 0002:0000a548       __ehfuncinfo$??__EioLog@U2@@YAXXZ 1002a548     moc_ClarkClassifyWorker.obj
 0002:0000a56c       __unwindtable$??__EperfLog@U2@@YAXXZ 1002a56c     moc_ClarkClassifyWorker.obj
 0002:0000a574       __ehfuncinfo$??__EperfLog@U2@@YAXXZ 1002a574     moc_ClarkClassifyWorker.obj
 0002:0000a598       __unwindtable$??__EscriptLog@U2@@YAXXZ 1002a598     moc_ClarkClassifyWorker.obj
 0002:0000a5a0       __ehfuncinfo$??__EscriptLog@U2@@YAXXZ 1002a5a0     moc_ClarkClassifyWorker.obj
 0002:0000a5c4       __unwindtable$??__EtaskLog@U2@@YAXXZ 1002a5c4     moc_ClarkClassifyWorker.obj
 0002:0000a5cc       __ehfuncinfo$??__EtaskLog@U2@@YAXXZ 1002a5cc     moc_ClarkClassifyWorker.obj
 0002:0000a5f0       __unwindtable$??__EuiLog@U2@@YAXXZ 1002a5f0     moc_ClarkClassifyWorker.obj
 0002:0000a5f8       __ehfuncinfo$??__EuiLog@U2@@YAXXZ 1002a5f8     moc_ClarkClassifyWorker.obj
 0002:0000a61c       __unwindtable$??__EuserActLog@U2@@YAXXZ 1002a61c     moc_ClarkClassifyWorker.obj
 0002:0000a624       __ehfuncinfo$??__EuserActLog@U2@@YAXXZ 1002a624     moc_ClarkClassifyWorker.obj
 0002:0000a648       __sehtable$__onexit        1002a648     MSVCRT:atonexit.obj
 0002:0000a668       __sehtable$??_M@YGXPAXIHP6EX0@Z@Z 1002a668     MSVCRT:ehvecdtr.obj
 0002:0000a688       __sehtable$?__ArrayUnwind@@YGXPAXIHP6EX0@Z@Z 1002a688     MSVCRT:ehvecdtr.obj
 0002:0000a6a8       __sehtable$___DllMainCRTStartup 1002a6a8     MSVCRT:crtdll.obj
 0002:0000a6d0       __sehtable$__IsNonwritableInCurrentImage 1002a6d0     MSVCRT:pesect.obj
 0002:0000a6f0       .edata                     1002a6f0     clark_support.exp
 0002:0000a718       rgpv                       1002a718     clark_support.exp
 0002:0000a71c       rgszName                   1002a71c     clark_support.exp
 0002:0000a720       rgwOrd                     1002a720     clark_support.exp
 0002:0000a722       szName                     1002a722     clark_support.exp
 0002:0000a734       $N00001                    1002a734     clark_support.exp
 0002:0000c858       .idata$6                   1002c858     U2Core:U2Core.dll
 0002:0000c8b2       .idata$6                   1002c8b2     U2Gui:U2Gui.dll
 0002:0000cb48       .idata$6                   1002cb48     U2Test:U2Test.dll
 0002:0000f432       .idata$6                   1002f432     U2Lang:U2Lang.dll
 0002:00010118       .idata$6                   10030118     U2Designer:U2Designer.dll
 0002:00010c5c       .idata$6                   10030c5c     ngs_reads_classification:ngs_reads_classification.dll
 0002:000110ba       .idata$6                   100310ba     Qt5Widgets:Qt5Widgets.dll
 0002:000111be       .idata$6                   100311be     Qt5Gui:Qt5Gui.dll
 0002:00011330       .idata$6                   10031330     Qt5Script:Qt5Script.dll
 0002:00011370       .idata$6                   10031370     Qt5Xml:Qt5Xml.dll
 0002:000127c8       .idata$6                   100327c8     Qt5Core:Qt5Core.dll
 0002:0001286e       .idata$6                   1003286e     msvcprt:MSVCP120.dll
 0002:000128f2       .idata$6                   100328f2     MSVCRT:MSVCR120.dll
 0002:00012b06       .idata$6                   10032b06     kernel32:KERNEL32.dll
 0003:0000000c       _Service_PluginViewer      1003300c     ClarkSupport.obj
 0003:00000014       _Service_Project           10033014     ClarkSupport.obj
 0003:0000001c       _Service_ProjectView       1003301c     ClarkSupport.obj
 0003:00000024       _Service_DNAGraphPack      10033024     ClarkSupport.obj
 0003:0000002c       _Service_DNAExport         1003302c     ClarkSupport.obj
 0003:00000034       _Service_TestRunner        10033034     ClarkSupport.obj
 0003:0000003c       _Service_ScriptRegistry    1003303c     ClarkSupport.obj
 0003:00000044       _Service_ExternalToolSupport 10033044     ClarkSupport.obj
 0003:0000004c       _Service_GUITesting        1003304c     ClarkSupport.obj
 0003:00000054       _Service_WorkflowDesigner  10033054     ClarkSupport.obj
 0003:0000005c       _Service_QueryDesigner     1003305c     ClarkSupport.obj
 0003:00000064       _Service_MinCoreServiceId  10033064     ClarkSupport.obj
 0003:0000006c       _Service_MaxCoreServiceId  1003306c     ClarkSupport.obj
 0003:00000d58       __Tuple_alloc              10033d58     ClarkBuildWorker.obj
 0003:00000d59       _ignore                    10033d59     ClarkBuildWorker.obj
 0003:00000d5a       _allocator_arg             10033d5a     ClarkBuildWorker.obj
 0003:00000d5b       _piecewise_construct       10033d5b     ClarkBuildWorker.obj
 0003:00000d5c       _taskLog                   10033d5c     ClarkBuildWorker.obj
 0003:00000d64       _algoLog                   10033d64     ClarkBuildWorker.obj
 0003:00000d6c       _userActLog                10033d6c     ClarkBuildWorker.obj
 0003:00000d74       _ioLog                     10033d74     ClarkBuildWorker.obj
 0003:00000d7c       _coreLog                   10033d7c     ClarkBuildWorker.obj
 0003:00000d84       _TAXONOMY_RANK             10033d84     ClarkBuildWorker.obj
 0003:00000d88       _uiLog                     10033d88     ClarkBuildWorker.obj
 0003:00000d90       _scriptLog                 10033d90     ClarkBuildWorker.obj
 0003:00000d98       _perfLog                   10033d98     ClarkBuildWorker.obj
 0003:00000da4       _cmdLog                    10033da4     ClarkBuildWorker.obj
 0003:00000dac       _GENOMIC_LIBRARY           10033dac     ClarkBuildWorker.obj
 0003:00000db0       _OUTPUT_PORT               10033db0     ClarkBuildWorker.obj
 0003:00000db4       _DB_URL                    10033db4     ClarkBuildWorker.obj
 0003:00000dc8       ?cvar@?1???0ClarkBuildTask@LocalWorkflow@U2@@QAE@ABVQString@@ABVQStringList@@H0@Z@4VGReportableCounter@3@A 10033dc8     ClarkBuildWorker.obj
 0003:00000df0       ?$S1@?1???0ClarkBuildTask@LocalWorkflow@U2@@QAE@ABVQString@@ABVQStringList@@H0@Z@4IA 10033df0     ClarkBuildWorker.obj
 0003:00000df4       __Tuple_alloc              10033df4     ClarkClassifyWorker.obj
 0003:00000df5       _ignore                    10033df5     ClarkClassifyWorker.obj
 0003:00000df6       _allocator_arg             10033df6     ClarkClassifyWorker.obj
 0003:00000df7       _piecewise_construct       10033df7     ClarkClassifyWorker.obj
 0003:00000df8       _REPORT_PREFIX             10033df8     ClarkClassifyWorker.obj
 0003:00000e10       _taskLog                   10033e10     ClarkClassifyWorker.obj
 0003:00000e18       _algoLog                   10033e18     ClarkClassifyWorker.obj
 0003:00000e20       _userActLog                10033e20     ClarkClassifyWorker.obj
 0003:00000e28       _ioLog                     10033e28     ClarkClassifyWorker.obj
 0003:00000e30       _coreLog                   10033e30     ClarkClassifyWorker.obj
 0003:00000e50       _uiLog                     10033e50     ClarkClassifyWorker.obj
 0003:00000e58       _scriptLog                 10033e58     ClarkClassifyWorker.obj
 0003:00000e60       _EXTENDED_REPORT_SUFFIX    10033e60     ClarkClassifyWorker.obj
 0003:00000e74       _perfLog                   10033e74     ClarkClassifyWorker.obj
 0003:00000e88       _cmdLog                    10033e88     ClarkClassifyWorker.obj
 0003:00000eb8       ?cvar@?1???0ClarkClassifyTask@LocalWorkflow@U2@@QAE@ABVClarkClassifySettings@23@ABVQString@@11@Z@4VGReportableCounter@3@A 10033eb8     ClarkClassifyWorker.obj
 0003:00000ee0       ?$S1@?1???0ClarkClassifyTask@LocalWorkflow@U2@@QAE@ABVClarkClassifySettings@23@ABVQString@@11@Z@4IA 10033ee0     ClarkClassifyWorker.obj
 0003:00000ef0       __Tuple_alloc              10033ef0     ClarkSupport.obj
 0003:00000ef1       _ignore                    10033ef1     ClarkSupport.obj
 0003:00000ef2       _allocator_arg             10033ef2     ClarkSupport.obj
 0003:00000ef3       _piecewise_construct       10033ef3     ClarkSupport.obj
 0003:00000ef8       _taskLog                   10033ef8     ClarkSupport.obj
 0003:00000f04       _algoLog                   10033f04     ClarkSupport.obj
 0003:00000f10       _userActLog                10033f10     ClarkSupport.obj
 0003:00000f1c       _ioLog                     10033f1c     ClarkSupport.obj
 0003:00000f28       _coreLog                   10033f28     ClarkSupport.obj
 0003:00000f30       _uiLog                     10033f30     ClarkSupport.obj
 0003:00000f38       _scriptLog                 10033f38     ClarkSupport.obj
 0003:00000f48       _perfLog                   10033f48     ClarkSupport.obj
 0003:00000f60       _cmdLog                    10033f60     ClarkSupport.obj
 0003:00000f70       __Tuple_alloc              10033f70     ClarkSupportPlugin.obj
 0003:00000f71       _ignore                    10033f71     ClarkSupportPlugin.obj
 0003:00000f72       _allocator_arg             10033f72     ClarkSupportPlugin.obj
 0003:00000f73       _piecewise_construct       10033f73     ClarkSupportPlugin.obj
 0003:00000f74       _taskLog                   10033f74     ClarkSupportPlugin.obj
 0003:00000f7c       _algoLog                   10033f7c     ClarkSupportPlugin.obj
 0003:00000f84       _userActLog                10033f84     ClarkSupportPlugin.obj
 0003:00000f8c       _ioLog                     10033f8c     ClarkSupportPlugin.obj
 0003:00000f98       _coreLog                   10033f98     ClarkSupportPlugin.obj
 0003:00000fa4       _uiLog                     10033fa4     ClarkSupportPlugin.obj
 0003:00000fac       _scriptLog                 10033fac     ClarkSupportPlugin.obj
 0003:00000fb4       _perfLog                   10033fb4     ClarkSupportPlugin.obj
 0003:00000fbc       _cmdLog                    10033fbc     ClarkSupportPlugin.obj
 0003:00000fc4       __Tuple_alloc              10033fc4     ClarkTests.obj
 0003:00000fc5       _ignore                    10033fc5     ClarkTests.obj
 0003:00000fc6       _allocator_arg             10033fc6     ClarkTests.obj
 0003:00000fc7       _piecewise_construct       10033fc7     ClarkTests.obj
 0003:00000fc8       _taskLog                   10033fc8     ClarkTests.obj
 0003:00000fd0       _algoLog                   10033fd0     ClarkTests.obj
 0003:00000fdc       _userActLog                10033fdc     ClarkTests.obj
 0003:00000fe4       _ioLog                     10033fe4     ClarkTests.obj
 0003:00000fec       _coreLog                   10033fec     ClarkTests.obj
 0003:00000ff8       _uiLog                     10033ff8     ClarkTests.obj
 0003:00001000       _scriptLog                 10034000     ClarkTests.obj
 0003:0000100c       _perfLog                   1003400c     ClarkTests.obj
 0003:00001014       _cmdLog                    10034014     ClarkTests.obj
 0003:0000102c       __Tuple_alloc              1003402c     moc_ClarkBuildWorker.obj
 0003:0000102d       _ignore                    1003402d     moc_ClarkBuildWorker.obj
 0003:0000102e       _allocator_arg             1003402e     moc_ClarkBuildWorker.obj
 0003:0000102f       _piecewise_construct       1003402f     moc_ClarkBuildWorker.obj
 0003:00001030       _taskLog                   10034030     moc_ClarkBuildWorker.obj
 0003:00001038       _algoLog                   10034038     moc_ClarkBuildWorker.obj
 0003:00001040       _userActLog                10034040     moc_ClarkBuildWorker.obj
 0003:00001048       _ioLog                     10034048     moc_ClarkBuildWorker.obj
 0003:00001050       _coreLog                   10034050     moc_ClarkBuildWorker.obj
 0003:00001058       _uiLog                     10034058     moc_ClarkBuildWorker.obj
 0003:00001060       _scriptLog                 10034060     moc_ClarkBuildWorker.obj
 0003:00001068       _perfLog                   10034068     moc_ClarkBuildWorker.obj
 0003:00001070       _cmdLog                    10034070     moc_ClarkBuildWorker.obj
 0003:0000107c       __Tuple_alloc              1003407c     moc_ClarkClassifyWorker.obj
 0003:0000107d       _ignore                    1003407d     moc_ClarkClassifyWorker.obj
 0003:0000107e       _allocator_arg             1003407e     moc_ClarkClassifyWorker.obj
 0003:0000107f       _piecewise_construct       1003407f     moc_ClarkClassifyWorker.obj
 0003:00001080       _taskLog                   10034080     moc_ClarkClassifyWorker.obj
 0003:00001088       _algoLog                   10034088     moc_ClarkClassifyWorker.obj
 0003:00001090       _userActLog                10034090     moc_ClarkClassifyWorker.obj
 0003:00001098       _ioLog                     10034098     moc_ClarkClassifyWorker.obj
 0003:000010a0       _coreLog                   100340a0     moc_ClarkClassifyWorker.obj
 0003:000010a8       _uiLog                     100340a8     moc_ClarkClassifyWorker.obj
 0003:000010b0       _scriptLog                 100340b0     moc_ClarkClassifyWorker.obj
 0003:000010b8       _perfLog                   100340b8     moc_ClarkClassifyWorker.obj
 0003:000010c0       _cmdLog                    100340c0     moc_ClarkClassifyWorker.obj
 0003:000010c8       __Tuple_alloc              100340c8     moc_ClarkSupport.obj
 0003:000010c9       _ignore                    100340c9     moc_ClarkSupport.obj
 0003:000010ca       _allocator_arg             100340ca     moc_ClarkSupport.obj
 0003:000010cb       _piecewise_construct       100340cb     moc_ClarkSupport.obj
 0003:000010cc       __Tuple_alloc              100340cc     moc_ClarkSupportPlugin.obj
 0003:000010cd       _ignore                    100340cd     moc_ClarkSupportPlugin.obj
 0003:000010ce       _allocator_arg             100340ce     moc_ClarkSupportPlugin.obj
 0003:000010cf       _piecewise_construct       100340cf     moc_ClarkSupportPlugin.obj
 0003:000010d0       ___proc_attached           100340d0     MSVCRT:crtdll.obj
 0003:000010d8       _GS_ExceptionRecord        100340d8     MSVCRT:gs_report.obj
 0003:00001128       _GS_ContextRecord          10034128     MSVCRT:gs_report.obj
 0003:000013f4       _DebuggerWasPresent        100343f4     MSVCRT:gs_report.obj
 0004:00000060       $R000000                   10035060     * linker generated manifest res *

 Exports

  ordinal    name

        1    _ugene_plugin_init
               exported name: ugene_plugin_init
